 kraken_support

 Timestamp is 5dee3773 (Mon Dec 09 19:00:51 2019)

 Preferred load address is 10000000

 Start         Length     Name                   Class
 0001:00000000 0000647bH .text$di                CODE
 0001:00006480 000159deH .text$mn                CODE
 0001:0001be60 00005694H .text$x                 CODE
 0001:00021500 0000129bH .text$yd                CODE
 0002:00000000 000008bcH .idata$5                DATA
 0002:000008bc 00000004H .CRT$XCA                DATA
 0002:000008c0 000003acH .CRT$XCU                DATA
 0002:00000c6c 00000004H .CRT$XCZ                DATA
 0002:00000c70 00000004H .CRT$XIA                DATA
 0002:00000c74 00000004H .CRT$XIAA               DATA
 0002:00000c78 00000004H .CRT$XIC                DATA
 0002:00000c7c 00000004H .CRT$XIZ                DATA
 0002:00000c80 00003380H .rdata                  DATA
 0002:00004000 00000074H .rdata$debug            DATA
 0002:00004074 00001558H .rdata$r                DATA
 0002:000055d0 000004a4H .rdata$sxdata           DATA
 0002:00005a74 00000004H .rtc$IAA                DATA
 0002:00005a78 00000004H .rtc$IZZ                DATA
 0002:00005a7c 00000004H .rtc$TAA                DATA
 0002:00005a80 00000004H .rtc$TZZ                DATA
 0002:00005a88 0000599cH .xdata$x                DATA
 0002:0000b430 00000057H .edata                  DATA
 0002:0000b488 000000f0H .idata$2                DATA
 0002:0000b578 00000014H .idata$3                DATA
 0002:0000b58c 000008bcH .idata$4                DATA
 0002:0000be48 0000760aH .idata$6                DATA
 0003:00000000 000000e4H .data                   DATA
 0003:000000e8 00000b28H .data$r                 DATA
 0003:00000c10 00000a74H .bss                    DATA
 0004:00000000 00000058H .rsrc$01                DATA
 0004:00000060 00000180H .rsrc$02                DATA

  Address         Publics by Value              Rva+Base       Lib:Object

 0000:00000000       ___guard_flags             00000000     <absolute>
 0000:00000000       ___guard_fids_count        00000000     <absolute>
 0000:00000000       ___guard_fids_table        00000000     <absolute>
 0000:00000000       __except_list              00000000     <absolute>
 0000:00000129       ___safe_se_handler_count   00000129     <absolute>
 0000:00009876       __ldused                   00009876     <absolute>
 0000:00009876       __fltused                  00009876     <absolute>
 0000:00000000       ___ImageBase               10000000     <linker-defined>
 0001:00006480       ??$_Allocate@D@std@@YAPADIPAD@Z 10007480 f i DatabaseSizeRelation.obj
 0001:000064b0       ??$addressof@D@std@@YAPADAAD@Z 100074b0 f i DatabaseSizeRelation.obj
 0001:000064c0       ??$atomic@H@?$QAtomicOpsBySize@$03@@CAPAJPAH@Z 100074c0 f i DatabaseSizeRelation.obj
 0001:000064d0       ??$construct@PADAAPAD@?$_Wrap_alloc@V?$allocator@D@std@@@std@@QAEXPAPADAAPAD@Z 100074d0 f i DatabaseSizeRelation.obj
 0001:000064f0       ??$construct@PADAAPAD@?$allocator@D@std@@QAEXPAPADAAPAD@Z 100074f0 f i DatabaseSizeRelation.obj
 0001:00006510       ??$construct@PADAAPAD@?$allocator_traits@V?$allocator@D@std@@@std@@SAXAAV?$allocator@D@1@PAPADAAPAD@Z 10007510 f i DatabaseSizeRelation.obj
 0001:00006530       ??$deref@H@?$QAtomicOpsBySize@$03@@SA_NAAH@Z 10007530 f i DatabaseSizeRelation.obj
 0001:00006550       ??$destroy@PAD@?$_Wrap_alloc@V?$allocator@D@std@@@std@@QAEXPAPAD@Z 10007550 f i DatabaseSizeRelation.obj
 0001:00006560       ??$destroy@PAD@?$allocator@D@std@@QAEXPAPAD@Z 10007560 f i DatabaseSizeRelation.obj
 0001:00006570       ??$destroy@PAD@?$allocator_traits@V?$allocator@D@std@@@std@@SAXAAV?$allocator@D@1@PAPAD@Z 10007570 f i DatabaseSizeRelation.obj
 0001:00006580       ??$forward@AAPAD@std@@YAAAPADAAPAD@Z 10007580 f i DatabaseSizeRelation.obj
 0001:00006590       ??$load@H@?$QGenericAtomicOps@U?$QAtomicOpsBySize@$03@@@@SAHABH@Z 10007590 f i DatabaseSizeRelation.obj
 0001:000065a0       ??0?$QMap@VQString@@VQVariant@@@@QAE@XZ 100075a0 f i DatabaseSizeRelation.obj
 0001:000065b0       ??0?$_String_alloc@$0A@U?$_String_base_types@DV?$allocator@D@std@@@std@@@std@@QAE@ABV?$allocator@D@1@@Z 100075b0 f i DatabaseSizeRelation.obj
 0001:000065d0       ??0?$_String_val@U?$_Simple_types@D@std@@@std@@QAE@XZ 100075d0 f i DatabaseSizeRelation.obj
 0001:000065f0       ??0?$_Wrap_alloc@V?$allocator@D@std@@@std@@QAE@XZ 100075f0 f i DatabaseSizeRelation.obj
 0001:00006600       ??0?$allocator@D@std@@QAE@XZ 10007600 f i DatabaseSizeRelation.obj
 0001:00006610       ??0?$basic_string@DU?$char_traits@D@std@@V?$allocator@D@2@@std@@QAE@PBD@Z 10007610 f i DatabaseSizeRelation.obj
 0001:00006670       ??0DatabaseSizeRelation@LocalWorkflow@U2@@QAE@ABV012@@Z 10007670 f i DatabaseSizeRelation.obj
 0001:00006690       ??0DatabaseSizeRelation@LocalWorkflow@U2@@QAE@ABVQString@@@Z 10007690 f   DatabaseSizeRelation.obj
 0001:00006740       ??0_Generic_error_category@std@@QAE@XZ 10007740 f i DatabaseSizeRelation.obj
 0001:00006750       ??0_Ignore@std@@QAE@XZ     10007750 f i DatabaseSizeRelation.obj
 0001:00006760       ??0_Iostream_error_category@std@@QAE@XZ 10007760 f i DatabaseSizeRelation.obj
 0001:00006770       ??0_System_error_category@std@@QAE@XZ 10007770 f i DatabaseSizeRelation.obj
 0001:00006780       ??0error_category@std@@QAE@XZ 10007780 f i DatabaseSizeRelation.obj
 0001:00006790       ??0error_condition@std@@QAE@HABVerror_category@1@@Z 10007790 f i DatabaseSizeRelation.obj
 0001:000067b0       ??1?$QMap@VQString@@VQVariant@@@@QAE@XZ 100077b0 f i DatabaseSizeRelation.obj
 0001:00006800       ??1?$basic_string@DU?$char_traits@D@std@@V?$allocator@D@2@@std@@QAE@XZ 10007800 f i DatabaseSizeRelation.obj
 0001:00006830       ??1DatabaseSizeRelation@LocalWorkflow@U2@@UAE@XZ 10007830 f i DatabaseSizeRelation.obj
 0001:00006840       ??1_Generic_error_category@std@@UAE@XZ 10007840 f i DatabaseSizeRelation.obj
 0001:00006850       ??1_Iostream_error_category@std@@UAE@XZ 10007850 f i DatabaseSizeRelation.obj
 0001:00006860       ??1_System_error_category@std@@UAE@XZ 10007860 f i DatabaseSizeRelation.obj
 0001:00006870       ??1error_category@std@@UAE@XZ 10007870 f i DatabaseSizeRelation.obj
 0001:00006880       ??2@YAPAXIPAX@Z            10007880 f i DatabaseSizeRelation.obj
 0001:00006890       ??3@YAXPAX0@Z              10007890 f i DatabaseSizeRelation.obj
 0001:000068a0       ??8error_category@std@@QBE_NABV01@@Z 100078a0 f i DatabaseSizeRelation.obj
 0001:000068b0       ??8error_condition@std@@QBE_NABV01@@Z 100078b0 f i DatabaseSizeRelation.obj
 0001:000068d0       ??H@YA?BVQString@@ABV0@PBD@Z 100078d0 f i DatabaseSizeRelation.obj
 0001:00006970       ??_GDatabaseSizeRelation@LocalWorkflow@U2@@UAEPAXI@Z 10007970 f i DatabaseSizeRelation.obj
 0001:00006970       ??_EDatabaseSizeRelation@LocalWorkflow@U2@@UAEPAXI@Z 10007970 f i DatabaseSizeRelation.obj
 0001:000069a0       ??_GQString@@QAEPAXI@Z     100079a0 f i DatabaseSizeRelation.obj
 0001:000069d0       ??_GQVariant@@QAEPAXI@Z    100079d0 f i DatabaseSizeRelation.obj
 0001:00006a00       ??_G_Generic_error_category@std@@UAEPAXI@Z 10007a00 f i DatabaseSizeRelation.obj
 0001:00006a00       ??_E_Generic_error_category@std@@UAEPAXI@Z 10007a00 f i DatabaseSizeRelation.obj
 0001:00006a30       ??_G_Iostream_error_category@std@@UAEPAXI@Z 10007a30 f i DatabaseSizeRelation.obj
 0001:00006a30       ??_E_Iostream_error_category@std@@UAEPAXI@Z 10007a30 f i DatabaseSizeRelation.obj
 0001:00006a60       ??_E_System_error_category@std@@UAEPAXI@Z 10007a60 f i DatabaseSizeRelation.obj
 0001:00006a60       ??_G_System_error_category@std@@UAEPAXI@Z 10007a60 f i DatabaseSizeRelation.obj
 0001:00006a90       ??_Eerror_category@std@@UAEPAXI@Z 10007a90 f i DatabaseSizeRelation.obj
 0001:00006a90       ??_Gerror_category@std@@UAEPAXI@Z 10007a90 f i DatabaseSizeRelation.obj
 0001:00006ac0       ?_Copy@?$basic_string@DU?$char_traits@D@std@@V?$allocator@D@2@@std@@QAEXII@Z 10007ac0 f i DatabaseSizeRelation.obj
 0001:00006c10       ?_Eos@?$basic_string@DU?$char_traits@D@std@@V?$allocator@D@2@@std@@QAEXI@Z 10007c10 f i DatabaseSizeRelation.obj
 0001:00006c40       ?_Getal@?$_String_alloc@$0A@U?$_String_base_types@DV?$allocator@D@std@@@std@@@std@@QBE?AU?$_Wrap_alloc@V?$allocator@D@std@@@2@XZ 10007c40 f i DatabaseSizeRelation.obj
 0001:00006c50       ?_Grow@?$basic_string@DU?$char_traits@D@std@@V?$allocator@D@2@@std@@QAE_NI_N@Z 10007c50 f i DatabaseSizeRelation.obj
 0001:00006d00       ?_Inside@?$basic_string@DU?$char_traits@D@std@@V?$allocator@D@2@@std@@QAE_NPBD@Z 10007d00 f i DatabaseSizeRelation.obj
 0001:00006d40       ?_Myptr@?$_String_val@U?$_Simple_types@D@std@@@std@@QAEPADXZ 10007d40 f i DatabaseSizeRelation.obj
 0001:00006d50       ?_Myptr@?$_String_val@U?$_Simple_types@D@std@@@std@@QBEPBDXZ 10007d50 f i DatabaseSizeRelation.obj
 0001:00006d60       ?_Tidy@?$basic_string@DU?$char_traits@D@std@@V?$allocator@D@2@@std@@QAEX_NI@Z 10007d60 f i DatabaseSizeRelation.obj
 0001:00006db0       ?_Xlen@?$basic_string@DU?$char_traits@D@std@@V?$allocator@D@2@@std@@QBEXXZ 10007db0 f i DatabaseSizeRelation.obj
 0001:00006dc0       ?_Xran@?$basic_string@DU?$char_traits@D@std@@V?$allocator@D@2@@std@@QBEXXZ 10007dc0 f i DatabaseSizeRelation.obj
 0001:00006dd0       ?allocate@?$_Wrap_alloc@V?$allocator@D@std@@@std@@QAEPADI@Z 10007dd0 f i DatabaseSizeRelation.obj
 0001:00006e00       ?allocate@?$allocator@D@std@@QAEPADI@Z 10007e00 f i DatabaseSizeRelation.obj
 0001:00006e30       ?assign@?$basic_string@DU?$char_traits@D@std@@V?$allocator@D@2@@std@@QAEAAV12@ABV12@II@Z 10007e30 f i DatabaseSizeRelation.obj
 0001:00006f50       ?assign@?$basic_string@DU?$char_traits@D@std@@V?$allocator@D@2@@std@@QAEAAV12@PBD@Z 10007f50 f i DatabaseSizeRelation.obj
 0001:00006fa0       ?assign@?$basic_string@DU?$char_traits@D@std@@V?$allocator@D@2@@std@@QAEAAV12@PBDI@Z 10007fa0 f i DatabaseSizeRelation.obj
 0001:000070a0       ?assign@?$char_traits@D@std@@SAXAADABD@Z 100080a0 f i DatabaseSizeRelation.obj
 0001:000070b0       ?category@error_code@std@@QBEABVerror_category@2@XZ 100080b0 f i DatabaseSizeRelation.obj
 0001:000070c0       ?category@error_condition@std@@QBEABVerror_category@2@XZ 100080c0 f i DatabaseSizeRelation.obj
 0001:000070d0       ?clone@DatabaseSizeRelation@LocalWorkflow@U2@@UBEPAV123@XZ 100080d0 f   DatabaseSizeRelation.obj
 0001:00007150       ?copy@?$char_traits@D@std@@SAPADPADPBDI@Z 10008150 f i DatabaseSizeRelation.obj
 0001:00007170       ?deallocate@?$_Wrap_alloc@V?$allocator@D@std@@@std@@QAEXPADI@Z 10008170 f i DatabaseSizeRelation.obj
 0001:00007190       ?deallocate@?$allocator@D@std@@QAEXPADI@Z 10008190 f i DatabaseSizeRelation.obj
 0001:000071b0       ?default_error_condition@_System_error_category@std@@UBE?AVerror_condition@2@H@Z 100081b0 f i DatabaseSizeRelation.obj
 0001:000071f0       ?default_error_condition@error_category@std@@UBE?AVerror_condition@2@H@Z 100081f0 f i DatabaseSizeRelation.obj
 0001:00007210       ?deref@?$QBasicAtomicInteger@H@@QAE_NXZ 10008210 f i DatabaseSizeRelation.obj
 0001:00007220       ?deref@RefCount@QtPrivate@@QAE_NXZ 10008220 f i DatabaseSizeRelation.obj
 0001:00007240       ?destroy@?$QMapData@VQString@@VQVariant@@@@QAEXXZ 10008240 f i DatabaseSizeRelation.obj
 0001:00007270       ?destroySubTree@?$QMapNode@VQString@@VQVariant@@@@QAEXXZ 10008270 f i DatabaseSizeRelation.obj
 0001:000072b0       ?equivalent@error_category@std@@UBE_NABVerror_code@2@H@Z 100082b0 f i DatabaseSizeRelation.obj
 0001:000072d0       ?equivalent@error_category@std@@UBE_NHABVerror_condition@2@@Z 100082d0 f i DatabaseSizeRelation.obj
 0001:00007310       ?erase@?$basic_string@DU?$char_traits@D@std@@V?$allocator@D@2@@std@@QAEAAV12@I@Z 10008310 f i DatabaseSizeRelation.obj
 0001:00007350       ?erase@?$basic_string@DU?$char_traits@D@std@@V?$allocator@D@2@@std@@QAEAAV12@II@Z 10008350 f i DatabaseSizeRelation.obj
 0001:000073f0       ?generic_category@std@@YAABVerror_category@1@XZ 100083f0 f i DatabaseSizeRelation.obj
 0001:00007400       ?getAffectResult@DatabaseSizeRelation@LocalWorkflow@U2@@UBE?AVQVariant@@ABV4@0PAVDelegateTags@3@1@Z 10008400 f   DatabaseSizeRelation.obj
 0001:00007520       ?leftNode@?$QMapNode@VQString@@VQVariant@@@@QBEPAU1@XZ 10008520 f i DatabaseSizeRelation.obj
 0001:00007530       ?length@?$char_traits@D@std@@SAIPBD@Z 10008530 f i DatabaseSizeRelation.obj
 0001:00007550       ?load@?$QBasicAtomicInteger@H@@QBEHXZ 10008550 f i DatabaseSizeRelation.obj
 0001:00007560       ?max_size@?$_Wrap_alloc@V?$allocator@D@std@@@std@@QBEIXZ 10008560 f i DatabaseSizeRelation.obj
 0001:00007570       ?max_size@?$allocator@D@std@@QBEIXZ 10008570 f i DatabaseSizeRelation.obj
 0001:00007580       ?max_size@?$allocator_traits@V?$allocator@D@std@@@std@@SAIABV?$allocator@D@2@@Z 10008580 f i DatabaseSizeRelation.obj
 0001:00007590       ?max_size@?$basic_string@DU?$char_traits@D@std@@V?$allocator@D@2@@std@@QBEIXZ 10008590 f i DatabaseSizeRelation.obj
 0001:000075a0       ?message@_Generic_error_category@std@@UBE?AV?$basic_string@DU?$char_traits@D@std@@V?$allocator@D@2@@2@H@Z 100085a0 f i DatabaseSizeRelation.obj
 0001:00007620       ?message@_Iostream_error_category@std@@UBE?AV?$basic_string@DU?$char_traits@D@std@@V?$allocator@D@2@@2@H@Z 10008620 f i DatabaseSizeRelation.obj
 0001:00007670       ?message@_System_error_category@std@@UBE?AV?$basic_string@DU?$char_traits@D@std@@V?$allocator@D@2@@2@H@Z 10008670 f i DatabaseSizeRelation.obj
 0001:000076f0       ?move@?$char_traits@D@std@@SAPADPADPBDI@Z 100086f0 f i DatabaseSizeRelation.obj
 0001:00007710       ?name@_Generic_error_category@std@@UBEPBDXZ 10008710 f i DatabaseSizeRelation.obj
 0001:00007720       ?name@_Iostream_error_category@std@@UBEPBDXZ 10008720 f i DatabaseSizeRelation.obj
 0001:00007730       ?name@_System_error_category@std@@UBEPBDXZ 10008730 f i DatabaseSizeRelation.obj
 0001:00007740       ?rightNode@?$QMapNode@VQString@@VQVariant@@@@QBEPAU1@XZ 10008740 f i DatabaseSizeRelation.obj
 0001:00007750       ?root@?$QMapData@VQString@@VQVariant@@@@QBEPAU?$QMapNode@VQString@@VQVariant@@@@XZ 10008750 f i DatabaseSizeRelation.obj
 0001:00007760       ?size@?$basic_string@DU?$char_traits@D@std@@V?$allocator@D@2@@std@@QBEIXZ 10008760 f i DatabaseSizeRelation.obj
 0001:00007770       ?system_category@std@@YAABVerror_category@1@XZ 10008770 f i DatabaseSizeRelation.obj
 0001:00007780       ?value@error_code@std@@QBEHXZ 10008780 f i DatabaseSizeRelation.obj
 0001:00007790       ?value@error_condition@std@@QBEHXZ 10008790 f i DatabaseSizeRelation.obj
 0001:000077a0       _hypot                     100087a0 f i DatabaseSizeRelation.obj
 0001:000077d0       ??$ref@H@?$QAtomicOpsBySize@$03@@SA_NAAH@Z 100087d0 f i KrakenBuildPrompter.obj
 0001:000077f0       ??0?$PrompterBase@VKrakenBuildPrompter@LocalWorkflow@U2@@@U2@@QAE@PAVActor@Workflow@1@_N@Z 100087f0 f i KrakenBuildPrompter.obj
 0001:00007820       ??0?$QForeachContainer@V?$QList@PAVPort@Workflow@U2@@@@@@QAE@ABV?$QList@PAVPort@Workflow@U2@@@@@Z 10008820 f i KrakenBuildPrompter.obj
 0001:00007860       ??0?$QList@PAVPort@Workflow@U2@@@@QAE@ABV0@@Z 10008860 f i KrakenBuildPrompter.obj
 0001:00007920       ??0KrakenBuildPrompter@LocalWorkflow@U2@@QAE@PAVActor@Workflow@2@@Z 10008920 f   KrakenBuildPrompter.obj
 0001:00007950       ??0QLatin1Char@@QAE@D@Z    10008950 f i KrakenBuildPrompter.obj
 0001:00007960       ??0const_iterator@?$QList@PAVPort@Workflow@U2@@@@QAE@PAUNode@1@@Z 10008960 f i KrakenBuildPrompter.obj
 0001:00007970       ??1?$PrompterBase@VKrakenBuildPrompter@LocalWorkflow@U2@@@U2@@UAE@XZ 10008970 f i KrakenBuildPrompter.obj
 0001:00007980       ??1?$QForeachContainer@V?$QList@PAVPort@Workflow@U2@@@@@@QAE@XZ 10008980 f i KrakenBuildPrompter.obj
 0001:000079b0       ??1?$QList@PAVPort@Workflow@U2@@@@QAE@XZ 100089b0 f i KrakenBuildPrompter.obj
 0001:000079e0       ??1KrakenBuildPrompter@LocalWorkflow@U2@@UAE@XZ 100089e0 f i KrakenBuildPrompter.obj
 0001:000079f0       ??9const_iterator@?$QList@PAVPort@Workflow@U2@@@@QBE_NABV01@@Z 100089f0 f i KrakenBuildPrompter.obj
 0001:00007a10       ??Dconst_iterator@?$QList@PAVPort@Workflow@U2@@@@QBEABQAVPort@Workflow@U2@@XZ 10008a10 f i KrakenBuildPrompter.obj
 0001:00007a20       ??Econst_iterator@?$QList@PAVPort@Workflow@U2@@@@QAEAAV01@XZ 10008a20 f i KrakenBuildPrompter.obj
 0001:00007a26       ??_E?$PrompterBase@VKrakenBuildPrompter@LocalWorkflow@U2@@@U2@@WM@AEPAXI@Z 10008a26 f i KrakenBuildPrompter.obj
 0001:00007a2e       ??_EKrakenBuildPrompter@LocalWorkflow@U2@@WM@AEPAXI@Z 10008a2e f i KrakenBuildPrompter.obj
 0001:00007a40       ??_G?$PrompterBase@VKrakenBuildPrompter@LocalWorkflow@U2@@@U2@@UAEPAXI@Z 10008a40 f i KrakenBuildPrompter.obj
 0001:00007a40       ??_E?$PrompterBase@VKrakenBuildPrompter@LocalWorkflow@U2@@@U2@@UAEPAXI@Z 10008a40 f i KrakenBuildPrompter.obj
 0001:00007a70       ??_EKrakenBuildPrompter@LocalWorkflow@U2@@UAEPAXI@Z 10008a70 f i KrakenBuildPrompter.obj
 0001:00007a70       ??_GKrakenBuildPrompter@LocalWorkflow@U2@@UAEPAXI@Z 10008a70 f i KrakenBuildPrompter.obj
 0001:00007aa0       ?begin@?$QList@PAVPort@Workflow@U2@@@@QBE?AVconst_iterator@1@XZ 10008aa0 f i KrakenBuildPrompter.obj
 0001:00007ac0       ?composeRichDoc@KrakenBuildPrompter@LocalWorkflow@U2@@EAE?AVQString@@XZ 10008ac0 f   KrakenBuildPrompter.obj
 0001:00007df0       ?createDescription@?$PrompterBase@VKrakenBuildPrompter@LocalWorkflow@U2@@@U2@@UAEPAVActorDocument@Workflow@2@PAVActor@42@@Z 10008df0 f i KrakenBuildPrompter.obj
 0001:00008090       ?dealloc@?$QList@PAVPort@Workflow@U2@@@@AAEXPAUData@QListData@@@Z 10009090 f i KrakenBuildPrompter.obj
 0001:000080b0       ?end@?$QList@PAVPort@Workflow@U2@@@@QBE?AVconst_iterator@1@XZ 100090b0 f i KrakenBuildPrompter.obj
 0001:000080d0       ?node_copy@?$QList@PAVPort@Workflow@U2@@@@AAEXPAUNode@1@00@Z 100090d0 f i KrakenBuildPrompter.obj
 0001:00008100       ?node_destruct@?$QList@PAVPort@Workflow@U2@@@@AAEXPAUNode@1@0@Z 10009100 f i KrakenBuildPrompter.obj
 0001:00008110       ?ref@?$QBasicAtomicInteger@H@@QAE_NXZ 10009110 f i KrakenBuildPrompter.obj
 0001:00008130       ?ref@RefCount@QtPrivate@@QAE_NXZ 10009130 f i KrakenBuildPrompter.obj
 0001:00008150       ?t@Node@?$QList@PAVPort@Workflow@U2@@@@QAEAAPAVPort@Workflow@U2@@XZ 10009150 f i KrakenBuildPrompter.obj
 0001:00008160       ?tr@KrakenBuildPrompter@LocalWorkflow@U2@@SA?AVQString@@PBD0H@Z 10009160 f i KrakenBuildPrompter.obj
 0001:00008190       ??$_Move@AAPAUData@QListData@@@std@@YA$$QAPAUData@QListData@@AAPAU12@@Z 10009190 f i KrakenBuildTask.obj
 0001:000081a0       ??$qSwap@PAUData@QListData@@@@YAXAAPAUData@QListData@@0@Z 100091a0 f i KrakenBuildTask.obj
 0001:000081c0       ??$swap@PAUData@QListData@@@std@@YAXAAPAUData@QListData@@0@Z 100091c0 f i KrakenBuildTask.obj
 0001:000081e0       ??0?$QFlags@W4Filter@QDir@@@@QAE@VQFlag@@@Z 100091e0 f i KrakenBuildTask.obj
 0001:000081f0       ??0?$QFlags@W4Filter@QDir@@@@QAE@W4Filter@QDir@@@Z 100091f0 f i KrakenBuildTask.obj
 0001:00008200       ??0?$QFlags@W4SortFlag@QDir@@@@QAE@W4SortFlag@QDir@@@Z 10009200 f i KrakenBuildTask.obj
 0001:00008210       ??0?$QFlags@W4TaskFlag@U2@@@@QAE@VQFlag@@@Z 10009210 f i KrakenBuildTask.obj
 0001:00008220       ??0?$QFlags@W4TaskFlag@U2@@@@QAE@W4TaskFlag@U2@@@Z 10009220 f i KrakenBuildTask.obj
 0001:00008230       ??0?$QForeachContainer@VQStringList@@@@QAE@ABVQStringList@@@Z 10009230 f i KrakenBuildTask.obj
 0001:00008270       ??0?$QList@PAVTask@U2@@@@QAE@$$QAV0@@Z 10009270 f i KrakenBuildTask.obj
 0001:00008290       ??0?$QList@PAVTask@U2@@@@QAE@ABV0@@Z 10009290 f i KrakenBuildTask.obj
 0001:00008350       ??0?$QList@PAVTask@U2@@@@QAE@XZ 10009350 f i KrakenBuildTask.obj
 0001:00008360       ??0?$QList@VQString@@@@QAE@ABV0@@Z 10009360 f i KrakenBuildTask.obj
 0001:00008420       ??0?$QList@VQString@@@@QAE@XZ 10009420 f i KrakenBuildTask.obj
 0001:00008430       ??0KrakenBuildTask@U2@@QAE@ABUKrakenBuildTaskSettings@1@@Z 10009430 f   KrakenBuildTask.obj
 0001:00008680       ??0KrakenBuildTaskSettings@U2@@QAE@ABU01@@Z 10009680 f i KrakenBuildTask.obj
 0001:00008740       ??0KrakenBuildTaskSettings@U2@@QAE@XZ 10009740 f   KrakenBuildTask.obj
 0001:000087f0       ??0QFlag@@QAE@H@Z          100097f0 f i KrakenBuildTask.obj
 0001:00008800       ??0QStringList@@QAE@ABV0@@Z 10009800 f i KrakenBuildTask.obj
 0001:00008820       ??0QStringList@@QAE@XZ     10009820 f i KrakenBuildTask.obj
 0001:00008830       ??0const_iterator@?$QList@VQString@@@@QAE@PAUNode@1@@Z 10009830 f i KrakenBuildTask.obj
 0001:00008840       ??1?$QForeachContainer@VQStringList@@@@QAE@XZ 10009840 f i KrakenBuildTask.obj
 0001:00008850       ??1?$QList@PAVTask@U2@@@@QAE@XZ 10009850 f i KrakenBuildTask.obj
 0001:00008880       ??1?$QList@VQString@@@@QAE@XZ 10009880 f i KrakenBuildTask.obj
 0001:000088e0       ??1KrakenBuildTask@U2@@UAE@XZ 100098e0 f i KrakenBuildTask.obj
 0001:00008970       ??1KrakenBuildTaskSettings@U2@@QAE@XZ 10009970 f i KrakenBuildTask.obj
 0001:000089f0       ??1QStringList@@QAE@XZ     100099f0 f i KrakenBuildTask.obj
 0001:00008a00       ??4?$QList@PAVTask@U2@@@@QAEAAV0@ABV0@@Z 10009a00 f i KrakenBuildTask.obj
 0001:00008a50       ??6?$QList@PAVTask@U2@@@@QAEAAV0@ABQAVTask@U2@@@Z 10009a50 f i KrakenBuildTask.obj
 0001:00008a70       ??6?$QList@PAVTask@U2@@@@QAEAAV0@ABV0@@Z 10009a70 f i KrakenBuildTask.obj
 0001:00008a90       ??6QStringList@@QAEAAV0@ABVQString@@@Z 10009a90 f i KrakenBuildTask.obj
 0001:00008ab0       ??9@YA_NABVQString@@0@Z    10009ab0 f i KrakenBuildTask.obj
 0001:00008ad0       ??9const_iterator@?$QList@VQString@@@@QBE_NABV01@@Z 10009ad0 f i KrakenBuildTask.obj
 0001:00008af0       ??BQFlag@@QBEHXZ           10009af0 f i KrakenBuildTask.obj
 0001:00008b00       ??Dconst_iterator@?$QList@VQString@@@@QBEABVQString@@XZ 10009b00 f i KrakenBuildTask.obj
 0001:00008b10       ??Econst_iterator@?$QList@VQString@@@@QAEAAV01@XZ 10009b10 f i KrakenBuildTask.obj
 0001:00008b20       ??H@YA?BVQString@@ABV0@0@Z 10009b20 f i KrakenBuildTask.obj
 0001:00008b90       ??U?$QFlags@W4Filter@QDir@@@@QBE?AV0@W4Filter@QDir@@@Z 10009b90 f i KrakenBuildTask.obj
 0001:00008bb0       ??U?$QFlags@W4TaskFlag@U2@@@@QBE?AV0@W4TaskFlag@U2@@@Z 10009bb0 f i KrakenBuildTask.obj
 0001:00008bd0       ??U@YA?AV?$QFlags@W4Filter@QDir@@@@W4Filter@QDir@@0@Z 10009bd0 f i KrakenBuildTask.obj
 0001:00008be0       ??Y?$QList@PAVTask@U2@@@@QAEAAV0@ABV0@@Z 10009be0 f i KrakenBuildTask.obj
 0001:00008cd0       ??_ECopyFileTask@U2@@UAEPAXI@Z 10009cd0 f i KrakenBuildTask.obj
 0001:00008cd0       ??_GCopyFileTask@U2@@UAEPAXI@Z 10009cd0 f i KrakenBuildTask.obj
 0001:00008d00       ??_EExternalToolLogParser@U2@@UAEPAXI@Z 10009d00 f i KrakenBuildTask.obj
 0001:00008d00       ??_GExternalToolLogParser@U2@@UAEPAXI@Z 10009d00 f i KrakenBuildTask.obj
 0001:00008d30       ??_EExternalToolRunTask@U2@@UAEPAXI@Z 10009d30 f i KrakenBuildTask.obj
 0001:00008d30       ??_GExternalToolRunTask@U2@@UAEPAXI@Z 10009d30 f i KrakenBuildTask.obj
 0001:00008d60       ??_GKrakenBuildTask@U2@@UAEPAXI@Z 10009d60 f i KrakenBuildTask.obj
 0001:00008d60       ??_EKrakenBuildTask@U2@@UAEPAXI@Z 10009d60 f i KrakenBuildTask.obj
 0001:00008e10       ??_ESequentialMultiTask@U2@@UAEPAXI@Z 10009e10 f i KrakenBuildTask.obj
 0001:00008e10       ??_GSequentialMultiTask@U2@@UAEPAXI@Z 10009e10 f i KrakenBuildTask.obj
 0001:00008e40       ?append@?$QList@PAVTask@U2@@@@QAEXABQAVTask@U2@@@Z 10009e40 f i KrakenBuildTask.obj
 0001:00008ed0       ?append@?$QList@VQString@@@@QAEXABVQString@@@Z 10009ed0 f i KrakenBuildTask.obj
 0001:00008fc0       ?begin@?$QList@VQString@@@@QBE?AVconst_iterator@1@XZ 10009fc0 f i KrakenBuildTask.obj
 0001:00008fe0       ?checkSettings@KrakenBuildTask@U2@@AAEXXZ 10009fe0 f   KrakenBuildTask.obj
 0001:000094c0       ?checkTaxonomy@KrakenBuildTask@U2@@AAEXXZ 1000a4c0 f   KrakenBuildTask.obj
 0001:00009550       ?contains@QStringList@@QBE_NABVQString@@W4CaseSensitivity@Qt@@@Z 1000a550 f i KrakenBuildTask.obj
 0001:00009570       ?dealloc@?$QList@PAVTask@U2@@@@AAEXPAUData@QListData@@@Z 1000a570 f i KrakenBuildTask.obj
 0001:00009590       ?dealloc@?$QList@VQString@@@@AAEXPAUData@QListData@@@Z 1000a590 f i KrakenBuildTask.obj
 0001:000095d0       ?detach_helper_grow@?$QList@PAVTask@U2@@@@AAEPAUNode@1@HH@Z 1000a5d0 f i KrakenBuildTask.obj
 0001:000096e0       ?detach_helper_grow@?$QList@VQString@@@@AAEPAUNode@1@HH@Z 1000a6e0 f i KrakenBuildTask.obj
 0001:00009860       ?end@?$QList@VQString@@@@QBE?AVconst_iterator@1@XZ 1000a860 f i KrakenBuildTask.obj
 0001:00009880       ?getAddToLibraryArguments@KrakenBuildTask@U2@@ABE?AVQStringList@@ABVQString@@@Z 1000a880 f   KrakenBuildTask.obj
 0001:00009960       ?getBuildArguments@KrakenBuildTask@U2@@ABE?AVQStringList@@XZ 1000a960 f   KrakenBuildTask.obj
 0001:00009c70       ?getCleanArguments@KrakenBuildTask@U2@@ABE?AVQStringList@@XZ 1000ac70 f   KrakenBuildTask.obj
 0001:00009d40       ?getResultDatabaseUrl@KrakenBuildTask@U2@@QBEABVQString@@XZ 1000ad40 f   KrakenBuildTask.obj
 0001:00009d50       ?getSettings@KrakenBuildTask@U2@@QBEABUKrakenBuildTaskSettings@2@XZ 1000ad50 f   KrakenBuildTask.obj
 0001:00009d70       ?getShrinkArguments@KrakenBuildTask@U2@@ABE?AVQStringList@@XZ 1000ad70 f   KrakenBuildTask.obj
 0001:0000a070       ?isEmpty@?$QList@PAVTask@U2@@@@QBE_NXZ 1000b070 f i KrakenBuildTask.obj
 0001:0000a080       ?isEmpty@?$QList@VQString@@@@QBE_NXZ 1000b080 f i KrakenBuildTask.obj
 0001:0000a090       ?isShared@RefCount@QtPrivate@@QBE_NXZ 1000b090 f i KrakenBuildTask.obj
 0001:0000a0b0       ?node_construct@?$QList@PAVTask@U2@@@@AAEXPAUNode@1@ABQAVTask@U2@@@Z 1000b0b0 f i KrakenBuildTask.obj
 0001:0000a0d0       ?node_construct@?$QList@VQString@@@@AAEXPAUNode@1@ABVQString@@@Z 1000b0d0 f i KrakenBuildTask.obj
 0001:0000a120       ?node_copy@?$QList@PAVTask@U2@@@@AAEXPAUNode@1@00@Z 1000b120 f i KrakenBuildTask.obj
 0001:0000a150       ?node_copy@?$QList@VQString@@@@AAEXPAUNode@1@00@Z 1000b150 f i KrakenBuildTask.obj
 0001:0000a1f0       ?node_destruct@?$QList@PAVTask@U2@@@@AAEXPAUNode@1@0@Z 1000b1f0 f i KrakenBuildTask.obj
 0001:0000a200       ?node_destruct@?$QList@PAVTask@U2@@@@AAEXPAUNode@1@@Z 1000b200 f i KrakenBuildTask.obj
 0001:0000a210       ?node_destruct@?$QList@VQString@@@@AAEXPAUNode@1@0@Z 1000b210 f i KrakenBuildTask.obj
 0001:0000a240       ?node_destruct@?$QList@VQString@@@@AAEXPAUNode@1@@Z 1000b240 f i KrakenBuildTask.obj
 0001:0000a250       ?prepare@KrakenBuildTask@U2@@EAEXXZ 1000b250 f   KrakenBuildTask.obj
 0001:0000ab20       ?prepareTaxonomyData@KrakenBuildTask@U2@@AAE?AV?$QList@PAVTask@U2@@@@XZ 1000bb20 f   KrakenBuildTask.obj
 0001:0000b090       ?size@?$QList@PAVTask@U2@@@@QBEHXZ 1000c090 f i KrakenBuildTask.obj
 0001:0000b0a0       ?swap@?$QList@PAVTask@U2@@@@QAEXAAV1@@Z 1000c0a0 f i KrakenBuildTask.obj
 0001:0000b0c0       ?t@Node@?$QList@VQString@@@@QAEAAVQString@@XZ 1000c0c0 f i KrakenBuildTask.obj
 0001:0000b0d0       ?tr@KrakenBuildTask@U2@@SA?AVQString@@PBD0H@Z 1000c0d0 f i KrakenBuildTask.obj
 0001:0000b100       ??$getAttributeValueWithoutScript@H@Attribute@U2@@QBEHXZ 1000c100 f i KrakenBuildValidator.obj
 0001:0000b140       ??$qMetaTypeId@H@@YAHXZ    1000c140 f i KrakenBuildValidator.obj
 0001:0000b150       ??$qvariant_cast@H@@YAHABVQVariant@@@Z 1000c150 f i KrakenBuildValidator.obj
 0001:0000b190       ??$value@H@QVariant@@QBEHXZ 1000c190 f i KrakenBuildValidator.obj
 0001:0000b1d0       ??0?$QForeachContainer@$$CBVQStringList@@@@QAE@ABVQStringList@@@Z 1000c1d0 f i KrakenBuildValidator.obj
 0001:0000b210       ??1?$QForeachContainer@$$CBVQStringList@@@@QAE@XZ 1000c210 f i KrakenBuildValidator.obj
 0001:0000b220       ??6?$QList@VWorkflowNotification@U2@@@@QAEAAV0@ABVWorkflowNotification@U2@@@Z 1000c220 f i KrakenBuildValidator.obj
 0001:0000b240       ??_GWorkflowNotification@U2@@QAEPAXI@Z 1000c240 f i KrakenBuildValidator.obj
 0001:0000b270       ?append@?$QList@VWorkflowNotification@U2@@@@QAEXABVWorkflowNotification@U2@@@Z 1000c270 f i KrakenBuildValidator.obj
 0001:0000b350       ?dealloc@?$QList@VWorkflowNotification@U2@@@@AAEXPAUData@QListData@@@Z 1000c350 f i KrakenBuildValidator.obj
 0001:0000b3b0       ?detach_helper_grow@?$QList@VWorkflowNotification@U2@@@@AAEPAUNode@1@HH@Z 1000c3b0 f i KrakenBuildValidator.obj
 0001:0000b500       ?invoke@?$MetaTypeInvoker@U?$QVariantValueHelper@H@QtPrivate@@ABVQVariant@@H@QtPrivate@@SAHABVQVariant@@@Z 1000c500 f i KrakenBuildValidator.obj
 0001:0000b540       ?metaType@?$QVariantValueHelper@H@QtPrivate@@SAHABVQVariant@@@Z 1000c540 f i KrakenBuildValidator.obj
 0001:0000b580       ?node_construct@?$QList@VWorkflowNotification@U2@@@@AAEXPAUNode@1@ABVWorkflowNotification@U2@@@Z 1000c580 f i KrakenBuildValidator.obj
 0001:0000b600       ?node_copy@?$QList@VWorkflowNotification@U2@@@@AAEXPAUNode@1@00@Z 1000c600 f i KrakenBuildValidator.obj
 0001:0000b6d0       ?node_destruct@?$QList@VWorkflowNotification@U2@@@@AAEXPAUNode@1@0@Z 1000c6d0 f i KrakenBuildValidator.obj
 0001:0000b710       ?node_destruct@?$QList@VWorkflowNotification@U2@@@@AAEXPAUNode@1@@Z 1000c710 f i KrakenBuildValidator.obj
 0001:0000b740       ?qt_metatype_id@?$QMetaTypeId2@H@@SAHXZ 1000c740 f i KrakenBuildValidator.obj
 0001:0000b750       ?tr@KrakenBuildValidator@Workflow@U2@@SA?AVQString@@PBD0H@Z 1000c750 f i KrakenBuildValidator.obj
 0001:0000b780       ?validate@KrakenBuildValidator@Workflow@U2@@UBE_NPBVActor@23@AAV?$QList@VWorkflowNotification@U2@@@@ABV?$QMap@VQString@@V1@@@@Z 1000c780 f   KrakenBuildValidator.obj
 0001:0000b7c0       ?validateMinimizerLength@KrakenBuildValidator@Workflow@U2@@ABE_NPBVActor@23@AAV?$QList@VWorkflowNotification@U2@@@@@Z 1000c7c0 f   KrakenBuildValidator.obj
 0001:0000b910       ?validateTaxonomy@KrakenBuildValidator@Workflow@U2@@ABE_NPBVActor@23@AAV?$QList@VWorkflowNotification@U2@@@@@Z 1000c910 f   KrakenBuildValidator.obj
 0001:0000bbe0       ??$acquireMemoryFence@H@?$QGenericAtomicOps@U?$QAtomicOpsBySize@$03@@@@SAXABH@Z 1000cbe0 f i KrakenBuildWorker.obj
 0001:0000bbf0       ??$getAttributeValue@H@Attribute@U2@@QBEHPAVWorkflowContext@Workflow@1@@Z 1000cbf0 f i KrakenBuildWorker.obj
 0001:0000bfc0       ??$getAttributeValue@V?$QList@VDataset@U2@@@@@Attribute@U2@@QBE?AV?$QList@VDataset@U2@@@@PAVWorkflowContext@Workflow@1@@Z 1000cfc0 f i KrakenBuildWorker.obj
 0001:0000bfe0       ??$getAttributeValue@VQString@@@Attribute@U2@@QBE?AVQString@@PAVWorkflowContext@Workflow@1@@Z 1000cfe0 f i KrakenBuildWorker.obj
 0001:0000c370       ??$getAttributeValue@_N@Attribute@U2@@QBE_NPAVWorkflowContext@Workflow@1@@Z 1000d370 f i KrakenBuildWorker.obj
 0001:0000c3b0       ??$getAttributeValueWithoutScript@V?$QList@VDataset@U2@@@@@Attribute@U2@@QBE?AV?$QList@VDataset@U2@@@@XZ 1000d3b0 f i KrakenBuildWorker.obj
 0001:0000c3d0       ??$getAttributeValueWithoutScript@VQString@@@Attribute@U2@@QBE?AVQString@@XZ 1000d3d0 f i KrakenBuildWorker.obj
 0001:0000c3f0       ??$getAttributeValueWithoutScript@_N@Attribute@U2@@QBE_NXZ 1000d3f0 f i KrakenBuildWorker.obj
 0001:0000c430       ??$getValue@H@BaseWorker@LocalWorkflow@U2@@IBEHABVQString@@@Z 1000d430 f i KrakenBuildWorker.obj
 0001:0000c460       ??$getValue@V?$QList@VDataset@U2@@@@@BaseWorker@LocalWorkflow@U2@@IBE?AV?$QList@VDataset@U2@@@@ABVQString@@@Z 1000d460 f i KrakenBuildWorker.obj
 0001:0000c4b0       ??$getValue@VQString@@@BaseWorker@LocalWorkflow@U2@@IBE?AVQString@@ABV3@@Z 1000d4b0 f i KrakenBuildWorker.obj
 0001:0000c5c0       ??$getValue@_N@BaseWorker@LocalWorkflow@U2@@IBE_NABVQString@@@Z 1000d5c0 f i KrakenBuildWorker.obj
 0001:0000c620       ??$loadAcquire@H@?$QGenericAtomicOps@U?$QAtomicOpsBySize@$03@@@@SAHABH@Z 1000d620 f i KrakenBuildWorker.obj
 0001:0000c630       ??$orderedMemoryFence@H@?$QGenericAtomicOps@U?$QAtomicOpsBySize@$03@@@@SAXABH@Z 1000d630 f i KrakenBuildWorker.obj
 0001:0000c640       ??$qMapLessThanKey@VDescriptor@U2@@@@YA_NABVDescriptor@U2@@0@Z 1000d640 f i KrakenBuildWorker.obj
 0001:0000c660       ??$qMapLessThanKey@VQString@@@@YA_NABVQString@@0@Z 1000d660 f i KrakenBuildWorker.obj
 0001:0000c670       ??$qMetaTypeId@V?$QList@VDataset@U2@@@@@@YAHXZ 1000d670 f i KrakenBuildWorker.obj
 0001:0000c680       ??$qMetaTypeId@VQString@@@@YAHXZ 1000d680 f i KrakenBuildWorker.obj
 0001:0000c690       ??$qMetaTypeId@_N@@YAHXZ   1000d690 f i KrakenBuildWorker.obj
 0001:0000c6a0       ??$qRegisterMetaType@V?$QList@VDataset@U2@@@@@@YAHPBDPAV?$QList@VDataset@U2@@@@W4DefinedType@?$MetaTypeDefinedHelper@V?$QList@VDataset@U2@@@@$00@QtPrivate@@@Z 1000d6a0 f i KrakenBuildWorker.obj
 0001:0000c760       ??$qRegisterNormalizedMetaType@V?$QList@VDataset@U2@@@@@@YAHABVQByteArray@@PAV?$QList@VDataset@U2@@@@W4DefinedType@?$MetaTypeDefinedHelper@V?$QList@VDataset@U2@@@@$00@QtPrivate@@@Z 1000d760 f i KrakenBuildWorker.obj
 0001:0000c7c0       ??$qobject_cast@PAVKrakenBuildTask@U2@@@@YAPAVKrakenBuildTask@U2@@PAVQObject@@@Z 1000d7c0 f i KrakenBuildWorker.obj
 0001:0000c7e0       ??$qvariant_cast@V?$QList@VDataset@U2@@@@@@YA?AV?$QList@VDataset@U2@@@@ABVQVariant@@@Z 1000d7e0 f i KrakenBuildWorker.obj
 0001:0000c800       ??$qvariant_cast@VQString@@@@YA?AVQString@@ABVQVariant@@@Z 1000d800 f i KrakenBuildWorker.obj
 0001:0000c820       ??$qvariant_cast@_N@@YA_NABVQVariant@@@Z 1000d820 f i KrakenBuildWorker.obj
 0001:0000c860       ??$releaseMemoryFence@H@?$QGenericAtomicOps@U?$QAtomicOpsBySize@$03@@@@SAXABH@Z 1000d860 f i KrakenBuildWorker.obj
 0001:0000c870       ??$storeRelease@HH@?$QGenericAtomicOps@U?$QAtomicOpsBySize@$03@@@@SAXAAHH@Z 1000d870 f i KrakenBuildWorker.obj
 0001:0000c880       ??$value@V?$QList@VDataset@U2@@@@@QVariant@@QBE?AV?$QList@VDataset@U2@@@@XZ 1000d880 f i KrakenBuildWorker.obj
 0001:0000c8a0       ??$value@VQString@@@QVariant@@QBE?AVQString@@XZ 1000d8a0 f i KrakenBuildWorker.obj
 0001:0000c8c0       ??$value@_N@QVariant@@QBE_NXZ 1000d8c0 f i KrakenBuildWorker.obj
 0001:0000c900       ??0?$QFlags@W4TypeFlag@QMetaType@@@@QAE@VQFlag@@@Z 1000d900 f i KrakenBuildWorker.obj
 0001:0000c910       ??0?$QForeachContainer@V?$QList@PAVURLContainer@U2@@@@@@QAE@ABV?$QList@PAVURLContainer@U2@@@@@Z 1000d910 f i KrakenBuildWorker.obj
 0001:0000c950       ??0?$QForeachContainer@V?$QList@VDescriptor@U2@@@@@@QAE@ABV?$QList@VDescriptor@U2@@@@@Z 1000d950 f i KrakenBuildWorker.obj
 0001:0000c990       ??0?$QList@PAVURLContainer@U2@@@@QAE@ABV0@@Z 1000d990 f i KrakenBuildWorker.obj
 0001:0000ca50       ??0?$QList@VDataset@U2@@@@QAE@$$QAV0@@Z 1000da50 f i KrakenBuildWorker.obj
 0001:0000ca70       ??0?$QList@VDataset@U2@@@@QAE@ABV0@@Z 1000da70 f i KrakenBuildWorker.obj
 0001:0000cb30       ??0?$QList@VDataset@U2@@@@QAE@XZ 1000db30 f i KrakenBuildWorker.obj
 0001:0000cb40       ??0?$QList@VDescriptor@U2@@@@QAE@$$QAV0@@Z 1000db40 f i KrakenBuildWorker.obj
 0001:0000cb60       ??0?$QList@VDescriptor@U2@@@@QAE@ABV0@@Z 1000db60 f i KrakenBuildWorker.obj
 0001:0000cc20       ??0?$QList@VDescriptor@U2@@@@QAE@XZ 1000dc20 f i KrakenBuildWorker.obj
 0001:0000cc30       ??0?$QMap@VQString@@VQScriptValue@@@@QAE@XZ 1000dc30 f i KrakenBuildWorker.obj
 0001:0000cc40       ??0KrakenBuildWorker@LocalWorkflow@U2@@QAE@PAVActor@Workflow@2@@Z 1000dc40 f   KrakenBuildWorker.obj
 0001:0000cc80       ??0const_iterator@?$QList@PAVURLContainer@U2@@@@QAE@PAUNode@1@@Z 1000dc80 f i KrakenBuildWorker.obj
 0001:0000cc90       ??0const_iterator@?$QList@VDescriptor@U2@@@@QAE@PAUNode@1@@Z 1000dc90 f i KrakenBuildWorker.obj
 0001:0000cca0       ??0const_iterator@?$QMap@VDescriptor@U2@@VQVariant@@@@QAE@PBU?$QMapNode@VDescriptor@U2@@VQVariant@@@@@Z 1000dca0 f i KrakenBuildWorker.obj
 0001:0000ccb0       ??0iterator@?$QMap@VQString@@VQScriptValue@@@@QAE@PAU?$QMapNode@VQString@@VQScriptValue@@@@@Z 1000dcb0 f i KrakenBuildWorker.obj
 0001:0000ccc0       ??0iterator@?$QMap@VQString@@VQVariant@@@@QAE@PAU?$QMapNode@VQString@@VQVariant@@@@@Z 1000dcc0 f i KrakenBuildWorker.obj
 0001:0000ccd0       ??1?$QExplicitlySharedDataPointer@VDataType@U2@@@@QAE@XZ 1000dcd0 f i KrakenBuildWorker.obj
 0001:0000ccf0       ??1?$QForeachContainer@V?$QList@PAVURLContainer@U2@@@@@@QAE@XZ 1000dcf0 f i KrakenBuildWorker.obj
 0001:0000cd20       ??1?$QForeachContainer@V?$QList@VDescriptor@U2@@@@@@QAE@XZ 1000dd20 f i KrakenBuildWorker.obj
 0001:0000cd50       ??1?$QList@PAVExternalToolListener@U2@@@@QAE@XZ 1000dd50 f i KrakenBuildWorker.obj
 0001:0000cd80       ??1?$QList@PAVURLContainer@U2@@@@QAE@XZ 1000dd80 f i KrakenBuildWorker.obj
 0001:0000cdb0       ??1?$QList@VDataset@U2@@@@QAE@XZ 1000ddb0 f i KrakenBuildWorker.obj
 0001:0000cde0       ??1?$QList@VDescriptor@U2@@@@QAE@XZ 1000dde0 f i KrakenBuildWorker.obj
 0001:0000ce10       ??1?$QMap@VQString@@VQScriptValue@@@@QAE@XZ 1000de10 f i KrakenBuildWorker.obj
 0001:0000ce60       ??1KrakenBuildWorker@LocalWorkflow@U2@@UAE@XZ 1000de60 f i KrakenBuildWorker.obj
 0001:0000ce70       ??8const_iterator@?$QMap@VDescriptor@U2@@VQVariant@@@@QBE_NABV01@@Z 1000de70 f i KrakenBuildWorker.obj
 0001:0000ce90       ??9const_iterator@?$QList@PAVURLContainer@U2@@@@QBE_NABV01@@Z 1000de90 f i KrakenBuildWorker.obj
 0001:0000ceb0       ??9const_iterator@?$QList@VDescriptor@U2@@@@QBE_NABV01@@Z 1000deb0 f i KrakenBuildWorker.obj
 0001:0000ced0       ??9const_iterator@?$QMap@VDescriptor@U2@@VQVariant@@@@QBE_NABV01@@Z 1000ded0 f i KrakenBuildWorker.obj
 0001:0000cef0       ??A?$QMap@VQString@@VQScriptValue@@@@QAEAAVQScriptValue@@ABVQString@@@Z 1000def0 f i KrakenBuildWorker.obj
 0001:0000cfc0       ??A?$QMap@VQString@@VQVariant@@@@QAEAAVQVariant@@ABVQString@@@Z 1000dfc0 f i KrakenBuildWorker.obj
 0001:0000d090       ??Dconst_iterator@?$QList@PAVURLContainer@U2@@@@QBEABQAVURLContainer@U2@@XZ 1000e090 f i KrakenBuildWorker.obj
 0001:0000d0a0       ??Dconst_iterator@?$QList@VDescriptor@U2@@@@QBEABVDescriptor@U2@@XZ 1000e0a0 f i KrakenBuildWorker.obj
 0001:0000d0b0       ??Diterator@?$QMap@VQString@@VQScriptValue@@@@QBEAAVQScriptValue@@XZ 1000e0b0 f i KrakenBuildWorker.obj
 0001:0000d0c0       ??Diterator@?$QMap@VQString@@VQVariant@@@@QBEAAVQVariant@@XZ 1000e0c0 f i KrakenBuildWorker.obj
 0001:0000d0d0       ??Econst_iterator@?$QList@PAVURLContainer@U2@@@@QAEAAV01@XZ 1000e0d0 f i KrakenBuildWorker.obj
 0001:0000d0e0       ??Econst_iterator@?$QList@VDescriptor@U2@@@@QAEAAV01@XZ 1000e0e0 f i KrakenBuildWorker.obj
 0001:0000d0f0       ??Econst_iterator@?$QMap@VDescriptor@U2@@VQVariant@@@@QAEAAV01@XZ 1000e0f0 f i KrakenBuildWorker.obj
 0001:0000d110       ??_5?$QFlags@W4TypeFlag@QMetaType@@@@QAEAAV0@W4TypeFlag@QMetaType@@@Z 1000e110 f i KrakenBuildWorker.obj
 0001:0000d11e       ??_EKrakenBuildWorker@LocalWorkflow@U2@@W7AEPAXI@Z 1000e11e f i KrakenBuildWorker.obj
 0001:0000d126       ??_EKrakenBuildWorker@LocalWorkflow@U2@@WBA@AEPAXI@Z 1000e126 f i KrakenBuildWorker.obj
 0001:0000d130       ??_G?$QList@VDataset@U2@@@@QAEPAXI@Z 1000e130 f i KrakenBuildWorker.obj
 0001:0000d170       ??_GDataset@U2@@QAEPAXI@Z  1000e170 f i KrakenBuildWorker.obj
 0001:0000d1a0       ??_GDescriptor@U2@@UAEPAXI@Z 1000e1a0 f i KrakenBuildWorker.obj
 0001:0000d1a0       ??_EDescriptor@U2@@UAEPAXI@Z 1000e1a0 f i KrakenBuildWorker.obj
 0001:0000d1d0       ??_EKrakenBuildWorker@LocalWorkflow@U2@@UAEPAXI@Z 1000e1d0 f i KrakenBuildWorker.obj
 0001:0000d1d0       ??_GKrakenBuildWorker@LocalWorkflow@U2@@UAEPAXI@Z 1000e1d0 f i KrakenBuildWorker.obj
 0001:0000d200       ??_GQScriptValue@@QAEPAXI@Z 1000e200 f i KrakenBuildWorker.obj
 0001:0000d230       ??_GTaskSignalMapper@U2@@UAEPAXI@Z 1000e230 f i KrakenBuildWorker.obj
 0001:0000d230       ??_ETaskSignalMapper@U2@@UAEPAXI@Z 1000e230 f i KrakenBuildWorker.obj
 0001:0000d260       ?Construct@?$QMetaTypeFunctionHelper@V?$QList@VDataset@U2@@@@$00@QtMetaTypePrivate@@SAPAXPAXPBX@Z 1000e260 f i KrakenBuildWorker.obj
 0001:0000d2f0       ?Create@?$QMetaTypeFunctionHelper@V?$QList@VDataset@U2@@@@$00@QtMetaTypePrivate@@SAPAXPBX@Z 1000e2f0 f i KrakenBuildWorker.obj
 0001:0000d390       ?Delete@?$QMetaTypeFunctionHelper@V?$QList@VDataset@U2@@@@$00@QtMetaTypePrivate@@SAXPAX@Z 1000e390 f i KrakenBuildWorker.obj
 0001:0000d3d0       ?Destruct@?$QMetaTypeFunctionHelper@V?$QList@VDataset@U2@@@@$00@QtMetaTypePrivate@@SAXPAX@Z 1000e3d0 f i KrakenBuildWorker.obj
 0001:0000d400       ?append@?$QList@VDescriptor@U2@@@@QAEXABVDescriptor@U2@@@Z 1000e400 f i KrakenBuildWorker.obj
 0001:0000d4f0       ?at@?$QList@VDataset@U2@@@@QBEABVDataset@U2@@H@Z 1000e4f0 f i KrakenBuildWorker.obj
 0001:0000d510       ?begin@?$QList@PAVURLContainer@U2@@@@QBE?AVconst_iterator@1@XZ 1000e510 f i KrakenBuildWorker.obj
 0001:0000d530       ?begin@?$QList@VDescriptor@U2@@@@QBE?AVconst_iterator@1@XZ 1000e530 f i KrakenBuildWorker.obj
 0001:0000d550       ?begin@?$QMap@VDescriptor@U2@@VQVariant@@@@QBE?AVconst_iterator@1@XZ 1000e550 f i KrakenBuildWorker.obj
 0001:0000d570       ?begin@?$QMapData@VDescriptor@U2@@VQVariant@@@@QAEPAU?$QMapNode@VDescriptor@U2@@VQVariant@@@@XZ 1000e570 f i KrakenBuildWorker.obj
 0001:0000d580       ?cleanup@KrakenBuildWorker@LocalWorkflow@U2@@UAEXXZ 1000e580 f   KrakenBuildWorker.obj
 0001:0000d590       ?copy@?$QMapNode@VQString@@VQScriptValue@@@@QBEPAU1@PAU?$QMapData@VQString@@VQScriptValue@@@@@Z 1000e590 f i KrakenBuildWorker.obj
 0001:0000d620       ?copy@?$QMapNode@VQString@@VQVariant@@@@QBEPAU1@PAU?$QMapData@VQString@@VQVariant@@@@@Z 1000e620 f i KrakenBuildWorker.obj
 0001:0000d6b0       ?create@?$QMapData@VQString@@VQScriptValue@@@@SAPAU1@XZ 1000e6b0 f i KrakenBuildWorker.obj
 0001:0000d6c0       ?create@?$QMapData@VQString@@VQVariant@@@@SAPAU1@XZ 1000e6c0 f i KrakenBuildWorker.obj
 0001:0000d6d0       ?createNode@?$QMapData@VQString@@VQScriptValue@@@@QAEPAU?$QMapNode@VQString@@VQScriptValue@@@@ABVQString@@ABVQScriptValue@@PAU2@_N@Z 1000e6d0 f i KrakenBuildWorker.obj
 0001:0000d790       ?createNode@?$QMapData@VQString@@VQVariant@@@@QAEPAU?$QMapNode@VQString@@VQVariant@@@@ABVQString@@ABVQVariant@@PAU2@_N@Z 1000e790 f i KrakenBuildWorker.obj
 0001:0000d850       ?dealloc@?$QList@PAVExternalToolListener@U2@@@@AAEXPAUData@QListData@@@Z 1000e850 f i KrakenBuildWorker.obj
 0001:0000d870       ?dealloc@?$QList@PAVURLContainer@U2@@@@AAEXPAUData@QListData@@@Z 1000e870 f i KrakenBuildWorker.obj
 0001:0000d890       ?dealloc@?$QList@VDataset@U2@@@@AAEXPAUData@QListData@@@Z 1000e890 f i KrakenBuildWorker.obj
 0001:0000d8f0       ?dealloc@?$QList@VDescriptor@U2@@@@AAEXPAUData@QListData@@@Z 1000e8f0 f i KrakenBuildWorker.obj
 0001:0000d940       ?destroy@?$QMapData@VQString@@VQScriptValue@@@@QAEXXZ 1000e940 f i KrakenBuildWorker.obj
 0001:0000d970       ?destroySubTree@?$QMapNode@VQString@@VQScriptValue@@@@QAEXXZ 1000e970 f i KrakenBuildWorker.obj
 0001:0000d9b0       ?detach@?$QMap@VQString@@VQScriptValue@@@@QAEXXZ 1000e9b0 f i KrakenBuildWorker.obj
 0001:0000d9d0       ?detach@?$QMap@VQString@@VQVariant@@@@QAEXXZ 1000e9d0 f i KrakenBuildWorker.obj
 0001:0000d9f0       ?detach_helper@?$QList@VDescriptor@U2@@@@AAEXH@Z 1000e9f0 f i KrakenBuildWorker.obj
 0001:0000dac0       ?detach_helper@?$QMap@VQString@@VQScriptValue@@@@AAEXXZ 1000eac0 f i KrakenBuildWorker.obj
 0001:0000db40       ?detach_helper@?$QMap@VQString@@VQVariant@@@@AAEXXZ 1000eb40 f i KrakenBuildWorker.obj
 0001:0000dbc0       ?detach_helper_grow@?$QList@VDescriptor@U2@@@@AAEPAUNode@1@HH@Z 1000ebc0 f i KrakenBuildWorker.obj
 0001:0000dd10       ?end@?$QList@PAVURLContainer@U2@@@@QBE?AVconst_iterator@1@XZ 1000ed10 f i KrakenBuildWorker.obj
 0001:0000dd30       ?end@?$QList@VDescriptor@U2@@@@QBE?AVconst_iterator@1@XZ 1000ed30 f i KrakenBuildWorker.obj
 0001:0000dd50       ?end@?$QMap@VDescriptor@U2@@VQVariant@@@@QBE?AVconst_iterator@1@XZ 1000ed50 f i KrakenBuildWorker.obj
 0001:0000dd70       ?end@?$QMapData@VDescriptor@U2@@VQVariant@@@@QAEPAU?$QMapNode@VDescriptor@U2@@VQVariant@@@@XZ 1000ed70 f i KrakenBuildWorker.obj
 0001:0000dd80       ?end@?$QMapData@VQString@@VQScriptValue@@@@QAEPAU?$QMapNode@VQString@@VQScriptValue@@@@XZ 1000ed80 f i KrakenBuildWorker.obj
 0001:0000dd90       ?end@?$QMapData@VQString@@VQVariant@@@@QAEPAU?$QMapNode@VQString@@VQVariant@@@@XZ 1000ed90 f i KrakenBuildWorker.obj
 0001:0000dda0       ?findNode@?$QMapData@VDescriptor@U2@@VQVariant@@@@QBEPAU?$QMapNode@VDescriptor@U2@@VQVariant@@@@ABVDescriptor@U2@@@Z 1000eda0 f i KrakenBuildWorker.obj
 0001:0000dde0       ?findNode@?$QMapData@VQString@@PAVIntegralBus@Workflow@U2@@@@QBEPAU?$QMapNode@VQString@@PAVIntegralBus@Workflow@U2@@@@ABVQString@@@Z 1000ede0 f i KrakenBuildWorker.obj
 0001:0000de20       ?findNode@?$QMapData@VQString@@VQScriptValue@@@@QBEPAU?$QMapNode@VQString@@VQScriptValue@@@@ABVQString@@@Z 1000ee20 f i KrakenBuildWorker.obj
 0001:0000de60       ?findNode@?$QMapData@VQString@@VQVariant@@@@QBEPAU?$QMapNode@VQString@@VQVariant@@@@ABVQString@@@Z 1000ee60 f i KrakenBuildWorker.obj
 0001:0000dea0       ?first@?$QList@VDataset@U2@@@@QBEABVDataset@U2@@XZ 1000eea0 f i KrakenBuildWorker.obj
 0001:0000deb0       ?getListenersCount@KrakenBuildWorker@LocalWorkflow@U2@@ABEHABUKrakenBuildTaskSettings@3@@Z 1000eeb0 f   KrakenBuildWorker.obj
 0001:0000def0       ?getSettings@KrakenBuildWorker@LocalWorkflow@U2@@AAE?AUKrakenBuildTaskSettings@3@XZ 1000eef0 f   KrakenBuildWorker.obj
 0001:0000e2f0       ?init@KrakenBuildWorker@LocalWorkflow@U2@@UAEXXZ 1000f2f0 f   KrakenBuildWorker.obj
 0001:0000e4b0       ?insert@?$QMap@VQString@@VQScriptValue@@@@QAE?AViterator@1@ABVQString@@ABVQScriptValue@@@Z 1000f4b0 f i KrakenBuildWorker.obj
 0001:0000e570       ?insert@?$QMap@VQString@@VQVariant@@@@QAE?AViterator@1@ABVQString@@ABVQVariant@@@Z 1000f570 f i KrakenBuildWorker.obj
 0001:0000e630       ?invoke@?$MetaTypeInvoker@U?$QVariantValueHelper@V?$QList@VDataset@U2@@@@@QtPrivate@@ABVQVariant@@V?$QList@VDataset@U2@@@@@QtPrivate@@SA?AV?$QList@VDataset@U2@@@@ABVQVariant@@@Z 1000f630 f i KrakenBuildWorker.obj
 0001:0000e650       ?invoke@?$MetaTypeInvoker@U?$QVariantValueHelper@VQString@@@QtPrivate@@ABVQVariant@@VQString@@@QtPrivate@@SA?AVQString@@ABVQVariant@@@Z 1000f650 f i KrakenBuildWorker.obj
 0001:0000e670       ?invoke@?$MetaTypeInvoker@U?$QVariantValueHelper@_N@QtPrivate@@ABVQVariant@@_N@QtPrivate@@SA_NABVQVariant@@@Z 1000f670 f i KrakenBuildWorker.obj
 0001:0000e6b0       ?isEmpty@?$QList@VDataset@U2@@@@QBE_NXZ 1000f6b0 f i KrakenBuildWorker.obj
 0001:0000e6c0       ?key@const_iterator@?$QMap@VDescriptor@U2@@VQVariant@@@@QBEABVDescriptor@U2@@XZ 1000f6c0 f i KrakenBuildWorker.obj
 0001:0000e6d0       ?leftNode@?$QMapNode@VDescriptor@U2@@VQVariant@@@@QBEPAU1@XZ 1000f6d0 f i KrakenBuildWorker.obj
 0001:0000e6e0       ?leftNode@?$QMapNode@VQString@@PAVIntegralBus@Workflow@U2@@@@QBEPAU1@XZ 1000f6e0 f i KrakenBuildWorker.obj
 0001:0000e6f0       ?leftNode@?$QMapNode@VQString@@VQScriptValue@@@@QBEPAU1@XZ 1000f6f0 f i KrakenBuildWorker.obj
 0001:0000e700       ?loadAcquire@?$QBasicAtomicInteger@H@@QBEHXZ 1000f700 f i KrakenBuildWorker.obj
 0001:0000e710       ?lowerBound@?$QMapNode@VDescriptor@U2@@VQVariant@@@@QAEPAU1@ABVDescriptor@U2@@@Z 1000f710 f i KrakenBuildWorker.obj
 0001:0000e750       ?lowerBound@?$QMapNode@VQString@@PAVIntegralBus@Workflow@U2@@@@QAEPAU1@ABVQString@@@Z 1000f750 f i KrakenBuildWorker.obj
 0001:0000e790       ?lowerBound@?$QMapNode@VQString@@VQScriptValue@@@@QAEPAU1@ABVQString@@@Z 1000f790 f i KrakenBuildWorker.obj
 0001:0000e7d0       ?lowerBound@?$QMapNode@VQString@@VQVariant@@@@QAEPAU1@ABVQString@@@Z 1000f7d0 f i KrakenBuildWorker.obj
 0001:0000e810       ?metaType@?$QVariantValueHelper@V?$QList@VDataset@U2@@@@@QtPrivate@@SA?AV?$QList@VDataset@U2@@@@ABVQVariant@@@Z 1000f810 f i KrakenBuildWorker.obj
 0001:0000e900       ?metaType@?$QVariantValueHelper@VQString@@@QtPrivate@@SA?AVQString@@ABVQVariant@@@Z 1000f900 f i KrakenBuildWorker.obj
 0001:0000e9c0       ?metaType@?$QVariantValueHelper@_N@QtPrivate@@SA_NABVQVariant@@@Z 1000f9c0 f i KrakenBuildWorker.obj
 0001:0000ea00       ?nextNode@?$QMapNode@VDescriptor@U2@@VQVariant@@@@QBEPBU1@XZ 1000fa00 f i KrakenBuildWorker.obj
 0001:0000ea10       ?node_construct@?$QList@VDescriptor@U2@@@@AAEXPAUNode@1@ABVDescriptor@U2@@@Z 1000fa10 f i KrakenBuildWorker.obj
 0001:0000eaa0       ?node_copy@?$QList@PAVURLContainer@U2@@@@AAEXPAUNode@1@00@Z 1000faa0 f i KrakenBuildWorker.obj
 0001:0000ead0       ?node_copy@?$QList@VDataset@U2@@@@AAEXPAUNode@1@00@Z 1000fad0 f i KrakenBuildWorker.obj
 0001:0000eba0       ?node_copy@?$QList@VDescriptor@U2@@@@AAEXPAUNode@1@00@Z 1000fba0 f i KrakenBuildWorker.obj
 0001:0000ec70       ?node_destruct@?$QList@PAVExternalToolListener@U2@@@@AAEXPAUNode@1@0@Z 1000fc70 f i KrakenBuildWorker.obj
 0001:0000ec80       ?node_destruct@?$QList@PAVURLContainer@U2@@@@AAEXPAUNode@1@0@Z 1000fc80 f i KrakenBuildWorker.obj
 0001:0000ec90       ?node_destruct@?$QList@VDataset@U2@@@@AAEXPAUNode@1@0@Z 1000fc90 f i KrakenBuildWorker.obj
 0001:0000ecd0       ?node_destruct@?$QList@VDescriptor@U2@@@@AAEXPAUNode@1@0@Z 1000fcd0 f i KrakenBuildWorker.obj
 0001:0000ed00       ?node_destruct@?$QList@VDescriptor@U2@@@@AAEXPAUNode@1@@Z 1000fd00 f i KrakenBuildWorker.obj
 0001:0000ed20       ?qt_metatype_id@?$QMetaTypeId2@V?$QList@VDataset@U2@@@@@@SAHXZ 1000fd20 f i KrakenBuildWorker.obj
 0001:0000ed30       ?qt_metatype_id@?$QMetaTypeId2@VQString@@@@SAHXZ 1000fd30 f i KrakenBuildWorker.obj
 0001:0000ed40       ?qt_metatype_id@?$QMetaTypeId2@_N@@SAHXZ 1000fd40 f i KrakenBuildWorker.obj
 0001:0000ed50       ?qt_metatype_id@?$QMetaTypeId@V?$QList@VDataset@U2@@@@@@SAHXZ 1000fd50 f i KrakenBuildWorker.obj
 0001:0000edf0       ?qt_metatype_id@?$QMetaTypeIdHelper@V?$QList@VDataset@U2@@@@$00@QtPrivate@@SAHXZ 1000fdf0 f i KrakenBuildWorker.obj
 0001:0000ee00       ?qt_noop@@YAXXZ            1000fe00 f i KrakenBuildWorker.obj
 0001:0000ee10       ?registerConverter@?$AssociativeContainerConverterHelper@V?$QList@VDataset@U2@@@@$0A@@QtPrivate@@SA_NH@Z 1000fe10 f i KrakenBuildWorker.obj
 0001:0000ee20       ?registerConverter@?$IsPair@V?$QList@VDataset@U2@@@@@QtPrivate@@SA_NH@Z 1000fe20 f i KrakenBuildWorker.obj
 0001:0000ee30       ?registerConverter@?$MetaTypeSmartPointerHelper@V?$QList@VDataset@U2@@@@X@QtPrivate@@SA_NH@Z 1000fe30 f i KrakenBuildWorker.obj
 0001:0000ee40       ?registerConverter@?$ValueTypeIsMetaType@V?$QList@VDataset@U2@@@@$0A@@QtPrivate@@SA_NH@Z 1000fe40 f i KrakenBuildWorker.obj
 0001:0000ee50       ?reserve@?$QList@VDescriptor@U2@@@@QAEXH@Z 1000fe50 f i KrakenBuildWorker.obj
 0001:0000ee80       ?rightNode@?$QMapNode@VDescriptor@U2@@VQVariant@@@@QBEPAU1@XZ 1000fe80 f i KrakenBuildWorker.obj
 0001:0000ee90       ?rightNode@?$QMapNode@VQString@@PAVIntegralBus@Workflow@U2@@@@QBEPAU1@XZ 1000fe90 f i KrakenBuildWorker.obj
 0001:0000eea0       ?rightNode@?$QMapNode@VQString@@VQScriptValue@@@@QBEPAU1@XZ 1000fea0 f i KrakenBuildWorker.obj
 0001:0000eeb0       ?root@?$QMapData@VDescriptor@U2@@VQVariant@@@@QBEPAU?$QMapNode@VDescriptor@U2@@VQVariant@@@@XZ 1000feb0 f i KrakenBuildWorker.obj
 0001:0000eec0       ?root@?$QMapData@VQString@@PAVIntegralBus@Workflow@U2@@@@QBEPAU?$QMapNode@VQString@@PAVIntegralBus@Workflow@U2@@@@XZ 1000fec0 f i KrakenBuildWorker.obj
 0001:0000eed0       ?root@?$QMapData@VQString@@VQScriptValue@@@@QBEPAU?$QMapNode@VQString@@VQScriptValue@@@@XZ 1000fed0 f i KrakenBuildWorker.obj
 0001:0000eee0       ?size@?$QList@VQString@@@@QBEHXZ 1000fee0 f i KrakenBuildWorker.obj
 0001:0000eef0       ?size@?$QMap@VDescriptor@U2@@VQVariant@@@@QBEHXZ 1000fef0 f i KrakenBuildWorker.obj
 0001:0000ef00       ?sl_taskFinished@KrakenBuildWorker@LocalWorkflow@U2@@AAEXPAVTask@3@@Z 1000ff00 f   KrakenBuildWorker.obj
 0001:0000f190       ?storeRelease@?$QBasicAtomicInteger@H@@QAEXH@Z 10010190 f i KrakenBuildWorker.obj
 0001:0000f1a0       ?t@Node@?$QList@PAVURLContainer@U2@@@@QAEAAPAVURLContainer@U2@@XZ 100101a0 f i KrakenBuildWorker.obj
 0001:0000f1b0       ?t@Node@?$QList@VDataset@U2@@@@QAEAAVDataset@U2@@XZ 100101b0 f i KrakenBuildWorker.obj
 0001:0000f1c0       ?t@Node@?$QList@VDescriptor@U2@@@@QAEAAVDescriptor@U2@@XZ 100101c0 f i KrakenBuildWorker.obj
 0001:0000f1d0       ?tick@KrakenBuildWorker@LocalWorkflow@U2@@UAEPAVTask@3@XZ 100101d0 f   KrakenBuildWorker.obj
 0001:0000f350       ?uniqueKeys@?$QMap@VDescriptor@U2@@VQVariant@@@@QBE?AV?$QList@VDescriptor@U2@@@@XZ 10010350 f i KrakenBuildWorker.obj
 0001:0000f450       ?value@?$MetaObjectForType@V?$QList@VDataset@U2@@@@$0A@@QtPrivate@@SAPBUQMetaObject@@XZ 10010450 f i KrakenBuildWorker.obj
 0001:0000f460       ?value@?$QMap@VDescriptor@U2@@VQVariant@@@@QBE?BVQVariant@@ABVDescriptor@U2@@ABV2@@Z 10010460 f i KrakenBuildWorker.obj
 0001:0000f4c0       ?value@?$QMap@VQString@@PAVIntegralBus@Workflow@U2@@@@QBEQAVIntegralBus@Workflow@U2@@ABVQString@@ABQAV234@@Z 100104c0 f i KrakenBuildWorker.obj
 0001:0000f510       ??$_Move@AAPAVDataType@U2@@@std@@YA$$QAPAVDataType@U2@@AAPAV12@@Z 10010510 f i KrakenBuildWorkerFactory.obj
 0001:0000f520       ??$qSwap@PAVDataType@U2@@@@YAXAAPAVDataType@U2@@0@Z 10010520 f i KrakenBuildWorkerFactory.obj
 0001:0000f540       ??$swap@PAVDataType@U2@@@std@@YAXAAPAVDataType@U2@@0@Z 10010540 f i KrakenBuildWorkerFactory.obj
 0001:0000f560       ??0?$QExplicitlySharedDataPointer@VDataType@U2@@@@QAE@ABV0@@Z 10010560 f i KrakenBuildWorkerFactory.obj
 0001:0000f580       ??0?$QExplicitlySharedDataPointer@VDataType@U2@@@@QAE@PAVDataType@U2@@@Z 10010580 f i KrakenBuildWorkerFactory.obj
 0001:0000f5a0       ??0?$QExplicitlySharedDataPointer@VDataType@U2@@@@QAE@XZ 100105a0 f i KrakenBuildWorkerFactory.obj
 0001:0000f5b0       ??0?$QFlags@W4Option@URLDelegate@U2@@@@QAE@VQFlag@@@Z 100105b0 f i KrakenBuildWorkerFactory.obj
 0001:0000f5c0       ??0?$QFlags@W4Option@URLDelegate@U2@@@@QAE@W4Option@URLDelegate@U2@@@Z 100105c0 f i KrakenBuildWorkerFactory.obj
 0001:0000f5d0       ??0?$QList@PAVAttribute@U2@@@@QAE@XZ 100105d0 f i KrakenBuildWorkerFactory.obj
 0001:0000f5e0       ??0?$QList@PAVPortDescriptor@Workflow@U2@@@@QAE@XZ 100105e0 f i KrakenBuildWorkerFactory.obj
 0001:0000f5f0       ??0?$QMap@VDescriptor@U2@@V?$QExplicitlySharedDataPointer@VDataType@U2@@@@@@QAE@XZ 100105f0 f i KrakenBuildWorkerFactory.obj
 0001:0000f600       ??0?$QMap@VQString@@PAVPropertyDelegate@U2@@@@QAE@XZ 10010600 f i KrakenBuildWorkerFactory.obj
 0001:0000f610       ??0KrakenBuildValidator@Workflow@U2@@QAE@XZ 10010610 f i KrakenBuildWorkerFactory.obj
 0001:0000f620       ??0KrakenBuildWorkerFactory@LocalWorkflow@U2@@QAE@XZ 10010620 f   KrakenBuildWorkerFactory.obj
 0001:0000f640       ??0iterator@?$QMap@VDescriptor@U2@@V?$QExplicitlySharedDataPointer@VDataType@U2@@@@@@QAE@PAU?$QMapNode@VDescriptor@U2@@V?$QExplicitlySharedDataPointer@VDataType@U2@@@@@@@Z 10010640 f i KrakenBuildWorkerFactory.obj
 0001:0000f650       ??0iterator@?$QMap@VQString@@PAVPropertyDelegate@U2@@@@QAE@PAU?$QMapNode@VQString@@PAVPropertyDelegate@U2@@@@@Z 10010650 f i KrakenBuildWorkerFactory.obj
 0001:0000f660       ??1?$QList@PAVAttribute@U2@@@@QAE@XZ 10010660 f i KrakenBuildWorkerFactory.obj
 0001:0000f690       ??1?$QList@PAVPortDescriptor@Workflow@U2@@@@QAE@XZ 10010690 f i KrakenBuildWorkerFactory.obj
 0001:0000f6c0       ??1?$QMap@VDescriptor@U2@@V?$QExplicitlySharedDataPointer@VDataType@U2@@@@@@QAE@XZ 100106c0 f i KrakenBuildWorkerFactory.obj
 0001:0000f710       ??1?$QMap@VQString@@PAVPropertyDelegate@U2@@@@QAE@XZ 10010710 f i KrakenBuildWorkerFactory.obj
 0001:0000f780       ??1KrakenBuildValidator@Workflow@U2@@UAE@XZ 10010780 f i KrakenBuildWorkerFactory.obj
 0001:0000f790       ??1KrakenBuildWorkerFactory@LocalWorkflow@U2@@UAE@XZ 10010790 f i KrakenBuildWorkerFactory.obj
 0001:0000f7a0       ??4?$QExplicitlySharedDataPointer@VDataType@U2@@@@QAEAAV0@$$QAV0@@Z 100107a0 f i KrakenBuildWorkerFactory.obj
 0001:0000f7c0       ??4?$QExplicitlySharedDataPointer@VDataType@U2@@@@QAEAAV0@ABV0@@Z 100107c0 f i KrakenBuildWorkerFactory.obj
 0001:0000f810       ??6?$QList@PAVAttribute@U2@@@@QAEAAV0@ABQAVAttribute@U2@@@Z 10010810 f i KrakenBuildWorkerFactory.obj
 0001:0000f830       ??6?$QList@PAVPortDescriptor@Workflow@U2@@@@QAEAAV0@ABQAVPortDescriptor@Workflow@U2@@@Z 10010830 f i KrakenBuildWorkerFactory.obj
 0001:0000f850       ??A?$QMap@VDescriptor@U2@@V?$QExplicitlySharedDataPointer@VDataType@U2@@@@@@QAEAAV?$QExplicitlySharedDataPointer@VDataType@U2@@@@ABVDescriptor@U2@@@Z 10010850 f i KrakenBuildWorkerFactory.obj
 0001:0000f910       ??A?$QMap@VQString@@PAVPropertyDelegate@U2@@@@QAEAAPAVPropertyDelegate@U2@@ABVQString@@@Z 10010910 f i KrakenBuildWorkerFactory.obj
 0001:0000f990       ??Diterator@?$QMap@VDescriptor@U2@@V?$QExplicitlySharedDataPointer@VDataType@U2@@@@@@QBEAAV?$QExplicitlySharedDataPointer@VDataType@U2@@@@XZ 10010990 f i KrakenBuildWorkerFactory.obj
 0001:0000f9a0       ??Diterator@?$QMap@VQString@@PAVPropertyDelegate@U2@@@@QBEAAPAVPropertyDelegate@U2@@XZ 100109a0 f i KrakenBuildWorkerFactory.obj
 0001:0000f9b0       ??U?$QFlags@W4Option@URLDelegate@U2@@@@QBE?AV0@W4Option@URLDelegate@U2@@@Z 100109b0 f i KrakenBuildWorkerFactory.obj
 0001:0000f9d0       ??U@YA?AV?$QFlags@W4Option@URLDelegate@U2@@@@W4Option@URLDelegate@U2@@0@Z 100109d0 f i KrakenBuildWorkerFactory.obj
 0001:0000f9e0       ??_EIntegralBusActorPrototype@Workflow@U2@@W7AEPAXI@Z 100109e0 f i KrakenBuildWorkerFactory.obj
 0001:0000f9e8       ??_EKrakenBuildWorkerFactory@LocalWorkflow@U2@@W7AEPAXI@Z 100109e8 f i KrakenBuildWorkerFactory.obj
 0001:0000f9f0       ??_G?$QExplicitlySharedDataPointer@VDataType@U2@@@@QAEPAXI@Z 100109f0 f i KrakenBuildWorkerFactory.obj
 0001:0000fa30       ??_EAttribute@U2@@UAEPAXI@Z 10010a30 f i KrakenBuildWorkerFactory.obj
 0001:0000fa30       ??_GAttribute@U2@@UAEPAXI@Z 10010a30 f i KrakenBuildWorkerFactory.obj
 0001:0000fa60       ??_GComboBoxDelegate@U2@@UAEPAXI@Z 10010a60 f i KrakenBuildWorkerFactory.obj
 0001:0000fa60       ??_EComboBoxDelegate@U2@@UAEPAXI@Z 10010a60 f i KrakenBuildWorkerFactory.obj
 0001:0000fa90       ??_GComboBoxWithBoolsDelegate@U2@@UAEPAXI@Z 10010a90 f i KrakenBuildWorkerFactory.obj
 0001:0000fa90       ??_EComboBoxWithBoolsDelegate@U2@@UAEPAXI@Z 10010a90 f i KrakenBuildWorkerFactory.obj
 0001:0000fac0       ??_GDelegateEditor@U2@@UAEPAXI@Z 10010ac0 f i KrakenBuildWorkerFactory.obj
 0001:0000fac0       ??_EDelegateEditor@U2@@UAEPAXI@Z 10010ac0 f i KrakenBuildWorkerFactory.obj
 0001:0000faf0       ??_GGenomicLibraryDelegate@LocalWorkflow@U2@@UAEPAXI@Z 10010af0 f i KrakenBuildWorkerFactory.obj
 0001:0000faf0       ??_EGenomicLibraryDelegate@LocalWorkflow@U2@@UAEPAXI@Z 10010af0 f i KrakenBuildWorkerFactory.obj
 0001:0000fb20       ??_GIntegralBusActorPrototype@Workflow@U2@@UAEPAXI@Z 10010b20 f i KrakenBuildWorkerFactory.obj
 0001:0000fb20       ??_EIntegralBusActorPrototype@Workflow@U2@@UAEPAXI@Z 10010b20 f i KrakenBuildWorkerFactory.obj
 0001:0000fb50       ??_GKrakenBuildValidator@Workflow@U2@@UAEPAXI@Z 10010b50 f i KrakenBuildWorkerFactory.obj
 0001:0000fb50       ??_EKrakenBuildValidator@Workflow@U2@@UAEPAXI@Z 10010b50 f i KrakenBuildWorkerFactory.obj
 0001:0000fb80       ??_EKrakenBuildWorkerFactory@LocalWorkflow@U2@@UAEPAXI@Z 10010b80 f i KrakenBuildWorkerFactory.obj
 0001:0000fb80       ??_GKrakenBuildWorkerFactory@LocalWorkflow@U2@@UAEPAXI@Z 10010b80 f i KrakenBuildWorkerFactory.obj
 0001:0000fbb0       ??_GMapDataType@U2@@UAEPAXI@Z 10010bb0 f i KrakenBuildWorkerFactory.obj
 0001:0000fbb0       ??_EMapDataType@U2@@UAEPAXI@Z 10010bb0 f i KrakenBuildWorkerFactory.obj
 0001:0000fbe0       ??_GPortDescriptor@Workflow@U2@@UAEPAXI@Z 10010be0 f i KrakenBuildWorkerFactory.obj
 0001:0000fbe0       ??_EPortDescriptor@Workflow@U2@@UAEPAXI@Z 10010be0 f i KrakenBuildWorkerFactory.obj
 0001:0000fc10       ??_GSpinBoxDelegate@U2@@UAEPAXI@Z 10010c10 f i KrakenBuildWorkerFactory.obj
 0001:0000fc10       ??_ESpinBoxDelegate@U2@@UAEPAXI@Z 10010c10 f i KrakenBuildWorkerFactory.obj
 0001:0000fc40       ??_EURLDelegate@U2@@UAEPAXI@Z 10010c40 f i KrakenBuildWorkerFactory.obj
 0001:0000fc40       ??_GURLDelegate@U2@@UAEPAXI@Z 10010c40 f i KrakenBuildWorkerFactory.obj
 0001:0000fc70       ??_EVisibilityRelation@U2@@UAEPAXI@Z 10010c70 f i KrakenBuildWorkerFactory.obj
 0001:0000fc70       ??_GVisibilityRelation@U2@@UAEPAXI@Z 10010c70 f i KrakenBuildWorkerFactory.obj
 0001:0000fca0       ?append@?$QList@PAVAttribute@U2@@@@QAEXABQAVAttribute@U2@@@Z 10010ca0 f i KrakenBuildWorkerFactory.obj
 0001:0000fd30       ?append@?$QList@PAVPortDescriptor@Workflow@U2@@@@QAEXABQAVPortDescriptor@Workflow@U2@@@Z 10010d30 f i KrakenBuildWorkerFactory.obj
 0001:0000fdc0       ?cleanup@KrakenBuildWorkerFactory@LocalWorkflow@U2@@SAXXZ 10010dc0 f   KrakenBuildWorkerFactory.obj
 0001:0000fe10       ?copy@?$QMapNode@VDescriptor@U2@@V?$QExplicitlySharedDataPointer@VDataType@U2@@@@@@QBEPAU1@PAU?$QMapData@VDescriptor@U2@@V?$QExplicitlySharedDataPointer@VDataType@U2@@@@@@@Z 10010e10 f i KrakenBuildWorkerFactory.obj
 0001:0000fea0       ?copy@?$QMapNode@VQString@@PAVPropertyDelegate@U2@@@@QBEPAU1@PAU?$QMapData@VQString@@PAVPropertyDelegate@U2@@@@@Z 10010ea0 f i KrakenBuildWorkerFactory.obj
 0001:0000ff30       ?create@?$QMapData@VDescriptor@U2@@V?$QExplicitlySharedDataPointer@VDataType@U2@@@@@@SAPAU1@XZ 10010f30 f i KrakenBuildWorkerFactory.obj
 0001:0000ff40       ?create@?$QMapData@VQString@@PAVPropertyDelegate@U2@@@@SAPAU1@XZ 10010f40 f i KrakenBuildWorkerFactory.obj
 0001:0000ff50       ?createNode@?$QMapData@VDescriptor@U2@@V?$QExplicitlySharedDataPointer@VDataType@U2@@@@@@QAEPAU?$QMapNode@VDescriptor@U2@@V?$QExplicitlySharedDataPointer@VDataType@U2@@@@@@ABVDescriptor@U2@@ABV?$QExplicitlySharedDataPointer@VDataType@U2@@@@PAU2@_N@Z 10010f50 f i KrakenBuildWorkerFactory.obj
 0001:00010010       ?createNode@?$QMapData@VQString@@PAVPropertyDelegate@U2@@@@QAEPAU?$QMapNode@VQString@@PAVPropertyDelegate@U2@@@@ABVQString@@ABQAVPropertyDelegate@U2@@PAU2@_N@Z 10011010 f i KrakenBuildWorkerFactory.obj
 0001:000100b0       ?createWorker@KrakenBuildWorkerFactory@LocalWorkflow@U2@@UAEPAVWorker@Workflow@3@PAVActor@53@@Z 100110b0 f   KrakenBuildWorkerFactory.obj
 0001:00010120       ?dealloc@?$QList@PAVAttribute@U2@@@@AAEXPAUData@QListData@@@Z 10011120 f i KrakenBuildWorkerFactory.obj
 0001:00010140       ?dealloc@?$QList@PAVPortDescriptor@Workflow@U2@@@@AAEXPAUData@QListData@@@Z 10011140 f i KrakenBuildWorkerFactory.obj
 0001:00010160       ?destroy@?$QMapData@VDescriptor@U2@@V?$QExplicitlySharedDataPointer@VDataType@U2@@@@@@QAEXXZ 10011160 f i KrakenBuildWorkerFactory.obj
 0001:00010190       ?destroy@?$QMapData@VQString@@PAVPropertyDelegate@U2@@@@QAEXXZ 10011190 f i KrakenBuildWorkerFactory.obj
 0001:000101e0       ?destroySubTree@?$QMapNode@VDescriptor@U2@@V?$QExplicitlySharedDataPointer@VDataType@U2@@@@@@QAEXXZ 100111e0 f i KrakenBuildWorkerFactory.obj
 0001:00010230       ?destroySubTree@?$QMapNode@VQString@@PAVPropertyDelegate@U2@@@@QAEXXZ 10011230 f i KrakenBuildWorkerFactory.obj
 0001:00010260       ?detach@?$QMap@VDescriptor@U2@@V?$QExplicitlySharedDataPointer@VDataType@U2@@@@@@QAEXXZ 10011260 f i KrakenBuildWorkerFactory.obj
 0001:00010280       ?detach@?$QMap@VQString@@PAVPropertyDelegate@U2@@@@QAEXXZ 10011280 f i KrakenBuildWorkerFactory.obj
 0001:000102a0       ?detach_helper@?$QMap@VDescriptor@U2@@V?$QExplicitlySharedDataPointer@VDataType@U2@@@@@@AAEXXZ 100112a0 f i KrakenBuildWorkerFactory.obj
 0001:00010320       ?detach_helper@?$QMap@VQString@@PAVPropertyDelegate@U2@@@@AAEXXZ 10011320 f i KrakenBuildWorkerFactory.obj
 0001:000103d0       ?detach_helper_grow@?$QList@PAVAttribute@U2@@@@AAEPAUNode@1@HH@Z 100113d0 f i KrakenBuildWorkerFactory.obj
 0001:000104e0       ?detach_helper_grow@?$QList@PAVPortDescriptor@Workflow@U2@@@@AAEPAUNode@1@HH@Z 100114e0 f i KrakenBuildWorkerFactory.obj
 0001:000105f0       ?end@?$QMapData@VDescriptor@U2@@V?$QExplicitlySharedDataPointer@VDataType@U2@@@@@@QAEPAU?$QMapNode@VDescriptor@U2@@V?$QExplicitlySharedDataPointer@VDataType@U2@@@@@@XZ 100115f0 f i KrakenBuildWorkerFactory.obj
 0001:00010600       ?end@?$QMapData@VQString@@PAVPropertyDelegate@U2@@@@QAEPAU?$QMapNode@VQString@@PAVPropertyDelegate@U2@@@@XZ 10011600 f i KrakenBuildWorkerFactory.obj
 0001:00010610       ?findNode@?$QMapData@VDescriptor@U2@@V?$QExplicitlySharedDataPointer@VDataType@U2@@@@@@QBEPAU?$QMapNode@VDescriptor@U2@@V?$QExplicitlySharedDataPointer@VDataType@U2@@@@@@ABVDescriptor@U2@@@Z 10011610 f i KrakenBuildWorkerFactory.obj
 0001:00010650       ?findNode@?$QMapData@VQString@@PAVPropertyDelegate@U2@@@@QBEPAU?$QMapNode@VQString@@PAVPropertyDelegate@U2@@@@ABVQString@@@Z 10011650 f i KrakenBuildWorkerFactory.obj
 0001:00010690       ?init@KrakenBuildWorkerFactory@LocalWorkflow@U2@@SAXXZ 10011690 f   KrakenBuildWorkerFactory.obj
 0001:00012bc0       ?insert@?$QMap@VDescriptor@U2@@V?$QExplicitlySharedDataPointer@VDataType@U2@@@@@@QAE?AViterator@1@ABVDescriptor@U2@@ABV?$QExplicitlySharedDataPointer@VDataType@U2@@@@@Z 10013bc0 f i KrakenBuildWorkerFactory.obj
 0001:00012cc0       ?insert@?$QMap@VQString@@PAVPropertyDelegate@U2@@@@QAE?AViterator@1@ABVQString@@ABQAVPropertyDelegate@U2@@@Z 10013cc0 f i KrakenBuildWorkerFactory.obj
 0001:00012d80       ?leftNode@?$QMapNode@VDescriptor@U2@@V?$QExplicitlySharedDataPointer@VDataType@U2@@@@@@QBEPAU1@XZ 10013d80 f i KrakenBuildWorkerFactory.obj
 0001:00012d90       ?leftNode@?$QMapNode@VQString@@PAVPropertyDelegate@U2@@@@QBEPAU1@XZ 10013d90 f i KrakenBuildWorkerFactory.obj
 0001:00012da0       ?lowerBound@?$QMapNode@VDescriptor@U2@@V?$QExplicitlySharedDataPointer@VDataType@U2@@@@@@QAEPAU1@ABVDescriptor@U2@@@Z 10013da0 f i KrakenBuildWorkerFactory.obj
 0001:00012de0       ?lowerBound@?$QMapNode@VQString@@PAVPropertyDelegate@U2@@@@QAEPAU1@ABVQString@@@Z 10013de0 f i KrakenBuildWorkerFactory.obj
 0001:00012e20       ?max@?$numeric_limits@H@std@@SAHXZ 10013e20 f i KrakenBuildWorkerFactory.obj
 0001:00012e30       ?node_construct@?$QList@PAVAttribute@U2@@@@AAEXPAUNode@1@ABQAVAttribute@U2@@@Z 10013e30 f i KrakenBuildWorkerFactory.obj
 0001:00012e50       ?node_construct@?$QList@PAVPortDescriptor@Workflow@U2@@@@AAEXPAUNode@1@ABQAVPortDescriptor@Workflow@U2@@@Z 10013e50 f i KrakenBuildWorkerFactory.obj
 0001:00012e70       ?node_copy@?$QList@PAVAttribute@U2@@@@AAEXPAUNode@1@00@Z 10013e70 f i KrakenBuildWorkerFactory.obj
 0001:00012ea0       ?node_copy@?$QList@PAVPortDescriptor@Workflow@U2@@@@AAEXPAUNode@1@00@Z 10013ea0 f i KrakenBuildWorkerFactory.obj
 0001:00012ed0       ?node_destruct@?$QList@PAVAttribute@U2@@@@AAEXPAUNode@1@0@Z 10013ed0 f i KrakenBuildWorkerFactory.obj
 0001:00012ee0       ?node_destruct@?$QList@PAVAttribute@U2@@@@AAEXPAUNode@1@@Z 10013ee0 f i KrakenBuildWorkerFactory.obj
 0001:00012ef0       ?node_destruct@?$QList@PAVPortDescriptor@Workflow@U2@@@@AAEXPAUNode@1@0@Z 10013ef0 f i KrakenBuildWorkerFactory.obj
 0001:00012f00       ?node_destruct@?$QList@PAVPortDescriptor@Workflow@U2@@@@AAEXPAUNode@1@@Z 10013f00 f i KrakenBuildWorkerFactory.obj
 0001:00012f10       ?rightNode@?$QMapNode@VDescriptor@U2@@V?$QExplicitlySharedDataPointer@VDataType@U2@@@@@@QBEPAU1@XZ 10013f10 f i KrakenBuildWorkerFactory.obj
 0001:00012f20       ?rightNode@?$QMapNode@VQString@@PAVPropertyDelegate@U2@@@@QBEPAU1@XZ 10013f20 f i KrakenBuildWorkerFactory.obj
 0001:00012f30       ?root@?$QMapData@VDescriptor@U2@@V?$QExplicitlySharedDataPointer@VDataType@U2@@@@@@QBEPAU?$QMapNode@VDescriptor@U2@@V?$QExplicitlySharedDataPointer@VDataType@U2@@@@@@XZ 10013f30 f i KrakenBuildWorkerFactory.obj
 0001:00012f40       ?root@?$QMapData@VQString@@PAVPropertyDelegate@U2@@@@QBEPAU?$QMapNode@VQString@@PAVPropertyDelegate@U2@@@@XZ 10013f40 f i KrakenBuildWorkerFactory.obj
 0001:00012f50       ?tr@KrakenSupport@U2@@SA?AVQString@@PBD0H@Z 10013f50 f i KrakenBuildWorkerFactory.obj
 0001:00012f80       ??0KrakenClassifyLogParser@U2@@QAE@XZ 10013f80 f   KrakenClassifyLogParser.obj
 0001:00012fa0       ??1KrakenClassifyLogParser@U2@@UAE@XZ 10013fa0 f i KrakenClassifyLogParser.obj
 0001:00012fb0       ??_EKrakenClassifyLogParser@U2@@UAEPAXI@Z 10013fb0 f i KrakenClassifyLogParser.obj
 0001:00012fb0       ??_GKrakenClassifyLogParser@U2@@UAEPAXI@Z 10013fb0 f i KrakenClassifyLogParser.obj
 0001:00012fe0       ?initWellKnownErrors@KrakenClassifyLogParser@U2@@CA?AVQStringList@@XZ 10013fe0 f   KrakenClassifyLogParser.obj
 0001:000131b0       ?isError@KrakenClassifyLogParser@U2@@EBE_NABVQString@@@Z 100141b0 f   KrakenClassifyLogParser.obj
 0001:00013320       ??0?$PrompterBase@VKrakenClassifyPrompter@LocalWorkflow@U2@@@U2@@QAE@PAVActor@Workflow@1@_N@Z 10014320 f i KrakenClassifyPrompter.obj
 0001:00013350       ??0KrakenClassifyPrompter@LocalWorkflow@U2@@QAE@PAVActor@Workflow@2@@Z 10014350 f   KrakenClassifyPrompter.obj
 0001:00013380       ??1?$PrompterBase@VKrakenClassifyPrompter@LocalWorkflow@U2@@@U2@@UAE@XZ 10014380 f i KrakenClassifyPrompter.obj
 0001:00013390       ??1KrakenClassifyPrompter@LocalWorkflow@U2@@UAE@XZ 10014390 f i KrakenClassifyPrompter.obj
 0001:00013396       ??_E?$PrompterBase@VKrakenClassifyPrompter@LocalWorkflow@U2@@@U2@@WM@AEPAXI@Z 10014396 f i KrakenClassifyPrompter.obj
 0001:0001339e       ??_EKrakenClassifyPrompter@LocalWorkflow@U2@@WM@AEPAXI@Z 1001439e f i KrakenClassifyPrompter.obj
 0001:000133b0       ??_G?$PrompterBase@VKrakenClassifyPrompter@LocalWorkflow@U2@@@U2@@UAEPAXI@Z 100143b0 f i KrakenClassifyPrompter.obj
 0001:000133b0       ??_E?$PrompterBase@VKrakenClassifyPrompter@LocalWorkflow@U2@@@U2@@UAEPAXI@Z 100143b0 f i KrakenClassifyPrompter.obj
 0001:000133e0       ??_EKrakenClassifyPrompter@LocalWorkflow@U2@@UAEPAXI@Z 100143e0 f i KrakenClassifyPrompter.obj
 0001:000133e0       ??_GKrakenClassifyPrompter@LocalWorkflow@U2@@UAEPAXI@Z 100143e0 f i KrakenClassifyPrompter.obj
 0001:00013410       ?composeRichDoc@KrakenClassifyPrompter@LocalWorkflow@U2@@EAE?AVQString@@XZ 10014410 f   KrakenClassifyPrompter.obj
 0001:00013660       ?createDescription@?$PrompterBase@VKrakenClassifyPrompter@LocalWorkflow@U2@@@U2@@UAEPAVActorDocument@Workflow@2@PAVActor@42@@Z 10014660 f i KrakenClassifyPrompter.obj
 0001:00013900       ?tr@KrakenClassifyPrompter@LocalWorkflow@U2@@SA?AVQString@@PBD0H@Z 10014900 f i KrakenClassifyPrompter.obj
 0001:00013930       ??0?$QFlags@W4OpenModeFlag@QIODevice@@@@QAE@W4OpenModeFlag@QIODevice@@@Z 10014930 f i KrakenClassifyTask.obj
 0001:00013940       ??0?$QMap@VQString@@I@@QAE@XZ 10014940 f i KrakenClassifyTask.obj
 0001:00013950       ??0KrakenClassifyTask@U2@@QAE@ABUKrakenClassifyTaskSettings@1@@Z 10014950 f   KrakenClassifyTask.obj
 0001:00013b20       ??0KrakenClassifyTaskSettings@U2@@QAE@ABU01@@Z 10014b20 f i KrakenClassifyTask.obj
 0001:00013bc0       ??0KrakenClassifyTaskSettings@U2@@QAE@XZ 10014bc0 f   KrakenClassifyTask.obj
 0001:00013c50       ??0iterator@?$QMap@VQString@@I@@QAE@PAU?$QMapNode@VQString@@I@@@Z 10014c50 f i KrakenClassifyTask.obj
 0001:00013c60       ??1?$QList@VQByteArray@@@@QAE@XZ 10014c60 f i KrakenClassifyTask.obj
 0001:00013cc0       ??1?$QMap@VQString@@I@@QAE@XZ 10014cc0 f i KrakenClassifyTask.obj
 0001:00013d30       ??1KrakenClassifyTask@U2@@UAE@XZ 10014d30 f i KrakenClassifyTask.obj
 0001:00013dd0       ??1KrakenClassifyTaskSettings@U2@@QAE@XZ 10014dd0 f i KrakenClassifyTask.obj
 0001:00013e50       ??A?$QList@VQByteArray@@@@QAEAAVQByteArray@@H@Z 10014e50 f i KrakenClassifyTask.obj
 0001:00013e80       ??_GKrakenClassifyTask@U2@@UAEPAXI@Z 10014e80 f i KrakenClassifyTask.obj
 0001:00013e80       ??_EKrakenClassifyTask@U2@@UAEPAXI@Z 10014e80 f i KrakenClassifyTask.obj
 0001:00013eb0       ??_GQByteArray@@QAEPAXI@Z  10014eb0 f i KrakenClassifyTask.obj
 0001:00013ee0       ?contains@?$QMap@VQString@@I@@QBE_NABVQString@@@Z 10014ee0 f i KrakenClassifyTask.obj
 0001:00013f20       ?copy@?$QMapNode@VQString@@I@@QBEPAU1@PAU?$QMapData@VQString@@I@@@Z 10014f20 f i KrakenClassifyTask.obj
 0001:00013fb0       ?create@?$QMapData@VQString@@I@@SAPAU1@XZ 10014fb0 f i KrakenClassifyTask.obj
 0001:00013fc0       ?createNode@?$QMapData@VQString@@I@@QAEPAU?$QMapNode@VQString@@I@@ABVQString@@ABIPAU2@_N@Z 10014fc0 f i KrakenClassifyTask.obj
 0001:00014060       ?dealloc@?$QList@VQByteArray@@@@AAEXPAUData@QListData@@@Z 10015060 f i KrakenClassifyTask.obj
 0001:000140a0       ?destroy@?$QMapData@VQString@@I@@QAEXXZ 100150a0 f i KrakenClassifyTask.obj
 0001:000140f0       ?destroySubTree@?$QMapNode@VQString@@I@@QAEXXZ 100150f0 f i KrakenClassifyTask.obj
 0001:00014120       ?detach@?$QList@VQByteArray@@@@QAEXXZ 10015120 f i KrakenClassifyTask.obj
 0001:00014140       ?detach@?$QMap@VQString@@I@@QAEXXZ 10015140 f i KrakenClassifyTask.obj
 0001:00014160       ?detach_helper@?$QList@VQByteArray@@@@AAEXH@Z 10015160 f i KrakenClassifyTask.obj
 0001:00014250       ?detach_helper@?$QList@VQByteArray@@@@AAEXXZ 10015250 f i KrakenClassifyTask.obj
 0001:00014260       ?detach_helper@?$QMap@VQString@@I@@AAEXXZ 10015260 f i KrakenClassifyTask.obj
 0001:00014310       ?end@?$QMapData@VQString@@I@@QAEPAU?$QMapNode@VQString@@I@@XZ 10015310 f i KrakenClassifyTask.obj
 0001:00014320       ?findNode@?$QMapData@VQString@@I@@QBEPAU?$QMapNode@VQString@@I@@ABVQString@@@Z 10015320 f i KrakenClassifyTask.obj
 0001:00014360       ?getArguments@KrakenClassifyTask@U2@@AAE?AVQStringList@@XZ 10015360 f   KrakenClassifyTask.obj
 0001:00014600       ?getClassificationUrl@KrakenClassifyTask@U2@@QBEABVQString@@XZ 10015600 f   KrakenClassifyTask.obj
 0001:00014610       ?getParsedReport@KrakenClassifyTask@U2@@QBEABV?$QMap@VQString@@I@@XZ 10015610 f   KrakenClassifyTask.obj
 0001:00014620       ?insert@?$QMap@VQString@@I@@QAE?AViterator@1@ABVQString@@ABI@Z 10015620 f i KrakenClassifyTask.obj
 0001:000146e0       ?leftNode@?$QMapNode@VQString@@I@@QBEPAU1@XZ 100156e0 f i KrakenClassifyTask.obj
 0001:000146f0       ?lowerBound@?$QMapNode@VQString@@I@@QAEPAU1@ABVQString@@@Z 100156f0 f i KrakenClassifyTask.obj
 0001:00014730       ?node_copy@?$QList@VQByteArray@@@@AAEXPAUNode@1@00@Z 10015730 f i KrakenClassifyTask.obj
 0001:000147d0       ?node_destruct@?$QList@VQByteArray@@@@AAEXPAUNode@1@0@Z 100157d0 f i KrakenClassifyTask.obj
 0001:00014800       ?prepare@KrakenClassifyTask@U2@@EAEXXZ 10015800 f   KrakenClassifyTask.obj
 0001:000149a0       ?rightNode@?$QMapNode@VQString@@I@@QBEPAU1@XZ 100159a0 f i KrakenClassifyTask.obj
 0001:000149b0       ?root@?$QMapData@VQString@@I@@QBEPAU?$QMapNode@VQString@@I@@XZ 100159b0 f i KrakenClassifyTask.obj
 0001:000149c0       ?run@KrakenClassifyTask@U2@@EAEXXZ 100159c0 f   KrakenClassifyTask.obj
 0001:00014e20       ?size@?$QList@VQByteArray@@@@QBEHXZ 10015e20 f i KrakenClassifyTask.obj
 0001:00014e30       ?t@Node@?$QList@VQByteArray@@@@QAEAAVQByteArray@@XZ 10015e30 f i KrakenClassifyTask.obj
 0001:00014e40       ?tr@KrakenClassifyTask@U2@@SA?AVQString@@PBD0H@Z 10015e40 f i KrakenClassifyTask.obj
 0001:00014e70       ?tr@KrakenClassifyValidator@Workflow@U2@@SA?AVQString@@PBD0H@Z 10015e70 f i KrakenClassifyValidator.obj
 0001:00014ea0       ?validate@KrakenClassifyValidator@Workflow@U2@@UBE_NPBVActor@23@AAV?$QList@VWorkflowNotification@U2@@@@ABV?$QMap@VQString@@V1@@@@Z 10015ea0 f   KrakenClassifyValidator.obj
 0001:00014ec0       ?validateDatabase@KrakenClassifyValidator@Workflow@U2@@ABE_NPBVActor@23@AAV?$QList@VWorkflowNotification@U2@@@@@Z 10015ec0 f   KrakenClassifyValidator.obj
 0001:00015470       ??$?0V?$QMap@VQString@@I@@@QAssociativeIterableImpl@QtMetaTypePrivate@@QAE@PBV?$QMap@VQString@@I@@@Z 10016470 f i KrakenClassifyWorker.obj
 0001:000154e0       ??$_Advance@Vconst_iterator@?$QMap@VQString@@I@@H@std@@YAXAAVconst_iterator@?$QMap@VQString@@I@@HUbidirectional_iterator_tag@0@@Z 100164e0 f i KrakenClassifyWorker.obj
 0001:00015520       ??$_Distance2@Vconst_iterator@?$QMap@VQString@@I@@H@std@@YAXVconst_iterator@?$QMap@VQString@@I@@0AAHUbidirectional_iterator_tag@0@@Z 10016520 f i KrakenClassifyWorker.obj
 0001:00015550       ??$_Iter_cat@Vconst_iterator@?$QMap@VQString@@I@@@std@@YA?AUbidirectional_iterator_tag@0@ABVconst_iterator@?$QMap@VQString@@I@@@Z 10016550 f i KrakenClassifyWorker.obj
 0001:00015560       ??$advance@Vconst_iterator@?$QMap@VQString@@I@@H@std@@YAXAAVconst_iterator@?$QMap@VQString@@I@@H@Z 10016560 f i KrakenClassifyWorker.obj
 0001:000155a0       ??$advanceImpl@V?$QMap@VQString@@I@@@QAssociativeIterableImpl@QtMetaTypePrivate@@SAXPAPAXH@Z 100165a0 f i KrakenClassifyWorker.obj
 0001:000155e0       ??$beginImpl@V?$QMap@VQString@@I@@@QAssociativeIterableImpl@QtMetaTypePrivate@@SAXPBXPAPAX@Z 100165e0 f i KrakenClassifyWorker.obj
 0001:00015620       ??$distance@Vconst_iterator@?$QMap@VQString@@I@@@std@@YAHVconst_iterator@?$QMap@VQString@@I@@0@Z 10016620 f i KrakenClassifyWorker.obj
 0001:00015650       ??$endImpl@V?$QMap@VQString@@I@@@QAssociativeIterableImpl@QtMetaTypePrivate@@SAXPBXPAPAX@Z 10016650 f i KrakenClassifyWorker.obj
 0001:00015680       ??$findImpl@V?$QMap@VQString@@I@@@QAssociativeIterableImpl@QtMetaTypePrivate@@SAXPBX0PAPAX@Z 10016680 f i KrakenClassifyWorker.obj
 0001:000156e0       ??$fromValue@V?$QMap@VQString@@I@@@QVariant@@SA?AV0@ABV?$QMap@VQString@@I@@@Z 100166e0 f i KrakenClassifyWorker.obj
 0001:00015700       ??$getKeyImpl@V?$QMap@VQString@@I@@@QAssociativeIterableImpl@QtMetaTypePrivate@@SA?AUVariantData@1@PBQAXHI@Z 10016700 f i KrakenClassifyWorker.obj
 0001:00015720       ??$getValueImpl@V?$QMap@VQString@@I@@@QAssociativeIterableImpl@QtMetaTypePrivate@@SA?AUVariantData@1@PBQAXHI@Z 10016720 f i KrakenClassifyWorker.obj
 0001:00015740       ??$qMetaTypeId@I@@YAHXZ    10016740 f i KrakenClassifyWorker.obj
 0001:00015750       ??$qMetaTypeId@V?$QMap@VQString@@I@@@@YAHXZ 10016750 f i KrakenClassifyWorker.obj
 0001:00015760       ??$qMetaTypeId@VQAssociativeIterableImpl@QtMetaTypePrivate@@@@YAHXZ 10016760 f i KrakenClassifyWorker.obj
 0001:00015770       ??$qRegisterMetaType@V?$QMap@VQString@@I@@@@YAHPBDPAV?$QMap@VQString@@I@@W4DefinedType@?$MetaTypeDefinedHelper@V?$QMap@VQString@@I@@$00@QtPrivate@@@Z 10016770 f i KrakenClassifyWorker.obj
 0001:000157e0       ??$qRegisterMetaType@VQAssociativeIterableImpl@QtMetaTypePrivate@@@@YAHPBDPAVQAssociativeIterableImpl@QtMetaTypePrivate@@W4DefinedType@?$MetaTypeDefinedHelper@VQAssociativeIterableImpl@QtMetaTypePrivate@@$00@QtPrivate@@@Z 100167e0 f i KrakenClassifyWorker.obj
 0001:000158a0       ??$qRegisterNormalizedMetaType@V?$QMap@VQString@@I@@@@YAHABVQByteArray@@PAV?$QMap@VQString@@I@@W4DefinedType@?$MetaTypeDefinedHelper@V?$QMap@VQString@@I@@$00@QtPrivate@@@Z 100168a0 f i KrakenClassifyWorker.obj
 0001:00015910       ??$qRegisterNormalizedMetaType@VQAssociativeIterableImpl@QtMetaTypePrivate@@@@YAHABVQByteArray@@PAVQAssociativeIterableImpl@QtMetaTypePrivate@@W4DefinedType@?$MetaTypeDefinedHelper@VQAssociativeIterableImpl@QtMetaTypePrivate@@$00@QtPrivate@@@Z 10016910 f i KrakenClassifyWorker.obj
 0001:00015970       ??$qVariantFromValue@V?$QMap@VQString@@I@@@@YA?AVQVariant@@ABV?$QMap@VQString@@I@@@Z 10016970 f i KrakenClassifyWorker.obj
 0001:000159a0       ??$qobject_cast@PAVKrakenClassifyTask@U2@@@@YAPAVKrakenClassifyTask@U2@@PAVQObject@@@Z 100169a0 f i KrakenClassifyWorker.obj
 0001:000159c0       ??$sizeImpl@V?$QMap@VQString@@I@@@QAssociativeIterableImpl@QtMetaTypePrivate@@SAHPBX@Z 100169c0 f i KrakenClassifyWorker.obj
 0001:00015a00       ??0?$ConverterFunctor@V?$QMap@VQString@@I@@VQAssociativeIterableImpl@QtMetaTypePrivate@@U?$QAssociativeIterableConvertFunctor@V?$QMap@VQString@@I@@@3@@QtPrivate@@QAE@U?$QAssociativeIterableConvertFunctor@V?$QMap@VQString@@I@@@QtMetaTypePrivate@@@Z 10016a00 f i KrakenClassifyWorker.obj
 0001:00015a10       ??0?$QHash@VQString@@UQHashDummyValue@@@@QAE@XZ 10016a10 f i KrakenClassifyWorker.obj
 0001:00015a20       ??0?$QMap@VQString@@I@@QAE@ABV0@@Z 10016a20 f i KrakenClassifyWorker.obj
 0001:00015a90       ??0?$QSet@VQString@@@@QAE@XZ 10016a90 f i KrakenClassifyWorker.obj
 0001:00015aa0       ??0AbstractConverterFunction@QtPrivate@@QAE@P6A_NPBU01@PBXPAX@Z@Z 10016aa0 f i KrakenClassifyWorker.obj
 0001:00015ab0       ??0KrakenClassifyWorker@LocalWorkflow@U2@@QAE@PAVActor@Workflow@2@@Z 10016ab0 f   KrakenClassifyWorker.obj
 0001:00015af0       ??0QAssociativeIterableImpl@QtMetaTypePrivate@@QAE@XZ 10016af0 f i KrakenClassifyWorker.obj
 0001:00015b60       ??0VariantData@QtMetaTypePrivate@@QAE@HPBXI@Z 10016b60 f i KrakenClassifyWorker.obj
 0001:00015b80       ??0const_iterator@?$QMap@VQString@@I@@QAE@PBU?$QMapNode@VQString@@I@@@Z 10016b80 f i KrakenClassifyWorker.obj
 0001:00015b90       ??0const_iterator@?$QMap@VQString@@I@@QAE@XZ 10016b90 f i KrakenClassifyWorker.obj
 0001:00015ba0       ??1?$ConverterFunctor@V?$QMap@VQString@@I@@VQAssociativeIterableImpl@QtMetaTypePrivate@@U?$QAssociativeIterableConvertFunctor@V?$QMap@VQString@@I@@@3@@QtPrivate@@QAE@XZ 10016ba0 f i KrakenClassifyWorker.obj
 0001:00015bc0       ??1?$QHash@VQString@@UQHashDummyValue@@@@QAE@XZ 10016bc0 f i KrakenClassifyWorker.obj
 0001:00015bf0       ??1?$QHashNode@VQString@@UQHashDummyValue@@@@QAE@XZ 10016bf0 f i KrakenClassifyWorker.obj
 0001:00015c00       ??1?$QSet@VQString@@@@QAE@XZ 10016c00 f i KrakenClassifyWorker.obj
 0001:00015c30       ??1KrakenClassifyWorker@LocalWorkflow@U2@@UAE@XZ 10016c30 f i KrakenClassifyWorker.obj
 0001:00015c40       ??8const_iterator@?$QMap@VQString@@I@@QBE_NABV01@@Z 10016c40 f i KrakenClassifyWorker.obj
 0001:00015c60       ??9const_iterator@?$QMap@VQString@@I@@QBE_NABV01@@Z 10016c60 f i KrakenClassifyWorker.obj
 0001:00015c80       ??Econst_iterator@?$QMap@VQString@@I@@QAEAAV01@XZ 10016c80 f i KrakenClassifyWorker.obj
 0001:00015ca0       ??Fconst_iterator@?$QMap@VQString@@I@@QAEAAV01@XZ 10016ca0 f i KrakenClassifyWorker.obj
 0001:00015cc0       ??R?$QAssociativeIterableConvertFunctor@V?$QMap@VQString@@I@@@QtMetaTypePrivate@@QBE?AVQAssociativeIterableImpl@1@ABV?$QMap@VQString@@I@@@Z 10016cc0 f i KrakenClassifyWorker.obj
 0001:00015cd5       ??_EKrakenClassifyWorker@LocalWorkflow@U2@@W7AEPAXI@Z 10016cd5 f i KrakenClassifyWorker.obj
 0001:00015cdd       ??_EKrakenClassifyWorker@LocalWorkflow@U2@@WBA@AEPAXI@Z 10016cdd f i KrakenClassifyWorker.obj
 0001:00015cf0       ??_G?$QHashNode@VQString@@UQHashDummyValue@@@@QAEPAXI@Z 10016cf0 f i KrakenClassifyWorker.obj
 0001:00015d20       ??_G?$QMap@VQString@@I@@QAEPAXI@Z 10016d20 f i KrakenClassifyWorker.obj
 0001:00015d50       ??_EFailTask@U2@@UAEPAXI@Z 10016d50 f i KrakenClassifyWorker.obj
 0001:00015d50       ??_GFailTask@U2@@UAEPAXI@Z 10016d50 f i KrakenClassifyWorker.obj
 0001:00015d80       ??_EKrakenClassifyWorker@LocalWorkflow@U2@@UAEPAXI@Z 10016d80 f i KrakenClassifyWorker.obj
 0001:00015d80       ??_GKrakenClassifyWorker@LocalWorkflow@U2@@UAEPAXI@Z 10016d80 f i KrakenClassifyWorker.obj
 0001:00015db0       ?Construct@?$QMetaTypeFunctionHelper@V?$QMap@VQString@@I@@$00@QtMetaTypePrivate@@SAPAXPAXPBX@Z 10016db0 f i KrakenClassifyWorker.obj
 0001:00015e40       ?Construct@?$QMetaTypeFunctionHelper@VQAssociativeIterableImpl@QtMetaTypePrivate@@$00@QtMetaTypePrivate@@SAPAXPAXPBX@Z 10016e40 f i KrakenClassifyWorker.obj
 0001:00015e90       ?Create@?$QMetaTypeFunctionHelper@V?$QMap@VQString@@I@@$00@QtMetaTypePrivate@@SAPAXPBX@Z 10016e90 f i KrakenClassifyWorker.obj
 0001:00015f30       ?Create@?$QMetaTypeFunctionHelper@VQAssociativeIterableImpl@QtMetaTypePrivate@@$00@QtMetaTypePrivate@@SAPAXPBX@Z 10016f30 f i KrakenClassifyWorker.obj
 0001:00015f90       ?Delete@?$QMetaTypeFunctionHelper@V?$QMap@VQString@@I@@$00@QtMetaTypePrivate@@SAXPAX@Z 10016f90 f i KrakenClassifyWorker.obj
 0001:00015fb0       ?Delete@?$QMetaTypeFunctionHelper@VQAssociativeIterableImpl@QtMetaTypePrivate@@$00@QtMetaTypePrivate@@SAXPAX@Z 10016fb0 f i KrakenClassifyWorker.obj
 0001:00015fc0       ?Destruct@?$QMetaTypeFunctionHelper@V?$QMap@VQString@@I@@$00@QtMetaTypePrivate@@SAXPAX@Z 10016fc0 f i KrakenClassifyWorker.obj
 0001:00015fd0       ?Destruct@?$QMetaTypeFunctionHelper@VQAssociativeIterableImpl@QtMetaTypePrivate@@$00@QtMetaTypePrivate@@SAXPAX@Z 10016fd0 f i KrakenClassifyWorker.obj
 0001:00015fe0       ?assign@?$IteratorOwnerCommon@Vconst_iterator@?$QMap@VQString@@I@@@QtMetaTypePrivate@@SAXPAPAXPBQAX@Z 10016fe0 f i KrakenClassifyWorker.obj
 0001:00016010       ?assign@?$IteratorOwnerCommon@Vconst_iterator@?$QMap@VQString@@I@@@QtMetaTypePrivate@@SAXPAPAXVconst_iterator@?$QMap@VQString@@I@@@Z 10017010 f i KrakenClassifyWorker.obj
 0001:00016040       ?begin@?$QMap@VQString@@I@@QBE?AVconst_iterator@1@XZ 10017040 f i KrakenClassifyWorker.obj
 0001:00016060       ?begin@?$QMapData@VQString@@I@@QAEPAU?$QMapNode@VQString@@I@@XZ 10017060 f i KrakenClassifyWorker.obj
 0001:00016070       ?cleanup@KrakenClassifyWorker@LocalWorkflow@U2@@UAEXXZ 10017070 f   KrakenClassifyWorker.obj
 0001:00016080       ?concrete@?$QHash@VQString@@UQHashDummyValue@@@@CAPAU?$QHashNode@VQString@@UQHashDummyValue@@@@PAUNode@QHashData@@@Z 10017080 f i KrakenClassifyWorker.obj
 0001:00016090       ?constFind@?$QMap@VQString@@I@@QBE?AVconst_iterator@1@ABVQString@@@Z 10017090 f i KrakenClassifyWorker.obj
 0001:000160e0       ?convert@?$ConverterFunctor@V?$QMap@VQString@@I@@VQAssociativeIterableImpl@QtMetaTypePrivate@@U?$QAssociativeIterableConvertFunctor@V?$QMap@VQString@@I@@@3@@QtPrivate@@SA_NPBUAbstractConverterFunction@2@PBXPAX@Z 100170e0 f i KrakenClassifyWorker.obj
 0001:00016130       ?dataFinished@KrakenClassifyWorker@LocalWorkflow@U2@@ABE_NXZ 10017130 f   KrakenClassifyWorker.obj
 0001:00016140       ?deleteNode2@?$QHash@VQString@@UQHashDummyValue@@@@CAXPAUNode@QHashData@@@Z 10017140 f i KrakenClassifyWorker.obj
 0001:00016150       ?destroy@?$IteratorOwnerCommon@Vconst_iterator@?$QMap@VQString@@I@@@QtMetaTypePrivate@@SAXPAPAX@Z 10017150 f i KrakenClassifyWorker.obj
 0001:00016170       ?end@?$QMap@VQString@@I@@QBE?AVconst_iterator@1@XZ 10017170 f i KrakenClassifyWorker.obj
 0001:00016190       ?equal@?$IteratorOwnerCommon@Vconst_iterator@?$QMap@VQString@@I@@@QtMetaTypePrivate@@SA_NPBQAX0@Z 10017190 f i KrakenClassifyWorker.obj
 0001:000161b0       ?find@?$QMap@VQString@@I@@QBE?AVconst_iterator@1@ABVQString@@@Z 100171b0 f i KrakenClassifyWorker.obj
 0001:00016200       ?freeData@?$QHash@VQString@@UQHashDummyValue@@@@AAEXPAUQHashData@@@Z 10017200 f i KrakenClassifyWorker.obj
 0001:00016220       ?getKey@?$AssociativeContainerAccessor@V?$QMap@VQString@@I@@$00@QtMetaTypePrivate@@SAABVQString@@ABVconst_iterator@?$QMap@VQString@@I@@@Z 10017220 f i KrakenClassifyWorker.obj
 0001:00016230       ?getSettings@KrakenClassifyWorker@LocalWorkflow@U2@@AAE?AUKrakenClassifyTaskSettings@3@AAVU2OpStatus@3@@Z 10017230 f   KrakenClassifyWorker.obj
 0001:00016910       ?getValue@?$AssociativeContainerAccessor@V?$QMap@VQString@@I@@$00@QtMetaTypePrivate@@SAABIABVconst_iterator@?$QMap@VQString@@I@@@Z 10017910 f i KrakenClassifyWorker.obj
 0001:00016920       ?init@KrakenClassifyWorker@LocalWorkflow@U2@@UAEXXZ 10017920 f   KrakenClassifyWorker.obj
 0001:00016ce0       ?isReadyToRun@KrakenClassifyWorker@LocalWorkflow@U2@@ABE_NXZ 10017ce0 f   KrakenClassifyWorker.obj
 0001:00016d00       ?key@const_iterator@?$QMap@VQString@@I@@QBEABVQString@@XZ 10017d00 f i KrakenClassifyWorker.obj
 0001:00016d10       ?nextNode@?$QMapNode@VQString@@I@@QBEPBU1@XZ 10017d10 f i KrakenClassifyWorker.obj
 0001:00016d20       ?previousNode@?$QMapNode@VQString@@I@@QBEPBU1@XZ 10017d20 f i KrakenClassifyWorker.obj
 0001:00016d30       ?qt_metatype_id@?$QMetaTypeId2@I@@SAHXZ 10017d30 f i KrakenClassifyWorker.obj
 0001:00016d40       ?qt_metatype_id@?$QMetaTypeId2@V?$QMap@VQString@@I@@@@SAHXZ 10017d40 f i KrakenClassifyWorker.obj
 0001:00016d50       ?qt_metatype_id@?$QMetaTypeId2@VQAssociativeIterableImpl@QtMetaTypePrivate@@@@SAHXZ 10017d50 f i KrakenClassifyWorker.obj
 0001:00016d60       ?qt_metatype_id@?$QMetaTypeId@V?$QMap@VQString@@I@@@@SAHXZ 10017d60 f i KrakenClassifyWorker.obj
 0001:00016e10       ?qt_metatype_id@?$QMetaTypeId@VQAssociativeIterableImpl@QtMetaTypePrivate@@@@SAHXZ 10017e10 f i KrakenClassifyWorker.obj
 0001:00016eb0       ?qt_metatype_id@?$QMetaTypeIdHelper@V?$QMap@VQString@@I@@$00@QtPrivate@@SAHXZ 10017eb0 f i KrakenClassifyWorker.obj
 0001:00016ec0       ?qt_metatype_id@?$QMetaTypeIdHelper@VQAssociativeIterableImpl@QtMetaTypePrivate@@$00@QtPrivate@@SAHXZ 10017ec0 f i KrakenClassifyWorker.obj
 0001:00016ed0       ?registerConverter@?$AssociativeContainerConverterHelper@VQAssociativeIterableImpl@QtMetaTypePrivate@@$0A@@QtPrivate@@SA_NH@Z 10017ed0 f i KrakenClassifyWorker.obj
 0001:00016ee0       ?registerConverter@?$AssociativeValueTypeIsMetaType@V?$QMap@VQString@@I@@$00@QtPrivate@@SA_NH@Z 10017ee0 f i KrakenClassifyWorker.obj
 0001:00016f50       ?registerConverter@?$IsPair@V?$QMap@VQString@@I@@@QtPrivate@@SA_NH@Z 10017f50 f i KrakenClassifyWorker.obj
 0001:00016f60       ?registerConverter@?$IsPair@VQAssociativeIterableImpl@QtMetaTypePrivate@@@QtPrivate@@SA_NH@Z 10017f60 f i KrakenClassifyWorker.obj
 0001:00016f70       ?registerConverter@?$MetaTypeSmartPointerHelper@V?$QMap@VQString@@I@@X@QtPrivate@@SA_NH@Z 10017f70 f i KrakenClassifyWorker.obj
 0001:00016f80       ?registerConverter@?$MetaTypeSmartPointerHelper@VQAssociativeIterableImpl@QtMetaTypePrivate@@X@QtPrivate@@SA_NH@Z 10017f80 f i KrakenClassifyWorker.obj
 0001:00016f90       ?registerConverter@?$SequentialContainerConverterHelper@V?$QMap@VQString@@I@@$0A@@QtPrivate@@SA_NH@Z 10017f90 f i KrakenClassifyWorker.obj
 0001:00016fa0       ?registerConverter@?$SequentialContainerConverterHelper@VQAssociativeIterableImpl@QtMetaTypePrivate@@$0A@@QtPrivate@@SA_NH@Z 10017fa0 f i KrakenClassifyWorker.obj
 0001:00016fb0       ?size@?$QMap@VQString@@I@@QBEHXZ 10017fb0 f i KrakenClassifyWorker.obj
 0001:00016fc0       ?sl_taskFinished@KrakenClassifyWorker@LocalWorkflow@U2@@AAEXPAVTask@3@@Z 10017fc0 f   KrakenClassifyWorker.obj
 0001:00017260       ?tick@KrakenClassifyWorker@LocalWorkflow@U2@@UAEPAVTask@3@XZ 10018260 f   KrakenClassifyWorker.obj
 0001:00017490       ?tr@KrakenClassifyWorker@LocalWorkflow@U2@@SA?AVQString@@PBD0H@Z 10018490 f i KrakenClassifyWorker.obj
 0001:000174c0       ?value@?$MetaObjectForType@V?$QMap@VQString@@I@@$0A@@QtPrivate@@SAPBUQMetaObject@@XZ 100184c0 f i KrakenClassifyWorker.obj
 0001:000174d0       ?value@?$MetaObjectForType@VQAssociativeIterableImpl@QtMetaTypePrivate@@$0A@@QtPrivate@@SAPBUQMetaObject@@XZ 100184d0 f i KrakenClassifyWorker.obj
 0001:000174e0       ?value@const_iterator@?$QMap@VQString@@I@@QBEABIXZ 100184e0 f i KrakenClassifyWorker.obj
 0001:000174f0       ??0?$QFlags@W4Flag@Attribute@U2@@@@QAE@VQFlag@@@Z 100184f0 f i KrakenClassifyWorkerFactory.obj
 0001:00017500       ??0?$QFlags@W4Flag@Attribute@U2@@@@QAE@W4Flag@Attribute@U2@@@Z 10018500 f i KrakenClassifyWorkerFactory.obj
 0001:00017510       ??0?$QList@VQVariant@@@@QAE@XZ 10018510 f i KrakenClassifyWorkerFactory.obj
 0001:00017520       ??0KrakenClassifyValidator@Workflow@U2@@QAE@XZ 10018520 f i KrakenClassifyWorkerFactory.obj
 0001:00017530       ??0KrakenClassifyWorkerFactory@LocalWorkflow@U2@@QAE@XZ 10018530 f   KrakenClassifyWorkerFactory.obj
 0001:00017550       ??1?$QList@VQVariant@@@@QAE@XZ 10018550 f i KrakenClassifyWorkerFactory.obj
 0001:00017580       ??1KrakenClassifyValidator@Workflow@U2@@UAE@XZ 10018580 f i KrakenClassifyWorkerFactory.obj
 0001:00017590       ??1KrakenClassifyWorkerFactory@LocalWorkflow@U2@@UAE@XZ 10018590 f i KrakenClassifyWorkerFactory.obj
 0001:000175a0       ??6?$QList@VQVariant@@@@QAEAAV0@ABVQVariant@@@Z 100185a0 f i KrakenClassifyWorkerFactory.obj
 0001:000175c0       ??U?$QFlags@W4Flag@Attribute@U2@@@@QBE?AV0@W4Flag@Attribute@U2@@@Z 100185c0 f i KrakenClassifyWorkerFactory.obj
 0001:000175e0       ??U@YA?AV?$QFlags@W4Flag@Attribute@U2@@@@W4Flag@Attribute@U2@@0@Z 100185e0 f i KrakenClassifyWorkerFactory.obj
 0001:000175f0       ??_EKrakenClassifyWorkerFactory@LocalWorkflow@U2@@W7AEPAXI@Z 100185f0 f i KrakenClassifyWorkerFactory.obj
 0001:00017600       ??_EDatabaseDelegate@LocalWorkflow@U2@@UAEPAXI@Z 10018600 f i KrakenClassifyWorkerFactory.obj
 0001:00017600       ??_GDatabaseDelegate@LocalWorkflow@U2@@UAEPAXI@Z 10018600 f i KrakenClassifyWorkerFactory.obj
 0001:00017630       ??_EKrakenClassifyValidator@Workflow@U2@@UAEPAXI@Z 10018630 f i KrakenClassifyWorkerFactory.obj
 0001:00017630       ??_GKrakenClassifyValidator@Workflow@U2@@UAEPAXI@Z 10018630 f i KrakenClassifyWorkerFactory.obj
 0001:00017660       ??_GKrakenClassifyWorkerFactory@LocalWorkflow@U2@@UAEPAXI@Z 10018660 f i KrakenClassifyWorkerFactory.obj
 0001:00017660       ??_EKrakenClassifyWorkerFactory@LocalWorkflow@U2@@UAEPAXI@Z 10018660 f i KrakenClassifyWorkerFactory.obj
 0001:00017690       ??_GPairedReadsPortValidator@Workflow@U2@@UAEPAXI@Z 10018690 f i KrakenClassifyWorkerFactory.obj
 0001:00017690       ??_EPairedReadsPortValidator@Workflow@U2@@UAEPAXI@Z 10018690 f i KrakenClassifyWorkerFactory.obj
 0001:000176c0       ??_GSlotRelationDescriptor@U2@@UAEPAXI@Z 100186c0 f i KrakenClassifyWorkerFactory.obj
 0001:000176c0       ??_ESlotRelationDescriptor@U2@@UAEPAXI@Z 100186c0 f i KrakenClassifyWorkerFactory.obj
 0001:000176f0       ?append@?$QList@VQVariant@@@@QAEXABVQVariant@@@Z 100186f0 f i KrakenClassifyWorkerFactory.obj
 0001:000177d0       ?cleanup@KrakenClassifyWorkerFactory@LocalWorkflow@U2@@SAXXZ 100187d0 f   KrakenClassifyWorkerFactory.obj
 0001:00017820       ?createWorker@KrakenClassifyWorkerFactory@LocalWorkflow@U2@@UAEPAVWorker@Workflow@3@PAVActor@53@@Z 10018820 f   KrakenClassifyWorkerFactory.obj
 0001:00017890       ?dealloc@?$QList@VQVariant@@@@AAEXPAUData@QListData@@@Z 10018890 f i KrakenClassifyWorkerFactory.obj
 0001:000178f0       ?detach_helper_grow@?$QList@VQVariant@@@@AAEPAUNode@1@HH@Z 100188f0 f i KrakenClassifyWorkerFactory.obj
 0001:00017a50       ?init@KrakenClassifyWorkerFactory@LocalWorkflow@U2@@SAXXZ 10018a50 f   KrakenClassifyWorkerFactory.obj
 0001:00019150       ?node_construct@?$QList@VQVariant@@@@AAEXPAUNode@1@ABVQVariant@@@Z 1001a150 f i KrakenClassifyWorkerFactory.obj
 0001:000191d0       ?node_copy@?$QList@VQVariant@@@@AAEXPAUNode@1@00@Z 1001a1d0 f i KrakenClassifyWorkerFactory.obj
 0001:000192a0       ?node_destruct@?$QList@VQVariant@@@@AAEXPAUNode@1@0@Z 1001a2a0 f i KrakenClassifyWorkerFactory.obj
 0001:000192e0       ?node_destruct@?$QList@VQVariant@@@@AAEXPAUNode@1@@Z 1001a2e0 f i KrakenClassifyWorkerFactory.obj
 0001:00019310       ??0KrakenSupport@U2@@QAE@ABVQString@@0@Z 1001a310 f   KrakenSupport.obj
 0001:00019520       ??1KrakenSupport@U2@@UAE@XZ 1001a520 f i KrakenSupport.obj
 0001:00019530       ??_EKrakenSupport@U2@@UAEPAXI@Z 1001a530 f i KrakenSupport.obj
 0001:00019530       ??_GKrakenSupport@U2@@UAEPAXI@Z 1001a530 f i KrakenSupport.obj
 0001:00019560       ?getAdditionalPaths@KrakenSupport@U2@@UBE?AVQStringList@@XZ 1001a560 f   KrakenSupport.obj
 0001:00019720       ?initBuild@KrakenSupport@U2@@AAEXXZ 1001a720 f   KrakenSupport.obj
 0001:000197a0       ?initClassify@KrakenSupport@U2@@AAEXXZ 1001a7a0 f   KrakenSupport.obj
 0001:00019820       ??0KrakenSupportPlugin@U2@@QAE@XZ 1001a820 f   KrakenSupportPlugin.obj
 0001:00019940       ??1KrakenSupportPlugin@U2@@UAE@XZ 1001a940 f   KrakenSupportPlugin.obj
 0001:000199c0       ??_GKrakenSupportPlugin@U2@@UAEPAXI@Z 1001a9c0 f i KrakenSupportPlugin.obj
 0001:000199c0       ??_EKrakenSupportPlugin@U2@@UAEPAXI@Z 1001a9c0 f i KrakenSupportPlugin.obj
 0001:00019a50       ?tr@KrakenSupportPlugin@U2@@SA?AVQString@@PBD0H@Z 1001aa50 f i KrakenSupportPlugin.obj
 0001:00019a80       _ugene_plugin_init         1001aa80 f   KrakenSupportPlugin.obj
 0001:00019aa0       ??0KrakenTranslateLogParser@U2@@QAE@XZ 1001aaa0 f   KrakenTranslateLogParser.obj
 0001:00019ac0       ??1KrakenTranslateLogParser@U2@@UAE@XZ 1001aac0 f i KrakenTranslateLogParser.obj
 0001:00019ad0       ??_GKrakenTranslateLogParser@U2@@UAEPAXI@Z 1001aad0 f i KrakenTranslateLogParser.obj
 0001:00019ad0       ??_EKrakenTranslateLogParser@U2@@UAEPAXI@Z 1001aad0 f i KrakenTranslateLogParser.obj
 0001:00019b00       ?initWellKnownErrors@KrakenTranslateLogParser@U2@@CA?AVQStringList@@XZ 1001ab00 f   KrakenTranslateLogParser.obj
 0001:00019c50       ?isError@KrakenTranslateLogParser@U2@@EBE_NABVQString@@@Z 1001ac50 f   KrakenTranslateLogParser.obj
 0001:00019dc0       ??C?$QScopedPointer@VQObjectData@@U?$QScopedPointerDeleter@VQObjectData@@@@@@QBEPAVQObjectData@@XZ 1001adc0 f i moc_KrakenBuildPrompter.obj
 0001:00019dd0       ?metaObject@KrakenBuildPrompter@LocalWorkflow@U2@@UBEPBUQMetaObject@@XZ 1001add0 f   moc_KrakenBuildPrompter.obj
 0001:00019df0       ?qt_metacall@KrakenBuildPrompter@LocalWorkflow@U2@@UAEHW4Call@QMetaObject@@HPAPAX@Z 1001adf0 f   moc_KrakenBuildPrompter.obj
 0001:00019e00       ?qt_metacast@KrakenBuildPrompter@LocalWorkflow@U2@@UAEPAXPBD@Z 1001ae00 f   moc_KrakenBuildPrompter.obj
 0001:00019e60       ?qt_static_metacall@KrakenBuildPrompter@LocalWorkflow@U2@@CAXPAVQObject@@W4Call@QMetaObject@@HPAPAX@Z 1001ae60 f   moc_KrakenBuildPrompter.obj
 0001:00019e70       ?metaObject@KrakenBuildTask@U2@@UBEPBUQMetaObject@@XZ 1001ae70 f   moc_KrakenBuildTask.obj
 0001:00019e90       ?qt_metacall@KrakenBuildTask@U2@@UAEHW4Call@QMetaObject@@HPAPAX@Z 1001ae90 f   moc_KrakenBuildTask.obj
 0001:00019ea0       ?qt_metacast@KrakenBuildTask@U2@@UAEPAXPBD@Z 1001aea0 f   moc_KrakenBuildTask.obj
 0001:00019f00       ?qt_static_metacall@KrakenBuildTask@U2@@CAXPAVQObject@@W4Call@QMetaObject@@HPAPAX@Z 1001af00 f   moc_KrakenBuildTask.obj
 0001:00019f10       ??$qMetaTypeId@PAVTask@U2@@@@YAHXZ 1001af10 f i moc_KrakenBuildWorker.obj
 0001:00019f20       ??$qRegisterMetaType@PAVTask@U2@@@@YAHXZ 1001af20 f i moc_KrakenBuildWorker.obj
 0001:00019f30       ??$qRegisterNormalizedMetaType@PAVTask@U2@@@@YAHABVQByteArray@@PAPAVTask@U2@@W4DefinedType@?$MetaTypeDefinedHelper@PAVTask@U2@@$00@QtPrivate@@@Z 1001af30 f i moc_KrakenBuildWorker.obj
 0001:00019f90       ?Construct@?$QMetaTypeFunctionHelper@PAVTask@U2@@$00@QtMetaTypePrivate@@SAPAXPAXPBX@Z 1001af90 f i moc_KrakenBuildWorker.obj
 0001:00019fc0       ?Create@?$QMetaTypeFunctionHelper@PAVTask@U2@@$00@QtMetaTypePrivate@@SAPAXPBX@Z 1001afc0 f i moc_KrakenBuildWorker.obj
 0001:0001a000       ?Delete@?$QMetaTypeFunctionHelper@PAVTask@U2@@$00@QtMetaTypePrivate@@SAXPAX@Z 1001b000 f i moc_KrakenBuildWorker.obj
 0001:0001a010       ?Destruct@?$QMetaTypeFunctionHelper@PAVTask@U2@@$00@QtMetaTypePrivate@@SAXPAX@Z 1001b010 f i moc_KrakenBuildWorker.obj
 0001:0001a020       ?metaObject@KrakenBuildWorker@LocalWorkflow@U2@@UBEPBUQMetaObject@@XZ 1001b020 f   moc_KrakenBuildWorker.obj
 0001:0001a040       ?qt_metacall@KrakenBuildWorker@LocalWorkflow@U2@@UAEHW4Call@QMetaObject@@HPAPAX@Z 1001b040 f   moc_KrakenBuildWorker.obj
 0001:0001a0a0       ?qt_metacast@KrakenBuildWorker@LocalWorkflow@U2@@UAEPAXPBD@Z 1001b0a0 f   moc_KrakenBuildWorker.obj
 0001:0001a100       ?qt_metatype_id@?$QMetaTypeId2@PAVTask@U2@@@@SAHXZ 1001b100 f i moc_KrakenBuildWorker.obj
 0001:0001a110       ?qt_metatype_id@?$QMetaTypeIdHelper@PAVTask@U2@@$00@QtPrivate@@SAHXZ 1001b110 f i moc_KrakenBuildWorker.obj
 0001:0001a120       ?qt_metatype_id@?$QMetaTypeIdQObject@PAVTask@U2@@$00@@SAHXZ 1001b120 f i moc_KrakenBuildWorker.obj
 0001:0001a200       ?qt_static_metacall@KrakenBuildWorker@LocalWorkflow@U2@@CAXPAVQObject@@W4Call@QMetaObject@@HPAPAX@Z 1001b200 f   moc_KrakenBuildWorker.obj
 0001:0001a260       ?registerConverter@?$AssociativeContainerConverterHelper@PAVTask@U2@@$0A@@QtPrivate@@SA_NH@Z 1001b260 f i moc_KrakenBuildWorker.obj
 0001:0001a270       ?registerConverter@?$IsPair@PAVTask@U2@@@QtPrivate@@SA_NH@Z 1001b270 f i moc_KrakenBuildWorker.obj
 0001:0001a280       ?registerConverter@?$MetaTypeSmartPointerHelper@PAVTask@U2@@X@QtPrivate@@SA_NH@Z 1001b280 f i moc_KrakenBuildWorker.obj
 0001:0001a290       ?registerConverter@?$SequentialContainerConverterHelper@PAVTask@U2@@$0A@@QtPrivate@@SA_NH@Z 1001b290 f i moc_KrakenBuildWorker.obj
 0001:0001a2a0       ?value@?$MetaObjectForType@PAVTask@U2@@$00@QtPrivate@@SAPBUQMetaObject@@XZ 1001b2a0 f i moc_KrakenBuildWorker.obj
 0001:0001a2b0       ?metaObject@KrakenClassifyPrompter@LocalWorkflow@U2@@UBEPBUQMetaObject@@XZ 1001b2b0 f   moc_KrakenClassifyPrompter.obj
 0001:0001a2d0       ?qt_metacall@KrakenClassifyPrompter@LocalWorkflow@U2@@UAEHW4Call@QMetaObject@@HPAPAX@Z 1001b2d0 f   moc_KrakenClassifyPrompter.obj
 0001:0001a2e0       ?qt_metacast@KrakenClassifyPrompter@LocalWorkflow@U2@@UAEPAXPBD@Z 1001b2e0 f   moc_KrakenClassifyPrompter.obj
 0001:0001a340       ?qt_static_metacall@KrakenClassifyPrompter@LocalWorkflow@U2@@CAXPAVQObject@@W4Call@QMetaObject@@HPAPAX@Z 1001b340 f   moc_KrakenClassifyPrompter.obj
 0001:0001a350       ?metaObject@KrakenClassifyTask@U2@@UBEPBUQMetaObject@@XZ 1001b350 f   moc_KrakenClassifyTask.obj
 0001:0001a370       ?qt_metacall@KrakenClassifyTask@U2@@UAEHW4Call@QMetaObject@@HPAPAX@Z 1001b370 f   moc_KrakenClassifyTask.obj
 0001:0001a380       ?qt_metacast@KrakenClassifyTask@U2@@UAEPAXPBD@Z 1001b380 f   moc_KrakenClassifyTask.obj
 0001:0001a3e0       ?qt_static_metacall@KrakenClassifyTask@U2@@CAXPAVQObject@@W4Call@QMetaObject@@HPAPAX@Z 1001b3e0 f   moc_KrakenClassifyTask.obj
 0001:0001a3f0       ?metaObject@KrakenClassifyWorker@LocalWorkflow@U2@@UBEPBUQMetaObject@@XZ 1001b3f0 f   moc_KrakenClassifyWorker.obj
 0001:0001a410       ?qt_metacall@KrakenClassifyWorker@LocalWorkflow@U2@@UAEHW4Call@QMetaObject@@HPAPAX@Z 1001b410 f   moc_KrakenClassifyWorker.obj
 0001:0001a470       ?qt_metacast@KrakenClassifyWorker@LocalWorkflow@U2@@UAEPAXPBD@Z 1001b470 f   moc_KrakenClassifyWorker.obj
 0001:0001a4d0       ?qt_static_metacall@KrakenClassifyWorker@LocalWorkflow@U2@@CAXPAVQObject@@W4Call@QMetaObject@@HPAPAX@Z 1001b4d0 f   moc_KrakenClassifyWorker.obj
 0001:0001a530       ?metaObject@KrakenSupport@U2@@UBEPBUQMetaObject@@XZ 1001b530 f   moc_KrakenSupport.obj
 0001:0001a550       ?qt_metacall@KrakenSupport@U2@@UAEHW4Call@QMetaObject@@HPAPAX@Z 1001b550 f   moc_KrakenSupport.obj
 0001:0001a560       ?qt_metacast@KrakenSupport@U2@@UAEPAXPBD@Z 1001b560 f   moc_KrakenSupport.obj
 0001:0001a5c0       ?qt_static_metacall@KrakenSupport@U2@@CAXPAVQObject@@W4Call@QMetaObject@@HPAPAX@Z 1001b5c0 f   moc_KrakenSupport.obj
 0001:0001a5d0       ?metaObject@KrakenSupportPlugin@U2@@UBEPBUQMetaObject@@XZ 1001b5d0 f   moc_KrakenSupportPlugin.obj
 0001:0001a5f0       ?qt_metacall@KrakenSupportPlugin@U2@@UAEHW4Call@QMetaObject@@HPAPAX@Z 1001b5f0 f   moc_KrakenSupportPlugin.obj
 0001:0001a600       ?qt_metacast@KrakenSupportPlugin@U2@@UAEPAXPBD@Z 1001b600 f   moc_KrakenSupportPlugin.obj
 0001:0001a660       ?qt_static_metacall@KrakenSupportPlugin@U2@@CAXPAVQObject@@W4Call@QMetaObject@@HPAPAX@Z 1001b660 f   moc_KrakenSupportPlugin.obj
 0001:0001a662       ?getAppSettings@AppContext@U2@@SAPAVAppSettings@2@XZ 1001b662 f   U2Core:U2Core.dll
 0001:0001a668       ??0Logger@U2@@QAE@ABVQString@@@Z 1001b668 f   U2Core:U2Core.dll
 0001:0001a66e       ??1Logger@U2@@UAE@XZ       1001b66e f   U2Core:U2Core.dll
 0001:0001a674       ?getTotalPhysicalMemory@AppResourcePool@U2@@SAHXZ 1001b674 f   U2Core:U2Core.dll
 0001:0001a67a       ?getDataPathRegistry@AppContext@U2@@SAPAVU2DataPathRegistry@2@XZ 1001b67a f   U2Core:U2Core.dll
 0001:0001a680       ?error@Logger@U2@@QAEXABVQString@@@Z 1001b680 f   U2Core:U2Core.dll
 0001:0001a686       ?getTaskName@Task@U2@@QBE?AVQString@@XZ 1001b686 f   U2Core:U2Core.dll
 0001:0001a68c       ?addSubTask@Task@U2@@QAEXPAV12@@Z 1001b68c f   U2Core:U2Core.dll
 0001:0001a692       ?setError@Task@U2@@QAEXABVQString@@@Z 1001b692 f   U2Core:U2Core.dll
 0001:0001a698       ?setTaskName@Task@U2@@IAEXABVQString@@@Z 1001b698 f   U2Core:U2Core.dll
 0001:0001a69e       ??0CopyFileTask@U2@@QAE@ABVQString@@0@Z 1001b69e f   U2Core:U2Core.dll
 0001:0001a6a4       ??1CopyFileTask@U2@@UAE@XZ 1001b6a4 f   U2Core:U2Core.dll
 0001:0001a6aa       ??1GCounter@U2@@UAE@XZ     1001b6aa f   U2Core:U2Core.dll
 0001:0001a6b0       ??0GReportableCounter@U2@@QAE@ABVQString@@0N@Z 1001b6b0 f   U2Core:U2Core.dll
 0001:0001a6b6       ??1SimpleEventCounter@U2@@UAE@XZ 1001b6b6 f   U2Core:U2Core.dll
 0001:0001a6bc       ?getPath@U2DataPath@U2@@QBEABVQString@@XZ 1001b6bc f   U2Core:U2Core.dll
 0001:0001a6c2       ?isValid@U2DataPath@U2@@QBE_NXZ 1001b6c2 f   U2Core:U2Core.dll
 0001:0001a6c8       ?getDataPathByName@U2DataPathRegistry@U2@@QAEPAVU2DataPath@2@ABVQString@@@Z 1001b6c8 f   U2Core:U2Core.dll
 0001:0001a6ce       ?prepareDirLocation@GUrlUtils@U2@@SA?AVQString@@ABV3@AAVU2OpStatus@2@@Z 1001b6ce f   U2Core:U2Core.dll
 0001:0001a6d4       ??0SequentialMultiTask@U2@@QAE@ABVQString@@ABV?$QList@PAVTask@U2@@@@V?$QFlags@W4TaskFlag@U2@@@@@Z 1001b6d4 f   U2Core:U2Core.dll
 0001:0001a6da       ??1SequentialMultiTask@U2@@UAE@XZ 1001b6da f   U2Core:U2Core.dll
 0001:0001a6e0       ??0ExternalToolRunTask@U2@@QAE@ABVQString@@ABVQStringList@@PAVExternalToolLogParser@1@010_N@Z 1001b6e0 f   U2Core:U2Core.dll
 0001:0001a6e6       ??1ExternalToolRunTask@U2@@UAE@XZ 1001b6e6 f   U2Core:U2Core.dll
 0001:0001a6ec       ??0ExternalToolSupportTask@U2@@QAE@ABVQString@@V?$QFlags@W4TaskFlag@U2@@@@@Z 1001b6ec f   U2Core:U2Core.dll
 0001:0001a6f2       ??1ExternalToolSupportTask@U2@@UAE@XZ 1001b6f2 f   U2Core:U2Core.dll
 0001:0001a6f8       ??0ExternalToolLogParser@U2@@QAE@_N@Z 1001b6f8 f   U2Core:U2Core.dll
 0001:0001a6fe       ??1ExternalToolLogParser@U2@@UAE@XZ 1001b6fe f   U2Core:U2Core.dll
 0001:0001a704       ?cleanup@Task@U2@@UAEXXZ   1001b704 f   U2Core:U2Core.dll
 0001:0001a70a       ?generateReport@Task@U2@@UBE?AVQString@@XZ 1001b70a f   U2Core:U2Core.dll
 0001:0001a710       ?getNumParallelSubtasks@Task@U2@@UBEHXZ 1001b710 f   U2Core:U2Core.dll
 0001:0001a716       ?getParentTask@Task@U2@@UBEPAV12@XZ 1001b716 f   U2Core:U2Core.dll
 0001:0001a71c       ?getProgress@ExternalToolLogParser@U2@@UAEHXZ 1001b71c f   U2Core:U2Core.dll
 0001:0001a722       ?getSubtaskWithErrors@Task@U2@@UBEPAV12@XZ 1001b722 f   U2Core:U2Core.dll
 0001:0001a728       ?getTaskId@Task@U2@@UBE_JXZ 1001b728 f   U2Core:U2Core.dll
 0001:0001a72e       ?getTopLevelParentTask@Task@U2@@UAEPAV12@XZ 1001b72e f   U2Core:U2Core.dll
 0001:0001a734       ?getWarnings@Task@U2@@UBE?AVQStringList@@XZ 1001b734 f   U2Core:U2Core.dll
 0001:0001a73a       ?hasSubtasksWithErrors@Task@U2@@UBE_NXZ 1001b73a f   U2Core:U2Core.dll
 0001:0001a740       ?hasWarning@Task@U2@@UBE_NXZ 1001b740 f   U2Core:U2Core.dll
 0001:0001a746       ?isError@ExternalToolLogParser@U2@@MBE_NABVQString@@@Z 1001b746 f   U2Core:U2Core.dll
 0001:0001a74c       ?isNotificationReport@Task@U2@@UBE_NXZ 1001b74c f   U2Core:U2Core.dll
 0001:0001a752       ?isReportingEnabled@Task@U2@@UBE_NXZ 1001b752 f   U2Core:U2Core.dll
 0001:0001a758       ?isReportingSupported@Task@U2@@UBE_NXZ 1001b758 f   U2Core:U2Core.dll
 0001:0001a75e       ?isTopLevelTask@Task@U2@@UBE_NXZ 1001b75e f   U2Core:U2Core.dll
 0001:0001a764       ?metaObject@CopyFileTask@U2@@UBEPBUQMetaObject@@XZ 1001b764 f   U2Core:U2Core.dll
 0001:0001a76a       ?metaObject@ExternalToolLogParser@U2@@UBEPBUQMetaObject@@XZ 1001b76a f   U2Core:U2Core.dll
 0001:0001a770       ?metaObject@ExternalToolRunTask@U2@@UBEPBUQMetaObject@@XZ 1001b770 f   U2Core:U2Core.dll
 0001:0001a776       ?metaObject@SequentialMultiTask@U2@@UBEPBUQMetaObject@@XZ 1001b776 f   U2Core:U2Core.dll
 0001:0001a77c       ?onSubTaskFinished@SequentialMultiTask@U2@@UAE?AV?$QList@PAVTask@U2@@@@PAVTask@2@@Z 1001b77c f   U2Core:U2Core.dll
 0001:0001a782       ?onSubTaskFinished@Task@U2@@MAE?AV?$QList@PAVTask@U2@@@@PAV12@@Z 1001b782 f   U2Core:U2Core.dll
 0001:0001a788       ?parseErrOutput@ExternalToolLogParser@U2@@UAEXABVQString@@@Z 1001b788 f   U2Core:U2Core.dll
 0001:0001a78e       ?parseOutput@ExternalToolLogParser@U2@@UAEXABVQString@@@Z 1001b78e f   U2Core:U2Core.dll
 0001:0001a794       ?prepare@SequentialMultiTask@U2@@UAEXXZ 1001b794 f   U2Core:U2Core.dll
 0001:0001a79a       ?prepare@Task@U2@@UAEXXZ   1001b79a f   U2Core:U2Core.dll
 0001:0001a7a0       ?processErrLine@ExternalToolLogParser@U2@@MAEXABVQString@@@Z 1001b7a0 f   U2Core:U2Core.dll
 0001:0001a7a6       ?processLine@ExternalToolLogParser@U2@@MAEXABVQString@@@Z 1001b7a6 f   U2Core:U2Core.dll
 0001:0001a7ac       ?propagateSubtaskError@Task@U2@@UAE_NXZ 1001b7ac f   U2Core:U2Core.dll
 0001:0001a7b2       ?qt_metacall@CopyFileTask@U2@@UAEHW4Call@QMetaObject@@HPAPAX@Z 1001b7b2 f   U2Core:U2Core.dll
 0001:0001a7b8       ?qt_metacall@ExternalToolLogParser@U2@@UAEHW4Call@QMetaObject@@HPAPAX@Z 1001b7b8 f   U2Core:U2Core.dll
 0001:0001a7be       ?qt_metacall@ExternalToolRunTask@U2@@UAEHW4Call@QMetaObject@@HPAPAX@Z 1001b7be f   U2Core:U2Core.dll
 0001:0001a7c4       ?qt_metacall@SequentialMultiTask@U2@@UAEHW4Call@QMetaObject@@HPAPAX@Z 1001b7c4 f   U2Core:U2Core.dll
 0001:0001a7ca       ?qt_metacast@CopyFileTask@U2@@UAEPAXPBD@Z 1001b7ca f   U2Core:U2Core.dll
 0001:0001a7d0       ?qt_metacast@ExternalToolLogParser@U2@@UAEPAXPBD@Z 1001b7d0 f   U2Core:U2Core.dll
 0001:0001a7d6       ?qt_metacast@ExternalToolRunTask@U2@@UAEPAXPBD@Z 1001b7d6 f   U2Core:U2Core.dll
 0001:0001a7dc       ?qt_metacast@SequentialMultiTask@U2@@UAEPAXPBD@Z 1001b7dc f   U2Core:U2Core.dll
 0001:0001a7e2       ?report@Task@U2@@UAE?AW4ReportResult@12@XZ 1001b7e2 f   U2Core:U2Core.dll
 0001:0001a7e8       ?run@CopyFileTask@U2@@EAEXXZ 1001b7e8 f   U2Core:U2Core.dll
 0001:0001a7ee       ?run@ExternalToolRunTask@U2@@UAEXXZ 1001b7ee f   U2Core:U2Core.dll
 0001:0001a7f4       ?run@Task@U2@@UAEXXZ       1001b7f4 f   U2Core:U2Core.dll
 0001:0001a7fa       ?setCollectChildrensWarningsFlag@Task@U2@@UAEX_N@Z 1001b7fa f   U2Core:U2Core.dll
 0001:0001a800       ?setLastError@ExternalToolLogParser@U2@@MAEXABVQString@@@Z 1001b800 f   U2Core:U2Core.dll
 0001:0001a806       ?setListenerForHelper@ExternalToolSupportTask@U2@@MAEXPAVExternalToolRunTaskHelper@2@H@Z 1001b806 f   U2Core:U2Core.dll
 0001:0001a80c       ?setListenerForTask@ExternalToolSupportTask@U2@@MAEXPAVExternalToolRunTask@2@H@Z 1001b80c f   U2Core:U2Core.dll
 0001:0001a812       ?setNoAutoDelete@Task@U2@@UAEX_N@Z 1001b812 f   U2Core:U2Core.dll
 0001:0001a818       ?setNotificationReport@Task@U2@@UAEX_N@Z 1001b818 f   U2Core:U2Core.dll
 0001:0001a81e       ?setReportingEnabled@Task@U2@@UAEX_N@Z 1001b81e f   U2Core:U2Core.dll
 0001:0001a824       ?setReportingSupported@Task@U2@@UAEX_N@Z 1001b824 f   U2Core:U2Core.dll
 0001:0001a82a       ?getPathByName@U2DataPath@U2@@QBE?AVQString@@ABV3@@Z 1001b82a f   U2Core:U2Core.dll
 0001:0001a830       ??0TaskSignalMapper@U2@@QAE@PAVTask@1@@Z 1001b830 f   U2Core:U2Core.dll
 0001:0001a836       ??0TaskStateInfo@U2@@QAE@XZ 1001b836 f   U2Core:U2Core.dll
 0001:0001a83c       ?getError@TaskStateInfo@U2@@UBE?AVQString@@XZ 1001b83c f   U2Core:U2Core.dll
 0001:0001a842       ?setError@TaskStateInfo@U2@@UAEXABVQString@@@Z 1001b842 f   U2Core:U2Core.dll
 0001:0001a848       ??1TaskStateInfo@U2@@UAE@XZ 1001b848 f   U2Core:U2Core.dll
 0001:0001a84e       ?hasError@Task@U2@@QBE_NXZ 1001b84e f   U2Core:U2Core.dll
 0001:0001a854       ?addListeners@ExternalToolSupportTask@U2@@QAEXABV?$QList@PAVExternalToolListener@U2@@@@@Z 1001b854 f   U2Core:U2Core.dll
 0001:0001a85a       ?runScript@ScriptTask@U2@@SA?AVQScriptValue@@PAVQScriptEngine@@ABV?$QMap@VQString@@VQScriptValue@@@@ABVQString@@AAVTaskStateInfo@2@@Z 1001b85a f   U2Core:U2Core.dll
 0001:0001a860       ?metaObject@TaskSignalMapper@U2@@UBEPBUQMetaObject@@XZ 1001b860 f   U2Core:U2Core.dll
 0001:0001a866       ?qt_metacall@TaskSignalMapper@U2@@UAEHW4Call@QMetaObject@@HPAPAX@Z 1001b866 f   U2Core:U2Core.dll
 0001:0001a86c       ?qt_metacast@TaskSignalMapper@U2@@UAEPAXPBD@Z 1001b86c f   U2Core:U2Core.dll
 0001:0001a872       ?trace@Logger@U2@@QAEXABVQString@@@Z 1001b872 f   U2Core:U2Core.dll
 0001:0001a878       ?info@Logger@U2@@QAEXABVQString@@@Z 1001b878 f   U2Core:U2Core.dll
 0001:0001a87e       ??0FailTask@U2@@QAE@ABVQString@@@Z 1001b87e f   U2Core:U2Core.dll
 0001:0001a884       ??1FailTask@U2@@UAE@XZ     1001b884 f   U2Core:U2Core.dll
 0001:0001a88a       ?createWorkingDir@FileAndDirectoryUtils@U2@@SA?AVQString@@ABV3@H00@Z 1001b88a f   U2Core:U2Core.dll
 0001:0001a890       ?rollFileName@GUrlUtils@U2@@SA?AVQString@@ABV3@0ABV?$QSet@VQString@@@@@Z 1001b890 f   U2Core:U2Core.dll
 0001:0001a896       ?createDirectory@GUrlUtils@U2@@SA?AVQString@@ABV3@0AAVU2OpStatus@2@@Z 1001b896 f   U2Core:U2Core.dll
 0001:0001a89c       ?getError@U2OpStatusImpl@U2@@UBE?AVQString@@XZ 1001b89c f   U2Core:U2Core.dll
 0001:0001a8a2       ??0U2OpStatus2Log@U2@@QAE@W4LogLevel@1@@Z 1001b8a2 f   U2Core:U2Core.dll
 0001:0001a8a8       ??1U2OpStatus2Log@U2@@UAE@XZ 1001b8a8 f   U2Core:U2Core.dll
 0001:0001a8ae       ?metaObject@FailTask@U2@@UBEPBUQMetaObject@@XZ 1001b8ae f   U2Core:U2Core.dll
 0001:0001a8b4       ?qt_metacall@FailTask@U2@@UAEHW4Call@QMetaObject@@HPAPAX@Z 1001b8b4 f   U2Core:U2Core.dll
 0001:0001a8ba       ?qt_metacast@FailTask@U2@@UAEPAXPBD@Z 1001b8ba f   U2Core:U2Core.dll
 0001:0001a8c0       ??0ExternalTool@U2@@QAE@VQString@@00@Z 1001b8c0 f   U2Core:U2Core.dll
 0001:0001a8c6       ??1ExternalTool@U2@@UAE@XZ 1001b8c6 f   U2Core:U2Core.dll
 0001:0001a8cc       ?extractAdditionalParameters@ExternalTool@U2@@UAEXABVQString@@@Z 1001b8cc f   U2Core:U2Core.dll
 0001:0001a8d2       ?getRunParameters@ExternalTool@U2@@UBE?AVQStringList@@XZ 1001b8d2 f   U2Core:U2Core.dll
 0001:0001a8d8       ?getToolRunnerAdditionalOptions@ExternalTool@U2@@UBE?AVQStringList@@XZ 1001b8d8 f   U2Core:U2Core.dll
 0001:0001a8de       ?performAdditionalChecks@ExternalTool@U2@@UAEXABVQString@@@Z 1001b8de f   U2Core:U2Core.dll
 0001:0001a8e4       ?getExternalToolRegistry@AppContext@U2@@SAPAVExternalToolRegistry@2@XZ 1001b8e4 f   U2Core:U2Core.dll
 0001:0001a8ea       ?registerEntry@ExternalToolRegistry@U2@@QAE_NPAVExternalTool@2@@Z 1001b8ea f   U2Core:U2Core.dll
 0001:0001a8f0       ?unregisterEntry@ExternalToolRegistry@U2@@QAEXABVQString@@@Z 1001b8f0 f   U2Core:U2Core.dll
 0001:0001a8f6       ?setToolkitDescription@ExternalToolRegistry@U2@@QAEXABVQString@@0@Z 1001b8f6 f   U2Core:U2Core.dll
 0001:0001a8fc       ??0Plugin@U2@@QAE@ABVQString@@0_NW4PluginState@1@@Z 1001b8fc f   U2Core:U2Core.dll
 0001:0001a902       ??1Plugin@U2@@UAE@XZ       1001b902 f   U2Core:U2Core.dll
 0001:0001a908       ?qt_metacast@Task@U2@@UAEPAXPBD@Z 1001b908 f   U2Core:U2Core.dll
 0001:0001a90e       ?qt_metacall@Task@U2@@UAEHW4Call@QMetaObject@@HPAPAX@Z 1001b90e f   U2Core:U2Core.dll
 0001:0001a914       ?qt_metacast@ExternalTool@U2@@UAEPAXPBD@Z 1001b914 f   U2Core:U2Core.dll
 0001:0001a91a       ?qt_metacall@ExternalTool@U2@@UAEHW4Call@QMetaObject@@HPAPAX@Z 1001b91a f   U2Core:U2Core.dll
 0001:0001a920       ?qt_metacast@Plugin@U2@@UAEPAXPBD@Z 1001b920 f   U2Core:U2Core.dll
 0001:0001a926       ?qt_metacall@Plugin@U2@@UAEHW4Call@QMetaObject@@HPAPAX@Z 1001b926 f   U2Core:U2Core.dll
 0001:0001a92c       ?prepareDocumentsFileFilter@DialogUtils@U2@@SA?AVQString@@ABV3@_NABVQStringList@@@Z 1001b92c f   U2Gui:U2Gui.dll
 0001:0001a932       ??0ValuesRelation@U2@@QAE@ABVQString@@ABV?$QMap@VQString@@VQVariant@@@@@Z 1001b932 f   U2Lang:U2Lang.dll
 0001:0001a938       ??1ValuesRelation@U2@@UAE@XZ 1001b938 f   U2Lang:U2Lang.dll
 0001:0001a93e       ??0ValuesRelation@U2@@QAE@ABV01@@Z 1001b93e f   U2Lang:U2Lang.dll
 0001:0001a944       ?getType@ValuesRelation@U2@@UBE?AW4RelationType@2@XZ 1001b944 f   U2Lang:U2Lang.dll
 0001:0001a94a       ?updateDelegateTags@ValuesRelation@U2@@UBEXABVQVariant@@PAVDelegateTags@2@@Z 1001b94a f   U2Lang:U2Lang.dll
 0001:0001a950       ?valueChangingRelation@AttributeRelation@U2@@UBE_NXZ 1001b950 f   U2Lang:U2Lang.dll
 0001:0001a956       ?getInputPorts@Actor@Workflow@U2@@QBE?AV?$QList@PAVPort@Workflow@U2@@@@XZ 1001b956 f   U2Lang:U2Lang.dll
 0001:0001a95c       ?getOutputPorts@Actor@Workflow@U2@@QBE?AV?$QList@PAVPort@Workflow@U2@@@@XZ 1001b95c f   U2Lang:U2Lang.dll
 0001:0001a962       ??0PrompterBaseImpl@U2@@QAE@PAVActor@Workflow@1@@Z 1001b962 f   U2Lang:U2Lang.dll
 0001:0001a968       ?getURL@PrompterBaseImpl@U2@@QAE?AVQString@@ABV3@PA_N00@Z 1001b968 f   U2Lang:U2Lang.dll
 0001:0001a96e       ?getParameter@PrompterBaseImpl@U2@@QAE?AVQVariant@@ABVQString@@@Z 1001b96e f   U2Lang:U2Lang.dll
 0001:0001a974       ?getHyperlink@PrompterBaseImpl@U2@@SA?AVQString@@ABV3@0@Z 1001b974 f   U2Lang:U2Lang.dll
 0001:0001a97a       ??1PrompterBaseImpl@U2@@UAE@XZ 1001b97a f   U2Lang:U2Lang.dll
 0001:0001a980       ?metaObject@PrompterBaseImpl@U2@@UBEPBUQMetaObject@@XZ 1001b980 f   U2Lang:U2Lang.dll
 0001:0001a986       ?qt_metacall@PrompterBaseImpl@U2@@UAEHW4Call@QMetaObject@@HPAPAX@Z 1001b986 f   U2Lang:U2Lang.dll
 0001:0001a98c       ?qt_metacast@PrompterBaseImpl@U2@@UAEPAXPBD@Z 1001b98c f   U2Lang:U2Lang.dll
 0001:0001a992       ?sl_actorModified@PrompterBaseImpl@U2@@MAEXXZ 1001b992 f   U2Lang:U2Lang.dll
 0001:0001a998       ?update@PrompterBaseImpl@U2@@UAEXABV?$QMap@VQString@@VQVariant@@@@@Z 1001b998 f   U2Lang:U2Lang.dll
 0001:0001a99e       ??0WorkflowNotification@U2@@QAE@ABVQString@@00@Z 1001b99e f   U2Lang:U2Lang.dll
 0001:0001a9a4       ??1WorkflowNotification@U2@@QAE@XZ 1001b9a4 f   U2Lang:U2Lang.dll
 0001:0001a9aa       ??0WorkflowNotification@U2@@QAE@ABV01@@Z 1001b9aa f   U2Lang:U2Lang.dll
 0001:0001a9b0       ?getId@Actor@Workflow@U2@@QBE?AVQString@@XZ 1001b9b0 f   U2Lang:U2Lang.dll
 0001:0001a9b6       ??1Descriptor@U2@@UAE@XZ   1001b9b6 f   U2Lang:U2Lang.dll
 0001:0001a9bc       ?getId@Descriptor@U2@@QBE?AVQString@@XZ 1001b9bc f   U2Lang:U2Lang.dll
 0001:0001a9c2       ??0Descriptor@U2@@QAE@ABV01@@Z 1001b9c2 f   U2Lang:U2Lang.dll
 0001:0001a9c8       ?URL_SLOT@BaseSlots@Workflow@U2@@SA?BVDescriptor@3@XZ 1001b9c8 f   U2Lang:U2Lang.dll
 0001:0001a9ce       ??0Dataset@U2@@QAE@ABV01@@Z 1001b9ce f   U2Lang:U2Lang.dll
 0001:0001a9d4       ??1Dataset@U2@@QAE@XZ      1001b9d4 f   U2Lang:U2Lang.dll
 0001:0001a9da       ?getUrls@Dataset@U2@@QBE?AV?$QList@PAVURLContainer@U2@@@@XZ 1001b9da f   U2Lang:U2Lang.dll
 0001:0001a9e0       ?initEngine@WorkflowScriptLibrary@U2@@SAXPAVWorkflowScriptEngine@2@@Z 1001b9e0 f   U2Lang:U2Lang.dll
 0001:0001a9e6       ??0MessageMetadata@U2@@QAE@XZ 1001b9e6 f   U2Lang:U2Lang.dll
 0001:0001a9ec       ??0MessageMetadata@U2@@QAE@ABVQString@@@Z 1001b9ec f   U2Lang:U2Lang.dll
 0001:0001a9f2       ??0MessageMetadata@U2@@QAE@ABVQString@@0@Z 1001b9f2 f   U2Lang:U2Lang.dll
 0001:0001a9f8       ?getId@MessageMetadata@U2@@QBEHXZ 1001b9f8 f   U2Lang:U2Lang.dll
 0001:0001a9fe       ??1MessageMetadata@U2@@QAE@XZ 1001b9fe f   U2Lang:U2Lang.dll
 0001:0001aa04       ??4MessageMetadata@U2@@QAEAAV01@ABV01@@Z 1001ba04 f   U2Lang:U2Lang.dll
 0001:0001aa0a       ?put@MessageMetadataStorage@U2@@QAEXABVMessageMetadata@2@@Z 1001ba0a f   U2Lang:U2Lang.dll
 0001:0001aa10       ?getMonitor@WorkflowContext@Workflow@U2@@QAEPAVWorkflowMonitor@23@XZ 1001ba10 f   U2Lang:U2Lang.dll
 0001:0001aa16       ?absolutePath@WorkflowContext@Workflow@U2@@QBE?AVQString@@ABV4@@Z 1001ba16 f   U2Lang:U2Lang.dll
 0001:0001aa1c       ?getMetadataStorage@WorkflowContext@Workflow@U2@@QAEAAVMessageMetadataStorage@3@XZ 1001ba1c f   U2Lang:U2Lang.dll
 0001:0001aa22       ??0WorkflowScriptEngine@U2@@QAE@PAVWorkflowContext@Workflow@1@@Z 1001ba22 f   U2Lang:U2Lang.dll
 0001:0001aa28       ??1WorkflowScriptEngine@U2@@UAE@XZ 1001ba28 f   U2Lang:U2Lang.dll
 0001:0001aa2e       ?isEmpty@AttributeScript@U2@@QBE_NXZ 1001ba2e f   U2Lang:U2Lang.dll
 0001:0001aa34       ?getScriptText@AttributeScript@U2@@QBEABVQString@@XZ 1001ba34 f   U2Lang:U2Lang.dll
 0001:0001aa3a       ?getScriptVars@AttributeScript@U2@@QBEABV?$QMap@VDescriptor@U2@@VQVariant@@@@XZ 1001ba3a f   U2Lang:U2Lang.dll
 0001:0001aa40       ??0Message@Workflow@U2@@QAE@V?$QExplicitlySharedDataPointer@VDataType@U2@@@@ABVQVariant@@H@Z 1001ba40 f   U2Lang:U2Lang.dll
 0001:0001aa46       ??1Message@Workflow@U2@@QAE@XZ 1001ba46 f   U2Lang:U2Lang.dll
 0001:0001aa4c       ?addOutputFile@WorkflowMonitor@Workflow@U2@@QAEXABVQString@@0_N@Z 1001ba4c f   U2Lang:U2Lang.dll
 0001:0001aa52       ?isOutUrlAttribute@RFSUtils@U2@@SA_NPAVAttribute@2@PAVActor@Workflow@2@AA_N@Z 1001ba52 f   U2Lang:U2Lang.dll
 0001:0001aa58       ?getBusType@IntegralBus@Workflow@U2@@QBE?AV?$QExplicitlySharedDataPointer@VDataType@U2@@@@XZ 1001ba58 f   U2Lang:U2Lang.dll
 0001:0001aa5e       ??0BaseWorker@LocalWorkflow@U2@@QAE@PAVActor@Workflow@2@_N@Z 1001ba5e f   U2Lang:U2Lang.dll
 0001:0001aa64       ??1BaseWorker@LocalWorkflow@U2@@UAE@XZ 1001ba64 f   U2Lang:U2Lang.dll
 0001:0001aa6a       ?createLogListeners@BaseWorker@LocalWorkflow@U2@@QBE?AV?$QList@PAVExternalToolListener@U2@@@@H@Z 1001ba6a f   U2Lang:U2Lang.dll
 0001:0001aa70       ?addCommunication@BaseWorker@LocalWorkflow@U2@@UAE_NABVQString@@PAVCommunicationChannel@Workflow@3@@Z 1001ba70 f   U2Lang:U2Lang.dll
 0001:0001aa76       ?canTaskBeCanceled@BaseWorker@LocalWorkflow@U2@@MBE_NPAVTask@3@@Z 1001ba76 f   U2Lang:U2Lang.dll
 0001:0001aa7c       ?getActorId@BaseWorker@LocalWorkflow@U2@@UBE?AVQString@@XZ 1001ba7c f   U2Lang:U2Lang.dll
 0001:0001aa82       ?getCommunication@BaseWorker@LocalWorkflow@U2@@UAEPAVCommunicationChannel@Workflow@3@ABVQString@@@Z 1001ba82 f   U2Lang:U2Lang.dll
 0001:0001aa88       ?getMessageAndSetupScriptValues@BaseWorker@LocalWorkflow@U2@@UAE?AVMessage@Workflow@3@PAVCommunicationChannel@53@@Z 1001ba88 f   U2Lang:U2Lang.dll
 0001:0001aa8e       ?getOutputFiles@BaseWorker@LocalWorkflow@U2@@UAE?AVQStringList@@XZ 1001ba8e f   U2Lang:U2Lang.dll
 0001:0001aa94       ?isDone@BaseWorker@LocalWorkflow@U2@@UBE_NXZ 1001ba94 f   U2Lang:U2Lang.dll
 0001:0001aa9a       ?isReady@BaseWorker@LocalWorkflow@U2@@UBE_NXZ 1001ba9a f   U2Lang:U2Lang.dll
 0001:0001aaa0       ?setDisplayName@Descriptor@U2@@UAEXABVQString@@@Z 1001baa0 f   U2Lang:U2Lang.dll
 0001:0001aaa6       ?setDocumentation@Descriptor@U2@@UAEXABVQString@@@Z 1001baa6 f   U2Lang:U2Lang.dll
 0001:0001aaac       ?setDone@BaseWorker@LocalWorkflow@U2@@UAEXXZ 1001baac f   U2Lang:U2Lang.dll
 0001:0001aab2       ??0VisibilityRelation@U2@@QAE@ABVQString@@ABVQVariant@@_N@Z 1001bab2 f   U2Lang:U2Lang.dll
 0001:0001aab8       ??1VisibilityRelation@U2@@UAE@XZ 1001bab8 f   U2Lang:U2Lang.dll
 0001:0001aabe       ??0Descriptor@U2@@QAE@ABVQString@@00@Z 1001babe f   U2Lang:U2Lang.dll
 0001:0001aac4       ??0Descriptor@U2@@QAE@ABVQString@@@Z 1001bac4 f   U2Lang:U2Lang.dll
 0001:0001aaca       ??0MapDataType@U2@@QAE@ABVDescriptor@1@ABV?$QMap@VDescriptor@U2@@V?$QExplicitlySharedDataPointer@VDataType@U2@@@@@@@Z 1001baca f   U2Lang:U2Lang.dll
 0001:0001aad0       ??1MapDataType@U2@@UAE@XZ  1001bad0 f   U2Lang:U2Lang.dll
 0001:0001aad6       ??0Attribute@U2@@QAE@ABVDescriptor@1@V?$QExplicitlySharedDataPointer@VDataType@U2@@@@_NABVQVariant@@@Z 1001bad6 f   U2Lang:U2Lang.dll
 0001:0001aadc       ??1Attribute@U2@@UAE@XZ    1001badc f   U2Lang:U2Lang.dll
 0001:0001aae2       ?addRelation@Attribute@U2@@QAEXPBVAttributeRelation@2@@Z 1001bae2 f   U2Lang:U2Lang.dll
 0001:0001aae8       ??1PropertyDelegate@U2@@UAE@XZ 1001bae8 f   U2Lang:U2Lang.dll
 0001:0001aaee       ??0PortDescriptor@Workflow@U2@@QAE@ABVDescriptor@2@V?$QExplicitlySharedDataPointer@VDataType@U2@@@@_N2I@Z 1001baee f   U2Lang:U2Lang.dll
 0001:0001aaf4       ??1PortDescriptor@Workflow@U2@@UAE@XZ 1001baf4 f   U2Lang:U2Lang.dll
 0001:0001aafa       ??0ActorPrototype@Workflow@U2@@QAE@ABVDescriptor@2@ABV?$QList@PAVPortDescriptor@Workflow@U2@@@@ABV?$QList@PAVAttribute@U2@@@@@Z 1001bafa f   U2Lang:U2Lang.dll
 0001:0001ab00       ??1ActorPrototype@Workflow@U2@@UAE@XZ 1001bb00 f   U2Lang:U2Lang.dll
 0001:0001ab06       ?setEditor@ActorPrototype@Workflow@U2@@QAEXPAVConfigurationEditor@3@@Z 1001bb06 f   U2Lang:U2Lang.dll
 0001:0001ab0c       ?setValidator@ActorPrototype@Workflow@U2@@QAEXPAVConfigurationValidator@3@@Z 1001bb0c f   U2Lang:U2Lang.dll
 0001:0001ab12       ?setPrompter@ActorPrototype@Workflow@U2@@QAEXPAVPrompter@23@@Z 1001bb12 f   U2Lang:U2Lang.dll
 0001:0001ab18       ?addExternalTool@ActorPrototype@Workflow@U2@@QAEXABVQString@@0@Z 1001bb18 f   U2Lang:U2Lang.dll
 0001:0001ab1e       ?registerProto@ActorPrototypeRegistry@Workflow@U2@@QAE_NABVDescriptor@3@PAVActorPrototype@23@@Z 1001bb1e f   U2Lang:U2Lang.dll
 0001:0001ab24       ?unregisterProto@ActorPrototypeRegistry@Workflow@U2@@QAEPAVActorPrototype@23@ABVQString@@@Z 1001bb24 f   U2Lang:U2Lang.dll
 0001:0001ab2a       ?STRING_TYPE@BaseTypes@U2@@SA?AV?$QExplicitlySharedDataPointer@VDataType@U2@@@@XZ 1001bb2a f   U2Lang:U2Lang.dll
 0001:0001ab30       ?BOOL_TYPE@BaseTypes@U2@@SA?AV?$QExplicitlySharedDataPointer@VDataType@U2@@@@XZ 1001bb30 f   U2Lang:U2Lang.dll
 0001:0001ab36       ?NUM_TYPE@BaseTypes@U2@@SA?AV?$QExplicitlySharedDataPointer@VDataType@U2@@@@XZ 1001bb36 f   U2Lang:U2Lang.dll
 0001:0001ab3c       ?URL_DATASETS_TYPE@BaseTypes@U2@@SA?AV?$QExplicitlySharedDataPointer@VDataType@U2@@@@XZ 1001bb3c f   U2Lang:U2Lang.dll
 0001:0001ab42       ?getInstance@WorkflowEnv@Workflow@U2@@KAPAV123@XZ 1001bb42 f   U2Lang:U2Lang.dll
 0001:0001ab48       ??0DomainFactory@Workflow@U2@@QAE@ABVQString@@@Z 1001bb48 f   U2Lang:U2Lang.dll
 0001:0001ab4e       ??1DomainFactory@Workflow@U2@@UAE@XZ 1001bb4e f   U2Lang:U2Lang.dll
 0001:0001ab54       ?clone@Attribute@U2@@UAEPAV12@XZ 1001bb54 f   U2Lang:U2Lang.dll
 0001:0001ab5a       ?clone@VisibilityRelation@U2@@UBEPAV12@XZ 1001bb5a f   U2Lang:U2Lang.dll
 0001:0001ab60       ?createConnection@DomainFactory@Workflow@U2@@UAEPAVCommunicationChannel@23@PAVLink@23@@Z 1001bb60 f   U2Lang:U2Lang.dll
 0001:0001ab66       ?createInstance@ActorPrototype@Workflow@U2@@UAEPAVActor@23@ABVQString@@PAVAttributeScript@3@ABV?$QMap@VQString@@VQVariant@@@@@Z 1001bb66 f   U2Lang:U2Lang.dll
 0001:0001ab6c       ?createPort@IntegralBusActorPrototype@Workflow@U2@@UAEPAVPort@23@ABVPortDescriptor@23@PAVActor@23@@Z 1001bb6c f   U2Lang:U2Lang.dll
 0001:0001ab72       ?createScheduler@DomainFactory@Workflow@U2@@UAEPAVScheduler@23@PAVSchema@23@@Z 1001bb72 f   U2Lang:U2Lang.dll
 0001:0001ab78       ?destroy@DomainFactory@Workflow@U2@@UAEXPAVScheduler@23@PAVSchema@23@@Z 1001bb78 f   U2Lang:U2Lang.dll
 0001:0001ab7e       ?getAffectResult@VisibilityRelation@U2@@UBE?AVQVariant@@ABV3@0PAVDelegateTags@2@1@Z 1001bb7e f   U2Lang:U2Lang.dll
 0001:0001ab84       ?getAllDescriptors@MapDataType@U2@@UBE?AV?$QList@VDescriptor@U2@@@@XZ 1001bb84 f   U2Lang:U2Lang.dll
 0001:0001ab8a       ?getAllEntries@?$IdRegistry@VDomainFactory@Workflow@U2@@@U2@@UBE?AV?$QList@PAVDomainFactory@Workflow@U2@@@@XZ 1001bb8a f   U2Lang:U2Lang.dll
 0001:0001ab90       ?getAllIds@?$IdRegistry@VDomainFactory@Workflow@U2@@@U2@@UBE?AV?$QList@VQString@@@@XZ 1001bb90 f   U2Lang:U2Lang.dll
 0001:0001ab96       ?getAttributePureValue@Attribute@U2@@UBEABVQVariant@@XZ 1001bb96 f   U2Lang:U2Lang.dll
 0001:0001ab9c       ?getById@?$IdRegistry@VDomainFactory@Workflow@U2@@@U2@@UAEPAVDomainFactory@Workflow@2@ABVQString@@@Z 1001bb9c f   U2Lang:U2Lang.dll
 0001:0001aba2       ?getDatatypeByDescriptor@MapDataType@U2@@UBE?AV?$QExplicitlySharedDataPointer@VDataType@U2@@@@ABVDescriptor@2@@Z 1001bba2 f   U2Lang:U2Lang.dll
 0001:0001aba8       ?getDatatypesMap@MapDataType@U2@@UBE?AV?$QMap@VDescriptor@U2@@V?$QExplicitlySharedDataPointer@VDataType@U2@@@@@@XZ 1001bba8 f   U2Lang:U2Lang.dll
 0001:0001abae       ?getDefaultPureValue@Attribute@U2@@UBEABVQVariant@@XZ 1001bbae f   U2Lang:U2Lang.dll
 0001:0001abb4       ?getGroup@Attribute@U2@@UAE?AW4AttributeGroup@2@XZ 1001bbb4 f   U2Lang:U2Lang.dll
 0001:0001abba       ?getItems@PropertyDelegate@U2@@UBEXAAV?$QMap@VQString@@VQVariant@@@@@Z 1001bbba f   U2Lang:U2Lang.dll
 0001:0001abc0       ?getType@PortDescriptor@Workflow@U2@@UBE?AV?$QExplicitlySharedDataPointer@VDataType@U2@@@@XZ 1001bbc0 f   U2Lang:U2Lang.dll
 0001:0001abc6       ?getType@VisibilityRelation@U2@@UBE?AW4RelationType@2@XZ 1001bbc6 f   U2Lang:U2Lang.dll
 0001:0001abcc       ?getWidget@ConfigurationEditor@U2@@UAEPAVQWidget@@XZ 1001bbcc f   U2Lang:U2Lang.dll
 0001:0001abd2       ?isAcceptableDrop@ActorPrototype@Workflow@U2@@UBE_NPBVQMimeData@@PAV?$QMap@VQString@@VQVariant@@@@@Z 1001bbd2 f   U2Lang:U2Lang.dll
 0001:0001abd8       ?isDefaultValue@Attribute@U2@@UBE_NXZ 1001bbd8 f   U2Lang:U2Lang.dll
 0001:0001abde       ?isEmpty@Attribute@U2@@UBE_NXZ 1001bbde f   U2Lang:U2Lang.dll
 0001:0001abe4       ?isEmpty@ConfigurationEditor@U2@@UBE_NXZ 1001bbe4 f   U2Lang:U2Lang.dll
 0001:0001abea       ?kind@MapDataType@U2@@UBE?AW4Kind@DataType@2@XZ 1001bbea f   U2Lang:U2Lang.dll
 0001:0001abf0       ?metaObject@ActorPrototype@Workflow@U2@@UBEPBUQMetaObject@@XZ 1001bbf0 f   U2Lang:U2Lang.dll
 0001:0001abf6       ?qt_metacall@ActorPrototype@Workflow@U2@@UAEHW4Call@QMetaObject@@HPAPAX@Z 1001bbf6 f   U2Lang:U2Lang.dll
 0001:0001abfc       ?qt_metacast@ActorPrototype@Workflow@U2@@UAEPAXPBD@Z 1001bbfc f   U2Lang:U2Lang.dll
 0001:0001ac02       ?registerEntry@?$IdRegistry@VDomainFactory@Workflow@U2@@@U2@@UAE_NPAVDomainFactory@Workflow@2@@Z 1001bc02 f   U2Lang:U2Lang.dll
 0001:0001ac08       ?setAttributeValue@Attribute@U2@@UAEXABVQVariant@@@Z 1001bc08 f   U2Lang:U2Lang.dll
 0001:0001ac0e       ?setDisplayName@ActorPrototype@Workflow@U2@@UAEXABVQString@@@Z 1001bc0e f   U2Lang:U2Lang.dll
 0001:0001ac14       ?setDocumentation@ActorPrototype@Workflow@U2@@UAEXABVQString@@@Z 1001bc14 f   U2Lang:U2Lang.dll
 0001:0001ac1a       ?setVisibleSlot@PortDescriptor@Workflow@U2@@UAEXABVQString@@_N@Z 1001bc1a f   U2Lang:U2Lang.dll
 0001:0001ac20       ?type@PropertyDelegate@U2@@UBE?AW4Type@12@XZ 1001bc20 f   U2Lang:U2Lang.dll
 0001:0001ac26       ?unregisterEntry@?$IdRegistry@VDomainFactory@Workflow@U2@@@U2@@UAEPAVDomainFactory@Workflow@2@ABVQString@@@Z 1001bc26 f   U2Lang:U2Lang.dll
 0001:0001ac2c       ?update@PropertyDelegate@U2@@UAEXXZ 1001bc2c f   U2Lang:U2Lang.dll
 0001:0001ac32       ?updateActorIds@Attribute@U2@@UAEXABV?$QMap@VQString@@V1@@@@Z 1001bc32 f   U2Lang:U2Lang.dll
 0001:0001ac38       ?updateDelegateTags@AttributeRelation@U2@@UBEXABVQVariant@@PAVDelegateTags@2@@Z 1001bc38 f   U2Lang:U2Lang.dll
 0001:0001ac3e       ?validate@ActorValidator@Workflow@U2@@UBE_NPBVConfiguration@3@AAV?$QList@VWorkflowNotification@U2@@@@@Z 1001bc3e f   U2Lang:U2Lang.dll
 0001:0001ac44       ?validate@Attribute@U2@@UAE_NAAV?$QList@VWorkflowNotification@U2@@@@@Z 1001bc44 f   U2Lang:U2Lang.dll
 0001:0001ac4a       ?valueChangingRelation@VisibilityRelation@U2@@UBE_NXZ 1001bc4a f   U2Lang:U2Lang.dll
 0001:0001ac50       ?getProducersOrUnset@PrompterBaseImpl@U2@@QAE?AVQString@@ABV3@0@Z 1001bc50 f   U2Lang:U2Lang.dll
 0001:0001ac56       ?getFileUrl@MessageMetadata@U2@@QBEABVQString@@XZ 1001bc56 f   U2Lang:U2Lang.dll
 0001:0001ac5c       ?get@MessageMetadataStorage@U2@@QBE?AVMessageMetadata@2@H@Z 1001bc5c f   U2Lang:U2Lang.dll
 0001:0001ac62       ?workingDir@WorkflowContext@Workflow@U2@@QBE?AVQString@@XZ 1001bc62 f   U2Lang:U2Lang.dll
 0001:0001ac68       ?getData@Message@Workflow@U2@@QBE?AVQVariant@@XZ 1001bc68 f   U2Lang:U2Lang.dll
 0001:0001ac6e       ?getMetadataId@Message@Workflow@U2@@QBEHXZ 1001bc6e f   U2Lang:U2Lang.dll
 0001:0001ac74       ?addInfo@WorkflowMonitor@Workflow@U2@@QAEXABVQString@@00@Z 1001bc74 f   U2Lang:U2Lang.dll
 0001:0001ac7a       ??0SlotRelationDescriptor@U2@@QAE@ABVQString@@0ABV?$QList@VQVariant@@@@@Z 1001bc7a f   U2Lang:U2Lang.dll
 0001:0001ac80       ??1SlotRelationDescriptor@U2@@UAE@XZ 1001bc80 f   U2Lang:U2Lang.dll
 0001:0001ac86       ??0Attribute@U2@@QAE@ABVDescriptor@1@V?$QExplicitlySharedDataPointer@VDataType@U2@@@@V?$QFlags@W4Flag@Attribute@U2@@@@ABVQVariant@@@Z 1001bc86 f   U2Lang:U2Lang.dll
 0001:0001ac8c       ?addSlotRelation@Attribute@U2@@QAEXPAVSlotRelationDescriptor@2@@Z 1001bc8c f   U2Lang:U2Lang.dll
 0001:0001ac92       ??0DelegateTags@U2@@QAE@PAVQObject@@@Z 1001bc92 f   U2Lang:U2Lang.dll
 0001:0001ac98       ?set@DelegateTags@U2@@QAEXABVQString@@ABVQVariant@@@Z 1001bc98 f   U2Lang:U2Lang.dll
 0001:0001ac9e       ??1DelegateTags@U2@@UAE@XZ 1001bc9e f   U2Lang:U2Lang.dll
 0001:0001aca4       ?setPortValidator@ActorPrototype@Workflow@U2@@QAEXABVQString@@PAVConfigurationValidator@3@@Z 1001bca4 f   U2Lang:U2Lang.dll
 0001:0001acaa       ??0PairedReadsPortValidator@Workflow@U2@@QAE@ABVQString@@0@Z 1001bcaa f   U2Lang:U2Lang.dll
 0001:0001acb0       ??1PairedReadsPortValidator@Workflow@U2@@UAE@XZ 1001bcb0 f   U2Lang:U2Lang.dll
 0001:0001acb6       ?clone@SlotRelationDescriptor@U2@@UBEPAV12@XZ 1001bcb6 f   U2Lang:U2Lang.dll
 0001:0001acbc       ?isSlotEnabled@SlotRelationDescriptor@U2@@UBE_NABVQVariant@@@Z 1001bcbc f   U2Lang:U2Lang.dll
 0001:0001acc2       ?validate@PairedReadsPortValidator@Workflow@U2@@UBE_NPBVIntegralBusPort@23@AAV?$QList@VWorkflowNotification@U2@@@@@Z 1001bcc2 f   U2Lang:U2Lang.dll
 0001:0001acc8       ?validate@PortValidator@Workflow@U2@@UBE_NPBVConfiguration@3@AAV?$QList@VWorkflowNotification@U2@@@@@Z 1001bcc8 f   U2Lang:U2Lang.dll
 0001:0001acce       ?qt_metacast@BaseWorker@LocalWorkflow@U2@@UAEPAXPBD@Z 1001bcce f   U2Lang:U2Lang.dll
 0001:0001acd4       ?qt_metacall@BaseWorker@LocalWorkflow@U2@@UAEHW4Call@QMetaObject@@HPAPAX@Z 1001bcd4 f   U2Lang:U2Lang.dll
 0001:0001acda       ??0DelegateEditor@U2@@QAE@ABV?$QMap@VQString@@PAVPropertyDelegate@U2@@@@@Z 1001bcda f   U2Designer:U2Designer.dll
 0001:0001ace0       ??1DelegateEditor@U2@@UAE@XZ 1001bce0 f   U2Designer:U2Designer.dll
 0001:0001ace6       ??0URLDelegate@U2@@QAE@ABVQString@@0ABV?$QFlags@W4Option@URLDelegate@U2@@@@PAVQObject@@0@Z 1001bce6 f   U2Designer:U2Designer.dll
 0001:0001acec       ??0URLDelegate@U2@@QAE@ABVQString@@0_N11PAVQObject@@011@Z 1001bcec f   U2Designer:U2Designer.dll
 0001:0001acf2       ??1URLDelegate@U2@@UAE@XZ  1001bcf2 f   U2Designer:U2Designer.dll
 0001:0001acf8       ??0SpinBoxDelegate@U2@@QAE@ABV?$QMap@VQString@@VQVariant@@@@PAVQObject@@@Z 1001bcf8 f   U2Designer:U2Designer.dll
 0001:0001acfe       ??1SpinBoxDelegate@U2@@UAE@XZ 1001bcfe f   U2Designer:U2Designer.dll
 0001:0001ad04       ??0ComboBoxDelegate@U2@@QAE@ABV?$QMap@VQString@@VQVariant@@@@PAVQObject@@@Z 1001bd04 f   U2Designer:U2Designer.dll
 0001:0001ad0a       ??1ComboBoxDelegate@U2@@UAE@XZ 1001bd0a f   U2Designer:U2Designer.dll
 0001:0001ad10       ??0ComboBoxWithBoolsDelegate@U2@@QAE@PAVQObject@@@Z 1001bd10 f   U2Designer:U2Designer.dll
 0001:0001ad16       ??1ComboBoxWithBoolsDelegate@U2@@UAE@XZ 1001bd16 f   U2Designer:U2Designer.dll
 0001:0001ad1c       ?addDelegate@DelegateEditor@U2@@UAEXPAVPropertyDelegate@2@ABVQString@@@Z 1001bd1c f   U2Designer:U2Designer.dll
 0001:0001ad22       ?clone@ComboBoxDelegate@U2@@UAEPAVPropertyDelegate@2@XZ 1001bd22 f   U2Designer:U2Designer.dll
 0001:0001ad28       ?clone@ComboBoxWithBoolsDelegate@U2@@UAEPAVPropertyDelegate@2@XZ 1001bd28 f   U2Designer:U2Designer.dll
 0001:0001ad2e       ?clone@DelegateEditor@U2@@UAEPAVConfigurationEditor@2@XZ 1001bd2e f   U2Designer:U2Designer.dll
 0001:0001ad34       ?clone@SpinBoxDelegate@U2@@UAEPAVPropertyDelegate@2@XZ 1001bd34 f   U2Designer:U2Designer.dll
 0001:0001ad3a       ?clone@URLDelegate@U2@@UAEPAVPropertyDelegate@2@XZ 1001bd3a f   U2Designer:U2Designer.dll
 0001:0001ad40       ?commit@DelegateEditor@U2@@UAEXXZ 1001bd40 f   U2Designer:U2Designer.dll
 0001:0001ad46       ?createEditor@ComboBoxDelegate@U2@@UBEPAVQWidget@@PAV3@ABVQStyleOptionViewItem@@ABVQModelIndex@@@Z 1001bd46 f   U2Designer:U2Designer.dll
 0001:0001ad4c       ?createEditor@SpinBoxDelegate@U2@@UBEPAVQWidget@@PAV3@ABVQStyleOptionViewItem@@ABVQModelIndex@@@Z 1001bd4c f   U2Designer:U2Designer.dll
 0001:0001ad52       ?createEditor@URLDelegate@U2@@UBEPAVQWidget@@PAV3@ABVQStyleOptionViewItem@@ABVQModelIndex@@@Z 1001bd52 f   U2Designer:U2Designer.dll
 0001:0001ad58       ?createWizardWidget@ComboBoxDelegate@U2@@UBEPAVPropertyWidget@2@AAVU2OpStatus@2@PAVQWidget@@@Z 1001bd58 f   U2Designer:U2Designer.dll
 0001:0001ad5e       ?createWizardWidget@SpinBoxDelegate@U2@@UBEPAVPropertyWidget@2@AAVU2OpStatus@2@PAVQWidget@@@Z 1001bd5e f   U2Designer:U2Designer.dll
 0001:0001ad64       ?createWizardWidget@URLDelegate@U2@@UBEPAVPropertyWidget@2@AAVU2OpStatus@2@PAVQWidget@@@Z 1001bd64 f   U2Designer:U2Designer.dll
 0001:0001ad6a       ?getDelegate@DelegateEditor@U2@@UAEPAVPropertyDelegate@2@ABVQString@@@Z 1001bd6a f   U2Designer:U2Designer.dll
 0001:0001ad70       ?getDisplayValue@ComboBoxDelegate@U2@@UBE?AVQVariant@@ABV3@@Z 1001bd70 f   U2Designer:U2Designer.dll
 0001:0001ad76       ?getDisplayValue@SpinBoxDelegate@U2@@UBE?AVQVariant@@ABV3@@Z 1001bd76 f   U2Designer:U2Designer.dll
 0001:0001ad7c       ?getDisplayValue@URLDelegate@U2@@UBE?AVQVariant@@ABV3@@Z 1001bd7c f   U2Designer:U2Designer.dll
 0001:0001ad82       ?getItems@ComboBoxDelegate@U2@@UBEXAAV?$QMap@VQString@@VQVariant@@@@@Z 1001bd82 f   U2Designer:U2Designer.dll
 0001:0001ad88       ?getItems@SpinBoxDelegate@U2@@UBEXAAV?$QMap@VQString@@VQVariant@@@@@Z 1001bd88 f   U2Designer:U2Designer.dll
 0001:0001ad8e       ?metaObject@ComboBoxDelegate@U2@@UBEPBUQMetaObject@@XZ 1001bd8e f   U2Designer:U2Designer.dll
 0001:0001ad94       ?metaObject@ComboBoxWithBoolsDelegate@U2@@UBEPBUQMetaObject@@XZ 1001bd94 f   U2Designer:U2Designer.dll
 0001:0001ad9a       ?metaObject@DelegateEditor@U2@@UBEPBUQMetaObject@@XZ 1001bd9a f   U2Designer:U2Designer.dll
 0001:0001ada0       ?metaObject@SpinBoxDelegate@U2@@UBEPBUQMetaObject@@XZ 1001bda0 f   U2Designer:U2Designer.dll
 0001:0001ada6       ?metaObject@URLDelegate@U2@@UBEPBUQMetaObject@@XZ 1001bda6 f   U2Designer:U2Designer.dll
 0001:0001adac       ?qt_metacall@ComboBoxDelegate@U2@@UAEHW4Call@QMetaObject@@HPAPAX@Z 1001bdac f   U2Designer:U2Designer.dll
 0001:0001adb2       ?qt_metacall@ComboBoxWithBoolsDelegate@U2@@UAEHW4Call@QMetaObject@@HPAPAX@Z 1001bdb2 f   U2Designer:U2Designer.dll
 0001:0001adb8       ?qt_metacall@DelegateEditor@U2@@UAEHW4Call@QMetaObject@@HPAPAX@Z 1001bdb8 f   U2Designer:U2Designer.dll
 0001:0001adbe       ?qt_metacall@SpinBoxDelegate@U2@@UAEHW4Call@QMetaObject@@HPAPAX@Z 1001bdbe f   U2Designer:U2Designer.dll
 0001:0001adc4       ?qt_metacall@URLDelegate@U2@@UAEHW4Call@QMetaObject@@HPAPAX@Z 1001bdc4 f   U2Designer:U2Designer.dll
 0001:0001adca       ?qt_metacast@ComboBoxDelegate@U2@@UAEPAXPBD@Z 1001bdca f   U2Designer:U2Designer.dll
 0001:0001add0       ?qt_metacast@ComboBoxWithBoolsDelegate@U2@@UAEPAXPBD@Z 1001bdd0 f   U2Designer:U2Designer.dll
 0001:0001add6       ?qt_metacast@DelegateEditor@U2@@UAEPAXPBD@Z 1001bdd6 f   U2Designer:U2Designer.dll
 0001:0001addc       ?qt_metacast@SpinBoxDelegate@U2@@UAEPAXPBD@Z 1001bddc f   U2Designer:U2Designer.dll
 0001:0001ade2       ?qt_metacast@URLDelegate@U2@@UAEPAXPBD@Z 1001bde2 f   U2Designer:U2Designer.dll
 0001:0001ade8       ?removeDelegate@DelegateEditor@U2@@UAEPAVPropertyDelegate@2@ABVQString@@@Z 1001bde8 f   U2Designer:U2Designer.dll
 0001:0001adee       ?setEditorData@ComboBoxDelegate@U2@@UBEXPAVQWidget@@ABVQModelIndex@@@Z 1001bdee f   U2Designer:U2Designer.dll
 0001:0001adf4       ?setEditorData@SpinBoxDelegate@U2@@UBEXPAVQWidget@@ABVQModelIndex@@@Z 1001bdf4 f   U2Designer:U2Designer.dll
 0001:0001adfa       ?setEditorData@URLDelegate@U2@@UBEXPAVQWidget@@ABVQModelIndex@@@Z 1001bdfa f   U2Designer:U2Designer.dll
 0001:0001ae00       ?setModelData@ComboBoxDelegate@U2@@UBEXPAVQWidget@@PAVQAbstractItemModel@@ABVQModelIndex@@@Z 1001be00 f   U2Designer:U2Designer.dll
 0001:0001ae06       ?setModelData@SpinBoxDelegate@U2@@UBEXPAVQWidget@@PAVQAbstractItemModel@@ABVQModelIndex@@@Z 1001be06 f   U2Designer:U2Designer.dll
 0001:0001ae0c       ?setModelData@URLDelegate@U2@@UBEXPAVQWidget@@PAVQAbstractItemModel@@ABVQModelIndex@@@Z 1001be0c f   U2Designer:U2Designer.dll
 0001:0001ae12       ?type@URLDelegate@U2@@UBE?AW4Type@PropertyDelegate@2@XZ 1001be12 f   U2Designer:U2Designer.dll
 0001:0001ae18       ?updateDelegate@DelegateEditor@U2@@UAEXABVQString@@@Z 1001be18 f   U2Designer:U2Designer.dll
 0001:0001ae1e       ?updateDelegates@DelegateEditor@U2@@UAEXXZ 1001be1e f   U2Designer:U2Designer.dll
 0001:0001ae24       ??0URLDelegate@U2@@QAE@ABVDelegateTags@1@ABVQString@@_N22PAVQObject@@22@Z 1001be24 f   U2Designer:U2Designer.dll
 0001:0001ae2a       ??0GenomicLibraryDelegate@LocalWorkflow@U2@@QAE@PAVQObject@@@Z 1001be2a f   ngs_reads_classification:ngs_reads_classification.dll
 0001:0001ae30       ?clone@GenomicLibraryDelegate@LocalWorkflow@U2@@UAEPAVPropertyDelegate@3@XZ 1001be30 f   ngs_reads_classification:ngs_reads_classification.dll
 0001:0001ae36       ?createEditor@GenomicLibraryDelegate@LocalWorkflow@U2@@UBEPAVQWidget@@PAV4@ABVQStyleOptionViewItem@@ABVQModelIndex@@@Z 1001be36 f   ngs_reads_classification:ngs_reads_classification.dll
 0001:0001ae3c       ?createWizardWidget@GenomicLibraryDelegate@LocalWorkflow@U2@@UBEPAVPropertyWidget@3@AAVU2OpStatus@3@PAVQWidget@@@Z 1001be3c f   ngs_reads_classification:ngs_reads_classification.dll
 0001:0001ae42       ?getDisplayValue@GenomicLibraryDelegate@LocalWorkflow@U2@@UBE?AVQVariant@@ABV4@@Z 1001be42 f   ngs_reads_classification:ngs_reads_classification.dll
 0001:0001ae48       ?metaObject@GenomicLibraryDelegate@LocalWorkflow@U2@@UBEPBUQMetaObject@@XZ 1001be48 f   ngs_reads_classification:ngs_reads_classification.dll
 0001:0001ae4e       ?qt_metacall@GenomicLibraryDelegate@LocalWorkflow@U2@@UAEHW4Call@QMetaObject@@HPAPAX@Z 1001be4e f   ngs_reads_classification:ngs_reads_classification.dll
 0001:0001ae54       ?qt_metacast@GenomicLibraryDelegate@LocalWorkflow@U2@@UAEPAXPBD@Z 1001be54 f   ngs_reads_classification:ngs_reads_classification.dll
 0001:0001ae5a       ?setEditorData@GenomicLibraryDelegate@LocalWorkflow@U2@@UBEXPAVQWidget@@ABVQModelIndex@@@Z 1001be5a f   ngs_reads_classification:ngs_reads_classification.dll
 0001:0001ae60       ?setModelData@GenomicLibraryDelegate@LocalWorkflow@U2@@UBEXPAVQWidget@@PAVQAbstractItemModel@@ABVQModelIndex@@@Z 1001be60 f   ngs_reads_classification:ngs_reads_classification.dll
 0001:0001ae66       ?getBaseFileNameWithSuffixes@NgsReadsClassificationUtils@U2@@SA?AVQString@@ABV3@ABVQStringList@@0_N@Z 1001be66 f   ngs_reads_classification:ngs_reads_classification.dll
 0001:0001ae6c       ?countClassified@NgsReadsClassificationUtils@U2@@SAHABV?$QMap@VQString@@I@@@Z 1001be6c f   ngs_reads_classification:ngs_reads_classification.dll
 0001:0001ae72       ?TAXONOMY_CLASSIFICATION_SLOT@TaxonomySupport@LocalWorkflow@U2@@SA?BVDescriptor@3@XZ 1001be72 f   ngs_reads_classification:ngs_reads_classification.dll
 0001:0001ae78       ?TAXONOMY_CLASSIFICATION_TYPE@TaxonomySupport@LocalWorkflow@U2@@SA?AV?$QExplicitlySharedDataPointer@VDataType@U2@@@@XZ 1001be78 f   ngs_reads_classification:ngs_reads_classification.dll
 0001:0001ae7e       ??0DatabaseDelegate@LocalWorkflow@U2@@QAE@ABVQString@@0000_N@Z 1001be7e f   ngs_reads_classification:ngs_reads_classification.dll
 0001:0001ae84       ??1DatabaseDelegate@LocalWorkflow@U2@@UAE@XZ 1001be84 f   ngs_reads_classification:ngs_reads_classification.dll
 0001:0001ae8a       ?update@DatabaseDelegate@LocalWorkflow@U2@@UAEXXZ 1001be8a f   ngs_reads_classification:ngs_reads_classification.dll
 0001:0001ae90       ?destroyEditor@QAbstractItemDelegate@@UBEXPAVQWidget@@ABVQModelIndex@@@Z 1001be90 f   Qt5Widgets:Qt5Widgets.dll
 0001:0001ae96       ?drawCheck@QItemDelegate@@MBEXPAVQPainter@@ABVQStyleOptionViewItem@@ABVQRect@@W4CheckState@Qt@@@Z 1001be96 f   Qt5Widgets:Qt5Widgets.dll
 0001:0001ae9c       ?drawDecoration@QItemDelegate@@MBEXPAVQPainter@@ABVQStyleOptionViewItem@@ABVQRect@@ABVQPixmap@@@Z 1001be9c f   Qt5Widgets:Qt5Widgets.dll
 0001:0001aea2       ?drawDisplay@QItemDelegate@@MBEXPAVQPainter@@ABVQStyleOptionViewItem@@ABVQRect@@ABVQString@@@Z 1001bea2 f   Qt5Widgets:Qt5Widgets.dll
 0001:0001aea8       ?drawFocus@QItemDelegate@@MBEXPAVQPainter@@ABVQStyleOptionViewItem@@ABVQRect@@@Z 1001bea8 f   Qt5Widgets:Qt5Widgets.dll
 0001:0001aeae       ?editorEvent@QItemDelegate@@MAE_NPAVQEvent@@PAVQAbstractItemModel@@ABVQStyleOptionViewItem@@ABVQModelIndex@@@Z 1001beae f   Qt5Widgets:Qt5Widgets.dll
 0001:0001aeb4       ?eventFilter@QItemDelegate@@MAE_NPAVQObject@@PAVQEvent@@@Z 1001beb4 f   Qt5Widgets:Qt5Widgets.dll
 0001:0001aeba       ?helpEvent@QAbstractItemDelegate@@UAE_NPAVQHelpEvent@@PAVQAbstractItemView@@ABVQStyleOptionViewItem@@ABVQModelIndex@@@Z 1001beba f   Qt5Widgets:Qt5Widgets.dll
 0001:0001aec0       ?paint@QItemDelegate@@UBEXPAVQPainter@@ABVQStyleOptionViewItem@@ABVQModelIndex@@@Z 1001bec0 f   Qt5Widgets:Qt5Widgets.dll
 0001:0001aec6       ?paintingRoles@QAbstractItemDelegate@@UBE?AV?$QVector@H@@XZ 1001bec6 f   Qt5Widgets:Qt5Widgets.dll
 0001:0001aecc       ?sizeHint@QItemDelegate@@UBE?AVQSize@@ABVQStyleOptionViewItem@@ABVQModelIndex@@@Z 1001becc f   Qt5Widgets:Qt5Widgets.dll
 0001:0001aed2       ?updateEditorGeometry@QItemDelegate@@UBEXPAVQWidget@@ABVQStyleOptionViewItem@@ABVQModelIndex@@@Z 1001bed2 f   Qt5Widgets:Qt5Widgets.dll
 0001:0001aed8       ?clear@QTextDocument@@UAEXXZ 1001bed8 f   Qt5Gui:Qt5Gui.dll
 0001:0001aede       ?createObject@QTextDocument@@MAEPAVQTextObject@@ABVQTextFormat@@@Z 1001bede f   Qt5Gui:Qt5Gui.dll
 0001:0001aee4       ?loadResource@QTextDocument@@MAE?AVQVariant@@HABVQUrl@@@Z 1001bee4 f   Qt5Gui:Qt5Gui.dll
 0001:0001aeea       ??0QScriptValue@@QAE@XZ    1001beea f   Qt5Script:Qt5Script.dll
 0001:0001aef0       ??1QScriptValue@@QAE@XZ    1001bef0 f   Qt5Script:Qt5Script.dll
 0001:0001aef6       ??0QScriptValue@@QAE@ABV0@@Z 1001bef6 f   Qt5Script:Qt5Script.dll
 0001:0001aefc       ??4QScriptValue@@QAEAAV0@ABV0@@Z 1001befc f   Qt5Script:Qt5Script.dll
 0001:0001af02       ?isNumber@QScriptValue@@QBE_NXZ 1001bf02 f   Qt5Script:Qt5Script.dll
 0001:0001af08       ?isString@QScriptValue@@QBE_NXZ 1001bf08 f   Qt5Script:Qt5Script.dll
 0001:0001af0e       ?toString@QScriptValue@@QBE?AVQString@@XZ 1001bf0e f   Qt5Script:Qt5Script.dll
 0001:0001af14       ?toInt32@QScriptValue@@QBEHXZ 1001bf14 f   Qt5Script:Qt5Script.dll
 0001:0001af1a       ??1QScriptEngine@@UAE@XZ   1001bf1a f   Qt5Script:Qt5Script.dll
 0001:0001af20       ?newVariant@QScriptEngine@@QAE?AVQScriptValue@@ABVQVariant@@@Z 1001bf20 f   Qt5Script:Qt5Script.dll
 0001:0001af26       ??0QString@@QAE@ABV0@@Z    1001bf26 f   Qt5Core:Qt5Core.dll
 0001:0001af2c       ??1QString@@QAE@XZ         1001bf2c f   Qt5Core:Qt5Core.dll
 0001:0001af32       ?append@QString@@QAEAAV1@ABV1@@Z 1001bf32 f   Qt5Core:Qt5Core.dll
 0001:0001af38       ?fromUtf8@QString@@SA?AV1@PBDH@Z 1001bf38 f   Qt5Core:Qt5Core.dll
 0001:0001af3e       ?fromAscii_helper@QString@@CAPAU?$QTypedArrayData@G@@PBDH@Z 1001bf3e f   Qt5Core:Qt5Core.dll
 0001:0001af44       ??0QFileInfo@@QAE@ABVQString@@@Z 1001bf44 f   Qt5Core:Qt5Core.dll
 0001:0001af4a       ??1QFileInfo@@QAE@XZ       1001bf4a f   Qt5Core:Qt5Core.dll
 0001:0001af50       ?exists@QFileInfo@@QBE_NXZ 1001bf50 f   Qt5Core:Qt5Core.dll
 0001:0001af56       ?size@QFileInfo@@QBE_JXZ   1001bf56 f   Qt5Core:Qt5Core.dll
 0001:0001af5c       ?freeTree@QMapDataBase@@QAEXPAUQMapNodeBase@@H@Z 1001bf5c f   Qt5Core:Qt5Core.dll
 0001:0001af62       ?freeData@QMapDataBase@@SAXPAU1@@Z 1001bf62 f   Qt5Core:Qt5Core.dll
 0001:0001af68       ??1QVariant@@QAE@XZ        1001bf68 f   Qt5Core:Qt5Core.dll
 0001:0001af6e       ??0QVariant@@QAE@ABV0@@Z   1001bf6e f   Qt5Core:Qt5Core.dll
 0001:0001af74       ??0QVariant@@QAE@_N@Z      1001bf74 f   Qt5Core:Qt5Core.dll
 0001:0001af7a       ?toString@QVariant@@QBE?AVQString@@XZ 1001bf7a f   Qt5Core:Qt5Core.dll
 0001:0001af80       ?tr@QMetaObject@@QBE?AVQString@@PBD0H@Z 1001bf80 f   Qt5Core:Qt5Core.dll
 0001:0001af86       ??1Connection@QMetaObject@@QAE@XZ 1001bf86 f   Qt5Core:Qt5Core.dll
 0001:0001af8c       ??0QChar@@QAE@UQLatin1Char@@@Z 1001bf8c f   Qt5Core:Qt5Core.dll
 0001:0001af92       ?arg@QString@@QBE?AV1@ABV1@HVQChar@@@Z 1001bf92 f   Qt5Core:Qt5Core.dll
 0001:0001af98       ??8@YA_NABVQString@@0@Z    1001bf98 f   Qt5Core:Qt5Core.dll
 0001:0001af9e       ?detach@QListData@@QAEPAUData@1@H@Z 1001bf9e f   Qt5Core:Qt5Core.dll
 0001:0001afa4       ?dispose@QListData@@SAXPAUData@1@@Z 1001bfa4 f   Qt5Core:Qt5Core.dll
 0001:0001afaa       ?connect@QObject@@QBE?AVConnection@QMetaObject@@PBV1@PBD1W4ConnectionType@Qt@@@Z 1001bfaa f   Qt5Core:Qt5Core.dll
 0001:0001afb0       ?childEvent@QObject@@MAEXPAVQChildEvent@@@Z 1001bfb0 f   Qt5Core:Qt5Core.dll
 0001:0001afb6       ?connectNotify@QObject@@MAEXABVQMetaMethod@@@Z 1001bfb6 f   Qt5Core:Qt5Core.dll
 0001:0001afbc       ?customEvent@QObject@@MAEXPAVQEvent@@@Z 1001bfbc f   Qt5Core:Qt5Core.dll
 0001:0001afc2       ?disconnectNotify@QObject@@MAEXABVQMetaMethod@@@Z 1001bfc2 f   Qt5Core:Qt5Core.dll
 0001:0001afc8       ?event@QObject@@UAE_NPAVQEvent@@@Z 1001bfc8 f   Qt5Core:Qt5Core.dll
 0001:0001afce       ?eventFilter@QObject@@UAE_NPAV1@PAVQEvent@@@Z 1001bfce f   Qt5Core:Qt5Core.dll
 0001:0001afd4       ?timerEvent@QObject@@MAEXPAVQTimerEvent@@@Z 1001bfd4 f   Qt5Core:Qt5Core.dll
 0001:0001afda       ??0QString@@QAE@XZ         1001bfda f   Qt5Core:Qt5Core.dll
 0001:0001afe0       ?arg@QString@@QBE?AV1@HHHVQChar@@@Z 1001bfe0 f   Qt5Core:Qt5Core.dll
 0001:0001afe6       ?number@QString@@SA?AV1@HH@Z 1001bfe6 f   Qt5Core:Qt5Core.dll
 0001:0001afec       ?number@QString@@SA?AV1@NDH@Z 1001bfec f   Qt5Core:Qt5Core.dll
 0001:0001aff2       ?detach_grow@QListData@@QAEPAUData@1@PAHH@Z 1001bff2 f   Qt5Core:Qt5Core.dll
 0001:0001aff8       ?append@QListData@@QAEPAPAXXZ 1001bff8 f   Qt5Core:Qt5Core.dll
 0001:0001affe       ?append@QListData@@QAEPAPAXABU1@@Z 1001bffe f   Qt5Core:Qt5Core.dll
 0001:0001b004       ?link@QFile@@SA_NABVQString@@0@Z 1001c004 f   Qt5Core:Qt5Core.dll
 0001:0001b00a       ?QStringList_contains@QtPrivate@@YA_NPBVQStringList@@ABVQString@@W4CaseSensitivity@Qt@@@Z 1001c00a f   Qt5Core:Qt5Core.dll
 0001:0001b010       ??0QDir@@QAE@ABVQString@@@Z 1001c010 f   Qt5Core:Qt5Core.dll
 0001:0001b016       ??1QDir@@QAE@XZ            1001c016 f   Qt5Core:Qt5Core.dll
 0001:0001b01c       ?entryList@QDir@@QBE?AVQStringList@@V?$QFlags@W4Filter@QDir@@@@V?$QFlags@W4SortFlag@QDir@@@@@Z 1001c01c f   Qt5Core:Qt5Core.dll
 0001:0001b022       ?userType@QVariant@@QBEHXZ 1001c022 f   Qt5Core:Qt5Core.dll
 0001:0001b028       ?constData@QVariant@@QBEPBXXZ 1001c028 f   Qt5Core:Qt5Core.dll
 0001:0001b02e       ?convert@QVariant@@QBE_NHPAX@Z 1001c02e f   Qt5Core:Qt5Core.dll
 0001:0001b034       ?translate@QCoreApplication@@SA?AVQString@@PBD00H@Z 1001c034 f   Qt5Core:Qt5Core.dll
 0001:0001b03a       ?cast@QMetaObject@@QBEPAVQObject@@PAV2@@Z 1001c03a f   Qt5Core:Qt5Core.dll
 0001:0001b040       ?normalizedType@QMetaObject@@SA?AVQByteArray@@PBD@Z 1001c040 f   Qt5Core:Qt5Core.dll
 0001:0001b046       ??1QByteArray@@QAE@XZ      1001c046 f   Qt5Core:Qt5Core.dll
 0001:0001b04c       ??0QString@@QAE@$$QAV0@@Z  1001c04c f   Qt5Core:Qt5Core.dll
 0001:0001b052       ??4QString@@QAEAAV0@$$QAV0@@Z 1001c052 f   Qt5Core:Qt5Core.dll
 0001:0001b058       ??M@YA_NABVQString@@0@Z    1001c058 f   Qt5Core:Qt5Core.dll
 0001:0001b05e       ?realloc@QListData@@QAEXH@Z 1001c05e f   Qt5Core:Qt5Core.dll
 0001:0001b064       ?registerNormalizedType@QMetaType@@SAHABVQByteArray@@P6AXPAX@ZP6APAXPBX@Z2P6APAX13@ZHV?$QFlags@W4TypeFlag@QMetaType@@@@PBUQMetaObject@@@Z 1001c064 f   Qt5Core:Qt5Core.dll
 0001:0001b06a       ?registerNormalizedTypedef@QMetaType@@SAHABVQByteArray@@H@Z 1001c06a f   Qt5Core:Qt5Core.dll
 0001:0001b070       ??1QObject@@UAE@XZ         1001c070 f   Qt5Core:Qt5Core.dll
 0001:0001b076       ?nextNode@QMapNodeBase@@QBEPBU1@XZ 1001c076 f   Qt5Core:Qt5Core.dll
 0001:0001b07c       ?freeNodeAndRebalance@QMapDataBase@@QAEXPAUQMapNodeBase@@@Z 1001c07c f   Qt5Core:Qt5Core.dll
 0001:0001b082       ?recalcMostLeftNode@QMapDataBase@@QAEXXZ 1001c082 f   Qt5Core:Qt5Core.dll
 0001:0001b088       ?createNode@QMapDataBase@@QAEPAUQMapNodeBase@@HHPAU2@_N@Z 1001c088 f   Qt5Core:Qt5Core.dll
 0001:0001b08e       ?createData@QMapDataBase@@SAPAU1@XZ 1001c08e f   Qt5Core:Qt5Core.dll
 0001:0001b094       ??0QVariant@@QAE@XZ        1001c094 f   Qt5Core:Qt5Core.dll
 0001:0001b09a       ??0QVariant@@QAE@ABVQString@@@Z 1001c09a f   Qt5Core:Qt5Core.dll
 0001:0001b0a0       ??0QVariant@@QAE@ABV?$QMap@VQString@@VQVariant@@@@@Z 1001c0a0 f   Qt5Core:Qt5Core.dll
 0001:0001b0a6       ??4QVariant@@QAEAAV0@ABV0@@Z 1001c0a6 f   Qt5Core:Qt5Core.dll
 0001:0001b0ac       ??4QVariant@@QAEAAV0@$$QAV0@@Z 1001c0ac f   Qt5Core:Qt5Core.dll
 0001:0001b0b2       ?idealThreadCount@QThread@@SAHXZ 1001c0b2 f   Qt5Core:Qt5Core.dll
 0001:0001b0b8       ??0QVariant@@QAE@H@Z       1001c0b8 f   Qt5Core:Qt5Core.dll
 0001:0001b0be       ??0QVariant@@QAE@PBD@Z     1001c0be f   Qt5Core:Qt5Core.dll
 0001:0001b0c4       ?indexOf@QString@@QBEHABV1@HW4CaseSensitivity@Qt@@@Z 1001c0c4 f   Qt5Core:Qt5Core.dll
 0001:0001b0ca       ??0QByteArray@@QAE@XZ      1001c0ca f   Qt5Core:Qt5Core.dll
 0001:0001b0d0       ??0QByteArray@@QAE@ABV0@@Z 1001c0d0 f   Qt5Core:Qt5Core.dll
 0001:0001b0d6       ??4QByteArray@@QAEAAV0@$$QAV0@@Z 1001c0d6 f   Qt5Core:Qt5Core.dll
 0001:0001b0dc       ?startsWith@QByteArray@@QBE_NPBD@Z 1001c0dc f   Qt5Core:Qt5Core.dll
 0001:0001b0e2       ?split@QByteArray@@QBE?AV?$QList@VQByteArray@@@@D@Z 1001c0e2 f   Qt5Core:Qt5Core.dll
 0001:0001b0e8       ?toUInt@QByteArray@@QBEIPA_NH@Z 1001c0e8 f   Qt5Core:Qt5Core.dll
 0001:0001b0ee       ??0QString@@QAE@ABVQByteArray@@@Z 1001c0ee f   Qt5Core:Qt5Core.dll
 0001:0001b0f4       ?readLine@QIODevice@@QAE?AVQByteArray@@_J@Z 1001c0f4 f   Qt5Core:Qt5Core.dll
 0001:0001b0fa       ?close@QFileDevice@@UAEXXZ 1001c0fa f   Qt5Core:Qt5Core.dll
 0001:0001b100       ??0QFile@@QAE@ABVQString@@@Z 1001c100 f   Qt5Core:Qt5Core.dll
 0001:0001b106       ??1QFile@@UAE@XZ           1001c106 f   Qt5Core:Qt5Core.dll
 0001:0001b10c       ?open@QFile@@UAE_NV?$QFlags@W4OpenModeFlag@QIODevice@@@@@Z 1001c10c f   Qt5Core:Qt5Core.dll
 0001:0001b112       ??4QString@@QAEAAV0@ABV0@@Z 1001c112 f   Qt5Core:Qt5Core.dll
 0001:0001b118       ?hasRegisteredConverterFunction@QMetaType@@SA_NHH@Z 1001c118 f   Qt5Core:Qt5Core.dll
 0001:0001b11e       ?registerConverterFunction@QMetaType@@SA_NPBUAbstractConverterFunction@QtPrivate@@HH@Z 1001c11e f   Qt5Core:Qt5Core.dll
 0001:0001b124       ?unregisterConverterFunction@QMetaType@@SAXHH@Z 1001c124 f   Qt5Core:Qt5Core.dll
 0001:0001b12a       ?previousNode@QMapNodeBase@@QBEPBU1@XZ 1001c12a f   Qt5Core:Qt5Core.dll
 0001:0001b130       ?free_helper@QHashData@@QAEXP6AXPAUNode@1@@Z@Z 1001c130 f   Qt5Core:Qt5Core.dll
 0001:0001b136       ??0QVariant@@QAE@HPBXI@Z   1001c136 f   Qt5Core:Qt5Core.dll
 0001:0001b13c       ?toMap@QVariant@@QBE?AV?$QMap@VQString@@VQVariant@@@@XZ 1001c13c f   Qt5Core:Qt5Core.dll
 0001:0001b142       ??4QString@@QAEAAV0@PBD@Z  1001c142 f   Qt5Core:Qt5Core.dll
 0001:0001b148       ?dir@QFileInfo@@QBE?AVQDir@@XZ 1001c148 f   Qt5Core:Qt5Core.dll
 0001:0001b14e       ??0QRegExp@@QAE@ABVQString@@W4CaseSensitivity@Qt@@W4PatternSyntax@0@@Z 1001c14e f   Qt5Core:Qt5Core.dll
 0001:0001b154       ??1QRegExp@@QAE@XZ         1001c154 f   Qt5Core:Qt5Core.dll
 0001:0001b15a       ??4QRegExp@@QAEAAV0@$$QAV0@@Z 1001c15a f   Qt5Core:Qt5Core.dll
 0001:0001b160       ?absolutePath@QDir@@QBE?AVQString@@XZ 1001c160 f   Qt5Core:Qt5Core.dll
 0001:0001b166       ?tr@QObject@@SA?AVQString@@PBD0H@Z 1001c166 f   Qt5Core:Qt5Core.dll
 0001:0001b16c       ?dynamicMetaObject@QObjectData@@QBEPAUQMetaObject@@XZ 1001c16c f   Qt5Core:Qt5Core.dll
 0001:0001b172       ?className@QMetaObject@@QBEPBDXZ 1001c172 f   Qt5Core:Qt5Core.dll
 0001:0001b178       ?reserve@QByteArray@@QAEXH@Z 1001c178 f   Qt5Core:Qt5Core.dll
 0001:0001b17e       ?append@QByteArray@@QAEAAV1@D@Z 1001c17e f   Qt5Core:Qt5Core.dll
 0001:0001b184       ?append@QByteArray@@QAEAAV1@PBD@Z 1001c184 f   Qt5Core:Qt5Core.dll
 0001:0001b18a       ?_Xbad_alloc@std@@YAXXZ    1001c18a f   msvcprt:MSVCP120.dll
 0001:0001b190       ?_Xlength_error@std@@YAXPBD@Z 1001c190 f   msvcprt:MSVCP120.dll
 0001:0001b196       ?_Xout_of_range@std@@YAXPBD@Z 1001c196 f   msvcprt:MSVCP120.dll
 0001:0001b19c       ?_Syserror_map@std@@YAPBDH@Z 1001c19c f   msvcprt:MSVCP120.dll
 0001:0001b1a2       ?_Winerror_map@std@@YAPBDH@Z 1001c1a2 f   msvcprt:MSVCP120.dll
 0001:0001b1a8       __purecall                 1001c1a8 f   MSVCRT:MSVCR120.dll
 0001:0001b1ae       ??2@YAPAXI@Z               1001c1ae f   MSVCRT:MSVCR120.dll
 0001:0001b1b4       ??3@YAXPAX@Z               1001c1b4 f   MSVCRT:MSVCR120.dll
 0001:0001b1ba       ___atonexitinit            1001c1ba f   MSVCRT:atonexit.obj
 0001:0001b1f6       __onexit                   1001c1f6 f   MSVCRT:atonexit.obj
 0001:0001b29f       _atexit                    1001c29f f   MSVCRT:atonexit.obj
 0001:0001b2b4       _memmove                   1001c2b4 f   MSVCRT:MSVCR120.dll
 0001:0001b2ba       __hypot                    1001c2ba f   MSVCRT:MSVCR120.dll
 0001:0001b2c0       @__security_check_cookie@4 1001c2c0 f   MSVCRT:secchk.obj
 0001:0001b2d0       __CxxThrowException@8      1001c2d0 f   MSVCRT:MSVCR120.dll
 0001:0001b2d6       ___CxxFrameHandler3        1001c2d6 f   MSVCRT:MSVCR120.dll
 0001:0001b2dc       _memcpy                    1001c2dc f   MSVCRT:MSVCR120.dll
 0001:0001b2e2       ??0type_info@@AAE@ABV0@@Z  1001c2e2 f   MSVCRT:ti_inst.obj
 0001:0001b2ed       ??4type_info@@AAEAAV0@ABV0@@Z 1001c2ed f   MSVCRT:ti_inst.obj
 0001:0001b2f2       ??_Etype_info@@UAEPAXI@Z   1001c2f2 f i MSVCRT:ti_inst.obj
 0001:0001b38c       _NtCurrentTeb              1001c38c f i MSVCRT:crtdll.obj
 0001:0001b393       __CRT_INIT@12              1001c393 f   MSVCRT:crtdll.obj
 0001:0001b58a       __DllMainCRTStartup@12     1001c58a f   MSVCRT:crtdll.obj
 0001:0001b6e0       __lock                     1001c6e0 f   MSVCRT:MSVCR120.dll
 0001:0001b6e6       __unlock                   1001c6e6 f   MSVCRT:MSVCR120.dll
 0001:0001b6ec       __calloc_crt               1001c6ec f   MSVCRT:MSVCR120.dll
 0001:0001b6f2       ___dllonexit               1001c6f2 f   MSVCRT:MSVCR120.dll
 0001:0001b700       __SEH_prolog4              1001c700 f   MSVCRT:sehprolg4.obj
 0001:0001b745       __SEH_epilog4              1001c745 f   MSVCRT:sehprolg4.obj
 0001:0001b759       __except_handler4          1001c759 f   MSVCRT:chandler4gs.obj
 0001:0001b77c       ___raise_securityfailure   1001c77c f   MSVCRT:gs_report.obj
 0001:0001b7b9       ___report_gsfailure        1001c7b9 f   MSVCRT:gs_report.obj
 0001:0001b8b4       ___report_rangecheckfailure 1001c8b4 f   MSVCRT:gs_report.obj
 0001:0001b8c0       ___report_securityfailure  1001c8c0 f   MSVCRT:gs_report.obj
 0001:0001b990       ___report_securityfailureEx 1001c990 f   MSVCRT:gs_report.obj
 0001:0001baa6       ??_M@YGXPAXIHP6EX0@Z@Z     1001caa6 f   MSVCRT:ehvecdtr.obj
 0001:0001bb2e       ?__ArrayUnwind@@YGXPAXIHP6EX0@Z@Z 1001cb2e f   MSVCRT:ehvecdtr.obj
 0001:0001bb8c       ??1type_info@@UAE@XZ       1001cb8c f   MSVCRT:MSVCR120.dll
 0001:0001bb92       ___CppXcptFilter           1001cb92 f   MSVCRT:MSVCR120.dll
 0001:0001bb98       __amsg_exit                1001cb98 f   MSVCRT:MSVCR120.dll
 0001:0001bba0       __FindPESection            1001cba0 f   MSVCRT:pesect.obj
 0001:0001bbf0       __IsNonwritableInCurrentImage 1001cbf0 f   MSVCRT:pesect.obj
 0001:0001bcb0       __ValidateImageBase        1001ccb0 f   MSVCRT:pesect.obj
 0001:0001bce2       _free                      1001cce2 f   MSVCRT:MSVCR120.dll
 0001:0001bce8       ___security_init_cookie    1001cce8 f   MSVCRT:gs_support.obj
 0001:0001bd84       _DllMain@12                1001cd84 f   MSVCRT:dllmain.obj
 0001:0001bda6       __malloc_crt               1001cda6 f   MSVCRT:MSVCR120.dll
 0001:0001bdac       __RTC_Initialize           1001cdac f   MSVCRT:initsect.obj
 0001:0001bdcc       __RTC_Terminate            1001cdcc f   MSVCRT:initsect.obj
 0001:0001bdec       __initterm                 1001cdec f   MSVCRT:MSVCR120.dll
 0001:0001bdf2       __initterm_e               1001cdf2 f   MSVCRT:MSVCR120.dll
 0001:0001bdf8       ___clean_type_info_names   1001cdf8 f   MSVCRT:tncleanup.obj
 0001:0001be04       __except_handler4_common   1001ce04 f   MSVCRT:MSVCR120.dll
 0001:0001be0a       __crt_debugger_hook        1001ce0a f   MSVCRT:MSVCR120.dll
 0001:0001be10       ___crtUnhandledException   1001ce10 f   MSVCRT:MSVCR120.dll
 0001:0001be16       ___crtTerminateProcess     1001ce16 f   MSVCRT:MSVCR120.dll
 0001:0001be1c       ?terminate@@YAXXZ          1001ce1c f   MSVCRT:MSVCR120.dll
 0001:0001be22       ___clean_type_info_names_internal 1001ce22 f   MSVCRT:MSVCR120.dll
 0001:0001be28       _EncodePointer@4           1001ce28 f   kernel32:KERNEL32.dll
 0001:0001be2e       _DecodePointer@4           1001ce2e f   kernel32:KERNEL32.dll
 0001:0001be34       _IsDebuggerPresent@0       1001ce34 f   kernel32:KERNEL32.dll
 0001:0001be3a       _IsProcessorFeaturePresent@4 1001ce3a f   kernel32:KERNEL32.dll
 0001:0001be40       _QueryPerformanceCounter@4 1001ce40 f   kernel32:KERNEL32.dll
 0001:0001be46       _GetCurrentProcessId@0     1001ce46 f   kernel32:KERNEL32.dll
 0001:0001be4c       _GetCurrentThreadId@0      1001ce4c f   kernel32:KERNEL32.dll
 0001:0001be52       _GetSystemTimeAsFileTime@4 1001ce52 f   kernel32:KERNEL32.dll
 0001:0001be58       _DisableThreadLibraryCalls@4 1001ce58 f   kernel32:KERNEL32.dll
 0001:00021e60       ??__Ff@?4??registerConverter@?$AssociativeValueTypeIsMetaType@V?$QMap@VQString@@I@@$00@QtPrivate@@SA_NH@Z@YAXXZ 10022e60 f i KrakenClassifyWorker.obj
 0002:00000000       __imp__GetSystemTimeAsFileTime@4 10024000     kernel32:KERNEL32.dll
 0002:00000004       __imp__GetCurrentThreadId@0 10024004     kernel32:KERNEL32.dll
 0002:00000008       __imp__GetCurrentProcessId@0 10024008     kernel32:KERNEL32.dll
 0002:0000000c       __imp__QueryPerformanceCounter@4 1002400c     kernel32:KERNEL32.dll
 0002:00000010       __imp__IsProcessorFeaturePresent@4 10024010     kernel32:KERNEL32.dll
 0002:00000014       __imp__IsDebuggerPresent@0 10024014     kernel32:KERNEL32.dll
 0002:00000018       __imp__DecodePointer@4     10024018     kernel32:KERNEL32.dll
 0002:0000001c       __imp__EncodePointer@4     1002401c     kernel32:KERNEL32.dll
 0002:00000020       __imp__DisableThreadLibraryCalls@4 10024020     kernel32:KERNEL32.dll
 0002:00000024       \177KERNEL32_NULL_THUNK_DATA 10024024     kernel32:KERNEL32.dll
 0002:00000028       __imp_?_Xbad_alloc@std@@YAXXZ 10024028     msvcprt:MSVCP120.dll
 0002:0000002c       __imp_?_Xout_of_range@std@@YAXPBD@Z 1002402c     msvcprt:MSVCP120.dll
 0002:00000030       __imp_?_Syserror_map@std@@YAPBDH@Z 10024030     msvcprt:MSVCP120.dll
 0002:00000034       __imp_?_Winerror_map@std@@YAPBDH@Z 10024034     msvcprt:MSVCP120.dll
 0002:00000038       __imp_?_Xlength_error@std@@YAXPBD@Z 10024038     msvcprt:MSVCP120.dll
 0002:0000003c       \177MSVCP120_NULL_THUNK_DATA 1002403c     msvcprt:MSVCP120.dll
 0002:00000040       __imp___unlock             10024040     MSVCRT:MSVCR120.dll
 0002:00000044       __imp___calloc_crt         10024044     MSVCRT:MSVCR120.dll
 0002:00000048       __imp____dllonexit         10024048     MSVCRT:MSVCR120.dll
 0002:0000004c       __imp___onexit             1002404c     MSVCRT:MSVCR120.dll
 0002:00000050       __imp_??1type_info@@UAE@XZ 10024050     MSVCRT:MSVCR120.dll
 0002:00000054       __imp_??3@YAXPAX@Z         10024054     MSVCRT:MSVCR120.dll
 0002:00000058       __imp___amsg_exit          10024058     MSVCRT:MSVCR120.dll
 0002:0000005c       __imp__free                1002405c     MSVCRT:MSVCR120.dll
 0002:00000060       __imp___malloc_crt         10024060     MSVCRT:MSVCR120.dll
 0002:00000064       __imp___lock               10024064     MSVCRT:MSVCR120.dll
 0002:00000068       __imp___initterm_e         10024068     MSVCRT:MSVCR120.dll
 0002:0000006c       __imp___except_handler4_common 1002406c     MSVCRT:MSVCR120.dll
 0002:00000070       __imp___crt_debugger_hook  10024070     MSVCRT:MSVCR120.dll
 0002:00000074       __imp____crtUnhandledException 10024074     MSVCRT:MSVCR120.dll
 0002:00000078       __imp____crtTerminateProcess 10024078     MSVCRT:MSVCR120.dll
 0002:0000007c       __imp_?terminate@@YAXXZ    1002407c     MSVCRT:MSVCR120.dll
 0002:00000080       __imp____clean_type_info_names_internal 10024080     MSVCRT:MSVCR120.dll
 0002:00000084       __imp_??2@YAPAXI@Z         10024084     MSVCRT:MSVCR120.dll
 0002:00000088       __imp___purecall           10024088     MSVCRT:MSVCR120.dll
 0002:0000008c       __imp__memcpy              1002408c     MSVCRT:MSVCR120.dll
 0002:00000090       __imp____CxxFrameHandler3  10024090     MSVCRT:MSVCR120.dll
 0002:00000094       __imp___CxxThrowException@8 10024094     MSVCRT:MSVCR120.dll
 0002:00000098       __imp___hypot              10024098     MSVCRT:MSVCR120.dll
 0002:0000009c       __imp___initterm           1002409c     MSVCRT:MSVCR120.dll
 0002:000000a0       __imp__memmove             100240a0     MSVCRT:MSVCR120.dll
 0002:000000a4       __imp____CppXcptFilter     100240a4     MSVCRT:MSVCR120.dll
 0002:000000a8       \177MSVCR120_NULL_THUNK_DATA 100240a8     MSVCRT:MSVCR120.dll
 0002:000000ac       __imp_?dynamicMetaObject@QObjectData@@QBEPAUQMetaObject@@XZ 100240ac     Qt5Core:Qt5Core.dll
 0002:000000b0       __imp_??4QRegExp@@QAEAAV0@$$QAV0@@Z 100240b0     Qt5Core:Qt5Core.dll
 0002:000000b4       __imp_?absolutePath@QDir@@QBE?AVQString@@XZ 100240b4     Qt5Core:Qt5Core.dll
 0002:000000b8       __imp_?tr@QObject@@SA?AVQString@@PBD0H@Z 100240b8     Qt5Core:Qt5Core.dll
 0002:000000bc       __imp_?className@QMetaObject@@QBEPBDXZ 100240bc     Qt5Core:Qt5Core.dll
 0002:000000c0       __imp_?reserve@QByteArray@@QAEXH@Z 100240c0     Qt5Core:Qt5Core.dll
 0002:000000c4       __imp_?append@QByteArray@@QAEAAV1@D@Z 100240c4     Qt5Core:Qt5Core.dll
 0002:000000c8       __imp_?append@QByteArray@@QAEAAV1@PBD@Z 100240c8     Qt5Core:Qt5Core.dll
 0002:000000cc       __imp_??0QRegExp@@QAE@ABVQString@@W4CaseSensitivity@Qt@@W4PatternSyntax@0@@Z 100240cc     Qt5Core:Qt5Core.dll
 0002:000000d0       __imp_?dir@QFileInfo@@QBE?AVQDir@@XZ 100240d0     Qt5Core:Qt5Core.dll
 0002:000000d4       __imp_??4QString@@QAEAAV0@PBD@Z 100240d4     Qt5Core:Qt5Core.dll
 0002:000000d8       __imp_?shared_null@QHashData@@2U1@B 100240d8     Qt5Core:Qt5Core.dll
 0002:000000dc       __imp_?toMap@QVariant@@QBE?AV?$QMap@VQString@@VQVariant@@@@XZ 100240dc     Qt5Core:Qt5Core.dll
 0002:000000e0       __imp_??0QVariant@@QAE@HPBXI@Z 100240e0     Qt5Core:Qt5Core.dll
 0002:000000e4       __imp_?free_helper@QHashData@@QAEXP6AXPAUNode@1@@Z@Z 100240e4     Qt5Core:Qt5Core.dll
 0002:000000e8       __imp_?previousNode@QMapNodeBase@@QBEPBU1@XZ 100240e8     Qt5Core:Qt5Core.dll
 0002:000000ec       __imp_?unregisterConverterFunction@QMetaType@@SAXHH@Z 100240ec     Qt5Core:Qt5Core.dll
 0002:000000f0       __imp_?registerConverterFunction@QMetaType@@SA_NPBUAbstractConverterFunction@QtPrivate@@HH@Z 100240f0     Qt5Core:Qt5Core.dll
 0002:000000f4       __imp_?hasRegisteredConverterFunction@QMetaType@@SA_NHH@Z 100240f4     Qt5Core:Qt5Core.dll
 0002:000000f8       __imp_??4QString@@QAEAAV0@ABV0@@Z 100240f8     Qt5Core:Qt5Core.dll
 0002:000000fc       __imp_?open@QFile@@UAE_NV?$QFlags@W4OpenModeFlag@QIODevice@@@@@Z 100240fc     Qt5Core:Qt5Core.dll
 0002:00000100       __imp_??1QFile@@UAE@XZ     10024100     Qt5Core:Qt5Core.dll
 0002:00000104       __imp_??0QFile@@QAE@ABVQString@@@Z 10024104     Qt5Core:Qt5Core.dll
 0002:00000108       __imp_?close@QFileDevice@@UAEXXZ 10024108     Qt5Core:Qt5Core.dll
 0002:0000010c       __imp_?readLine@QIODevice@@QAE?AVQByteArray@@_J@Z 1002410c     Qt5Core:Qt5Core.dll
 0002:00000110       __imp_??0QString@@QAE@ABVQByteArray@@@Z 10024110     Qt5Core:Qt5Core.dll
 0002:00000114       __imp_?toUInt@QByteArray@@QBEIPA_NH@Z 10024114     Qt5Core:Qt5Core.dll
 0002:00000118       __imp_??0QString@@QAE@ABV0@@Z 10024118     Qt5Core:Qt5Core.dll
 0002:0000011c       __imp_??1QString@@QAE@XZ   1002411c     Qt5Core:Qt5Core.dll
 0002:00000120       __imp_?append@QString@@QAEAAV1@ABV1@@Z 10024120     Qt5Core:Qt5Core.dll
 0002:00000124       __imp_?fromUtf8@QString@@SA?AV1@PBDH@Z 10024124     Qt5Core:Qt5Core.dll
 0002:00000128       __imp_?fromAscii_helper@QString@@CAPAU?$QTypedArrayData@G@@PBDH@Z 10024128     Qt5Core:Qt5Core.dll
 0002:0000012c       __imp_??0QFileInfo@@QAE@ABVQString@@@Z 1002412c     Qt5Core:Qt5Core.dll
 0002:00000130       __imp_??1QFileInfo@@QAE@XZ 10024130     Qt5Core:Qt5Core.dll
 0002:00000134       __imp_?exists@QFileInfo@@QBE_NXZ 10024134     Qt5Core:Qt5Core.dll
 0002:00000138       __imp_?size@QFileInfo@@QBE_JXZ 10024138     Qt5Core:Qt5Core.dll
 0002:0000013c       __imp_?freeTree@QMapDataBase@@QAEXPAUQMapNodeBase@@H@Z 1002413c     Qt5Core:Qt5Core.dll
 0002:00000140       __imp_?freeData@QMapDataBase@@SAXPAU1@@Z 10024140     Qt5Core:Qt5Core.dll
 0002:00000144       __imp_??1QVariant@@QAE@XZ  10024144     Qt5Core:Qt5Core.dll
 0002:00000148       __imp_??0QVariant@@QAE@ABV0@@Z 10024148     Qt5Core:Qt5Core.dll
 0002:0000014c       __imp_??0QVariant@@QAE@_N@Z 1002414c     Qt5Core:Qt5Core.dll
 0002:00000150       __imp_?toString@QVariant@@QBE?AVQString@@XZ 10024150     Qt5Core:Qt5Core.dll
 0002:00000154       __imp_?shared_null@QMapDataBase@@2U1@B 10024154     Qt5Core:Qt5Core.dll
 0002:00000158       __imp_?tr@QMetaObject@@QBE?AVQString@@PBD0H@Z 10024158     Qt5Core:Qt5Core.dll
 0002:0000015c       __imp_??1Connection@QMetaObject@@QAE@XZ 1002415c     Qt5Core:Qt5Core.dll
 0002:00000160       __imp_??0QChar@@QAE@UQLatin1Char@@@Z 10024160     Qt5Core:Qt5Core.dll
 0002:00000164       __imp_?arg@QString@@QBE?AV1@ABV1@HVQChar@@@Z 10024164     Qt5Core:Qt5Core.dll
 0002:00000168       __imp_??8@YA_NABVQString@@0@Z 10024168     Qt5Core:Qt5Core.dll
 0002:0000016c       __imp_?detach@QListData@@QAEPAUData@1@H@Z 1002416c     Qt5Core:Qt5Core.dll
 0002:00000170       __imp_?dispose@QListData@@SAXPAUData@1@@Z 10024170     Qt5Core:Qt5Core.dll
 0002:00000174       __imp_?connect@QObject@@QBE?AVConnection@QMetaObject@@PBV1@PBD1W4ConnectionType@Qt@@@Z 10024174     Qt5Core:Qt5Core.dll
 0002:00000178       __imp_?childEvent@QObject@@MAEXPAVQChildEvent@@@Z 10024178     Qt5Core:Qt5Core.dll
 0002:0000017c       __imp_?connectNotify@QObject@@MAEXABVQMetaMethod@@@Z 1002417c     Qt5Core:Qt5Core.dll
 0002:00000180       __imp_?customEvent@QObject@@MAEXPAVQEvent@@@Z 10024180     Qt5Core:Qt5Core.dll
 0002:00000184       __imp_?disconnectNotify@QObject@@MAEXABVQMetaMethod@@@Z 10024184     Qt5Core:Qt5Core.dll
 0002:00000188       __imp_?event@QObject@@UAE_NPAVQEvent@@@Z 10024188     Qt5Core:Qt5Core.dll
 0002:0000018c       __imp_?eventFilter@QObject@@UAE_NPAV1@PAVQEvent@@@Z 1002418c     Qt5Core:Qt5Core.dll
 0002:00000190       __imp_?timerEvent@QObject@@MAEXPAVQTimerEvent@@@Z 10024190     Qt5Core:Qt5Core.dll
 0002:00000194       __imp_??0QString@@QAE@XZ   10024194     Qt5Core:Qt5Core.dll
 0002:00000198       __imp_?arg@QString@@QBE?AV1@HHHVQChar@@@Z 10024198     Qt5Core:Qt5Core.dll
 0002:0000019c       __imp_?number@QString@@SA?AV1@HH@Z 1002419c     Qt5Core:Qt5Core.dll
 0002:000001a0       __imp_?number@QString@@SA?AV1@NDH@Z 100241a0     Qt5Core:Qt5Core.dll
 0002:000001a4       __imp_?detach_grow@QListData@@QAEPAUData@1@PAHH@Z 100241a4     Qt5Core:Qt5Core.dll
 0002:000001a8       __imp_?append@QListData@@QAEPAPAXXZ 100241a8     Qt5Core:Qt5Core.dll
 0002:000001ac       __imp_?append@QListData@@QAEPAPAXABU1@@Z 100241ac     Qt5Core:Qt5Core.dll
 0002:000001b0       __imp_?link@QFile@@SA_NABVQString@@0@Z 100241b0     Qt5Core:Qt5Core.dll
 0002:000001b4       __imp_?QStringList_contains@QtPrivate@@YA_NPBVQStringList@@ABVQString@@W4CaseSensitivity@Qt@@@Z 100241b4     Qt5Core:Qt5Core.dll
 0002:000001b8       __imp_??0QDir@@QAE@ABVQString@@@Z 100241b8     Qt5Core:Qt5Core.dll
 0002:000001bc       __imp_??1QDir@@QAE@XZ      100241bc     Qt5Core:Qt5Core.dll
 0002:000001c0       __imp_?entryList@QDir@@QBE?AVQStringList@@V?$QFlags@W4Filter@QDir@@@@V?$QFlags@W4SortFlag@QDir@@@@@Z 100241c0     Qt5Core:Qt5Core.dll
 0002:000001c4       __imp_?shared_null@QListData@@2UData@1@B 100241c4     Qt5Core:Qt5Core.dll
 0002:000001c8       __imp_?userType@QVariant@@QBEHXZ 100241c8     Qt5Core:Qt5Core.dll
 0002:000001cc       __imp_?constData@QVariant@@QBEPBXXZ 100241cc     Qt5Core:Qt5Core.dll
 0002:000001d0       __imp_?convert@QVariant@@QBE_NHPAX@Z 100241d0     Qt5Core:Qt5Core.dll
 0002:000001d4       __imp_?translate@QCoreApplication@@SA?AVQString@@PBD00H@Z 100241d4     Qt5Core:Qt5Core.dll
 0002:000001d8       __imp_?cast@QMetaObject@@QBEPAVQObject@@PAV2@@Z 100241d8     Qt5Core:Qt5Core.dll
 0002:000001dc       __imp_?normalizedType@QMetaObject@@SA?AVQByteArray@@PBD@Z 100241dc     Qt5Core:Qt5Core.dll
 0002:000001e0       __imp_??1QByteArray@@QAE@XZ 100241e0     Qt5Core:Qt5Core.dll
 0002:000001e4       __imp_??0QString@@QAE@$$QAV0@@Z 100241e4     Qt5Core:Qt5Core.dll
 0002:000001e8       __imp_??4QString@@QAEAAV0@$$QAV0@@Z 100241e8     Qt5Core:Qt5Core.dll
 0002:000001ec       __imp_??M@YA_NABVQString@@0@Z 100241ec     Qt5Core:Qt5Core.dll
 0002:000001f0       __imp_?realloc@QListData@@QAEXH@Z 100241f0     Qt5Core:Qt5Core.dll
 0002:000001f4       __imp_?registerNormalizedType@QMetaType@@SAHABVQByteArray@@P6AXPAX@ZP6APAXPBX@Z2P6APAX13@ZHV?$QFlags@W4TypeFlag@QMetaType@@@@PBUQMetaObject@@@Z 100241f4     Qt5Core:Qt5Core.dll
 0002:000001f8       __imp_?registerNormalizedTypedef@QMetaType@@SAHABVQByteArray@@H@Z 100241f8     Qt5Core:Qt5Core.dll
 0002:000001fc       __imp_??1QObject@@UAE@XZ   100241fc     Qt5Core:Qt5Core.dll
 0002:00000200       __imp_?nextNode@QMapNodeBase@@QBEPBU1@XZ 10024200     Qt5Core:Qt5Core.dll
 0002:00000204       __imp_?freeNodeAndRebalance@QMapDataBase@@QAEXPAUQMapNodeBase@@@Z 10024204     Qt5Core:Qt5Core.dll
 0002:00000208       __imp_?recalcMostLeftNode@QMapDataBase@@QAEXXZ 10024208     Qt5Core:Qt5Core.dll
 0002:0000020c       __imp_?createNode@QMapDataBase@@QAEPAUQMapNodeBase@@HHPAU2@_N@Z 1002420c     Qt5Core:Qt5Core.dll
 0002:00000210       __imp_?createData@QMapDataBase@@SAPAU1@XZ 10024210     Qt5Core:Qt5Core.dll
 0002:00000214       __imp_??0QVariant@@QAE@XZ  10024214     Qt5Core:Qt5Core.dll
 0002:00000218       __imp_??0QVariant@@QAE@ABVQString@@@Z 10024218     Qt5Core:Qt5Core.dll
 0002:0000021c       __imp_??0QVariant@@QAE@ABV?$QMap@VQString@@VQVariant@@@@@Z 1002421c     Qt5Core:Qt5Core.dll
 0002:00000220       __imp_??4QVariant@@QAEAAV0@ABV0@@Z 10024220     Qt5Core:Qt5Core.dll
 0002:00000224       __imp_??4QVariant@@QAEAAV0@$$QAV0@@Z 10024224     Qt5Core:Qt5Core.dll
 0002:00000228       __imp_?idealThreadCount@QThread@@SAHXZ 10024228     Qt5Core:Qt5Core.dll
 0002:0000022c       __imp_??0QVariant@@QAE@H@Z 1002422c     Qt5Core:Qt5Core.dll
 0002:00000230       __imp_??0QVariant@@QAE@PBD@Z 10024230     Qt5Core:Qt5Core.dll
 0002:00000234       __imp_?indexOf@QString@@QBEHABV1@HW4CaseSensitivity@Qt@@@Z 10024234     Qt5Core:Qt5Core.dll
 0002:00000238       __imp_??0QByteArray@@QAE@XZ 10024238     Qt5Core:Qt5Core.dll
 0002:0000023c       __imp_??0QByteArray@@QAE@ABV0@@Z 1002423c     Qt5Core:Qt5Core.dll
 0002:00000240       __imp_??4QByteArray@@QAEAAV0@$$QAV0@@Z 10024240     Qt5Core:Qt5Core.dll
 0002:00000244       __imp_?startsWith@QByteArray@@QBE_NPBD@Z 10024244     Qt5Core:Qt5Core.dll
 0002:00000248       __imp_?split@QByteArray@@QBE?AV?$QList@VQByteArray@@@@D@Z 10024248     Qt5Core:Qt5Core.dll
 0002:0000024c       __imp_??1QRegExp@@QAE@XZ   1002424c     Qt5Core:Qt5Core.dll
 0002:00000250       \177Qt5Core_NULL_THUNK_DATA 10024250     Qt5Core:Qt5Core.dll
 0002:00000254       __imp_?clear@QTextDocument@@UAEXXZ 10024254     Qt5Gui:Qt5Gui.dll
 0002:00000258       __imp_?createObject@QTextDocument@@MAEPAVQTextObject@@ABVQTextFormat@@@Z 10024258     Qt5Gui:Qt5Gui.dll
 0002:0000025c       __imp_?loadResource@QTextDocument@@MAE?AVQVariant@@HABVQUrl@@@Z 1002425c     Qt5Gui:Qt5Gui.dll
 0002:00000260       \177Qt5Gui_NULL_THUNK_DATA 10024260     Qt5Gui:Qt5Gui.dll
 0002:00000264       __imp_?isString@QScriptValue@@QBE_NXZ 10024264     Qt5Script:Qt5Script.dll
 0002:00000268       __imp_?isNumber@QScriptValue@@QBE_NXZ 10024268     Qt5Script:Qt5Script.dll
 0002:0000026c       __imp_??4QScriptValue@@QAEAAV0@ABV0@@Z 1002426c     Qt5Script:Qt5Script.dll
 0002:00000270       __imp_??0QScriptValue@@QAE@ABV0@@Z 10024270     Qt5Script:Qt5Script.dll
 0002:00000274       __imp_??1QScriptValue@@QAE@XZ 10024274     Qt5Script:Qt5Script.dll
 0002:00000278       __imp_??0QScriptValue@@QAE@XZ 10024278     Qt5Script:Qt5Script.dll
 0002:0000027c       __imp_?toString@QScriptValue@@QBE?AVQString@@XZ 1002427c     Qt5Script:Qt5Script.dll
 0002:00000280       __imp_?toInt32@QScriptValue@@QBEHXZ 10024280     Qt5Script:Qt5Script.dll
 0002:00000284       __imp_??1QScriptEngine@@UAE@XZ 10024284     Qt5Script:Qt5Script.dll
 0002:00000288       __imp_?newVariant@QScriptEngine@@QAE?AVQScriptValue@@ABVQVariant@@@Z 10024288     Qt5Script:Qt5Script.dll
 0002:0000028c       \177Qt5Script_NULL_THUNK_DATA 1002428c     Qt5Script:Qt5Script.dll
 0002:00000290       __imp_?updateEditorGeometry@QItemDelegate@@UBEXPAVQWidget@@ABVQStyleOptionViewItem@@ABVQModelIndex@@@Z 10024290     Qt5Widgets:Qt5Widgets.dll
 0002:00000294       __imp_?paintingRoles@QAbstractItemDelegate@@UBE?AV?$QVector@H@@XZ 10024294     Qt5Widgets:Qt5Widgets.dll
 0002:00000298       __imp_?paint@QItemDelegate@@UBEXPAVQPainter@@ABVQStyleOptionViewItem@@ABVQModelIndex@@@Z 10024298     Qt5Widgets:Qt5Widgets.dll
 0002:0000029c       __imp_?helpEvent@QAbstractItemDelegate@@UAE_NPAVQHelpEvent@@PAVQAbstractItemView@@ABVQStyleOptionViewItem@@ABVQModelIndex@@@Z 1002429c     Qt5Widgets:Qt5Widgets.dll
 0002:000002a0       __imp_?eventFilter@QItemDelegate@@MAE_NPAVQObject@@PAVQEvent@@@Z 100242a0     Qt5Widgets:Qt5Widgets.dll
 0002:000002a4       __imp_?editorEvent@QItemDelegate@@MAE_NPAVQEvent@@PAVQAbstractItemModel@@ABVQStyleOptionViewItem@@ABVQModelIndex@@@Z 100242a4     Qt5Widgets:Qt5Widgets.dll
 0002:000002a8       __imp_?drawFocus@QItemDelegate@@MBEXPAVQPainter@@ABVQStyleOptionViewItem@@ABVQRect@@@Z 100242a8     Qt5Widgets:Qt5Widgets.dll
 0002:000002ac       __imp_?destroyEditor@QAbstractItemDelegate@@UBEXPAVQWidget@@ABVQModelIndex@@@Z 100242ac     Qt5Widgets:Qt5Widgets.dll
 0002:000002b0       __imp_?drawDisplay@QItemDelegate@@MBEXPAVQPainter@@ABVQStyleOptionViewItem@@ABVQRect@@ABVQString@@@Z 100242b0     Qt5Widgets:Qt5Widgets.dll
 0002:000002b4       __imp_?drawDecoration@QItemDelegate@@MBEXPAVQPainter@@ABVQStyleOptionViewItem@@ABVQRect@@ABVQPixmap@@@Z 100242b4     Qt5Widgets:Qt5Widgets.dll
 0002:000002b8       __imp_?drawCheck@QItemDelegate@@MBEXPAVQPainter@@ABVQStyleOptionViewItem@@ABVQRect@@W4CheckState@Qt@@@Z 100242b8     Qt5Widgets:Qt5Widgets.dll
 0002:000002bc       __imp_?sizeHint@QItemDelegate@@UBE?AVQSize@@ABVQStyleOptionViewItem@@ABVQModelIndex@@@Z 100242bc     Qt5Widgets:Qt5Widgets.dll
 0002:000002c0       \177Qt5Widgets_NULL_THUNK_DATA 100242c0     Qt5Widgets:Qt5Widgets.dll
 0002:000002c4       __imp_??0Logger@U2@@QAE@ABVQString@@@Z 100242c4     U2Core:U2Core.dll
 0002:000002c8       __imp_??1Logger@U2@@UAE@XZ 100242c8     U2Core:U2Core.dll
 0002:000002cc       __imp_?getTotalPhysicalMemory@AppResourcePool@U2@@SAHXZ 100242cc     U2Core:U2Core.dll
 0002:000002d0       __imp_?getDataPathRegistry@AppContext@U2@@SAPAVU2DataPathRegistry@2@XZ 100242d0     U2Core:U2Core.dll
 0002:000002d4       __imp_?error@Logger@U2@@QAEXABVQString@@@Z 100242d4     U2Core:U2Core.dll
 0002:000002d8       __imp_?getTaskName@Task@U2@@QBE?AVQString@@XZ 100242d8     U2Core:U2Core.dll
 0002:000002dc       __imp_?addSubTask@Task@U2@@QAEXPAV12@@Z 100242dc     U2Core:U2Core.dll
 0002:000002e0       __imp_?setError@Task@U2@@QAEXABVQString@@@Z 100242e0     U2Core:U2Core.dll
 0002:000002e4       __imp_?setTaskName@Task@U2@@IAEXABVQString@@@Z 100242e4     U2Core:U2Core.dll
 0002:000002e8       __imp_??0CopyFileTask@U2@@QAE@ABVQString@@0@Z 100242e8     U2Core:U2Core.dll
 0002:000002ec       __imp_??1CopyFileTask@U2@@UAE@XZ 100242ec     U2Core:U2Core.dll
 0002:000002f0       __imp_??1GCounter@U2@@UAE@XZ 100242f0     U2Core:U2Core.dll
 0002:000002f4       __imp_??0GReportableCounter@U2@@QAE@ABVQString@@0N@Z 100242f4     U2Core:U2Core.dll
 0002:000002f8       __imp_??1SimpleEventCounter@U2@@UAE@XZ 100242f8     U2Core:U2Core.dll
 0002:000002fc       __imp_?getPath@U2DataPath@U2@@QBEABVQString@@XZ 100242fc     U2Core:U2Core.dll
 0002:00000300       __imp_?isValid@U2DataPath@U2@@QBE_NXZ 10024300     U2Core:U2Core.dll
 0002:00000304       __imp_?getDataPathByName@U2DataPathRegistry@U2@@QAEPAVU2DataPath@2@ABVQString@@@Z 10024304     U2Core:U2Core.dll
 0002:00000308       __imp_?prepareDirLocation@GUrlUtils@U2@@SA?AVQString@@ABV3@AAVU2OpStatus@2@@Z 10024308     U2Core:U2Core.dll
 0002:0000030c       __imp_??0SequentialMultiTask@U2@@QAE@ABVQString@@ABV?$QList@PAVTask@U2@@@@V?$QFlags@W4TaskFlag@U2@@@@@Z 1002430c     U2Core:U2Core.dll
 0002:00000310       __imp_??1SequentialMultiTask@U2@@UAE@XZ 10024310     U2Core:U2Core.dll
 0002:00000314       __imp_??0ExternalToolRunTask@U2@@QAE@ABVQString@@ABVQStringList@@PAVExternalToolLogParser@1@010_N@Z 10024314     U2Core:U2Core.dll
 0002:00000318       __imp_??1ExternalToolRunTask@U2@@UAE@XZ 10024318     U2Core:U2Core.dll
 0002:0000031c       __imp_??0ExternalToolSupportTask@U2@@QAE@ABVQString@@V?$QFlags@W4TaskFlag@U2@@@@@Z 1002431c     U2Core:U2Core.dll
 0002:00000320       __imp_??1ExternalToolSupportTask@U2@@UAE@XZ 10024320     U2Core:U2Core.dll
 0002:00000324       __imp_??0ExternalToolLogParser@U2@@QAE@_N@Z 10024324     U2Core:U2Core.dll
 0002:00000328       __imp_??1ExternalToolLogParser@U2@@UAE@XZ 10024328     U2Core:U2Core.dll
 0002:0000032c       __imp_?cleanup@Task@U2@@UAEXXZ 1002432c     U2Core:U2Core.dll
 0002:00000330       __imp_?generateReport@Task@U2@@UBE?AVQString@@XZ 10024330     U2Core:U2Core.dll
 0002:00000334       __imp_?getNumParallelSubtasks@Task@U2@@UBEHXZ 10024334     U2Core:U2Core.dll
 0002:00000338       __imp_?getParentTask@Task@U2@@UBEPAV12@XZ 10024338     U2Core:U2Core.dll
 0002:0000033c       __imp_?getProgress@ExternalToolLogParser@U2@@UAEHXZ 1002433c     U2Core:U2Core.dll
 0002:00000340       __imp_?getSubtaskWithErrors@Task@U2@@UBEPAV12@XZ 10024340     U2Core:U2Core.dll
 0002:00000344       __imp_?getTaskId@Task@U2@@UBE_JXZ 10024344     U2Core:U2Core.dll
 0002:00000348       __imp_?getTopLevelParentTask@Task@U2@@UAEPAV12@XZ 10024348     U2Core:U2Core.dll
 0002:0000034c       __imp_?getWarnings@Task@U2@@UBE?AVQStringList@@XZ 1002434c     U2Core:U2Core.dll
 0002:00000350       __imp_?hasSubtasksWithErrors@Task@U2@@UBE_NXZ 10024350     U2Core:U2Core.dll
 0002:00000354       __imp_?hasWarning@Task@U2@@UBE_NXZ 10024354     U2Core:U2Core.dll
 0002:00000358       __imp_?isError@ExternalToolLogParser@U2@@MBE_NABVQString@@@Z 10024358     U2Core:U2Core.dll
 0002:0000035c       __imp_?isNotificationReport@Task@U2@@UBE_NXZ 1002435c     U2Core:U2Core.dll
 0002:00000360       __imp_?isReportingEnabled@Task@U2@@UBE_NXZ 10024360     U2Core:U2Core.dll
 0002:00000364       __imp_?isReportingSupported@Task@U2@@UBE_NXZ 10024364     U2Core:U2Core.dll
 0002:00000368       __imp_?isTopLevelTask@Task@U2@@UBE_NXZ 10024368     U2Core:U2Core.dll
 0002:0000036c       __imp_?staticMetaObject@Plugin@U2@@2UQMetaObject@@B 1002436c     U2Core:U2Core.dll
 0002:00000370       __imp_?qt_metacall@Plugin@U2@@UAEHW4Call@QMetaObject@@HPAPAX@Z 10024370     U2Core:U2Core.dll
 0002:00000374       __imp_?qt_metacast@Plugin@U2@@UAEPAXPBD@Z 10024374     U2Core:U2Core.dll
 0002:00000378       __imp_?staticMetaObject@ExternalTool@U2@@2UQMetaObject@@B 10024378     U2Core:U2Core.dll
 0002:0000037c       __imp_?qt_metacall@ExternalTool@U2@@UAEHW4Call@QMetaObject@@HPAPAX@Z 1002437c     U2Core:U2Core.dll
 0002:00000380       __imp_?qt_metacast@ExternalTool@U2@@UAEPAXPBD@Z 10024380     U2Core:U2Core.dll
 0002:00000384       __imp_?staticMetaObject@Task@U2@@2UQMetaObject@@B 10024384     U2Core:U2Core.dll
 0002:00000388       __imp_?qt_metacall@Task@U2@@UAEHW4Call@QMetaObject@@HPAPAX@Z 10024388     U2Core:U2Core.dll
 0002:0000038c       __imp_?qt_metacast@Task@U2@@UAEPAXPBD@Z 1002438c     U2Core:U2Core.dll
 0002:00000390       __imp_??1Plugin@U2@@UAE@XZ 10024390     U2Core:U2Core.dll
 0002:00000394       __imp_??0Plugin@U2@@QAE@ABVQString@@0_NW4PluginState@1@@Z 10024394     U2Core:U2Core.dll
 0002:00000398       __imp_?setToolkitDescription@ExternalToolRegistry@U2@@QAEXABVQString@@0@Z 10024398     U2Core:U2Core.dll
 0002:0000039c       __imp_?unregisterEntry@ExternalToolRegistry@U2@@QAEXABVQString@@@Z 1002439c     U2Core:U2Core.dll
 0002:000003a0       __imp_?registerEntry@ExternalToolRegistry@U2@@QAE_NPAVExternalTool@2@@Z 100243a0     U2Core:U2Core.dll
 0002:000003a4       __imp_?getExternalToolRegistry@AppContext@U2@@SAPAVExternalToolRegistry@2@XZ 100243a4     U2Core:U2Core.dll
 0002:000003a8       __imp_?performAdditionalChecks@ExternalTool@U2@@UAEXABVQString@@@Z 100243a8     U2Core:U2Core.dll
 0002:000003ac       __imp_?getToolRunnerAdditionalOptions@ExternalTool@U2@@UBE?AVQStringList@@XZ 100243ac     U2Core:U2Core.dll
 0002:000003b0       __imp_?getRunParameters@ExternalTool@U2@@UBE?AVQStringList@@XZ 100243b0     U2Core:U2Core.dll
 0002:000003b4       __imp_?extractAdditionalParameters@ExternalTool@U2@@UAEXABVQString@@@Z 100243b4     U2Core:U2Core.dll
 0002:000003b8       __imp_??1ExternalTool@U2@@UAE@XZ 100243b8     U2Core:U2Core.dll
 0002:000003bc       __imp_??0ExternalTool@U2@@QAE@VQString@@00@Z 100243bc     U2Core:U2Core.dll
 0002:000003c0       __imp_?PLAIN_TEXT@BaseDocumentFormats@U2@@2VQString@@B 100243c0     U2Core:U2Core.dll
 0002:000003c4       __imp_?qt_metacast@FailTask@U2@@UAEPAXPBD@Z 100243c4     U2Core:U2Core.dll
 0002:000003c8       __imp_?qt_metacall@FailTask@U2@@UAEHW4Call@QMetaObject@@HPAPAX@Z 100243c8     U2Core:U2Core.dll
 0002:000003cc       __imp_?metaObject@FailTask@U2@@UBEPBUQMetaObject@@XZ 100243cc     U2Core:U2Core.dll
 0002:000003d0       __imp_??1U2OpStatus2Log@U2@@UAE@XZ 100243d0     U2Core:U2Core.dll
 0002:000003d4       __imp_??0U2OpStatus2Log@U2@@QAE@W4LogLevel@1@@Z 100243d4     U2Core:U2Core.dll
 0002:000003d8       __imp_?getError@U2OpStatusImpl@U2@@UBE?AVQString@@XZ 100243d8     U2Core:U2Core.dll
 0002:000003dc       __imp_?createDirectory@GUrlUtils@U2@@SA?AVQString@@ABV3@0AAVU2OpStatus@2@@Z 100243dc     U2Core:U2Core.dll
 0002:000003e0       __imp_?rollFileName@GUrlUtils@U2@@SA?AVQString@@ABV3@0ABV?$QSet@VQString@@@@@Z 100243e0     U2Core:U2Core.dll
 0002:000003e4       __imp_?createWorkingDir@FileAndDirectoryUtils@U2@@SA?AVQString@@ABV3@H00@Z 100243e4     U2Core:U2Core.dll
 0002:000003e8       __imp_??1FailTask@U2@@UAE@XZ 100243e8     U2Core:U2Core.dll
 0002:000003ec       __imp_??0FailTask@U2@@QAE@ABVQString@@@Z 100243ec     U2Core:U2Core.dll
 0002:000003f0       __imp_?info@Logger@U2@@QAEXABVQString@@@Z 100243f0     U2Core:U2Core.dll
 0002:000003f4       __imp_?trace@Logger@U2@@QAEXABVQString@@@Z 100243f4     U2Core:U2Core.dll
 0002:000003f8       __imp_?qt_metacast@TaskSignalMapper@U2@@UAEPAXPBD@Z 100243f8     U2Core:U2Core.dll
 0002:000003fc       __imp_?qt_metacall@TaskSignalMapper@U2@@UAEHW4Call@QMetaObject@@HPAPAX@Z 100243fc     U2Core:U2Core.dll
 0002:00000400       __imp_?metaObject@TaskSignalMapper@U2@@UBEPBUQMetaObject@@XZ 10024400     U2Core:U2Core.dll
 0002:00000404       __imp_?runScript@ScriptTask@U2@@SA?AVQScriptValue@@PAVQScriptEngine@@ABV?$QMap@VQString@@VQScriptValue@@@@ABVQString@@AAVTaskStateInfo@2@@Z 10024404     U2Core:U2Core.dll
 0002:00000408       __imp_?addListeners@ExternalToolSupportTask@U2@@QAEXABV?$QList@PAVExternalToolListener@U2@@@@@Z 10024408     U2Core:U2Core.dll
 0002:0000040c       __imp_?hasError@Task@U2@@QBE_NXZ 1002440c     U2Core:U2Core.dll
 0002:00000410       __imp_??1TaskStateInfo@U2@@UAE@XZ 10024410     U2Core:U2Core.dll
 0002:00000414       __imp_?setError@TaskStateInfo@U2@@UAEXABVQString@@@Z 10024414     U2Core:U2Core.dll
 0002:00000418       __imp_?getError@TaskStateInfo@U2@@UBE?AVQString@@XZ 10024418     U2Core:U2Core.dll
 0002:0000041c       __imp_??0TaskStateInfo@U2@@QAE@XZ 1002441c     U2Core:U2Core.dll
 0002:00000420       __imp_??0TaskSignalMapper@U2@@QAE@PAVTask@1@@Z 10024420     U2Core:U2Core.dll
 0002:00000424       __imp_?getPathByName@U2DataPath@U2@@QBE?AVQString@@ABV3@@Z 10024424     U2Core:U2Core.dll
 0002:00000428       __imp_??_7SimpleEventCounter@U2@@6B@ 10024428     U2Core:U2Core.dll
 0002:0000042c       __imp_?setReportingSupported@Task@U2@@UAEX_N@Z 1002442c     U2Core:U2Core.dll
 0002:00000430       __imp_?setReportingEnabled@Task@U2@@UAEX_N@Z 10024430     U2Core:U2Core.dll
 0002:00000434       __imp_?setNotificationReport@Task@U2@@UAEX_N@Z 10024434     U2Core:U2Core.dll
 0002:00000438       __imp_?setNoAutoDelete@Task@U2@@UAEX_N@Z 10024438     U2Core:U2Core.dll
 0002:0000043c       __imp_?setListenerForTask@ExternalToolSupportTask@U2@@MAEXPAVExternalToolRunTask@2@H@Z 1002443c     U2Core:U2Core.dll
 0002:00000440       __imp_?setListenerForHelper@ExternalToolSupportTask@U2@@MAEXPAVExternalToolRunTaskHelper@2@H@Z 10024440     U2Core:U2Core.dll
 0002:00000444       __imp_?setLastError@ExternalToolLogParser@U2@@MAEXABVQString@@@Z 10024444     U2Core:U2Core.dll
 0002:00000448       __imp_?setCollectChildrensWarningsFlag@Task@U2@@UAEX_N@Z 10024448     U2Core:U2Core.dll
 0002:0000044c       __imp_?run@Task@U2@@UAEXXZ 1002444c     U2Core:U2Core.dll
 0002:00000450       __imp_?run@ExternalToolRunTask@U2@@UAEXXZ 10024450     U2Core:U2Core.dll
 0002:00000454       __imp_?run@CopyFileTask@U2@@EAEXXZ 10024454     U2Core:U2Core.dll
 0002:00000458       __imp_?getAppSettings@AppContext@U2@@SAPAVAppSettings@2@XZ 10024458     U2Core:U2Core.dll
 0002:0000045c       __imp_?report@Task@U2@@UAE?AW4ReportResult@12@XZ 1002445c     U2Core:U2Core.dll
 0002:00000460       __imp_?qt_metacast@SequentialMultiTask@U2@@UAEPAXPBD@Z 10024460     U2Core:U2Core.dll
 0002:00000464       __imp_?qt_metacast@ExternalToolRunTask@U2@@UAEPAXPBD@Z 10024464     U2Core:U2Core.dll
 0002:00000468       __imp_?qt_metacast@ExternalToolLogParser@U2@@UAEPAXPBD@Z 10024468     U2Core:U2Core.dll
 0002:0000046c       __imp_?qt_metacast@CopyFileTask@U2@@UAEPAXPBD@Z 1002446c     U2Core:U2Core.dll
 0002:00000470       __imp_?qt_metacall@SequentialMultiTask@U2@@UAEHW4Call@QMetaObject@@HPAPAX@Z 10024470     U2Core:U2Core.dll
 0002:00000474       __imp_?qt_metacall@ExternalToolRunTask@U2@@UAEHW4Call@QMetaObject@@HPAPAX@Z 10024474     U2Core:U2Core.dll
 0002:00000478       __imp_?qt_metacall@ExternalToolLogParser@U2@@UAEHW4Call@QMetaObject@@HPAPAX@Z 10024478     U2Core:U2Core.dll
 0002:0000047c       __imp_?qt_metacall@CopyFileTask@U2@@UAEHW4Call@QMetaObject@@HPAPAX@Z 1002447c     U2Core:U2Core.dll
 0002:00000480       __imp_?propagateSubtaskError@Task@U2@@UAE_NXZ 10024480     U2Core:U2Core.dll
 0002:00000484       __imp_?processLine@ExternalToolLogParser@U2@@MAEXABVQString@@@Z 10024484     U2Core:U2Core.dll
 0002:00000488       __imp_?processErrLine@ExternalToolLogParser@U2@@MAEXABVQString@@@Z 10024488     U2Core:U2Core.dll
 0002:0000048c       __imp_?prepare@Task@U2@@UAEXXZ 1002448c     U2Core:U2Core.dll
 0002:00000490       __imp_?prepare@SequentialMultiTask@U2@@UAEXXZ 10024490     U2Core:U2Core.dll
 0002:00000494       __imp_?parseOutput@ExternalToolLogParser@U2@@UAEXABVQString@@@Z 10024494     U2Core:U2Core.dll
 0002:00000498       __imp_?parseErrOutput@ExternalToolLogParser@U2@@UAEXABVQString@@@Z 10024498     U2Core:U2Core.dll
 0002:0000049c       __imp_?onSubTaskFinished@Task@U2@@MAE?AV?$QList@PAVTask@U2@@@@PAV12@@Z 1002449c     U2Core:U2Core.dll
 0002:000004a0       __imp_?onSubTaskFinished@SequentialMultiTask@U2@@UAE?AV?$QList@PAVTask@U2@@@@PAVTask@2@@Z 100244a0     U2Core:U2Core.dll
 0002:000004a4       __imp_?metaObject@SequentialMultiTask@U2@@UBEPBUQMetaObject@@XZ 100244a4     U2Core:U2Core.dll
 0002:000004a8       __imp_?metaObject@ExternalToolRunTask@U2@@UBEPBUQMetaObject@@XZ 100244a8     U2Core:U2Core.dll
 0002:000004ac       __imp_?metaObject@ExternalToolLogParser@U2@@UBEPBUQMetaObject@@XZ 100244ac     U2Core:U2Core.dll
 0002:000004b0       __imp_?metaObject@CopyFileTask@U2@@UBEPBUQMetaObject@@XZ 100244b0     U2Core:U2Core.dll
 0002:000004b4       \177U2Core_NULL_THUNK_DATA 100244b4     U2Core:U2Core.dll
 0002:000004b8       __imp_??1ComboBoxDelegate@U2@@UAE@XZ 100244b8     U2Designer:U2Designer.dll
 0002:000004bc       __imp_??0ComboBoxWithBoolsDelegate@U2@@QAE@PAVQObject@@@Z 100244bc     U2Designer:U2Designer.dll
 0002:000004c0       __imp_??1ComboBoxWithBoolsDelegate@U2@@UAE@XZ 100244c0     U2Designer:U2Designer.dll
 0002:000004c4       __imp_?addDelegate@DelegateEditor@U2@@UAEXPAVPropertyDelegate@2@ABVQString@@@Z 100244c4     U2Designer:U2Designer.dll
 0002:000004c8       __imp_?clone@ComboBoxDelegate@U2@@UAEPAVPropertyDelegate@2@XZ 100244c8     U2Designer:U2Designer.dll
 0002:000004cc       __imp_?clone@ComboBoxWithBoolsDelegate@U2@@UAEPAVPropertyDelegate@2@XZ 100244cc     U2Designer:U2Designer.dll
 0002:000004d0       __imp_?clone@DelegateEditor@U2@@UAEPAVConfigurationEditor@2@XZ 100244d0     U2Designer:U2Designer.dll
 0002:000004d4       __imp_?clone@SpinBoxDelegate@U2@@UAEPAVPropertyDelegate@2@XZ 100244d4     U2Designer:U2Designer.dll
 0002:000004d8       __imp_?clone@URLDelegate@U2@@UAEPAVPropertyDelegate@2@XZ 100244d8     U2Designer:U2Designer.dll
 0002:000004dc       __imp_?commit@DelegateEditor@U2@@UAEXXZ 100244dc     U2Designer:U2Designer.dll
 0002:000004e0       __imp_?createEditor@ComboBoxDelegate@U2@@UBEPAVQWidget@@PAV3@ABVQStyleOptionViewItem@@ABVQModelIndex@@@Z 100244e0     U2Designer:U2Designer.dll
 0002:000004e4       __imp_?createEditor@SpinBoxDelegate@U2@@UBEPAVQWidget@@PAV3@ABVQStyleOptionViewItem@@ABVQModelIndex@@@Z 100244e4     U2Designer:U2Designer.dll
 0002:000004e8       __imp_?createEditor@URLDelegate@U2@@UBEPAVQWidget@@PAV3@ABVQStyleOptionViewItem@@ABVQModelIndex@@@Z 100244e8     U2Designer:U2Designer.dll
 0002:000004ec       __imp_?createWizardWidget@ComboBoxDelegate@U2@@UBEPAVPropertyWidget@2@AAVU2OpStatus@2@PAVQWidget@@@Z 100244ec     U2Designer:U2Designer.dll
 0002:000004f0       __imp_?createWizardWidget@SpinBoxDelegate@U2@@UBEPAVPropertyWidget@2@AAVU2OpStatus@2@PAVQWidget@@@Z 100244f0     U2Designer:U2Designer.dll
 0002:000004f4       __imp_?createWizardWidget@URLDelegate@U2@@UBEPAVPropertyWidget@2@AAVU2OpStatus@2@PAVQWidget@@@Z 100244f4     U2Designer:U2Designer.dll
 0002:000004f8       __imp_?getDelegate@DelegateEditor@U2@@UAEPAVPropertyDelegate@2@ABVQString@@@Z 100244f8     U2Designer:U2Designer.dll
 0002:000004fc       __imp_?getDisplayValue@ComboBoxDelegate@U2@@UBE?AVQVariant@@ABV3@@Z 100244fc     U2Designer:U2Designer.dll
 0002:00000500       __imp_?getDisplayValue@SpinBoxDelegate@U2@@UBE?AVQVariant@@ABV3@@Z 10024500     U2Designer:U2Designer.dll
 0002:00000504       __imp_?getDisplayValue@URLDelegate@U2@@UBE?AVQVariant@@ABV3@@Z 10024504     U2Designer:U2Designer.dll
 0002:00000508       __imp_?getItems@ComboBoxDelegate@U2@@UBEXAAV?$QMap@VQString@@VQVariant@@@@@Z 10024508     U2Designer:U2Designer.dll
 0002:0000050c       __imp_?getItems@SpinBoxDelegate@U2@@UBEXAAV?$QMap@VQString@@VQVariant@@@@@Z 1002450c     U2Designer:U2Designer.dll
 0002:00000510       __imp_?metaObject@ComboBoxDelegate@U2@@UBEPBUQMetaObject@@XZ 10024510     U2Designer:U2Designer.dll
 0002:00000514       __imp_?metaObject@ComboBoxWithBoolsDelegate@U2@@UBEPBUQMetaObject@@XZ 10024514     U2Designer:U2Designer.dll
 0002:00000518       __imp_?metaObject@DelegateEditor@U2@@UBEPBUQMetaObject@@XZ 10024518     U2Designer:U2Designer.dll
 0002:0000051c       __imp_?metaObject@SpinBoxDelegate@U2@@UBEPBUQMetaObject@@XZ 1002451c     U2Designer:U2Designer.dll
 0002:00000520       __imp_?metaObject@URLDelegate@U2@@UBEPBUQMetaObject@@XZ 10024520     U2Designer:U2Designer.dll
 0002:00000524       __imp_?qt_metacall@ComboBoxDelegate@U2@@UAEHW4Call@QMetaObject@@HPAPAX@Z 10024524     U2Designer:U2Designer.dll
 0002:00000528       __imp_?qt_metacall@ComboBoxWithBoolsDelegate@U2@@UAEHW4Call@QMetaObject@@HPAPAX@Z 10024528     U2Designer:U2Designer.dll
 0002:0000052c       __imp_?qt_metacall@DelegateEditor@U2@@UAEHW4Call@QMetaObject@@HPAPAX@Z 1002452c     U2Designer:U2Designer.dll
 0002:00000530       __imp_?qt_metacall@SpinBoxDelegate@U2@@UAEHW4Call@QMetaObject@@HPAPAX@Z 10024530     U2Designer:U2Designer.dll
 0002:00000534       __imp_?qt_metacall@URLDelegate@U2@@UAEHW4Call@QMetaObject@@HPAPAX@Z 10024534     U2Designer:U2Designer.dll
 0002:00000538       __imp_?qt_metacast@ComboBoxDelegate@U2@@UAEPAXPBD@Z 10024538     U2Designer:U2Designer.dll
 0002:0000053c       __imp_?qt_metacast@ComboBoxWithBoolsDelegate@U2@@UAEPAXPBD@Z 1002453c     U2Designer:U2Designer.dll
 0002:00000540       __imp_?qt_metacast@DelegateEditor@U2@@UAEPAXPBD@Z 10024540     U2Designer:U2Designer.dll
 0002:00000544       __imp_?qt_metacast@SpinBoxDelegate@U2@@UAEPAXPBD@Z 10024544     U2Designer:U2Designer.dll
 0002:00000548       __imp_?qt_metacast@URLDelegate@U2@@UAEPAXPBD@Z 10024548     U2Designer:U2Designer.dll
 0002:0000054c       __imp_?removeDelegate@DelegateEditor@U2@@UAEPAVPropertyDelegate@2@ABVQString@@@Z 1002454c     U2Designer:U2Designer.dll
 0002:00000550       __imp_?setEditorData@ComboBoxDelegate@U2@@UBEXPAVQWidget@@ABVQModelIndex@@@Z 10024550     U2Designer:U2Designer.dll
 0002:00000554       __imp_?setEditorData@SpinBoxDelegate@U2@@UBEXPAVQWidget@@ABVQModelIndex@@@Z 10024554     U2Designer:U2Designer.dll
 0002:00000558       __imp_?setEditorData@URLDelegate@U2@@UBEXPAVQWidget@@ABVQModelIndex@@@Z 10024558     U2Designer:U2Designer.dll
 0002:0000055c       __imp_?setModelData@ComboBoxDelegate@U2@@UBEXPAVQWidget@@PAVQAbstractItemModel@@ABVQModelIndex@@@Z 1002455c     U2Designer:U2Designer.dll
 0002:00000560       __imp_?setModelData@SpinBoxDelegate@U2@@UBEXPAVQWidget@@PAVQAbstractItemModel@@ABVQModelIndex@@@Z 10024560     U2Designer:U2Designer.dll
 0002:00000564       __imp_?setModelData@URLDelegate@U2@@UBEXPAVQWidget@@PAVQAbstractItemModel@@ABVQModelIndex@@@Z 10024564     U2Designer:U2Designer.dll
 0002:00000568       __imp_?type@URLDelegate@U2@@UBE?AW4Type@PropertyDelegate@2@XZ 10024568     U2Designer:U2Designer.dll
 0002:0000056c       __imp_?updateDelegate@DelegateEditor@U2@@UAEXABVQString@@@Z 1002456c     U2Designer:U2Designer.dll
 0002:00000570       __imp_?updateDelegates@DelegateEditor@U2@@UAEXXZ 10024570     U2Designer:U2Designer.dll
 0002:00000574       __imp_??0URLDelegate@U2@@QAE@ABVDelegateTags@1@ABVQString@@_N22PAVQObject@@22@Z 10024574     U2Designer:U2Designer.dll
 0002:00000578       __imp_??1DelegateEditor@U2@@UAE@XZ 10024578     U2Designer:U2Designer.dll
 0002:0000057c       __imp_??0URLDelegate@U2@@QAE@ABVQString@@0ABV?$QFlags@W4Option@URLDelegate@U2@@@@PAVQObject@@0@Z 1002457c     U2Designer:U2Designer.dll
 0002:00000580       __imp_??0URLDelegate@U2@@QAE@ABVQString@@0_N11PAVQObject@@011@Z 10024580     U2Designer:U2Designer.dll
 0002:00000584       __imp_??1URLDelegate@U2@@UAE@XZ 10024584     U2Designer:U2Designer.dll
 0002:00000588       __imp_??0SpinBoxDelegate@U2@@QAE@ABV?$QMap@VQString@@VQVariant@@@@PAVQObject@@@Z 10024588     U2Designer:U2Designer.dll
 0002:0000058c       __imp_??1SpinBoxDelegate@U2@@UAE@XZ 1002458c     U2Designer:U2Designer.dll
 0002:00000590       __imp_??0ComboBoxDelegate@U2@@QAE@ABV?$QMap@VQString@@VQVariant@@@@PAVQObject@@@Z 10024590     U2Designer:U2Designer.dll
 0002:00000594       __imp_??0DelegateEditor@U2@@QAE@ABV?$QMap@VQString@@PAVPropertyDelegate@U2@@@@@Z 10024594     U2Designer:U2Designer.dll
 0002:00000598       \177U2Designer_NULL_THUNK_DATA 10024598     U2Designer:U2Designer.dll
 0002:0000059c       __imp_?prepareDocumentsFileFilter@DialogUtils@U2@@SA?AVQString@@ABV3@_NABVQStringList@@@Z 1002459c     U2Gui:U2Gui.dll
 0002:000005a0       \177U2Gui_NULL_THUNK_DATA  100245a0     U2Gui:U2Gui.dll
 0002:000005a4       __imp_??0PrompterBaseImpl@U2@@QAE@PAVActor@Workflow@1@@Z 100245a4     U2Lang:U2Lang.dll
 0002:000005a8       __imp_?getURL@PrompterBaseImpl@U2@@QAE?AVQString@@ABV3@PA_N00@Z 100245a8     U2Lang:U2Lang.dll
 0002:000005ac       __imp_?getParameter@PrompterBaseImpl@U2@@QAE?AVQVariant@@ABVQString@@@Z 100245ac     U2Lang:U2Lang.dll
 0002:000005b0       __imp_?getHyperlink@PrompterBaseImpl@U2@@SA?AVQString@@ABV3@0@Z 100245b0     U2Lang:U2Lang.dll
 0002:000005b4       __imp_??1PrompterBaseImpl@U2@@UAE@XZ 100245b4     U2Lang:U2Lang.dll
 0002:000005b8       __imp_?metaObject@PrompterBaseImpl@U2@@UBEPBUQMetaObject@@XZ 100245b8     U2Lang:U2Lang.dll
 0002:000005bc       __imp_?qt_metacall@PrompterBaseImpl@U2@@UAEHW4Call@QMetaObject@@HPAPAX@Z 100245bc     U2Lang:U2Lang.dll
 0002:000005c0       __imp_?qt_metacast@PrompterBaseImpl@U2@@UAEPAXPBD@Z 100245c0     U2Lang:U2Lang.dll
 0002:000005c4       __imp_?sl_actorModified@PrompterBaseImpl@U2@@MAEXXZ 100245c4     U2Lang:U2Lang.dll
 0002:000005c8       __imp_?update@PrompterBaseImpl@U2@@UAEXABV?$QMap@VQString@@VQVariant@@@@@Z 100245c8     U2Lang:U2Lang.dll
 0002:000005cc       __imp_??0WorkflowNotification@U2@@QAE@ABVQString@@00@Z 100245cc     U2Lang:U2Lang.dll
 0002:000005d0       __imp_??1WorkflowNotification@U2@@QAE@XZ 100245d0     U2Lang:U2Lang.dll
 0002:000005d4       __imp_?getOutputPorts@Actor@Workflow@U2@@QBE?AV?$QList@PAVPort@Workflow@U2@@@@XZ 100245d4     U2Lang:U2Lang.dll
 0002:000005d8       __imp_?getId@Actor@Workflow@U2@@QBE?AVQString@@XZ 100245d8     U2Lang:U2Lang.dll
 0002:000005dc       __imp_?U2_ERROR@WorkflowNotification@U2@@2VQString@@B 100245dc     U2Lang:U2Lang.dll
 0002:000005e0       __imp_??1Descriptor@U2@@UAE@XZ 100245e0     U2Lang:U2Lang.dll
 0002:000005e4       __imp_?getId@Descriptor@U2@@QBE?AVQString@@XZ 100245e4     U2Lang:U2Lang.dll
 0002:000005e8       __imp_??0Descriptor@U2@@QAE@ABV01@@Z 100245e8     U2Lang:U2Lang.dll
 0002:000005ec       __imp_?URL_SLOT@BaseSlots@Workflow@U2@@SA?BVDescriptor@3@XZ 100245ec     U2Lang:U2Lang.dll
 0002:000005f0       __imp_??0Dataset@U2@@QAE@ABV01@@Z 100245f0     U2Lang:U2Lang.dll
 0002:000005f4       __imp_??1Dataset@U2@@QAE@XZ 100245f4     U2Lang:U2Lang.dll
 0002:000005f8       __imp_?updateDelegateTags@ValuesRelation@U2@@UBEXABVQVariant@@PAVDelegateTags@2@@Z 100245f8     U2Lang:U2Lang.dll
 0002:000005fc       __imp_?getType@ValuesRelation@U2@@UBE?AW4RelationType@2@XZ 100245fc     U2Lang:U2Lang.dll
 0002:00000600       __imp_??0ValuesRelation@U2@@QAE@ABV01@@Z 10024600     U2Lang:U2Lang.dll
 0002:00000604       __imp_??1ValuesRelation@U2@@UAE@XZ 10024604     U2Lang:U2Lang.dll
 0002:00000608       __imp_??0ValuesRelation@U2@@QAE@ABVQString@@ABV?$QMap@VQString@@VQVariant@@@@@Z 10024608     U2Lang:U2Lang.dll
 0002:0000060c       __imp_?getInputPorts@Actor@Workflow@U2@@QBE?AV?$QList@PAVPort@Workflow@U2@@@@XZ 1002460c     U2Lang:U2Lang.dll
 0002:00000610       __imp_??0WorkflowNotification@U2@@QAE@ABV01@@Z 10024610     U2Lang:U2Lang.dll
 0002:00000614       __imp_?valueChangingRelation@AttributeRelation@U2@@UBE_NXZ 10024614     U2Lang:U2Lang.dll
 0002:00000618       __imp_?staticMetaObject@BaseWorker@LocalWorkflow@U2@@2UQMetaObject@@B 10024618     U2Lang:U2Lang.dll
 0002:0000061c       __imp_?qt_metacall@BaseWorker@LocalWorkflow@U2@@UAEHW4Call@QMetaObject@@HPAPAX@Z 1002461c     U2Lang:U2Lang.dll
 0002:00000620       __imp_?qt_metacast@BaseWorker@LocalWorkflow@U2@@UAEPAXPBD@Z 10024620     U2Lang:U2Lang.dll
 0002:00000624       __imp_?staticMetaObject@PrompterBaseImpl@U2@@2UQMetaObject@@B 10024624     U2Lang:U2Lang.dll
 0002:00000628       __imp_?FORMAT@DelegateTags@U2@@2VQString@@B 10024628     U2Lang:U2Lang.dll
 0002:0000062c       __imp_?FILTER@DelegateTags@U2@@2VQString@@B 1002462c     U2Lang:U2Lang.dll
 0002:00000630       __imp_?PLACEHOLDER_TEXT@DelegateTags@U2@@2VQString@@B 10024630     U2Lang:U2Lang.dll
 0002:00000634       __imp_?validate@PortValidator@Workflow@U2@@UBE_NPBVConfiguration@3@AAV?$QList@VWorkflowNotification@U2@@@@@Z 10024634     U2Lang:U2Lang.dll
 0002:00000638       __imp_?validate@PairedReadsPortValidator@Workflow@U2@@UBE_NPBVIntegralBusPort@23@AAV?$QList@VWorkflowNotification@U2@@@@@Z 10024638     U2Lang:U2Lang.dll
 0002:0000063c       __imp_?isSlotEnabled@SlotRelationDescriptor@U2@@UBE_NABVQVariant@@@Z 1002463c     U2Lang:U2Lang.dll
 0002:00000640       __imp_?clone@SlotRelationDescriptor@U2@@UBEPAV12@XZ 10024640     U2Lang:U2Lang.dll
 0002:00000644       __imp_??1PairedReadsPortValidator@Workflow@U2@@UAE@XZ 10024644     U2Lang:U2Lang.dll
 0002:00000648       __imp_??0PairedReadsPortValidator@Workflow@U2@@QAE@ABVQString@@0@Z 10024648     U2Lang:U2Lang.dll
 0002:0000064c       __imp_??1DelegateTags@U2@@UAE@XZ 1002464c     U2Lang:U2Lang.dll
 0002:00000650       __imp_?set@DelegateTags@U2@@QAEXABVQString@@ABVQVariant@@@Z 10024650     U2Lang:U2Lang.dll
 0002:00000654       __imp_??0DelegateTags@U2@@QAE@PAVQObject@@@Z 10024654     U2Lang:U2Lang.dll
 0002:00000658       __imp_?addSlotRelation@Attribute@U2@@QAEXPAVSlotRelationDescriptor@2@@Z 10024658     U2Lang:U2Lang.dll
 0002:0000065c       __imp_??0Attribute@U2@@QAE@ABVDescriptor@1@V?$QExplicitlySharedDataPointer@VDataType@U2@@@@V?$QFlags@W4Flag@Attribute@U2@@@@ABVQVariant@@@Z 1002465c     U2Lang:U2Lang.dll
 0002:00000660       __imp_??1SlotRelationDescriptor@U2@@UAE@XZ 10024660     U2Lang:U2Lang.dll
 0002:00000664       __imp_??0SlotRelationDescriptor@U2@@QAE@ABVQString@@0ABV?$QList@VQVariant@@@@@Z 10024664     U2Lang:U2Lang.dll
 0002:00000668       __imp_?U2_INFO@WorkflowNotification@U2@@2VQString@@B 10024668     U2Lang:U2Lang.dll
 0002:0000066c       __imp_?addInfo@WorkflowMonitor@Workflow@U2@@QAEXABVQString@@00@Z 1002466c     U2Lang:U2Lang.dll
 0002:00000670       __imp_?getMetadataId@Message@Workflow@U2@@QBEHXZ 10024670     U2Lang:U2Lang.dll
 0002:00000674       __imp_?getData@Message@Workflow@U2@@QBE?AVQVariant@@XZ 10024674     U2Lang:U2Lang.dll
 0002:00000678       __imp_?workingDir@WorkflowContext@Workflow@U2@@QBE?AVQString@@XZ 10024678     U2Lang:U2Lang.dll
 0002:0000067c       __imp_?get@MessageMetadataStorage@U2@@QBE?AVMessageMetadata@2@H@Z 1002467c     U2Lang:U2Lang.dll
 0002:00000680       __imp_?getFileUrl@MessageMetadata@U2@@QBEABVQString@@XZ 10024680     U2Lang:U2Lang.dll
 0002:00000684       __imp_?getProducersOrUnset@PrompterBaseImpl@U2@@QAE?AVQString@@ABV3@0@Z 10024684     U2Lang:U2Lang.dll
 0002:00000688       __imp_?ID@LocalDomainFactory@LocalWorkflow@U2@@2VQString@@B 10024688     U2Lang:U2Lang.dll
 0002:0000068c       __imp_??_7ActorValidator@Workflow@U2@@6B@ 1002468c     U2Lang:U2Lang.dll
 0002:00000690       __imp_??_7ConfigurationValidator@U2@@6B@ 10024690     U2Lang:U2Lang.dll
 0002:00000694       __imp_?valueChangingRelation@VisibilityRelation@U2@@UBE_NXZ 10024694     U2Lang:U2Lang.dll
 0002:00000698       __imp_?validate@Attribute@U2@@UAE_NAAV?$QList@VWorkflowNotification@U2@@@@@Z 10024698     U2Lang:U2Lang.dll
 0002:0000069c       __imp_?validate@ActorValidator@Workflow@U2@@UBE_NPBVConfiguration@3@AAV?$QList@VWorkflowNotification@U2@@@@@Z 1002469c     U2Lang:U2Lang.dll
 0002:000006a0       __imp_?updateDelegateTags@AttributeRelation@U2@@UBEXABVQVariant@@PAVDelegateTags@2@@Z 100246a0     U2Lang:U2Lang.dll
 0002:000006a4       __imp_?updateActorIds@Attribute@U2@@UAEXABV?$QMap@VQString@@V1@@@@Z 100246a4     U2Lang:U2Lang.dll
 0002:000006a8       __imp_?update@PropertyDelegate@U2@@UAEXXZ 100246a8     U2Lang:U2Lang.dll
 0002:000006ac       __imp_?unregisterEntry@?$IdRegistry@VDomainFactory@Workflow@U2@@@U2@@UAEPAVDomainFactory@Workflow@2@ABVQString@@@Z 100246ac     U2Lang:U2Lang.dll
 0002:000006b0       __imp_?type@PropertyDelegate@U2@@UBE?AW4Type@12@XZ 100246b0     U2Lang:U2Lang.dll
 0002:000006b4       __imp_?setVisibleSlot@PortDescriptor@Workflow@U2@@UAEXABVQString@@_N@Z 100246b4     U2Lang:U2Lang.dll
 0002:000006b8       __imp_?setDocumentation@ActorPrototype@Workflow@U2@@UAEXABVQString@@@Z 100246b8     U2Lang:U2Lang.dll
 0002:000006bc       __imp_?setDisplayName@ActorPrototype@Workflow@U2@@UAEXABVQString@@@Z 100246bc     U2Lang:U2Lang.dll
 0002:000006c0       __imp_?setAttributeValue@Attribute@U2@@UAEXABVQVariant@@@Z 100246c0     U2Lang:U2Lang.dll
 0002:000006c4       __imp_?registerEntry@?$IdRegistry@VDomainFactory@Workflow@U2@@@U2@@UAE_NPAVDomainFactory@Workflow@2@@Z 100246c4     U2Lang:U2Lang.dll
 0002:000006c8       __imp_?qt_metacast@ActorPrototype@Workflow@U2@@UAEPAXPBD@Z 100246c8     U2Lang:U2Lang.dll
 0002:000006cc       __imp_?qt_metacall@ActorPrototype@Workflow@U2@@UAEHW4Call@QMetaObject@@HPAPAX@Z 100246cc     U2Lang:U2Lang.dll
 0002:000006d0       __imp_?metaObject@ActorPrototype@Workflow@U2@@UBEPBUQMetaObject@@XZ 100246d0     U2Lang:U2Lang.dll
 0002:000006d4       __imp_?kind@MapDataType@U2@@UBE?AW4Kind@DataType@2@XZ 100246d4     U2Lang:U2Lang.dll
 0002:000006d8       __imp_?isEmpty@ConfigurationEditor@U2@@UBE_NXZ 100246d8     U2Lang:U2Lang.dll
 0002:000006dc       __imp_?isEmpty@Attribute@U2@@UBE_NXZ 100246dc     U2Lang:U2Lang.dll
 0002:000006e0       __imp_?isDefaultValue@Attribute@U2@@UBE_NXZ 100246e0     U2Lang:U2Lang.dll
 0002:000006e4       __imp_?isAcceptableDrop@ActorPrototype@Workflow@U2@@UBE_NPBVQMimeData@@PAV?$QMap@VQString@@VQVariant@@@@@Z 100246e4     U2Lang:U2Lang.dll
 0002:000006e8       __imp_?getWidget@ConfigurationEditor@U2@@UAEPAVQWidget@@XZ 100246e8     U2Lang:U2Lang.dll
 0002:000006ec       __imp_?getType@VisibilityRelation@U2@@UBE?AW4RelationType@2@XZ 100246ec     U2Lang:U2Lang.dll
 0002:000006f0       __imp_?getType@PortDescriptor@Workflow@U2@@UBE?AV?$QExplicitlySharedDataPointer@VDataType@U2@@@@XZ 100246f0     U2Lang:U2Lang.dll
 0002:000006f4       __imp_?getItems@PropertyDelegate@U2@@UBEXAAV?$QMap@VQString@@VQVariant@@@@@Z 100246f4     U2Lang:U2Lang.dll
 0002:000006f8       __imp_?getGroup@Attribute@U2@@UAE?AW4AttributeGroup@2@XZ 100246f8     U2Lang:U2Lang.dll
 0002:000006fc       __imp_?getDefaultPureValue@Attribute@U2@@UBEABVQVariant@@XZ 100246fc     U2Lang:U2Lang.dll
 0002:00000700       __imp_?getDatatypesMap@MapDataType@U2@@UBE?AV?$QMap@VDescriptor@U2@@V?$QExplicitlySharedDataPointer@VDataType@U2@@@@@@XZ 10024700     U2Lang:U2Lang.dll
 0002:00000704       __imp_?getDatatypeByDescriptor@MapDataType@U2@@UBE?AV?$QExplicitlySharedDataPointer@VDataType@U2@@@@ABVDescriptor@2@@Z 10024704     U2Lang:U2Lang.dll
 0002:00000708       __imp_?getById@?$IdRegistry@VDomainFactory@Workflow@U2@@@U2@@UAEPAVDomainFactory@Workflow@2@ABVQString@@@Z 10024708     U2Lang:U2Lang.dll
 0002:0000070c       __imp_?getAttributePureValue@Attribute@U2@@UBEABVQVariant@@XZ 1002470c     U2Lang:U2Lang.dll
 0002:00000710       __imp_?getAllIds@?$IdRegistry@VDomainFactory@Workflow@U2@@@U2@@UBE?AV?$QList@VQString@@@@XZ 10024710     U2Lang:U2Lang.dll
 0002:00000714       __imp_?getAllEntries@?$IdRegistry@VDomainFactory@Workflow@U2@@@U2@@UBE?AV?$QList@PAVDomainFactory@Workflow@U2@@@@XZ 10024714     U2Lang:U2Lang.dll
 0002:00000718       __imp_?getAllDescriptors@MapDataType@U2@@UBE?AV?$QList@VDescriptor@U2@@@@XZ 10024718     U2Lang:U2Lang.dll
 0002:0000071c       __imp_?getAffectResult@VisibilityRelation@U2@@UBE?AVQVariant@@ABV3@0PAVDelegateTags@2@1@Z 1002471c     U2Lang:U2Lang.dll
 0002:00000720       __imp_?destroy@DomainFactory@Workflow@U2@@UAEXPAVScheduler@23@PAVSchema@23@@Z 10024720     U2Lang:U2Lang.dll
 0002:00000724       __imp_?createScheduler@DomainFactory@Workflow@U2@@UAEPAVScheduler@23@PAVSchema@23@@Z 10024724     U2Lang:U2Lang.dll
 0002:00000728       __imp_?createPort@IntegralBusActorPrototype@Workflow@U2@@UAEPAVPort@23@ABVPortDescriptor@23@PAVActor@23@@Z 10024728     U2Lang:U2Lang.dll
 0002:0000072c       __imp_?createInstance@ActorPrototype@Workflow@U2@@UAEPAVActor@23@ABVQString@@PAVAttributeScript@3@ABV?$QMap@VQString@@VQVariant@@@@@Z 1002472c     U2Lang:U2Lang.dll
 0002:00000730       __imp_?createConnection@DomainFactory@Workflow@U2@@UAEPAVCommunicationChannel@23@PAVLink@23@@Z 10024730     U2Lang:U2Lang.dll
 0002:00000734       __imp_?clone@VisibilityRelation@U2@@UBEPAV12@XZ 10024734     U2Lang:U2Lang.dll
 0002:00000738       __imp_?clone@Attribute@U2@@UAEPAV12@XZ 10024738     U2Lang:U2Lang.dll
 0002:0000073c       __imp_??1DomainFactory@Workflow@U2@@UAE@XZ 1002473c     U2Lang:U2Lang.dll
 0002:00000740       __imp_??0DomainFactory@Workflow@U2@@QAE@ABVQString@@@Z 10024740     U2Lang:U2Lang.dll
 0002:00000744       __imp_?getInstance@WorkflowEnv@Workflow@U2@@KAPAV123@XZ 10024744     U2Lang:U2Lang.dll
 0002:00000748       __imp_?URL_DATASETS_TYPE@BaseTypes@U2@@SA?AV?$QExplicitlySharedDataPointer@VDataType@U2@@@@XZ 10024748     U2Lang:U2Lang.dll
 0002:0000074c       __imp_?NUM_TYPE@BaseTypes@U2@@SA?AV?$QExplicitlySharedDataPointer@VDataType@U2@@@@XZ 1002474c     U2Lang:U2Lang.dll
 0002:00000750       __imp_?BOOL_TYPE@BaseTypes@U2@@SA?AV?$QExplicitlySharedDataPointer@VDataType@U2@@@@XZ 10024750     U2Lang:U2Lang.dll
 0002:00000754       __imp_?STRING_TYPE@BaseTypes@U2@@SA?AV?$QExplicitlySharedDataPointer@VDataType@U2@@@@XZ 10024754     U2Lang:U2Lang.dll
 0002:00000758       __imp_?unregisterProto@ActorPrototypeRegistry@Workflow@U2@@QAEPAVActorPrototype@23@ABVQString@@@Z 10024758     U2Lang:U2Lang.dll
 0002:0000075c       __imp_?registerProto@ActorPrototypeRegistry@Workflow@U2@@QAE_NABVDescriptor@3@PAVActorPrototype@23@@Z 1002475c     U2Lang:U2Lang.dll
 0002:00000760       __imp_?addExternalTool@ActorPrototype@Workflow@U2@@QAEXABVQString@@0@Z 10024760     U2Lang:U2Lang.dll
 0002:00000764       __imp_?setPrompter@ActorPrototype@Workflow@U2@@QAEXPAVPrompter@23@@Z 10024764     U2Lang:U2Lang.dll
 0002:00000768       __imp_?setValidator@ActorPrototype@Workflow@U2@@QAEXPAVConfigurationValidator@3@@Z 10024768     U2Lang:U2Lang.dll
 0002:0000076c       __imp_?setEditor@ActorPrototype@Workflow@U2@@QAEXPAVConfigurationEditor@3@@Z 1002476c     U2Lang:U2Lang.dll
 0002:00000770       __imp_??1ActorPrototype@Workflow@U2@@UAE@XZ 10024770     U2Lang:U2Lang.dll
 0002:00000774       __imp_??0ActorPrototype@Workflow@U2@@QAE@ABVDescriptor@2@ABV?$QList@PAVPortDescriptor@Workflow@U2@@@@ABV?$QList@PAVAttribute@U2@@@@@Z 10024774     U2Lang:U2Lang.dll
 0002:00000778       __imp_??1PortDescriptor@Workflow@U2@@UAE@XZ 10024778     U2Lang:U2Lang.dll
 0002:0000077c       __imp_??0PortDescriptor@Workflow@U2@@QAE@ABVDescriptor@2@V?$QExplicitlySharedDataPointer@VDataType@U2@@@@_N2I@Z 1002477c     U2Lang:U2Lang.dll
 0002:00000780       __imp_??1PropertyDelegate@U2@@UAE@XZ 10024780     U2Lang:U2Lang.dll
 0002:00000784       __imp_?addRelation@Attribute@U2@@QAEXPBVAttributeRelation@2@@Z 10024784     U2Lang:U2Lang.dll
 0002:00000788       __imp_??1Attribute@U2@@UAE@XZ 10024788     U2Lang:U2Lang.dll
 0002:0000078c       __imp_??0Attribute@U2@@QAE@ABVDescriptor@1@V?$QExplicitlySharedDataPointer@VDataType@U2@@@@_NABVQVariant@@@Z 1002478c     U2Lang:U2Lang.dll
 0002:00000790       __imp_??1MapDataType@U2@@UAE@XZ 10024790     U2Lang:U2Lang.dll
 0002:00000794       __imp_??0MapDataType@U2@@QAE@ABVDescriptor@1@ABV?$QMap@VDescriptor@U2@@V?$QExplicitlySharedDataPointer@VDataType@U2@@@@@@@Z 10024794     U2Lang:U2Lang.dll
 0002:00000798       __imp_??0Descriptor@U2@@QAE@ABVQString@@@Z 10024798     U2Lang:U2Lang.dll
 0002:0000079c       __imp_??0Descriptor@U2@@QAE@ABVQString@@00@Z 1002479c     U2Lang:U2Lang.dll
 0002:000007a0       __imp_??1VisibilityRelation@U2@@UAE@XZ 100247a0     U2Lang:U2Lang.dll
 0002:000007a4       __imp_??0VisibilityRelation@U2@@QAE@ABVQString@@ABVQVariant@@_N@Z 100247a4     U2Lang:U2Lang.dll
 0002:000007a8       __imp_?setDone@BaseWorker@LocalWorkflow@U2@@UAEXXZ 100247a8     U2Lang:U2Lang.dll
 0002:000007ac       __imp_?setDocumentation@Descriptor@U2@@UAEXABVQString@@@Z 100247ac     U2Lang:U2Lang.dll
 0002:000007b0       __imp_?setDisplayName@Descriptor@U2@@UAEXABVQString@@@Z 100247b0     U2Lang:U2Lang.dll
 0002:000007b4       __imp_?isReady@BaseWorker@LocalWorkflow@U2@@UBE_NXZ 100247b4     U2Lang:U2Lang.dll
 0002:000007b8       __imp_?isDone@BaseWorker@LocalWorkflow@U2@@UBE_NXZ 100247b8     U2Lang:U2Lang.dll
 0002:000007bc       __imp_?getOutputFiles@BaseWorker@LocalWorkflow@U2@@UAE?AVQStringList@@XZ 100247bc     U2Lang:U2Lang.dll
 0002:000007c0       __imp_?getMessageAndSetupScriptValues@BaseWorker@LocalWorkflow@U2@@UAE?AVMessage@Workflow@3@PAVCommunicationChannel@53@@Z 100247c0     U2Lang:U2Lang.dll
 0002:000007c4       __imp_?getCommunication@BaseWorker@LocalWorkflow@U2@@UAEPAVCommunicationChannel@Workflow@3@ABVQString@@@Z 100247c4     U2Lang:U2Lang.dll
 0002:000007c8       __imp_?getActorId@BaseWorker@LocalWorkflow@U2@@UBE?AVQString@@XZ 100247c8     U2Lang:U2Lang.dll
 0002:000007cc       __imp_?canTaskBeCanceled@BaseWorker@LocalWorkflow@U2@@MBE_NPAVTask@3@@Z 100247cc     U2Lang:U2Lang.dll
 0002:000007d0       __imp_?addCommunication@BaseWorker@LocalWorkflow@U2@@UAE_NABVQString@@PAVCommunicationChannel@Workflow@3@@Z 100247d0     U2Lang:U2Lang.dll
 0002:000007d4       __imp_?createLogListeners@BaseWorker@LocalWorkflow@U2@@QBE?AV?$QList@PAVExternalToolListener@U2@@@@H@Z 100247d4     U2Lang:U2Lang.dll
 0002:000007d8       __imp_??1BaseWorker@LocalWorkflow@U2@@UAE@XZ 100247d8     U2Lang:U2Lang.dll
 0002:000007dc       __imp_??0BaseWorker@LocalWorkflow@U2@@QAE@PAVActor@Workflow@2@_N@Z 100247dc     U2Lang:U2Lang.dll
 0002:000007e0       __imp_?getBusType@IntegralBus@Workflow@U2@@QBE?AV?$QExplicitlySharedDataPointer@VDataType@U2@@@@XZ 100247e0     U2Lang:U2Lang.dll
 0002:000007e4       __imp_?isOutUrlAttribute@RFSUtils@U2@@SA_NPAVAttribute@2@PAVActor@Workflow@2@AA_N@Z 100247e4     U2Lang:U2Lang.dll
 0002:000007e8       __imp_?addOutputFile@WorkflowMonitor@Workflow@U2@@QAEXABVQString@@0_N@Z 100247e8     U2Lang:U2Lang.dll
 0002:000007ec       __imp_??1Message@Workflow@U2@@QAE@XZ 100247ec     U2Lang:U2Lang.dll
 0002:000007f0       __imp_??0Message@Workflow@U2@@QAE@V?$QExplicitlySharedDataPointer@VDataType@U2@@@@ABVQVariant@@H@Z 100247f0     U2Lang:U2Lang.dll
 0002:000007f4       __imp_?getScriptVars@AttributeScript@U2@@QBEABV?$QMap@VDescriptor@U2@@VQVariant@@@@XZ 100247f4     U2Lang:U2Lang.dll
 0002:000007f8       __imp_?getScriptText@AttributeScript@U2@@QBEABVQString@@XZ 100247f8     U2Lang:U2Lang.dll
 0002:000007fc       __imp_?isEmpty@AttributeScript@U2@@QBE_NXZ 100247fc     U2Lang:U2Lang.dll
 0002:00000800       __imp_??1WorkflowScriptEngine@U2@@UAE@XZ 10024800     U2Lang:U2Lang.dll
 0002:00000804       __imp_??0WorkflowScriptEngine@U2@@QAE@PAVWorkflowContext@Workflow@1@@Z 10024804     U2Lang:U2Lang.dll
 0002:00000808       __imp_?getMetadataStorage@WorkflowContext@Workflow@U2@@QAEAAVMessageMetadataStorage@3@XZ 10024808     U2Lang:U2Lang.dll
 0002:0000080c       __imp_?absolutePath@WorkflowContext@Workflow@U2@@QBE?AVQString@@ABV4@@Z 1002480c     U2Lang:U2Lang.dll
 0002:00000810       __imp_?getMonitor@WorkflowContext@Workflow@U2@@QAEPAVWorkflowMonitor@23@XZ 10024810     U2Lang:U2Lang.dll
 0002:00000814       __imp_?put@MessageMetadataStorage@U2@@QAEXABVMessageMetadata@2@@Z 10024814     U2Lang:U2Lang.dll
 0002:00000818       __imp_??4MessageMetadata@U2@@QAEAAV01@ABV01@@Z 10024818     U2Lang:U2Lang.dll
 0002:0000081c       __imp_??1MessageMetadata@U2@@QAE@XZ 1002481c     U2Lang:U2Lang.dll
 0002:00000820       __imp_?getId@MessageMetadata@U2@@QBEHXZ 10024820     U2Lang:U2Lang.dll
 0002:00000824       __imp_??0MessageMetadata@U2@@QAE@ABVQString@@0@Z 10024824     U2Lang:U2Lang.dll
 0002:00000828       __imp_??0MessageMetadata@U2@@QAE@ABVQString@@@Z 10024828     U2Lang:U2Lang.dll
 0002:0000082c       __imp_??0MessageMetadata@U2@@QAE@XZ 1002482c     U2Lang:U2Lang.dll
 0002:00000830       __imp_?initEngine@WorkflowScriptLibrary@U2@@SAXPAVWorkflowScriptEngine@2@@Z 10024830     U2Lang:U2Lang.dll
 0002:00000834       __imp_?getUrls@Dataset@U2@@QBE?AV?$QList@PAVURLContainer@U2@@@@XZ 10024834     U2Lang:U2Lang.dll
 0002:00000838       __imp_?setPortValidator@ActorPrototype@Workflow@U2@@QAEXABVQString@@PAVConfigurationValidator@3@@Z 10024838     U2Lang:U2Lang.dll
 0002:0000083c       \177U2Lang_NULL_THUNK_DATA 1002483c     U2Lang:U2Lang.dll
 0002:00000840       __imp_?WORKFLOW_CLASSIFY_TOOL_ID@NgsReadsClassificationPlugin@U2@@2VQString@@B 10024840     ngs_reads_classification:ngs_reads_classification.dll
 0002:00000844       __imp_?MINIKRAKEN_4_GB_ITEM_ID@NgsReadsClassificationPlugin@U2@@2VQString@@B 10024844     ngs_reads_classification:ngs_reads_classification.dll
 0002:00000848       __imp_?MINIKRAKEN_4_GB_DATA_ID@NgsReadsClassificationPlugin@U2@@2VQString@@B 10024848     ngs_reads_classification:ngs_reads_classification.dll
 0002:0000084c       __imp_?update@DatabaseDelegate@LocalWorkflow@U2@@UAEXXZ 1002484c     ngs_reads_classification:ngs_reads_classification.dll
 0002:00000850       __imp_??1DatabaseDelegate@LocalWorkflow@U2@@UAE@XZ 10024850     ngs_reads_classification:ngs_reads_classification.dll
 0002:00000854       __imp_??0DatabaseDelegate@LocalWorkflow@U2@@QAE@ABVQString@@0000_N@Z 10024854     ngs_reads_classification:ngs_reads_classification.dll
 0002:00000858       __imp_?TAXONOMY_CLASSIFICATION_TYPE@TaxonomySupport@LocalWorkflow@U2@@SA?AV?$QExplicitlySharedDataPointer@VDataType@U2@@@@XZ 10024858     ngs_reads_classification:ngs_reads_classification.dll
 0002:0000085c       __imp_?TAXONOMY_CLASSIFICATION_SLOT@TaxonomySupport@LocalWorkflow@U2@@SA?BVDescriptor@3@XZ 1002485c     ngs_reads_classification:ngs_reads_classification.dll
 0002:00000860       __imp_?CLASSIFICATION_SUFFIX@NgsReadsClassificationUtils@U2@@2VQString@@B 10024860     ngs_reads_classification:ngs_reads_classification.dll
 0002:00000864       __imp_?TAXONOMY_CLASSIFICATION_SLOT_ID@TaxonomySupport@LocalWorkflow@U2@@2VQString@@B 10024864     ngs_reads_classification:ngs_reads_classification.dll
 0002:00000868       __imp_?countClassified@NgsReadsClassificationUtils@U2@@SAHABV?$QMap@VQString@@I@@@Z 10024868     ngs_reads_classification:ngs_reads_classification.dll
 0002:0000086c       __imp_?getBaseFileNameWithSuffixes@NgsReadsClassificationUtils@U2@@SA?AVQString@@ABV3@ABVQStringList@@0_N@Z 1002486c     ngs_reads_classification:ngs_reads_classification.dll
 0002:00000870       __imp_?WORKFLOW_ELEMENTS_GROUP@NgsReadsClassificationPlugin@U2@@2VQString@@B 10024870     ngs_reads_classification:ngs_reads_classification.dll
 0002:00000874       __imp_?setModelData@GenomicLibraryDelegate@LocalWorkflow@U2@@UBEXPAVQWidget@@PAVQAbstractItemModel@@ABVQModelIndex@@@Z 10024874     ngs_reads_classification:ngs_reads_classification.dll
 0002:00000878       __imp_?setEditorData@GenomicLibraryDelegate@LocalWorkflow@U2@@UBEXPAVQWidget@@ABVQModelIndex@@@Z 10024878     ngs_reads_classification:ngs_reads_classification.dll
 0002:0000087c       __imp_?qt_metacast@GenomicLibraryDelegate@LocalWorkflow@U2@@UAEPAXPBD@Z 1002487c     ngs_reads_classification:ngs_reads_classification.dll
 0002:00000880       __imp_?qt_metacall@GenomicLibraryDelegate@LocalWorkflow@U2@@UAEHW4Call@QMetaObject@@HPAPAX@Z 10024880     ngs_reads_classification:ngs_reads_classification.dll
 0002:00000884       __imp_?metaObject@GenomicLibraryDelegate@LocalWorkflow@U2@@UBEPBUQMetaObject@@XZ 10024884     ngs_reads_classification:ngs_reads_classification.dll
 0002:00000888       __imp_?getDisplayValue@GenomicLibraryDelegate@LocalWorkflow@U2@@UBE?AVQVariant@@ABV4@@Z 10024888     ngs_reads_classification:ngs_reads_classification.dll
 0002:0000088c       __imp_?createWizardWidget@GenomicLibraryDelegate@LocalWorkflow@U2@@UBEPAVPropertyWidget@3@AAVU2OpStatus@3@PAVQWidget@@@Z 1002488c     ngs_reads_classification:ngs_reads_classification.dll
 0002:00000890       __imp_?createEditor@GenomicLibraryDelegate@LocalWorkflow@U2@@UBEPAVQWidget@@PAV4@ABVQStyleOptionViewItem@@ABVQModelIndex@@@Z 10024890     ngs_reads_classification:ngs_reads_classification.dll
 0002:00000894       __imp_?clone@GenomicLibraryDelegate@LocalWorkflow@U2@@UAEPAVPropertyDelegate@3@XZ 10024894     ngs_reads_classification:ngs_reads_classification.dll
 0002:00000898       __imp_??0GenomicLibraryDelegate@LocalWorkflow@U2@@QAE@PAVQObject@@@Z 10024898     ngs_reads_classification:ngs_reads_classification.dll
 0002:0000089c       __imp_?TAXON_NUCL_WGS_ACCESSION_2_TAXID_ITEM_ID@NgsReadsClassificationPlugin@U2@@2VQString@@B 1002489c     ngs_reads_classification:ngs_reads_classification.dll
 0002:000008a0       __imp_?TAXON_NUCL_GSS_ACCESSION_2_TAXID_ITEM_ID@NgsReadsClassificationPlugin@U2@@2VQString@@B 100248a0     ngs_reads_classification:ngs_reads_classification.dll
 0002:000008a4       __imp_?TAXON_NUCL_GB_ACCESSION_2_TAXID_ITEM_ID@NgsReadsClassificationPlugin@U2@@2VQString@@B 100248a4     ngs_reads_classification:ngs_reads_classification.dll
 0002:000008a8       __imp_?TAXON_NUCL_EST_ACCESSION_2_TAXID_ITEM_ID@NgsReadsClassificationPlugin@U2@@2VQString@@B 100248a8     ngs_reads_classification:ngs_reads_classification.dll
 0002:000008ac       __imp_?TAXON_NAMES_ITEM_ID@NgsReadsClassificationPlugin@U2@@2VQString@@B 100248ac     ngs_reads_classification:ngs_reads_classification.dll
 0002:000008b0       __imp_?TAXON_NODES_ITEM_ID@NgsReadsClassificationPlugin@U2@@2VQString@@B 100248b0     ngs_reads_classification:ngs_reads_classification.dll
 0002:000008b4       __imp_?TAXONOMY_DATA_ID@NgsReadsClassificationPlugin@U2@@2VQString@@B 100248b4     ngs_reads_classification:ngs_reads_classification.dll
 0002:000008b8       \177ngs_reads_classification_NULL_THUNK_DATA 100248b8     ngs_reads_classification:ngs_reads_classification.dll
 0002:000008bc       ___xc_a                    100248bc     MSVCRT:cinitexe.obj
 0002:00000c6c       ___xc_z                    10024c6c     MSVCRT:cinitexe.obj
 0002:00000c70       ___xi_a                    10024c70     MSVCRT:cinitexe.obj
 0002:00000c7c       ___xi_z                    10024c7c     MSVCRT:cinitexe.obj
 0002:00000cbc       ??_7error_category@std@@6B@ 10024cbc     DatabaseSizeRelation.obj
 0002:00000cd8       ??_7_Generic_error_category@std@@6B@ 10024cd8     DatabaseSizeRelation.obj
 0002:00000cf0       ??_C@_07DCLBNMLN@generic?$AA@ 10024cf0     DatabaseSizeRelation.obj
 0002:00000cf8       ??_C@_0O@BFJCFAAK@unknown?5error?$AA@ 10024cf8     DatabaseSizeRelation.obj
 0002:00000d0c       ??_7_Iostream_error_category@std@@6B@ 10024d0c     DatabaseSizeRelation.obj
 0002:00000d24       ??_C@_08LLGCOLLL@iostream?$AA@ 10024d24     DatabaseSizeRelation.obj
 0002:00000d30       ??_C@_0BG@PADBLCHM@iostream?5stream?5error?$AA@ 10024d30     DatabaseSizeRelation.obj
 0002:00000d4c       ??_7_System_error_category@std@@6B@ 10024d4c     DatabaseSizeRelation.obj
 0002:00000d64       ??_C@_06FHFOAHML@system?$AA@ 10024d64     DatabaseSizeRelation.obj
 0002:00000d6c       ??_C@_0L@JLHNEGIN@Algorithms?$AA@ 10024d6c     DatabaseSizeRelation.obj
 0002:00000d78       ??_C@_07PGLPGHFC@Console?$AA@ 10024d78     DatabaseSizeRelation.obj
 0002:00000d80       ??_C@_0O@BOFHOPCF@Core?5Services?$AA@ 10024d80     DatabaseSizeRelation.obj
 0002:00000d90       ??_C@_0N@PPADAKBM@Input?1Output?$AA@ 10024d90     DatabaseSizeRelation.obj
 0002:00000da0       ??_C@_0M@KPPBKPKK@Performance?$AA@ 10024da0     DatabaseSizeRelation.obj
 0002:00000dac       ??_C@_07BFDHHBBI@Scripts?$AA@ 10024dac     DatabaseSizeRelation.obj
 0002:00000db4       ??_C@_05EEGKELMG@Tasks?$AA@ 10024db4     DatabaseSizeRelation.obj
 0002:00000dbc       ??_C@_0P@NIIOBHGA@User?5Interface?$AA@ 10024dbc     DatabaseSizeRelation.obj
 0002:00000dcc       ??_C@_0N@JINCGGMN@User?5Actions?$AA@ 10024dcc     DatabaseSizeRelation.obj
 0002:00000de0       ??_7DatabaseSizeRelation@LocalWorkflow@U2@@6B@ 10024de0     DatabaseSizeRelation.obj
 0002:00000df8       ??_C@_0O@NJHJECGA@?1database?4kdb?$AA@ 10024df8     DatabaseSizeRelation.obj
 0002:00000e08       ??_C@_0BA@JFNIOLAK@string?5too?5long?$AA@ 10024e08     DatabaseSizeRelation.obj
 0002:00000e18       ??_C@_0BI@CFPLBAOH@invalid?5string?5position?$AA@ 10024e18     DatabaseSizeRelation.obj
 0002:00000e30       ??_C@_00CNPNBAHC@?$AA@     10024e30     KrakenBuildPrompter.obj
 0002:00000e38       ??_7?$PrompterBase@VKrakenBuildPrompter@LocalWorkflow@U2@@@U2@@6BActorDocument@Workflow@1@@ 10024e38     KrakenBuildPrompter.obj
 0002:00000e80       ??_7?$PrompterBase@VKrakenBuildPrompter@LocalWorkflow@U2@@@U2@@6BPrompter@Workflow@1@@ 10024e80     KrakenBuildPrompter.obj
 0002:00000e8c       ??_7KrakenBuildPrompter@LocalWorkflow@U2@@6BActorDocument@Workflow@2@@ 10024e8c     KrakenBuildPrompter.obj
 0002:00000ed4       ??_7KrakenBuildPrompter@LocalWorkflow@U2@@6BPrompter@Workflow@2@@ 10024ed4     KrakenBuildPrompter.obj
 0002:00000edc       ??_C@_0CN@GADOJEAG@Use?5custom?5data?5to?5build?5?$CF1?5Krak@ 10024edc     KrakenBuildPrompter.obj
 0002:00000f0c       ??_C@_0CB@BCNNDEOF@Shrink?5Kraken?5database?5?$CF1?5to?5?$CF2?4@ 10024f0c     KrakenBuildPrompter.obj
 0002:00000f30       ??_C@_0BE@LGBLLFOL@1sl_actorModified?$CI?$CJ?$AA@ 10024f30     KrakenBuildPrompter.obj
 0002:00000f44       ??_C@_0BD@FGIDJNMI@2si_labelChanged?$CI?$CJ?$AA@ 10024f44     KrakenBuildPrompter.obj
 0002:00000f58       ??_C@_0P@DIBOLHGA@2si_modified?$CI?$CJ?$AA@ 10024f58     KrakenBuildPrompter.obj
 0002:00000f68       ??_C@_0BC@HBGBGNIM@2bindingChanged?$CI?$CJ?$AA@ 10024f68     KrakenBuildPrompter.obj
 0002:00000f84       ??_SCopyFileTask@U2@@6B@   10024f84     KrakenBuildTask.obj
 0002:00001014       ??_SSequentialMultiTask@U2@@6B@ 10025014     KrakenBuildTask.obj
 0002:000010a4       ??_SExternalToolRunTask@U2@@6B@ 100250a4     KrakenBuildTask.obj
 0002:00001134       ??_SExternalToolLogParser@U2@@6B@ 10025134     KrakenBuildTask.obj
 0002:00001180       ??_7KrakenBuildTask@U2@@6B@ 10025180     KrakenBuildTask.obj
 0002:00001214       ??_C@_05DMEBLLNM@build?$AA@ 10025214     KrakenBuildTask.obj
 0002:0000121c       ??_C@_06FKMIDIGA@shrink?$AA@ 1002521c     KrakenBuildTask.obj
 0002:00001224       ??_C@_0BD@LIGABAMJ@?$CF1?5Kraken?5database?$AA@ 10025224     KrakenBuildTask.obj
 0002:00001238       ??_C@_0BA@CNJLLDBG@KrakenBuildTask?$AA@ 10025238     KrakenBuildTask.obj
 0002:00001248       ??_C@_05DLONLOOK@Build?$AA@ 10025248     KrakenBuildTask.obj
 0002:00001250       ??_C@_06JFHFABPM@Shrink?$AA@ 10025250     KrakenBuildTask.obj
 0002:00001258       ??_C@_0CK@IGBIANDN@Trying?5to?5recover?5from?5error?3?5?$CF1@ 10025258     KrakenBuildTask.obj
 0002:00001284       ??_C@_0BA@IHMBOPHE@An?5unknown?5mode?$AA@ 10025284     KrakenBuildTask.obj
 0002:00001294       ??_C@_0BI@CKLBCGO@src?2KrakenBuildTask?4cpp?$AA@ 10025294     KrakenBuildTask.obj
 0002:000012ac       ??_C@_0BF@EDNEEPFK@Sequential?5execution?$AA@ 100252ac     KrakenBuildTask.obj
 0002:000012c4       ??_C@_0N@DFEPOLHD@Unknown?5mode?$AA@ 100252c4     KrakenBuildTask.obj
 0002:000012d4       ??_C@_0BM@GIICOGOA@Input?5database?5URL?5is?5empty?$AA@ 100252d4     KrakenBuildTask.obj
 0002:000012f0       ??_C@_0BN@IAIDMBGK@Input?5database?5doesn?8t?5exist?$AA@ 100252f0     KrakenBuildTask.obj
 0002:00001310       ??_C@_0BK@JJDJOPO@New?5database?5URL?5is?5empty?$AA@ 10025310     KrakenBuildTask.obj
 0002:0000132c       ??_C@_0DC@PNEKCFAO@Genomes?5URLs?5list?5to?5build?5datab@ 1002532c     KrakenBuildTask.obj
 0002:00001360       ??_C@_0DN@PDEKLLLE@K?9mers?5count?5to?5move?5to?5a?5new?5da@ 10025360     KrakenBuildTask.obj
 0002:000013a0       ??_C@_0CG@GCMAFGIB@K?9mer?5length?5is?5out?5of?5boundarie@ 100253a0     KrakenBuildTask.obj
 0002:000013c8       ??_C@_0CK@POKIKMPL@Minimizer?5length?5is?5out?5of?5bound@ 100253c8     KrakenBuildTask.obj
 0002:000013f4       ??_C@_0CP@NDCOICFG@Minimizer?5length?5is?5not?5less?5tha@ 100253f4     KrakenBuildTask.obj
 0002:00001424       ??_C@_0DA@FOHLOALB@Maximum?5database?5size?5cannot?5be?5@ 10025424     KrakenBuildTask.obj
 0002:00001454       ??_C@_0CO@DBEKCBHA@Shrink?5block?5offset?5cannot?5be?5le@ 10025454     KrakenBuildTask.obj
 0002:00001484       ??_C@_0CO@BNNNHEOA@Jellyfish?5hash?5size?5cannot?5be?5le@ 10025484     KrakenBuildTask.obj
 0002:000014b4       ??_C@_0CJ@KNGACNAJ@Threads?5number?5cannot?5be?5less?5th@ 100254b4     KrakenBuildTask.obj
 0002:000014e0       ??_C@_0BK@PGODFLIK@Taxonomy?5data?5are?5not?5set?$AA@ 100254e0     KrakenBuildTask.obj
 0002:000014fc       ??_C@_09MOLNGKFO@?1taxonomy?$AA@ 100254fc     KrakenBuildTask.obj
 0002:00001508       ??_C@_0BK@OAKDHIKP@Cannot?5find?5taxonomy?5data?$AA@ 10025508     KrakenBuildTask.obj
 0002:00001524       ??_C@_01KMDKNFGN@?1?$AA@   10025524     KrakenBuildTask.obj
 0002:00001528       ??_C@_0DG@OLPAAICA@Can?8t?5create?5a?5symbolic?5link?5to?5@ 10025528     KrakenBuildTask.obj
 0002:00001560       ??_C@_0BB@FKOHAGMK@?9?9add?9to?9library?$AA@ 10025560     KrakenBuildTask.obj
 0002:00001574       ??_C@_04EKMBPOGN@?9?9db?$AA@ 10025574     KrakenBuildTask.obj
 0002:0000157c       ??_C@_07CELIOKMN@?9?9build?$AA@ 1002557c     KrakenBuildTask.obj
 0002:00001584       ??_C@_09JKEFGKKN@?9?9threads?$AA@ 10025584     KrakenBuildTask.obj
 0002:00001590       ??_C@_0L@JEKMINNE@?9?9kmer?9len?$AA@ 10025590     KrakenBuildTask.obj
 0002:0000159c       ??_C@_0BA@KKKPOPHA@?9?9minimizer?9len?$AA@ 1002559c     KrakenBuildTask.obj
 0002:000015ac       ??_C@_0BG@BHFEPIGM@?9?9jellyfish?9hash?9size?$AA@ 100255ac     KrakenBuildTask.obj
 0002:000015c4       ??_C@_0O@FLAFJECB@?9?9max?9db?9size?$AA@ 100255c4     KrakenBuildTask.obj
 0002:000015d4       ??_C@_0P@NEJNNOML@?9?9work?9on?9disk?$AA@ 100255d4     KrakenBuildTask.obj
 0002:000015e4       ??_C@_07DKPFAIPK@?9?9clean?$AA@ 100255e4     KrakenBuildTask.obj
 0002:000015ec       ??_C@_08DAGAOBMD@?9?9shrink?$AA@ 100255ec     KrakenBuildTask.obj
 0002:000015f8       ??_C@_08IKDEHBJG@?9?9new?9db?$AA@ 100255f8     KrakenBuildTask.obj
 0002:00001604       ??_C@_0BG@POAOJIHE@?9?9shrink?9block?9offset?$AA@ 10025604     KrakenBuildTask.obj
 0002:00001620       __real@3f50000000000000    10025620     KrakenBuildTask.obj
 0002:00001628       __real@3ff0000000000000    10025628     KrakenBuildTask.obj
 0002:00001630       ??_C@_0BJ@BCCOGGEF@MinimizerLengthValidator?$AA@ 10025630     KrakenBuildValidator.obj
 0002:0000164c       ??_C@_0DC@IBAJOJDB@Minimizer?5length?5has?5to?5be?5less?5@ 1002564c     KrakenBuildValidator.obj
 0002:00001680       ??_C@_0DK@FGLPPHNF@Taxonomy?5classification?5data?5fro@ 10025680     KrakenBuildValidator.obj
 0002:000016c0       ??_C@_0EL@ENMJCHGK@Taxonomy?5classification?5data?5fro@ 100256c0     KrakenBuildValidator.obj
 0002:00001710       ??_STaskSignalMapper@U2@@6B@ 10025710     KrakenBuildWorker.obj
 0002:00001740       ??_SDescriptor@U2@@6B@     10025740     KrakenBuildWorker.obj
 0002:0000174c       ??_C@_0BD@FOHBGHEI@QList?$DMU2?3?3Dataset?$DO?$AA@ 1002574c     KrakenBuildWorker.obj
 0002:00001760       ??_C@_0BF@COKBMJP@Script?5task?5canceled?$AA@ 10025760     KrakenBuildWorker.obj
 0002:0000177c       ??_7KrakenBuildWorker@LocalWorkflow@U2@@6BQObject@@@ 1002577c     KrakenBuildWorker.obj
 0002:000017c0       ??_7KrakenBuildWorker@LocalWorkflow@U2@@6BWorker@Workflow@2@@ 100257c0     KrakenBuildWorker.obj
 0002:000017dc       ??_7KrakenBuildWorker@LocalWorkflow@U2@@6BCommunicationSubject@Workflow@2@@ 100257dc     KrakenBuildWorker.obj
 0002:000017e8       ??_C@_0BK@LMMJOEHE@Port?5with?5id?5?8?$CF1?8?5is?5NULL?$AA@ 100257e8     KrakenBuildWorker.obj
 0002:00001804       ??_C@_0BK@KIFABPPL@src?2KrakenBuildWorker?4cpp?$AA@ 10025804     KrakenBuildWorker.obj
 0002:00001820       ??_C@_0BJ@JJNIMNNJ@1sl_taskFinished?$CITask?5?$CK?$CJ?$AA@ 10025820     KrakenBuildWorker.obj
 0002:0000183c       ??_C@_0BJ@DHBKDAMN@2si_taskFinished?$CITask?5?$CK?$CJ?$AA@ 1002583c     KrakenBuildWorker.obj
 0002:00001858       ??_C@_09DMOIMEE@Dataset?51?$AA@ 10025858     KrakenBuildWorker.obj
 0002:00001868       ??_SVisibilityRelation@U2@@6B@ 10025868     KrakenBuildWorkerFactory.obj
 0002:00001884       ??_SMapDataType@U2@@6B@    10025884     KrakenBuildWorkerFactory.obj
 0002:000018a4       ??_SAttribute@U2@@6B@      100258a4     KrakenBuildWorkerFactory.obj
 0002:000018dc       ??_SDelegateEditor@U2@@6B@ 100258dc     KrakenBuildWorkerFactory.obj
 0002:00001934       ??_SURLDelegate@U2@@6B@    10025934     KrakenBuildWorkerFactory.obj
 0002:000019b4       ??_SSpinBoxDelegate@U2@@6B@ 100259b4     KrakenBuildWorkerFactory.obj
 0002:00001a34       ??_SComboBoxDelegate@U2@@6B@ 10025a34     KrakenBuildWorkerFactory.obj
 0002:00001ab4       ??_SComboBoxWithBoolsDelegate@U2@@6B@ 10025ab4     KrakenBuildWorkerFactory.obj
 0002:00001b34       ??_SPortDescriptor@Workflow@U2@@6B@ 10025b34     KrakenBuildWorkerFactory.obj
 0002:00001b4c       ??_SIntegralBusActorPrototype@Workflow@U2@@6BQObject@@@ 10025b4c     KrakenBuildWorkerFactory.obj
 0002:00001b88       ??_SIntegralBusActorPrototype@Workflow@U2@@6BVisualDescriptor@2@@ 10025b88     KrakenBuildWorkerFactory.obj
 0002:00001b98       ??_7KrakenBuildValidator@Workflow@U2@@6B@ 10025b98     KrakenBuildWorkerFactory.obj
 0002:00001ba8       ??_7KrakenBuildWorkerFactory@LocalWorkflow@U2@@6B?$IdRegistry@VDomainFactory@Workflow@U2@@@2@@ 10025ba8     KrakenBuildWorkerFactory.obj
 0002:00001bd4       ??_7KrakenBuildWorkerFactory@LocalWorkflow@U2@@6BDescriptor@2@@ 10025bd4     KrakenBuildWorkerFactory.obj
 0002:00001be4       ??_SGenomicLibraryDelegate@LocalWorkflow@U2@@6B@ 10025be4     KrakenBuildWorkerFactory.obj
 0002:00001c60       ??_C@_0N@GGBOLOCK@kraken?9build?$AA@ 10025c60     KrakenBuildWorkerFactory.obj
 0002:00001c70       ??_C@_03KEJHNBPP@out?$AA@  10025c70     KrakenBuildWorkerFactory.obj
 0002:00001c74       ??_C@_04GMGOKAFF@mode?$AA@ 10025c74     KrakenBuildWorkerFactory.obj
 0002:00001c7c       ??_C@_0P@EBHHPCKG@input?9database?$AA@ 10025c7c     KrakenBuildWorkerFactory.obj
 0002:00001c8c       ??_C@_08PBOCEOLL@database?$AA@ 10025c8c     KrakenBuildWorkerFactory.obj
 0002:00001c98       ??_C@_0BA@GJNMLPPF@genomic?9library?$AA@ 10025c98     KrakenBuildWorkerFactory.obj
 0002:00001ca8       ??_C@_0BB@IFJAPLCN@number?9of?9k?9mers?$AA@ 10025ca8     KrakenBuildWorkerFactory.obj
 0002:00001cbc       ??_C@_0N@OFIHBBIE@k?9mer?9length?$AA@ 10025cbc     KrakenBuildWorkerFactory.obj
 0002:00001ccc       ??_C@_0BB@DPPGHOBL@minimizer?9length?$AA@ 10025ccc     KrakenBuildWorkerFactory.obj
 0002:00001ce0       ??_C@_0BG@KLIJOLBE@maximum?9database?9size?$AA@ 10025ce0     KrakenBuildWorkerFactory.obj
 0002:00001cf8       ??_C@_0BE@BMLOFKJB@shrink?9block?9offset?$AA@ 10025cf8     KrakenBuildWorkerFactory.obj
 0002:00001d0c       ??_C@_05CCAMFJOL@clean?$AA@ 10025d0c     KrakenBuildWorkerFactory.obj
 0002:00001d14       ??_C@_0N@CGPNPLP@work?9on?9disk?$AA@ 10025d14     KrakenBuildWorkerFactory.obj
 0002:00001d24       ??_C@_0BE@PFOEDKIJ@jellyfish?9hash?9size?$AA@ 10025d24     KrakenBuildWorkerFactory.obj
 0002:00001d38       ??_C@_07NFPADACG@threads?$AA@ 10025d38     KrakenBuildWorkerFactory.obj
 0002:00001d40       ??_C@_0M@FOOCJNHH@Output?5URL?4?$AA@ 10025d40     KrakenBuildWorkerFactory.obj
 0002:00001d4c       ??_C@_0L@OALCHELH@Output?5URL?$AA@ 10025d4c     KrakenBuildWorkerFactory.obj
 0002:00001d58       ??_C@_0CM@GFPCBDAO@URL?5to?5the?5folder?5with?5the?5Krake@ 10025d58     KrakenBuildWorkerFactory.obj
 0002:00001d84       ??_C@_0BH@DGGGNADM@Output?5Kraken?5database?$AA@ 10025d84     KrakenBuildWorkerFactory.obj
 0002:00001d9c       ??_C@_04HKKABCEL@?9out?$AA@ 10025d9c     KrakenBuildWorkerFactory.obj
 0002:00001da8       ??_C@_0LE@JLOLNEOK@Select?5?$CCBuild?$CC?5to?5create?5a?5new?5d@ 10025da8     KrakenBuildWorkerFactory.obj
 0002:00001e5c       ??_C@_04KNKPIPFB@Mode?$AA@ 10025e5c     KrakenBuildWorkerFactory.obj
 0002:00001e68       ??_C@_0GD@CHCFDEKN@Name?5of?5the?5input?5database?5that?5@ 10025e68     KrakenBuildWorkerFactory.obj
 0002:00001ecc       ??_C@_0P@DMEMEHII@Input?5database?$AA@ 10025ecc     KrakenBuildWorkerFactory.obj
 0002:00001ee0       ??_C@_0IA@GCDHOCPL@Name?5of?5the?5output?5Kraken?5databa@ 10025ee0     KrakenBuildWorkerFactory.obj
 0002:00001f60       ??_C@_08HDBDMMBI@Database?$AA@ 10025f60     KrakenBuildWorkerFactory.obj
 0002:00001f70       ??_C@_0MO@CDCJOOIF@Genomes?5that?5should?5be?5used?5to?5b@ 10025f70     KrakenBuildWorkerFactory.obj
 0002:00002040       ??_C@_0BA@IPKMCDNP@Genomic?5library?$AA@ 10026040     KrakenBuildWorkerFactory.obj
 0002:00002050       ??_C@_0GG@PKCPLMHK@The?5new?5database?5will?5contain?5th@ 10026050     KrakenBuildWorkerFactory.obj
 0002:000020b8       ??_C@_0BB@PLKCJBAB@Number?5of?5k?9mers?$AA@ 100260b8     KrakenBuildWorkerFactory.obj
 0002:000020cc       ??_C@_0CB@KHNJOKBD@K?9mer?5length?5in?5bp?5?$CI?9?9kmer?9len?$CJ?4@ 100260cc     KrakenBuildWorkerFactory.obj
 0002:000020f0       ??_C@_0N@MNPMEPKA@K?9mer?5length?$AA@ 100260f0     KrakenBuildWorkerFactory.obj
 0002:00002100       ??_C@_0BIA@GPAAEMCC@Minimizer?5length?5in?5bp?5?$CI?9?9minimi@ 10026100     KrakenBuildWorkerFactory.obj
 0002:00002280       ??_C@_0BB@IKFAFJDA@Minimizer?5length?$AA@ 10026280     KrakenBuildWorkerFactory.obj
 0002:00002298       ??_C@_0BBF@OELDCMFI@By?5default?0?5a?5full?5database?5buil@ 10026298     KrakenBuildWorkerFactory.obj
 0002:000023b0       ??_C@_0BG@GDIGBIAF@Maximum?5database?5size?$AA@ 100263b0     KrakenBuildWorkerFactory.obj
 0002:000023c8       ??_C@_0HC@KMCNNHKI@When?5shrinking?0?5select?5the?5k?9mer@ 100263c8     KrakenBuildWorkerFactory.obj
 0002:0000243c       ??_C@_0BE@CKLNGPBA@Shrink?5block?5offset?$AA@ 1002643c     KrakenBuildWorkerFactory.obj
 0002:00002450       ??_C@_0FA@KDAJFNMO@Remove?5unneeded?5files?5from?5a?5bui@ 10026450     KrakenBuildWorkerFactory.obj
 0002:000024a0       ??_C@_05CFKAFMNN@Clean?$AA@ 100264a0     KrakenBuildWorkerFactory.obj
 0002:000024a8       ??_C@_0FO@NKBNJJGK@Perform?5most?5operations?5on?5disk?5@ 100264a8     KrakenBuildWorkerFactory.obj
 0002:00002508       ??_C@_0N@PMMAGAMD@Work?5on?5disk?$AA@ 10026508     KrakenBuildWorkerFactory.obj
 0002:00002518       ??_C@_0BDB@MIOBPPEH@The?5?$CCkraken?9build?$CC?5tool?5uses?5the@ 10026518     KrakenBuildWorkerFactory.obj
 0002:0000264c       ??_C@_0BE@JIBCDEFL@Jellyfish?5hash?5size?$AA@ 1002664c     KrakenBuildWorkerFactory.obj
 0002:00002660       ??_C@_0CC@FJELABGN@Use?5multiple?5threads?5?$CI?9?9threads?$CJ@ 10026660     KrakenBuildWorkerFactory.obj
 0002:00002684       ??_C@_0BC@GJADDMKB@Number?5of?5threads?$AA@ 10026684     KrakenBuildWorkerFactory.obj
 0002:00002698       ??_C@_0BA@MCPNCJJO@kraken?1database?$AA@ 10026698     KrakenBuildWorkerFactory.obj
 0002:000026a8       ??_C@_07CCOEHHFD@minimum?$AA@ 100266a8     KrakenBuildWorkerFactory.obj
 0002:000026b0       ??_C@_07MEIENILC@maximum?$AA@ 100266b0     KrakenBuildWorkerFactory.obj
 0002:000026b8       ??_C@_0M@MFGNCGHE@accelerated?$AA@ 100266b8     KrakenBuildWorkerFactory.obj
 0002:000026c4       ??_C@_06EMCDFPCG@suffix?$AA@ 100266c4     KrakenBuildWorkerFactory.obj
 0002:000026cc       ??_C@_03FBAAJIGL@?5Mb?$AA@ 100266cc     KrakenBuildWorkerFactory.obj
 0002:000026d0       ??_C@_0BB@HBOHNBEB@specialValueText?$AA@ 100266d0     KrakenBuildWorkerFactory.obj
 0002:000026e4       ??_C@_08OHNNABNB@No?5limit?$AA@ 100266e4     KrakenBuildWorkerFactory.obj
 0002:000026f0       ??_C@_02HNCEFBEF@?5M?$AA@  100266f0     KrakenBuildWorkerFactory.obj
 0002:000026f4       ??_C@_04MCHAEEKC@Skip?$AA@ 100266f4     KrakenBuildWorkerFactory.obj
 0002:00002700       ??_C@_0EM@HBLJNIIE@Build?5a?5Kraken?5database?5from?5a?5g@ 10026700     KrakenBuildWorkerFactory.obj
 0002:0000274c       ??_C@_0BG@DNGHNMMB@Build?5Kraken?5Database?$AA@ 1002674c     KrakenBuildWorkerFactory.obj
 0002:00002768       ??_7KrakenClassifyLogParser@U2@@6B@ 10026768     KrakenClassifyLogParser.obj
 0002:000027b0       ??_C@_0BA@NGPCNOJ@Must?5specify?5DB?$AA@ 100267b0     KrakenClassifyLogParser.obj
 0002:000027c0       ??_C@_0CN@MLBDIIPK@does?5not?5contain?5necessary?5file?5@ 100267c0     KrakenClassifyLogParser.obj
 0002:000027f0       ??_C@_0CI@FBIPMBAN@?9?9paired?5requires?5exactly?5two?5fi@ 100267f0     KrakenClassifyLogParser.obj
 0002:00002818       ??_C@_0BL@GKJCAKFJ@mismatched?5mate?5pair?5names?$AA@ 10026818     KrakenClassifyLogParser.obj
 0002:00002834       ??_C@_0BM@DFJFCBLE@can?8t?5determine?5what?5format?$AA@ 10026834     KrakenClassifyLogParser.obj
 0002:00002850       ??_C@_0DD@GCAHBFEB@can?8t?5open?5database?4idx?3?5No?5such@ 10026850     KrakenClassifyLogParser.obj
 0002:00002884       ??_C@_0BL@JDODHMKN@mismatched?5sequence?5counts?$AA@ 10026884     KrakenClassifyLogParser.obj
 0002:000028a0       ??_C@_0CA@LAIKEMDJ@Need?5to?5specify?5input?5filenames?$AA@ 100268a0     KrakenClassifyLogParser.obj
 0002:000028c4       ??_7?$PrompterBase@VKrakenClassifyPrompter@LocalWorkflow@U2@@@U2@@6BActorDocument@Workflow@1@@ 100268c4     KrakenClassifyPrompter.obj
 0002:0000290c       ??_7?$PrompterBase@VKrakenClassifyPrompter@LocalWorkflow@U2@@@U2@@6BPrompter@Workflow@1@@ 1002690c     KrakenClassifyPrompter.obj
 0002:00002918       ??_7KrakenClassifyPrompter@LocalWorkflow@U2@@6BActorDocument@Workflow@2@@ 10026918     KrakenClassifyPrompter.obj
 0002:00002960       ??_7KrakenClassifyPrompter@LocalWorkflow@U2@@6BPrompter@Workflow@2@@ 10026960     KrakenClassifyPrompter.obj
 0002:00002968       ??_C@_0EA@PMNCDKIH@Classify?5sequences?5from?5?$DMu?$DO?$CF1?$DM?1u@ 10026968     KrakenClassifyPrompter.obj
 0002:000029a8       ??_C@_0EH@KEOKEAON@Classify?5paired?9end?5reads?5from?5?$DM@ 100269a8     KrakenClassifyPrompter.obj
 0002:000029f4       ??_7KrakenClassifyTask@U2@@6B@ 100269f4     KrakenClassifyTask.obj
 0002:00002a88       ??_C@_0L@PCJLLKLK@single?9end?$AA@ 10026a88     KrakenClassifyTask.obj
 0002:00002a94       ??_C@_0L@HGFAFILP@paired?9end?$AA@ 10026a94     KrakenClassifyTask.obj
 0002:00002aa0       ??_C@_0BL@NPCCMJJP@Classify?5reads?5with?5Kraken?$AA@ 10026aa0     KrakenClassifyTask.obj
 0002:00002abc       ??_C@_0BD@FCNPPCDI@KrakenClassifyTask?$AA@ 10026abc     KrakenClassifyTask.obj
 0002:00002ad0       ??_C@_0BD@HKKHAEBH@Reads?5URL?5is?5empty?$AA@ 10026ad0     KrakenClassifyTask.obj
 0002:00002ae4       ??_C@_0BN@INGDPKFL@Kraken?5database?5URL?5is?5empty?$AA@ 10026ae4     KrakenClassifyTask.obj
 0002:00002b04       ??_C@_0CD@IDNFHIKN@Kraken?5classification?5URL?5is?5emp@ 10026b04     KrakenClassifyTask.obj
 0002:00002b28       ??_C@_07CNDOMBAK@?9?9quick?$AA@ 10026b28     KrakenClassifyTask.obj
 0002:00002b30       ??_C@_0L@NJGGJGCM@?9?9min?9hits?$AA@ 10026b30     KrakenClassifyTask.obj
 0002:00002b3c       ??_C@_08FACOKJIG@?9?9output?$AA@ 10026b3c     KrakenClassifyTask.obj
 0002:00002b48       ??_C@_09CNPFMGML@?9?9preload?$AA@ 10026b48     KrakenClassifyTask.obj
 0002:00002b54       ??_C@_08DNGCCPLF@?9?9paired?$AA@ 10026b54     KrakenClassifyTask.obj
 0002:00002b60       ??_C@_0O@HBHGMGKG@?9?9check?9names?$AA@ 10026b60     KrakenClassifyTask.obj
 0002:00002b70       ??_C@_0CG@IHMCOLO@Cannot?5open?5classification?5repor@ 10026b70     KrakenClassifyTask.obj
 0002:00002b98       ??_C@_02KDKAKODN@C?7?$AA@  10026b98     KrakenClassifyTask.obj
 0002:00002b9c       ??_C@_02LLALHBPP@U?7?$AA@  10026b9c     KrakenClassifyTask.obj
 0002:00002ba0       ??_C@_0CD@HNGOICBL@Found?5Kraken?5classification?3?5?$CF1?$DN@ 10026ba0     KrakenClassifyTask.obj
 0002:00002bc8       ??_C@_0EO@GBJCHADO@Duplicate?5sequence?5name?5?8?$CF1?8?5hav@ 10026bc8     KrakenClassifyTask.obj
 0002:00002c18       ??_C@_0BK@EMCDHGEH@Broken?5Kraken?5report?5?3?5?$CF1?$AA@ 10026c18     KrakenClassifyTask.obj
 0002:00002c34       ??_C@_0BI@IHPDBDA@KrakenClassifyValidator?$AA@ 10026c34     KrakenClassifyValidator.obj
 0002:00002c4c       ??_C@_0CI@PPNEEPAN@The?5database?5folder?5?$CC?$CF1?$CC?5doesn?8t@ 10026c4c     KrakenClassifyValidator.obj
 0002:00002c74       ??_C@_0N@JMEGLBAL@database?4kdb?$AA@ 10026c74     KrakenClassifyValidator.obj
 0002:00002c84       ??_C@_0N@IGGCIDFL@database?4idx?$AA@ 10026c84     KrakenClassifyValidator.obj
 0002:00002c94       ??_C@_0BD@PAHDILNG@taxonomy?1nodes?4dmp?$AA@ 10026c94     KrakenClassifyValidator.obj
 0002:00002ca8       ??_C@_0BD@CHPOELGP@taxonomy?1names?4dmp?$AA@ 10026ca8     KrakenClassifyValidator.obj
 0002:00002cbc       ??_C@_0DA@NHHLJLMN@The?5mandatory?5database?5file?5?$CC?$CF1?$CC@ 10026cbc     KrakenClassifyValidator.obj
 0002:00002cec       ??_C@_0CM@ICPJCNAJ@QtMetaTypePrivate?3?3QAssociativeI@ 10026cec     KrakenClassifyWorker.obj
 0002:00002d1c       ??_SFailTask@U2@@6B@       10026d1c     KrakenClassifyWorker.obj
 0002:00002da8       ??_C@_0DA@ENPGIFBJ@U2?3?3LocalWorkflow?3?3TaxonomyClass@ 10026da8     KrakenClassifyWorker.obj
 0002:00002ddc       ??_7KrakenClassifyWorker@LocalWorkflow@U2@@6BQObject@@@ 10026ddc     KrakenClassifyWorker.obj
 0002:00002e20       ??_7KrakenClassifyWorker@LocalWorkflow@U2@@6BWorker@Workflow@2@@ 10026e20     KrakenClassifyWorker.obj
 0002:00002e3c       ??_7KrakenClassifyWorker@LocalWorkflow@U2@@6BCommunicationSubject@Workflow@2@@ 10026e3c     KrakenClassifyWorker.obj
 0002:00002e48       ??_C@_06JPGCMMNF@Kraken?$AA@ 10026e48     KrakenClassifyWorker.obj
 0002:00002e50       ??_C@_0BN@HGFPBHKI@src?2KrakenClassifyWorker?4cpp?$AA@ 10026e50     KrakenClassifyWorker.obj
 0002:00002e70       ??_C@_0DF@GPCBDEIK@There?5were?5?$CF1?5input?5reads?0?5?$CF2?5re@ 10026e70     KrakenClassifyWorker.obj
 0002:00002ea8       ??_C@_01IDAFKMJL@_?$AA@    10026ea8     KrakenClassifyWorker.obj
 0002:00002eac       ??_C@_0O@MMLICHBP@Kraken_?$CF1?4txt?$AA@ 10026eac     KrakenClassifyWorker.obj
 0002:00002ebc       ??_C@_03CLFHJCDC@txt?$AA@  10026ebc     KrakenClassifyWorker.obj
 0002:00002ec0       ??_C@_04LOAJBDKD@true?$AA@ 10026ec0     KrakenClassifyWorkerFactory.obj
 0002:00002ecc       ??_SSlotRelationDescriptor@U2@@6B@ 10026ecc     KrakenClassifyWorkerFactory.obj
 0002:00002edc       ??_SPairedReadsPortValidator@Workflow@U2@@6B@ 10026edc     KrakenClassifyWorkerFactory.obj
 0002:00002eec       ??_7KrakenClassifyValidator@Workflow@U2@@6B@ 10026eec     KrakenClassifyWorkerFactory.obj
 0002:00002efc       ??_7KrakenClassifyWorkerFactory@LocalWorkflow@U2@@6B?$IdRegistry@VDomainFactory@Workflow@U2@@@2@@ 10026efc     KrakenClassifyWorkerFactory.obj
 0002:00002f28       ??_7KrakenClassifyWorkerFactory@LocalWorkflow@U2@@6BDescriptor@2@@ 10026f28     KrakenClassifyWorkerFactory.obj
 0002:00002f3c       ??_SDatabaseDelegate@LocalWorkflow@U2@@6B@ 10026f3c     KrakenClassifyWorkerFactory.obj
 0002:00002fb8       ??_C@_0BA@CGDKDLFJ@kraken?9classify?$AA@ 10026fb8     KrakenClassifyWorkerFactory.obj
 0002:00002fc8       ??_C@_02LMMGJAGL@in?$AA@   10026fc8     KrakenClassifyWorkerFactory.obj
 0002:00002fcc       ??_C@_0L@LGHLPLD@reads?9url1?$AA@ 10026fcc     KrakenClassifyWorkerFactory.obj
 0002:00002fd8       ??_C@_0L@CAEKOMHA@reads?9url2?$AA@ 10026fd8     KrakenClassifyWorkerFactory.obj
 0002:00002fe4       ??_C@_0L@HPPLHBN@input?9data?$AA@ 10026fe4     KrakenClassifyWorkerFactory.obj
 0002:00002ff0       ??_C@_0L@JDEFPCKN@output?9url?$AA@ 10026ff0     KrakenClassifyWorkerFactory.obj
 0002:00002ffc       ??_C@_0BA@NAHJCFJC@quick?9operation?$AA@ 10026ffc     KrakenClassifyWorkerFactory.obj
 0002:0000300c       ??_C@_08KDEDHJNO@min?9hits?$AA@ 1002700c     KrakenClassifyWorkerFactory.obj
 0002:00003018       ??_C@_07GCEAJMEA@preload?$AA@ 10027018     KrakenClassifyWorkerFactory.obj
 0002:00003020       ??_C@_0BE@IHKBOJBH@SE?5reads?5or?5contigs?$AA@ 10027020     KrakenClassifyWorkerFactory.obj
 0002:00003034       ??_C@_08BKAKNCGK@PE?5reads?$AA@ 10027034     KrakenClassifyWorkerFactory.obj
 0002:00003040       ??_C@_0N@JCLPICJJ@Input?5URL?51?4?$AA@ 10027040     KrakenClassifyWorkerFactory.obj
 0002:00003050       ??_C@_0M@LBNKAPAD@Input?5URL?51?$AA@ 10027050     KrakenClassifyWorkerFactory.obj
 0002:0000305c       ??_C@_0N@JAPJDMMA@Input?5URL?52?4?$AA@ 1002705c     KrakenClassifyWorkerFactory.obj
 0002:0000306c       ??_C@_0M@JKPHFMMA@Input?5URL?52?$AA@ 1002706c     KrakenClassifyWorkerFactory.obj
 0002:00003078       ??_C@_0BAF@MDCIJEPN@URL?$CIs?$CJ?5to?5FASTQ?5or?5FASTA?5file?$CIs?$CJ@ 10027078     KrakenClassifyWorkerFactory.obj
 0002:00003180       ??_C@_0BA@GLOOOALC@Input?5sequences?$AA@ 10027180     KrakenClassifyWorkerFactory.obj
 0002:00003190       ??_C@_0FA@KJMADBIC@A?5map?5of?5sequence?5names?5with?5the@ 10027190     KrakenClassifyWorkerFactory.obj
 0002:000031e0       ??_C@_0BG@KAPCJDCF@Kraken?5Classification?$AA@ 100271e0     KrakenClassifyWorkerFactory.obj
 0002:000031f8       ??_C@_03DAJLOBIG@?9in?$AA@ 100271f8     KrakenClassifyWorkerFactory.obj
 0002:00003200       ??_C@_0BIC@MFFKKPNE@To?5classify?5single?9end?5?$CISE?$CJ?5read@ 10027200     KrakenClassifyWorkerFactory.obj
 0002:00003384       ??_C@_0L@DNPNCLBE@Input?5data?$AA@ 10027384     KrakenClassifyWorkerFactory.obj
 0002:00003390       ??_C@_0DF@NEOCIJKM@A?5path?5to?5the?5folder?5with?5the?5Kr@ 10027390     KrakenClassifyWorkerFactory.obj
 0002:000033c8       ??_C@_0BO@FKBHNKFL@Specify?5the?5output?5file?5name?4?$AA@ 100273c8     KrakenClassifyWorkerFactory.obj
 0002:000033e8       ??_C@_0M@LEIJPAKP@Output?5file?$AA@ 100273e8     KrakenClassifyWorkerFactory.obj
 0002:000033f8       ??_C@_0JE@EFMMJCBH@Stop?5classification?5of?5an?5input?5@ 100273f8     KrakenClassifyWorkerFactory.obj
 0002:0000348c       ??_C@_0BA@MNCBDOI@Quick?5operation?$AA@ 1002748c     KrakenClassifyWorkerFactory.obj
 0002:000034a0       ??_C@_0NN@IPELMFDB@The?5number?5of?5hits?5that?5are?5requ@ 100274a0     KrakenClassifyWorkerFactory.obj
 0002:00003580       ??_C@_0BH@NMMILFKE@Minimum?5number?5of?5hits?$AA@ 10027580     KrakenClassifyWorkerFactory.obj
 0002:00003598       ??_C@_0BBB@HDHAOFP@Load?5the?5Kraken?5database?5into?5RA@ 10027598     KrakenClassifyWorkerFactory.obj
 0002:000036ac       ??_C@_0BK@MBNCKPDD@Load?5database?5into?5memory?$AA@ 100276ac     KrakenClassifyWorkerFactory.obj
 0002:000036c8       ??_C@_0CA@BBFPBJKD@Classify?5tool?4?5Hidden?5attribute?$AA@ 100276c8     KrakenClassifyWorkerFactory.obj
 0002:000036e8       ??_C@_04LBDCJOFB@Auto?$AA@ 100276e8     KrakenClassifyWorkerFactory.obj
 0002:000036f0       ??_C@_0O@CMCHHPHE@kraken?1output?$AA@ 100276f0     KrakenClassifyWorkerFactory.obj
 0002:00003700       ??_C@_0LD@PJICIECK@Kraken?5is?5a?5taxonomic?5sequence?5c@ 10027700     KrakenClassifyWorkerFactory.obj
 0002:000037b4       ??_C@_0BP@ONJHABCG@Classify?5Sequences?5with?5Kraken?$AA@ 100277b4     KrakenClassifyWorkerFactory.obj
 0002:000037d8       ??_7KrakenSupport@U2@@6B@  100277d8     KrakenSupport.obj
 0002:00003818       ??_C@_0BD@INIEADMO@USUPP_KRAKEN_BUILD?$AA@ 10027818     KrakenSupport.obj
 0002:0000382c       ??_C@_06FANPPFEJ@kraken?$AA@ 1002782c     KrakenSupport.obj
 0002:00003834       ??_C@_0N@NHAFOJML@USUPP_KRAKEN?$AA@ 10027834     KrakenSupport.obj
 0002:00003844       ??_C@_09GAJKMFCA@?9?9version?$AA@ 10027844     KrakenSupport.obj
 0002:00003850       ??_C@_0BA@BIEDGII@Kraken?5version?5?$AA@ 10027850     KrakenSupport.obj
 0002:00003860       ??_C@_0DA@EEOIFEAO@Kraken?5version?5?$CI?2d?$CL?2?4?2d?$CL?$CI?2?4?2d?$CL?$CJ?$DP@ 10027860     KrakenSupport.obj
 0002:00003890       ??_C@_0L@NLHBDLEH@USUPP_PERL?$AA@ 10027890     KrakenSupport.obj
 0002:0000389c       ??_C@_0L@BNJNKHPO@?1jellyfish?$AA@ 1002789c     KrakenSupport.obj
 0002:000038a8       ??_C@_05ODOGGFMP@?1util?$AA@ 100278a8     KrakenSupport.obj
 0002:000038b0       ??_C@_0CN@GJNAPEOC@The?5tool?5is?5used?5to?5build?5a?5Krak@ 100278b0     KrakenSupport.obj
 0002:000038e0       ??_C@_0IP@KFAIBKMK@The?5tool?5is?5used?5to?5classify?5a?5s@ 100278e0     KrakenSupport.obj
 0002:00003974       ??_7KrakenSupportPlugin@U2@@6B@ 10027974     KrakenSupportPlugin.obj
 0002:000039a0       ??_C@_0BN@HDEDDFCB@Kraken?5external?5tool?5support?$AA@ 100279a0     KrakenSupportPlugin.obj
 0002:000039c0       ??_C@_0GM@JPOANEIL@The?5plugin?5supports?5Kraken?3?5taxo@ 100279c0     KrakenSupportPlugin.obj
 0002:00003a30       ??_C@_0FM@HAIBDKME@Kraken?5is?5a?5taxonomic?5sequence?5c@ 10027a30     KrakenSupportPlugin.obj
 0002:00003a90       ??_7KrakenTranslateLogParser@U2@@6B@ 10027a90     KrakenTranslateLogParser.obj
 0002:00003ad8       ??_C@_0P@ODIACOAP@unable?5to?5find?$AA@ 10027ad8     KrakenTranslateLogParser.obj
 0002:00003ae8       ??_C@_0BK@FMDHKPNF@No?5such?5file?5or?5directory?$AA@ 10027ae8     KrakenTranslateLogParser.obj
 0002:00003b04       ??_C@_0CC@LKALPDKM@Use?5of?5uninitialized?5value?5$taxi@ 10027b04     KrakenTranslateLogParser.obj
 0002:00003f88       ?value@?$integral_constant@_N$0A@@std@@2_NB 10027f88     MSVCRT:ti_inst.obj
 0002:00003f89       ?value@?$integral_constant@_N$00@std@@2_NB 10027f89     MSVCRT:ti_inst.obj
 0002:00003f90       ??_7type_info@@6B@         10027f90     MSVCRT:ti_inst.obj
 0002:00003f94       __pDefaultRawDllMain       10027f94     MSVCRT:crtdll.obj
 0002:00003f94       __pRawDllMain              10027f94     MSVCRT:crtdll.obj
 0002:00003fa0       ?ProcessDetach@NativeDll@<CrtImplementationDetails>@@0IB 10027fa0     MSVCRT:initsect.obj
 0002:00003fa4       ?ProcessAttach@NativeDll@<CrtImplementationDetails>@@0IB 10027fa4     MSVCRT:initsect.obj
 0002:00003fa8       ?ThreadAttach@NativeDll@<CrtImplementationDetails>@@0IB 10027fa8     MSVCRT:initsect.obj
 0002:00003fac       ?ThreadDetach@NativeDll@<CrtImplementationDetails>@@0IB 10027fac     MSVCRT:initsect.obj
 0002:00003fb0       ?ProcessVerifier@NativeDll@<CrtImplementationDetails>@@0IB 10027fb0     MSVCRT:initsect.obj
 0002:00003fb8       __load_config_used         10027fb8     MSVCRT:loadcfg.obj
 0002:00004074       ??_R4error_category@std@@6B@ 10028074     DatabaseSizeRelation.obj
 0002:00004088       ??_R3error_category@std@@8 10028088     DatabaseSizeRelation.obj
 0002:00004098       ??_R2error_category@std@@8 10028098     DatabaseSizeRelation.obj
 0002:000040a0       ??_R1A@?0A@EA@error_category@std@@8 100280a0     DatabaseSizeRelation.obj
 0002:000040bc       ??_R4_Generic_error_category@std@@6B@ 100280bc     DatabaseSizeRelation.obj
 0002:000040d0       ??_R3_Generic_error_category@std@@8 100280d0     DatabaseSizeRelation.obj
 0002:000040e0       ??_R2_Generic_error_category@std@@8 100280e0     DatabaseSizeRelation.obj
 0002:000040ec       ??_R1A@?0A@EA@_Generic_error_category@std@@8 100280ec     DatabaseSizeRelation.obj
 0002:00004108       ??_R4_Iostream_error_category@std@@6B@ 10028108     DatabaseSizeRelation.obj
 0002:0000411c       ??_R3_Iostream_error_category@std@@8 1002811c     DatabaseSizeRelation.obj
 0002:0000412c       ??_R2_Iostream_error_category@std@@8 1002812c     DatabaseSizeRelation.obj
 0002:0000413c       ??_R1A@?0A@EA@_Iostream_error_category@std@@8 1002813c     DatabaseSizeRelation.obj
 0002:00004158       ??_R4_System_error_category@std@@6B@ 10028158     DatabaseSizeRelation.obj
 0002:0000416c       ??_R3_System_error_category@std@@8 1002816c     DatabaseSizeRelation.obj
 0002:0000417c       ??_R2_System_error_category@std@@8 1002817c     DatabaseSizeRelation.obj
 0002:0000418c       ??_R1A@?0A@EA@_System_error_category@std@@8 1002818c     DatabaseSizeRelation.obj
 0002:000041a8       ??_R4DatabaseSizeRelation@LocalWorkflow@U2@@6B@ 100281a8     DatabaseSizeRelation.obj
 0002:000041bc       ??_R3DatabaseSizeRelation@LocalWorkflow@U2@@8 100281bc     DatabaseSizeRelation.obj
 0002:000041cc       ??_R2DatabaseSizeRelation@LocalWorkflow@U2@@8 100281cc     DatabaseSizeRelation.obj
 0002:000041dc       ??_R1A@?0A@EA@DatabaseSizeRelation@LocalWorkflow@U2@@8 100281dc     DatabaseSizeRelation.obj
 0002:000041f8       ??_R1A@?0A@EA@ValuesRelation@U2@@8 100281f8     DatabaseSizeRelation.obj
 0002:00004214       ??_R3ValuesRelation@U2@@8  10028214     DatabaseSizeRelation.obj
 0002:00004224       ??_R2ValuesRelation@U2@@8  10028224     DatabaseSizeRelation.obj
 0002:00004230       ??_R1A@?0A@EA@AttributeRelation@U2@@8 10028230     DatabaseSizeRelation.obj
 0002:0000424c       ??_R3AttributeRelation@U2@@8 1002824c     DatabaseSizeRelation.obj
 0002:0000425c       ??_R2AttributeRelation@U2@@8 1002825c     DatabaseSizeRelation.obj
 0002:00004264       ??_R1A@?0A@EA@QObject@@8   10028264     KrakenBuildPrompter.obj
 0002:00004280       ??_R3QObject@@8            10028280     KrakenBuildPrompter.obj
 0002:00004290       ??_R2QObject@@8            10028290     KrakenBuildPrompter.obj
 0002:00004298       ??_R4KrakenBuildPrompter@LocalWorkflow@U2@@6BActorDocument@Workflow@2@@ 10028298     KrakenBuildPrompter.obj
 0002:000042ac       ??_R3KrakenBuildPrompter@LocalWorkflow@U2@@8 100282ac     KrakenBuildPrompter.obj
 0002:000042bc       ??_R2KrakenBuildPrompter@LocalWorkflow@U2@@8 100282bc     KrakenBuildPrompter.obj
 0002:000042dc       ??_R1A@?0A@EA@KrakenBuildPrompter@LocalWorkflow@U2@@8 100282dc     KrakenBuildPrompter.obj
 0002:000042f8       ??_R1A@?0A@EA@?$PrompterBase@VKrakenBuildPrompter@LocalWorkflow@U2@@@U2@@8 100282f8     KrakenBuildPrompter.obj
 0002:00004314       ??_R3?$PrompterBase@VKrakenBuildPrompter@LocalWorkflow@U2@@@U2@@8 10028314     KrakenBuildPrompter.obj
 0002:00004324       ??_R2?$PrompterBase@VKrakenBuildPrompter@LocalWorkflow@U2@@@U2@@8 10028324     KrakenBuildPrompter.obj
 0002:00004340       ??_R1A@?0A@EA@PrompterBaseImpl@U2@@8 10028340     KrakenBuildPrompter.obj
 0002:0000435c       ??_R3PrompterBaseImpl@U2@@8 1002835c     KrakenBuildPrompter.obj
 0002:0000436c       ??_R2PrompterBaseImpl@U2@@8 1002836c     KrakenBuildPrompter.obj
 0002:00004384       ??_R1A@?0A@EA@ActorDocument@Workflow@U2@@8 10028384     KrakenBuildPrompter.obj
 0002:000043a0       ??_R3ActorDocument@Workflow@U2@@8 100283a0     KrakenBuildPrompter.obj
 0002:000043b0       ??_R2ActorDocument@Workflow@U2@@8 100283b0     KrakenBuildPrompter.obj
 0002:000043c0       ??_R1A@?0A@EA@QTextDocument@@8 100283c0     KrakenBuildPrompter.obj
 0002:000043dc       ??_R3QTextDocument@@8      100283dc     KrakenBuildPrompter.obj
 0002:000043ec       ??_R2QTextDocument@@8      100283ec     KrakenBuildPrompter.obj
 0002:000043f8       ??_R1M@?0A@EA@Prompter@Workflow@U2@@8 100283f8     KrakenBuildPrompter.obj
 0002:00004414       ??_R3Prompter@Workflow@U2@@8 10028414     KrakenBuildPrompter.obj
 0002:00004424       ??_R2Prompter@Workflow@U2@@8 10028424     KrakenBuildPrompter.obj
 0002:0000442c       ??_R1A@?0A@EA@Prompter@Workflow@U2@@8 1002842c     KrakenBuildPrompter.obj
 0002:00004448       ??_R4KrakenBuildPrompter@LocalWorkflow@U2@@6BPrompter@Workflow@2@@ 10028448     KrakenBuildPrompter.obj
 0002:0000445c       ??_R4?$PrompterBase@VKrakenBuildPrompter@LocalWorkflow@U2@@@U2@@6BActorDocument@Workflow@1@@ 1002845c     KrakenBuildPrompter.obj
 0002:00004470       ??_R4?$PrompterBase@VKrakenBuildPrompter@LocalWorkflow@U2@@@U2@@6BPrompter@Workflow@1@@ 10028470     KrakenBuildPrompter.obj
 0002:00004484       ??_R4CopyFileTask@U2@@6B@  10028484     KrakenBuildTask.obj
 0002:00004498       ??_R3CopyFileTask@U2@@8    10028498     KrakenBuildTask.obj
 0002:000044a8       ??_R2CopyFileTask@U2@@8    100284a8     KrakenBuildTask.obj
 0002:000044b8       ??_R1A@?0A@EA@CopyFileTask@U2@@8 100284b8     KrakenBuildTask.obj
 0002:000044d4       ??_R1A@?0A@EA@Task@U2@@8   100284d4     KrakenBuildTask.obj
 0002:000044f0       ??_R3Task@U2@@8            100284f0     KrakenBuildTask.obj
 0002:00004500       ??_R2Task@U2@@8            10028500     KrakenBuildTask.obj
 0002:0000450c       ??_R4SequentialMultiTask@U2@@6B@ 1002850c     KrakenBuildTask.obj
 0002:00004520       ??_R3SequentialMultiTask@U2@@8 10028520     KrakenBuildTask.obj
 0002:00004530       ??_R2SequentialMultiTask@U2@@8 10028530     KrakenBuildTask.obj
 0002:00004540       ??_R1A@?0A@EA@SequentialMultiTask@U2@@8 10028540     KrakenBuildTask.obj
 0002:0000455c       ??_R4ExternalToolLogParser@U2@@6B@ 1002855c     KrakenBuildTask.obj
 0002:00004570       ??_R3ExternalToolLogParser@U2@@8 10028570     KrakenBuildTask.obj
 0002:00004580       ??_R2ExternalToolLogParser@U2@@8 10028580     KrakenBuildTask.obj
 0002:0000458c       ??_R1A@?0A@EA@ExternalToolLogParser@U2@@8 1002858c     KrakenBuildTask.obj
 0002:000045a8       ??_R4ExternalToolRunTask@U2@@6B@ 100285a8     KrakenBuildTask.obj
 0002:000045bc       ??_R3ExternalToolRunTask@U2@@8 100285bc     KrakenBuildTask.obj
 0002:000045cc       ??_R2ExternalToolRunTask@U2@@8 100285cc     KrakenBuildTask.obj
 0002:000045dc       ??_R1A@?0A@EA@ExternalToolRunTask@U2@@8 100285dc     KrakenBuildTask.obj
 0002:000045f8       ??_R4KrakenBuildTask@U2@@6B@ 100285f8     KrakenBuildTask.obj
 0002:0000460c       ??_R3KrakenBuildTask@U2@@8 1002860c     KrakenBuildTask.obj
 0002:0000461c       ??_R2KrakenBuildTask@U2@@8 1002861c     KrakenBuildTask.obj
 0002:00004630       ??_R1A@?0A@EA@KrakenBuildTask@U2@@8 10028630     KrakenBuildTask.obj
 0002:0000464c       ??_R1A@?0A@EA@ExternalToolSupportTask@U2@@8 1002864c     KrakenBuildTask.obj
 0002:00004668       ??_R3ExternalToolSupportTask@U2@@8 10028668     KrakenBuildTask.obj
 0002:00004678       ??_R2ExternalToolSupportTask@U2@@8 10028678     KrakenBuildTask.obj
 0002:00004688       ??_R4TaskSignalMapper@U2@@6B@ 10028688     KrakenBuildWorker.obj
 0002:0000469c       ??_R3TaskSignalMapper@U2@@8 1002869c     KrakenBuildWorker.obj
 0002:000046ac       ??_R2TaskSignalMapper@U2@@8 100286ac     KrakenBuildWorker.obj
 0002:000046b8       ??_R1A@?0A@EA@TaskSignalMapper@U2@@8 100286b8     KrakenBuildWorker.obj
 0002:000046d4       ??_R4Descriptor@U2@@6B@    100286d4     KrakenBuildWorker.obj
 0002:000046e8       ??_R3Descriptor@U2@@8      100286e8     KrakenBuildWorker.obj
 0002:000046f8       ??_R2Descriptor@U2@@8      100286f8     KrakenBuildWorker.obj
 0002:00004700       ??_R1A@?0A@EA@Descriptor@U2@@8 10028700     KrakenBuildWorker.obj
 0002:0000471c       ??_R4KrakenBuildWorker@LocalWorkflow@U2@@6BQObject@@@ 1002871c     KrakenBuildWorker.obj
 0002:00004730       ??_R3KrakenBuildWorker@LocalWorkflow@U2@@8 10028730     KrakenBuildWorker.obj
 0002:00004740       ??_R2KrakenBuildWorker@LocalWorkflow@U2@@8 10028740     KrakenBuildWorker.obj
 0002:00004758       ??_R1A@?0A@EA@KrakenBuildWorker@LocalWorkflow@U2@@8 10028758     KrakenBuildWorker.obj
 0002:00004774       ??_R1A@?0A@EA@BaseWorker@LocalWorkflow@U2@@8 10028774     KrakenBuildWorker.obj
 0002:00004790       ??_R3BaseWorker@LocalWorkflow@U2@@8 10028790     KrakenBuildWorker.obj
 0002:000047a0       ??_R2BaseWorker@LocalWorkflow@U2@@8 100287a0     KrakenBuildWorker.obj
 0002:000047b4       ??_R17?0A@EA@Worker@Workflow@U2@@8 100287b4     KrakenBuildWorker.obj
 0002:000047d0       ??_R3Worker@Workflow@U2@@8 100287d0     KrakenBuildWorker.obj
 0002:000047e0       ??_R2Worker@Workflow@U2@@8 100287e0     KrakenBuildWorker.obj
 0002:000047e8       ??_R1A@?0A@EA@Worker@Workflow@U2@@8 100287e8     KrakenBuildWorker.obj
 0002:00004804       ??_R1BA@?0A@EA@CommunicationSubject@Workflow@U2@@8 10028804     KrakenBuildWorker.obj
 0002:00004820       ??_R3CommunicationSubject@Workflow@U2@@8 10028820     KrakenBuildWorker.obj
 0002:00004830       ??_R2CommunicationSubject@Workflow@U2@@8 10028830     KrakenBuildWorker.obj
 0002:00004838       ??_R1A@?0A@EA@CommunicationSubject@Workflow@U2@@8 10028838     KrakenBuildWorker.obj
 0002:00004854       ??_R4KrakenBuildWorker@LocalWorkflow@U2@@6BWorker@Workflow@2@@ 10028854     KrakenBuildWorker.obj
 0002:00004868       ??_R4KrakenBuildWorker@LocalWorkflow@U2@@6BCommunicationSubject@Workflow@2@@ 10028868     KrakenBuildWorker.obj
 0002:0000487c       ??_R4VisibilityRelation@U2@@6B@ 1002887c     KrakenBuildWorkerFactory.obj
 0002:00004890       ??_R3VisibilityRelation@U2@@8 10028890     KrakenBuildWorkerFactory.obj
 0002:000048a0       ??_R2VisibilityRelation@U2@@8 100288a0     KrakenBuildWorkerFactory.obj
 0002:000048ac       ??_R1A@?0A@EA@VisibilityRelation@U2@@8 100288ac     KrakenBuildWorkerFactory.obj
 0002:000048c8       ??_R4MapDataType@U2@@6B@   100288c8     KrakenBuildWorkerFactory.obj
 0002:000048dc       ??_R3MapDataType@U2@@8     100288dc     KrakenBuildWorkerFactory.obj
 0002:000048ec       ??_R2MapDataType@U2@@8     100288ec     KrakenBuildWorkerFactory.obj
 0002:00004900       ??_R1A@?0A@EA@MapDataType@U2@@8 10028900     KrakenBuildWorkerFactory.obj
 0002:0000491c       ??_R1A@?0A@EA@DataType@U2@@8 1002891c     KrakenBuildWorkerFactory.obj
 0002:00004938       ??_R3DataType@U2@@8        10028938     KrakenBuildWorkerFactory.obj
 0002:00004948       ??_R2DataType@U2@@8        10028948     KrakenBuildWorkerFactory.obj
 0002:00004958       ??_R1BA@?0A@EA@QSharedData@@8 10028958     KrakenBuildWorkerFactory.obj
 0002:00004974       ??_R3QSharedData@@8        10028974     KrakenBuildWorkerFactory.obj
 0002:00004984       ??_R2QSharedData@@8        10028984     KrakenBuildWorkerFactory.obj
 0002:0000498c       ??_R1A@?0A@EA@QSharedData@@8 1002898c     KrakenBuildWorkerFactory.obj
 0002:000049a8       ??_R4Attribute@U2@@6B@     100289a8     KrakenBuildWorkerFactory.obj
 0002:000049bc       ??_R3Attribute@U2@@8       100289bc     KrakenBuildWorkerFactory.obj
 0002:000049cc       ??_R2Attribute@U2@@8       100289cc     KrakenBuildWorkerFactory.obj
 0002:000049d8       ??_R1A@?0A@EA@Attribute@U2@@8 100289d8     KrakenBuildWorkerFactory.obj
 0002:000049f4       ??_R3ConfigurationEditor@U2@@8 100289f4     KrakenBuildWorkerFactory.obj
 0002:00004a04       ??_R2ConfigurationEditor@U2@@8 10028a04     KrakenBuildWorkerFactory.obj
 0002:00004a10       ??_R1A@?0A@EA@ConfigurationEditor@U2@@8 10028a10     KrakenBuildWorkerFactory.obj
 0002:00004a2c       ??_R4DelegateEditor@U2@@6B@ 10028a2c     KrakenBuildWorkerFactory.obj
 0002:00004a40       ??_R3DelegateEditor@U2@@8  10028a40     KrakenBuildWorkerFactory.obj
 0002:00004a50       ??_R2DelegateEditor@U2@@8  10028a50     KrakenBuildWorkerFactory.obj
 0002:00004a60       ??_R1A@?0A@EA@DelegateEditor@U2@@8 10028a60     KrakenBuildWorkerFactory.obj
 0002:00004a7c       ??_R4URLDelegate@U2@@6B@   10028a7c     KrakenBuildWorkerFactory.obj
 0002:00004a90       ??_R3URLDelegate@U2@@8     10028a90     KrakenBuildWorkerFactory.obj
 0002:00004aa0       ??_R2URLDelegate@U2@@8     10028aa0     KrakenBuildWorkerFactory.obj
 0002:00004ab8       ??_R1A@?0A@EA@URLDelegate@U2@@8 10028ab8     KrakenBuildWorkerFactory.obj
 0002:00004ad4       ??_R1A@?0A@EA@PropertyDelegate@U2@@8 10028ad4     KrakenBuildWorkerFactory.obj
 0002:00004af0       ??_R3PropertyDelegate@U2@@8 10028af0     KrakenBuildWorkerFactory.obj
 0002:00004b00       ??_R2PropertyDelegate@U2@@8 10028b00     KrakenBuildWorkerFactory.obj
 0002:00004b14       ??_R1A@?0A@EA@QItemDelegate@@8 10028b14     KrakenBuildWorkerFactory.obj
 0002:00004b30       ??_R3QItemDelegate@@8      10028b30     KrakenBuildWorkerFactory.obj
 0002:00004b40       ??_R2QItemDelegate@@8      10028b40     KrakenBuildWorkerFactory.obj
 0002:00004b50       ??_R1A@?0A@EA@QAbstractItemDelegate@@8 10028b50     KrakenBuildWorkerFactory.obj
 0002:00004b6c       ??_R3QAbstractItemDelegate@@8 10028b6c     KrakenBuildWorkerFactory.obj
 0002:00004b7c       ??_R2QAbstractItemDelegate@@8 10028b7c     KrakenBuildWorkerFactory.obj
 0002:00004b88       ??_R4SpinBoxDelegate@U2@@6B@ 10028b88     KrakenBuildWorkerFactory.obj
 0002:00004b9c       ??_R3SpinBoxDelegate@U2@@8 10028b9c     KrakenBuildWorkerFactory.obj
 0002:00004bac       ??_R2SpinBoxDelegate@U2@@8 10028bac     KrakenBuildWorkerFactory.obj
 0002:00004bc4       ??_R1A@?0A@EA@SpinBoxDelegate@U2@@8 10028bc4     KrakenBuildWorkerFactory.obj
 0002:00004be0       ??_R4ComboBoxDelegate@U2@@6B@ 10028be0     KrakenBuildWorkerFactory.obj
 0002:00004bf4       ??_R3ComboBoxDelegate@U2@@8 10028bf4     KrakenBuildWorkerFactory.obj
 0002:00004c04       ??_R2ComboBoxDelegate@U2@@8 10028c04     KrakenBuildWorkerFactory.obj
 0002:00004c1c       ??_R1A@?0A@EA@ComboBoxDelegate@U2@@8 10028c1c     KrakenBuildWorkerFactory.obj
 0002:00004c38       ??_R4ComboBoxWithBoolsDelegate@U2@@6B@ 10028c38     KrakenBuildWorkerFactory.obj
 0002:00004c4c       ??_R3ComboBoxWithBoolsDelegate@U2@@8 10028c4c     KrakenBuildWorkerFactory.obj
 0002:00004c5c       ??_R2ComboBoxWithBoolsDelegate@U2@@8 10028c5c     KrakenBuildWorkerFactory.obj
 0002:00004c78       ??_R1A@?0A@EA@ComboBoxWithBoolsDelegate@U2@@8 10028c78     KrakenBuildWorkerFactory.obj
 0002:00004c94       ??_R4PortDescriptor@Workflow@U2@@6B@ 10028c94     KrakenBuildWorkerFactory.obj
 0002:00004ca8       ??_R3PortDescriptor@Workflow@U2@@8 10028ca8     KrakenBuildWorkerFactory.obj
 0002:00004cb8       ??_R2PortDescriptor@Workflow@U2@@8 10028cb8     KrakenBuildWorkerFactory.obj
 0002:00004cc4       ??_R1A@?0A@EA@PortDescriptor@Workflow@U2@@8 10028cc4     KrakenBuildWorkerFactory.obj
 0002:00004ce0       ??_R17?0A@EA@Descriptor@U2@@8 10028ce0     KrakenBuildWorkerFactory.obj
 0002:00004cfc       ??_R4IntegralBusActorPrototype@Workflow@U2@@6BQObject@@@ 10028cfc     KrakenBuildWorkerFactory.obj
 0002:00004d10       ??_R3IntegralBusActorPrototype@Workflow@U2@@8 10028d10     KrakenBuildWorkerFactory.obj
 0002:00004d20       ??_R2IntegralBusActorPrototype@Workflow@U2@@8 10028d20     KrakenBuildWorkerFactory.obj
 0002:00004d38       ??_R1A@?0A@EA@IntegralBusActorPrototype@Workflow@U2@@8 10028d38     KrakenBuildWorkerFactory.obj
 0002:00004d54       ??_R1A@?0A@EA@ActorPrototype@Workflow@U2@@8 10028d54     KrakenBuildWorkerFactory.obj
 0002:00004d70       ??_R3ActorPrototype@Workflow@U2@@8 10028d70     KrakenBuildWorkerFactory.obj
 0002:00004d80       ??_R2ActorPrototype@Workflow@U2@@8 10028d80     KrakenBuildWorkerFactory.obj
 0002:00004d94       ??_R17?0A@EA@VisualDescriptor@U2@@8 10028d94     KrakenBuildWorkerFactory.obj
 0002:00004db0       ??_R3VisualDescriptor@U2@@8 10028db0     KrakenBuildWorkerFactory.obj
 0002:00004dc0       ??_R2VisualDescriptor@U2@@8 10028dc0     KrakenBuildWorkerFactory.obj
 0002:00004dcc       ??_R1A@?0A@EA@VisualDescriptor@U2@@8 10028dcc     KrakenBuildWorkerFactory.obj
 0002:00004de8       ??_R4IntegralBusActorPrototype@Workflow@U2@@6BVisualDescriptor@2@@ 10028de8     KrakenBuildWorkerFactory.obj
 0002:00004dfc       ??_R4KrakenBuildValidator@Workflow@U2@@6B@ 10028dfc     KrakenBuildWorkerFactory.obj
 0002:00004e10       ??_R3KrakenBuildValidator@Workflow@U2@@8 10028e10     KrakenBuildWorkerFactory.obj
 0002:00004e20       ??_R2KrakenBuildValidator@Workflow@U2@@8 10028e20     KrakenBuildWorkerFactory.obj
 0002:00004e30       ??_R1A@?0A@EA@KrakenBuildValidator@Workflow@U2@@8 10028e30     KrakenBuildWorkerFactory.obj
 0002:00004e4c       ??_R1A@?0A@EA@ActorValidator@Workflow@U2@@8 10028e4c     KrakenBuildWorkerFactory.obj
 0002:00004e68       ??_R3ActorValidator@Workflow@U2@@8 10028e68     KrakenBuildWorkerFactory.obj
 0002:00004e78       ??_R2ActorValidator@Workflow@U2@@8 10028e78     KrakenBuildWorkerFactory.obj
 0002:00004e84       ??_R1A@?0A@EA@ConfigurationValidator@U2@@8 10028e84     KrakenBuildWorkerFactory.obj
 0002:00004ea0       ??_R3ConfigurationValidator@U2@@8 10028ea0     KrakenBuildWorkerFactory.obj
 0002:00004eb0       ??_R2ConfigurationValidator@U2@@8 10028eb0     KrakenBuildWorkerFactory.obj
 0002:00004eb8       ??_R4KrakenBuildWorkerFactory@LocalWorkflow@U2@@6B?$IdRegistry@VDomainFactory@Workflow@U2@@@2@@ 10028eb8     KrakenBuildWorkerFactory.obj
 0002:00004ecc       ??_R3KrakenBuildWorkerFactory@LocalWorkflow@U2@@8 10028ecc     KrakenBuildWorkerFactory.obj
 0002:00004edc       ??_R2KrakenBuildWorkerFactory@LocalWorkflow@U2@@8 10028edc     KrakenBuildWorkerFactory.obj
 0002:00004ef0       ??_R1A@?0A@EA@KrakenBuildWorkerFactory@LocalWorkflow@U2@@8 10028ef0     KrakenBuildWorkerFactory.obj
 0002:00004f0c       ??_R1A@?0A@EA@DomainFactory@Workflow@U2@@8 10028f0c     KrakenBuildWorkerFactory.obj
 0002:00004f28       ??_R3DomainFactory@Workflow@U2@@8 10028f28     KrakenBuildWorkerFactory.obj
 0002:00004f38       ??_R2DomainFactory@Workflow@U2@@8 10028f38     KrakenBuildWorkerFactory.obj
 0002:00004f48       ??_R1A@?0A@EA@?$IdRegistry@VDomainFactory@Workflow@U2@@@U2@@8 10028f48     KrakenBuildWorkerFactory.obj
 0002:00004f64       ??_R3?$IdRegistry@VDomainFactory@Workflow@U2@@@U2@@8 10028f64     KrakenBuildWorkerFactory.obj
 0002:00004f74       ??_R2?$IdRegistry@VDomainFactory@Workflow@U2@@@U2@@8 10028f74     KrakenBuildWorkerFactory.obj
 0002:00004f7c       ??_R4KrakenBuildWorkerFactory@LocalWorkflow@U2@@6BDescriptor@2@@ 10028f7c     KrakenBuildWorkerFactory.obj
 0002:00004f90       ??_R4GenomicLibraryDelegate@LocalWorkflow@U2@@6B@ 10028f90     KrakenBuildWorkerFactory.obj
 0002:00004fa4       ??_R3GenomicLibraryDelegate@LocalWorkflow@U2@@8 10028fa4     KrakenBuildWorkerFactory.obj
 0002:00004fb4       ??_R2GenomicLibraryDelegate@LocalWorkflow@U2@@8 10028fb4     KrakenBuildWorkerFactory.obj
 0002:00004fcc       ??_R1A@?0A@EA@GenomicLibraryDelegate@LocalWorkflow@U2@@8 10028fcc     KrakenBuildWorkerFactory.obj
 0002:00004fe8       ??_R4KrakenClassifyLogParser@U2@@6B@ 10028fe8     KrakenClassifyLogParser.obj
 0002:00004ffc       ??_R3KrakenClassifyLogParser@U2@@8 10028ffc     KrakenClassifyLogParser.obj
 0002:0000500c       ??_R2KrakenClassifyLogParser@U2@@8 1002900c     KrakenClassifyLogParser.obj
 0002:0000501c       ??_R1A@?0A@EA@KrakenClassifyLogParser@U2@@8 1002901c     KrakenClassifyLogParser.obj
 0002:00005038       ??_R4KrakenClassifyPrompter@LocalWorkflow@U2@@6BActorDocument@Workflow@2@@ 10029038     KrakenClassifyPrompter.obj
 0002:0000504c       ??_R3KrakenClassifyPrompter@LocalWorkflow@U2@@8 1002904c     KrakenClassifyPrompter.obj
 0002:0000505c       ??_R2KrakenClassifyPrompter@LocalWorkflow@U2@@8 1002905c     KrakenClassifyPrompter.obj
 0002:0000507c       ??_R1A@?0A@EA@KrakenClassifyPrompter@LocalWorkflow@U2@@8 1002907c     KrakenClassifyPrompter.obj
 0002:00005098       ??_R1A@?0A@EA@?$PrompterBase@VKrakenClassifyPrompter@LocalWorkflow@U2@@@U2@@8 10029098     KrakenClassifyPrompter.obj
 0002:000050b4       ??_R3?$PrompterBase@VKrakenClassifyPrompter@LocalWorkflow@U2@@@U2@@8 100290b4     KrakenClassifyPrompter.obj
 0002:000050c4       ??_R2?$PrompterBase@VKrakenClassifyPrompter@LocalWorkflow@U2@@@U2@@8 100290c4     KrakenClassifyPrompter.obj
 0002:000050e0       ??_R4KrakenClassifyPrompter@LocalWorkflow@U2@@6BPrompter@Workflow@2@@ 100290e0     KrakenClassifyPrompter.obj
 0002:000050f4       ??_R4?$PrompterBase@VKrakenClassifyPrompter@LocalWorkflow@U2@@@U2@@6BActorDocument@Workflow@1@@ 100290f4     KrakenClassifyPrompter.obj
 0002:00005108       ??_R4?$PrompterBase@VKrakenClassifyPrompter@LocalWorkflow@U2@@@U2@@6BPrompter@Workflow@1@@ 10029108     KrakenClassifyPrompter.obj
 0002:0000511c       ??_R4KrakenClassifyTask@U2@@6B@ 1002911c     KrakenClassifyTask.obj
 0002:00005130       ??_R3KrakenClassifyTask@U2@@8 10029130     KrakenClassifyTask.obj
 0002:00005140       ??_R2KrakenClassifyTask@U2@@8 10029140     KrakenClassifyTask.obj
 0002:00005154       ??_R1A@?0A@EA@KrakenClassifyTask@U2@@8 10029154     KrakenClassifyTask.obj
 0002:00005170       ??_R4FailTask@U2@@6B@      10029170     KrakenClassifyWorker.obj
 0002:00005184       ??_R3FailTask@U2@@8        10029184     KrakenClassifyWorker.obj
 0002:00005194       ??_R2FailTask@U2@@8        10029194     KrakenClassifyWorker.obj
 0002:000051a4       ??_R1A@?0A@EA@FailTask@U2@@8 100291a4     KrakenClassifyWorker.obj
 0002:000051c0       ??_R4KrakenClassifyWorker@LocalWorkflow@U2@@6BQObject@@@ 100291c0     KrakenClassifyWorker.obj
 0002:000051d4       ??_R3KrakenClassifyWorker@LocalWorkflow@U2@@8 100291d4     KrakenClassifyWorker.obj
 0002:000051e4       ??_R2KrakenClassifyWorker@LocalWorkflow@U2@@8 100291e4     KrakenClassifyWorker.obj
 0002:000051fc       ??_R1A@?0A@EA@KrakenClassifyWorker@LocalWorkflow@U2@@8 100291fc     KrakenClassifyWorker.obj
 0002:00005218       ??_R4KrakenClassifyWorker@LocalWorkflow@U2@@6BWorker@Workflow@2@@ 10029218     KrakenClassifyWorker.obj
 0002:0000522c       ??_R4KrakenClassifyWorker@LocalWorkflow@U2@@6BCommunicationSubject@Workflow@2@@ 1002922c     KrakenClassifyWorker.obj
 0002:00005240       ??_R4SlotRelationDescriptor@U2@@6B@ 10029240     KrakenClassifyWorkerFactory.obj
 0002:00005254       ??_R3SlotRelationDescriptor@U2@@8 10029254     KrakenClassifyWorkerFactory.obj
 0002:00005264       ??_R2SlotRelationDescriptor@U2@@8 10029264     KrakenClassifyWorkerFactory.obj
 0002:0000526c       ??_R1A@?0A@EA@SlotRelationDescriptor@U2@@8 1002926c     KrakenClassifyWorkerFactory.obj
 0002:00005288       ??_R4PairedReadsPortValidator@Workflow@U2@@6B@ 10029288     KrakenClassifyWorkerFactory.obj
 0002:0000529c       ??_R3PairedReadsPortValidator@Workflow@U2@@8 1002929c     KrakenClassifyWorkerFactory.obj
 0002:000052ac       ??_R2PairedReadsPortValidator@Workflow@U2@@8 100292ac     KrakenClassifyWorkerFactory.obj
 0002:000052bc       ??_R1A@?0A@EA@PairedReadsPortValidator@Workflow@U2@@8 100292bc     KrakenClassifyWorkerFactory.obj
 0002:000052d8       ??_R1A@?0A@EA@PortValidator@Workflow@U2@@8 100292d8     KrakenClassifyWorkerFactory.obj
 0002:000052f4       ??_R3PortValidator@Workflow@U2@@8 100292f4     KrakenClassifyWorkerFactory.obj
 0002:00005304       ??_R2PortValidator@Workflow@U2@@8 10029304     KrakenClassifyWorkerFactory.obj
 0002:00005310       ??_R4KrakenClassifyValidator@Workflow@U2@@6B@ 10029310     KrakenClassifyWorkerFactory.obj
 0002:00005324       ??_R3KrakenClassifyValidator@Workflow@U2@@8 10029324     KrakenClassifyWorkerFactory.obj
 0002:00005334       ??_R2KrakenClassifyValidator@Workflow@U2@@8 10029334     KrakenClassifyWorkerFactory.obj
 0002:00005344       ??_R1A@?0A@EA@KrakenClassifyValidator@Workflow@U2@@8 10029344     KrakenClassifyWorkerFactory.obj
 0002:00005360       ??_R4KrakenClassifyWorkerFactory@LocalWorkflow@U2@@6B?$IdRegistry@VDomainFactory@Workflow@U2@@@2@@ 10029360     KrakenClassifyWorkerFactory.obj
 0002:00005374       ??_R3KrakenClassifyWorkerFactory@LocalWorkflow@U2@@8 10029374     KrakenClassifyWorkerFactory.obj
 0002:00005384       ??_R2KrakenClassifyWorkerFactory@LocalWorkflow@U2@@8 10029384     KrakenClassifyWorkerFactory.obj
 0002:00005398       ??_R1A@?0A@EA@KrakenClassifyWorkerFactory@LocalWorkflow@U2@@8 10029398     KrakenClassifyWorkerFactory.obj
 0002:000053b4       ??_R4KrakenClassifyWorkerFactory@LocalWorkflow@U2@@6BDescriptor@2@@ 100293b4     KrakenClassifyWorkerFactory.obj
 0002:000053c8       ??_R4DatabaseDelegate@LocalWorkflow@U2@@6B@ 100293c8     KrakenClassifyWorkerFactory.obj
 0002:000053dc       ??_R3DatabaseDelegate@LocalWorkflow@U2@@8 100293dc     KrakenClassifyWorkerFactory.obj
 0002:000053ec       ??_R2DatabaseDelegate@LocalWorkflow@U2@@8 100293ec     KrakenClassifyWorkerFactory.obj
 0002:00005408       ??_R1A@?0A@EA@DatabaseDelegate@LocalWorkflow@U2@@8 10029408     KrakenClassifyWorkerFactory.obj
 0002:00005424       ??_R4KrakenSupport@U2@@6B@ 10029424     KrakenSupport.obj
 0002:00005438       ??_R3KrakenSupport@U2@@8   10029438     KrakenSupport.obj
 0002:00005448       ??_R2KrakenSupport@U2@@8   10029448     KrakenSupport.obj
 0002:00005458       ??_R1A@?0A@EA@KrakenSupport@U2@@8 10029458     KrakenSupport.obj
 0002:00005474       ??_R1A@?0A@EA@ExternalTool@U2@@8 10029474     KrakenSupport.obj
 0002:00005490       ??_R3ExternalTool@U2@@8    10029490     KrakenSupport.obj
 0002:000054a0       ??_R2ExternalTool@U2@@8    100294a0     KrakenSupport.obj
 0002:000054ac       ??_R4KrakenSupportPlugin@U2@@6B@ 100294ac     KrakenSupportPlugin.obj
 0002:000054c0       ??_R3KrakenSupportPlugin@U2@@8 100294c0     KrakenSupportPlugin.obj
 0002:000054d0       ??_R2KrakenSupportPlugin@U2@@8 100294d0     KrakenSupportPlugin.obj
 0002:000054e0       ??_R1A@?0A@EA@KrakenSupportPlugin@U2@@8 100294e0     KrakenSupportPlugin.obj
 0002:000054fc       ??_R1A@?0A@EA@Plugin@U2@@8 100294fc     KrakenSupportPlugin.obj
 0002:00005518       ??_R3Plugin@U2@@8          10029518     KrakenSupportPlugin.obj
 0002:00005528       ??_R2Plugin@U2@@8          10029528     KrakenSupportPlugin.obj
 0002:00005534       ??_R4KrakenTranslateLogParser@U2@@6B@ 10029534     KrakenTranslateLogParser.obj
 0002:00005548       ??_R3KrakenTranslateLogParser@U2@@8 10029548     KrakenTranslateLogParser.obj
 0002:00005558       ??_R2KrakenTranslateLogParser@U2@@8 10029558     KrakenTranslateLogParser.obj
 0002:00005568       ??_R1A@?0A@EA@KrakenTranslateLogParser@U2@@8 10029568     KrakenTranslateLogParser.obj
 0002:00005584       ??_R4type_info@@6B@        10029584     MSVCRT:ti_inst.obj
 0002:00005598       ??_R3type_info@@8          10029598     MSVCRT:ti_inst.obj
 0002:000055a8       ??_R2type_info@@8          100295a8     MSVCRT:ti_inst.obj
 0002:000055b0       ??_R1A@?0A@EA@type_info@@8 100295b0     MSVCRT:ti_inst.obj
 0002:000055d0       ___safe_se_handler_table   100295d0     <linker-defined>
 0002:00005a74       ___rtc_iaa                 10029a74     MSVCRT:initsect.obj
 0002:00005a78       ___rtc_izz                 10029a78     MSVCRT:initsect.obj
 0002:00005a7c       ___rtc_taa                 10029a7c     MSVCRT:initsect.obj
 0002:00005a80       ___rtc_tzz                 10029a80     MSVCRT:initsect.obj
 0002:0000b488       __IMPORT_DESCRIPTOR_U2Core 1002f488     U2Core:U2Core.dll
 0002:0000b49c       __IMPORT_DESCRIPTOR_U2Gui  1002f49c     U2Gui:U2Gui.dll
 0002:0000b4b0       __IMPORT_DESCRIPTOR_U2Lang 1002f4b0     U2Lang:U2Lang.dll
 0002:0000b4c4       __IMPORT_DESCRIPTOR_U2Designer 1002f4c4     U2Designer:U2Designer.dll
 0002:0000b4d8       __IMPORT_DESCRIPTOR_ngs_reads_classification 1002f4d8     ngs_reads_classification:ngs_reads_classification.dll
 0002:0000b4ec       __IMPORT_DESCRIPTOR_Qt5Widgets 1002f4ec     Qt5Widgets:Qt5Widgets.dll
 0002:0000b500       __IMPORT_DESCRIPTOR_Qt5Gui 1002f500     Qt5Gui:Qt5Gui.dll
 0002:0000b514       __IMPORT_DESCRIPTOR_Qt5Script 1002f514     Qt5Script:Qt5Script.dll
 0002:0000b528       __IMPORT_DESCRIPTOR_Qt5Core 1002f528     Qt5Core:Qt5Core.dll
 0002:0000b53c       __IMPORT_DESCRIPTOR_MSVCP120 1002f53c     msvcprt:MSVCP120.dll
 0002:0000b550       __IMPORT_DESCRIPTOR_MSVCR120 1002f550     MSVCRT:MSVCR120.dll
 0002:0000b564       __IMPORT_DESCRIPTOR_KERNEL32 1002f564     kernel32:KERNEL32.dll
 0002:0000b578       __NULL_IMPORT_DESCRIPTOR   1002f578     U2Core:U2Core.dll
 0003:00000000       ?_Generic_object@?$_Error_objects@H@std@@2V_Generic_error_category@2@A 10038000     DatabaseSizeRelation.obj
 0003:00000004       ?_Iostream_object@?$_Error_objects@H@std@@2V_Iostream_error_category@2@A 10038004     DatabaseSizeRelation.obj
 0003:00000008       ?_System_object@?$_Error_objects@H@std@@2V_System_error_category@2@A 10038008     DatabaseSizeRelation.obj
 0003:0000000c       ?staticMetaObject@KrakenBuildPrompter@LocalWorkflow@U2@@2UQMetaObject@@B 1003800c     moc_KrakenBuildPrompter.obj
 0003:00000024       ?staticMetaObject@KrakenBuildTask@U2@@2UQMetaObject@@B 10038024     moc_KrakenBuildTask.obj
 0003:0000003c       ?staticMetaObject@KrakenBuildWorker@LocalWorkflow@U2@@2UQMetaObject@@B 1003803c     moc_KrakenBuildWorker.obj
 0003:00000054       ?staticMetaObject@KrakenClassifyPrompter@LocalWorkflow@U2@@2UQMetaObject@@B 10038054     moc_KrakenClassifyPrompter.obj
 0003:0000006c       ?staticMetaObject@KrakenClassifyTask@U2@@2UQMetaObject@@B 1003806c     moc_KrakenClassifyTask.obj
 0003:00000084       ?staticMetaObject@KrakenClassifyWorker@LocalWorkflow@U2@@2UQMetaObject@@B 10038084     moc_KrakenClassifyWorker.obj
 0003:0000009c       ?staticMetaObject@KrakenSupport@U2@@2UQMetaObject@@B 1003809c     moc_KrakenSupport.obj
 0003:000000b4       ?staticMetaObject@KrakenSupportPlugin@U2@@2UQMetaObject@@B 100380b4     moc_KrakenSupportPlugin.obj
 0003:000000cc       ___security_cookie         100380cc     MSVCRT:gs_cookie.obj
 0003:000000d0       ___security_cookie_complement 100380d0     MSVCRT:gs_cookie.obj
 0003:000000e0       ___native_dllmain_reason   100380e0     MSVCRT:natstart.obj
 0003:000000e8       ??_R0?AVerror_category@std@@@8 100380e8     DatabaseSizeRelation.obj
 0003:0000010c       ??_R0?AV_Generic_error_category@std@@@8 1003810c     DatabaseSizeRelation.obj
 0003:00000138       ??_R0?AV_Iostream_error_category@std@@@8 10038138     DatabaseSizeRelation.obj
 0003:00000164       ??_R0?AV_System_error_category@std@@@8 10038164     DatabaseSizeRelation.obj
 0003:00000190       ??_R0?AVDatabaseSizeRelation@LocalWorkflow@U2@@@8 10038190     DatabaseSizeRelation.obj
 0003:000001c4       ??_R0?AVValuesRelation@U2@@@8 100381c4     DatabaseSizeRelation.obj
 0003:000001e4       ??_R0?AVAttributeRelation@U2@@@8 100381e4     DatabaseSizeRelation.obj
 0003:00000208       ??_R0?AVQObject@@@8        10038208     KrakenBuildPrompter.obj
 0003:00000220       ??_R0?AVKrakenBuildPrompter@LocalWorkflow@U2@@@8 10038220     KrakenBuildPrompter.obj
 0003:00000258       ??_R0?AV?$PrompterBase@VKrakenBuildPrompter@LocalWorkflow@U2@@@U2@@@8 10038258     KrakenBuildPrompter.obj
 0003:000002a0       ??_R0?AVPrompterBaseImpl@U2@@@8 100382a0     KrakenBuildPrompter.obj
 0003:000002c4       ??_R0?AVActorDocument@Workflow@U2@@@8 100382c4     KrakenBuildPrompter.obj
 0003:000002ec       ??_R0?AVQTextDocument@@@8  100382ec     KrakenBuildPrompter.obj
 0003:00000308       ??_R0?AVPrompter@Workflow@U2@@@8 10038308     KrakenBuildPrompter.obj
 0003:0000032c       ??_R0?AVCopyFileTask@U2@@@8 1003832c     KrakenBuildTask.obj
 0003:0000034c       ??_R0?AVTask@U2@@@8        1003834c     KrakenBuildTask.obj
 0003:00000364       ??_R0?AVSequentialMultiTask@U2@@@8 10038364     KrakenBuildTask.obj
 0003:0000038c       ??_R0?AVExternalToolLogParser@U2@@@8 1003838c     KrakenBuildTask.obj
 0003:000003b4       ??_R0?AVExternalToolRunTask@U2@@@8 100383b4     KrakenBuildTask.obj
 0003:000003dc       ??_R0?AVKrakenBuildTask@U2@@@8 100383dc     KrakenBuildTask.obj
 0003:00000400       ??_R0?AVExternalToolSupportTask@U2@@@8 10038400     KrakenBuildTask.obj
 0003:0000042c       ??_R0?AVTaskSignalMapper@U2@@@8 1003842c     KrakenBuildWorker.obj
 0003:00000450       ??_R0?AVDescriptor@U2@@@8  10038450     KrakenBuildWorker.obj
 0003:0000046c       ??_R0?AVKrakenBuildWorker@LocalWorkflow@U2@@@8 1003846c     KrakenBuildWorker.obj
 0003:000004a0       ??_R0?AVBaseWorker@LocalWorkflow@U2@@@8 100384a0     KrakenBuildWorker.obj
 0003:000004cc       ??_R0?AVWorker@Workflow@U2@@@8 100384cc     KrakenBuildWorker.obj
 0003:000004f0       ??_R0?AVCommunicationSubject@Workflow@U2@@@8 100384f0     KrakenBuildWorker.obj
 0003:00000520       ??_R0?AVVisibilityRelation@U2@@@8 10038520     KrakenBuildWorkerFactory.obj
 0003:00000544       ??_R0?AVMapDataType@U2@@@8 10038544     KrakenBuildWorkerFactory.obj
 0003:00000564       ??_R0?AVDataType@U2@@@8    10038564     KrakenBuildWorkerFactory.obj
 0003:00000580       ??_R0?AVQSharedData@@@8    10038580     KrakenBuildWorkerFactory.obj
 0003:0000059c       ??_R0?AVAttribute@U2@@@8   1003859c     KrakenBuildWorkerFactory.obj
 0003:000005b8       ??_R0?AVConfigurationEditor@U2@@@8 100385b8     KrakenBuildWorkerFactory.obj
 0003:000005e0       ??_R0?AVDelegateEditor@U2@@@8 100385e0     KrakenBuildWorkerFactory.obj
 0003:00000600       ??_R0?AVURLDelegate@U2@@@8 10038600     KrakenBuildWorkerFactory.obj
 0003:00000620       ??_R0?AVPropertyDelegate@U2@@@8 10038620     KrakenBuildWorkerFactory.obj
 0003:00000644       ??_R0?AVQItemDelegate@@@8  10038644     KrakenBuildWorkerFactory.obj
 0003:00000660       ??_R0?AVQAbstractItemDelegate@@@8 10038660     KrakenBuildWorkerFactory.obj
 0003:00000684       ??_R0?AVSpinBoxDelegate@U2@@@8 10038684     KrakenBuildWorkerFactory.obj
 0003:000006a8       ??_R0?AVComboBoxDelegate@U2@@@8 100386a8     KrakenBuildWorkerFactory.obj
 0003:000006cc       ??_R0?AVComboBoxWithBoolsDelegate@U2@@@8 100386cc     KrakenBuildWorkerFactory.obj
 0003:000006f8       ??_R0?AVPortDescriptor@Workflow@U2@@@8 100386f8     KrakenBuildWorkerFactory.obj
 0003:00000724       ??_R0?AVIntegralBusActorPrototype@Workflow@U2@@@8 10038724     KrakenBuildWorkerFactory.obj
 0003:00000758       ??_R0?AVActorPrototype@Workflow@U2@@@8 10038758     KrakenBuildWorkerFactory.obj
 0003:00000784       ??_R0?AVVisualDescriptor@U2@@@8 10038784     KrakenBuildWorkerFactory.obj
 0003:000007a8       ??_R0?AVKrakenBuildValidator@Workflow@U2@@@8 100387a8     KrakenBuildWorkerFactory.obj
 0003:000007d8       ??_R0?AVActorValidator@Workflow@U2@@@8 100387d8     KrakenBuildWorkerFactory.obj
 0003:00000804       ??_R0?AVConfigurationValidator@U2@@@8 10038804     KrakenBuildWorkerFactory.obj
 0003:0000082c       ??_R0?AVKrakenBuildWorkerFactory@LocalWorkflow@U2@@@8 1003882c     KrakenBuildWorkerFactory.obj
 0003:00000864       ??_R0?AVDomainFactory@Workflow@U2@@@8 10038864     KrakenBuildWorkerFactory.obj
 0003:0000088c       ??_R0?AV?$IdRegistry@VDomainFactory@Workflow@U2@@@U2@@@8 1003888c     KrakenBuildWorkerFactory.obj
 0003:000008c8       ??_R0?AVGenomicLibraryDelegate@LocalWorkflow@U2@@@8 100388c8     KrakenBuildWorkerFactory.obj
 0003:00000900       ??_R0?AVKrakenClassifyLogParser@U2@@@8 10038900     KrakenClassifyLogParser.obj
 0003:0000092c       ??_R0?AVKrakenClassifyPrompter@LocalWorkflow@U2@@@8 1003892c     KrakenClassifyPrompter.obj
 0003:00000968       ??_R0?AV?$PrompterBase@VKrakenClassifyPrompter@LocalWorkflow@U2@@@U2@@@8 10038968     KrakenClassifyPrompter.obj
 0003:000009b4       ??_R0?AVKrakenClassifyTask@U2@@@8 100389b4     KrakenClassifyTask.obj
 0003:000009d8       ??_R0?AVFailTask@U2@@@8    100389d8     KrakenClassifyWorker.obj
 0003:000009f4       ??_R0?AVKrakenClassifyWorker@LocalWorkflow@U2@@@8 100389f4     KrakenClassifyWorker.obj
 0003:00000a28       ??_R0?AVSlotRelationDescriptor@U2@@@8 10038a28     KrakenClassifyWorkerFactory.obj
 0003:00000a50       ??_R0?AVPairedReadsPortValidator@Workflow@U2@@@8 10038a50     KrakenClassifyWorkerFactory.obj
 0003:00000a84       ??_R0?AVPortValidator@Workflow@U2@@@8 10038a84     KrakenClassifyWorkerFactory.obj
 0003:00000aac       ??_R0?AVKrakenClassifyValidator@Workflow@U2@@@8 10038aac     KrakenClassifyWorkerFactory.obj
 0003:00000ae0       ??_R0?AVKrakenClassifyWorkerFactory@LocalWorkflow@U2@@@8 10038ae0     KrakenClassifyWorkerFactory.obj
 0003:00000b1c       ??_R0?AVDatabaseDelegate@LocalWorkflow@U2@@@8 10038b1c     KrakenClassifyWorkerFactory.obj
 0003:00000b4c       ??_R0?AVKrakenSupport@U2@@@8 10038b4c     KrakenSupport.obj
 0003:00000b6c       ??_R0?AVExternalTool@U2@@@8 10038b6c     KrakenSupport.obj
 0003:00000b8c       ??_R0?AVKrakenSupportPlugin@U2@@@8 10038b8c     KrakenSupportPlugin.obj
 0003:00000bb4       ??_R0?AVPlugin@U2@@@8      10038bb4     KrakenSupportPlugin.obj
 0003:00000bcc       ??_R0?AVKrakenTranslateLogParser@U2@@@8 10038bcc     KrakenTranslateLogParser.obj
 0003:00000bf8       ??_R0?AVtype_info@@@8      10038bf8     MSVCRT:ti_inst.obj
 0003:00000c5c       ?id@?$num_put@DV?$back_insert_iterator@V?$basic_string@DU?$char_traits@D@std@@V?$allocator@D@2@@std@@@std@@@std@@2V0locale@2@A 10038c5c     DatabaseSizeRelation.obj
 0003:00000c60       ?id@?$num_put@_WV?$back_insert_iterator@V?$basic_string@_WU?$char_traits@_W@std@@V?$allocator@_W@2@@std@@@std@@@std@@2V0locale@2@A 10038c60     DatabaseSizeRelation.obj
 0003:00000cb4       ?BUILD@KrakenBuildTaskSettings@U2@@2VQString@@B 10038cb4     KrakenBuildTask.obj
 0003:00000cf0       ?SHRINK@KrakenBuildTaskSettings@U2@@2VQString@@B 10038cf0     KrakenBuildTask.obj
 0003:00000dd4       ?metatype_id@?1??qt_metatype_id@?$QMetaTypeId@V?$QList@VDataset@U2@@@@@@SAHXZ@4V?$QBasicAtomicInteger@H@@A 10038dd4     KrakenBuildWorker.obj
 0003:00000ddc       ?NEW_DATABASE_NAME_ATTR_ID@KrakenBuildWorkerFactory@LocalWorkflow@U2@@2VQString@@B 10038ddc     KrakenBuildWorkerFactory.obj
 0003:00000de0       ?MINIMIZER_LENGTH_ATTR_ID@KrakenBuildWorkerFactory@LocalWorkflow@U2@@2VQString@@B 10038de0     KrakenBuildWorkerFactory.obj
 0003:00000e0c       ?K_MER_LENGTH_ATTR_ID@KrakenBuildWorkerFactory@LocalWorkflow@U2@@2VQString@@B 10038e0c     KrakenBuildWorkerFactory.obj
 0003:00000e10       ?INPUT_DATABASE_NAME_ATTR_ID@KrakenBuildWorkerFactory@LocalWorkflow@U2@@2VQString@@B 10038e10     KrakenBuildWorkerFactory.obj
 0003:00000e14       ?GENOMIC_LIBRARY_ATTR_ID@KrakenBuildWorkerFactory@LocalWorkflow@U2@@2VQString@@B 10038e14     KrakenBuildWorkerFactory.obj
 0003:00000e20       ?JELLYFISH_HASH_SIZE_ATTR_ID@KrakenBuildWorkerFactory@LocalWorkflow@U2@@2VQString@@B 10038e20     KrakenBuildWorkerFactory.obj
 0003:00000e34       ?ACTOR_ID@KrakenBuildWorkerFactory@LocalWorkflow@U2@@2VQString@@B 10038e34     KrakenBuildWorkerFactory.obj
 0003:00000e38       ?WORK_ON_DISK_ATTR_ID@KrakenBuildWorkerFactory@LocalWorkflow@U2@@2VQString@@B 10038e38     KrakenBuildWorkerFactory.obj
 0003:00000e3c       ?MAXIMUM_DATABASE_SIZE_ATTR_ID@KrakenBuildWorkerFactory@LocalWorkflow@U2@@2VQString@@B 10038e3c     KrakenBuildWorkerFactory.obj
 0003:00000e48       ?MODE_ATTR_ID@KrakenBuildWorkerFactory@LocalWorkflow@U2@@2VQString@@B 10038e48     KrakenBuildWorkerFactory.obj
 0003:00000e4c       ?NUMBER_OF_K_MERS_ATTR_ID@KrakenBuildWorkerFactory@LocalWorkflow@U2@@2VQString@@B 10038e4c     KrakenBuildWorkerFactory.obj
 0003:00000e50       ?CLEAN_ATTR_ID@KrakenBuildWorkerFactory@LocalWorkflow@U2@@2VQString@@B 10038e50     KrakenBuildWorkerFactory.obj
 0003:00000e54       ?THREADS_NUMBER_ATTR_ID@KrakenBuildWorkerFactory@LocalWorkflow@U2@@2VQString@@B 10038e54     KrakenBuildWorkerFactory.obj
 0003:00000e58       ?OUTPUT_PORT_ID@KrakenBuildWorkerFactory@LocalWorkflow@U2@@2VQString@@B 10038e58     KrakenBuildWorkerFactory.obj
 0003:00000e5c       ?SHRINK_BLOCK_OFFSET_ATTR_ID@KrakenBuildWorkerFactory@LocalWorkflow@U2@@2VQString@@B 10038e5c     KrakenBuildWorkerFactory.obj
 0003:00000eac       ?wellKnownErrors@KrakenClassifyLogParser@U2@@0VQStringList@@B 10038eac     KrakenClassifyLogParser.obj
 0003:00000f10       ?SINGLE_END@KrakenClassifyTaskSettings@U2@@2VQString@@B 10038f10     KrakenClassifyTask.obj
 0003:00000f3c       ?PAIRED_END@KrakenClassifyTaskSettings@U2@@2VQString@@B 10038f3c     KrakenClassifyTask.obj
 0003:00000fcc       ?KRAKEN_DIR@KrakenClassifyWorker@LocalWorkflow@U2@@0VQString@@B 10038fcc     KrakenClassifyWorker.obj
 0003:00001018       ?metatype_id@?1??qt_metatype_id@?$QMetaTypeId@VQAssociativeIterableImpl@QtMetaTypePrivate@@@@SAHXZ@4V?$QBasicAtomicInteger@H@@A 10039018     KrakenClassifyWorker.obj
 0003:0000101c       ?metatype_id@?1??qt_metatype_id@?$QMetaTypeId@V?$QMap@VQString@@I@@@@SAHXZ@4V?$QBasicAtomicInteger@H@@A 1003901c     KrakenClassifyWorker.obj
 0003:00001020       ?f@?4??registerConverter@?$AssociativeValueTypeIsMetaType@V?$QMap@VQString@@I@@$00@QtPrivate@@SA_NH@Z@4U?$ConverterFunctor@V?$QMap@VQString@@I@@VQAssociativeIterableImpl@QtMetaTypePrivate@@U?$QAssociativeIterableConvertFunctor@V?$QMap@VQString@@I@@@3@@3@B 10039020     KrakenClassifyWorker.obj
 0003:00001028       ??_B?4??registerConverter@?$AssociativeValueTypeIsMetaType@V?$QMap@VQString@@I@@$00@QtPrivate@@SA_NH@Z@54 10039028     KrakenClassifyWorker.obj
 0003:00001030       ?QUICK_OPERATION_ATTR_ID@KrakenClassifyWorkerFactory@LocalWorkflow@U2@@2VQString@@B 10039030     KrakenClassifyWorkerFactory.obj
 0003:00001034       ?INPUT_PORT_ID@KrakenClassifyWorkerFactory@LocalWorkflow@U2@@2VQString@@B 10039034     KrakenClassifyWorkerFactory.obj
 0003:00001038       ?SINGLE_END_TEXT@KrakenClassifyWorkerFactory@LocalWorkflow@U2@@2VQString@@B 10039038     KrakenClassifyWorkerFactory.obj
 0003:0000103c       ?PAIRED_END_TEXT@KrakenClassifyWorkerFactory@LocalWorkflow@U2@@2VQString@@B 1003903c     KrakenClassifyWorkerFactory.obj
 0003:00001040       ?OUTPUT_PORT_ID@KrakenClassifyWorkerFactory@LocalWorkflow@U2@@2VQString@@B 10039040     KrakenClassifyWorkerFactory.obj
 0003:00001044       ?THREADS_NUMBER_ATTR_ID@KrakenClassifyWorkerFactory@LocalWorkflow@U2@@2VQString@@B 10039044     KrakenClassifyWorkerFactory.obj
 0003:00001070       ?PRELOAD_DATABASE_ATTR_ID@KrakenClassifyWorkerFactory@LocalWorkflow@U2@@2VQString@@B 10039070     KrakenClassifyWorkerFactory.obj
 0003:00001074       ?ACTOR_ID@KrakenClassifyWorkerFactory@LocalWorkflow@U2@@2VQString@@B 10039074     KrakenClassifyWorkerFactory.obj
 0003:00001078       ?PAIRED_INPUT_SLOT@KrakenClassifyWorkerFactory@LocalWorkflow@U2@@2VQString@@B 10039078     KrakenClassifyWorkerFactory.obj
 0003:0000108c       ?WORKFLOW_CLASSIFY_TOOL_KRAKEN@KrakenClassifyWorkerFactory@LocalWorkflow@U2@@2VQString@@B 1003908c     KrakenClassifyWorkerFactory.obj
 0003:000010a0       ?INPUT_DATA_ATTR_ID@KrakenClassifyWorkerFactory@LocalWorkflow@U2@@2VQString@@B 100390a0     KrakenClassifyWorkerFactory.obj
 0003:000010a4       ?DATABASE_ATTR_ID@KrakenClassifyWorkerFactory@LocalWorkflow@U2@@2VQString@@B 100390a4     KrakenClassifyWorkerFactory.obj
 0003:000010a8       ?MIN_HITS_NUMBER_ATTR_ID@KrakenClassifyWorkerFactory@LocalWorkflow@U2@@2VQString@@B 100390a8     KrakenClassifyWorkerFactory.obj
 0003:000010ac       ?OUTPUT_URL_ATTR_ID@KrakenClassifyWorkerFactory@LocalWorkflow@U2@@2VQString@@B 100390ac     KrakenClassifyWorkerFactory.obj
 0003:000010b0       ?INPUT_SLOT@KrakenClassifyWorkerFactory@LocalWorkflow@U2@@2VQString@@B 100390b0     KrakenClassifyWorkerFactory.obj
 0003:000010b8       ?CLASSIFY_TOOL@KrakenSupport@U2@@2VQString@@B 100390b8     KrakenSupport.obj
 0003:000010bc       ?BUILD_TOOL@KrakenSupport@U2@@2VQString@@B 100390bc     KrakenSupport.obj
 0003:000010c0       ?CLASSIFY_TOOL_ID@KrakenSupport@U2@@2VQString@@B 100390c0     KrakenSupport.obj
 0003:000010c4       ?GROUP_NAME@KrakenSupport@U2@@2VQString@@B 100390c4     KrakenSupport.obj
 0003:000010c8       ?BUILD_TOOL_ID@KrakenSupport@U2@@2VQString@@B 100390c8     KrakenSupport.obj
 0003:000010f0       ?PLUGIN_NAME@KrakenSupportPlugin@U2@@2VQString@@B 100390f0     KrakenSupportPlugin.obj
 0003:00001114       ?PLUGIN_DESCRIPRION@KrakenSupportPlugin@U2@@2VQString@@B 10039114     KrakenSupportPlugin.obj
 0003:00001144       ?wellKnownErrors@KrakenTranslateLogParser@U2@@0VQStringList@@B 10039144     KrakenTranslateLogParser.obj
 0003:00001254       ?metatype_id@?1??qt_metatype_id@?$QMetaTypeIdQObject@PAVTask@U2@@$00@@SAHXZ@4V?$QBasicAtomicInteger@H@@A 10039254     moc_KrakenBuildWorker.obj
 0003:00001668       ?__type_info_root_node@@3U__type_info_node@@A 10039668     MSVCRT:tncleanup.obj
 0003:00001670       ___native_startup_lock     10039670     <common>
 0003:00001674       ___native_startup_state    10039674     <common>
 0003:00001678       ___dyn_tls_init_callback   10039678     <common>
 0003:0000167c       ___onexitend               1003967c     <common>
 0003:00001680       ___onexitbegin             10039680     <common>

 entry point at        0001:0001b58a

 Static symbols

 0000:fffbf000       .debug$S                   10000000     MSVCRT:MSVCR120.dll
 0000:fffbf000       .debug$S                   10000000     MSVCRT:MSVCR120.dll
 0000:fffbf000       .debug$S                   10000000     MSVCRT:MSVCR120.dll
 0000:fffbf000       .debug$S                   10000000     MSVCRT:MSVCR120.dll
 0000:fffbf000       .debug$S                   10000000     MSVCRT:MSVCR120.dll
 0000:fffbf000       .debug$S                   10000000     MSVCRT:MSVCR120.dll
 0000:fffbf000       .debug$S                   10000000     MSVCRT:MSVCR120.dll
 0001:fffff000       __unwindfunclet$??1KrakenClassifyTaskSettings@U2@@QAE@XZ$0 10000000 f   KrakenClassifyWorker.obj
 0002:fffdc000       __catchsym$?detach_helper_grow@?$QList@VQString@@@@AAEPAUNode@1@HH@Z$5 10000000     KrakenClassifyValidator.obj
 0002:fffdc000       __unwindtable$?node_construct@?$QList@VQString@@@@AAEXPAUNode@1@ABVQString@@@Z 10000000     KrakenClassifyValidator.obj
 0002:fffdc000       __catchsym$?append@?$QList@VQString@@@@QAEXABVQString@@@Z$13 10000000     KrakenClassifyValidator.obj
 0002:fffdc000       __catchsym$?node_copy@?$QList@VQString@@@@AAEXPAUNode@1@00@Z$6 10000000     KrakenClassifyValidator.obj
 0001:fffff000       __unwindfunclet$??$getAttributeValue@H@Attribute@U2@@QBEHPAVWorkflowContext@Workflow@1@@Z$0 10000000 f   KrakenClassifyWorker.obj
 0000:fffbf000       .debug$S                   10000000     U2Lang:U2Lang.dll
 0001:fffff000       __unwindfunclet$??$getAttributeValue@VQString@@@Attribute@U2@@QBE?AVQString@@PAVWorkflowContext@Workflow@1@@Z$0 10000000 f   KrakenClassifyWorker.obj
 0001:fffff000       __unwindfunclet$?uniqueKeys@?$QMap@VDescriptor@U2@@VQVariant@@@@QBE?AV?$QList@VDescriptor@U2@@@@XZ$1 10000000 f   KrakenClassifyWorker.obj
 0001:fffff000       __ehhandler$?_Copy@?$basic_string@DU?$char_traits@D@std@@V?$allocator@D@2@@std@@QAEXII@Z 10000000 f   moc_KrakenSupportPlugin.obj
 0000:fffbf000       .debug$S                   10000000     U2Lang:U2Lang.dll
 0001:fffff000       __unwindfunclet$??A?$QMap@VQString@@VQScriptValue@@@@QAEAAVQScriptValue@@ABVQString@@@Z$0 10000000 f   KrakenClassifyWorker.obj
 0000:fffbf000       .debug$S                   10000000     U2Lang:U2Lang.dll
 0000:fffbf000       .debug$S                   10000000     U2Lang:U2Lang.dll
 0001:fffff000       __unwindfunclet$?node_copy@?$QList@VDescriptor@U2@@@@AAEXPAUNode@1@00@Z$4 10000000 f   KrakenClassifyWorker.obj
 0000:fffbf000       .debug$S                   10000000     U2Lang:U2Lang.dll
 0002:fffdc000       __catchsym$?_Copy@?$basic_string@DU?$char_traits@D@std@@V?$allocator@D@2@@std@@QAEXII@Z$5 10000000     moc_KrakenSupportPlugin.obj
 0000:fffbf000       .debug$S                   10000000     MSVCRT:MSVCR120.dll
 0000:fffbf000       .debug$S                   10000000     MSVCRT:MSVCR120.dll
 0000:fffbf000       .debug$S                   10000000     MSVCRT:MSVCR120.dll
 0000:fffbf000       .debug$S                   10000000     MSVCRT:MSVCR120.dll
 0000:fffbf000       .debug$S                   10000000     U2Lang:U2Lang.dll
 0002:fffdc000       ?_Generic_object$initializer$@?$_Error_objects@H@std@@2P6AXXZA 10000000     moc_KrakenSupportPlugin.obj
 0002:fffdc000       ?_Iostream_object$initializer$@?$_Error_objects@H@std@@2P6AXXZA 10000000     moc_KrakenSupportPlugin.obj
 0002:fffdc000       ?_System_object$initializer$@?$_Error_objects@H@std@@2P6AXXZA 10000000     moc_KrakenSupportPlugin.obj
 0001:fffff000       __unwindfunclet$?node_construct@?$QList@VDescriptor@U2@@@@AAEXPAUNode@1@ABVDescriptor@U2@@@Z$0 10000000 f   KrakenClassifyWorker.obj
 0000:fffbf000       .debug$S                   10000000     U2Lang:U2Lang.dll
 0002:fffdc000       ?_System_object$initializer$@?$_Error_objects@H@std@@2P6AXXZA 10000000     KrakenBuildPrompter.obj
 0002:fffdc000       ?_Iostream_object$initializer$@?$_Error_objects@H@std@@2P6AXXZA 10000000     KrakenBuildPrompter.obj
 0002:fffdc000       ?_Generic_object$initializer$@?$_Error_objects@H@std@@2P6AXXZA 10000000     KrakenBuildPrompter.obj
 0002:fffdc000       __catchsym$?_Copy@?$basic_string@DU?$char_traits@D@std@@V?$allocator@D@2@@std@@QAEXII@Z$5 10000000     KrakenBuildPrompter.obj
 0000:fffbf000       .debug$S                   10000000     U2Lang:U2Lang.dll
 0001:fffff000       __ehhandler$?detach_helper@?$QList@VDescriptor@U2@@@@AAEXH@Z 10000000 f   KrakenClassifyWorker.obj
 0000:fffbf000       .debug$S                   10000000     U2Lang:U2Lang.dll
 0001:fffff000       __ehhandler$?_Copy@?$basic_string@DU?$char_traits@D@std@@V?$allocator@D@2@@std@@QAEXII@Z 10000000 f   moc_KrakenSupport.obj
 0001:fffff000       __ehhandler$?detach_helper_grow@?$QList@VDescriptor@U2@@@@AAEPAUNode@1@HH@Z 10000000 f   KrakenClassifyWorker.obj
 0001:fffff000       __unwindfunclet$?append@?$QList@VDescriptor@U2@@@@QAEXABVDescriptor@U2@@@Z$6 10000000 f   KrakenClassifyWorker.obj
 0000:fffbf000       .debug$S                   10000000     U2Lang:U2Lang.dll
 0000:fffbf000       .debug$S                   10000000     U2Lang:U2Lang.dll
 0001:fffff000       __ehhandler$??0?$QList@VDescriptor@U2@@@@QAE@ABV0@@Z 10000000 f   KrakenClassifyWorker.obj
 0000:fffbf000       .debug$S                   10000000     U2Lang:U2Lang.dll
 0002:fffdc000       __catchsym$?_Copy@?$basic_string@DU?$char_traits@D@std@@V?$allocator@D@2@@std@@QAEXII@Z$5 10000000     moc_KrakenSupport.obj
 0000:fffbf000       .debug$S                   10000000     MSVCRT:MSVCR120.dll
 0000:fffbf000       .debug$S                   10000000     MSVCRT:MSVCR120.dll
 0000:fffbf000       .debug$S                   10000000     MSVCRT:MSVCR120.dll
 0000:fffbf000       .debug$S                   10000000     MSVCRT:MSVCR120.dll
 0000:fffbf000       .debug$S                   10000000     U2Lang:U2Lang.dll
 0002:fffdc000       ?_Generic_object$initializer$@?$_Error_objects@H@std@@2P6AXXZA 10000000     moc_KrakenSupport.obj
 0002:fffdc000       ?_Iostream_object$initializer$@?$_Error_objects@H@std@@2P6AXXZA 10000000     moc_KrakenSupport.obj
 0002:fffdc000       ?_System_object$initializer$@?$_Error_objects@H@std@@2P6AXXZA 10000000     moc_KrakenSupport.obj
 0000:fffbf000       .debug$S                   10000000     U2Lang:U2Lang.dll
 0000:fffbf000       .debug$S                   10000000     U2Lang:U2Lang.dll
 0001:fffff000       __ehhandler$?_Copy@?$basic_string@DU?$char_traits@D@std@@V?$allocator@D@2@@std@@QAEXII@Z 10000000 f   KrakenBuildPrompter.obj
 0001:fffff000       __unwindfunclet$??0KrakenClassifyTaskSettings@U2@@QAE@ABU01@@Z$0 10000000 f   KrakenClassifyWorker.obj
 0000:fffbf000       .debug$S                   10000000     U2Lang:U2Lang.dll
 0000:fffbf000       .debug$S                   10000000     U2Lang:U2Lang.dll
 0001:fffff000       __unwindfunclet$??$getValue@VQString@@@BaseWorker@LocalWorkflow@U2@@IBE?AVQString@@ABV3@@Z$0 10000000 f   KrakenClassifyWorker.obj
 0000:fffbf000       .debug$S                   10000000     U2Lang:U2Lang.dll
 0001:fffff000       __unwindfunclet$?createNode@?$QMapData@VQString@@VQVariant@@@@QAEPAU?$QMapNode@VQString@@VQVariant@@@@ABVQString@@ABVQVariant@@PAU2@_N@Z$4 10000000 f   KrakenClassifyWorker.obj
 0000:fffbf000       .debug$S                   10000000     U2Lang:U2Lang.dll
 0001:fffff000       __unwindfunclet$?createNode@?$QMapData@VQString@@VQScriptValue@@@@QAEPAU?$QMapNode@VQString@@VQScriptValue@@@@ABVQString@@ABVQScriptValue@@PAU2@_N@Z$4 10000000 f   KrakenClassifyWorker.obj
 0001:fffff000       __unwindfunclet$??A?$QMap@VQString@@VQVariant@@@@QAEAAVQVariant@@ABVQString@@@Z$0 10000000 f   KrakenClassifyWorker.obj
 0000:fffbf000       .debug$S                   10000000     U2Lang:U2Lang.dll
 0001:fffff000       __unwindfunclet$?node_copy@?$QList@VQString@@@@AAEXPAUNode@1@00@Z$5 10000000 f   KrakenClassifyWorker.obj
 0001:fffff000       __ehhandler$?_Copy@?$basic_string@DU?$char_traits@D@std@@V?$allocator@D@2@@std@@QAEXII@Z 10000000 f   KrakenClassifyWorkerFactory.obj
 0002:fffdc000       ?_System_object$initializer$@?$_Error_objects@H@std@@2P6AXXZA 10000000     KrakenBuildTask.obj
 0002:fffdc000       ?_Iostream_object$initializer$@?$_Error_objects@H@std@@2P6AXXZA 10000000     KrakenBuildTask.obj
 0002:fffdc000       ?_Generic_object$initializer$@?$_Error_objects@H@std@@2P6AXXZA 10000000     KrakenBuildTask.obj
 0000:fffbf000       .debug$S                   10000000     U2Core:U2Core.dll
 0000:fffbf000       .debug$S                   10000000     U2Core:U2Core.dll
 0000:fffbf000       .debug$S                   10000000     U2Core:U2Core.dll
 0000:fffbf000       .debug$S                   10000000     U2Core:U2Core.dll
 0000:fffbf000       .debug$S                   10000000     U2Core:U2Core.dll
 0002:fffdc000       __unwindtable$??H@YA?BVQString@@ABV0@PBD@Z 10000000     KrakenBuildTask.obj
 0001:fffff000       __unwindfunclet$??H@YA?BVQString@@ABV0@PBD@Z$0 10000000 f   KrakenClassifyWorkerFactory.obj
 0002:fffdc000       __catchsym$?_Copy@?$basic_string@DU?$char_traits@D@std@@V?$allocator@D@2@@std@@QAEXII@Z$5 10000000     KrakenBuildTask.obj
 0002:fffdc000       __catchsym$?append@?$QList@VWorkflowNotification@U2@@@@QAEXABVWorkflowNotification@U2@@@Z$11 10000000     KrakenClassifyValidator.obj
 0001:fffff000       __ehhandler$?_Copy@?$basic_string@DU?$char_traits@D@std@@V?$allocator@D@2@@std@@QAEXII@Z 10000000 f   moc_KrakenClassifyWorker.obj
 0001:fffff000       __unwindfunclet$?node_construct@?$QList@VQString@@@@AAEXPAUNode@1@ABVQString@@@Z$1 10000000 f   KrakenClassifyWorker.obj
 0002:fffdc000       __catchsym$?detach_helper_grow@?$QList@VWorkflowNotification@U2@@@@AAEPAUNode@1@HH@Z$5 10000000     KrakenClassifyValidator.obj
 0001:fffff000       __ehhandler$?detach_helper_grow@?$QList@VQString@@@@AAEPAUNode@1@HH@Z 10000000 f   KrakenClassifyWorker.obj
 0002:fffdc000       __unwindtable$?node_construct@?$QList@VWorkflowNotification@U2@@@@AAEXPAUNode@1@ABVWorkflowNotification@U2@@@Z 10000000     KrakenClassifyValidator.obj
 0001:fffff000       __unwindfunclet$??A?$QMap@VQString@@VQVariant@@@@QAEAAVQVariant@@ABVQString@@@Z$0 10000000 f   KrakenClassifyWorkerFactory.obj
 0002:fffdc000       __catchsym$?node_copy@?$QList@VWorkflowNotification@U2@@@@AAEXPAUNode@1@00@Z$6 10000000     KrakenClassifyValidator.obj
 0001:fffff000       __unwindfunclet$??H@YA?BVQString@@ABV0@PBD@Z$0 10000000 f   KrakenBuildTask.obj
 0001:fffff000       __unwindfunclet$?append@?$QList@VQString@@@@QAEXABVQString@@@Z$7 10000000 f   KrakenClassifyWorker.obj
 0002:fffdc000       __unwindtable$?metaType@?$QVariantValueHelper@VQString@@@QtPrivate@@SA?AVQString@@ABVQVariant@@@Z 10000000     KrakenClassifyValidator.obj
 0000:fffbf000       .debug$S                   10000000     U2Lang:U2Lang.dll
 0001:fffff000       __ehhandler$?_Copy@?$basic_string@DU?$char_traits@D@std@@V?$allocator@D@2@@std@@QAEXII@Z 10000000 f   KrakenBuildTask.obj
 0001:fffff000       __unwindfunclet$?createNode@?$QMapData@VQString@@I@@QAEPAU?$QMapNode@VQString@@I@@ABVQString@@ABIPAU2@_N@Z$4 10000000 f   KrakenClassifyWorker.obj
 0000:fffbf000       .debug$S                   10000000     U2Lang:U2Lang.dll
 0001:fffff000       __unwindfunclet$??H@YA?BVQString@@ABV0@PBD@Z$0 10000000 f   KrakenClassifyWorker.obj
 0001:fffff000       __unwindfunclet$??H@YA?BVQString@@ABV0@0@Z$0 10000000 f   KrakenClassifyWorker.obj
 0002:fffdc000       ?_System_object$initializer$@?$_Error_objects@H@std@@2P6AXXZA 10000000     KrakenSupport.obj
 0001:fffff000       __ehhandler$?_Copy@?$basic_string@DU?$char_traits@D@std@@V?$allocator@D@2@@std@@QAEXII@Z 10000000 f   KrakenClassifyWorker.obj
 0001:fffff000       __unwindfunclet$?metaType@?$QVariantValueHelper@VQString@@@QtPrivate@@SA?AVQString@@ABVQVariant@@@Z$0 10000000 f   KrakenClassifyWorker.obj
 0002:fffdc000       ?_Iostream_object$initializer$@?$_Error_objects@H@std@@2P6AXXZA 10000000     KrakenSupport.obj
 0002:fffdc000       ?_Generic_object$initializer$@?$_Error_objects@H@std@@2P6AXXZA 10000000     KrakenSupport.obj
 0000:fffbf000       .debug$S                   10000000     U2Lang:U2Lang.dll
 0001:fffff000       __unwindfunclet$?qt_metatype_id@?$QMetaTypeIdQObject@PAVTask@U2@@$00@@SAHXZ$0 10000000 f   moc_KrakenClassifyWorker.obj
 0000:fffbf000       .debug$S                   10000000     U2Lang:U2Lang.dll
 0000:fffbf000       .debug$S                   10000000     U2Lang:U2Lang.dll
 0002:fffdc000       __catchsym$?_Copy@?$basic_string@DU?$char_traits@D@std@@V?$allocator@D@2@@std@@QAEXII@Z$5 10000000     KrakenClassifyWorker.obj
 0000:fffbf000       .debug$S                   10000000     U2Lang:U2Lang.dll
 0002:fffdc000       __catchsym$?_Copy@?$basic_string@DU?$char_traits@D@std@@V?$allocator@D@2@@std@@QAEXII@Z$5 10000000     moc_KrakenClassifyWorker.obj
 0000:fffbf000       .debug$S                   10000000     MSVCRT:MSVCR120.dll
 0000:fffbf000       .debug$S                   10000000     MSVCRT:MSVCR120.dll
 0000:fffbf000       .debug$S                   10000000     MSVCRT:MSVCR120.dll
 0000:fffbf000       .debug$S                   10000000     MSVCRT:MSVCR120.dll
 0000:fffbf000       .debug$S                   10000000     MSVCRT:MSVCR120.dll
 0000:fffbf000       .debug$S                   10000000     MSVCRT:MSVCR120.dll
 0000:fffbf000       .debug$S                   10000000     MSVCRT:MSVCR120.dll
 0000:fffbf000       .debug$S                   10000000     MSVCRT:MSVCR120.dll
 0000:fffbf000       .debug$S                   10000000     MSVCRT:MSVCR120.dll
 0000:fffbf000       .debug$S                   10000000     MSVCRT:MSVCR120.dll
 0000:fffbf000       .debug$S                   10000000     MSVCRT:MSVCR120.dll
 0000:fffbf000       .debug$S                   10000000     U2Lang:U2Lang.dll
 0002:fffdc000       __unwindtable$??H@YA?BVQString@@ABV0@0@Z 10000000     KrakenClassifyWorker.obj
 0000:fffbf000       .debug$S                   10000000     U2Lang:U2Lang.dll
 0002:fffdc000       __unwindtable$??H@YA?BVQString@@ABV0@PBD@Z 10000000     KrakenClassifyWorker.obj
 0000:fffbf000       .debug$S                   10000000     U2Lang:U2Lang.dll
 0002:fffdc000       ?_System_object$initializer$@?$_Error_objects@H@std@@2P6AXXZA 10000000     KrakenBuildValidator.obj
 0002:fffdc000       ?_Iostream_object$initializer$@?$_Error_objects@H@std@@2P6AXXZA 10000000     KrakenBuildValidator.obj
 0000:fffbf000       .debug$S                   10000000     U2Lang:U2Lang.dll
 0002:fffdc000       __unwindtable$?qt_metatype_id@?$QMetaTypeIdQObject@PAVTask@U2@@$00@@SAHXZ 10000000     moc_KrakenClassifyWorker.obj
 0000:fffbf000       .debug$S                   10000000     msvcprt:MSVCP120.dll
 0000:fffbf000       .debug$S                   10000000     msvcprt:MSVCP120.dll
 0000:fffbf000       .debug$S                   10000000     msvcprt:MSVCP120.dll
 0000:fffbf000       .debug$S                   10000000     msvcprt:MSVCP120.dll
 0000:fffbf000       .debug$S                   10000000     msvcprt:MSVCP120.dll
 0000:fffbf000       .debug$S                   10000000     kernel32:KERNEL32.dll
 0000:fffbf000       .debug$S                   10000000     kernel32:KERNEL32.dll
 0000:fffbf000       .debug$S                   10000000     kernel32:KERNEL32.dll
 0000:fffbf000       .debug$S                   10000000     kernel32:KERNEL32.dll
 0000:fffbf000       .debug$S                   10000000     kernel32:KERNEL32.dll
 0000:fffbf000       .debug$S                   10000000     kernel32:KERNEL32.dll
 0000:fffbf000       .debug$S                   10000000     kernel32:KERNEL32.dll
 0000:fffbf000       .debug$S                   10000000     kernel32:KERNEL32.dll
 0002:fffdc000       ?_Generic_object$initializer$@?$_Error_objects@H@std@@2P6AXXZA 10000000     KrakenBuildValidator.obj
 0000:fffbf000       .debug$S                   10000000     U2Core:U2Core.dll
 0000:fffbf000       .debug$S                   10000000     U2Core:U2Core.dll
 0000:fffbf000       .debug$S                   10000000     U2Core:U2Core.dll
 0000:fffbf000       .debug$S                   10000000     U2Core:U2Core.dll
 0000:fffbf000       .debug$S                   10000000     U2Core:U2Core.dll
 0000:fffbf000       .debug$S                   10000000     U2Core:U2Core.dll
 0000:fffbf000       .debug$S                   10000000     U2Core:U2Core.dll
 0000:fffbf000       .debug$S                   10000000     U2Core:U2Core.dll
 0000:fffbf000       .debug$S                   10000000     U2Core:U2Core.dll
 0002:fffdc000       ?_Generic_object$initializer$@?$_Error_objects@H@std@@2P6AXXZA 10000000     moc_KrakenClassifyWorker.obj
 0002:fffdc000       ?_Iostream_object$initializer$@?$_Error_objects@H@std@@2P6AXXZA 10000000     moc_KrakenClassifyWorker.obj
 0002:fffdc000       ?_System_object$initializer$@?$_Error_objects@H@std@@2P6AXXZA 10000000     moc_KrakenClassifyWorker.obj
 0000:fffbf000       .debug$S                   10000000     U2Core:U2Core.dll
 0000:fffbf000       .debug$S                   10000000     U2Core:U2Core.dll
 0000:fffbf000       .debug$S                   10000000     U2Core:U2Core.dll
 0000:fffbf000       .debug$S                   10000000     U2Core:U2Core.dll
 0002:fffdc000       __catchsym$?node_copy@?$QList@VQString@@@@AAEXPAUNode@1@00@Z$6 10000000     KrakenBuildValidator.obj
 0000:fffbf000       .debug$S                   10000000     U2Lang:U2Lang.dll
 0000:fffbf000       .debug$S                   10000000     U2Lang:U2Lang.dll
 0000:fffbf000       .debug$S                   10000000     U2Lang:U2Lang.dll
 0002:fffdc000       __unwindtable$?node_construct@?$QList@VQString@@@@AAEXPAUNode@1@ABVQString@@@Z 10000000     KrakenBuildValidator.obj
 0000:fffbf000       .debug$S                   10000000     U2Lang:U2Lang.dll
 0002:fffdc000       __catchsym$?detach_helper_grow@?$QList@VQString@@@@AAEPAUNode@1@HH@Z$5 10000000     KrakenBuildValidator.obj
 0000:fffbf000       .debug$S                   10000000     U2Lang:U2Lang.dll
 0000:fffbf000       .debug$S                   10000000     U2Lang:U2Lang.dll
 0000:fffbf000       .debug$S                   10000000     U2Lang:U2Lang.dll
 0000:fffbf000       .debug$S                   10000000     U2Lang:U2Lang.dll
 0002:fffdc000       __catchsym$?append@?$QList@VQString@@@@QAEXABVQString@@@Z$13 10000000     KrakenBuildValidator.obj
 0000:fffbf000       .debug$S                   10000000     U2Lang:U2Lang.dll
 0000:fffbf000       .debug$S                   10000000     U2Lang:U2Lang.dll
 0002:fffdc000       __catchsym$?append@?$QList@VQString@@@@QAEXABVQString@@@Z$13 10000000     KrakenClassifyWorker.obj
 0000:fffbf000       .debug$S                   10000000     U2Lang:U2Lang.dll
 0002:fffdc000       __catchsym$??0?$QList@VQString@@@@QAE@ABV0@@Z$2 10000000     KrakenBuildValidator.obj
 0000:fffbf000       .debug$S                   10000000     U2Lang:U2Lang.dll
 0000:fffbf000       .debug$S                   10000000     U2Lang:U2Lang.dll
 0002:fffdc000       __catchsym$?node_copy@?$QList@VQString@@@@AAEXPAUNode@1@00@Z$6 10000000     KrakenSupport.obj
 0002:fffdc000       __catchsym$?_Copy@?$basic_string@DU?$char_traits@D@std@@V?$allocator@D@2@@std@@QAEXII@Z$5 10000000     KrakenBuildValidator.obj
 0002:fffdc000       __catchsym$??0?$QList@VQString@@@@QAE@ABV0@@Z$2 10000000     KrakenClassifyValidator.obj
 0002:fffdc000       __unwindtable$?node_construct@?$QList@VQString@@@@AAEXPAUNode@1@ABVQString@@@Z 10000000     KrakenSupport.obj
 0001:fffff000       __ehhandler$?_Copy@?$basic_string@DU?$char_traits@D@std@@V?$allocator@D@2@@std@@QAEXII@Z 10000000 f   moc_KrakenClassifyTask.obj
 0002:fffdc000       __catchsym$?detach_helper_grow@?$QList@VQString@@@@AAEPAUNode@1@HH@Z$5 10000000     KrakenClassifyWorker.obj
 0002:fffdc000       ?_System_object$initializer$@?$_Error_objects@H@std@@2P6AXXZA 10000000     KrakenClassifyWorkerFactory.obj
 0002:fffdc000       __catchsym$?detach_helper_grow@?$QList@VQString@@@@AAEPAUNode@1@HH@Z$5 10000000     KrakenSupport.obj
 0002:fffdc000       ?_Iostream_object$initializer$@?$_Error_objects@H@std@@2P6AXXZA 10000000     KrakenClassifyWorkerFactory.obj
 0001:fffff000       __unwindfunclet$?node_copy@?$QList@VQString@@@@AAEXPAUNode@1@00@Z$5 10000000 f   KrakenBuildValidator.obj
 0002:fffdc000       ?_Generic_object$initializer$@?$_Error_objects@H@std@@2P6AXXZA 10000000     KrakenClassifyWorkerFactory.obj
 0002:fffdc000       __unwindtable$??H@YA?BVQString@@ABV0@PBD@Z 10000000     KrakenClassifyValidator.obj
 0001:fffff000       __unwindfunclet$?node_construct@?$QList@VQString@@@@AAEXPAUNode@1@ABVQString@@@Z$1 10000000 f   KrakenBuildValidator.obj
 0002:fffdc000       __catchsym$?append@?$QList@VQString@@@@QAEXABVQString@@@Z$13 10000000     KrakenSupport.obj
 0002:fffdc000       __unwindtable$??H@YA?BVQString@@ABV0@0@Z 10000000     KrakenClassifyValidator.obj
 0002:fffdc000       __unwindtable$?node_construct@?$QList@VQString@@@@AAEXPAUNode@1@ABVQString@@@Z 10000000     KrakenClassifyWorker.obj
 0001:fffff000       __ehhandler$?detach_helper_grow@?$QList@VQString@@@@AAEPAUNode@1@HH@Z 10000000 f   KrakenBuildValidator.obj
 0002:fffdc000       __catchsym$??0?$QList@VQString@@@@QAE@ABV0@@Z$2 10000000     KrakenSupport.obj
 0001:fffff000       __unwindfunclet$?append@?$QList@VQString@@@@QAEXABVQString@@@Z$7 10000000 f   KrakenBuildValidator.obj
 0002:fffdc000       __unwindtable$??H@YA?BVQString@@ABV0@PBD@Z 10000000     KrakenSupport.obj
 0002:fffdc000       __catchsym$?node_copy@?$QList@VQString@@@@AAEXPAUNode@1@00@Z$6 10000000     KrakenClassifyWorker.obj
 0002:fffdc000       __catchsym$?_Copy@?$basic_string@DU?$char_traits@D@std@@V?$allocator@D@2@@std@@QAEXII@Z$5 10000000     KrakenSupport.obj
 0002:fffdc000       __unwindtable$??A?$QMap@VQString@@VQVariant@@@@QAEAAVQVariant@@ABVQString@@@Z 10000000     KrakenClassifyWorker.obj
 0001:fffff000       __ehhandler$??0?$QList@VQString@@@@QAE@ABV0@@Z 10000000 f   KrakenBuildValidator.obj
 0000:fffbf000       .debug$S                   10000000     U2Lang:U2Lang.dll
 0000:fffbf000       .debug$S                   10000000     U2Lang:U2Lang.dll
 0002:fffdc000       __catchsym$?_Copy@?$basic_string@DU?$char_traits@D@std@@V?$allocator@D@2@@std@@QAEXII@Z$5 10000000     KrakenClassifyValidator.obj
 0000:fffbf000       .debug$S                   10000000     U2Lang:U2Lang.dll
 0000:fffbf000       .debug$S                   10000000     U2Lang:U2Lang.dll
 0002:fffdc000       __catchsym$?_Copy@?$basic_string@DU?$char_traits@D@std@@V?$allocator@D@2@@std@@QAEXII@Z$5 10000000     moc_KrakenClassifyTask.obj
 0000:fffbf000       .debug$S                   10000000     kernel32:KERNEL32.dll
 0000:fffbf000       .debug$S                   10000000     Qt5Core:Qt5Core.dll
 0000:fffbf000       .debug$S                   10000000     Qt5Core:Qt5Core.dll
 0000:fffbf000       .debug$S                   10000000     Qt5Core:Qt5Core.dll
 0000:fffbf000       .debug$S                   10000000     Qt5Core:Qt5Core.dll
 0000:fffbf000       .debug$S                   10000000     Qt5Core:Qt5Core.dll
 0000:fffbf000       .debug$S                   10000000     Qt5Core:Qt5Core.dll
 0000:fffbf000       .debug$S                   10000000     Qt5Core:Qt5Core.dll
 0000:fffbf000       .debug$S                   10000000     Qt5Core:Qt5Core.dll
 0000:fffbf000       .debug$S                   10000000     Qt5Core:Qt5Core.dll
 0000:fffbf000       .debug$S                   10000000     Qt5Core:Qt5Core.dll
 0000:fffbf000       .debug$S                   10000000     Qt5Core:Qt5Core.dll
 0000:fffbf000       .debug$S                   10000000     Qt5Core:Qt5Core.dll
 0000:fffbf000       .debug$S                   10000000     Qt5Core:Qt5Core.dll
 0000:fffbf000       .debug$S                   10000000     Qt5Core:Qt5Core.dll
 0000:fffbf000       .debug$S                   10000000     Qt5Core:Qt5Core.dll
 0000:fffbf000       .debug$S                   10000000     Qt5Core:Qt5Core.dll
 0000:fffbf000       .debug$S                   10000000     Qt5Core:Qt5Core.dll
 0000:fffbf000       .debug$S                   10000000     Qt5Core:Qt5Core.dll
 0000:fffbf000       .debug$S                   10000000     Qt5Core:Qt5Core.dll
 0000:fffbf000       .debug$S                   10000000     Qt5Core:Qt5Core.dll
 0000:fffbf000       .debug$S                   10000000     Qt5Core:Qt5Core.dll
 0000:fffbf000       .debug$S                   10000000     Qt5Core:Qt5Core.dll
 0000:fffbf000       .debug$S                   10000000     Qt5Core:Qt5Core.dll
 0000:fffbf000       .debug$S                   10000000     Qt5Core:Qt5Core.dll
 0000:fffbf000       .debug$S                   10000000     Qt5Core:Qt5Core.dll
 0000:fffbf000       .debug$S                   10000000     Qt5Core:Qt5Core.dll
 0000:fffbf000       .debug$S                   10000000     Qt5Core:Qt5Core.dll
 0000:fffbf000       .debug$S                   10000000     Qt5Core:Qt5Core.dll
 0000:fffbf000       .debug$S                   10000000     Qt5Core:Qt5Core.dll
 0000:fffbf000       .debug$S                   10000000     Qt5Core:Qt5Core.dll
 0000:fffbf000       .debug$S                   10000000     U2Lang:U2Lang.dll
 0001:fffff000       __ehhandler$?_Copy@?$basic_string@DU?$char_traits@D@std@@V?$allocator@D@2@@std@@QAEXII@Z 10000000 f   KrakenBuildValidator.obj
 0000:fffbf000       .debug$S                   10000000     U2Lang:U2Lang.dll
 0000:fffbf000       .debug$S                   10000000     U2Lang:U2Lang.dll
 0000:fffbf000       .debug$S                   10000000     U2Lang:U2Lang.dll
 0000:fffbf000       .debug$S                   10000000     U2Lang:U2Lang.dll
 0000:fffbf000       .debug$S                   10000000     U2Lang:U2Lang.dll
 0000:fffbf000       .debug$S                   10000000     U2Lang:U2Lang.dll
 0000:fffbf000       .debug$S                   10000000     U2Lang:U2Lang.dll
 0000:fffbf000       .debug$S                   10000000     U2Lang:U2Lang.dll
 0002:fffdc000       ?_Generic_object$initializer$@?$_Error_objects@H@std@@2P6AXXZA 10000000     moc_KrakenClassifyTask.obj
 0002:fffdc000       ?_Iostream_object$initializer$@?$_Error_objects@H@std@@2P6AXXZA 10000000     moc_KrakenClassifyTask.obj
 0002:fffdc000       ?_System_object$initializer$@?$_Error_objects@H@std@@2P6AXXZA 10000000     moc_KrakenClassifyTask.obj
 0000:fffbf000       .debug$S                   10000000     U2Lang:U2Lang.dll
 0000:fffbf000       .debug$S                   10000000     U2Lang:U2Lang.dll
 0000:fffbf000       .debug$S                   10000000     U2Lang:U2Lang.dll
 0000:fffbf000       .debug$S                   10000000     U2Lang:U2Lang.dll
 0002:fffdc000       ?_System_object$initializer$@?$_Error_objects@H@std@@2P6AXXZA 10000000     KrakenBuildWorker.obj
 0002:fffdc000       ?_Iostream_object$initializer$@?$_Error_objects@H@std@@2P6AXXZA 10000000     KrakenBuildWorker.obj
 0002:fffdc000       ?_Generic_object$initializer$@?$_Error_objects@H@std@@2P6AXXZA 10000000     KrakenBuildWorker.obj
 0000:fffbf000       .debug$S                   10000000     U2Core:U2Core.dll
 0000:fffbf000       .debug$S                   10000000     U2Core:U2Core.dll
 0000:fffbf000       .debug$S                   10000000     U2Core:U2Core.dll
 0000:fffbf000       .debug$S                   10000000     U2Core:U2Core.dll
 0000:fffbf000       .debug$S                   10000000     U2Core:U2Core.dll
 0000:fffbf000       .debug$S                   10000000     U2Core:U2Core.dll
 0000:fffbf000       .debug$S                   10000000     U2Core:U2Core.dll
 0000:fffbf000       .debug$S                   10000000     U2Core:U2Core.dll
 0000:fffbf000       .debug$S                   10000000     U2Core:U2Core.dll
 0000:fffbf000       .debug$S                   10000000     U2Core:U2Core.dll
 0000:fffbf000       .debug$S                   10000000     U2Core:U2Core.dll
 0000:fffbf000       .debug$S                   10000000     U2Core:U2Core.dll
 0000:fffbf000       .debug$S                   10000000     U2Core:U2Core.dll
 0002:fffdc000       __unwindtable$??0KrakenBuildTaskSettings@U2@@QAE@ABU01@@Z 10000000     KrakenBuildWorker.obj
 0000:fffbf000       .debug$S                   10000000     U2Lang:U2Lang.dll
 0002:fffdc000       __unwindtable$??1KrakenBuildTaskSettings@U2@@QAE@XZ 10000000     KrakenBuildWorker.obj
 0000:fffbf000       .debug$S                   10000000     U2Lang:U2Lang.dll
 0002:fffdc000       __catchsym$?node_copy@?$QList@VQString@@@@AAEXPAUNode@1@00@Z$6 10000000     KrakenBuildWorker.obj
 0000:fffbf000       .debug$S                   10000000     U2Lang:U2Lang.dll
 0000:fffbf000       .debug$S                   10000000     U2Lang:U2Lang.dll
 0001:fffff000       __ehhandler$?_Copy@?$basic_string@DU?$char_traits@D@std@@V?$allocator@D@2@@std@@QAEXII@Z 10000000 f   moc_KrakenClassifyPrompter.obj
 0000:fffbf000       .debug$S                   10000000     U2Lang:U2Lang.dll
 0000:fffbf000       .debug$S                   10000000     U2Lang:U2Lang.dll
 0000:fffbf000       .debug$S                   10000000     U2Lang:U2Lang.dll
 0002:fffdc000       __unwindtable$?node_construct@?$QList@VQString@@@@AAEXPAUNode@1@ABVQString@@@Z 10000000     KrakenBuildWorker.obj
 0000:fffbf000       .debug$S                   10000000     U2Lang:U2Lang.dll
 0002:fffdc000       __catchsym$?detach_helper_grow@?$QList@VQString@@@@AAEPAUNode@1@HH@Z$5 10000000     KrakenBuildWorker.obj
 0000:fffbf000       .debug$S                   10000000     U2Lang:U2Lang.dll
 0000:fffbf000       .debug$S                   10000000     U2Lang:U2Lang.dll
 0002:fffdc000       ?_Generic_object$initializer$@?$_Error_objects@H@std@@2P6AXXZA 10000000     KrakenClassifyValidator.obj
 0000:fffbf000       .debug$S                   10000000     U2Lang:U2Lang.dll
 0002:fffdc000       __catchsym$?append@?$QList@VQString@@@@QAEXABVQString@@@Z$13 10000000     KrakenBuildWorker.obj
 0002:fffdc000       ?_Iostream_object$initializer$@?$_Error_objects@H@std@@2P6AXXZA 10000000     KrakenClassifyValidator.obj
 0000:fffbf000       .debug$S                   10000000     U2Lang:U2Lang.dll
 0000:fffbf000       .debug$S                   10000000     U2Lang:U2Lang.dll
 0002:fffdc000       ?_System_object$initializer$@?$_Error_objects@H@std@@2P6AXXZA 10000000     KrakenClassifyValidator.obj
 0002:fffdc000       __catchsym$??0?$QList@VQString@@@@QAE@ABV0@@Z$2 10000000     KrakenBuildWorker.obj
 0001:fffff000       __unwindfunclet$?metaType@?$QVariantValueHelper@VQString@@@QtPrivate@@SA?AVQString@@ABVQVariant@@@Z$0 10000000 f   KrakenClassifyValidator.obj
 0001:fffff000       __ehhandler$?_Copy@?$basic_string@DU?$char_traits@D@std@@V?$allocator@D@2@@std@@QAEXII@Z 10000000 f   KrakenClassifyTask.obj
 0000:fffbf000       .debug$S                   10000000     U2Lang:U2Lang.dll
 0002:fffdc000       __catchsym$?_Copy@?$basic_string@DU?$char_traits@D@std@@V?$allocator@D@2@@std@@QAEXII@Z$5 10000000     KrakenBuildWorker.obj
 0000:fffbf000       .debug$S                   10000000     U2Lang:U2Lang.dll
 0001:fffff000       __unwindfunclet$?node_copy@?$QList@VWorkflowNotification@U2@@@@AAEXPAUNode@1@00@Z$4 10000000 f   KrakenClassifyValidator.obj
 0000:fffbf000       .debug$S                   10000000     U2Lang:U2Lang.dll
 0001:fffff000       __ehhandler$??0?$QList@VQString@@@@QAE@ABV0@@Z 10000000 f   KrakenClassifyTask.obj
 0002:fffdc000       __catchsym$?_Copy@?$basic_string@DU?$char_traits@D@std@@V?$allocator@D@2@@std@@QAEXII@Z$5 10000000     moc_KrakenClassifyPrompter.obj
 0000:fffbf000       .debug$S                   10000000     Qt5Core:Qt5Core.dll
 0000:fffbf000       .debug$S                   10000000     Qt5Core:Qt5Core.dll
 0000:fffbf000       .debug$S                   10000000     Qt5Core:Qt5Core.dll
 0000:fffbf000       .debug$S                   10000000     Qt5Core:Qt5Core.dll
 0000:fffbf000       .debug$S                   10000000     Qt5Core:Qt5Core.dll
 0000:fffbf000       .debug$S                   10000000     Qt5Core:Qt5Core.dll
 0000:fffbf000       .debug$S                   10000000     Qt5Core:Qt5Core.dll
 0000:fffbf000       .debug$S                   10000000     Qt5Core:Qt5Core.dll
 0000:fffbf000       .debug$S                   10000000     Qt5Core:Qt5Core.dll
 0000:fffbf000       .debug$S                   10000000     Qt5Core:Qt5Core.dll
 0000:fffbf000       .debug$S                   10000000     Qt5Core:Qt5Core.dll
 0000:fffbf000       .debug$S                   10000000     Qt5Core:Qt5Core.dll
 0000:fffbf000       .debug$S                   10000000     Qt5Core:Qt5Core.dll
 0000:fffbf000       .debug$S                   10000000     Qt5Core:Qt5Core.dll
 0000:fffbf000       .debug$S                   10000000     Qt5Core:Qt5Core.dll
 0000:fffbf000       .debug$S                   10000000     Qt5Core:Qt5Core.dll
 0000:fffbf000       .debug$S                   10000000     Qt5Core:Qt5Core.dll
 0000:fffbf000       .debug$S                   10000000     Qt5Core:Qt5Core.dll
 0000:fffbf000       .debug$S                   10000000     Qt5Core:Qt5Core.dll
 0000:fffbf000       .debug$S                   10000000     Qt5Core:Qt5Core.dll
 0000:fffbf000       .debug$S                   10000000     Qt5Core:Qt5Core.dll
 0000:fffbf000       .debug$S                   10000000     Qt5Core:Qt5Core.dll
 0000:fffbf000       .debug$S                   10000000     Qt5Core:Qt5Core.dll
 0000:fffbf000       .debug$S                   10000000     Qt5Core:Qt5Core.dll
 0000:fffbf000       .debug$S                   10000000     Qt5Core:Qt5Core.dll
 0000:fffbf000       .debug$S                   10000000     Qt5Core:Qt5Core.dll
 0000:fffbf000       .debug$S                   10000000     Qt5Core:Qt5Core.dll
 0000:fffbf000       .debug$S                   10000000     Qt5Core:Qt5Core.dll
 0000:fffbf000       .debug$S                   10000000     Qt5Core:Qt5Core.dll
 0000:fffbf000       .debug$S                   10000000     Qt5Core:Qt5Core.dll
 0000:fffbf000       .debug$S                   10000000     Qt5Core:Qt5Core.dll
 0001:fffff000       __unwindfunclet$?node_construct@?$QList@VWorkflowNotification@U2@@@@AAEXPAUNode@1@ABVWorkflowNotification@U2@@@Z$0 10000000 f   KrakenClassifyValidator.obj
 0000:fffbf000       .debug$S                   10000000     U2Lang:U2Lang.dll
 0001:fffff000       __ehhandler$?detach_helper_grow@?$QList@VWorkflowNotification@U2@@@@AAEPAUNode@1@HH@Z 10000000 f   KrakenClassifyValidator.obj
 0000:fffbf000       .debug$S                   10000000     U2Lang:U2Lang.dll
 0001:fffff000       __unwindfunclet$?append@?$QList@VWorkflowNotification@U2@@@@QAEXABVWorkflowNotification@U2@@@Z$6 10000000 f   KrakenClassifyValidator.obj
 0001:fffff000       __unwindfunclet$?append@?$QList@VQString@@@@QAEXABVQString@@@Z$7 10000000 f   KrakenClassifyTask.obj
 0001:fffff000       __unwindfunclet$??0KrakenBuildTaskSettings@U2@@QAE@ABU01@@Z$0 10000000 f   KrakenBuildWorker.obj
 0001:fffff000       __ehhandler$?detach_helper_grow@?$QList@VQString@@@@AAEPAUNode@1@HH@Z 10000000 f   KrakenClassifyTask.obj
 0001:fffff000       __unwindfunclet$?node_copy@?$QList@VQString@@@@AAEXPAUNode@1@00@Z$5 10000000 f   KrakenSupport.obj
 0001:fffff000       __unwindfunclet$?node_construct@?$QList@VQString@@@@AAEXPAUNode@1@ABVQString@@@Z$1 10000000 f   KrakenSupport.obj
 0002:fffdc000       ?_Generic_object$initializer$@?$_Error_objects@H@std@@2P6AXXZA 10000000     moc_KrakenClassifyPrompter.obj
 0002:fffdc000       ?_Iostream_object$initializer$@?$_Error_objects@H@std@@2P6AXXZA 10000000     moc_KrakenClassifyPrompter.obj
 0002:fffdc000       ?_System_object$initializer$@?$_Error_objects@H@std@@2P6AXXZA 10000000     moc_KrakenClassifyPrompter.obj
 0001:fffff000       __unwindfunclet$??1KrakenBuildTaskSettings@U2@@QAE@XZ$0 10000000 f   KrakenBuildWorker.obj
 0001:fffff000       __unwindfunclet$??A?$QMap@VDescriptor@U2@@V?$QExplicitlySharedDataPointer@VDataType@U2@@@@@@QAEAAV?$QExplicitlySharedDataPointer@VDataType@U2@@@@ABVDescriptor@U2@@@Z$0 10000000 f   KrakenClassifyWorkerFactory.obj
 0001:fffff000       __unwindfunclet$?node_copy@?$QList@VQString@@@@AAEXPAUNode@1@00@Z$5 10000000 f   KrakenBuildWorker.obj
 0002:fffdc000       __catchsym$?createNode@?$QMapData@VQString@@PAVPropertyDelegate@U2@@@@QAEPAU?$QMapNode@VQString@@PAVPropertyDelegate@U2@@@@ABVQString@@ABQAVPropertyDelegate@U2@@PAU2@_N@Z$5 10000000     KrakenClassifyWorkerFactory.obj
 0001:fffff000       __ehhandler$?append@?$QList@PAVAttribute@U2@@@@QAEXABQAVAttribute@U2@@@Z 10000000 f   KrakenClassifyWorkerFactory.obj
 0001:fffff000       __unwindfunclet$?node_construct@?$QList@VQString@@@@AAEXPAUNode@1@ABVQString@@@Z$1 10000000 f   KrakenBuildWorker.obj
 0001:fffff000       __ehhandler$?detach_helper_grow@?$QList@VQString@@@@AAEPAUNode@1@HH@Z 10000000 f   KrakenSupport.obj
 0001:fffff000       __unwindfunclet$?append@?$QList@VQString@@@@QAEXABVQString@@@Z$7 10000000 f   KrakenSupport.obj
 0002:fffdc000       __catchsym$?createNode@?$QMapData@VDescriptor@U2@@V?$QExplicitlySharedDataPointer@VDataType@U2@@@@@@QAEPAU?$QMapNode@VDescriptor@U2@@V?$QExplicitlySharedDataPointer@VDataType@U2@@@@@@ABVDescriptor@U2@@ABV?$QExplicitlySharedDataPointer@VDataType@U2@@@@PAU2@_N@Z$6 10000000     KrakenClassifyWorkerFactory.obj
 0001:fffff000       __ehhandler$?detach_helper_grow@?$QList@VQString@@@@AAEPAUNode@1@HH@Z 10000000 f   KrakenBuildWorker.obj
 0001:fffff000       __ehhandler$?detach_helper_grow@?$QList@PAVAttribute@U2@@@@AAEPAUNode@1@HH@Z 10000000 f   KrakenClassifyWorkerFactory.obj
 0001:fffff000       __unwindfunclet$?append@?$QList@VQString@@@@QAEXABVQString@@@Z$7 10000000 f   KrakenBuildWorker.obj
 0001:fffff000       __ehhandler$?append@?$QList@PAVPortDescriptor@Workflow@U2@@@@QAEXABQAVPortDescriptor@Workflow@U2@@@Z 10000000 f   KrakenClassifyWorkerFactory.obj
 0002:fffdc000       __catchsym$?createNode@?$QMapData@VQString@@VQVariant@@@@QAEPAU?$QMapNode@VQString@@VQVariant@@@@ABVQString@@ABVQVariant@@PAU2@_N@Z$7 10000000     KrakenClassifyWorkerFactory.obj
 0001:fffff000       __ehhandler$?detach_helper_grow@?$QList@PAVPortDescriptor@Workflow@U2@@@@AAEPAUNode@1@HH@Z 10000000 f   KrakenClassifyWorkerFactory.obj
 0001:fffff000       __unwindfunclet$?node_copy@?$QList@VQString@@@@AAEXPAUNode@1@00@Z$5 10000000 f   KrakenClassifyValidator.obj
 0001:fffff000       __ehhandler$??0?$QList@VQString@@@@QAE@ABV0@@Z 10000000 f   KrakenBuildWorker.obj
 0000:fffbf000       .debug$S                   10000000     U2Lang:U2Lang.dll
 0000:fffbf000       .debug$S                   10000000     U2Lang:U2Lang.dll
 0001:fffff000       __ehhandler$?_Copy@?$basic_string@DU?$char_traits@D@std@@V?$allocator@D@2@@std@@QAEXII@Z 10000000 f   KrakenBuildWorker.obj
 0000:fffbf000       .debug$S                   10000000     U2Lang:U2Lang.dll
 0000:fffbf000       .debug$S                   10000000     U2Lang:U2Lang.dll
 0002:fffdc000       __catchsym$?detach_helper_grow@?$QList@PAVPortDescriptor@Workflow@U2@@@@AAEPAUNode@1@HH@Z$5 10000000     KrakenClassifyWorkerFactory.obj
 0001:fffff000       __ehhandler$??0?$QList@VQString@@@@QAE@ABV0@@Z 10000000 f   KrakenSupport.obj
 0001:fffff000       __unwindfunclet$??H@YA?BVQString@@ABV0@PBD@Z$0 10000000 f   KrakenSupport.obj
 0002:fffdc000       __catchsym$?append@?$QList@PAVPortDescriptor@Workflow@U2@@@@QAEXABQAVPortDescriptor@Workflow@U2@@@Z$6 10000000     KrakenClassifyWorkerFactory.obj
 0001:fffff000       __unwindfunclet$?node_construct@?$QList@VQString@@@@AAEXPAUNode@1@ABVQString@@@Z$1 10000000 f   KrakenClassifyValidator.obj
 0001:fffff000       __ehhandler$?_Copy@?$basic_string@DU?$char_traits@D@std@@V?$allocator@D@2@@std@@QAEXII@Z 10000000 f   moc_KrakenBuildWorker.obj
 0002:fffdc000       __catchsym$?detach_helper_grow@?$QList@PAVAttribute@U2@@@@AAEPAUNode@1@HH@Z$5 10000000     KrakenClassifyWorkerFactory.obj
 0001:fffff000       __ehhandler$?_Copy@?$basic_string@DU?$char_traits@D@std@@V?$allocator@D@2@@std@@QAEXII@Z 10000000 f   KrakenSupport.obj
 0001:fffff000       __ehhandler$?detach_helper_grow@?$QList@VQString@@@@AAEPAUNode@1@HH@Z 10000000 f   KrakenClassifyValidator.obj
 0002:fffdc000       __catchsym$?append@?$QList@PAVAttribute@U2@@@@QAEXABQAVAttribute@U2@@@Z$6 10000000     KrakenClassifyWorkerFactory.obj
 0001:fffff000       __unwindfunclet$?node_construct@?$QList@VQString@@@@AAEXPAUNode@1@ABVQString@@@Z$1 10000000 f   KrakenClassifyTask.obj
 0002:fffdc000       __unwindtable$??A?$QMap@VDescriptor@U2@@V?$QExplicitlySharedDataPointer@VDataType@U2@@@@@@QAEAAV?$QExplicitlySharedDataPointer@VDataType@U2@@@@ABVDescriptor@U2@@@Z 10000000     KrakenClassifyWorkerFactory.obj
 0001:fffff000       __unwindfunclet$?node_copy@?$QList@VQString@@@@AAEXPAUNode@1@00@Z$5 10000000 f   KrakenClassifyTask.obj
 0002:fffdc000       ?_System_object$initializer$@?$_Error_objects@H@std@@2P6AXXZA 10000000     KrakenBuildWorkerFactory.obj
 0002:fffdc000       ?_Iostream_object$initializer$@?$_Error_objects@H@std@@2P6AXXZA 10000000     KrakenBuildWorkerFactory.obj
 0002:fffdc000       ?_Generic_object$initializer$@?$_Error_objects@H@std@@2P6AXXZA 10000000     KrakenBuildWorkerFactory.obj
 0000:fffbf000       .debug$S                   10000000     U2Core:U2Core.dll
 0000:fffbf000       .debug$S                   10000000     U2Core:U2Core.dll
 0000:fffbf000       .debug$S                   10000000     U2Core:U2Core.dll
 0000:fffbf000       .debug$S                   10000000     U2Core:U2Core.dll
 0000:fffbf000       .debug$S                   10000000     U2Core:U2Core.dll
 0000:fffbf000       .debug$S                   10000000     U2Core:U2Core.dll
 0000:fffbf000       .debug$S                   10000000     U2Core:U2Core.dll
 0000:fffbf000       .debug$S                   10000000     U2Core:U2Core.dll
 0000:fffbf000       .debug$S                   10000000     U2Core:U2Core.dll
 0000:fffbf000       .debug$S                   10000000     U2Core:U2Core.dll
 0000:fffbf000       .debug$S                   10000000     U2Core:U2Core.dll
 0000:fffbf000       .debug$S                   10000000     U2Core:U2Core.dll
 0000:fffbf000       .debug$S                   10000000     U2Lang:U2Lang.dll
 0001:fffff000       __unwindfunclet$?append@?$QList@VQString@@@@QAEXABVQString@@@Z$7 10000000 f   KrakenClassifyValidator.obj
 0000:fffbf000       .debug$S                   10000000     U2Lang:U2Lang.dll
 0001:fffff000       __ehhandler$??0?$QList@VQString@@@@QAE@ABV0@@Z 10000000 f   KrakenClassifyValidator.obj
 0002:fffdc000       __catchsym$?_Copy@?$basic_string@DU?$char_traits@D@std@@V?$allocator@D@2@@std@@QAEXII@Z$5 10000000     moc_KrakenBuildWorker.obj
 0000:fffbf000       .debug$S                   10000000     Qt5Core:Qt5Core.dll
 0000:fffbf000       .debug$S                   10000000     Qt5Core:Qt5Core.dll
 0000:fffbf000       .debug$S                   10000000     Qt5Core:Qt5Core.dll
 0000:fffbf000       .debug$S                   10000000     Qt5Core:Qt5Core.dll
 0000:fffbf000       .debug$S                   10000000     Qt5Core:Qt5Core.dll
 0000:fffbf000       .debug$S                   10000000     Qt5Core:Qt5Core.dll
 0000:fffbf000       .debug$S                   10000000     Qt5Core:Qt5Core.dll
 0000:fffbf000       .debug$S                   10000000     Qt5Core:Qt5Core.dll
 0000:fffbf000       .debug$S                   10000000     Qt5Core:Qt5Core.dll
 0000:fffbf000       .debug$S                   10000000     Qt5Core:Qt5Core.dll
 0000:fffbf000       .debug$S                   10000000     Qt5Core:Qt5Core.dll
 0000:fffbf000       .debug$S                   10000000     Qt5Core:Qt5Core.dll
 0000:fffbf000       .debug$S                   10000000     Qt5Core:Qt5Core.dll
 0000:fffbf000       .debug$S                   10000000     Qt5Core:Qt5Core.dll
 0000:fffbf000       .debug$S                   10000000     Qt5Core:Qt5Core.dll
 0000:fffbf000       .debug$S                   10000000     Qt5Core:Qt5Core.dll
 0000:fffbf000       .debug$S                   10000000     Qt5Core:Qt5Core.dll
 0000:fffbf000       .debug$S                   10000000     Qt5Core:Qt5Core.dll
 0000:fffbf000       .debug$S                   10000000     Qt5Core:Qt5Core.dll
 0000:fffbf000       .debug$S                   10000000     Qt5Core:Qt5Core.dll
 0000:fffbf000       .debug$S                   10000000     Qt5Core:Qt5Core.dll
 0000:fffbf000       .debug$S                   10000000     Qt5Core:Qt5Core.dll
 0000:fffbf000       .debug$S                   10000000     Qt5Core:Qt5Core.dll
 0000:fffbf000       .debug$S                   10000000     Qt5Core:Qt5Core.dll
 0000:fffbf000       .debug$S                   10000000     Qt5Core:Qt5Core.dll
 0000:fffbf000       .debug$S                   10000000     Qt5Core:Qt5Core.dll
 0000:fffbf000       .debug$S                   10000000     Qt5Core:Qt5Core.dll
 0000:fffbf000       .debug$S                   10000000     Qt5Core:Qt5Core.dll
 0000:fffbf000       .debug$S                   10000000     Qt5Core:Qt5Core.dll
 0000:fffbf000       .debug$S                   10000000     Qt5Core:Qt5Core.dll
 0000:fffbf000       .debug$S                   10000000     Qt5Core:Qt5Core.dll
 0000:fffbf000       .debug$S                   10000000     Qt5Core:Qt5Core.dll
 0000:fffbf000       .debug$S                   10000000     Qt5Core:Qt5Core.dll
 0000:fffbf000       .debug$S                   10000000     U2Core:U2Core.dll
 0002:fffdc000       __catchsym$?createNode@?$QMapData@VQString@@VQVariant@@@@QAEPAU?$QMapNode@VQString@@VQVariant@@@@ABVQString@@ABVQVariant@@PAU2@_N@Z$7 10000000     KrakenBuildWorkerFactory.obj
 0002:fffdc000       __catchsym$?_Copy@?$basic_string@DU?$char_traits@D@std@@V?$allocator@D@2@@std@@QAEXII@Z$5 10000000     KrakenClassifyTask.obj
 0000:fffbf000       .debug$S                   10000000     U2Lang:U2Lang.dll
 0000:fffbf000       .debug$S                   10000000     U2Lang:U2Lang.dll
 0000:fffbf000       .debug$S                   10000000     U2Lang:U2Lang.dll
 0002:fffdc000       __unwindtable$??A?$QMap@VQString@@VQVariant@@@@QAEAAVQVariant@@ABVQString@@@Z 10000000     KrakenBuildWorkerFactory.obj
 0000:fffbf000       .debug$S                   10000000     U2Lang:U2Lang.dll
 0002:fffdc000       __unwindtable$??H@YA?BVQString@@ABV0@PBD@Z 10000000     KrakenBuildWorkerFactory.obj
 0000:fffbf000       .debug$S                   10000000     U2Lang:U2Lang.dll
 0002:fffdc000       ?_Generic_object$initializer$@?$_Error_objects@H@std@@2P6AXXZA 10000000     moc_KrakenBuildWorker.obj
 0002:fffdc000       ?_Iostream_object$initializer$@?$_Error_objects@H@std@@2P6AXXZA 10000000     moc_KrakenBuildWorker.obj
 0002:fffdc000       ?_System_object$initializer$@?$_Error_objects@H@std@@2P6AXXZA 10000000     moc_KrakenBuildWorker.obj
 0002:fffdc000       __catchsym$?_Copy@?$basic_string@DU?$char_traits@D@std@@V?$allocator@D@2@@std@@QAEXII@Z$5 10000000     KrakenBuildWorkerFactory.obj
 0000:fffbf000       .debug$S                   10000000     U2Lang:U2Lang.dll
 0000:fffbf000       .debug$S                   10000000     U2Lang:U2Lang.dll
 0000:fffbf000       .debug$S                   10000000     U2Lang:U2Lang.dll
 0000:fffbf000       .debug$S                   10000000     U2Lang:U2Lang.dll
 0002:fffdc000       ?_System_object$initializer$@?$_Error_objects@H@std@@2P6AXXZA 10000000     KrakenSupportPlugin.obj
 0001:fffff000       __unwindfunclet$?createNode@?$QMapData@VQString@@VQVariant@@@@QAEPAU?$QMapNode@VQString@@VQVariant@@@@ABVQString@@ABVQVariant@@PAU2@_N@Z$4 10000000 f   KrakenBuildWorkerFactory.obj
 0000:fffbf000       .debug$S                   10000000     U2Lang:U2Lang.dll
 0000:fffbf000       .debug$S                   10000000     U2Lang:U2Lang.dll
 0000:fffbf000       .debug$S                   10000000     U2Lang:U2Lang.dll
 0001:fffff000       __unwindfunclet$??A?$QMap@VQString@@VQVariant@@@@QAEAAVQVariant@@ABVQString@@@Z$0 10000000 f   KrakenBuildWorkerFactory.obj
 0002:fffdc000       ?_Iostream_object$initializer$@?$_Error_objects@H@std@@2P6AXXZA 10000000     KrakenSupportPlugin.obj
 0002:fffdc000       ?_Generic_object$initializer$@?$_Error_objects@H@std@@2P6AXXZA 10000000     KrakenSupportPlugin.obj
 0001:fffff000       __unwindfunclet$??H@YA?BVQString@@ABV0@PBD@Z$0 10000000 f   KrakenBuildWorkerFactory.obj
 0000:fffbf000       .debug$S                   10000000     U2Lang:U2Lang.dll
 0000:fffbf000       .debug$S                   10000000     U2Lang:U2Lang.dll
 0000:fffbf000       .debug$S                   10000000     U2Lang:U2Lang.dll
 0001:fffff000       __ehhandler$?_Copy@?$basic_string@DU?$char_traits@D@std@@V?$allocator@D@2@@std@@QAEXII@Z 10000000 f   KrakenBuildWorkerFactory.obj
 0000:fffbf000       .debug$S                   10000000     U2Lang:U2Lang.dll
 0000:fffbf000       .debug$S                   10000000     U2Lang:U2Lang.dll
 0000:fffbf000       .debug$S                   10000000     U2Lang:U2Lang.dll
 0000:fffbf000       .debug$S                   10000000     U2Lang:U2Lang.dll
 0000:fffbf000       .debug$S                   10000000     U2Lang:U2Lang.dll
 0000:fffbf000       .debug$S                   10000000     U2Lang:U2Lang.dll
 0000:fffbf000       .debug$S                   10000000     U2Lang:U2Lang.dll
 0000:fffbf000       .debug$S                   10000000     U2Lang:U2Lang.dll
 0000:fffbf000       .debug$S                   10000000     U2Lang:U2Lang.dll
 0001:fffff000       __ehhandler$?_Copy@?$basic_string@DU?$char_traits@D@std@@V?$allocator@D@2@@std@@QAEXII@Z 10000000 f   moc_KrakenBuildTask.obj
 0000:fffbf000       .debug$S                   10000000     U2Lang:U2Lang.dll
 0000:fffbf000       .debug$S                   10000000     U2Lang:U2Lang.dll
 0000:fffbf000       .debug$S                   10000000     U2Lang:U2Lang.dll
 0000:fffbf000       .debug$S                   10000000     U2Lang:U2Lang.dll
 0000:fffbf000       .debug$S                   10000000     U2Lang:U2Lang.dll
 0000:fffbf000       .debug$S                   10000000     U2Lang:U2Lang.dll
 0000:fffbf000       .debug$S                   10000000     U2Lang:U2Lang.dll
 0000:fffbf000       .debug$S                   10000000     U2Lang:U2Lang.dll
 0000:fffbf000       .debug$S                   10000000     U2Lang:U2Lang.dll
 0000:fffbf000       .debug$S                   10000000     U2Lang:U2Lang.dll
 0000:fffbf000       .debug$S                   10000000     U2Lang:U2Lang.dll
 0000:fffbf000       .debug$S                   10000000     U2Lang:U2Lang.dll
 0000:fffbf000       .debug$S                   10000000     U2Lang:U2Lang.dll
 0002:fffdc000       __unwindtable$??A?$QMap@VQString@@VQVariant@@@@QAEAAVQVariant@@ABVQString@@@Z 10000000     KrakenClassifyWorkerFactory.obj
 0000:fffbf000       .debug$S                   10000000     U2Lang:U2Lang.dll
 0002:fffdc000       __unwindtable$??H@YA?BVQString@@ABV0@PBD@Z 10000000     KrakenClassifyWorkerFactory.obj
 0000:fffbf000       .debug$S                   10000000     U2Lang:U2Lang.dll
 0002:fffdc000       __catchsym$?_Copy@?$basic_string@DU?$char_traits@D@std@@V?$allocator@D@2@@std@@QAEXII@Z$5 10000000     KrakenClassifyWorkerFactory.obj
 0000:fffbf000       .debug$S                   10000000     U2Gui:U2Gui.dll
 0002:fffdc000       __catchsym$??0?$QList@VQString@@@@QAE@ABV0@@Z$2 10000000     KrakenClassifyTask.obj
 0001:fffff000       __unwindfunclet$?createNode@?$QMapData@VQString@@PAVPropertyDelegate@U2@@@@QAEPAU?$QMapNode@VQString@@PAVPropertyDelegate@U2@@@@ABVQString@@ABQAVPropertyDelegate@U2@@PAU2@_N@Z$4 10000000 f   KrakenClassifyWorkerFactory.obj
 0001:fffff000       __unwindfunclet$??H@YA?BVQString@@ABV0@PBD@Z$0 10000000 f   KrakenClassifyValidator.obj
 0001:fffff000       __unwindfunclet$??H@YA?BVQString@@ABV0@0@Z$0 10000000 f   KrakenClassifyValidator.obj
 0000:fffbf000       .debug$S                   10000000     U2Lang:U2Lang.dll
 0002:fffdc000       __catchsym$?_Copy@?$basic_string@DU?$char_traits@D@std@@V?$allocator@D@2@@std@@QAEXII@Z$5 10000000     moc_KrakenBuildTask.obj
 0000:fffbf000       .debug$S                   10000000     Qt5Core:Qt5Core.dll
 0000:fffbf000       .debug$S                   10000000     Qt5Core:Qt5Core.dll
 0000:fffbf000       .debug$S                   10000000     Qt5Core:Qt5Core.dll
 0000:fffbf000       .debug$S                   10000000     Qt5Core:Qt5Core.dll
 0000:fffbf000       .debug$S                   10000000     Qt5Core:Qt5Core.dll
 0000:fffbf000       .debug$S                   10000000     Qt5Core:Qt5Core.dll
 0000:fffbf000       .debug$S                   10000000     Qt5Core:Qt5Core.dll
 0000:fffbf000       .debug$S                   10000000     Qt5Core:Qt5Core.dll
 0000:fffbf000       .debug$S                   10000000     Qt5Core:Qt5Core.dll
 0000:fffbf000       .debug$S                   10000000     Qt5Core:Qt5Core.dll
 0000:fffbf000       .debug$S                   10000000     Qt5Core:Qt5Core.dll
 0000:fffbf000       .debug$S                   10000000     Qt5Script:Qt5Script.dll
 0000:fffbf000       .debug$S                   10000000     Qt5Script:Qt5Script.dll
 0000:fffbf000       .debug$S                   10000000     Qt5Script:Qt5Script.dll
 0000:fffbf000       .debug$S                   10000000     Qt5Script:Qt5Script.dll
 0000:fffbf000       .debug$S                   10000000     Qt5Script:Qt5Script.dll
 0000:fffbf000       .debug$S                   10000000     Qt5Script:Qt5Script.dll
 0000:fffbf000       .debug$S                   10000000     Qt5Script:Qt5Script.dll
 0000:fffbf000       .debug$S                   10000000     Qt5Script:Qt5Script.dll
 0000:fffbf000       .debug$S                   10000000     Qt5Script:Qt5Script.dll
 0000:fffbf000       .debug$S                   10000000     Qt5Script:Qt5Script.dll
 0000:fffbf000       .debug$S                   10000000     Qt5Gui:Qt5Gui.dll
 0000:fffbf000       .debug$S                   10000000     Qt5Gui:Qt5Gui.dll
 0000:fffbf000       .debug$S                   10000000     Qt5Gui:Qt5Gui.dll
 0000:fffbf000       .debug$S                   10000000     Qt5Widgets:Qt5Widgets.dll
 0000:fffbf000       .debug$S                   10000000     Qt5Widgets:Qt5Widgets.dll
 0000:fffbf000       .debug$S                   10000000     Qt5Widgets:Qt5Widgets.dll
 0000:fffbf000       .debug$S                   10000000     Qt5Widgets:Qt5Widgets.dll
 0000:fffbf000       .debug$S                   10000000     Qt5Widgets:Qt5Widgets.dll
 0000:fffbf000       .debug$S                   10000000     Qt5Widgets:Qt5Widgets.dll
 0000:fffbf000       .debug$S                   10000000     Qt5Widgets:Qt5Widgets.dll
 0002:fffdc000       ?_System_object$initializer$@?$_Error_objects@H@std@@2P6AXXZA 10000000     KrakenClassifyLogParser.obj
 0002:fffdc000       ?_Iostream_object$initializer$@?$_Error_objects@H@std@@2P6AXXZA 10000000     KrakenClassifyLogParser.obj
 0002:fffdc000       ?_Generic_object$initializer$@?$_Error_objects@H@std@@2P6AXXZA 10000000     KrakenClassifyLogParser.obj
 0000:fffbf000       .debug$S                   10000000     U2Core:U2Core.dll
 0000:fffbf000       .debug$S                   10000000     U2Core:U2Core.dll
 0000:fffbf000       .debug$S                   10000000     U2Core:U2Core.dll
 0000:fffbf000       .debug$S                   10000000     U2Core:U2Core.dll
 0000:fffbf000       .debug$S                   10000000     U2Core:U2Core.dll
 0000:fffbf000       .debug$S                   10000000     U2Core:U2Core.dll
 0000:fffbf000       .debug$S                   10000000     U2Core:U2Core.dll
 0002:fffdc000       ?_Generic_object$initializer$@?$_Error_objects@H@std@@2P6AXXZA 10000000     moc_KrakenBuildTask.obj
 0002:fffdc000       ?_Iostream_object$initializer$@?$_Error_objects@H@std@@2P6AXXZA 10000000     moc_KrakenBuildTask.obj
 0002:fffdc000       ?_System_object$initializer$@?$_Error_objects@H@std@@2P6AXXZA 10000000     moc_KrakenBuildTask.obj
 0000:fffbf000       .debug$S                   10000000     U2Core:U2Core.dll
 0000:fffbf000       .debug$S                   10000000     U2Core:U2Core.dll
 0000:fffbf000       .debug$S                   10000000     U2Core:U2Core.dll
 0000:fffbf000       .debug$S                   10000000     U2Core:U2Core.dll
 0000:fffbf000       .debug$S                   10000000     U2Core:U2Core.dll
 0000:fffbf000       .debug$S                   10000000     U2Core:U2Core.dll
 0002:fffdc000       __catchsym$?node_copy@?$QList@VQString@@@@AAEXPAUNode@1@00@Z$6 10000000     KrakenClassifyLogParser.obj
 0000:fffbf000       .debug$S                   10000000     U2Lang:U2Lang.dll
 0001:fffff000       __unwindfunclet$?createNode@?$QMapData@VDescriptor@U2@@V?$QExplicitlySharedDataPointer@VDataType@U2@@@@@@QAEPAU?$QMapNode@VDescriptor@U2@@V?$QExplicitlySharedDataPointer@VDataType@U2@@@@@@ABVDescriptor@U2@@ABV?$QExplicitlySharedDataPointer@VDataType@U2@@@@PAU2@_N@Z$4 10000000 f   KrakenClassifyWorkerFactory.obj
 0000:fffbf000       .debug$S                   10000000     U2Lang:U2Lang.dll
 0002:fffdc000       __unwindtable$?node_construct@?$QList@VQString@@@@AAEXPAUNode@1@ABVQString@@@Z 10000000     KrakenClassifyLogParser.obj
 0000:fffbf000       .debug$S                   10000000     U2Lang:U2Lang.dll
 0002:fffdc000       __catchsym$?detach_helper_grow@?$QList@VQString@@@@AAEPAUNode@1@HH@Z$5 10000000     KrakenClassifyLogParser.obj
 0000:fffbf000       .debug$S                   10000000     U2Lang:U2Lang.dll
 0000:fffbf000       .debug$S                   10000000     U2Lang:U2Lang.dll
 0000:fffbf000       .debug$S                   10000000     U2Lang:U2Lang.dll
 0001:fffff000       __unwindfunclet$?createNode@?$QMapData@VQString@@VQVariant@@@@QAEPAU?$QMapNode@VQString@@VQVariant@@@@ABVQString@@ABVQVariant@@PAU2@_N@Z$4 10000000 f   KrakenClassifyWorkerFactory.obj
 0002:fffdc000       __catchsym$?append@?$QList@VQString@@@@QAEXABVQString@@@Z$13 10000000     KrakenClassifyLogParser.obj
 0000:fffbf000       .debug$S                   10000000     U2Lang:U2Lang.dll
 0000:fffbf000       .debug$S                   10000000     U2Lang:U2Lang.dll
 0000:fffbf000       .debug$S                   10000000     U2Lang:U2Lang.dll
 0000:fffbf000       .debug$S                   10000000     U2Lang:U2Lang.dll
 0002:fffdc000       __catchsym$??0?$QList@VQString@@@@QAE@ABV0@@Z$2 10000000     KrakenClassifyLogParser.obj
 0000:fffbf000       .debug$S                   10000000     U2Lang:U2Lang.dll
 0000:fffbf000       .debug$S                   10000000     U2Lang:U2Lang.dll
 0000:fffbf000       .debug$S                   10000000     U2Lang:U2Lang.dll
 0002:fffdc000       __catchsym$?_Copy@?$basic_string@DU?$char_traits@D@std@@V?$allocator@D@2@@std@@QAEXII@Z$5 10000000     KrakenClassifyLogParser.obj
 0001:fffff000       __ehhandler$?_Copy@?$basic_string@DU?$char_traits@D@std@@V?$allocator@D@2@@std@@QAEXII@Z 10000000 f   moc_KrakenBuildPrompter.obj
 0000:fffbf000       .debug$S                   10000000     U2Designer:U2Designer.dll
 0002:fffdc000       __catchsym$??0?$QList@VDescriptor@U2@@@@QAE@ABV0@@Z$2 10000000     KrakenClassifyWorker.obj
 0000:fffbf000       .debug$S                   10000000     U2Designer:U2Designer.dll
 0000:fffbf000       .debug$S                   10000000     U2Designer:U2Designer.dll
 0000:fffbf000       .debug$S                   10000000     U2Designer:U2Designer.dll
 0000:fffbf000       .debug$S                   10000000     U2Designer:U2Designer.dll
 0001:fffff000       __unwindfunclet$?node_copy@?$QList@VQString@@@@AAEXPAUNode@1@00@Z$5 10000000 f   KrakenClassifyLogParser.obj
 0002:fffdc000       __catchsym$?append@?$QList@VDescriptor@U2@@@@QAEXABVDescriptor@U2@@@Z$9 10000000     KrakenClassifyWorker.obj
 0000:fffbf000       .debug$S                   10000000     U2Designer:U2Designer.dll
 0001:fffff000       __unwindfunclet$?node_construct@?$QList@VQString@@@@AAEXPAUNode@1@ABVQString@@@Z$1 10000000 f   KrakenClassifyLogParser.obj
 0000:fffbf000       .debug$S                   10000000     U2Designer:U2Designer.dll
 0000:fffbf000       .debug$S                   10000000     U2Designer:U2Designer.dll
 0000:fffbf000       .debug$S                   10000000     U2Designer:U2Designer.dll
 0001:fffff000       __ehhandler$?detach_helper_grow@?$QList@VQString@@@@AAEPAUNode@1@HH@Z 10000000 f   KrakenClassifyLogParser.obj
 0000:fffbf000       .debug$S                   10000000     U2Designer:U2Designer.dll
 0001:fffff000       __unwindfunclet$?append@?$QList@VQString@@@@QAEXABVQString@@@Z$7 10000000 f   KrakenClassifyLogParser.obj
 0002:fffdc000       __catchsym$?detach_helper_grow@?$QList@VDescriptor@U2@@@@AAEPAUNode@1@HH@Z$5 10000000     KrakenClassifyWorker.obj
 0000:fffbf000       .debug$S                   10000000     U2Designer:U2Designer.dll
 0000:fffbf000       .debug$S                   10000000     U2Designer:U2Designer.dll
 0002:fffdc000       __catchsym$?detach_helper@?$QList@VDescriptor@U2@@@@AAEXH@Z$2 10000000     KrakenClassifyWorker.obj
 0000:fffbf000       .debug$S                   10000000     U2Designer:U2Designer.dll
 0000:fffbf000       .debug$S                   10000000     U2Designer:U2Designer.dll
 0002:fffdc000       __unwindtable$?node_construct@?$QList@VDescriptor@U2@@@@AAEXPAUNode@1@ABVDescriptor@U2@@@Z 10000000     KrakenClassifyWorker.obj
 0000:fffbf000       .debug$S                   10000000     U2Designer:U2Designer.dll
 0002:fffdc000       __catchsym$?_Copy@?$basic_string@DU?$char_traits@D@std@@V?$allocator@D@2@@std@@QAEXII@Z$5 10000000     moc_KrakenBuildPrompter.obj
 0000:fffbf000       .debug$S                   10000000     Qt5Widgets:Qt5Widgets.dll
 0000:fffbf000       .debug$S                   10000000     Qt5Widgets:Qt5Widgets.dll
 0000:fffbf000       .debug$S                   10000000     Qt5Widgets:Qt5Widgets.dll
 0000:fffbf000       .debug$S                   10000000     Qt5Widgets:Qt5Widgets.dll
 0000:fffbf000       .debug$S                   10000000     Qt5Widgets:Qt5Widgets.dll
 0000:fffbf000       .debug$S                   10000000     ngs_reads_classification:ngs_reads_classification.dll
 0000:fffbf000       .debug$S                   10000000     ngs_reads_classification:ngs_reads_classification.dll
 0000:fffbf000       .debug$S                   10000000     ngs_reads_classification:ngs_reads_classification.dll
 0000:fffbf000       .debug$S                   10000000     ngs_reads_classification:ngs_reads_classification.dll
 0000:fffbf000       .debug$S                   10000000     ngs_reads_classification:ngs_reads_classification.dll
 0000:fffbf000       .debug$S                   10000000     ngs_reads_classification:ngs_reads_classification.dll
 0000:fffbf000       .debug$S                   10000000     ngs_reads_classification:ngs_reads_classification.dll
 0000:fffbf000       .debug$S                   10000000     ngs_reads_classification:ngs_reads_classification.dll
 0000:fffbf000       .debug$S                   10000000     ngs_reads_classification:ngs_reads_classification.dll
 0000:fffbf000       .debug$S                   10000000     ngs_reads_classification:ngs_reads_classification.dll
 0000:fffbf000       .debug$S                   10000000     ngs_reads_classification:ngs_reads_classification.dll
 0000:fffbf000       .debug$S                   10000000     ngs_reads_classification:ngs_reads_classification.dll
 0000:fffbf000       .debug$S                   10000000     ngs_reads_classification:ngs_reads_classification.dll
 0000:fffbf000       .debug$S                   10000000     ngs_reads_classification:ngs_reads_classification.dll
 0000:fffbf000       .debug$S                   10000000     ngs_reads_classification:ngs_reads_classification.dll
 0000:fffbf000       .debug$S                   10000000     ngs_reads_classification:ngs_reads_classification.dll
 0000:fffbf000       .debug$S                   10000000     ngs_reads_classification:ngs_reads_classification.dll
 0000:fffbf000       .debug$S                   10000000     ngs_reads_classification:ngs_reads_classification.dll
 0000:fffbf000       .debug$S                   10000000     ngs_reads_classification:ngs_reads_classification.dll
 0000:fffbf000       .debug$S                   10000000     ngs_reads_classification:ngs_reads_classification.dll
 0000:fffbf000       .debug$S                   10000000     ngs_reads_classification:ngs_reads_classification.dll
 0000:fffbf000       .debug$S                   10000000     ngs_reads_classification:ngs_reads_classification.dll
 0000:fffbf000       .debug$S                   10000000     ngs_reads_classification:ngs_reads_classification.dll
 0000:fffbf000       .debug$S                   10000000     ngs_reads_classification:ngs_reads_classification.dll
 0000:fffbf000       .debug$S                   10000000     ngs_reads_classification:ngs_reads_classification.dll
 0000:fffbf000       .debug$S                   10000000     ngs_reads_classification:ngs_reads_classification.dll
 0001:fffff000       __ehhandler$??0?$QList@VQString@@@@QAE@ABV0@@Z 10000000 f   KrakenClassifyLogParser.obj
 0000:fffbf000       .debug$S                   10000000     U2Designer:U2Designer.dll
 0002:fffdc000       __catchsym$?node_copy@?$QList@VDescriptor@U2@@@@AAEXPAUNode@1@00@Z$6 10000000     KrakenClassifyWorker.obj
 0001:fffff000       __ehhandler$?_Copy@?$basic_string@DU?$char_traits@D@std@@V?$allocator@D@2@@std@@QAEXII@Z 10000000 f   KrakenClassifyLogParser.obj
 0000:fffbf000       .debug$S                   10000000     U2Designer:U2Designer.dll
 0002:fffdc000       __unwindtable$??A?$QMap@VQString@@VQScriptValue@@@@QAEAAVQScriptValue@@ABVQString@@@Z 10000000     KrakenClassifyWorker.obj
 0000:fffbf000       .debug$S                   10000000     U2Designer:U2Designer.dll
 0002:fffdc000       __unwindtable$?uniqueKeys@?$QMap@VDescriptor@U2@@VQVariant@@@@QBE?AV?$QList@VDescriptor@U2@@@@XZ 10000000     KrakenClassifyWorker.obj
 0002:fffdc000       __ehfuncinfo$??$getAttributeValue@VQString@@@Attribute@U2@@QBE?AVQString@@PAVWorkflowContext@Workflow@1@@Z 10000000     KrakenClassifyWorker.obj
 0002:fffdc000       __ehfuncinfo$??$getAttributeValue@H@Attribute@U2@@QBEHPAVWorkflowContext@Workflow@1@@Z 10000000     KrakenClassifyWorker.obj
 0002:fffdc000       ?_Generic_object$initializer$@?$_Error_objects@H@std@@2P6AXXZA 10000000     moc_KrakenBuildPrompter.obj
 0002:fffdc000       ?_Iostream_object$initializer$@?$_Error_objects@H@std@@2P6AXXZA 10000000     moc_KrakenBuildPrompter.obj
 0002:fffdc000       ?_System_object$initializer$@?$_Error_objects@H@std@@2P6AXXZA 10000000     moc_KrakenBuildPrompter.obj
 0000:fffbf000       .debug$S                   10000000     U2Lang:U2Lang.dll
 0000:fffbf000       .debug$S                   10000000     U2Lang:U2Lang.dll
 0000:fffbf000       .debug$S                   10000000     U2Lang:U2Lang.dll
 0000:fffbf000       .debug$S                   10000000     U2Lang:U2Lang.dll
 0000:fffbf000       .debug$S                   10000000     U2Designer:U2Designer.dll
 0002:fffdc000       __unwindtable$??1KrakenClassifyTaskSettings@U2@@QAE@XZ 10000000     KrakenClassifyWorker.obj
 0000:fffbf000       .debug$S                   10000000     U2Designer:U2Designer.dll
 0002:fffdc000       ?_System_object$initializer$@?$_Error_objects@H@std@@2P6AXXZA 10000000     KrakenClassifyPrompter.obj
 0002:fffdc000       ?_Iostream_object$initializer$@?$_Error_objects@H@std@@2P6AXXZA 10000000     KrakenClassifyPrompter.obj
 0002:fffdc000       ?_Generic_object$initializer$@?$_Error_objects@H@std@@2P6AXXZA 10000000     KrakenClassifyPrompter.obj
 0000:fffbf000       .debug$S                   10000000     U2Core:U2Core.dll
 0000:fffbf000       .debug$S                   10000000     U2Core:U2Core.dll
 0000:fffbf000       .debug$S                   10000000     U2Core:U2Core.dll
 0000:fffbf000       .debug$S                   10000000     U2Core:U2Core.dll
 0000:fffbf000       .debug$S                   10000000     U2Core:U2Core.dll
 0000:fffbf000       .debug$S                   10000000     U2Core:U2Core.dll
 0000:fffbf000       .debug$S                   10000000     U2Core:U2Core.dll
 0000:fffbf000       .debug$S                   10000000     U2Core:U2Core.dll
 0000:fffbf000       .debug$S                   10000000     U2Core:U2Core.dll
 0000:fffbf000       .debug$S                   10000000     U2Core:U2Core.dll
 0000:fffbf000       .debug$S                   10000000     U2Core:U2Core.dll
 0000:fffbf000       .debug$S                   10000000     U2Core:U2Core.dll
 0000:fffbf000       .debug$S                   10000000     U2Core:U2Core.dll
 0002:fffdc000       __catchsym$??0?$QList@PAVPort@Workflow@U2@@@@QAE@ABV0@@Z$2 10000000     KrakenClassifyPrompter.obj
 0000:fffbf000       .debug$S                   10000000     U2Designer:U2Designer.dll
 0000:fffbf000       .debug$S                   10000000     U2Designer:U2Designer.dll
 0001:fffff000       __ehhandler$?_Copy@?$basic_string@DU?$char_traits@D@std@@V?$allocator@D@2@@std@@QAEXII@Z 10000000 f   KrakenTranslateLogParser.obj
 0002:fffdc000       __unwindtable$??0KrakenClassifyTaskSettings@U2@@QAE@ABU01@@Z 10000000     KrakenClassifyWorker.obj
 0000:fffbf000       .debug$S                   10000000     U2Designer:U2Designer.dll
 0001:fffff000       __ehhandler$??0?$QList@VQString@@@@QAE@ABV0@@Z 10000000 f   KrakenTranslateLogParser.obj
 0002:fffdc000       __unwindtable$??$getValue@VQString@@@BaseWorker@LocalWorkflow@U2@@IBE?AVQString@@ABV3@@Z 10000000     KrakenClassifyWorker.obj
 0000:fffbf000       .debug$S                   10000000     U2Lang:U2Lang.dll
 0000:fffbf000       .debug$S                   10000000     U2Lang:U2Lang.dll
 0000:fffbf000       .debug$S                   10000000     U2Lang:U2Lang.dll
 0001:fffff000       __unwindfunclet$?append@?$QList@VQString@@@@QAEXABVQString@@@Z$7 10000000 f   KrakenTranslateLogParser.obj
 0000:fffbf000       .debug$S                   10000000     U2Designer:U2Designer.dll
 0001:fffff000       __ehhandler$?detach_helper_grow@?$QList@VQString@@@@AAEPAUNode@1@HH@Z 10000000 f   KrakenTranslateLogParser.obj
 0000:fffbf000       .debug$S                   10000000     U2Lang:U2Lang.dll
 0000:fffbf000       .debug$S                   10000000     U2Lang:U2Lang.dll
 0000:fffbf000       .debug$S                   10000000     U2Designer:U2Designer.dll
 0001:fffff000       __unwindfunclet$?node_construct@?$QList@VQString@@@@AAEXPAUNode@1@ABVQString@@@Z$1 10000000 f   KrakenTranslateLogParser.obj
 0002:fffdc000       __catchsym$?_Copy@?$basic_string@DU?$char_traits@D@std@@V?$allocator@D@2@@std@@QAEXII@Z$5 10000000     KrakenSupportPlugin.obj
 0000:fffbf000       .debug$S                   10000000     U2Lang:U2Lang.dll
 0001:fffff000       __unwindfunclet$?node_copy@?$QList@VQString@@@@AAEXPAUNode@1@00@Z$5 10000000 f   KrakenTranslateLogParser.obj
 0000:fffbf000       .debug$S                   10000000     U2Lang:U2Lang.dll
 0000:fffbf000       .debug$S                   10000000     U2Core:U2Core.dll
 0002:fffdc000       __catchsym$?_Copy@?$basic_string@DU?$char_traits@D@std@@V?$allocator@D@2@@std@@QAEXII@Z$5 10000000     KrakenClassifyPrompter.obj
 0001:fffff000       __ehhandler$?_Copy@?$basic_string@DU?$char_traits@D@std@@V?$allocator@D@2@@std@@QAEXII@Z 10000000 f   KrakenClassifyValidator.obj
 0000:fffbf000       .debug$S                   10000000     U2Lang:U2Lang.dll
 0002:fffdc000       __catchsym$?append@?$QList@VQString@@@@QAEXABVQString@@@Z$13 10000000     KrakenClassifyTask.obj
 0002:fffdc000       ?_System_object$initializer$@?$_Error_objects@H@std@@2P6AXXZA 10000000     KrakenClassifyWorker.obj
 0002:fffdc000       ?_Iostream_object$initializer$@?$_Error_objects@H@std@@2P6AXXZA 10000000     KrakenClassifyWorker.obj
 0001:fffff000       __ehhandler$??0?$QList@PAVPort@Workflow@U2@@@@QAE@ABV0@@Z 10000000 f   KrakenClassifyPrompter.obj
 0002:fffdc000       __catchsym$?createNode@?$QMapData@VQString@@VQVariant@@@@QAEPAU?$QMapNode@VQString@@VQVariant@@@@ABVQString@@ABVQVariant@@PAU2@_N@Z$7 10000000     KrakenClassifyWorker.obj
 0002:fffdc000       __catchsym$?detach_helper_grow@?$QList@VQString@@@@AAEPAUNode@1@HH@Z$5 10000000     KrakenClassifyTask.obj
 0001:fffff000       __ehhandler$?_Copy@?$basic_string@DU?$char_traits@D@std@@V?$allocator@D@2@@std@@QAEXII@Z 10000000 f   KrakenClassifyPrompter.obj
 0002:fffdc000       __unwindtable$?node_construct@?$QList@VQString@@@@AAEXPAUNode@1@ABVQString@@@Z 10000000     KrakenClassifyTask.obj
 0002:fffdc000       __catchsym$?createNode@?$QMapData@VQString@@VQScriptValue@@@@QAEPAU?$QMapNode@VQString@@VQScriptValue@@@@ABVQString@@ABVQScriptValue@@PAU2@_N@Z$7 10000000     KrakenClassifyWorker.obj
 0002:fffdc000       ?_Generic_object$initializer$@?$_Error_objects@H@std@@2P6AXXZA 10000000     KrakenClassifyWorker.obj
 0002:fffdc000       __catchsym$?createNode@?$QMapData@VQString@@I@@QAEPAU?$QMapNode@VQString@@I@@ABVQString@@ABIPAU2@_N@Z$5 10000000     KrakenClassifyWorker.obj
 0000:fffbf000       .debug$S                   10000000     U2Lang:U2Lang.dll
 0002:fffdc000       __unwindtable$?metaType@?$QVariantValueHelper@VQString@@@QtPrivate@@SA?AVQString@@ABVQVariant@@@Z 10000000     KrakenClassifyWorker.obj
 0000:fffbf000       .debug$S                   10000000     U2Lang:U2Lang.dll
 0000:fffbf000       .debug$S                   10000000     U2Lang:U2Lang.dll
 0000:fffbf000       .debug$S                   10000000     U2Lang:U2Lang.dll
 0000:fffbf000       .debug$S                   10000000     U2Lang:U2Lang.dll
 0000:fffbf000       .debug$S                   10000000     U2Lang:U2Lang.dll
 0000:fffbf000       .debug$S                   10000000     U2Lang:U2Lang.dll
 0002:fffdc000       ?_System_object$initializer$@?$_Error_objects@H@std@@2P6AXXZA 10000000     KrakenClassifyTask.obj
 0002:fffdc000       ?_Iostream_object$initializer$@?$_Error_objects@H@std@@2P6AXXZA 10000000     KrakenClassifyTask.obj
 0002:fffdc000       ?_Generic_object$initializer$@?$_Error_objects@H@std@@2P6AXXZA 10000000     KrakenClassifyTask.obj
 0000:fffbf000       .debug$S                   10000000     U2Lang:U2Lang.dll
 0002:fffdc000       __catchsym$?node_copy@?$QList@VQString@@@@AAEXPAUNode@1@00@Z$6 10000000     KrakenClassifyTask.obj
 0000:fffbf000       .debug$S                   10000000     U2Lang:U2Lang.dll
 0000:fffbf000       .debug$S                   10000000     U2Core:U2Core.dll
 0002:fffdc000       __catchsym$?_Copy@?$basic_string@DU?$char_traits@D@std@@V?$allocator@D@2@@std@@QAEXII@Z$5 10000000     KrakenTranslateLogParser.obj
 0000:fffbf000       .debug$S                   10000000     U2Lang:U2Lang.dll
 0000:fffbf000       .debug$S                   10000000     U2Core:U2Core.dll
 0000:fffbf000       .debug$S                   10000000     U2Core:U2Core.dll
 0002:fffdc000       __catchsym$??0?$QList@VQString@@@@QAE@ABV0@@Z$2 10000000     KrakenTranslateLogParser.obj
 0000:fffbf000       .debug$S                   10000000     U2Core:U2Core.dll
 0000:fffbf000       .debug$S                   10000000     U2Lang:U2Lang.dll
 0000:fffbf000       .debug$S                   10000000     U2Lang:U2Lang.dll
 0000:fffbf000       .debug$S                   10000000     U2Core:U2Core.dll
 0002:fffdc000       __catchsym$?append@?$QList@VQString@@@@QAEXABVQString@@@Z$13 10000000     KrakenTranslateLogParser.obj
 0000:fffbf000       .debug$S                   10000000     U2Lang:U2Lang.dll
 0000:fffbf000       .debug$S                   10000000     U2Core:U2Core.dll
 0000:fffbf000       .debug$S                   10000000     U2Lang:U2Lang.dll
 0000:fffbf000       .debug$S                   10000000     U2Core:U2Core.dll
 0002:fffdc000       __catchsym$?detach_helper_grow@?$QList@VQString@@@@AAEPAUNode@1@HH@Z$5 10000000     KrakenTranslateLogParser.obj
 0000:fffbf000       .debug$S                   10000000     U2Core:U2Core.dll
 0002:fffdc000       __unwindtable$?node_construct@?$QList@VQString@@@@AAEXPAUNode@1@ABVQString@@@Z 10000000     KrakenTranslateLogParser.obj
 0000:fffbf000       .debug$S                   10000000     U2Core:U2Core.dll
 0000:fffbf000       .debug$S                   10000000     U2Lang:U2Lang.dll
 0000:fffbf000       .debug$S                   10000000     U2Core:U2Core.dll
 0002:fffdc000       __catchsym$?node_copy@?$QList@VQString@@@@AAEXPAUNode@1@00@Z$6 10000000     KrakenTranslateLogParser.obj
 0000:fffbf000       .debug$S                   10000000     ngs_reads_classification:ngs_reads_classification.dll
 0000:fffbf000       .debug$S                   10000000     ngs_reads_classification:ngs_reads_classification.dll
 0000:fffbf000       .debug$S                   10000000     ngs_reads_classification:ngs_reads_classification.dll
 0000:fffbf000       .debug$S                   10000000     ngs_reads_classification:ngs_reads_classification.dll
 0000:fffbf000       .debug$S                   10000000     U2Designer:U2Designer.dll
 0000:fffbf000       .debug$S                   10000000     U2Designer:U2Designer.dll
 0000:fffbf000       .debug$S                   10000000     U2Designer:U2Designer.dll
 0000:fffbf000       .debug$S                   10000000     U2Designer:U2Designer.dll
 0000:fffbf000       .debug$S                   10000000     U2Designer:U2Designer.dll
 0000:fffbf000       .debug$S                   10000000     U2Designer:U2Designer.dll
 0000:fffbf000       .debug$S                   10000000     U2Designer:U2Designer.dll
 0000:fffbf000       .debug$S                   10000000     U2Designer:U2Designer.dll
 0000:fffbf000       .debug$S                   10000000     U2Designer:U2Designer.dll
 0000:fffbf000       .debug$S                   10000000     U2Designer:U2Designer.dll
 0000:fffbf000       .debug$S                   10000000     U2Designer:U2Designer.dll
 0000:fffbf000       .debug$S                   10000000     U2Designer:U2Designer.dll
 0000:fffbf000       .debug$S                   10000000     U2Designer:U2Designer.dll
 0000:fffbf000       .debug$S                   10000000     U2Designer:U2Designer.dll
 0000:fffbf000       .debug$S                   10000000     U2Designer:U2Designer.dll
 0000:fffbf000       .debug$S                   10000000     U2Designer:U2Designer.dll
 0000:fffbf000       .debug$S                   10000000     U2Designer:U2Designer.dll
 0000:fffbf000       .debug$S                   10000000     U2Designer:U2Designer.dll
 0000:fffbf000       .debug$S                   10000000     U2Designer:U2Designer.dll
 0000:fffbf000       .debug$S                   10000000     U2Designer:U2Designer.dll
 0000:fffbf000       .debug$S                   10000000     U2Designer:U2Designer.dll
 0000:fffbf000       .debug$S                   10000000     U2Designer:U2Designer.dll
 0000:fffbf000       .debug$S                   10000000     U2Designer:U2Designer.dll
 0000:fffbf000       .debug$S                   10000000     U2Designer:U2Designer.dll
 0000:fffbf000       .debug$S                   10000000     U2Designer:U2Designer.dll
 0000:fffbf000       .debug$S                   10000000     U2Designer:U2Designer.dll
 0000:fffbf000       .debug$S                   10000000     U2Designer:U2Designer.dll
 0000:fffbf000       .debug$S                   10000000     U2Designer:U2Designer.dll
 0000:fffbf000       .debug$S                   10000000     U2Designer:U2Designer.dll
 0000:fffbf000       .debug$S                   10000000     U2Designer:U2Designer.dll
 0000:fffbf000       .debug$S                   10000000     U2Designer:U2Designer.dll
 0000:fffbf000       .debug$S                   10000000     U2Core:U2Core.dll
 0000:fffbf000       .debug$S                   10000000     U2Core:U2Core.dll
 0000:fffbf000       .debug$S                   10000000     U2Core:U2Core.dll
 0000:fffbf000       .debug$S                   10000000     U2Core:U2Core.dll
 0000:fffbf000       .debug$S                   10000000     U2Core:U2Core.dll
 0000:fffbf000       .debug$S                   10000000     U2Core:U2Core.dll
 0000:fffbf000       .debug$S                   10000000     U2Core:U2Core.dll
 0000:fffbf000       .debug$S                   10000000     U2Core:U2Core.dll
 0000:fffbf000       .debug$S                   10000000     U2Core:U2Core.dll
 0000:fffbf000       .debug$S                   10000000     U2Core:U2Core.dll
 0002:fffdc000       ?_Generic_object$initializer$@?$_Error_objects@H@std@@2P6AXXZA 10000000     KrakenTranslateLogParser.obj
 0002:fffdc000       ?_Iostream_object$initializer$@?$_Error_objects@H@std@@2P6AXXZA 10000000     KrakenTranslateLogParser.obj
 0002:fffdc000       ?_System_object$initializer$@?$_Error_objects@H@std@@2P6AXXZA 10000000     KrakenTranslateLogParser.obj
 0000:fffbf000       .debug$S                   10000000     U2Core:U2Core.dll
 0000:fffbf000       .debug$S                   10000000     U2Core:U2Core.dll
 0000:fffbf000       .debug$S                   10000000     U2Core:U2Core.dll
 0000:fffbf000       .debug$S                   10000000     U2Core:U2Core.dll
 0000:fffbf000       .debug$S                   10000000     U2Core:U2Core.dll
 0000:fffbf000       .debug$S                   10000000     U2Core:U2Core.dll
 0000:fffbf000       .debug$S                   10000000     U2Core:U2Core.dll
 0000:fffbf000       .debug$S                   10000000     U2Core:U2Core.dll
 0000:fffbf000       .debug$S                   10000000     U2Core:U2Core.dll
 0000:fffbf000       .debug$S                   10000000     U2Core:U2Core.dll
 0000:fffbf000       .debug$S                   10000000     U2Core:U2Core.dll
 0000:fffbf000       .debug$S                   10000000     U2Core:U2Core.dll
 0000:fffbf000       .debug$S                   10000000     U2Core:U2Core.dll
 0000:fffbf000       .debug$S                   10000000     U2Core:U2Core.dll
 0000:fffbf000       .debug$S                   10000000     U2Core:U2Core.dll
 0000:fffbf000       .debug$S                   10000000     U2Core:U2Core.dll
 0000:fffbf000       .debug$S                   10000000     U2Core:U2Core.dll
 0000:fffbf000       .debug$S                   10000000     U2Core:U2Core.dll
 0000:fffbf000       .debug$S                   10000000     U2Core:U2Core.dll
 0000:fffbf000       .debug$S                   10000000     U2Core:U2Core.dll
 0000:fffbf000       .debug$S                   10000000     U2Core:U2Core.dll
 0000:fffbf000       .debug$S                   10000000     U2Core:U2Core.dll
 0000:fffbf000       .debug$S                   10000000     U2Core:U2Core.dll
 0000:fffbf000       .debug$S                   10000000     U2Core:U2Core.dll
 0000:fffbf000       .debug$S                   10000000     U2Core:U2Core.dll
 0000:fffbf000       .debug$S                   10000000     U2Core:U2Core.dll
 0000:fffbf000       .debug$S                   10000000     U2Core:U2Core.dll
 0000:fffbf000       .debug$S                   10000000     U2Core:U2Core.dll
 0001:fffff000       __ehhandler$?_Copy@?$basic_string@DU?$char_traits@D@std@@V?$allocator@D@2@@std@@QAEXII@Z 10000000 f   KrakenSupportPlugin.obj
 0000:fffbf000       .debug$S                   10000000     U2Lang:U2Lang.dll
 0000:fffbf000       .debug$S                   10000000     U2Lang:U2Lang.dll
 0000:fffbf000       .debug$S                   10000000     U2Core:U2Core.dll
 0000:fffbf000       .debug$S                   10000000     U2Core:U2Core.dll
 0000:fffbf000       .debug$S                   10000000     U2Core:U2Core.dll
 0000:fffbf000       .debug$S                   10000000     U2Core:U2Core.dll
 0000:fffbf000       .debug$S                   10000000     U2Core:U2Core.dll
 0002:fffdc008       __ehfuncinfo$??H@YA?BVQString@@ABV0@0@Z 10000008     KrakenClassifyWorker.obj
 0001:fffff008       __ehhandler$??A?$QMap@VDescriptor@U2@@V?$QExplicitlySharedDataPointer@VDataType@U2@@@@@@QAEAAV?$QExplicitlySharedDataPointer@VDataType@U2@@@@ABVDescriptor@U2@@@Z 10000008 f   KrakenClassifyWorkerFactory.obj
 0002:fffdc008       __ehfuncinfo$??A?$QMap@VQString@@VQVariant@@@@QAEAAVQVariant@@ABVQString@@@Z 10000008     KrakenClassifyWorkerFactory.obj
 0002:fffdc008       __ehfuncinfo$?qt_metatype_id@?$QMetaTypeIdQObject@PAVTask@U2@@$00@@SAHXZ 10000008     moc_KrakenClassifyWorker.obj
 0002:fffdc008       __ehfuncinfo$?uniqueKeys@?$QMap@VDescriptor@U2@@VQVariant@@@@QBE?AV?$QList@VDescriptor@U2@@@@XZ 10000008     KrakenClassifyWorker.obj
 0002:fffdc008       __ehfuncinfo$??A?$QMap@VQString@@VQScriptValue@@@@QAEAAVQScriptValue@@ABVQString@@@Z 10000008     KrakenClassifyWorker.obj
 0002:fffdc008       __ehfuncinfo$??A?$QMap@VQString@@VQVariant@@@@QAEAAVQVariant@@ABVQString@@@Z 10000008     KrakenClassifyWorker.obj
 0002:fffdc008       __ehfuncinfo$??A?$QMap@VDescriptor@U2@@V?$QExplicitlySharedDataPointer@VDataType@U2@@@@@@QAEAAV?$QExplicitlySharedDataPointer@VDataType@U2@@@@ABVDescriptor@U2@@@Z 10000008     KrakenClassifyWorkerFactory.obj
 0002:fffdc008       __ehfuncinfo$??A?$QMap@VQString@@VQVariant@@@@QAEAAVQVariant@@ABVQString@@@Z 10000008     KrakenBuildWorkerFactory.obj
 0002:fffdc008       __ehfuncinfo$??H@YA?BVQString@@ABV0@0@Z 10000008     KrakenClassifyValidator.obj
 0001:fffff009       __unwindfunclet$??0KrakenBuildTaskSettings@U2@@QAE@ABU01@@Z$1 10000009 f   KrakenBuildWorker.obj
 0001:fffff009       __ehhandler$?qt_metatype_id@?$QMetaTypeIdQObject@PAVTask@U2@@$00@@SAHXZ 10000009 f   moc_KrakenClassifyWorker.obj
 0001:fffff009       __ehhandler$??A?$QMap@VQString@@VQScriptValue@@@@QAEAAVQScriptValue@@ABVQString@@@Z 10000009 f   KrakenClassifyWorker.obj
 0001:fffff009       __ehhandler$??A?$QMap@VQString@@VQVariant@@@@QAEAAVQVariant@@ABVQString@@@Z 10000009 f   KrakenClassifyWorkerFactory.obj
 0001:fffff009       __ehhandler$??A?$QMap@VQString@@VQVariant@@@@QAEAAVQVariant@@ABVQString@@@Z 10000009 f   KrakenBuildWorkerFactory.obj
 0001:fffff009       __unwindfunclet$??1KrakenBuildTaskSettings@U2@@QAE@XZ$1 10000009 f   KrakenBuildWorker.obj
 0001:fffff009       __unwindfunclet$??$getAttributeValue@H@Attribute@U2@@QBEHPAVWorkflowContext@Workflow@1@@Z$1 10000009 f   KrakenClassifyWorker.obj
 0001:fffff009       __ehhandler$??A?$QMap@VQString@@VQVariant@@@@QAEAAVQVariant@@ABVQString@@@Z 10000009 f   KrakenClassifyWorker.obj
 0001:fffff009       __unwindfunclet$??0KrakenClassifyTaskSettings@U2@@QAE@ABU01@@Z$1 10000009 f   KrakenClassifyWorker.obj
 0001:fffff009       __unwindfunclet$??1KrakenClassifyTaskSettings@U2@@QAE@XZ$1 10000009 f   KrakenClassifyWorker.obj
 0001:fffff00b       __ehhandler$?node_copy@?$QList@VDescriptor@U2@@@@AAEXPAUNode@1@00@Z 1000000b f   KrakenClassifyWorker.obj
 0001:fffff00b       __ehhandler$?node_construct@?$QList@VWorkflowNotification@U2@@@@AAEXPAUNode@1@ABVWorkflowNotification@U2@@@Z 1000000b f   KrakenClassifyValidator.obj
 0001:fffff00b       __ehhandler$?node_construct@?$QList@VDescriptor@U2@@@@AAEXPAUNode@1@ABVDescriptor@U2@@@Z 1000000b f   KrakenClassifyWorker.obj
 0001:fffff00b       __ehhandler$?node_copy@?$QList@VWorkflowNotification@U2@@@@AAEXPAUNode@1@00@Z 1000000b f   KrakenClassifyValidator.obj
 0001:fffff00b       __ehhandler$?append@?$QList@VWorkflowNotification@U2@@@@QAEXABVWorkflowNotification@U2@@@Z 1000000b f   KrakenClassifyValidator.obj
 0001:fffff00b       __ehhandler$?append@?$QList@VDescriptor@U2@@@@QAEXABVDescriptor@U2@@@Z 1000000b f   KrakenClassifyWorker.obj
 0002:fffdc010       __ehfuncinfo$??H@YA?BVQString@@ABV0@PBD@Z 10000010     KrakenSupport.obj
 0002:fffdc010       __catchsym$?_Copy@?$basic_string@DU?$char_traits@D@std@@V?$allocator@D@2@@std@@QAEXII@Z$4 10000010     KrakenClassifyValidator.obj
 0002:fffdc010       __catchsym$?_Copy@?$basic_string@DU?$char_traits@D@std@@V?$allocator@D@2@@std@@QAEXII@Z$4 10000010     moc_KrakenClassifyTask.obj
 0002:fffdc010       __ehfuncinfo$??$getValue@VQString@@@BaseWorker@LocalWorkflow@U2@@IBE?AVQString@@ABV3@@Z 10000010     KrakenClassifyWorker.obj
 0002:fffdc010       __unwindtable$??0?$QList@PAVPort@Workflow@U2@@@@QAE@ABV0@@Z 10000010     KrakenClassifyPrompter.obj
 0002:fffdc010       __catchsym$?_Copy@?$basic_string@DU?$char_traits@D@std@@V?$allocator@D@2@@std@@QAEXII@Z$4 10000010     KrakenSupportPlugin.obj
 0002:fffdc010       __catchsym$?_Copy@?$basic_string@DU?$char_traits@D@std@@V?$allocator@D@2@@std@@QAEXII@Z$4 10000010     moc_KrakenSupport.obj
 0002:fffdc010       __catchsym$?_Copy@?$basic_string@DU?$char_traits@D@std@@V?$allocator@D@2@@std@@QAEXII@Z$4 10000010     KrakenBuildPrompter.obj
 0002:fffdc010       __catchsym$?_Copy@?$basic_string@DU?$char_traits@D@std@@V?$allocator@D@2@@std@@QAEXII@Z$4 10000010     KrakenClassifyPrompter.obj
 0002:fffdc010       __catchsym$?_Copy@?$basic_string@DU?$char_traits@D@std@@V?$allocator@D@2@@std@@QAEXII@Z$4 10000010     moc_KrakenSupportPlugin.obj
 0002:fffdc010       __tryblocktable$?node_copy@?$QList@VDescriptor@U2@@@@AAEXPAUNode@1@00@Z 10000010     KrakenClassifyWorker.obj
 0002:fffdc010       __catchsym$?_Copy@?$basic_string@DU?$char_traits@D@std@@V?$allocator@D@2@@std@@QAEXII@Z$4 10000010     moc_KrakenBuildPrompter.obj
 0002:fffdc010       __catchsym$?createNode@?$QMapData@VQString@@VQVariant@@@@QAEPAU?$QMapNode@VQString@@VQVariant@@@@ABVQString@@ABVQVariant@@PAU2@_N@Z$6 10000010     KrakenClassifyWorker.obj
 0002:fffdc010       __ehfuncinfo$?node_construct@?$QList@VDescriptor@U2@@@@AAEXPAUNode@1@ABVDescriptor@U2@@@Z 10000010     KrakenClassifyWorker.obj
 0002:fffdc010       __catchsym$?detach_helper_grow@?$QList@VQString@@@@AAEPAUNode@1@HH@Z$4 10000010     KrakenClassifyTask.obj
 0002:fffdc010       __unwindtable$?detach_helper@?$QList@VDescriptor@U2@@@@AAEXH@Z 10000010     KrakenClassifyWorker.obj
 0002:fffdc010       __tryblocktable$?node_copy@?$QList@VQString@@@@AAEXPAUNode@1@00@Z 10000010     KrakenClassifyWorker.obj
 0002:fffdc010       __catchsym$?detach_helper_grow@?$QList@VDescriptor@U2@@@@AAEPAUNode@1@HH@Z$4 10000010     KrakenClassifyWorker.obj
 0002:fffdc010       __ehfuncinfo$?node_construct@?$QList@VQString@@@@AAEXPAUNode@1@ABVQString@@@Z 10000010     KrakenClassifyTask.obj
 0002:fffdc010       __tryblocktable$?node_copy@?$QList@VQString@@@@AAEXPAUNode@1@00@Z 10000010     KrakenBuildWorker.obj
 0002:fffdc010       __ehfuncinfo$?node_construct@?$QList@VQString@@@@AAEXPAUNode@1@ABVQString@@@Z 10000010     KrakenBuildWorker.obj
 0002:fffdc010       __catchsym$?append@?$QList@VDescriptor@U2@@@@QAEXABVDescriptor@U2@@@Z$8 10000010     KrakenClassifyWorker.obj
 0002:fffdc010       __ehfuncinfo$??H@YA?BVQString@@ABV0@PBD@Z 10000010     KrakenBuildTask.obj
 0002:fffdc010       __catchsym$?append@?$QList@VWorkflowNotification@U2@@@@QAEXABVWorkflowNotification@U2@@@Z$10 10000010     KrakenClassifyValidator.obj
 0002:fffdc010       __catchsym$?_Copy@?$basic_string@DU?$char_traits@D@std@@V?$allocator@D@2@@std@@QAEXII@Z$4 10000010     KrakenClassifyLogParser.obj
 0002:fffdc010       __catchsym$?_Copy@?$basic_string@DU?$char_traits@D@std@@V?$allocator@D@2@@std@@QAEXII@Z$4 10000010     KrakenBuildTask.obj
 0002:fffdc010       __unwindtable$??0?$QList@VDescriptor@U2@@@@QAE@ABV0@@Z 10000010     KrakenClassifyWorker.obj
 0002:fffdc010       __unwindtable$??0?$QList@VQString@@@@QAE@ABV0@@Z 10000010     KrakenClassifyLogParser.obj
 0002:fffdc010       __catchsym$?createNode@?$QMapData@VQString@@VQScriptValue@@@@QAEPAU?$QMapNode@VQString@@VQScriptValue@@@@ABVQString@@ABVQScriptValue@@PAU2@_N@Z$6 10000010     KrakenClassifyWorker.obj
 0002:fffdc010       __catchsym$?detach_helper_grow@?$QList@VWorkflowNotification@U2@@@@AAEPAUNode@1@HH@Z$4 10000010     KrakenClassifyValidator.obj
 0002:fffdc010       __catchsym$?append@?$QList@VQString@@@@QAEXABVQString@@@Z$12 10000010     KrakenClassifyLogParser.obj
 0002:fffdc010       __catchsym$?detach_helper_grow@?$QList@VQString@@@@AAEPAUNode@1@HH@Z$4 10000010     KrakenBuildWorker.obj
 0002:fffdc010       __tryblocktable$?createNode@?$QMapData@VQString@@I@@QAEPAU?$QMapNode@VQString@@I@@ABVQString@@ABIPAU2@_N@Z 10000010     KrakenClassifyWorker.obj
 0002:fffdc010       __catchsym$?detach_helper_grow@?$QList@VQString@@@@AAEPAUNode@1@HH@Z$4 10000010     KrakenClassifyLogParser.obj
 0002:fffdc010       __ehfuncinfo$?node_construct@?$QList@VQString@@@@AAEXPAUNode@1@ABVQString@@@Z 10000010     KrakenClassifyLogParser.obj
 0002:fffdc010       __unwindtable$??0?$QList@VQString@@@@QAE@ABV0@@Z 10000010     KrakenSupport.obj
 0002:fffdc010       __tryblocktable$?node_copy@?$QList@VQString@@@@AAEXPAUNode@1@00@Z 10000010     KrakenClassifyLogParser.obj
 0002:fffdc010       __catchsym$?_Copy@?$basic_string@DU?$char_traits@D@std@@V?$allocator@D@2@@std@@QAEXII@Z$4 10000010     moc_KrakenBuildTask.obj
 0002:fffdc010       __catchsym$?append@?$QList@VQString@@@@QAEXABVQString@@@Z$12 10000010     KrakenClassifyTask.obj
 0002:fffdc010       __tryblocktable$?node_copy@?$QList@VWorkflowNotification@U2@@@@AAEXPAUNode@1@00@Z 10000010     KrakenClassifyValidator.obj
 0002:fffdc010       __ehfuncinfo$?metaType@?$QVariantValueHelper@VQString@@@QtPrivate@@SA?AVQString@@ABVQVariant@@@Z 10000010     KrakenClassifyValidator.obj
 0002:fffdc010       __ehfuncinfo$?metaType@?$QVariantValueHelper@VQString@@@QtPrivate@@SA?AVQString@@ABVQVariant@@@Z 10000010     KrakenClassifyWorker.obj
 0002:fffdc010       __catchsym$?_Copy@?$basic_string@DU?$char_traits@D@std@@V?$allocator@D@2@@std@@QAEXII@Z$4 10000010     KrakenClassifyWorker.obj
 0002:fffdc010       __catchsym$?_Copy@?$basic_string@DU?$char_traits@D@std@@V?$allocator@D@2@@std@@QAEXII@Z$4 10000010     moc_KrakenClassifyWorker.obj
 0002:fffdc010       __unwindtable$??0?$QList@VQString@@@@QAE@ABV0@@Z 10000010     KrakenClassifyTask.obj
 0002:fffdc010       __tryblocktable$?node_copy@?$QList@VQString@@@@AAEXPAUNode@1@00@Z 10000010     KrakenTranslateLogParser.obj
 0002:fffdc010       __catchsym$?_Copy@?$basic_string@DU?$char_traits@D@std@@V?$allocator@D@2@@std@@QAEXII@Z$4 10000010     KrakenClassifyWorkerFactory.obj
 0002:fffdc010       __ehfuncinfo$??H@YA?BVQString@@ABV0@PBD@Z 10000010     KrakenClassifyWorkerFactory.obj
 0002:fffdc010       __tryblocktable$?node_copy@?$QList@VQString@@@@AAEXPAUNode@1@00@Z 10000010     KrakenClassifyTask.obj
 0002:fffdc010       __ehfuncinfo$??H@YA?BVQString@@ABV0@PBD@Z 10000010     KrakenClassifyWorker.obj
 0002:fffdc010       __tryblocktable$?node_copy@?$QList@VQString@@@@AAEXPAUNode@1@00@Z 10000010     KrakenClassifyValidator.obj
 0002:fffdc010       __catchsym$?_Copy@?$basic_string@DU?$char_traits@D@std@@V?$allocator@D@2@@std@@QAEXII@Z$4 10000010     KrakenTranslateLogParser.obj
 0002:fffdc010       __tryblocktable$?node_copy@?$QList@VQString@@@@AAEXPAUNode@1@00@Z 10000010     KrakenBuildValidator.obj
 0002:fffdc010       __catchsym$?_Copy@?$basic_string@DU?$char_traits@D@std@@V?$allocator@D@2@@std@@QAEXII@Z$4 10000010     KrakenBuildWorkerFactory.obj
 0002:fffdc010       __ehfuncinfo$??H@YA?BVQString@@ABV0@PBD@Z 10000010     KrakenBuildWorkerFactory.obj
 0002:fffdc010       __unwindtable$??0?$QList@VQString@@@@QAE@ABV0@@Z 10000010     KrakenTranslateLogParser.obj
 0002:fffdc010       __ehfuncinfo$?node_construct@?$QList@VQString@@@@AAEXPAUNode@1@ABVQString@@@Z 10000010     KrakenBuildValidator.obj
 0002:fffdc010       __catchsym$?createNode@?$QMapData@VQString@@VQVariant@@@@QAEPAU?$QMapNode@VQString@@VQVariant@@@@ABVQString@@ABVQVariant@@PAU2@_N@Z$6 10000010     KrakenBuildWorkerFactory.obj
 0002:fffdc010       __catchsym$?_Copy@?$basic_string@DU?$char_traits@D@std@@V?$allocator@D@2@@std@@QAEXII@Z$4 10000010     KrakenClassifyTask.obj
 0002:fffdc010       __catchsym$?_Copy@?$basic_string@DU?$char_traits@D@std@@V?$allocator@D@2@@std@@QAEXII@Z$4 10000010     moc_KrakenBuildWorker.obj
 0002:fffdc010       __catchsym$?detach_helper_grow@?$QList@VQString@@@@AAEPAUNode@1@HH@Z$4 10000010     KrakenBuildValidator.obj
 0002:fffdc010       __catchsym$?append@?$QList@VQString@@@@QAEXABVQString@@@Z$12 10000010     KrakenBuildValidator.obj
 0002:fffdc010       __catchsym$?append@?$QList@VQString@@@@QAEXABVQString@@@Z$12 10000010     KrakenClassifyValidator.obj
 0002:fffdc010       __catchsym$?append@?$QList@VQString@@@@QAEXABVQString@@@Z$12 10000010     KrakenBuildWorker.obj
 0002:fffdc010       __ehfuncinfo$?node_construct@?$QList@VQString@@@@AAEXPAUNode@1@ABVQString@@@Z 10000010     KrakenClassifyWorker.obj
 0002:fffdc010       __tryblocktable$?append@?$QList@PAVAttribute@U2@@@@QAEXABQAVAttribute@U2@@@Z 10000010     KrakenClassifyWorkerFactory.obj
 0002:fffdc010       __ehfuncinfo$??H@YA?BVQString@@ABV0@PBD@Z 10000010     KrakenClassifyValidator.obj
 0002:fffdc010       __catchsym$?append@?$QList@VQString@@@@QAEXABVQString@@@Z$12 10000010     KrakenClassifyWorker.obj
 0002:fffdc010       __catchsym$?detach_helper_grow@?$QList@PAVAttribute@U2@@@@AAEPAUNode@1@HH@Z$4 10000010     KrakenClassifyWorkerFactory.obj
 0002:fffdc010       __catchsym$?append@?$QList@VQString@@@@QAEXABVQString@@@Z$12 10000010     KrakenSupport.obj
 0002:fffdc010       __tryblocktable$?append@?$QList@PAVPortDescriptor@Workflow@U2@@@@QAEXABQAVPortDescriptor@Workflow@U2@@@Z 10000010     KrakenClassifyWorkerFactory.obj
 0002:fffdc010       __unwindtable$??0?$QList@VQString@@@@QAE@ABV0@@Z 10000010     KrakenBuildWorker.obj
 0002:fffdc010       __unwindtable$??0?$QList@VQString@@@@QAE@ABV0@@Z 10000010     KrakenBuildValidator.obj
 0002:fffdc010       __tryblocktable$?node_copy@?$QList@VQString@@@@AAEXPAUNode@1@00@Z 10000010     KrakenSupport.obj
 0002:fffdc010       __catchsym$?detach_helper_grow@?$QList@PAVPortDescriptor@Workflow@U2@@@@AAEPAUNode@1@HH@Z$4 10000010     KrakenClassifyWorkerFactory.obj
 0002:fffdc010       __catchsym$?_Copy@?$basic_string@DU?$char_traits@D@std@@V?$allocator@D@2@@std@@QAEXII@Z$4 10000010     KrakenBuildValidator.obj
 0002:fffdc010       __catchsym$?createNode@?$QMapData@VQString@@VQVariant@@@@QAEPAU?$QMapNode@VQString@@VQVariant@@@@ABVQString@@ABVQVariant@@PAU2@_N@Z$6 10000010     KrakenClassifyWorkerFactory.obj
 0002:fffdc010       __tryblocktable$?createNode@?$QMapData@VDescriptor@U2@@V?$QExplicitlySharedDataPointer@VDataType@U2@@@@@@QAEPAU?$QMapNode@VDescriptor@U2@@V?$QExplicitlySharedDataPointer@VDataType@U2@@@@@@ABVDescriptor@U2@@ABV?$QExplicitlySharedDataPointer@VDataType@U2@@@@PAU2@_N@Z 10000010     KrakenClassifyWorkerFactory.obj
 0002:fffdc010       __catchsym$?append@?$QList@VQString@@@@QAEXABVQString@@@Z$12 10000010     KrakenTranslateLogParser.obj
 0002:fffdc010       __tryblocktable$?createNode@?$QMapData@VQString@@PAVPropertyDelegate@U2@@@@QAEPAU?$QMapNode@VQString@@PAVPropertyDelegate@U2@@@@ABVQString@@ABQAVPropertyDelegate@U2@@PAU2@_N@Z 10000010     KrakenClassifyWorkerFactory.obj
 0002:fffdc010       __catchsym$?_Copy@?$basic_string@DU?$char_traits@D@std@@V?$allocator@D@2@@std@@QAEXII@Z$4 10000010     moc_KrakenClassifyPrompter.obj
 0002:fffdc010       __catchsym$?_Copy@?$basic_string@DU?$char_traits@D@std@@V?$allocator@D@2@@std@@QAEXII@Z$4 10000010     KrakenBuildWorker.obj
 0002:fffdc010       __ehfuncinfo$?node_construct@?$QList@VQString@@@@AAEXPAUNode@1@ABVQString@@@Z 10000010     KrakenClassifyValidator.obj
 0002:fffdc010       __catchsym$?detach_helper_grow@?$QList@VQString@@@@AAEPAUNode@1@HH@Z$4 10000010     KrakenClassifyWorker.obj
 0002:fffdc010       __unwindtable$??0?$QList@VQString@@@@QAE@ABV0@@Z 10000010     KrakenClassifyValidator.obj
 0002:fffdc010       __catchsym$?detach_helper_grow@?$QList@VQString@@@@AAEPAUNode@1@HH@Z$4 10000010     KrakenTranslateLogParser.obj
 0002:fffdc010       __ehfuncinfo$?node_construct@?$QList@VQString@@@@AAEXPAUNode@1@ABVQString@@@Z 10000010     KrakenTranslateLogParser.obj
 0002:fffdc010       __catchsym$?detach_helper_grow@?$QList@VQString@@@@AAEPAUNode@1@HH@Z$4 10000010     KrakenClassifyValidator.obj
 0002:fffdc010       __ehfuncinfo$?node_construct@?$QList@VQString@@@@AAEXPAUNode@1@ABVQString@@@Z 10000010     KrakenSupport.obj
 0002:fffdc010       __ehfuncinfo$?node_construct@?$QList@VWorkflowNotification@U2@@@@AAEXPAUNode@1@ABVWorkflowNotification@U2@@@Z 10000010     KrakenClassifyValidator.obj
 0002:fffdc010       __catchsym$?detach_helper_grow@?$QList@VQString@@@@AAEPAUNode@1@HH@Z$4 10000010     KrakenSupport.obj
 0002:fffdc010       __catchsym$?_Copy@?$basic_string@DU?$char_traits@D@std@@V?$allocator@D@2@@std@@QAEXII@Z$4 10000010     KrakenSupport.obj
 0001:fffff011       __ehhandler$?node_copy@?$QList@VQString@@@@AAEXPAUNode@1@00@Z 10000011 f   KrakenSupport.obj
 0001:fffff011       __ehhandler$?node_construct@?$QList@VQString@@@@AAEXPAUNode@1@ABVQString@@@Z 10000011 f   KrakenSupport.obj
 0001:fffff011       __ehhandler$?node_copy@?$QList@VQString@@@@AAEXPAUNode@1@00@Z 10000011 f   KrakenBuildValidator.obj
 0001:fffff011       __ehhandler$?node_copy@?$QList@VQString@@@@AAEXPAUNode@1@00@Z 10000011 f   KrakenBuildWorker.obj
 0001:fffff011       __ehhandler$?node_construct@?$QList@VQString@@@@AAEXPAUNode@1@ABVQString@@@Z 10000011 f   KrakenBuildWorker.obj
 0001:fffff011       __unwindfunclet$?append@?$QList@VQString@@@@QAEXABVQString@@@Z$11 10000011 f   KrakenSupport.obj
 0001:fffff011       __unwindfunclet$?append@?$QList@VQString@@@@QAEXABVQString@@@Z$11 10000011 f   KrakenBuildWorker.obj
 0001:fffff011       __ehhandler$?node_construct@?$QList@VQString@@@@AAEXPAUNode@1@ABVQString@@@Z 10000011 f   KrakenBuildValidator.obj
 0001:fffff011       __ehhandler$?node_copy@?$QList@VQString@@@@AAEXPAUNode@1@00@Z 10000011 f   KrakenClassifyValidator.obj
 0001:fffff011       __ehhandler$?node_construct@?$QList@VQString@@@@AAEXPAUNode@1@ABVQString@@@Z 10000011 f   KrakenClassifyValidator.obj
 0001:fffff011       __ehhandler$?node_construct@?$QList@VQString@@@@AAEXPAUNode@1@ABVQString@@@Z 10000011 f   KrakenClassifyTask.obj
 0001:fffff011       __ehhandler$?node_copy@?$QList@VQString@@@@AAEXPAUNode@1@00@Z 10000011 f   KrakenClassifyTask.obj
 0001:fffff011       __unwindfunclet$?append@?$QList@VQString@@@@QAEXABVQString@@@Z$11 10000011 f   KrakenBuildValidator.obj
 0001:fffff011       __unwindfunclet$?append@?$QList@VQString@@@@QAEXABVQString@@@Z$11 10000011 f   KrakenClassifyValidator.obj
 0001:fffff011       __unwindfunclet$?append@?$QList@VQString@@@@QAEXABVQString@@@Z$11 10000011 f   KrakenClassifyWorker.obj
 0001:fffff011       __ehhandler$?node_construct@?$QList@VQString@@@@AAEXPAUNode@1@ABVQString@@@Z 10000011 f   KrakenClassifyWorker.obj
 0001:fffff011       __ehhandler$?node_copy@?$QList@VQString@@@@AAEXPAUNode@1@00@Z 10000011 f   KrakenClassifyLogParser.obj
 0001:fffff011       __ehhandler$?node_construct@?$QList@VQString@@@@AAEXPAUNode@1@ABVQString@@@Z 10000011 f   KrakenClassifyLogParser.obj
 0001:fffff011       __ehhandler$?node_copy@?$QList@VQString@@@@AAEXPAUNode@1@00@Z 10000011 f   KrakenClassifyWorker.obj
 0001:fffff011       __unwindfunclet$?append@?$QList@VQString@@@@QAEXABVQString@@@Z$11 10000011 f   KrakenClassifyLogParser.obj
 0001:fffff011       __unwindfunclet$?append@?$QList@VQString@@@@QAEXABVQString@@@Z$11 10000011 f   KrakenTranslateLogParser.obj
 0001:fffff011       __ehhandler$?node_construct@?$QList@VQString@@@@AAEXPAUNode@1@ABVQString@@@Z 10000011 f   KrakenTranslateLogParser.obj
 0001:fffff011       __ehhandler$?node_copy@?$QList@VQString@@@@AAEXPAUNode@1@00@Z 10000011 f   KrakenTranslateLogParser.obj
 0001:fffff011       __unwindfunclet$??$getAttributeValue@H@Attribute@U2@@QBEHPAVWorkflowContext@Workflow@1@@Z$2 10000011 f   KrakenClassifyWorker.obj
 0001:fffff011       __unwindfunclet$?append@?$QList@VQString@@@@QAEXABVQString@@@Z$11 10000011 f   KrakenClassifyTask.obj
 0001:fffff014       __unwindfunclet$?createNode@?$QMapData@VQString@@VQVariant@@@@QAEPAU?$QMapNode@VQString@@VQVariant@@@@ABVQString@@ABVQVariant@@PAU2@_N@Z$5 10000014 f   KrakenBuildWorkerFactory.obj
 0001:fffff014       __ehhandler$?createNode@?$QMapData@VQString@@I@@QAEPAU?$QMapNode@VQString@@I@@ABVQString@@ABIPAU2@_N@Z 10000014 f   KrakenClassifyWorker.obj
 0001:fffff014       __unwindfunclet$?createNode@?$QMapData@VQString@@VQScriptValue@@@@QAEPAU?$QMapNode@VQString@@VQScriptValue@@@@ABVQString@@ABVQScriptValue@@PAU2@_N@Z$5 10000014 f   KrakenClassifyWorker.obj
 0001:fffff014       __unwindfunclet$?createNode@?$QMapData@VQString@@VQVariant@@@@QAEPAU?$QMapNode@VQString@@VQVariant@@@@ABVQString@@ABVQVariant@@PAU2@_N@Z$5 10000014 f   KrakenClassifyWorkerFactory.obj
 0001:fffff014       __ehhandler$?createNode@?$QMapData@VQString@@PAVPropertyDelegate@U2@@@@QAEPAU?$QMapNode@VQString@@PAVPropertyDelegate@U2@@@@ABVQString@@ABQAVPropertyDelegate@U2@@PAU2@_N@Z 10000014 f   KrakenClassifyWorkerFactory.obj
 0001:fffff014       __ehhandler$?createNode@?$QMapData@VDescriptor@U2@@V?$QExplicitlySharedDataPointer@VDataType@U2@@@@@@QAEPAU?$QMapNode@VDescriptor@U2@@V?$QExplicitlySharedDataPointer@VDataType@U2@@@@@@ABVDescriptor@U2@@ABV?$QExplicitlySharedDataPointer@VDataType@U2@@@@PAU2@_N@Z 10000014 f   KrakenClassifyWorkerFactory.obj
 0001:fffff014       __unwindfunclet$?createNode@?$QMapData@VQString@@VQVariant@@@@QAEPAU?$QMapNode@VQString@@VQVariant@@@@ABVQString@@ABVQVariant@@PAU2@_N@Z$5 10000014 f   KrakenClassifyWorker.obj
 0001:fffff015       __unwindfunclet$??0KrakenClassifyTaskSettings@U2@@QAE@ABU01@@Z$2 10000015 f   KrakenClassifyWorker.obj
 0001:fffff015       __unwindfunclet$??1KrakenBuildTaskSettings@U2@@QAE@XZ$2 10000015 f   KrakenBuildWorker.obj
 0001:fffff015       __unwindfunclet$??1KrakenClassifyTaskSettings@U2@@QAE@XZ$2 10000015 f   KrakenClassifyWorker.obj
 0001:fffff015       __unwindfunclet$??0KrakenBuildTaskSettings@U2@@QAE@ABU01@@Z$2 10000015 f   KrakenBuildWorker.obj
 0002:fffdc018       __ehfuncinfo$??0KrakenBuildTaskSettings@U2@@QAE@ABU01@@Z 10000018     KrakenBuildWorker.obj
 0002:fffdc018       __ehfuncinfo$??1KrakenBuildTaskSettings@U2@@QAE@XZ 10000018     KrakenBuildWorker.obj
 0002:fffdc018       __ehfuncinfo$??0KrakenClassifyTaskSettings@U2@@QAE@ABU01@@Z 10000018     KrakenClassifyWorker.obj
 0002:fffdc018       __ehfuncinfo$??1KrakenClassifyTaskSettings@U2@@QAE@XZ 10000018     KrakenClassifyWorker.obj
 0001:fffff019       __unwindfunclet$??$getAttributeValue@H@Attribute@U2@@QBEHPAVWorkflowContext@Workflow@1@@Z$3 10000019 f   KrakenClassifyWorker.obj
 0001:fffff019       __ehhandler$?uniqueKeys@?$QMap@VDescriptor@U2@@VQVariant@@@@QBE?AV?$QList@VDescriptor@U2@@@@XZ 10000019 f   KrakenClassifyWorker.obj
 0001:fffff01a       __unwindfunclet$??H@YA?BVQString@@ABV0@PBD@Z$1 1000001a f   KrakenClassifyWorkerFactory.obj
 0001:fffff01a       __unwindfunclet$??H@YA?BVQString@@ABV0@PBD@Z$1 1000001a f   KrakenBuildTask.obj
 0001:fffff01a       __unwindfunclet$??$getValue@VQString@@@BaseWorker@LocalWorkflow@U2@@IBE?AVQString@@ABV3@@Z$1 1000001a f   KrakenClassifyWorker.obj
 0001:fffff01a       __unwindfunclet$??H@YA?BVQString@@ABV0@PBD@Z$1 1000001a f   KrakenSupport.obj
 0001:fffff01a       __ehhandler$??H@YA?BVQString@@ABV0@0@Z 1000001a f   KrakenClassifyValidator.obj
 0001:fffff01a       __unwindfunclet$?metaType@?$QVariantValueHelper@VQString@@@QtPrivate@@SA?AVQString@@ABVQVariant@@@Z$1 1000001a f   KrakenClassifyValidator.obj
 0001:fffff01a       __unwindfunclet$??H@YA?BVQString@@ABV0@PBD@Z$1 1000001a f   KrakenClassifyWorker.obj
 0001:fffff01a       __ehhandler$??H@YA?BVQString@@ABV0@0@Z 1000001a f   KrakenClassifyWorker.obj
 0001:fffff01a       __unwindfunclet$??$getAttributeValue@VQString@@@Attribute@U2@@QBE?AVQString@@PAVWorkflowContext@Workflow@1@@Z$1 1000001a f   KrakenClassifyWorker.obj
 0001:fffff01a       __unwindfunclet$??H@YA?BVQString@@ABV0@PBD@Z$1 1000001a f   KrakenClassifyValidator.obj
 0001:fffff01a       __unwindfunclet$??H@YA?BVQString@@ABV0@PBD@Z$1 1000001a f   KrakenBuildWorkerFactory.obj
 0001:fffff01a       __unwindfunclet$?metaType@?$QVariantValueHelper@VQString@@@QtPrivate@@SA?AVQString@@ABVQVariant@@@Z$1 1000001a f   KrakenClassifyWorker.obj
 0002:fffdc020       __unwindtable$?detach_helper_grow@?$QList@VQString@@@@AAEPAUNode@1@HH@Z 10000020     KrakenBuildValidator.obj
 0002:fffdc020       __unwindtable$?_Copy@?$basic_string@DU?$char_traits@D@std@@V?$allocator@D@2@@std@@QAEXII@Z 10000020     KrakenClassifyTask.obj
 0002:fffdc020       __ehfuncinfo$?createNode@?$QMapData@VQString@@VQVariant@@@@QAEPAU?$QMapNode@VQString@@VQVariant@@@@ABVQString@@ABVQVariant@@PAU2@_N@Z 10000020     KrakenBuildWorkerFactory.obj
 0002:fffdc020       __unwindtable$?_Copy@?$basic_string@DU?$char_traits@D@std@@V?$allocator@D@2@@std@@QAEXII@Z 10000020     KrakenBuildWorkerFactory.obj
 0002:fffdc020       __ehfuncinfo$?append@?$QList@VQString@@@@QAEXABVQString@@@Z 10000020     KrakenClassifyWorker.obj
 0002:fffdc020       __unwindtable$?_Copy@?$basic_string@DU?$char_traits@D@std@@V?$allocator@D@2@@std@@QAEXII@Z 10000020     moc_KrakenBuildWorker.obj
 0002:fffdc020       __unwindtable$?detach_helper_grow@?$QList@PAVAttribute@U2@@@@AAEPAUNode@1@HH@Z 10000020     KrakenClassifyWorkerFactory.obj
 0002:fffdc020       __tryblocktable$??0?$QList@VQString@@@@QAE@ABV0@@Z 10000020     KrakenClassifyTask.obj
 0002:fffdc020       __unwindtable$?_Copy@?$basic_string@DU?$char_traits@D@std@@V?$allocator@D@2@@std@@QAEXII@Z 10000020     moc_KrakenClassifyWorker.obj
 0002:fffdc020       __unwindtable$?_Copy@?$basic_string@DU?$char_traits@D@std@@V?$allocator@D@2@@std@@QAEXII@Z 10000020     KrakenClassifyWorkerFactory.obj
 0002:fffdc020       __ehfuncinfo$?append@?$QList@VQString@@@@QAEXABVQString@@@Z 10000020     KrakenClassifyTask.obj
 0002:fffdc020       __unwindtable$?_Copy@?$basic_string@DU?$char_traits@D@std@@V?$allocator@D@2@@std@@QAEXII@Z 10000020     KrakenClassifyWorker.obj
 0002:fffdc020       __ehfuncinfo$?append@?$QList@VQString@@@@QAEXABVQString@@@Z 10000020     KrakenBuildValidator.obj
 0002:fffdc020       __tryblocktable$??0?$QList@VQString@@@@QAE@ABV0@@Z 10000020     KrakenBuildValidator.obj
 0002:fffdc020       __unwindtable$?detach_helper_grow@?$QList@PAVPortDescriptor@Workflow@U2@@@@AAEPAUNode@1@HH@Z 10000020     KrakenClassifyWorkerFactory.obj
 0002:fffdc020       __unwindtable$?detach_helper_grow@?$QList@VQString@@@@AAEPAUNode@1@HH@Z 10000020     KrakenClassifyWorker.obj
 0002:fffdc020       __ehfuncinfo$?createNode@?$QMapData@VQString@@VQVariant@@@@QAEPAU?$QMapNode@VQString@@VQVariant@@@@ABVQString@@ABVQVariant@@PAU2@_N@Z 10000020     KrakenClassifyWorkerFactory.obj
 0002:fffdc020       __unwindtable$?_Copy@?$basic_string@DU?$char_traits@D@std@@V?$allocator@D@2@@std@@QAEXII@Z 10000020     moc_KrakenBuildTask.obj
 0002:fffdc020       __tryblocktable$??0?$QList@VQString@@@@QAE@ABV0@@Z 10000020     KrakenClassifyValidator.obj
 0002:fffdc020       __unwindtable$?_Copy@?$basic_string@DU?$char_traits@D@std@@V?$allocator@D@2@@std@@QAEXII@Z 10000020     KrakenBuildValidator.obj
 0002:fffdc020       __ehfuncinfo$?append@?$QList@VQString@@@@QAEXABVQString@@@Z 10000020     KrakenClassifyValidator.obj
 0002:fffdc020       __unwindtable$?detach_helper_grow@?$QList@VQString@@@@AAEPAUNode@1@HH@Z 10000020     KrakenTranslateLogParser.obj
 0002:fffdc020       __unwindtable$?_Copy@?$basic_string@DU?$char_traits@D@std@@V?$allocator@D@2@@std@@QAEXII@Z 10000020     KrakenBuildTask.obj
 0002:fffdc020       __unwindtable$?detach_helper_grow@?$QList@VQString@@@@AAEPAUNode@1@HH@Z 10000020     KrakenSupport.obj
 0002:fffdc020       __unwindtable$?detach_helper_grow@?$QList@VQString@@@@AAEPAUNode@1@HH@Z 10000020     KrakenClassifyLogParser.obj
 0002:fffdc020       __ehfuncinfo$?append@?$QList@VQString@@@@QAEXABVQString@@@Z 10000020     KrakenClassifyLogParser.obj
 0002:fffdc020       __tryblocktable$??0?$QList@VQString@@@@QAE@ABV0@@Z 10000020     KrakenClassifyLogParser.obj
 0002:fffdc020       __unwindtable$?detach_helper_grow@?$QList@VWorkflowNotification@U2@@@@AAEPAUNode@1@HH@Z 10000020     KrakenClassifyValidator.obj
 0002:fffdc020       __unwindtable$?_Copy@?$basic_string@DU?$char_traits@D@std@@V?$allocator@D@2@@std@@QAEXII@Z 10000020     KrakenBuildWorker.obj
 0002:fffdc020       __tryblocktable$??0?$QList@VDescriptor@U2@@@@QAE@ABV0@@Z 10000020     KrakenClassifyWorker.obj
 0002:fffdc020       __ehfuncinfo$?append@?$QList@VDescriptor@U2@@@@QAEXABVDescriptor@U2@@@Z 10000020     KrakenClassifyWorker.obj
 0002:fffdc020       __unwindtable$?_Copy@?$basic_string@DU?$char_traits@D@std@@V?$allocator@D@2@@std@@QAEXII@Z 10000020     KrakenClassifyLogParser.obj
 0002:fffdc020       __unwindtable$?detach_helper_grow@?$QList@VDescriptor@U2@@@@AAEPAUNode@1@HH@Z 10000020     KrakenClassifyWorker.obj
 0002:fffdc020       __ehfuncinfo$?append@?$QList@VWorkflowNotification@U2@@@@QAEXABVWorkflowNotification@U2@@@Z 10000020     KrakenClassifyValidator.obj
 0002:fffdc020       __tryblocktable$?detach_helper@?$QList@VDescriptor@U2@@@@AAEXH@Z 10000020     KrakenClassifyWorker.obj
 0002:fffdc020       __unwindtable$?_Copy@?$basic_string@DU?$char_traits@D@std@@V?$allocator@D@2@@std@@QAEXII@Z 10000020     moc_KrakenClassifyPrompter.obj
 0002:fffdc020       __tryblocktable$??0?$QList@VQString@@@@QAE@ABV0@@Z 10000020     KrakenBuildWorker.obj
 0002:fffdc020       __unwindtable$?_Copy@?$basic_string@DU?$char_traits@D@std@@V?$allocator@D@2@@std@@QAEXII@Z 10000020     KrakenClassifyValidator.obj
 0002:fffdc020       __unwindtable$?_Copy@?$basic_string@DU?$char_traits@D@std@@V?$allocator@D@2@@std@@QAEXII@Z 10000020     moc_KrakenBuildPrompter.obj
 0002:fffdc020       __ehfuncinfo$?append@?$QList@VQString@@@@QAEXABVQString@@@Z 10000020     KrakenTranslateLogParser.obj
 0002:fffdc020       __ehfuncinfo$?append@?$QList@VQString@@@@QAEXABVQString@@@Z 10000020     KrakenSupport.obj
 0002:fffdc020       __ehfuncinfo$?append@?$QList@VQString@@@@QAEXABVQString@@@Z 10000020     KrakenBuildWorker.obj
 0002:fffdc020       __tryblocktable$??0?$QList@VQString@@@@QAE@ABV0@@Z 10000020     KrakenSupport.obj
 0002:fffdc020       __unwindtable$?_Copy@?$basic_string@DU?$char_traits@D@std@@V?$allocator@D@2@@std@@QAEXII@Z 10000020     moc_KrakenSupport.obj
 0002:fffdc020       __tryblocktable$??0?$QList@PAVPort@Workflow@U2@@@@QAE@ABV0@@Z 10000020     KrakenClassifyPrompter.obj
 0002:fffdc020       __unwindtable$?_Copy@?$basic_string@DU?$char_traits@D@std@@V?$allocator@D@2@@std@@QAEXII@Z 10000020     KrakenBuildPrompter.obj
 0002:fffdc020       __unwindtable$?detach_helper_grow@?$QList@VQString@@@@AAEPAUNode@1@HH@Z 10000020     KrakenBuildWorker.obj
 0002:fffdc020       __unwindtable$?_Copy@?$basic_string@DU?$char_traits@D@std@@V?$allocator@D@2@@std@@QAEXII@Z 10000020     KrakenSupportPlugin.obj
 0002:fffdc020       __unwindtable$?_Copy@?$basic_string@DU?$char_traits@D@std@@V?$allocator@D@2@@std@@QAEXII@Z 10000020     KrakenClassifyPrompter.obj
 0002:fffdc020       __ehfuncinfo$?createNode@?$QMapData@VQString@@VQVariant@@@@QAEPAU?$QMapNode@VQString@@VQVariant@@@@ABVQString@@ABVQVariant@@PAU2@_N@Z 10000020     KrakenClassifyWorker.obj
 0002:fffdc020       __unwindtable$?_Copy@?$basic_string@DU?$char_traits@D@std@@V?$allocator@D@2@@std@@QAEXII@Z 10000020     moc_KrakenSupportPlugin.obj
 0002:fffdc020       __unwindtable$?detach_helper_grow@?$QList@VQString@@@@AAEPAUNode@1@HH@Z 10000020     KrakenClassifyTask.obj
 0002:fffdc020       __unwindtable$?_Copy@?$basic_string@DU?$char_traits@D@std@@V?$allocator@D@2@@std@@QAEXII@Z 10000020     KrakenSupport.obj
 0002:fffdc020       __unwindtable$?_Copy@?$basic_string@DU?$char_traits@D@std@@V?$allocator@D@2@@std@@QAEXII@Z 10000020     moc_KrakenClassifyTask.obj
 0002:fffdc020       __ehfuncinfo$?createNode@?$QMapData@VQString@@VQScriptValue@@@@QAEPAU?$QMapNode@VQString@@VQScriptValue@@@@ABVQString@@ABVQScriptValue@@PAU2@_N@Z 10000020     KrakenClassifyWorker.obj
 0002:fffdc020       __unwindtable$?_Copy@?$basic_string@DU?$char_traits@D@std@@V?$allocator@D@2@@std@@QAEXII@Z 10000020     KrakenTranslateLogParser.obj
 0002:fffdc020       __tryblocktable$??0?$QList@VQString@@@@QAE@ABV0@@Z 10000020     KrakenTranslateLogParser.obj
 0002:fffdc020       __unwindtable$?detach_helper_grow@?$QList@VQString@@@@AAEPAUNode@1@HH@Z 10000020     KrakenClassifyValidator.obj
 0001:fffff021       __ehhandler$??0KrakenBuildTaskSettings@U2@@QAE@ABU01@@Z 10000021 f   KrakenBuildWorker.obj
 0001:fffff021       __unwindfunclet$??$getAttributeValue@H@Attribute@U2@@QBEHPAVWorkflowContext@Workflow@1@@Z$4 10000021 f   KrakenClassifyWorker.obj
 0001:fffff021       __ehhandler$??1KrakenClassifyTaskSettings@U2@@QAE@XZ 10000021 f   KrakenClassifyWorker.obj
 0001:fffff021       __ehhandler$??1KrakenBuildTaskSettings@U2@@QAE@XZ 10000021 f   KrakenBuildWorker.obj
 0001:fffff021       __ehhandler$??0KrakenClassifyTaskSettings@U2@@QAE@ABU01@@Z 10000021 f   KrakenClassifyWorker.obj
 0001:fffff022       __ehhandler$?append@?$QList@VQString@@@@QAEXABVQString@@@Z 10000022 f   KrakenSupport.obj
 0001:fffff022       __ehhandler$?append@?$QList@VQString@@@@QAEXABVQString@@@Z 10000022 f   KrakenClassifyWorker.obj
 0001:fffff022       __ehhandler$?append@?$QList@VQString@@@@QAEXABVQString@@@Z 10000022 f   KrakenTranslateLogParser.obj
 0001:fffff022       __ehhandler$?append@?$QList@VQString@@@@QAEXABVQString@@@Z 10000022 f   KrakenClassifyTask.obj
 0001:fffff022       __ehhandler$?append@?$QList@VQString@@@@QAEXABVQString@@@Z 10000022 f   KrakenBuildWorker.obj
 0001:fffff022       __ehhandler$?append@?$QList@VQString@@@@QAEXABVQString@@@Z 10000022 f   KrakenBuildValidator.obj
 0001:fffff022       __ehhandler$?append@?$QList@VQString@@@@QAEXABVQString@@@Z 10000022 f   KrakenClassifyValidator.obj
 0001:fffff022       __ehhandler$?append@?$QList@VQString@@@@QAEXABVQString@@@Z 10000022 f   KrakenClassifyLogParser.obj
 0001:fffff023       __unwindfunclet$??$getAttributeValue@VQString@@@Attribute@U2@@QBE?AVQString@@PAVWorkflowContext@Workflow@1@@Z$2 10000023 f   KrakenClassifyWorker.obj
 0001:fffff023       __ehhandler$??$getValue@VQString@@@BaseWorker@LocalWorkflow@U2@@IBE?AVQString@@ABV3@@Z 10000023 f   KrakenClassifyWorker.obj
 0001:fffff023       __ehhandler$?metaType@?$QVariantValueHelper@VQString@@@QtPrivate@@SA?AVQString@@ABVQVariant@@@Z 10000023 f   KrakenClassifyValidator.obj
 0001:fffff023       __ehhandler$??H@YA?BVQString@@ABV0@PBD@Z 10000023 f   KrakenClassifyWorker.obj
 0001:fffff023       __ehhandler$??H@YA?BVQString@@ABV0@PBD@Z 10000023 f   KrakenClassifyValidator.obj
 0001:fffff023       __ehhandler$??H@YA?BVQString@@ABV0@PBD@Z 10000023 f   KrakenBuildTask.obj
 0001:fffff023       __ehhandler$??H@YA?BVQString@@ABV0@PBD@Z 10000023 f   KrakenClassifyWorkerFactory.obj
 0001:fffff023       __ehhandler$??H@YA?BVQString@@ABV0@PBD@Z 10000023 f   KrakenSupport.obj
 0001:fffff023       __ehhandler$??H@YA?BVQString@@ABV0@PBD@Z 10000023 f   KrakenBuildWorkerFactory.obj
 0001:fffff023       __ehhandler$?metaType@?$QVariantValueHelper@VQString@@@QtPrivate@@SA?AVQString@@ABVQVariant@@@Z 10000023 f   KrakenClassifyWorker.obj
 0002:fffdc024       __ehfuncinfo$?append@?$QList@PAVPortDescriptor@Workflow@U2@@@@QAEXABQAVPortDescriptor@Workflow@U2@@@Z 10000024     KrakenClassifyWorkerFactory.obj
 0002:fffdc024       __ehfuncinfo$?createNode@?$QMapData@VQString@@I@@QAEPAU?$QMapNode@VQString@@I@@ABVQString@@ABIPAU2@_N@Z 10000024     KrakenClassifyWorker.obj
 0002:fffdc024       __ehfuncinfo$?node_copy@?$QList@VWorkflowNotification@U2@@@@AAEXPAUNode@1@00@Z 10000024     KrakenClassifyValidator.obj
 0002:fffdc024       __ehfuncinfo$?node_copy@?$QList@VQString@@@@AAEXPAUNode@1@00@Z 10000024     KrakenBuildWorker.obj
 0002:fffdc024       __unwindtable$??$getAttributeValue@H@Attribute@U2@@QBEHPAVWorkflowContext@Workflow@1@@Z 10000024     KrakenClassifyWorker.obj
 0002:fffdc024       __ehfuncinfo$?node_copy@?$QList@VDescriptor@U2@@@@AAEXPAUNode@1@00@Z 10000024     KrakenClassifyWorker.obj
 0002:fffdc024       __ehfuncinfo$?node_copy@?$QList@VQString@@@@AAEXPAUNode@1@00@Z 10000024     KrakenClassifyTask.obj
 0002:fffdc024       __ehfuncinfo$?node_copy@?$QList@VQString@@@@AAEXPAUNode@1@00@Z 10000024     KrakenClassifyWorker.obj
 0002:fffdc024       __ehfuncinfo$?node_copy@?$QList@VQString@@@@AAEXPAUNode@1@00@Z 10000024     KrakenTranslateLogParser.obj
 0002:fffdc024       __ehfuncinfo$?node_copy@?$QList@VQString@@@@AAEXPAUNode@1@00@Z 10000024     KrakenBuildValidator.obj
 0002:fffdc024       __ehfuncinfo$?node_copy@?$QList@VQString@@@@AAEXPAUNode@1@00@Z 10000024     KrakenClassifyLogParser.obj
 0002:fffdc024       __ehfuncinfo$?createNode@?$QMapData@VDescriptor@U2@@V?$QExplicitlySharedDataPointer@VDataType@U2@@@@@@QAEPAU?$QMapNode@VDescriptor@U2@@V?$QExplicitlySharedDataPointer@VDataType@U2@@@@@@ABVDescriptor@U2@@ABV?$QExplicitlySharedDataPointer@VDataType@U2@@@@PAU2@_N@Z 10000024     KrakenClassifyWorkerFactory.obj
 0002:fffdc024       __ehfuncinfo$?node_copy@?$QList@VQString@@@@AAEXPAUNode@1@00@Z 10000024     KrakenClassifyValidator.obj
 0002:fffdc024       __ehfuncinfo$?createNode@?$QMapData@VQString@@PAVPropertyDelegate@U2@@@@QAEPAU?$QMapNode@VQString@@PAVPropertyDelegate@U2@@@@ABVQString@@ABQAVPropertyDelegate@U2@@PAU2@_N@Z 10000024     KrakenClassifyWorkerFactory.obj
 0002:fffdc024       __ehfuncinfo$?append@?$QList@PAVAttribute@U2@@@@QAEXABQAVAttribute@U2@@@Z 10000024     KrakenClassifyWorkerFactory.obj
 0002:fffdc024       __unwindtable$??$getAttributeValue@VQString@@@Attribute@U2@@QBE?AVQString@@PAVWorkflowContext@Workflow@1@@Z 10000024     KrakenClassifyWorker.obj
 0002:fffdc024       __ehfuncinfo$?node_copy@?$QList@VQString@@@@AAEXPAUNode@1@00@Z 10000024     KrakenSupport.obj
 0001:fffff028       __ehhandler$?createNode@?$QMapData@VQString@@VQVariant@@@@QAEPAU?$QMapNode@VQString@@VQVariant@@@@ABVQString@@ABVQVariant@@PAU2@_N@Z 10000028 f   KrakenClassifyWorker.obj
 0001:fffff028       __ehhandler$?createNode@?$QMapData@VQString@@VQScriptValue@@@@QAEPAU?$QMapNode@VQString@@VQScriptValue@@@@ABVQString@@ABVQScriptValue@@PAU2@_N@Z 10000028 f   KrakenClassifyWorker.obj
 0001:fffff028       __ehhandler$?createNode@?$QMapData@VQString@@VQVariant@@@@QAEPAU?$QMapNode@VQString@@VQVariant@@@@ABVQString@@ABVQVariant@@PAU2@_N@Z 10000028 f   KrakenBuildWorkerFactory.obj
 0001:fffff028       __ehhandler$?createNode@?$QMapData@VQString@@VQVariant@@@@QAEPAU?$QMapNode@VQString@@VQVariant@@@@ABVQString@@ABVQVariant@@PAU2@_N@Z 10000028 f   KrakenClassifyWorkerFactory.obj
 0001:fffff02a       __unwindfunclet$??$getAttributeValue@H@Attribute@U2@@QBEHPAVWorkflowContext@Workflow@1@@Z$5 1000002a f   KrakenClassifyWorker.obj
 0001:fffff02b       __unwindfunclet$??$getAttributeValue@VQString@@@Attribute@U2@@QBE?AVQString@@PAVWorkflowContext@Workflow@1@@Z$3 1000002b f   KrakenClassifyWorker.obj
 0001:fffff033       __unwindfunclet$??$getAttributeValue@VQString@@@Attribute@U2@@QBE?AVQString@@PAVWorkflowContext@Workflow@1@@Z$4 10000033 f   KrakenClassifyWorker.obj
 0001:fffff033       __unwindfunclet$??$getAttributeValue@H@Attribute@U2@@QBEHPAVWorkflowContext@Workflow@1@@Z$6 10000033 f   KrakenClassifyWorker.obj
 0002:fffdc034       __ehfuncinfo$??0?$QList@VQString@@@@QAE@ABV0@@Z 10000034     KrakenTranslateLogParser.obj
 0002:fffdc034       __ehfuncinfo$?detach_helper@?$QList@VDescriptor@U2@@@@AAEXH@Z 10000034     KrakenClassifyWorker.obj
 0002:fffdc034       __ehfuncinfo$??0?$QList@VQString@@@@QAE@ABV0@@Z 10000034     KrakenClassifyLogParser.obj
 0002:fffdc034       __ehfuncinfo$??0?$QList@VQString@@@@QAE@ABV0@@Z 10000034     KrakenBuildWorker.obj
 0002:fffdc034       __ehfuncinfo$??0?$QList@VQString@@@@QAE@ABV0@@Z 10000034     KrakenSupport.obj
 0002:fffdc034       __ehfuncinfo$??0?$QList@VDescriptor@U2@@@@QAE@ABV0@@Z 10000034     KrakenClassifyWorker.obj
 0002:fffdc034       __ehfuncinfo$??0?$QList@VQString@@@@QAE@ABV0@@Z 10000034     KrakenClassifyValidator.obj
 0002:fffdc034       __ehfuncinfo$??0?$QList@VQString@@@@QAE@ABV0@@Z 10000034     KrakenClassifyTask.obj
 0002:fffdc034       __ehfuncinfo$??0?$QList@VQString@@@@QAE@ABV0@@Z 10000034     KrakenBuildValidator.obj
 0002:fffdc034       __ehfuncinfo$??0?$QList@PAVPort@Workflow@U2@@@@QAE@ABV0@@Z 10000034     KrakenClassifyPrompter.obj
 0001:fffff03b       __unwindfunclet$??$getAttributeValue@VQString@@@Attribute@U2@@QBE?AVQString@@PAVWorkflowContext@Workflow@1@@Z$5 1000003b f   KrakenClassifyWorker.obj
 0001:fffff03c       __unwindfunclet$??$getAttributeValue@H@Attribute@U2@@QBEHPAVWorkflowContext@Workflow@1@@Z$7 1000003c f   KrakenClassifyWorker.obj
 0002:fffdc040       __ehfuncinfo$?detach_helper_grow@?$QList@PAVAttribute@U2@@@@AAEPAUNode@1@HH@Z 10000040     KrakenClassifyWorkerFactory.obj
 0002:fffdc040       __ehfuncinfo$?_Copy@?$basic_string@DU?$char_traits@D@std@@V?$allocator@D@2@@std@@QAEXII@Z 10000040     moc_KrakenSupportPlugin.obj
 0002:fffdc040       __ehfuncinfo$?_Copy@?$basic_string@DU?$char_traits@D@std@@V?$allocator@D@2@@std@@QAEXII@Z 10000040     moc_KrakenSupport.obj
 0002:fffdc040       __ehfuncinfo$?_Copy@?$basic_string@DU?$char_traits@D@std@@V?$allocator@D@2@@std@@QAEXII@Z 10000040     KrakenBuildPrompter.obj
 0002:fffdc040       __ehfuncinfo$?_Copy@?$basic_string@DU?$char_traits@D@std@@V?$allocator@D@2@@std@@QAEXII@Z 10000040     KrakenClassifyWorker.obj
 0002:fffdc040       __ehfuncinfo$?_Copy@?$basic_string@DU?$char_traits@D@std@@V?$allocator@D@2@@std@@QAEXII@Z 10000040     moc_KrakenBuildWorker.obj
 0002:fffdc040       __ehfuncinfo$?_Copy@?$basic_string@DU?$char_traits@D@std@@V?$allocator@D@2@@std@@QAEXII@Z 10000040     moc_KrakenClassifyWorker.obj
 0002:fffdc040       __ehfuncinfo$?_Copy@?$basic_string@DU?$char_traits@D@std@@V?$allocator@D@2@@std@@QAEXII@Z 10000040     KrakenBuildWorker.obj
 0002:fffdc040       __ehfuncinfo$?_Copy@?$basic_string@DU?$char_traits@D@std@@V?$allocator@D@2@@std@@QAEXII@Z 10000040     KrakenBuildWorkerFactory.obj
 0002:fffdc040       __ehfuncinfo$?_Copy@?$basic_string@DU?$char_traits@D@std@@V?$allocator@D@2@@std@@QAEXII@Z 10000040     KrakenClassifyTask.obj
 0002:fffdc040       __ehfuncinfo$?_Copy@?$basic_string@DU?$char_traits@D@std@@V?$allocator@D@2@@std@@QAEXII@Z 10000040     KrakenClassifyPrompter.obj
 0002:fffdc040       __ehfuncinfo$?_Copy@?$basic_string@DU?$char_traits@D@std@@V?$allocator@D@2@@std@@QAEXII@Z 10000040     KrakenClassifyValidator.obj
 0002:fffdc040       __ehfuncinfo$?_Copy@?$basic_string@DU?$char_traits@D@std@@V?$allocator@D@2@@std@@QAEXII@Z 10000040     KrakenSupport.obj
 0002:fffdc040       __ehfuncinfo$?_Copy@?$basic_string@DU?$char_traits@D@std@@V?$allocator@D@2@@std@@QAEXII@Z 10000040     moc_KrakenClassifyPrompter.obj
 0002:fffdc040       __ehfuncinfo$?_Copy@?$basic_string@DU?$char_traits@D@std@@V?$allocator@D@2@@std@@QAEXII@Z 10000040     KrakenBuildTask.obj
 0002:fffdc040       __ehfuncinfo$?_Copy@?$basic_string@DU?$char_traits@D@std@@V?$allocator@D@2@@std@@QAEXII@Z 10000040     moc_KrakenBuildPrompter.obj
 0002:fffdc040       __ehfuncinfo$?detach_helper_grow@?$QList@VQString@@@@AAEPAUNode@1@HH@Z 10000040     KrakenBuildValidator.obj
 0002:fffdc040       __ehfuncinfo$?detach_helper_grow@?$QList@VQString@@@@AAEPAUNode@1@HH@Z 10000040     KrakenSupport.obj
 0002:fffdc040       __ehfuncinfo$?detach_helper_grow@?$QList@VQString@@@@AAEPAUNode@1@HH@Z 10000040     KrakenBuildWorker.obj
 0002:fffdc040       __ehfuncinfo$?_Copy@?$basic_string@DU?$char_traits@D@std@@V?$allocator@D@2@@std@@QAEXII@Z 10000040     KrakenClassifyWorkerFactory.obj
 0002:fffdc040       __ehfuncinfo$?_Copy@?$basic_string@DU?$char_traits@D@std@@V?$allocator@D@2@@std@@QAEXII@Z 10000040     moc_KrakenBuildTask.obj
 0002:fffdc040       __ehfuncinfo$?_Copy@?$basic_string@DU?$char_traits@D@std@@V?$allocator@D@2@@std@@QAEXII@Z 10000040     moc_KrakenClassifyTask.obj
 0002:fffdc040       __ehfuncinfo$?_Copy@?$basic_string@DU?$char_traits@D@std@@V?$allocator@D@2@@std@@QAEXII@Z 10000040     KrakenSupportPlugin.obj
 0002:fffdc040       __ehfuncinfo$?detach_helper_grow@?$QList@VQString@@@@AAEPAUNode@1@HH@Z 10000040     KrakenClassifyTask.obj
 0002:fffdc040       __ehfuncinfo$?detach_helper_grow@?$QList@VWorkflowNotification@U2@@@@AAEPAUNode@1@HH@Z 10000040     KrakenClassifyValidator.obj
 0002:fffdc040       __ehfuncinfo$?detach_helper_grow@?$QList@VDescriptor@U2@@@@AAEPAUNode@1@HH@Z 10000040     KrakenClassifyWorker.obj
 0002:fffdc040       __ehfuncinfo$?_Copy@?$basic_string@DU?$char_traits@D@std@@V?$allocator@D@2@@std@@QAEXII@Z 10000040     KrakenClassifyLogParser.obj
 0002:fffdc040       __ehfuncinfo$?detach_helper_grow@?$QList@VQString@@@@AAEPAUNode@1@HH@Z 10000040     KrakenClassifyWorker.obj
 0002:fffdc040       __ehfuncinfo$?detach_helper_grow@?$QList@VQString@@@@AAEPAUNode@1@HH@Z 10000040     KrakenClassifyValidator.obj
 0002:fffdc040       __ehfuncinfo$?detach_helper_grow@?$QList@VQString@@@@AAEPAUNode@1@HH@Z 10000040     KrakenClassifyLogParser.obj
 0002:fffdc040       __ehfuncinfo$?_Copy@?$basic_string@DU?$char_traits@D@std@@V?$allocator@D@2@@std@@QAEXII@Z 10000040     KrakenBuildValidator.obj
 0002:fffdc040       __ehfuncinfo$?detach_helper_grow@?$QList@VQString@@@@AAEPAUNode@1@HH@Z 10000040     KrakenTranslateLogParser.obj
 0002:fffdc040       __ehfuncinfo$?_Copy@?$basic_string@DU?$char_traits@D@std@@V?$allocator@D@2@@std@@QAEXII@Z 10000040     KrakenTranslateLogParser.obj
 0002:fffdc040       __ehfuncinfo$?detach_helper_grow@?$QList@PAVPortDescriptor@Workflow@U2@@@@AAEPAUNode@1@HH@Z 10000040     KrakenClassifyWorkerFactory.obj
 0002:fffdc044       __tryblocktable$?createNode@?$QMapData@VQString@@VQVariant@@@@QAEPAU?$QMapNode@VQString@@VQVariant@@@@ABVQString@@ABVQVariant@@PAU2@_N@Z 10000044     KrakenClassifyWorkerFactory.obj
 0001:fffff044       __unwindfunclet$??$getAttributeValue@VQString@@@Attribute@U2@@QBE?AVQString@@PAVWorkflowContext@Workflow@1@@Z$6 10000044 f   KrakenClassifyWorker.obj
 0002:fffdc044       __tryblocktable$?append@?$QList@VQString@@@@QAEXABVQString@@@Z 10000044     KrakenTranslateLogParser.obj
 0002:fffdc044       __tryblocktable$?append@?$QList@VQString@@@@QAEXABVQString@@@Z 10000044     KrakenClassifyLogParser.obj
 0002:fffdc044       __tryblocktable$?append@?$QList@VQString@@@@QAEXABVQString@@@Z 10000044     KrakenClassifyValidator.obj
 0002:fffdc044       __tryblocktable$?createNode@?$QMapData@VQString@@VQVariant@@@@QAEPAU?$QMapNode@VQString@@VQVariant@@@@ABVQString@@ABVQVariant@@PAU2@_N@Z 10000044     KrakenBuildWorkerFactory.obj
 0002:fffdc044       __tryblocktable$?createNode@?$QMapData@VQString@@VQVariant@@@@QAEPAU?$QMapNode@VQString@@VQVariant@@@@ABVQString@@ABVQVariant@@PAU2@_N@Z 10000044     KrakenClassifyWorker.obj
 0002:fffdc044       __tryblocktable$?append@?$QList@VQString@@@@QAEXABVQString@@@Z 10000044     KrakenSupport.obj
 0002:fffdc044       __tryblocktable$?append@?$QList@VDescriptor@U2@@@@QAEXABVDescriptor@U2@@@Z 10000044     KrakenClassifyWorker.obj
 0002:fffdc044       __tryblocktable$?append@?$QList@VQString@@@@QAEXABVQString@@@Z 10000044     KrakenBuildValidator.obj
 0002:fffdc044       __tryblocktable$?append@?$QList@VWorkflowNotification@U2@@@@QAEXABVWorkflowNotification@U2@@@Z 10000044     KrakenClassifyValidator.obj
 0002:fffdc044       __tryblocktable$?append@?$QList@VQString@@@@QAEXABVQString@@@Z 10000044     KrakenBuildWorker.obj
 0002:fffdc044       __tryblocktable$?append@?$QList@VQString@@@@QAEXABVQString@@@Z 10000044     KrakenClassifyWorker.obj
 0002:fffdc044       __tryblocktable$?createNode@?$QMapData@VQString@@VQScriptValue@@@@QAEPAU?$QMapNode@VQString@@VQScriptValue@@@@ABVQString@@ABVQScriptValue@@PAU2@_N@Z 10000044     KrakenClassifyWorker.obj
 0002:fffdc044       __tryblocktable$?append@?$QList@VQString@@@@QAEXABVQString@@@Z 10000044     KrakenClassifyTask.obj
 0001:fffff045       __unwindfunclet$??$getAttributeValue@H@Attribute@U2@@QBEHPAVWorkflowContext@Workflow@1@@Z$8 10000045 f   KrakenClassifyWorker.obj
 0002:fffdc048       __unwindtable$?node_copy@?$QList@VWorkflowNotification@U2@@@@AAEXPAUNode@1@00@Z 10000048     KrakenClassifyValidator.obj
 0002:fffdc048       __unwindtable$?createNode@?$QMapData@VQString@@I@@QAEPAU?$QMapNode@VQString@@I@@ABVQString@@ABIPAU2@_N@Z 10000048     KrakenClassifyWorker.obj
 0002:fffdc048       __unwindtable$?node_copy@?$QList@VQString@@@@AAEXPAUNode@1@00@Z 10000048     KrakenBuildWorker.obj
 0002:fffdc048       __unwindtable$?node_copy@?$QList@VQString@@@@AAEXPAUNode@1@00@Z 10000048     KrakenSupport.obj
 0002:fffdc048       __unwindtable$?node_copy@?$QList@VQString@@@@AAEXPAUNode@1@00@Z 10000048     KrakenClassifyWorker.obj
 0002:fffdc048       __unwindtable$?node_copy@?$QList@VDescriptor@U2@@@@AAEXPAUNode@1@00@Z 10000048     KrakenClassifyWorker.obj
 0002:fffdc048       __unwindtable$?node_copy@?$QList@VQString@@@@AAEXPAUNode@1@00@Z 10000048     KrakenClassifyTask.obj
 0002:fffdc048       __unwindtable$?node_copy@?$QList@VQString@@@@AAEXPAUNode@1@00@Z 10000048     KrakenClassifyLogParser.obj
 0002:fffdc048       __unwindtable$?node_copy@?$QList@VQString@@@@AAEXPAUNode@1@00@Z 10000048     KrakenBuildValidator.obj
 0002:fffdc048       __unwindtable$?node_copy@?$QList@VQString@@@@AAEXPAUNode@1@00@Z 10000048     KrakenClassifyValidator.obj
 0002:fffdc048       __unwindtable$?append@?$QList@PAVAttribute@U2@@@@QAEXABQAVAttribute@U2@@@Z 10000048     KrakenClassifyWorkerFactory.obj
 0002:fffdc048       __unwindtable$?node_copy@?$QList@VQString@@@@AAEXPAUNode@1@00@Z 10000048     KrakenTranslateLogParser.obj
 0002:fffdc048       __unwindtable$?append@?$QList@PAVPortDescriptor@Workflow@U2@@@@QAEXABQAVPortDescriptor@Workflow@U2@@@Z 10000048     KrakenClassifyWorkerFactory.obj
 0002:fffdc048       __unwindtable$?createNode@?$QMapData@VDescriptor@U2@@V?$QExplicitlySharedDataPointer@VDataType@U2@@@@@@QAEPAU?$QMapNode@VDescriptor@U2@@V?$QExplicitlySharedDataPointer@VDataType@U2@@@@@@ABVDescriptor@U2@@ABV?$QExplicitlySharedDataPointer@VDataType@U2@@@@PAU2@_N@Z 10000048     KrakenClassifyWorkerFactory.obj
 0002:fffdc048       __unwindtable$?createNode@?$QMapData@VQString@@PAVPropertyDelegate@U2@@@@QAEPAU?$QMapNode@VQString@@PAVPropertyDelegate@U2@@@@ABVQString@@ABQAVPropertyDelegate@U2@@PAU2@_N@Z 10000048     KrakenClassifyWorkerFactory.obj
 0001:fffff04d       __unwindfunclet$??$getAttributeValue@VQString@@@Attribute@U2@@QBE?AVQString@@PAVWorkflowContext@Workflow@1@@Z$7 1000004d f   KrakenClassifyWorker.obj
 0001:fffff04e       __unwindfunclet$??$getAttributeValue@H@Attribute@U2@@QBEHPAVWorkflowContext@Workflow@1@@Z$9 1000004e f   KrakenClassifyWorker.obj
 0001:fffff056       __unwindfunclet$??$getAttributeValue@VQString@@@Attribute@U2@@QBE?AVQString@@PAVWorkflowContext@Workflow@1@@Z$8 10000056 f   KrakenClassifyWorker.obj
 0001:fffff057       __unwindfunclet$??$getAttributeValue@H@Attribute@U2@@QBEHPAVWorkflowContext@Workflow@1@@Z$10 10000057 f   KrakenClassifyWorker.obj
 0001:fffff05f       __unwindfunclet$??$getAttributeValue@VQString@@@Attribute@U2@@QBE?AVQString@@PAVWorkflowContext@Workflow@1@@Z$9 1000005f f   KrakenClassifyWorker.obj
 0001:fffff060       __unwindfunclet$??$getAttributeValue@H@Attribute@U2@@QBEHPAVWorkflowContext@Workflow@1@@Z$11 10000060 f   KrakenClassifyWorker.obj
 0001:fffff062       __catch$?node_copy@?$QList@VQString@@@@AAEXPAUNode@1@00@Z$2 10000062 f   KrakenBuildValidator.obj
 0001:fffff062       __catch$?node_copy@?$QList@VQString@@@@AAEXPAUNode@1@00@Z$2 10000062 f   KrakenClassifyLogParser.obj
 0001:fffff062       __catch$?node_copy@?$QList@VQString@@@@AAEXPAUNode@1@00@Z$2 10000062 f   KrakenTranslateLogParser.obj
 0001:fffff062       __catch$?node_copy@?$QList@VQString@@@@AAEXPAUNode@1@00@Z$2 10000062 f   KrakenSupport.obj
 0001:fffff062       __catch$?node_copy@?$QList@VQString@@@@AAEXPAUNode@1@00@Z$2 10000062 f   KrakenBuildWorker.obj
 0001:fffff062       __catch$?node_copy@?$QList@VQString@@@@AAEXPAUNode@1@00@Z$2 10000062 f   KrakenClassifyWorker.obj
 0001:fffff062       __catch$?node_copy@?$QList@VQString@@@@AAEXPAUNode@1@00@Z$2 10000062 f   KrakenClassifyTask.obj
 0001:fffff062       __catch$?node_copy@?$QList@VQString@@@@AAEXPAUNode@1@00@Z$2 10000062 f   KrakenClassifyValidator.obj
 0002:fffdc064       __tryblocktable$?_Copy@?$basic_string@DU?$char_traits@D@std@@V?$allocator@D@2@@std@@QAEXII@Z 10000064     KrakenClassifyPrompter.obj
 0002:fffdc064       __tryblocktable$?_Copy@?$basic_string@DU?$char_traits@D@std@@V?$allocator@D@2@@std@@QAEXII@Z 10000064     moc_KrakenClassifyWorker.obj
 0002:fffdc064       __tryblocktable$?_Copy@?$basic_string@DU?$char_traits@D@std@@V?$allocator@D@2@@std@@QAEXII@Z 10000064     KrakenBuildPrompter.obj
 0002:fffdc064       __tryblocktable$?_Copy@?$basic_string@DU?$char_traits@D@std@@V?$allocator@D@2@@std@@QAEXII@Z 10000064     moc_KrakenBuildWorker.obj
 0002:fffdc064       __tryblocktable$?_Copy@?$basic_string@DU?$char_traits@D@std@@V?$allocator@D@2@@std@@QAEXII@Z 10000064     KrakenBuildWorker.obj
 0002:fffdc064       __tryblocktable$?_Copy@?$basic_string@DU?$char_traits@D@std@@V?$allocator@D@2@@std@@QAEXII@Z 10000064     KrakenBuildWorkerFactory.obj
 0002:fffdc064       __tryblocktable$?_Copy@?$basic_string@DU?$char_traits@D@std@@V?$allocator@D@2@@std@@QAEXII@Z 10000064     KrakenBuildTask.obj
 0002:fffdc064       __tryblocktable$?detach_helper_grow@?$QList@PAVAttribute@U2@@@@AAEPAUNode@1@HH@Z 10000064     KrakenClassifyWorkerFactory.obj
 0002:fffdc064       __tryblocktable$?_Copy@?$basic_string@DU?$char_traits@D@std@@V?$allocator@D@2@@std@@QAEXII@Z 10000064     moc_KrakenClassifyPrompter.obj
 0002:fffdc064       __tryblocktable$?_Copy@?$basic_string@DU?$char_traits@D@std@@V?$allocator@D@2@@std@@QAEXII@Z 10000064     KrakenSupport.obj
 0002:fffdc064       __tryblocktable$?_Copy@?$basic_string@DU?$char_traits@D@std@@V?$allocator@D@2@@std@@QAEXII@Z 10000064     moc_KrakenBuildPrompter.obj
 0002:fffdc064       __tryblocktable$?detach_helper_grow@?$QList@VQString@@@@AAEPAUNode@1@HH@Z 10000064     KrakenBuildValidator.obj
 0002:fffdc064       __tryblocktable$?detach_helper_grow@?$QList@VQString@@@@AAEPAUNode@1@HH@Z 10000064     KrakenSupport.obj
 0002:fffdc064       __tryblocktable$?_Copy@?$basic_string@DU?$char_traits@D@std@@V?$allocator@D@2@@std@@QAEXII@Z 10000064     KrakenClassifyTask.obj
 0002:fffdc064       __tryblocktable$?detach_helper_grow@?$QList@VQString@@@@AAEPAUNode@1@HH@Z 10000064     KrakenClassifyValidator.obj
 0002:fffdc064       __tryblocktable$?detach_helper_grow@?$QList@VQString@@@@AAEPAUNode@1@HH@Z 10000064     KrakenBuildWorker.obj
 0002:fffdc064       __tryblocktable$?_Copy@?$basic_string@DU?$char_traits@D@std@@V?$allocator@D@2@@std@@QAEXII@Z 10000064     KrakenClassifyWorkerFactory.obj
 0002:fffdc064       __tryblocktable$?_Copy@?$basic_string@DU?$char_traits@D@std@@V?$allocator@D@2@@std@@QAEXII@Z 10000064     KrakenSupportPlugin.obj
 0002:fffdc064       __tryblocktable$?detach_helper_grow@?$QList@VDescriptor@U2@@@@AAEPAUNode@1@HH@Z 10000064     KrakenClassifyWorker.obj
 0002:fffdc064       __tryblocktable$?detach_helper_grow@?$QList@VWorkflowNotification@U2@@@@AAEPAUNode@1@HH@Z 10000064     KrakenClassifyValidator.obj
 0002:fffdc064       __tryblocktable$?_Copy@?$basic_string@DU?$char_traits@D@std@@V?$allocator@D@2@@std@@QAEXII@Z 10000064     moc_KrakenClassifyTask.obj
 0002:fffdc064       __tryblocktable$?_Copy@?$basic_string@DU?$char_traits@D@std@@V?$allocator@D@2@@std@@QAEXII@Z 10000064     moc_KrakenSupport.obj
 0002:fffdc064       __tryblocktable$?_Copy@?$basic_string@DU?$char_traits@D@std@@V?$allocator@D@2@@std@@QAEXII@Z 10000064     moc_KrakenSupportPlugin.obj
 0002:fffdc064       __tryblocktable$?detach_helper_grow@?$QList@VQString@@@@AAEPAUNode@1@HH@Z 10000064     KrakenClassifyTask.obj
 0002:fffdc064       __tryblocktable$?_Copy@?$basic_string@DU?$char_traits@D@std@@V?$allocator@D@2@@std@@QAEXII@Z 10000064     moc_KrakenBuildTask.obj
 0002:fffdc064       __tryblocktable$?_Copy@?$basic_string@DU?$char_traits@D@std@@V?$allocator@D@2@@std@@QAEXII@Z 10000064     KrakenClassifyLogParser.obj
 0002:fffdc064       __tryblocktable$?detach_helper_grow@?$QList@PAVPortDescriptor@Workflow@U2@@@@AAEPAUNode@1@HH@Z 10000064     KrakenClassifyWorkerFactory.obj
 0002:fffdc064       __tryblocktable$?_Copy@?$basic_string@DU?$char_traits@D@std@@V?$allocator@D@2@@std@@QAEXII@Z 10000064     KrakenClassifyValidator.obj
 0002:fffdc064       __tryblocktable$?_Copy@?$basic_string@DU?$char_traits@D@std@@V?$allocator@D@2@@std@@QAEXII@Z 10000064     KrakenClassifyWorker.obj
 0002:fffdc064       __tryblocktable$?detach_helper_grow@?$QList@VQString@@@@AAEPAUNode@1@HH@Z 10000064     KrakenTranslateLogParser.obj
 0002:fffdc064       __tryblocktable$?detach_helper_grow@?$QList@VQString@@@@AAEPAUNode@1@HH@Z 10000064     KrakenClassifyLogParser.obj
 0002:fffdc064       __tryblocktable$?_Copy@?$basic_string@DU?$char_traits@D@std@@V?$allocator@D@2@@std@@QAEXII@Z 10000064     KrakenBuildValidator.obj
 0002:fffdc064       __tryblocktable$?_Copy@?$basic_string@DU?$char_traits@D@std@@V?$allocator@D@2@@std@@QAEXII@Z 10000064     KrakenTranslateLogParser.obj
 0002:fffdc064       __tryblocktable$?detach_helper_grow@?$QList@VQString@@@@AAEPAUNode@1@HH@Z 10000064     KrakenClassifyWorker.obj
 0001:fffff068       __unwindfunclet$??$getAttributeValue@VQString@@@Attribute@U2@@QBE?AVQString@@PAVWorkflowContext@Workflow@1@@Z$10 10000068 f   KrakenClassifyWorker.obj
 0001:fffff069       __ehhandler$??$getAttributeValue@H@Attribute@U2@@QBEHPAVWorkflowContext@Workflow@1@@Z 10000069 f   KrakenClassifyWorker.obj
 0002:fffdc06c       __unwindtable$?append@?$QList@VQString@@@@QAEXABVQString@@@Z 1000006c     KrakenClassifyLogParser.obj
 0002:fffdc06c       __unwindtable$?append@?$QList@VQString@@@@QAEXABVQString@@@Z 1000006c     KrakenClassifyWorker.obj
 0002:fffdc06c       __unwindtable$?createNode@?$QMapData@VQString@@VQVariant@@@@QAEPAU?$QMapNode@VQString@@VQVariant@@@@ABVQString@@ABVQVariant@@PAU2@_N@Z 1000006c     KrakenClassifyWorkerFactory.obj
 0002:fffdc06c       __unwindtable$?append@?$QList@VWorkflowNotification@U2@@@@QAEXABVWorkflowNotification@U2@@@Z 1000006c     KrakenClassifyValidator.obj
 0002:fffdc06c       __unwindtable$?append@?$QList@VQString@@@@QAEXABVQString@@@Z 1000006c     KrakenBuildValidator.obj
 0002:fffdc06c       __unwindtable$?append@?$QList@VQString@@@@QAEXABVQString@@@Z 1000006c     KrakenClassifyTask.obj
 0002:fffdc06c       __unwindtable$?createNode@?$QMapData@VQString@@VQVariant@@@@QAEPAU?$QMapNode@VQString@@VQVariant@@@@ABVQString@@ABVQVariant@@PAU2@_N@Z 1000006c     KrakenBuildWorkerFactory.obj
 0002:fffdc06c       __unwindtable$?append@?$QList@VQString@@@@QAEXABVQString@@@Z 1000006c     KrakenClassifyValidator.obj
 0002:fffdc06c       __unwindtable$?append@?$QList@VQString@@@@QAEXABVQString@@@Z 1000006c     KrakenSupport.obj
 0002:fffdc06c       __unwindtable$?append@?$QList@VDescriptor@U2@@@@QAEXABVDescriptor@U2@@@Z 1000006c     KrakenClassifyWorker.obj
 0002:fffdc06c       __unwindtable$?append@?$QList@VQString@@@@QAEXABVQString@@@Z 1000006c     KrakenBuildWorker.obj
 0002:fffdc06c       __unwindtable$?createNode@?$QMapData@VQString@@VQVariant@@@@QAEPAU?$QMapNode@VQString@@VQVariant@@@@ABVQString@@ABVQVariant@@PAU2@_N@Z 1000006c     KrakenClassifyWorker.obj
 0002:fffdc06c       __unwindtable$?append@?$QList@VQString@@@@QAEXABVQString@@@Z 1000006c     KrakenTranslateLogParser.obj
 0002:fffdc06c       __unwindtable$?createNode@?$QMapData@VQString@@VQScriptValue@@@@QAEPAU?$QMapNode@VQString@@VQScriptValue@@@@ABVQString@@ABVQScriptValue@@PAU2@_N@Z 1000006c     KrakenClassifyWorker.obj
 0001:fffff071       __unwindfunclet$??$getAttributeValue@VQString@@@Attribute@U2@@QBE?AVQString@@PAVWorkflowContext@Workflow@1@@Z$11 10000071 f   KrakenClassifyWorker.obj
 0001:fffff07a       __unwindfunclet$??$getAttributeValue@VQString@@@Attribute@U2@@QBE?AVQString@@PAVWorkflowContext@Workflow@1@@Z$12 1000007a f   KrakenClassifyWorker.obj
 0001:fffff07d       __catch$?append@?$QList@VQString@@@@QAEXABVQString@@@Z$0 1000007d f   KrakenClassifyWorker.obj
 0001:fffff07d       __catch$?append@?$QList@VQString@@@@QAEXABVQString@@@Z$0 1000007d f   KrakenSupport.obj
 0001:fffff07d       __catch$?append@?$QList@VQString@@@@QAEXABVQString@@@Z$0 1000007d f   KrakenBuildWorker.obj
 0001:fffff07d       __catch$?append@?$QList@VQString@@@@QAEXABVQString@@@Z$0 1000007d f   KrakenClassifyTask.obj
 0001:fffff07d       __catch$?append@?$QList@VQString@@@@QAEXABVQString@@@Z$0 1000007d f   KrakenClassifyValidator.obj
 0001:fffff07d       __catch$?append@?$QList@VQString@@@@QAEXABVQString@@@Z$0 1000007d f   KrakenTranslateLogParser.obj
 0001:fffff07d       __catch$?append@?$QList@VQString@@@@QAEXABVQString@@@Z$0 1000007d f   KrakenBuildValidator.obj
 0001:fffff07d       __catch$?append@?$QList@VQString@@@@QAEXABVQString@@@Z$0 1000007d f   KrakenClassifyLogParser.obj
 0001:fffff07e       __catch$?node_copy@?$QList@VWorkflowNotification@U2@@@@AAEXPAUNode@1@00@Z$0 1000007e f   KrakenClassifyValidator.obj
 0001:fffff083       __ehhandler$??$getAttributeValue@VQString@@@Attribute@U2@@QBE?AVQString@@PAVWorkflowContext@Workflow@1@@Z 10000083 f   KrakenClassifyWorker.obj
 0001:fffff085       __catch$?createNode@?$QMapData@VQString@@PAVPropertyDelegate@U2@@@@QAEPAU?$QMapNode@VQString@@PAVPropertyDelegate@U2@@@@ABVQString@@ABQAVPropertyDelegate@U2@@PAU2@_N@Z$2 10000085 f   KrakenClassifyWorkerFactory.obj
 0001:fffff085       __catch$?append@?$QList@PAVAttribute@U2@@@@QAEXABQAVAttribute@U2@@@Z$4 10000085 f   KrakenClassifyWorkerFactory.obj
 0001:fffff085       __catch$?createNode@?$QMapData@VQString@@I@@QAEPAU?$QMapNode@VQString@@I@@ABVQString@@ABIPAU2@_N@Z$2 10000085 f   KrakenClassifyWorker.obj
 0001:fffff085       __catch$?append@?$QList@PAVPortDescriptor@Workflow@U2@@@@QAEXABQAVPortDescriptor@Workflow@U2@@@Z$4 10000085 f   KrakenClassifyWorkerFactory.obj
 0001:fffff085       __catch$?node_copy@?$QList@VDescriptor@U2@@@@AAEXPAUNode@1@00@Z$0 10000085 f   KrakenClassifyWorker.obj
 0001:fffff08e       __catch$?createNode@?$QMapData@VQString@@VQVariant@@@@QAEPAU?$QMapNode@VQString@@VQVariant@@@@ABVQString@@ABVQVariant@@PAU2@_N@Z$0 1000008e f   KrakenBuildWorkerFactory.obj
 0001:fffff08e       __catch$?createNode@?$QMapData@VQString@@VQScriptValue@@@@QAEPAU?$QMapNode@VQString@@VQScriptValue@@@@ABVQString@@ABVQScriptValue@@PAU2@_N@Z$0 1000008e f   KrakenClassifyWorker.obj
 0001:fffff08e       __catch$?createNode@?$QMapData@VQString@@VQVariant@@@@QAEPAU?$QMapNode@VQString@@VQVariant@@@@ABVQString@@ABVQVariant@@PAU2@_N@Z$0 1000008e f   KrakenClassifyWorker.obj
 0001:fffff08e       __catch$?createNode@?$QMapData@VQString@@VQVariant@@@@QAEPAU?$QMapNode@VQString@@VQVariant@@@@ABVQString@@ABVQVariant@@PAU2@_N@Z$0 1000008e f   KrakenClassifyWorkerFactory.obj
 0001:fffff096       __catch$?_Copy@?$basic_string@DU?$char_traits@D@std@@V?$allocator@D@2@@std@@QAEXII@Z$0 10000096 f   KrakenBuildTask.obj
 0001:fffff096       __catch$?_Copy@?$basic_string@DU?$char_traits@D@std@@V?$allocator@D@2@@std@@QAEXII@Z$0 10000096 f   moc_KrakenClassifyWorker.obj
 0001:fffff096       __catch$?_Copy@?$basic_string@DU?$char_traits@D@std@@V?$allocator@D@2@@std@@QAEXII@Z$0 10000096 f   KrakenTranslateLogParser.obj
 0001:fffff096       __catch$?_Copy@?$basic_string@DU?$char_traits@D@std@@V?$allocator@D@2@@std@@QAEXII@Z$0 10000096 f   moc_KrakenBuildTask.obj
 0001:fffff096       __catch$?_Copy@?$basic_string@DU?$char_traits@D@std@@V?$allocator@D@2@@std@@QAEXII@Z$0 10000096 f   KrakenClassifyWorker.obj
 0001:fffff096       __catch$?_Copy@?$basic_string@DU?$char_traits@D@std@@V?$allocator@D@2@@std@@QAEXII@Z$0 10000096 f   moc_KrakenBuildWorker.obj
 0001:fffff096       __catch$?_Copy@?$basic_string@DU?$char_traits@D@std@@V?$allocator@D@2@@std@@QAEXII@Z$0 10000096 f   KrakenSupport.obj
 0001:fffff096       __catch$?_Copy@?$basic_string@DU?$char_traits@D@std@@V?$allocator@D@2@@std@@QAEXII@Z$0 10000096 f   KrakenClassifyPrompter.obj
 0001:fffff096       __catch$?_Copy@?$basic_string@DU?$char_traits@D@std@@V?$allocator@D@2@@std@@QAEXII@Z$0 10000096 f   moc_KrakenClassifyPrompter.obj
 0001:fffff096       __catch$?_Copy@?$basic_string@DU?$char_traits@D@std@@V?$allocator@D@2@@std@@QAEXII@Z$0 10000096 f   KrakenClassifyLogParser.obj
 0001:fffff096       __catch$?_Copy@?$basic_string@DU?$char_traits@D@std@@V?$allocator@D@2@@std@@QAEXII@Z$0 10000096 f   KrakenClassifyTask.obj
 0001:fffff096       __catch$?_Copy@?$basic_string@DU?$char_traits@D@std@@V?$allocator@D@2@@std@@QAEXII@Z$0 10000096 f   KrakenClassifyWorkerFactory.obj
 0001:fffff096       __catch$?_Copy@?$basic_string@DU?$char_traits@D@std@@V?$allocator@D@2@@std@@QAEXII@Z$0 10000096 f   KrakenBuildValidator.obj
 0001:fffff096       __catch$?_Copy@?$basic_string@DU?$char_traits@D@std@@V?$allocator@D@2@@std@@QAEXII@Z$0 10000096 f   moc_KrakenSupport.obj
 0001:fffff096       __catch$?_Copy@?$basic_string@DU?$char_traits@D@std@@V?$allocator@D@2@@std@@QAEXII@Z$0 10000096 f   moc_KrakenBuildPrompter.obj
 0001:fffff096       __catch$?_Copy@?$basic_string@DU?$char_traits@D@std@@V?$allocator@D@2@@std@@QAEXII@Z$0 10000096 f   KrakenClassifyValidator.obj
 0001:fffff096       __catch$?_Copy@?$basic_string@DU?$char_traits@D@std@@V?$allocator@D@2@@std@@QAEXII@Z$0 10000096 f   moc_KrakenSupportPlugin.obj
 0001:fffff096       __catch$?_Copy@?$basic_string@DU?$char_traits@D@std@@V?$allocator@D@2@@std@@QAEXII@Z$0 10000096 f   KrakenSupportPlugin.obj
 0001:fffff096       __catch$?_Copy@?$basic_string@DU?$char_traits@D@std@@V?$allocator@D@2@@std@@QAEXII@Z$0 10000096 f   KrakenBuildPrompter.obj
 0001:fffff096       __catch$?_Copy@?$basic_string@DU?$char_traits@D@std@@V?$allocator@D@2@@std@@QAEXII@Z$0 10000096 f   moc_KrakenClassifyTask.obj
 0001:fffff096       __catch$?_Copy@?$basic_string@DU?$char_traits@D@std@@V?$allocator@D@2@@std@@QAEXII@Z$0 10000096 f   KrakenBuildWorkerFactory.obj
 0001:fffff096       __catch$?_Copy@?$basic_string@DU?$char_traits@D@std@@V?$allocator@D@2@@std@@QAEXII@Z$0 10000096 f   KrakenBuildWorker.obj
 0001:fffff09d       __catch$?createNode@?$QMapData@VDescriptor@U2@@V?$QExplicitlySharedDataPointer@VDataType@U2@@@@@@QAEPAU?$QMapNode@VDescriptor@U2@@V?$QExplicitlySharedDataPointer@VDataType@U2@@@@@@ABVDescriptor@U2@@ABV?$QExplicitlySharedDataPointer@VDataType@U2@@@@PAU2@_N@Z$2 1000009d f   KrakenClassifyWorkerFactory.obj
 0001:fffff09e       __catch$??0?$QList@VQString@@@@QAE@ABV0@@Z$0 1000009e f   KrakenBuildWorker.obj
 0001:fffff09e       __catch$??0?$QList@VQString@@@@QAE@ABV0@@Z$0 1000009e f   KrakenClassifyLogParser.obj
 0001:fffff09e       __catch$??0?$QList@VQString@@@@QAE@ABV0@@Z$0 1000009e f   KrakenSupport.obj
 0001:fffff09e       __catch$??0?$QList@VQString@@@@QAE@ABV0@@Z$0 1000009e f   KrakenClassifyValidator.obj
 0001:fffff09e       __catch$??0?$QList@VQString@@@@QAE@ABV0@@Z$0 1000009e f   KrakenBuildValidator.obj
 0001:fffff09e       __catch$??0?$QList@VQString@@@@QAE@ABV0@@Z$0 1000009e f   KrakenClassifyTask.obj
 0001:fffff09e       __catch$??0?$QList@PAVPort@Workflow@U2@@@@QAE@ABV0@@Z$0 1000009e f   KrakenClassifyPrompter.obj
 0001:fffff09e       __catch$??0?$QList@VDescriptor@U2@@@@QAE@ABV0@@Z$0 1000009e f   KrakenClassifyWorker.obj
 0001:fffff09e       __catch$??0?$QList@VQString@@@@QAE@ABV0@@Z$0 1000009e f   KrakenTranslateLogParser.obj
 0001:fffff0a0       __catch$?append@?$QList@VWorkflowNotification@U2@@@@QAEXABVWorkflowNotification@U2@@@Z$0 100000a0 f   KrakenClassifyValidator.obj
 0001:fffff0a0       __catch$?append@?$QList@VWorkflowNotification@U2@@@@QAEXABVWorkflowNotification@U2@@@Z$2 100000a0 f   KrakenClassifyValidator.obj
 0001:fffff0a3       __catch$?createNode@?$QMapData@VQString@@VQScriptValue@@@@QAEPAU?$QMapNode@VQString@@VQScriptValue@@@@ABVQString@@ABVQScriptValue@@PAU2@_N@Z$2 100000a3 f   KrakenClassifyWorker.obj
 0001:fffff0a3       __catch$?createNode@?$QMapData@VQString@@VQVariant@@@@QAEPAU?$QMapNode@VQString@@VQVariant@@@@ABVQString@@ABVQVariant@@PAU2@_N@Z$2 100000a3 f   KrakenBuildWorkerFactory.obj
 0001:fffff0a3       __catch$?createNode@?$QMapData@VQString@@VQVariant@@@@QAEPAU?$QMapNode@VQString@@VQVariant@@@@ABVQString@@ABVQVariant@@PAU2@_N@Z$2 100000a3 f   KrakenClassifyWorkerFactory.obj
 0001:fffff0a3       __catch$?createNode@?$QMapData@VQString@@VQVariant@@@@QAEPAU?$QMapNode@VQString@@VQVariant@@@@ABVQString@@ABVQVariant@@PAU2@_N@Z$2 100000a3 f   KrakenClassifyWorker.obj
 0001:fffff0aa       __catch$?detach_helper@?$QList@VDescriptor@U2@@@@AAEXH@Z$0 100000aa f   KrakenClassifyWorker.obj
 0001:fffff0ac       __catch$?append@?$QList@VDescriptor@U2@@@@QAEXABVDescriptor@U2@@@Z$2 100000ac f   KrakenClassifyWorker.obj
 0001:fffff0ac       __catch$?append@?$QList@VDescriptor@U2@@@@QAEXABVDescriptor@U2@@@Z$0 100000ac f   KrakenClassifyWorker.obj
 0001:fffff0ce       __catch$?append@?$QList@VQString@@@@QAEXABVQString@@@Z$4 100000ce f   KrakenClassifyLogParser.obj
 0001:fffff0ce       __catch$?append@?$QList@VQString@@@@QAEXABVQString@@@Z$4 100000ce f   KrakenBuildValidator.obj
 0001:fffff0ce       __catch$?append@?$QList@VQString@@@@QAEXABVQString@@@Z$4 100000ce f   KrakenClassifyWorker.obj
 0001:fffff0ce       __catch$?append@?$QList@VQString@@@@QAEXABVQString@@@Z$4 100000ce f   KrakenClassifyValidator.obj
 0001:fffff0ce       __catch$?append@?$QList@VQString@@@@QAEXABVQString@@@Z$4 100000ce f   KrakenSupport.obj
 0001:fffff0ce       __catch$?append@?$QList@VQString@@@@QAEXABVQString@@@Z$4 100000ce f   KrakenBuildWorker.obj
 0001:fffff0ce       __catch$?append@?$QList@VQString@@@@QAEXABVQString@@@Z$4 100000ce f   KrakenClassifyTask.obj
 0001:fffff0ce       __catch$?append@?$QList@VQString@@@@QAEXABVQString@@@Z$4 100000ce f   KrakenTranslateLogParser.obj
 0001:fffff0d3       __catch$?_Copy@?$basic_string@DU?$char_traits@D@std@@V?$allocator@D@2@@std@@QAEXII@Z$1 100000d3 f   moc_KrakenSupportPlugin.obj
 0001:fffff0d3       __catch$?_Copy@?$basic_string@DU?$char_traits@D@std@@V?$allocator@D@2@@std@@QAEXII@Z$1 100000d3 f   moc_KrakenClassifyTask.obj
 0001:fffff0d3       __catch$?_Copy@?$basic_string@DU?$char_traits@D@std@@V?$allocator@D@2@@std@@QAEXII@Z$1 100000d3 f   KrakenSupportPlugin.obj
 0001:fffff0d3       __catch$?_Copy@?$basic_string@DU?$char_traits@D@std@@V?$allocator@D@2@@std@@QAEXII@Z$1 100000d3 f   KrakenClassifyValidator.obj
 0001:fffff0d3       __catch$?_Copy@?$basic_string@DU?$char_traits@D@std@@V?$allocator@D@2@@std@@QAEXII@Z$1 100000d3 f   KrakenBuildValidator.obj
 0001:fffff0d3       __catch$?_Copy@?$basic_string@DU?$char_traits@D@std@@V?$allocator@D@2@@std@@QAEXII@Z$1 100000d3 f   KrakenTranslateLogParser.obj
 0001:fffff0d3       __catch$?_Copy@?$basic_string@DU?$char_traits@D@std@@V?$allocator@D@2@@std@@QAEXII@Z$1 100000d3 f   KrakenClassifyPrompter.obj
 0001:fffff0d3       __catch$?_Copy@?$basic_string@DU?$char_traits@D@std@@V?$allocator@D@2@@std@@QAEXII@Z$1 100000d3 f   moc_KrakenSupport.obj
 0001:fffff0d3       __catch$?_Copy@?$basic_string@DU?$char_traits@D@std@@V?$allocator@D@2@@std@@QAEXII@Z$1 100000d3 f   KrakenClassifyTask.obj
 0001:fffff0d3       __catch$?_Copy@?$basic_string@DU?$char_traits@D@std@@V?$allocator@D@2@@std@@QAEXII@Z$1 100000d3 f   moc_KrakenBuildPrompter.obj
 0001:fffff0d3       __catch$?_Copy@?$basic_string@DU?$char_traits@D@std@@V?$allocator@D@2@@std@@QAEXII@Z$1 100000d3 f   KrakenClassifyLogParser.obj
 0001:fffff0d3       __catch$?_Copy@?$basic_string@DU?$char_traits@D@std@@V?$allocator@D@2@@std@@QAEXII@Z$1 100000d3 f   KrakenBuildPrompter.obj
 0001:fffff0d3       __catch$?_Copy@?$basic_string@DU?$char_traits@D@std@@V?$allocator@D@2@@std@@QAEXII@Z$1 100000d3 f   KrakenSupport.obj
 0001:fffff0d3       __catch$?_Copy@?$basic_string@DU?$char_traits@D@std@@V?$allocator@D@2@@std@@QAEXII@Z$1 100000d3 f   moc_KrakenClassifyPrompter.obj
 0001:fffff0d3       __catch$?_Copy@?$basic_string@DU?$char_traits@D@std@@V?$allocator@D@2@@std@@QAEXII@Z$1 100000d3 f   moc_KrakenBuildWorker.obj
 0001:fffff0d3       __catch$?_Copy@?$basic_string@DU?$char_traits@D@std@@V?$allocator@D@2@@std@@QAEXII@Z$1 100000d3 f   moc_KrakenBuildTask.obj
 0001:fffff0d3       __catch$?_Copy@?$basic_string@DU?$char_traits@D@std@@V?$allocator@D@2@@std@@QAEXII@Z$1 100000d3 f   KrakenBuildWorkerFactory.obj
 0001:fffff0d3       __catch$?_Copy@?$basic_string@DU?$char_traits@D@std@@V?$allocator@D@2@@std@@QAEXII@Z$1 100000d3 f   KrakenClassifyWorker.obj
 0001:fffff0d3       __catch$?_Copy@?$basic_string@DU?$char_traits@D@std@@V?$allocator@D@2@@std@@QAEXII@Z$1 100000d3 f   moc_KrakenClassifyWorker.obj
 0001:fffff0d3       __catch$?_Copy@?$basic_string@DU?$char_traits@D@std@@V?$allocator@D@2@@std@@QAEXII@Z$1 100000d3 f   KrakenBuildTask.obj
 0001:fffff0d3       __catch$?_Copy@?$basic_string@DU?$char_traits@D@std@@V?$allocator@D@2@@std@@QAEXII@Z$1 100000d3 f   KrakenClassifyWorkerFactory.obj
 0001:fffff0d3       __catch$?_Copy@?$basic_string@DU?$char_traits@D@std@@V?$allocator@D@2@@std@@QAEXII@Z$1 100000d3 f   KrakenBuildWorker.obj
 0001:fffff0ef       __catch$?detach_helper_grow@?$QList@VWorkflowNotification@U2@@@@AAEPAUNode@1@HH@Z$2 100000ef f   KrakenClassifyValidator.obj
 0001:fffff0ef       __catch$?detach_helper_grow@?$QList@VDescriptor@U2@@@@AAEPAUNode@1@HH@Z$2 100000ef f   KrakenClassifyWorker.obj
 0001:fffff0f1       __catch$?detach_helper_grow@?$QList@PAVPortDescriptor@Workflow@U2@@@@AAEPAUNode@1@HH@Z$2 100000f1 f   KrakenClassifyWorkerFactory.obj
 0001:fffff0f1       __catch$?detach_helper_grow@?$QList@PAVAttribute@U2@@@@AAEPAUNode@1@HH@Z$2 100000f1 f   KrakenClassifyWorkerFactory.obj
 0001:fffff0f1       __catch$?detach_helper_grow@?$QList@PAVAttribute@U2@@@@AAEPAUNode@1@HH@Z$0 100000f1 f   KrakenClassifyWorkerFactory.obj
 0001:fffff0f1       __catch$?detach_helper_grow@?$QList@PAVPortDescriptor@Workflow@U2@@@@AAEPAUNode@1@HH@Z$0 100000f1 f   KrakenClassifyWorkerFactory.obj
 0001:fffff11e       __catch$?detach_helper_grow@?$QList@VQString@@@@AAEPAUNode@1@HH@Z$2 1000011e f   KrakenClassifyValidator.obj
 0001:fffff11e       __catch$?detach_helper_grow@?$QList@VQString@@@@AAEPAUNode@1@HH@Z$2 1000011e f   KrakenClassifyTask.obj
 0001:fffff11e       __catch$?detach_helper_grow@?$QList@VQString@@@@AAEPAUNode@1@HH@Z$2 1000011e f   KrakenBuildValidator.obj
 0001:fffff11e       __catch$?detach_helper_grow@?$QList@VQString@@@@AAEPAUNode@1@HH@Z$2 1000011e f   KrakenClassifyWorker.obj
 0001:fffff11e       __catch$?detach_helper_grow@?$QList@VQString@@@@AAEPAUNode@1@HH@Z$2 1000011e f   KrakenTranslateLogParser.obj
 0001:fffff11e       __catch$?detach_helper_grow@?$QList@VQString@@@@AAEPAUNode@1@HH@Z$2 1000011e f   KrakenBuildWorker.obj
 0001:fffff11e       __catch$?detach_helper_grow@?$QList@VQString@@@@AAEPAUNode@1@HH@Z$2 1000011e f   KrakenSupport.obj
 0001:fffff11e       __catch$?detach_helper_grow@?$QList@VQString@@@@AAEPAUNode@1@HH@Z$2 1000011e f   KrakenClassifyLogParser.obj
 0001:fffff12a       __catch$?detach_helper_grow@?$QList@VDescriptor@U2@@@@AAEPAUNode@1@HH@Z$0 1000012a f   KrakenClassifyWorker.obj
 0001:fffff12a       __catch$?detach_helper_grow@?$QList@VWorkflowNotification@U2@@@@AAEPAUNode@1@HH@Z$0 1000012a f   KrakenClassifyValidator.obj
 0001:fffff159       __catch$?detach_helper_grow@?$QList@VQString@@@@AAEPAUNode@1@HH@Z$0 10000159 f   KrakenBuildValidator.obj
 0001:fffff159       __catch$?detach_helper_grow@?$QList@VQString@@@@AAEPAUNode@1@HH@Z$0 10000159 f   KrakenSupport.obj
 0001:fffff159       __catch$?detach_helper_grow@?$QList@VQString@@@@AAEPAUNode@1@HH@Z$0 10000159 f   KrakenClassifyValidator.obj
 0001:fffff159       __catch$?detach_helper_grow@?$QList@VQString@@@@AAEPAUNode@1@HH@Z$0 10000159 f   KrakenTranslateLogParser.obj
 0001:fffff159       __catch$?detach_helper_grow@?$QList@VQString@@@@AAEPAUNode@1@HH@Z$0 10000159 f   KrakenBuildWorker.obj
 0001:fffff159       __catch$?detach_helper_grow@?$QList@VQString@@@@AAEPAUNode@1@HH@Z$0 10000159 f   KrakenClassifyTask.obj
 0001:fffff159       __catch$?detach_helper_grow@?$QList@VQString@@@@AAEPAUNode@1@HH@Z$0 10000159 f   KrakenClassifyWorker.obj
 0001:fffff159       __catch$?detach_helper_grow@?$QList@VQString@@@@AAEPAUNode@1@HH@Z$0 10000159 f   KrakenClassifyLogParser.obj
 0001:00000000       ??__E?_Generic_object@?$_Error_objects@H@std@@2V_Generic_error_category@2@A@@YAXXZ 10001000 f   DatabaseSizeRelation.obj
 0001:00000010       ??__E?_Iostream_object@?$_Error_objects@H@std@@2V_Iostream_error_category@2@A@@YAXXZ 10001010 f   DatabaseSizeRelation.obj
 0001:00000020       ??__E?_System_object@?$_Error_objects@H@std@@2V_System_error_category@2@A@@YAXXZ 10001020 f   DatabaseSizeRelation.obj
 0001:00000030       ??__EalgoLog@U2@@YAXXZ     10001030 f   DatabaseSizeRelation.obj
 0001:000000b0       ??__EcmdLog@U2@@YAXXZ      100010b0 f   DatabaseSizeRelation.obj
 0001:00000130       ??__EcoreLog@U2@@YAXXZ     10001130 f   DatabaseSizeRelation.obj
 0001:000001b0       ??__EioLog@U2@@YAXXZ       100011b0 f   DatabaseSizeRelation.obj
 0001:00000230       ??__EperfLog@U2@@YAXXZ     10001230 f   DatabaseSizeRelation.obj
 0001:000002b0       ??__EscriptLog@U2@@YAXXZ   100012b0 f   DatabaseSizeRelation.obj
 0001:00000330       ??__EtaskLog@U2@@YAXXZ     10001330 f   DatabaseSizeRelation.obj
 0001:000003b0       ??__EuiLog@U2@@YAXXZ       100013b0 f   DatabaseSizeRelation.obj
 0001:00000430       ??__EuserActLog@U2@@YAXXZ  10001430 f   DatabaseSizeRelation.obj
 0001:000004b0       ??__E?_Generic_object@?$_Error_objects@H@std@@2V_Generic_error_category@2@A@@YAXXZ 100014b0 f   KrakenBuildPrompter.obj
 0001:000004c0       ??__E?_Iostream_object@?$_Error_objects@H@std@@2V_Iostream_error_category@2@A@@YAXXZ 100014c0 f   KrakenBuildPrompter.obj
 0001:000004d0       ??__E?_System_object@?$_Error_objects@H@std@@2V_System_error_category@2@A@@YAXXZ 100014d0 f   KrakenBuildPrompter.obj
 0001:000004e0       ??__EalgoLog@U2@@YAXXZ     100014e0 f   KrakenBuildPrompter.obj
 0001:00000560       ??__EcmdLog@U2@@YAXXZ      10001560 f   KrakenBuildPrompter.obj
 0001:000005e0       ??__EcoreLog@U2@@YAXXZ     100015e0 f   KrakenBuildPrompter.obj
 0001:00000660       ??__EioLog@U2@@YAXXZ       10001660 f   KrakenBuildPrompter.obj
 0001:000006e0       ??__EperfLog@U2@@YAXXZ     100016e0 f   KrakenBuildPrompter.obj
 0001:00000760       ??__EscriptLog@U2@@YAXXZ   10001760 f   KrakenBuildPrompter.obj
 0001:000007e0       ??__EtaskLog@U2@@YAXXZ     100017e0 f   KrakenBuildPrompter.obj
 0001:00000860       ??__EuiLog@U2@@YAXXZ       10001860 f   KrakenBuildPrompter.obj
 0001:000008e0       ??__EuserActLog@U2@@YAXXZ  100018e0 f   KrakenBuildPrompter.obj
 0001:00000960       ??__E?BUILD@KrakenBuildTaskSettings@U2@@2VQString@@B@@YAXXZ 10001960 f   KrakenBuildTask.obj
 0001:00000980       ??__E?SHRINK@KrakenBuildTaskSettings@U2@@2VQString@@B@@YAXXZ 10001980 f   KrakenBuildTask.obj
 0001:000009a0       ??__E?_Generic_object@?$_Error_objects@H@std@@2V_Generic_error_category@2@A@@YAXXZ 100019a0 f   KrakenBuildTask.obj
 0001:000009b0       ??__E?_Iostream_object@?$_Error_objects@H@std@@2V_Iostream_error_category@2@A@@YAXXZ 100019b0 f   KrakenBuildTask.obj
 0001:000009c0       ??__E?_System_object@?$_Error_objects@H@std@@2V_System_error_category@2@A@@YAXXZ 100019c0 f   KrakenBuildTask.obj
 0001:000009d0       ??__EalgoLog@U2@@YAXXZ     100019d0 f   KrakenBuildTask.obj
 0001:00000a50       ??__EcmdLog@U2@@YAXXZ      10001a50 f   KrakenBuildTask.obj
 0001:00000ad0       ??__EcoreLog@U2@@YAXXZ     10001ad0 f   KrakenBuildTask.obj
 0001:00000b50       ??__EioLog@U2@@YAXXZ       10001b50 f   KrakenBuildTask.obj
 0001:00000bd0       ??__EperfLog@U2@@YAXXZ     10001bd0 f   KrakenBuildTask.obj
 0001:00000c50       ??__EscriptLog@U2@@YAXXZ   10001c50 f   KrakenBuildTask.obj
 0001:00000cd0       ??__EtaskLog@U2@@YAXXZ     10001cd0 f   KrakenBuildTask.obj
 0001:00000d50       ??__EuiLog@U2@@YAXXZ       10001d50 f   KrakenBuildTask.obj
 0001:00000dd0       ??__EuserActLog@U2@@YAXXZ  10001dd0 f   KrakenBuildTask.obj
 0001:00000e50       ??__E?_Generic_object@?$_Error_objects@H@std@@2V_Generic_error_category@2@A@@YAXXZ 10001e50 f   KrakenBuildValidator.obj
 0001:00000e60       ??__E?_Iostream_object@?$_Error_objects@H@std@@2V_Iostream_error_category@2@A@@YAXXZ 10001e60 f   KrakenBuildValidator.obj
 0001:00000e70       ??__E?_System_object@?$_Error_objects@H@std@@2V_System_error_category@2@A@@YAXXZ 10001e70 f   KrakenBuildValidator.obj
 0001:00000e80       ??__EalgoLog@U2@@YAXXZ     10001e80 f   KrakenBuildValidator.obj
 0001:00000f00       ??__EcmdLog@U2@@YAXXZ      10001f00 f   KrakenBuildValidator.obj
 0001:00000f80       ??__EcoreLog@U2@@YAXXZ     10001f80 f   KrakenBuildValidator.obj
 0001:00001000       ??__EioLog@U2@@YAXXZ       10002000 f   KrakenBuildValidator.obj
 0001:00001080       ??__EperfLog@U2@@YAXXZ     10002080 f   KrakenBuildValidator.obj
 0001:00001100       ??__EscriptLog@U2@@YAXXZ   10002100 f   KrakenBuildValidator.obj
 0001:00001180       ??__EtaskLog@U2@@YAXXZ     10002180 f   KrakenBuildValidator.obj
 0001:00001200       ??__EuiLog@U2@@YAXXZ       10002200 f   KrakenBuildValidator.obj
 0001:00001280       ??__EuserActLog@U2@@YAXXZ  10002280 f   KrakenBuildValidator.obj
 0001:00001300       ??__E?_Generic_object@?$_Error_objects@H@std@@2V_Generic_error_category@2@A@@YAXXZ 10002300 f   KrakenBuildWorker.obj
 0001:00001310       ??__E?_Iostream_object@?$_Error_objects@H@std@@2V_Iostream_error_category@2@A@@YAXXZ 10002310 f   KrakenBuildWorker.obj
 0001:00001320       ??__E?_System_object@?$_Error_objects@H@std@@2V_System_error_category@2@A@@YAXXZ 10002320 f   KrakenBuildWorker.obj
 0001:00001330       ??__EalgoLog@U2@@YAXXZ     10002330 f   KrakenBuildWorker.obj
 0001:000013b0       ??__EcmdLog@U2@@YAXXZ      100023b0 f   KrakenBuildWorker.obj
 0001:00001430       ??__EcoreLog@U2@@YAXXZ     10002430 f   KrakenBuildWorker.obj
 0001:000014b0       ??__EioLog@U2@@YAXXZ       100024b0 f   KrakenBuildWorker.obj
 0001:00001530       ??__EperfLog@U2@@YAXXZ     10002530 f   KrakenBuildWorker.obj
 0001:000015b0       ??__EscriptLog@U2@@YAXXZ   100025b0 f   KrakenBuildWorker.obj
 0001:00001630       ??__EtaskLog@U2@@YAXXZ     10002630 f   KrakenBuildWorker.obj
 0001:000016b0       ??__EuiLog@U2@@YAXXZ       100026b0 f   KrakenBuildWorker.obj
 0001:00001730       ??__EuserActLog@U2@@YAXXZ  10002730 f   KrakenBuildWorker.obj
 0001:000017b0       ??__E?ACTOR_ID@KrakenBuildWorkerFactory@LocalWorkflow@U2@@2VQString@@B@@YAXXZ 100027b0 f   KrakenBuildWorkerFactory.obj
 0001:000017d0       ??__E?CLEAN_ATTR_ID@KrakenBuildWorkerFactory@LocalWorkflow@U2@@2VQString@@B@@YAXXZ 100027d0 f   KrakenBuildWorkerFactory.obj
 0001:000017f0       ??__E?GENOMIC_LIBRARY_ATTR_ID@KrakenBuildWorkerFactory@LocalWorkflow@U2@@2VQString@@B@@YAXXZ 100027f0 f   KrakenBuildWorkerFactory.obj
 0001:00001810       ??__E?INPUT_DATABASE_NAME_ATTR_ID@KrakenBuildWorkerFactory@LocalWorkflow@U2@@2VQString@@B@@YAXXZ 10002810 f   KrakenBuildWorkerFactory.obj
 0001:00001830       ??__E?JELLYFISH_HASH_SIZE_ATTR_ID@KrakenBuildWorkerFactory@LocalWorkflow@U2@@2VQString@@B@@YAXXZ 10002830 f   KrakenBuildWorkerFactory.obj
 0001:00001850       ??__E?K_MER_LENGTH_ATTR_ID@KrakenBuildWorkerFactory@LocalWorkflow@U2@@2VQString@@B@@YAXXZ 10002850 f   KrakenBuildWorkerFactory.obj
 0001:00001870       ??__E?MAXIMUM_DATABASE_SIZE_ATTR_ID@KrakenBuildWorkerFactory@LocalWorkflow@U2@@2VQString@@B@@YAXXZ 10002870 f   KrakenBuildWorkerFactory.obj
 0001:00001890       ??__E?MINIMIZER_LENGTH_ATTR_ID@KrakenBuildWorkerFactory@LocalWorkflow@U2@@2VQString@@B@@YAXXZ 10002890 f   KrakenBuildWorkerFactory.obj
 0001:000018b0       ??__E?MODE_ATTR_ID@KrakenBuildWorkerFactory@LocalWorkflow@U2@@2VQString@@B@@YAXXZ 100028b0 f   KrakenBuildWorkerFactory.obj
 0001:000018d0       ??__E?NEW_DATABASE_NAME_ATTR_ID@KrakenBuildWorkerFactory@LocalWorkflow@U2@@2VQString@@B@@YAXXZ 100028d0 f   KrakenBuildWorkerFactory.obj
 0001:000018f0       ??__E?NUMBER_OF_K_MERS_ATTR_ID@KrakenBuildWorkerFactory@LocalWorkflow@U2@@2VQString@@B@@YAXXZ 100028f0 f   KrakenBuildWorkerFactory.obj
 0001:00001910       ??__E?OUTPUT_PORT_ID@KrakenBuildWorkerFactory@LocalWorkflow@U2@@2VQString@@B@@YAXXZ 10002910 f   KrakenBuildWorkerFactory.obj
 0001:00001930       ??__E?SHRINK_BLOCK_OFFSET_ATTR_ID@KrakenBuildWorkerFactory@LocalWorkflow@U2@@2VQString@@B@@YAXXZ 10002930 f   KrakenBuildWorkerFactory.obj
 0001:00001950       ??__E?THREADS_NUMBER_ATTR_ID@KrakenBuildWorkerFactory@LocalWorkflow@U2@@2VQString@@B@@YAXXZ 10002950 f   KrakenBuildWorkerFactory.obj
 0001:00001970       ??__E?WORK_ON_DISK_ATTR_ID@KrakenBuildWorkerFactory@LocalWorkflow@U2@@2VQString@@B@@YAXXZ 10002970 f   KrakenBuildWorkerFactory.obj
 0001:00001990       ??__E?_Generic_object@?$_Error_objects@H@std@@2V_Generic_error_category@2@A@@YAXXZ 10002990 f   KrakenBuildWorkerFactory.obj
 0001:000019a0       ??__E?_Iostream_object@?$_Error_objects@H@std@@2V_Iostream_error_category@2@A@@YAXXZ 100029a0 f   KrakenBuildWorkerFactory.obj
 0001:000019b0       ??__E?_System_object@?$_Error_objects@H@std@@2V_System_error_category@2@A@@YAXXZ 100029b0 f   KrakenBuildWorkerFactory.obj
 0001:000019c0       ??__EalgoLog@U2@@YAXXZ     100029c0 f   KrakenBuildWorkerFactory.obj
 0001:00001a40       ??__EcmdLog@U2@@YAXXZ      10002a40 f   KrakenBuildWorkerFactory.obj
 0001:00001ac0       ??__EcoreLog@U2@@YAXXZ     10002ac0 f   KrakenBuildWorkerFactory.obj
 0001:00001b40       ??__EioLog@U2@@YAXXZ       10002b40 f   KrakenBuildWorkerFactory.obj
 0001:00001bc0       ??__EperfLog@U2@@YAXXZ     10002bc0 f   KrakenBuildWorkerFactory.obj
 0001:00001c40       ??__EscriptLog@U2@@YAXXZ   10002c40 f   KrakenBuildWorkerFactory.obj
 0001:00001cc0       ??__EtaskLog@U2@@YAXXZ     10002cc0 f   KrakenBuildWorkerFactory.obj
 0001:00001d40       ??__EuiLog@U2@@YAXXZ       10002d40 f   KrakenBuildWorkerFactory.obj
 0001:00001dc0       ??__EuserActLog@U2@@YAXXZ  10002dc0 f   KrakenBuildWorkerFactory.obj
 0001:00001e40       ??__E?_Generic_object@?$_Error_objects@H@std@@2V_Generic_error_category@2@A@@YAXXZ 10002e40 f   KrakenClassifyLogParser.obj
 0001:00001e50       ??__E?_Iostream_object@?$_Error_objects@H@std@@2V_Iostream_error_category@2@A@@YAXXZ 10002e50 f   KrakenClassifyLogParser.obj
 0001:00001e60       ??__E?_System_object@?$_Error_objects@H@std@@2V_System_error_category@2@A@@YAXXZ 10002e60 f   KrakenClassifyLogParser.obj
 0001:00001e70       ??__E?wellKnownErrors@KrakenClassifyLogParser@U2@@0VQStringList@@B@@YAXXZ 10002e70 f   KrakenClassifyLogParser.obj
 0001:00001e90       ??__EalgoLog@U2@@YAXXZ     10002e90 f   KrakenClassifyLogParser.obj
 0001:00001f10       ??__EcmdLog@U2@@YAXXZ      10002f10 f   KrakenClassifyLogParser.obj
 0001:00001f90       ??__EcoreLog@U2@@YAXXZ     10002f90 f   KrakenClassifyLogParser.obj
 0001:00002010       ??__EioLog@U2@@YAXXZ       10003010 f   KrakenClassifyLogParser.obj
 0001:00002090       ??__EperfLog@U2@@YAXXZ     10003090 f   KrakenClassifyLogParser.obj
 0001:00002110       ??__EscriptLog@U2@@YAXXZ   10003110 f   KrakenClassifyLogParser.obj
 0001:00002190       ??__EtaskLog@U2@@YAXXZ     10003190 f   KrakenClassifyLogParser.obj
 0001:00002210       ??__EuiLog@U2@@YAXXZ       10003210 f   KrakenClassifyLogParser.obj
 0001:00002290       ??__EuserActLog@U2@@YAXXZ  10003290 f   KrakenClassifyLogParser.obj
 0001:00002310       ??__E?_Generic_object@?$_Error_objects@H@std@@2V_Generic_error_category@2@A@@YAXXZ 10003310 f   KrakenClassifyPrompter.obj
 0001:00002320       ??__E?_Iostream_object@?$_Error_objects@H@std@@2V_Iostream_error_category@2@A@@YAXXZ 10003320 f   KrakenClassifyPrompter.obj
 0001:00002330       ??__E?_System_object@?$_Error_objects@H@std@@2V_System_error_category@2@A@@YAXXZ 10003330 f   KrakenClassifyPrompter.obj
 0001:00002340       ??__EalgoLog@U2@@YAXXZ     10003340 f   KrakenClassifyPrompter.obj
 0001:000023c0       ??__EcmdLog@U2@@YAXXZ      100033c0 f   KrakenClassifyPrompter.obj
 0001:00002440       ??__EcoreLog@U2@@YAXXZ     10003440 f   KrakenClassifyPrompter.obj
 0001:000024c0       ??__EioLog@U2@@YAXXZ       100034c0 f   KrakenClassifyPrompter.obj
 0001:00002540       ??__EperfLog@U2@@YAXXZ     10003540 f   KrakenClassifyPrompter.obj
 0001:000025c0       ??__EscriptLog@U2@@YAXXZ   100035c0 f   KrakenClassifyPrompter.obj
 0001:00002640       ??__EtaskLog@U2@@YAXXZ     10003640 f   KrakenClassifyPrompter.obj
 0001:000026c0       ??__EuiLog@U2@@YAXXZ       100036c0 f   KrakenClassifyPrompter.obj
 0001:00002740       ??__EuserActLog@U2@@YAXXZ  10003740 f   KrakenClassifyPrompter.obj
 0001:000027c0       ??__E?PAIRED_END@KrakenClassifyTaskSettings@U2@@2VQString@@B@@YAXXZ 100037c0 f   KrakenClassifyTask.obj
 0001:000027e0       ??__E?SINGLE_END@KrakenClassifyTaskSettings@U2@@2VQString@@B@@YAXXZ 100037e0 f   KrakenClassifyTask.obj
 0001:00002800       ??__E?_Generic_object@?$_Error_objects@H@std@@2V_Generic_error_category@2@A@@YAXXZ 10003800 f   KrakenClassifyTask.obj
 0001:00002810       ??__E?_Iostream_object@?$_Error_objects@H@std@@2V_Iostream_error_category@2@A@@YAXXZ 10003810 f   KrakenClassifyTask.obj
 0001:00002820       ??__E?_System_object@?$_Error_objects@H@std@@2V_System_error_category@2@A@@YAXXZ 10003820 f   KrakenClassifyTask.obj
 0001:00002830       ??__EalgoLog@U2@@YAXXZ     10003830 f   KrakenClassifyTask.obj
 0001:000028b0       ??__EcmdLog@U2@@YAXXZ      100038b0 f   KrakenClassifyTask.obj
 0001:00002930       ??__EcoreLog@U2@@YAXXZ     10003930 f   KrakenClassifyTask.obj
 0001:000029b0       ??__EioLog@U2@@YAXXZ       100039b0 f   KrakenClassifyTask.obj
 0001:00002a30       ??__EperfLog@U2@@YAXXZ     10003a30 f   KrakenClassifyTask.obj
 0001:00002ab0       ??__EscriptLog@U2@@YAXXZ   10003ab0 f   KrakenClassifyTask.obj
 0001:00002b30       ??__EtaskLog@U2@@YAXXZ     10003b30 f   KrakenClassifyTask.obj
 0001:00002bb0       ??__EuiLog@U2@@YAXXZ       10003bb0 f   KrakenClassifyTask.obj
 0001:00002c30       ??__EuserActLog@U2@@YAXXZ  10003c30 f   KrakenClassifyTask.obj
 0001:00002cb0       ??__E?_Generic_object@?$_Error_objects@H@std@@2V_Generic_error_category@2@A@@YAXXZ 10003cb0 f   KrakenClassifyValidator.obj
 0001:00002cc0       ??__E?_Iostream_object@?$_Error_objects@H@std@@2V_Iostream_error_category@2@A@@YAXXZ 10003cc0 f   KrakenClassifyValidator.obj
 0001:00002cd0       ??__E?_System_object@?$_Error_objects@H@std@@2V_System_error_category@2@A@@YAXXZ 10003cd0 f   KrakenClassifyValidator.obj
 0001:00002ce0       ??__EalgoLog@U2@@YAXXZ     10003ce0 f   KrakenClassifyValidator.obj
 0001:00002d60       ??__EcmdLog@U2@@YAXXZ      10003d60 f   KrakenClassifyValidator.obj
 0001:00002de0       ??__EcoreLog@U2@@YAXXZ     10003de0 f   KrakenClassifyValidator.obj
 0001:00002e60       ??__EioLog@U2@@YAXXZ       10003e60 f   KrakenClassifyValidator.obj
 0001:00002ee0       ??__EperfLog@U2@@YAXXZ     10003ee0 f   KrakenClassifyValidator.obj
 0001:00002f60       ??__EscriptLog@U2@@YAXXZ   10003f60 f   KrakenClassifyValidator.obj
 0001:00002fe0       ??__EtaskLog@U2@@YAXXZ     10003fe0 f   KrakenClassifyValidator.obj
 0001:00003060       ??__EuiLog@U2@@YAXXZ       10004060 f   KrakenClassifyValidator.obj
 0001:000030e0       ??__EuserActLog@U2@@YAXXZ  100040e0 f   KrakenClassifyValidator.obj
 0001:00003160       ??__E?KRAKEN_DIR@KrakenClassifyWorker@LocalWorkflow@U2@@0VQString@@B@@YAXXZ 10004160 f   KrakenClassifyWorker.obj
 0001:00003180       ??__E?_Generic_object@?$_Error_objects@H@std@@2V_Generic_error_category@2@A@@YAXXZ 10004180 f   KrakenClassifyWorker.obj
 0001:00003190       ??__E?_Iostream_object@?$_Error_objects@H@std@@2V_Iostream_error_category@2@A@@YAXXZ 10004190 f   KrakenClassifyWorker.obj
 0001:000031a0       ??__E?_System_object@?$_Error_objects@H@std@@2V_System_error_category@2@A@@YAXXZ 100041a0 f   KrakenClassifyWorker.obj
 0001:000031b0       ??__EalgoLog@U2@@YAXXZ     100041b0 f   KrakenClassifyWorker.obj
 0001:00003230       ??__EcmdLog@U2@@YAXXZ      10004230 f   KrakenClassifyWorker.obj
 0001:000032b0       ??__EcoreLog@U2@@YAXXZ     100042b0 f   KrakenClassifyWorker.obj
 0001:00003330       ??__EioLog@U2@@YAXXZ       10004330 f   KrakenClassifyWorker.obj
 0001:000033b0       ??__EperfLog@U2@@YAXXZ     100043b0 f   KrakenClassifyWorker.obj
 0001:00003430       ??__EscriptLog@U2@@YAXXZ   10004430 f   KrakenClassifyWorker.obj
 0001:000034b0       ??__EtaskLog@U2@@YAXXZ     100044b0 f   KrakenClassifyWorker.obj
 0001:00003530       ??__EuiLog@U2@@YAXXZ       10004530 f   KrakenClassifyWorker.obj
 0001:000035b0       ??__EuserActLog@U2@@YAXXZ  100045b0 f   KrakenClassifyWorker.obj
 0001:00003630       ??__E?ACTOR_ID@KrakenClassifyWorkerFactory@LocalWorkflow@U2@@2VQString@@B@@YAXXZ 10004630 f   KrakenClassifyWorkerFactory.obj
 0001:00003650       ??__E?DATABASE_ATTR_ID@KrakenClassifyWorkerFactory@LocalWorkflow@U2@@2VQString@@B@@YAXXZ 10004650 f   KrakenClassifyWorkerFactory.obj
 0001:00003670       ??__E?INPUT_DATA_ATTR_ID@KrakenClassifyWorkerFactory@LocalWorkflow@U2@@2VQString@@B@@YAXXZ 10004670 f   KrakenClassifyWorkerFactory.obj
 0001:00003690       ??__E?INPUT_PORT_ID@KrakenClassifyWorkerFactory@LocalWorkflow@U2@@2VQString@@B@@YAXXZ 10004690 f   KrakenClassifyWorkerFactory.obj
 0001:000036b0       ??__E?INPUT_SLOT@KrakenClassifyWorkerFactory@LocalWorkflow@U2@@2VQString@@B@@YAXXZ 100046b0 f   KrakenClassifyWorkerFactory.obj
 0001:000036d0       ??__E?MIN_HITS_NUMBER_ATTR_ID@KrakenClassifyWorkerFactory@LocalWorkflow@U2@@2VQString@@B@@YAXXZ 100046d0 f   KrakenClassifyWorkerFactory.obj
 0001:000036f0       ??__E?OUTPUT_PORT_ID@KrakenClassifyWorkerFactory@LocalWorkflow@U2@@2VQString@@B@@YAXXZ 100046f0 f   KrakenClassifyWorkerFactory.obj
 0001:00003710       ??__E?OUTPUT_URL_ATTR_ID@KrakenClassifyWorkerFactory@LocalWorkflow@U2@@2VQString@@B@@YAXXZ 10004710 f   KrakenClassifyWorkerFactory.obj
 0001:00003730       ??__E?PAIRED_END_TEXT@KrakenClassifyWorkerFactory@LocalWorkflow@U2@@2VQString@@B@@YAXXZ 10004730 f   KrakenClassifyWorkerFactory.obj
 0001:00003750       ??__E?PAIRED_INPUT_SLOT@KrakenClassifyWorkerFactory@LocalWorkflow@U2@@2VQString@@B@@YAXXZ 10004750 f   KrakenClassifyWorkerFactory.obj
 0001:00003770       ??__E?PRELOAD_DATABASE_ATTR_ID@KrakenClassifyWorkerFactory@LocalWorkflow@U2@@2VQString@@B@@YAXXZ 10004770 f   KrakenClassifyWorkerFactory.obj
 0001:00003790       ??__E?QUICK_OPERATION_ATTR_ID@KrakenClassifyWorkerFactory@LocalWorkflow@U2@@2VQString@@B@@YAXXZ 10004790 f   KrakenClassifyWorkerFactory.obj
 0001:000037b0       ??__E?SINGLE_END_TEXT@KrakenClassifyWorkerFactory@LocalWorkflow@U2@@2VQString@@B@@YAXXZ 100047b0 f   KrakenClassifyWorkerFactory.obj
 0001:000037d0       ??__E?THREADS_NUMBER_ATTR_ID@KrakenClassifyWorkerFactory@LocalWorkflow@U2@@2VQString@@B@@YAXXZ 100047d0 f   KrakenClassifyWorkerFactory.obj
 0001:000037f0       ??__E?WORKFLOW_CLASSIFY_TOOL_KRAKEN@KrakenClassifyWorkerFactory@LocalWorkflow@U2@@2VQString@@B@@YAXXZ 100047f0 f   KrakenClassifyWorkerFactory.obj
 0001:00003810       ??__E?_Generic_object@?$_Error_objects@H@std@@2V_Generic_error_category@2@A@@YAXXZ 10004810 f   KrakenClassifyWorkerFactory.obj
 0001:00003820       ??__E?_Iostream_object@?$_Error_objects@H@std@@2V_Iostream_error_category@2@A@@YAXXZ 10004820 f   KrakenClassifyWorkerFactory.obj
 0001:00003830       ??__E?_System_object@?$_Error_objects@H@std@@2V_System_error_category@2@A@@YAXXZ 10004830 f   KrakenClassifyWorkerFactory.obj
 0001:00003840       ??__EalgoLog@U2@@YAXXZ     10004840 f   KrakenClassifyWorkerFactory.obj
 0001:000038c0       ??__EcmdLog@U2@@YAXXZ      100048c0 f   KrakenClassifyWorkerFactory.obj
 0001:00003940       ??__EcoreLog@U2@@YAXXZ     10004940 f   KrakenClassifyWorkerFactory.obj
 0001:000039c0       ??__EioLog@U2@@YAXXZ       100049c0 f   KrakenClassifyWorkerFactory.obj
 0001:00003a40       ??__EperfLog@U2@@YAXXZ     10004a40 f   KrakenClassifyWorkerFactory.obj
 0001:00003ac0       ??__EscriptLog@U2@@YAXXZ   10004ac0 f   KrakenClassifyWorkerFactory.obj
 0001:00003b40       ??__EtaskLog@U2@@YAXXZ     10004b40 f   KrakenClassifyWorkerFactory.obj
 0001:00003bc0       ??__EuiLog@U2@@YAXXZ       10004bc0 f   KrakenClassifyWorkerFactory.obj
 0001:00003c40       ??__EuserActLog@U2@@YAXXZ  10004c40 f   KrakenClassifyWorkerFactory.obj
 0001:00003cc0       ??__E?BUILD_TOOL@KrakenSupport@U2@@2VQString@@B@@YAXXZ 10004cc0 f   KrakenSupport.obj
 0001:00003ce0       ??__E?BUILD_TOOL_ID@KrakenSupport@U2@@2VQString@@B@@YAXXZ 10004ce0 f   KrakenSupport.obj
 0001:00003d00       ??__E?CLASSIFY_TOOL@KrakenSupport@U2@@2VQString@@B@@YAXXZ 10004d00 f   KrakenSupport.obj
 0001:00003d20       ??__E?CLASSIFY_TOOL_ID@KrakenSupport@U2@@2VQString@@B@@YAXXZ 10004d20 f   KrakenSupport.obj
 0001:00003d40       ??__E?GROUP_NAME@KrakenSupport@U2@@2VQString@@B@@YAXXZ 10004d40 f   KrakenSupport.obj
 0001:00003d60       ??__E?_Generic_object@?$_Error_objects@H@std@@2V_Generic_error_category@2@A@@YAXXZ 10004d60 f   KrakenSupport.obj
 0001:00003d70       ??__E?_Iostream_object@?$_Error_objects@H@std@@2V_Iostream_error_category@2@A@@YAXXZ 10004d70 f   KrakenSupport.obj
 0001:00003d80       ??__E?_System_object@?$_Error_objects@H@std@@2V_System_error_category@2@A@@YAXXZ 10004d80 f   KrakenSupport.obj
 0001:00003d90       ??__E?PLUGIN_DESCRIPRION@KrakenSupportPlugin@U2@@2VQString@@B@@YAXXZ 10004d90 f   KrakenSupportPlugin.obj
 0001:00003dc0       ??__E?PLUGIN_NAME@KrakenSupportPlugin@U2@@2VQString@@B@@YAXXZ 10004dc0 f   KrakenSupportPlugin.obj
 0001:00003df0       ??__E?_Generic_object@?$_Error_objects@H@std@@2V_Generic_error_category@2@A@@YAXXZ 10004df0 f   KrakenSupportPlugin.obj
 0001:00003e00       ??__E?_Iostream_object@?$_Error_objects@H@std@@2V_Iostream_error_category@2@A@@YAXXZ 10004e00 f   KrakenSupportPlugin.obj
 0001:00003e10       ??__E?_System_object@?$_Error_objects@H@std@@2V_System_error_category@2@A@@YAXXZ 10004e10 f   KrakenSupportPlugin.obj
 0001:00003e20       ??__EalgoLog@U2@@YAXXZ     10004e20 f   KrakenSupportPlugin.obj
 0001:00003ea0       ??__EcmdLog@U2@@YAXXZ      10004ea0 f   KrakenSupportPlugin.obj
 0001:00003f20       ??__EcoreLog@U2@@YAXXZ     10004f20 f   KrakenSupportPlugin.obj
 0001:00003fb0       ??__EioLog@U2@@YAXXZ       10004fb0 f   KrakenSupportPlugin.obj
 0001:00004030       ??__EperfLog@U2@@YAXXZ     10005030 f   KrakenSupportPlugin.obj
 0001:000040b0       ??__EscriptLog@U2@@YAXXZ   100050b0 f   KrakenSupportPlugin.obj
 0001:00004130       ??__EtaskLog@U2@@YAXXZ     10005130 f   KrakenSupportPlugin.obj
 0001:000041b0       ??__EuiLog@U2@@YAXXZ       100051b0 f   KrakenSupportPlugin.obj
 0001:00004230       ??__EuserActLog@U2@@YAXXZ  10005230 f   KrakenSupportPlugin.obj
 0001:000042b0       ??__E?_Generic_object@?$_Error_objects@H@std@@2V_Generic_error_category@2@A@@YAXXZ 100052b0 f   KrakenTranslateLogParser.obj
 0001:000042c0       ??__E?_Iostream_object@?$_Error_objects@H@std@@2V_Iostream_error_category@2@A@@YAXXZ 100052c0 f   KrakenTranslateLogParser.obj
 0001:000042d0       ??__E?_System_object@?$_Error_objects@H@std@@2V_System_error_category@2@A@@YAXXZ 100052d0 f   KrakenTranslateLogParser.obj
 0001:000042e0       ??__E?wellKnownErrors@KrakenTranslateLogParser@U2@@0VQStringList@@B@@YAXXZ 100052e0 f   KrakenTranslateLogParser.obj
 0001:00004300       ??__EalgoLog@U2@@YAXXZ     10005300 f   KrakenTranslateLogParser.obj
 0001:00004380       ??__EcmdLog@U2@@YAXXZ      10005380 f   KrakenTranslateLogParser.obj
 0001:00004400       ??__EcoreLog@U2@@YAXXZ     10005400 f   KrakenTranslateLogParser.obj
 0001:00004480       ??__EioLog@U2@@YAXXZ       10005480 f   KrakenTranslateLogParser.obj
 0001:00004500       ??__EperfLog@U2@@YAXXZ     10005500 f   KrakenTranslateLogParser.obj
 0001:00004580       ??__EscriptLog@U2@@YAXXZ   10005580 f   KrakenTranslateLogParser.obj
 0001:00004600       ??__EtaskLog@U2@@YAXXZ     10005600 f   KrakenTranslateLogParser.obj
 0001:00004680       ??__EuiLog@U2@@YAXXZ       10005680 f   KrakenTranslateLogParser.obj
 0001:00004700       ??__EuserActLog@U2@@YAXXZ  10005700 f   KrakenTranslateLogParser.obj
 0001:00004780       ??__E?_Generic_object@?$_Error_objects@H@std@@2V_Generic_error_category@2@A@@YAXXZ 10005780 f   moc_KrakenBuildPrompter.obj
 0001:00004790       ??__E?_Iostream_object@?$_Error_objects@H@std@@2V_Iostream_error_category@2@A@@YAXXZ 10005790 f   moc_KrakenBuildPrompter.obj
 0001:000047a0       ??__E?_System_object@?$_Error_objects@H@std@@2V_System_error_category@2@A@@YAXXZ 100057a0 f   moc_KrakenBuildPrompter.obj
 0001:000047b0       ??__E?staticMetaObject@KrakenBuildPrompter@LocalWorkflow@U2@@2UQMetaObject@@B@@YAXXZ 100057b0 f   moc_KrakenBuildPrompter.obj
 0001:000047c0       ??__EalgoLog@U2@@YAXXZ     100057c0 f   moc_KrakenBuildPrompter.obj
 0001:00004840       ??__EcmdLog@U2@@YAXXZ      10005840 f   moc_KrakenBuildPrompter.obj
 0001:000048c0       ??__EcoreLog@U2@@YAXXZ     100058c0 f   moc_KrakenBuildPrompter.obj
 0001:00004940       ??__EioLog@U2@@YAXXZ       10005940 f   moc_KrakenBuildPrompter.obj
 0001:000049c0       ??__EperfLog@U2@@YAXXZ     100059c0 f   moc_KrakenBuildPrompter.obj
 0001:00004a40       ??__EscriptLog@U2@@YAXXZ   10005a40 f   moc_KrakenBuildPrompter.obj
 0001:00004ac0       ??__EtaskLog@U2@@YAXXZ     10005ac0 f   moc_KrakenBuildPrompter.obj
 0001:00004b40       ??__EuiLog@U2@@YAXXZ       10005b40 f   moc_KrakenBuildPrompter.obj
 0001:00004bc0       ??__EuserActLog@U2@@YAXXZ  10005bc0 f   moc_KrakenBuildPrompter.obj
 0001:00004c40       ??__E?_Generic_object@?$_Error_objects@H@std@@2V_Generic_error_category@2@A@@YAXXZ 10005c40 f   moc_KrakenBuildTask.obj
 0001:00004c50       ??__E?_Iostream_object@?$_Error_objects@H@std@@2V_Iostream_error_category@2@A@@YAXXZ 10005c50 f   moc_KrakenBuildTask.obj
 0001:00004c60       ??__E?_System_object@?$_Error_objects@H@std@@2V_System_error_category@2@A@@YAXXZ 10005c60 f   moc_KrakenBuildTask.obj
 0001:00004c70       ??__E?staticMetaObject@KrakenBuildTask@U2@@2UQMetaObject@@B@@YAXXZ 10005c70 f   moc_KrakenBuildTask.obj
 0001:00004c80       ??__EalgoLog@U2@@YAXXZ     10005c80 f   moc_KrakenBuildTask.obj
 0001:00004d00       ??__EcmdLog@U2@@YAXXZ      10005d00 f   moc_KrakenBuildTask.obj
 0001:00004d80       ??__EcoreLog@U2@@YAXXZ     10005d80 f   moc_KrakenBuildTask.obj
 0001:00004e00       ??__EioLog@U2@@YAXXZ       10005e00 f   moc_KrakenBuildTask.obj
 0001:00004e80       ??__EperfLog@U2@@YAXXZ     10005e80 f   moc_KrakenBuildTask.obj
 0001:00004f00       ??__EscriptLog@U2@@YAXXZ   10005f00 f   moc_KrakenBuildTask.obj
 0001:00004f80       ??__EtaskLog@U2@@YAXXZ     10005f80 f   moc_KrakenBuildTask.obj
 0001:00005000       ??__EuiLog@U2@@YAXXZ       10006000 f   moc_KrakenBuildTask.obj
 0001:00005080       ??__EuserActLog@U2@@YAXXZ  10006080 f   moc_KrakenBuildTask.obj
 0001:00005100       ??__E?_Generic_object@?$_Error_objects@H@std@@2V_Generic_error_category@2@A@@YAXXZ 10006100 f   moc_KrakenBuildWorker.obj
 0001:00005110       ??__E?_Iostream_object@?$_Error_objects@H@std@@2V_Iostream_error_category@2@A@@YAXXZ 10006110 f   moc_KrakenBuildWorker.obj
 0001:00005120       ??__E?_System_object@?$_Error_objects@H@std@@2V_System_error_category@2@A@@YAXXZ 10006120 f   moc_KrakenBuildWorker.obj
 0001:00005130       ??__E?staticMetaObject@KrakenBuildWorker@LocalWorkflow@U2@@2UQMetaObject@@B@@YAXXZ 10006130 f   moc_KrakenBuildWorker.obj
 0001:00005140       ??__EalgoLog@U2@@YAXXZ     10006140 f   moc_KrakenBuildWorker.obj
 0001:000051c0       ??__EcmdLog@U2@@YAXXZ      100061c0 f   moc_KrakenBuildWorker.obj
 0001:00005240       ??__EcoreLog@U2@@YAXXZ     10006240 f   moc_KrakenBuildWorker.obj
 0001:000052c0       ??__EioLog@U2@@YAXXZ       100062c0 f   moc_KrakenBuildWorker.obj
 0001:00005340       ??__EperfLog@U2@@YAXXZ     10006340 f   moc_KrakenBuildWorker.obj
 0001:000053c0       ??__EscriptLog@U2@@YAXXZ   100063c0 f   moc_KrakenBuildWorker.obj
 0001:00005440       ??__EtaskLog@U2@@YAXXZ     10006440 f   moc_KrakenBuildWorker.obj
 0001:000054c0       ??__EuiLog@U2@@YAXXZ       100064c0 f   moc_KrakenBuildWorker.obj
 0001:00005540       ??__EuserActLog@U2@@YAXXZ  10006540 f   moc_KrakenBuildWorker.obj
 0001:000055c0       ??__E?_Generic_object@?$_Error_objects@H@std@@2V_Generic_error_category@2@A@@YAXXZ 100065c0 f   moc_KrakenClassifyPrompter.obj
 0001:000055d0       ??__E?_Iostream_object@?$_Error_objects@H@std@@2V_Iostream_error_category@2@A@@YAXXZ 100065d0 f   moc_KrakenClassifyPrompter.obj
 0001:000055e0       ??__E?_System_object@?$_Error_objects@H@std@@2V_System_error_category@2@A@@YAXXZ 100065e0 f   moc_KrakenClassifyPrompter.obj
 0001:000055f0       ??__E?staticMetaObject@KrakenClassifyPrompter@LocalWorkflow@U2@@2UQMetaObject@@B@@YAXXZ 100065f0 f   moc_KrakenClassifyPrompter.obj
 0001:00005600       ??__EalgoLog@U2@@YAXXZ     10006600 f   moc_KrakenClassifyPrompter.obj
 0001:00005680       ??__EcmdLog@U2@@YAXXZ      10006680 f   moc_KrakenClassifyPrompter.obj
 0001:00005700       ??__EcoreLog@U2@@YAXXZ     10006700 f   moc_KrakenClassifyPrompter.obj
 0001:00005780       ??__EioLog@U2@@YAXXZ       10006780 f   moc_KrakenClassifyPrompter.obj
 0001:00005800       ??__EperfLog@U2@@YAXXZ     10006800 f   moc_KrakenClassifyPrompter.obj
 0001:00005880       ??__EscriptLog@U2@@YAXXZ   10006880 f   moc_KrakenClassifyPrompter.obj
 0001:00005900       ??__EtaskLog@U2@@YAXXZ     10006900 f   moc_KrakenClassifyPrompter.obj
 0001:00005980       ??__EuiLog@U2@@YAXXZ       10006980 f   moc_KrakenClassifyPrompter.obj
 0001:00005a00       ??__EuserActLog@U2@@YAXXZ  10006a00 f   moc_KrakenClassifyPrompter.obj
 0001:00005a80       ??__E?_Generic_object@?$_Error_objects@H@std@@2V_Generic_error_category@2@A@@YAXXZ 10006a80 f   moc_KrakenClassifyTask.obj
 0001:00005a90       ??__E?_Iostream_object@?$_Error_objects@H@std@@2V_Iostream_error_category@2@A@@YAXXZ 10006a90 f   moc_KrakenClassifyTask.obj
 0001:00005aa0       ??__E?_System_object@?$_Error_objects@H@std@@2V_System_error_category@2@A@@YAXXZ 10006aa0 f   moc_KrakenClassifyTask.obj
 0001:00005ab0       ??__E?staticMetaObject@KrakenClassifyTask@U2@@2UQMetaObject@@B@@YAXXZ 10006ab0 f   moc_KrakenClassifyTask.obj
 0001:00005ac0       ??__EalgoLog@U2@@YAXXZ     10006ac0 f   moc_KrakenClassifyTask.obj
 0001:00005b40       ??__EcmdLog@U2@@YAXXZ      10006b40 f   moc_KrakenClassifyTask.obj
 0001:00005bc0       ??__EcoreLog@U2@@YAXXZ     10006bc0 f   moc_KrakenClassifyTask.obj
 0001:00005c40       ??__EioLog@U2@@YAXXZ       10006c40 f   moc_KrakenClassifyTask.obj
 0001:00005cc0       ??__EperfLog@U2@@YAXXZ     10006cc0 f   moc_KrakenClassifyTask.obj
 0001:00005d40       ??__EscriptLog@U2@@YAXXZ   10006d40 f   moc_KrakenClassifyTask.obj
 0001:00005dc0       ??__EtaskLog@U2@@YAXXZ     10006dc0 f   moc_KrakenClassifyTask.obj
 0001:00005e40       ??__EuiLog@U2@@YAXXZ       10006e40 f   moc_KrakenClassifyTask.obj
 0001:00005ec0       ??__EuserActLog@U2@@YAXXZ  10006ec0 f   moc_KrakenClassifyTask.obj
 0001:00005f40       ??__E?_Generic_object@?$_Error_objects@H@std@@2V_Generic_error_category@2@A@@YAXXZ 10006f40 f   moc_KrakenClassifyWorker.obj
 0001:00005f50       ??__E?_Iostream_object@?$_Error_objects@H@std@@2V_Iostream_error_category@2@A@@YAXXZ 10006f50 f   moc_KrakenClassifyWorker.obj
 0001:00005f60       ??__E?_System_object@?$_Error_objects@H@std@@2V_System_error_category@2@A@@YAXXZ 10006f60 f   moc_KrakenClassifyWorker.obj
 0001:00005f70       ??__E?staticMetaObject@KrakenClassifyWorker@LocalWorkflow@U2@@2UQMetaObject@@B@@YAXXZ 10006f70 f   moc_KrakenClassifyWorker.obj
 0001:00005f80       ??__EalgoLog@U2@@YAXXZ     10006f80 f   moc_KrakenClassifyWorker.obj
 0001:00006000       ??__EcmdLog@U2@@YAXXZ      10007000 f   moc_KrakenClassifyWorker.obj
 0001:00006080       ??__EcoreLog@U2@@YAXXZ     10007080 f   moc_KrakenClassifyWorker.obj
 0001:00006100       ??__EioLog@U2@@YAXXZ       10007100 f   moc_KrakenClassifyWorker.obj
 0001:00006180       ??__EperfLog@U2@@YAXXZ     10007180 f   moc_KrakenClassifyWorker.obj
 0001:00006200       ??__EscriptLog@U2@@YAXXZ   10007200 f   moc_KrakenClassifyWorker.obj
 0001:00006280       ??__EtaskLog@U2@@YAXXZ     10007280 f   moc_KrakenClassifyWorker.obj
 0001:00006300       ??__EuiLog@U2@@YAXXZ       10007300 f   moc_KrakenClassifyWorker.obj
 0001:00006380       ??__EuserActLog@U2@@YAXXZ  10007380 f   moc_KrakenClassifyWorker.obj
 0001:00006400       ??__E?_Generic_object@?$_Error_objects@H@std@@2V_Generic_error_category@2@A@@YAXXZ 10007400 f   moc_KrakenSupport.obj
 0001:00006410       ??__E?_Iostream_object@?$_Error_objects@H@std@@2V_Iostream_error_category@2@A@@YAXXZ 10007410 f   moc_KrakenSupport.obj
 0001:00006420       ??__E?_System_object@?$_Error_objects@H@std@@2V_System_error_category@2@A@@YAXXZ 10007420 f   moc_KrakenSupport.obj
 0001:00006430       ??__E?staticMetaObject@KrakenSupport@U2@@2UQMetaObject@@B@@YAXXZ 10007430 f   moc_KrakenSupport.obj
 0001:00006440       ??__E?_Generic_object@?$_Error_objects@H@std@@2V_Generic_error_category@2@A@@YAXXZ 10007440 f   moc_KrakenSupportPlugin.obj
 0001:00006450       ??__E?_Iostream_object@?$_Error_objects@H@std@@2V_Iostream_error_category@2@A@@YAXXZ 10007450 f   moc_KrakenSupportPlugin.obj
 0001:00006460       ??__E?_System_object@?$_Error_objects@H@std@@2V_System_error_category@2@A@@YAXXZ 10007460 f   moc_KrakenSupportPlugin.obj
 0001:00006470       ??__E?staticMetaObject@KrakenSupportPlugin@U2@@2UQMetaObject@@B@@YAXXZ 10007470 f   moc_KrakenSupportPlugin.obj
 0001:00006b56       __catch$?_Copy@?$basic_string@DU?$char_traits@D@std@@V?$allocator@D@2@@std@@QAEXII@Z$0 10007b56 f i DatabaseSizeRelation.obj
 0001:00006b93       __catch$?_Copy@?$basic_string@DU?$char_traits@D@std@@V?$allocator@D@2@@std@@QAEXII@Z$1 10007b93 f i DatabaseSizeRelation.obj
 0001:000078fe       __catch$??0?$QList@PAVPort@Workflow@U2@@@@QAE@ABV0@@Z$0 100088fe f i KrakenBuildPrompter.obj
 0001:0000832e       __catch$??0?$QList@PAVTask@U2@@@@QAE@ABV0@@Z$0 1000932e f i KrakenBuildTask.obj
 0001:000083fe       __catch$??0?$QList@VQString@@@@QAE@ABV0@@Z$0 100093fe f i KrakenBuildTask.obj
 0001:00008c9f       __catch$??Y?$QList@PAVTask@U2@@@@QAEAAV0@ABV0@@Z$0 10009c9f f i KrakenBuildTask.obj
 0001:00008ec5       __catch$?append@?$QList@PAVTask@U2@@@@QAEXABQAVTask@U2@@@Z$4 10009ec5 f i KrakenBuildTask.obj
 0001:00008f4d       __catch$?append@?$QList@VQString@@@@QAEXABVQString@@@Z$0 10009f4d f i KrakenBuildTask.obj
 0001:00008f9e       __catch$?append@?$QList@VQString@@@@QAEXABVQString@@@Z$4 10009f9e f i KrakenBuildTask.obj
 0001:000096c1       __catch$?detach_helper_grow@?$QList@PAVTask@U2@@@@AAEPAUNode@1@HH@Z$0 1000a6c1 f i KrakenBuildTask.obj
 0001:000096c1       __catch$?detach_helper_grow@?$QList@PAVTask@U2@@@@AAEPAUNode@1@HH@Z$2 1000a6c1 f i KrakenBuildTask.obj
 0001:000097fe       __catch$?detach_helper_grow@?$QList@VQString@@@@AAEPAUNode@1@HH@Z$2 1000a7fe f i KrakenBuildTask.obj
 0001:00009839       __catch$?detach_helper_grow@?$QList@VQString@@@@AAEPAUNode@1@HH@Z$0 1000a839 f i KrakenBuildTask.obj
 0001:0000a1b2       __catch$?node_copy@?$QList@VQString@@@@AAEXPAUNode@1@00@Z$2 1000b1b2 f i KrakenBuildTask.obj
 0001:0000b310       __catch$?append@?$QList@VWorkflowNotification@U2@@@@QAEXABVWorkflowNotification@U2@@@Z$0 1000c310 f i KrakenBuildValidator.obj
 0001:0000b310       __catch$?append@?$QList@VWorkflowNotification@U2@@@@QAEXABVWorkflowNotification@U2@@@Z$2 1000c310 f i KrakenBuildValidator.obj
 0001:0000b49f       __catch$?detach_helper_grow@?$QList@VWorkflowNotification@U2@@@@AAEPAUNode@1@HH@Z$2 1000c49f f i KrakenBuildValidator.obj
 0001:0000b4da       __catch$?detach_helper_grow@?$QList@VWorkflowNotification@U2@@@@AAEPAUNode@1@HH@Z$0 1000c4da f i KrakenBuildValidator.obj
 0001:0000b67e       __catch$?node_copy@?$QList@VWorkflowNotification@U2@@@@AAEXPAUNode@1@00@Z$0 1000c67e f i KrakenBuildValidator.obj
 0001:0000ca2e       __catch$??0?$QList@PAVURLContainer@U2@@@@QAE@ABV0@@Z$0 1000da2e f i KrakenBuildWorker.obj
 0001:0000cb0e       __catch$??0?$QList@VDataset@U2@@@@QAE@ABV0@@Z$0 1000db0e f i KrakenBuildWorker.obj
 0001:0000cbfe       __catch$??0?$QList@VDescriptor@U2@@@@QAE@ABV0@@Z$0 1000dbfe f i KrakenBuildWorker.obj
 0001:0000d4ac       __catch$?append@?$QList@VDescriptor@U2@@@@QAEXABVDescriptor@U2@@@Z$0 1000e4ac f i KrakenBuildWorker.obj
 0001:0000d4ac       __catch$?append@?$QList@VDescriptor@U2@@@@QAEXABVDescriptor@U2@@@Z$2 1000e4ac f i KrakenBuildWorker.obj
 0001:0000d75e       __catch$?createNode@?$QMapData@VQString@@VQScriptValue@@@@QAEPAU?$QMapNode@VQString@@VQScriptValue@@@@ABVQString@@ABVQScriptValue@@PAU2@_N@Z$0 1000e75e f i KrakenBuildWorker.obj
 0001:0000d773       __catch$?createNode@?$QMapData@VQString@@VQScriptValue@@@@QAEPAU?$QMapNode@VQString@@VQScriptValue@@@@ABVQString@@ABVQScriptValue@@PAU2@_N@Z$2 1000e773 f i KrakenBuildWorker.obj
 0001:0000d81e       __catch$?createNode@?$QMapData@VQString@@VQVariant@@@@QAEPAU?$QMapNode@VQString@@VQVariant@@@@ABVQString@@ABVQVariant@@PAU2@_N@Z$0 1000e81e f i KrakenBuildWorker.obj
 0001:0000d833       __catch$?createNode@?$QMapData@VQString@@VQVariant@@@@QAEPAU?$QMapNode@VQString@@VQVariant@@@@ABVQString@@ABVQVariant@@PAU2@_N@Z$2 1000e833 f i KrakenBuildWorker.obj
 0001:0000da9a       __catch$?detach_helper@?$QList@VDescriptor@U2@@@@AAEXH@Z$0 1000ea9a f i KrakenBuildWorker.obj
 0001:0000dcaf       __catch$?detach_helper_grow@?$QList@VDescriptor@U2@@@@AAEPAUNode@1@HH@Z$2 1000ecaf f i KrakenBuildWorker.obj
 0001:0000dcea       __catch$?detach_helper_grow@?$QList@VDescriptor@U2@@@@AAEPAUNode@1@HH@Z$0 1000ecea f i KrakenBuildWorker.obj
 0001:0000eb4e       __catch$?node_copy@?$QList@VDataset@U2@@@@AAEXPAUNode@1@00@Z$0 1000fb4e f i KrakenBuildWorker.obj
 0001:0000ec25       __catch$?node_copy@?$QList@VDescriptor@U2@@@@AAEXPAUNode@1@00@Z$0 1000fc25 f i KrakenBuildWorker.obj
 0001:0000fd25       __catch$?append@?$QList@PAVAttribute@U2@@@@QAEXABQAVAttribute@U2@@@Z$4 10010d25 f i KrakenBuildWorkerFactory.obj
 0001:0000fdb5       __catch$?append@?$QList@PAVPortDescriptor@Workflow@U2@@@@QAEXABQAVPortDescriptor@Workflow@U2@@@Z$4 10010db5 f i KrakenBuildWorkerFactory.obj
 0001:0000ffed       __catch$?createNode@?$QMapData@VDescriptor@U2@@V?$QExplicitlySharedDataPointer@VDataType@U2@@@@@@QAEPAU?$QMapNode@VDescriptor@U2@@V?$QExplicitlySharedDataPointer@VDataType@U2@@@@@@ABVDescriptor@U2@@ABV?$QExplicitlySharedDataPointer@VDataType@U2@@@@PAU2@_N@Z$2 10010fed f i KrakenBuildWorkerFactory.obj
 0001:00010095       __catch$?createNode@?$QMapData@VQString@@PAVPropertyDelegate@U2@@@@QAEPAU?$QMapNode@VQString@@PAVPropertyDelegate@U2@@@@ABVQString@@ABQAVPropertyDelegate@U2@@PAU2@_N@Z$2 10011095 f i KrakenBuildWorkerFactory.obj
 0001:000104c1       __catch$?detach_helper_grow@?$QList@PAVAttribute@U2@@@@AAEPAUNode@1@HH@Z$2 100114c1 f i KrakenBuildWorkerFactory.obj
 0001:000104c1       __catch$?detach_helper_grow@?$QList@PAVAttribute@U2@@@@AAEPAUNode@1@HH@Z$0 100114c1 f i KrakenBuildWorkerFactory.obj
 0001:000105d1       __catch$?detach_helper_grow@?$QList@PAVPortDescriptor@Workflow@U2@@@@AAEPAUNode@1@HH@Z$0 100115d1 f i KrakenBuildWorkerFactory.obj
 0001:000105d1       __catch$?detach_helper_grow@?$QList@PAVPortDescriptor@Workflow@U2@@@@AAEPAUNode@1@HH@Z$2 100115d1 f i KrakenBuildWorkerFactory.obj
 0001:00014045       __catch$?createNode@?$QMapData@VQString@@I@@QAEPAU?$QMapNode@VQString@@I@@ABVQString@@ABIPAU2@_N@Z$2 10015045 f i KrakenClassifyTask.obj
 0001:00014231       __catch$?detach_helper@?$QList@VQByteArray@@@@AAEXH@Z$0 10015231 f i KrakenClassifyTask.obj
 0001:00014792       __catch$?node_copy@?$QList@VQByteArray@@@@AAEXPAUNode@1@00@Z$2 10015792 f i KrakenClassifyTask.obj
 0001:00017790       __catch$?append@?$QList@VQVariant@@@@QAEXABVQVariant@@@Z$2 10018790 f i KrakenClassifyWorkerFactory.obj
 0001:00017790       __catch$?append@?$QList@VQVariant@@@@QAEXABVQVariant@@@Z$0 10018790 f i KrakenClassifyWorkerFactory.obj
 0001:000179df       __catch$?detach_helper_grow@?$QList@VQVariant@@@@AAEPAUNode@1@HH@Z$2 100189df f i KrakenClassifyWorkerFactory.obj
 0001:00017a1a       __catch$?detach_helper_grow@?$QList@VQVariant@@@@AAEPAUNode@1@HH@Z$0 10018a1a f i KrakenClassifyWorkerFactory.obj
 0001:0001924e       __catch$?node_copy@?$QList@VQVariant@@@@AAEXPAUNode@1@00@Z$0 1001a24e f i KrakenClassifyWorkerFactory.obj
 0001:0001b340       _pre_c_init                1001c340 f   MSVCRT:crtdll.obj
 0001:0001b5ad       ___DllMainCRTStartup       1001c5ad f   MSVCRT:crtdll.obj
 0001:0001b700       $$000000                   1001c700     MSVCRT:sehprolg4.obj
 0001:0001bb15       ?ArrayUnwindFilter@@YAHPAU_EXCEPTION_POINTERS@@@Z 1001cb15 f   MSVCRT:ehvecdtr.obj
 0001:0001be60       __unwindfunclet$??0DatabaseSizeRelation@LocalWorkflow@U2@@QAE@ABVQString@@@Z$0 1001ce60 f   DatabaseSizeRelation.obj
 0001:0001be68       __unwindfunclet$??0DatabaseSizeRelation@LocalWorkflow@U2@@QAE@ABVQString@@@Z$1 1001ce68 f   DatabaseSizeRelation.obj
 0001:0001be71       __ehhandler$??0DatabaseSizeRelation@LocalWorkflow@U2@@QAE@ABVQString@@@Z 1001ce71 f   DatabaseSizeRelation.obj
 0001:0001be90       __unwindfunclet$??H@YA?BVQString@@ABV0@PBD@Z$0 1001ce90 f   DatabaseSizeRelation.obj
 0001:0001beaa       __unwindfunclet$??H@YA?BVQString@@ABV0@PBD@Z$1 1001ceaa f   DatabaseSizeRelation.obj
 0001:0001beb3       __ehhandler$??H@YA?BVQString@@ABV0@PBD@Z 1001ceb3 f   DatabaseSizeRelation.obj
 0001:0001bed0       __unwindfunclet$??__EalgoLog@U2@@YAXXZ$0 1001ced0 f   DatabaseSizeRelation.obj
 0001:0001bed9       __ehhandler$??__EalgoLog@U2@@YAXXZ 1001ced9 f   DatabaseSizeRelation.obj
 0001:0001bf00       __unwindfunclet$??__EcmdLog@U2@@YAXXZ$0 1001cf00 f   DatabaseSizeRelation.obj
 0001:0001bf09       __ehhandler$??__EcmdLog@U2@@YAXXZ 1001cf09 f   DatabaseSizeRelation.obj
 0001:0001bf30       __unwindfunclet$??__EcoreLog@U2@@YAXXZ$0 1001cf30 f   DatabaseSizeRelation.obj
 0001:0001bf39       __ehhandler$??__EcoreLog@U2@@YAXXZ 1001cf39 f   DatabaseSizeRelation.obj
 0001:0001bf60       __unwindfunclet$??__EioLog@U2@@YAXXZ$0 1001cf60 f   DatabaseSizeRelation.obj
 0001:0001bf69       __ehhandler$??__EioLog@U2@@YAXXZ 1001cf69 f   DatabaseSizeRelation.obj
 0001:0001bf90       __unwindfunclet$??__EperfLog@U2@@YAXXZ$0 1001cf90 f   DatabaseSizeRelation.obj
 0001:0001bf99       __ehhandler$??__EperfLog@U2@@YAXXZ 1001cf99 f   DatabaseSizeRelation.obj
 0001:0001bfc0       __unwindfunclet$??__EscriptLog@U2@@YAXXZ$0 1001cfc0 f   DatabaseSizeRelation.obj
 0001:0001bfc9       __ehhandler$??__EscriptLog@U2@@YAXXZ 1001cfc9 f   DatabaseSizeRelation.obj
 0001:0001bff0       __unwindfunclet$??__EtaskLog@U2@@YAXXZ$0 1001cff0 f   DatabaseSizeRelation.obj
 0001:0001bff9       __ehhandler$??__EtaskLog@U2@@YAXXZ 1001cff9 f   DatabaseSizeRelation.obj
 0001:0001c020       __unwindfunclet$??__EuiLog@U2@@YAXXZ$0 1001d020 f   DatabaseSizeRelation.obj
 0001:0001c029       __ehhandler$??__EuiLog@U2@@YAXXZ 1001d029 f   DatabaseSizeRelation.obj
 0001:0001c050       __unwindfunclet$??__EuserActLog@U2@@YAXXZ$0 1001d050 f   DatabaseSizeRelation.obj
 0001:0001c059       __ehhandler$??__EuserActLog@U2@@YAXXZ 1001d059 f   DatabaseSizeRelation.obj
 0001:0001c080       __ehhandler$?_Copy@?$basic_string@DU?$char_traits@D@std@@V?$allocator@D@2@@std@@QAEXII@Z 1001d080 f   DatabaseSizeRelation.obj
 0001:0001c0a0       __unwindfunclet$?clone@DatabaseSizeRelation@LocalWorkflow@U2@@UBEPAV123@XZ$0 1001d0a0 f   DatabaseSizeRelation.obj
 0001:0001c0ab       __ehhandler$?clone@DatabaseSizeRelation@LocalWorkflow@U2@@UBEPAV123@XZ 1001d0ab f   DatabaseSizeRelation.obj
 0001:0001c0d0       __unwindfunclet$?getAffectResult@DatabaseSizeRelation@LocalWorkflow@U2@@UBE?AVQVariant@@ABV4@0PAVDelegateTags@3@1@Z$0 1001d0d0 f   DatabaseSizeRelation.obj
 0001:0001c0d9       __unwindfunclet$?getAffectResult@DatabaseSizeRelation@LocalWorkflow@U2@@UBE?AVQVariant@@ABV4@0PAVDelegateTags@3@1@Z$1 1001d0d9 f   DatabaseSizeRelation.obj
 0001:0001c0f3       __unwindfunclet$?getAffectResult@DatabaseSizeRelation@LocalWorkflow@U2@@UBE?AVQVariant@@ABV4@0PAVDelegateTags@3@1@Z$2 1001d0f3 f   DatabaseSizeRelation.obj
 0001:0001c0fc       __unwindfunclet$?getAffectResult@DatabaseSizeRelation@LocalWorkflow@U2@@UBE?AVQVariant@@ABV4@0PAVDelegateTags@3@1@Z$3 1001d0fc f   DatabaseSizeRelation.obj
 0001:0001c105       __ehhandler$?getAffectResult@DatabaseSizeRelation@LocalWorkflow@U2@@UBE?AVQVariant@@ABV4@0PAVDelegateTags@3@1@Z 1001d105 f   DatabaseSizeRelation.obj
 0001:0001c120       __ehhandler$??0?$QList@PAVPort@Workflow@U2@@@@QAE@ABV0@@Z 1001d120 f   KrakenBuildPrompter.obj
 0001:0001c140       __unwindfunclet$??__EalgoLog@U2@@YAXXZ$0 1001d140 f   KrakenBuildPrompter.obj
 0001:0001c149       __ehhandler$??__EalgoLog@U2@@YAXXZ 1001d149 f   KrakenBuildPrompter.obj
 0001:0001c170       __unwindfunclet$??__EcmdLog@U2@@YAXXZ$0 1001d170 f   KrakenBuildPrompter.obj
 0001:0001c179       __ehhandler$??__EcmdLog@U2@@YAXXZ 1001d179 f   KrakenBuildPrompter.obj
 0001:0001c1a0       __unwindfunclet$??__EcoreLog@U2@@YAXXZ$0 1001d1a0 f   KrakenBuildPrompter.obj
 0001:0001c1a9       __ehhandler$??__EcoreLog@U2@@YAXXZ 1001d1a9 f   KrakenBuildPrompter.obj
 0001:0001c1d0       __unwindfunclet$??__EioLog@U2@@YAXXZ$0 1001d1d0 f   KrakenBuildPrompter.obj
 0001:0001c1d9       __ehhandler$??__EioLog@U2@@YAXXZ 1001d1d9 f   KrakenBuildPrompter.obj
 0001:0001c200       __unwindfunclet$??__EperfLog@U2@@YAXXZ$0 1001d200 f   KrakenBuildPrompter.obj
 0001:0001c209       __ehhandler$??__EperfLog@U2@@YAXXZ 1001d209 f   KrakenBuildPrompter.obj
 0001:0001c230       __unwindfunclet$??__EscriptLog@U2@@YAXXZ$0 1001d230 f   KrakenBuildPrompter.obj
 0001:0001c239       __ehhandler$??__EscriptLog@U2@@YAXXZ 1001d239 f   KrakenBuildPrompter.obj
 0001:0001c260       __unwindfunclet$??__EtaskLog@U2@@YAXXZ$0 1001d260 f   KrakenBuildPrompter.obj
 0001:0001c269       __ehhandler$??__EtaskLog@U2@@YAXXZ 1001d269 f   KrakenBuildPrompter.obj
 0001:0001c290       __unwindfunclet$??__EuiLog@U2@@YAXXZ$0 1001d290 f   KrakenBuildPrompter.obj
 0001:0001c299       __ehhandler$??__EuiLog@U2@@YAXXZ 1001d299 f   KrakenBuildPrompter.obj
 0001:0001c2c0       __unwindfunclet$??__EuserActLog@U2@@YAXXZ$0 1001d2c0 f   KrakenBuildPrompter.obj
 0001:0001c2c9       __ehhandler$??__EuserActLog@U2@@YAXXZ 1001d2c9 f   KrakenBuildPrompter.obj
 0001:0001c2f0       __unwindfunclet$?composeRichDoc@KrakenBuildPrompter@LocalWorkflow@U2@@EAE?AVQString@@XZ$0 1001d2f0 f   KrakenBuildPrompter.obj
 0001:0001c2f9       __unwindfunclet$?composeRichDoc@KrakenBuildPrompter@LocalWorkflow@U2@@EAE?AVQString@@XZ$1 1001d2f9 f   KrakenBuildPrompter.obj
 0001:0001c302       __unwindfunclet$?composeRichDoc@KrakenBuildPrompter@LocalWorkflow@U2@@EAE?AVQString@@XZ$2 1001d302 f   KrakenBuildPrompter.obj
 0001:0001c30b       __unwindfunclet$?composeRichDoc@KrakenBuildPrompter@LocalWorkflow@U2@@EAE?AVQString@@XZ$3 1001d30b f   KrakenBuildPrompter.obj
 0001:0001c314       __unwindfunclet$?composeRichDoc@KrakenBuildPrompter@LocalWorkflow@U2@@EAE?AVQString@@XZ$4 1001d314 f   KrakenBuildPrompter.obj
 0001:0001c31d       __unwindfunclet$?composeRichDoc@KrakenBuildPrompter@LocalWorkflow@U2@@EAE?AVQString@@XZ$5 1001d31d f   KrakenBuildPrompter.obj
 0001:0001c326       __unwindfunclet$?composeRichDoc@KrakenBuildPrompter@LocalWorkflow@U2@@EAE?AVQString@@XZ$6 1001d326 f   KrakenBuildPrompter.obj
 0001:0001c32f       __unwindfunclet$?composeRichDoc@KrakenBuildPrompter@LocalWorkflow@U2@@EAE?AVQString@@XZ$7 1001d32f f   KrakenBuildPrompter.obj
 0001:0001c349       __unwindfunclet$?composeRichDoc@KrakenBuildPrompter@LocalWorkflow@U2@@EAE?AVQString@@XZ$8 1001d349 f   KrakenBuildPrompter.obj
 0001:0001c352       __unwindfunclet$?composeRichDoc@KrakenBuildPrompter@LocalWorkflow@U2@@EAE?AVQString@@XZ$9 1001d352 f   KrakenBuildPrompter.obj
 0001:0001c35b       __unwindfunclet$?composeRichDoc@KrakenBuildPrompter@LocalWorkflow@U2@@EAE?AVQString@@XZ$10 1001d35b f   KrakenBuildPrompter.obj
 0001:0001c364       __unwindfunclet$?composeRichDoc@KrakenBuildPrompter@LocalWorkflow@U2@@EAE?AVQString@@XZ$11 1001d364 f   KrakenBuildPrompter.obj
 0001:0001c36d       __unwindfunclet$?composeRichDoc@KrakenBuildPrompter@LocalWorkflow@U2@@EAE?AVQString@@XZ$12 1001d36d f   KrakenBuildPrompter.obj
 0001:0001c376       __unwindfunclet$?composeRichDoc@KrakenBuildPrompter@LocalWorkflow@U2@@EAE?AVQString@@XZ$13 1001d376 f   KrakenBuildPrompter.obj
 0001:0001c37f       __unwindfunclet$?composeRichDoc@KrakenBuildPrompter@LocalWorkflow@U2@@EAE?AVQString@@XZ$14 1001d37f f   KrakenBuildPrompter.obj
 0001:0001c388       __unwindfunclet$?composeRichDoc@KrakenBuildPrompter@LocalWorkflow@U2@@EAE?AVQString@@XZ$15 1001d388 f   KrakenBuildPrompter.obj
 0001:0001c391       __unwindfunclet$?composeRichDoc@KrakenBuildPrompter@LocalWorkflow@U2@@EAE?AVQString@@XZ$16 1001d391 f   KrakenBuildPrompter.obj
 0001:0001c39a       __unwindfunclet$?composeRichDoc@KrakenBuildPrompter@LocalWorkflow@U2@@EAE?AVQString@@XZ$17 1001d39a f   KrakenBuildPrompter.obj
 0001:0001c3a3       __ehhandler$?composeRichDoc@KrakenBuildPrompter@LocalWorkflow@U2@@EAE?AVQString@@XZ 1001d3a3 f   KrakenBuildPrompter.obj
 0001:0001c3c0       __unwindfunclet$?createDescription@?$PrompterBase@VKrakenBuildPrompter@LocalWorkflow@U2@@@U2@@UAEPAVActorDocument@Workflow@2@PAVActor@42@@Z$0 1001d3c0 f   KrakenBuildPrompter.obj
 0001:0001c3cb       __unwindfunclet$?createDescription@?$PrompterBase@VKrakenBuildPrompter@LocalWorkflow@U2@@@U2@@UAEPAVActorDocument@Workflow@2@PAVActor@42@@Z$3 1001d3cb f   KrakenBuildPrompter.obj
 0001:0001c3d3       __unwindfunclet$?createDescription@?$PrompterBase@VKrakenBuildPrompter@LocalWorkflow@U2@@@U2@@UAEPAVActorDocument@Workflow@2@PAVActor@42@@Z$4 1001d3d3 f   KrakenBuildPrompter.obj
 0001:0001c3db       __unwindfunclet$?createDescription@?$PrompterBase@VKrakenBuildPrompter@LocalWorkflow@U2@@@U2@@UAEPAVActorDocument@Workflow@2@PAVActor@42@@Z$6 1001d3db f   KrakenBuildPrompter.obj
 0001:0001c3e3       __unwindfunclet$?createDescription@?$PrompterBase@VKrakenBuildPrompter@LocalWorkflow@U2@@@U2@@UAEPAVActorDocument@Workflow@2@PAVActor@42@@Z$7 1001d3e3 f   KrakenBuildPrompter.obj
 0001:0001c3eb       __ehhandler$?createDescription@?$PrompterBase@VKrakenBuildPrompter@LocalWorkflow@U2@@@U2@@UAEPAVActorDocument@Workflow@2@PAVActor@42@@Z 1001d3eb f   KrakenBuildPrompter.obj
 0001:0001c410       __ehhandler$??0?$QList@PAVTask@U2@@@@QAE@ABV0@@Z 1001d410 f   KrakenBuildTask.obj
 0001:0001c430       __ehhandler$??0?$QList@VQString@@@@QAE@ABV0@@Z 1001d430 f   KrakenBuildTask.obj
 0001:0001c450       __unwindfunclet$??0KrakenBuildTask@U2@@QAE@ABUKrakenBuildTaskSettings@1@@Z$0 1001d450 f   KrakenBuildTask.obj
 0001:0001c459       __unwindfunclet$??0KrakenBuildTask@U2@@QAE@ABUKrakenBuildTaskSettings@1@@Z$1 1001d459 f   KrakenBuildTask.obj
 0001:0001c462       __unwindfunclet$??0KrakenBuildTask@U2@@QAE@ABUKrakenBuildTaskSettings@1@@Z$2 1001d462 f   KrakenBuildTask.obj
 0001:0001c470       __unwindfunclet$??0KrakenBuildTask@U2@@QAE@ABUKrakenBuildTaskSettings@1@@Z$3 1001d470 f   KrakenBuildTask.obj
 0001:0001c47e       __unwindfunclet$??0KrakenBuildTask@U2@@QAE@ABUKrakenBuildTaskSettings@1@@Z$4 1001d47e f   KrakenBuildTask.obj
 0001:0001c487       __unwindfunclet$??0KrakenBuildTask@U2@@QAE@ABUKrakenBuildTaskSettings@1@@Z$5 1001d487 f   KrakenBuildTask.obj
 0001:0001c490       __unwindfunclet$??0KrakenBuildTask@U2@@QAE@ABUKrakenBuildTaskSettings@1@@Z$6 1001d490 f   KrakenBuildTask.obj
 0001:0001c499       __unwindfunclet$??0KrakenBuildTask@U2@@QAE@ABUKrakenBuildTaskSettings@1@@Z$7 1001d499 f   KrakenBuildTask.obj
 0001:0001c4b3       __unwindfunclet$??0KrakenBuildTask@U2@@QAE@ABUKrakenBuildTaskSettings@1@@Z$8 1001d4b3 f   KrakenBuildTask.obj
 0001:0001c4cd       __unwindfunclet$??0KrakenBuildTask@U2@@QAE@ABUKrakenBuildTaskSettings@1@@Z$9 1001d4cd f   KrakenBuildTask.obj
 0001:0001c4d6       __unwindfunclet$??0KrakenBuildTask@U2@@QAE@ABUKrakenBuildTaskSettings@1@@Z$10 1001d4d6 f   KrakenBuildTask.obj
 0001:0001c4df       __ehhandler$??0KrakenBuildTask@U2@@QAE@ABUKrakenBuildTaskSettings@1@@Z 1001d4df f   KrakenBuildTask.obj
 0001:0001c500       __unwindfunclet$??0KrakenBuildTaskSettings@U2@@QAE@ABU01@@Z$0 1001d500 f   KrakenBuildTask.obj
 0001:0001c509       __unwindfunclet$??0KrakenBuildTaskSettings@U2@@QAE@ABU01@@Z$1 1001d509 f   KrakenBuildTask.obj
 0001:0001c515       __unwindfunclet$??0KrakenBuildTaskSettings@U2@@QAE@ABU01@@Z$2 1001d515 f   KrakenBuildTask.obj
 0001:0001c521       __ehhandler$??0KrakenBuildTaskSettings@U2@@QAE@ABU01@@Z 1001d521 f   KrakenBuildTask.obj
 0001:0001c540       __unwindfunclet$??0KrakenBuildTaskSettings@U2@@QAE@XZ$0 1001d540 f   KrakenBuildTask.obj
 0001:0001c549       __unwindfunclet$??0KrakenBuildTaskSettings@U2@@QAE@XZ$1 1001d549 f   KrakenBuildTask.obj
 0001:0001c555       __ehhandler$??0KrakenBuildTaskSettings@U2@@QAE@XZ 1001d555 f   KrakenBuildTask.obj
 0001:0001c570       __unwindfunclet$??1KrakenBuildTask@U2@@UAE@XZ$0 1001d570 f   KrakenBuildTask.obj
 0001:0001c579       __unwindfunclet$??1KrakenBuildTask@U2@@UAE@XZ$2 1001d579 f   KrakenBuildTask.obj
 0001:0001c582       __unwindfunclet$??1KrakenBuildTask@U2@@UAE@XZ$3 1001d582 f   KrakenBuildTask.obj
 0001:0001c58e       __unwindfunclet$??1KrakenBuildTask@U2@@UAE@XZ$4 1001d58e f   KrakenBuildTask.obj
 0001:0001c59a       __ehhandler$??1KrakenBuildTask@U2@@UAE@XZ 1001d59a f   KrakenBuildTask.obj
 0001:0001c5c0       __unwindfunclet$??1KrakenBuildTaskSettings@U2@@QAE@XZ$0 1001d5c0 f   KrakenBuildTask.obj
 0001:0001c5c9       __unwindfunclet$??1KrakenBuildTaskSettings@U2@@QAE@XZ$1 1001d5c9 f   KrakenBuildTask.obj
 0001:0001c5d5       __unwindfunclet$??1KrakenBuildTaskSettings@U2@@QAE@XZ$2 1001d5d5 f   KrakenBuildTask.obj
 0001:0001c5e1       __ehhandler$??1KrakenBuildTaskSettings@U2@@QAE@XZ 1001d5e1 f   KrakenBuildTask.obj
 0001:0001c600       __unwindfunclet$??H@YA?BVQString@@ABV0@0@Z$0 1001d600 f   KrakenBuildTask.obj
 0001:0001c61a       __ehhandler$??H@YA?BVQString@@ABV0@0@Z 1001d61a f   KrakenBuildTask.obj
 0001:0001c640       __ehhandler$??Y?$QList@PAVTask@U2@@@@QAEAAV0@ABV0@@Z 1001d640 f   KrakenBuildTask.obj
 0001:0001c660       __unwindfunclet$??_GKrakenBuildTask@U2@@UAEPAXI@Z$0 1001d660 f   KrakenBuildTask.obj
 0001:0001c669       __unwindfunclet$??_GKrakenBuildTask@U2@@UAEPAXI@Z$2 1001d669 f   KrakenBuildTask.obj
 0001:0001c672       __unwindfunclet$??_GKrakenBuildTask@U2@@UAEPAXI@Z$3 1001d672 f   KrakenBuildTask.obj
 0001:0001c67e       __unwindfunclet$??_GKrakenBuildTask@U2@@UAEPAXI@Z$4 1001d67e f   KrakenBuildTask.obj
 0001:0001c68a       __ehhandler$??_GKrakenBuildTask@U2@@UAEPAXI@Z 1001d68a f   KrakenBuildTask.obj
 0001:0001c6b0       __unwindfunclet$??__EalgoLog@U2@@YAXXZ$0 1001d6b0 f   KrakenBuildTask.obj
 0001:0001c6b9       __ehhandler$??__EalgoLog@U2@@YAXXZ 1001d6b9 f   KrakenBuildTask.obj
 0001:0001c6e0       __unwindfunclet$??__EcmdLog@U2@@YAXXZ$0 1001d6e0 f   KrakenBuildTask.obj
 0001:0001c6e9       __ehhandler$??__EcmdLog@U2@@YAXXZ 1001d6e9 f   KrakenBuildTask.obj
 0001:0001c710       __unwindfunclet$??__EcoreLog@U2@@YAXXZ$0 1001d710 f   KrakenBuildTask.obj
 0001:0001c719       __ehhandler$??__EcoreLog@U2@@YAXXZ 1001d719 f   KrakenBuildTask.obj
 0001:0001c740       __unwindfunclet$??__EioLog@U2@@YAXXZ$0 1001d740 f   KrakenBuildTask.obj
 0001:0001c749       __ehhandler$??__EioLog@U2@@YAXXZ 1001d749 f   KrakenBuildTask.obj
 0001:0001c770       __unwindfunclet$??__EperfLog@U2@@YAXXZ$0 1001d770 f   KrakenBuildTask.obj
 0001:0001c779       __ehhandler$??__EperfLog@U2@@YAXXZ 1001d779 f   KrakenBuildTask.obj
 0001:0001c7a0       __unwindfunclet$??__EscriptLog@U2@@YAXXZ$0 1001d7a0 f   KrakenBuildTask.obj
 0001:0001c7a9       __ehhandler$??__EscriptLog@U2@@YAXXZ 1001d7a9 f   KrakenBuildTask.obj
 0001:0001c7d0       __unwindfunclet$??__EtaskLog@U2@@YAXXZ$0 1001d7d0 f   KrakenBuildTask.obj
 0001:0001c7d9       __ehhandler$??__EtaskLog@U2@@YAXXZ 1001d7d9 f   KrakenBuildTask.obj
 0001:0001c800       __unwindfunclet$??__EuiLog@U2@@YAXXZ$0 1001d800 f   KrakenBuildTask.obj
 0001:0001c809       __ehhandler$??__EuiLog@U2@@YAXXZ 1001d809 f   KrakenBuildTask.obj
 0001:0001c830       __unwindfunclet$??__EuserActLog@U2@@YAXXZ$0 1001d830 f   KrakenBuildTask.obj
 0001:0001c839       __ehhandler$??__EuserActLog@U2@@YAXXZ 1001d839 f   KrakenBuildTask.obj
 0001:0001c860       __ehhandler$?append@?$QList@PAVTask@U2@@@@QAEXABQAVTask@U2@@@Z 1001d860 f   KrakenBuildTask.obj
 0001:0001c880       __unwindfunclet$?append@?$QList@VQString@@@@QAEXABVQString@@@Z$7 1001d880 f   KrakenBuildTask.obj
 0001:0001c891       __unwindfunclet$?append@?$QList@VQString@@@@QAEXABVQString@@@Z$11 1001d891 f   KrakenBuildTask.obj
 0001:0001c8a2       __ehhandler$?append@?$QList@VQString@@@@QAEXABVQString@@@Z 1001d8a2 f   KrakenBuildTask.obj
 0001:0001c8c0       __unwindfunclet$?checkSettings@KrakenBuildTask@U2@@AAEXXZ$0 1001d8c0 f   KrakenBuildTask.obj
 0001:0001c8c9       __unwindfunclet$?checkSettings@KrakenBuildTask@U2@@AAEXXZ$1 1001d8c9 f   KrakenBuildTask.obj
 0001:0001c8d2       __unwindfunclet$?checkSettings@KrakenBuildTask@U2@@AAEXXZ$2 1001d8d2 f   KrakenBuildTask.obj
 0001:0001c8ec       __unwindfunclet$?checkSettings@KrakenBuildTask@U2@@AAEXXZ$3 1001d8ec f   KrakenBuildTask.obj
 0001:0001c8f5       __unwindfunclet$?checkSettings@KrakenBuildTask@U2@@AAEXXZ$4 1001d8f5 f   KrakenBuildTask.obj
 0001:0001c8fe       __unwindfunclet$?checkSettings@KrakenBuildTask@U2@@AAEXXZ$5 1001d8fe f   KrakenBuildTask.obj
 0001:0001c907       __unwindfunclet$?checkSettings@KrakenBuildTask@U2@@AAEXXZ$6 1001d907 f   KrakenBuildTask.obj
 0001:0001c910       __unwindfunclet$?checkSettings@KrakenBuildTask@U2@@AAEXXZ$11 1001d910 f   KrakenBuildTask.obj
 0001:0001c919       __unwindfunclet$?checkSettings@KrakenBuildTask@U2@@AAEXXZ$12 1001d919 f   KrakenBuildTask.obj
 0001:0001c922       __unwindfunclet$?checkSettings@KrakenBuildTask@U2@@AAEXXZ$13 1001d922 f   KrakenBuildTask.obj
 0001:0001c92b       __unwindfunclet$?checkSettings@KrakenBuildTask@U2@@AAEXXZ$14 1001d92b f   KrakenBuildTask.obj
 0001:0001c934       __unwindfunclet$?checkSettings@KrakenBuildTask@U2@@AAEXXZ$15 1001d934 f   KrakenBuildTask.obj
 0001:0001c93d       __unwindfunclet$?checkSettings@KrakenBuildTask@U2@@AAEXXZ$16 1001d93d f   KrakenBuildTask.obj
 0001:0001c946       __unwindfunclet$?checkSettings@KrakenBuildTask@U2@@AAEXXZ$17 1001d946 f   KrakenBuildTask.obj
 0001:0001c94f       __unwindfunclet$?checkSettings@KrakenBuildTask@U2@@AAEXXZ$18 1001d94f f   KrakenBuildTask.obj
 0001:0001c958       __unwindfunclet$?checkSettings@KrakenBuildTask@U2@@AAEXXZ$19 1001d958 f   KrakenBuildTask.obj
 0001:0001c961       __unwindfunclet$?checkSettings@KrakenBuildTask@U2@@AAEXXZ$9 1001d961 f   KrakenBuildTask.obj
 0001:0001c96a       __unwindfunclet$?checkSettings@KrakenBuildTask@U2@@AAEXXZ$10 1001d96a f   KrakenBuildTask.obj
 0001:0001c973       __unwindfunclet$?checkSettings@KrakenBuildTask@U2@@AAEXXZ$7 1001d973 f   KrakenBuildTask.obj
 0001:0001c97c       __unwindfunclet$?checkSettings@KrakenBuildTask@U2@@AAEXXZ$8 1001d97c f   KrakenBuildTask.obj
 0001:0001c985       __ehhandler$?checkSettings@KrakenBuildTask@U2@@AAEXXZ 1001d985 f   KrakenBuildTask.obj
 0001:0001c9a0       __unwindfunclet$?checkTaxonomy@KrakenBuildTask@U2@@AAEXXZ$0 1001d9a0 f   KrakenBuildTask.obj
 0001:0001c9a9       __ehhandler$?checkTaxonomy@KrakenBuildTask@U2@@AAEXXZ 1001d9a9 f   KrakenBuildTask.obj
 0001:0001c9d0       __ehhandler$?detach_helper_grow@?$QList@PAVTask@U2@@@@AAEPAUNode@1@HH@Z 1001d9d0 f   KrakenBuildTask.obj
 0001:0001c9f0       __ehhandler$?detach_helper_grow@?$QList@VQString@@@@AAEPAUNode@1@HH@Z 1001d9f0 f   KrakenBuildTask.obj
 0001:0001ca10       __unwindfunclet$?getAddToLibraryArguments@KrakenBuildTask@U2@@ABE?AVQStringList@@ABVQString@@@Z$0 1001da10 f   KrakenBuildTask.obj
 0001:0001ca29       __unwindfunclet$?getAddToLibraryArguments@KrakenBuildTask@U2@@ABE?AVQStringList@@ABVQString@@@Z$1 1001da29 f   KrakenBuildTask.obj
 0001:0001ca32       __unwindfunclet$?getAddToLibraryArguments@KrakenBuildTask@U2@@ABE?AVQStringList@@ABVQString@@@Z$2 1001da32 f   KrakenBuildTask.obj
 0001:0001ca3b       __ehhandler$?getAddToLibraryArguments@KrakenBuildTask@U2@@ABE?AVQStringList@@ABVQString@@@Z 1001da3b f   KrakenBuildTask.obj
 0001:0001ca60       __unwindfunclet$?getBuildArguments@KrakenBuildTask@U2@@ABE?AVQStringList@@XZ$0 1001da60 f   KrakenBuildTask.obj
 0001:0001ca79       __unwindfunclet$?getBuildArguments@KrakenBuildTask@U2@@ABE?AVQStringList@@XZ$1 1001da79 f   KrakenBuildTask.obj
 0001:0001ca82       __unwindfunclet$?getBuildArguments@KrakenBuildTask@U2@@ABE?AVQStringList@@XZ$2 1001da82 f   KrakenBuildTask.obj
 0001:0001ca8b       __unwindfunclet$?getBuildArguments@KrakenBuildTask@U2@@ABE?AVQStringList@@XZ$3 1001da8b f   KrakenBuildTask.obj
 0001:0001ca94       __unwindfunclet$?getBuildArguments@KrakenBuildTask@U2@@ABE?AVQStringList@@XZ$4 1001da94 f   KrakenBuildTask.obj
 0001:0001ca9d       __unwindfunclet$?getBuildArguments@KrakenBuildTask@U2@@ABE?AVQStringList@@XZ$5 1001da9d f   KrakenBuildTask.obj
 0001:0001caa6       __unwindfunclet$?getBuildArguments@KrakenBuildTask@U2@@ABE?AVQStringList@@XZ$6 1001daa6 f   KrakenBuildTask.obj
 0001:0001caaf       __unwindfunclet$?getBuildArguments@KrakenBuildTask@U2@@ABE?AVQStringList@@XZ$7 1001daaf f   KrakenBuildTask.obj
 0001:0001cab8       __unwindfunclet$?getBuildArguments@KrakenBuildTask@U2@@ABE?AVQStringList@@XZ$8 1001dab8 f   KrakenBuildTask.obj
 0001:0001cac1       __unwindfunclet$?getBuildArguments@KrakenBuildTask@U2@@ABE?AVQStringList@@XZ$9 1001dac1 f   KrakenBuildTask.obj
 0001:0001caca       __unwindfunclet$?getBuildArguments@KrakenBuildTask@U2@@ABE?AVQStringList@@XZ$10 1001daca f   KrakenBuildTask.obj
 0001:0001cad3       __unwindfunclet$?getBuildArguments@KrakenBuildTask@U2@@ABE?AVQStringList@@XZ$11 1001dad3 f   KrakenBuildTask.obj
 0001:0001cadc       __unwindfunclet$?getBuildArguments@KrakenBuildTask@U2@@ABE?AVQStringList@@XZ$12 1001dadc f   KrakenBuildTask.obj
 0001:0001cae5       __unwindfunclet$?getBuildArguments@KrakenBuildTask@U2@@ABE?AVQStringList@@XZ$13 1001dae5 f   KrakenBuildTask.obj
 0001:0001caee       __ehhandler$?getBuildArguments@KrakenBuildTask@U2@@ABE?AVQStringList@@XZ 1001daee f   KrakenBuildTask.obj
 0001:0001cb10       __unwindfunclet$?getCleanArguments@KrakenBuildTask@U2@@ABE?AVQStringList@@XZ$0 1001db10 f   KrakenBuildTask.obj
 0001:0001cb29       __unwindfunclet$?getCleanArguments@KrakenBuildTask@U2@@ABE?AVQStringList@@XZ$1 1001db29 f   KrakenBuildTask.obj
 0001:0001cb32       __unwindfunclet$?getCleanArguments@KrakenBuildTask@U2@@ABE?AVQStringList@@XZ$2 1001db32 f   KrakenBuildTask.obj
 0001:0001cb3b       __ehhandler$?getCleanArguments@KrakenBuildTask@U2@@ABE?AVQStringList@@XZ 1001db3b f   KrakenBuildTask.obj
 0001:0001cb60       __unwindfunclet$?getShrinkArguments@KrakenBuildTask@U2@@ABE?AVQStringList@@XZ$0 1001db60 f   KrakenBuildTask.obj
 0001:0001cb79       __unwindfunclet$?getShrinkArguments@KrakenBuildTask@U2@@ABE?AVQStringList@@XZ$1 1001db79 f   KrakenBuildTask.obj
 0001:0001cb82       __unwindfunclet$?getShrinkArguments@KrakenBuildTask@U2@@ABE?AVQStringList@@XZ$2 1001db82 f   KrakenBuildTask.obj
 0001:0001cb8b       __unwindfunclet$?getShrinkArguments@KrakenBuildTask@U2@@ABE?AVQStringList@@XZ$3 1001db8b f   KrakenBuildTask.obj
 0001:0001cb94       __unwindfunclet$?getShrinkArguments@KrakenBuildTask@U2@@ABE?AVQStringList@@XZ$4 1001db94 f   KrakenBuildTask.obj
 0001:0001cb9d       __unwindfunclet$?getShrinkArguments@KrakenBuildTask@U2@@ABE?AVQStringList@@XZ$5 1001db9d f   KrakenBuildTask.obj
 0001:0001cba6       __unwindfunclet$?getShrinkArguments@KrakenBuildTask@U2@@ABE?AVQStringList@@XZ$6 1001dba6 f   KrakenBuildTask.obj
 0001:0001cbaf       __unwindfunclet$?getShrinkArguments@KrakenBuildTask@U2@@ABE?AVQStringList@@XZ$7 1001dbaf f   KrakenBuildTask.obj
 0001:0001cbb8       __unwindfunclet$?getShrinkArguments@KrakenBuildTask@U2@@ABE?AVQStringList@@XZ$8 1001dbb8 f   KrakenBuildTask.obj
 0001:0001cbc1       __unwindfunclet$?getShrinkArguments@KrakenBuildTask@U2@@ABE?AVQStringList@@XZ$9 1001dbc1 f   KrakenBuildTask.obj
 0001:0001cbca       __unwindfunclet$?getShrinkArguments@KrakenBuildTask@U2@@ABE?AVQStringList@@XZ$10 1001dbca f   KrakenBuildTask.obj
 0001:0001cbd3       __unwindfunclet$?getShrinkArguments@KrakenBuildTask@U2@@ABE?AVQStringList@@XZ$11 1001dbd3 f   KrakenBuildTask.obj
 0001:0001cbdc       __unwindfunclet$?getShrinkArguments@KrakenBuildTask@U2@@ABE?AVQStringList@@XZ$12 1001dbdc f   KrakenBuildTask.obj
 0001:0001cbe5       __unwindfunclet$?getShrinkArguments@KrakenBuildTask@U2@@ABE?AVQStringList@@XZ$13 1001dbe5 f   KrakenBuildTask.obj
 0001:0001cbee       __ehhandler$?getShrinkArguments@KrakenBuildTask@U2@@ABE?AVQStringList@@XZ 1001dbee f   KrakenBuildTask.obj
 0001:0001cc10       __unwindfunclet$?node_construct@?$QList@VQString@@@@AAEXPAUNode@1@ABVQString@@@Z$1 1001dc10 f   KrakenBuildTask.obj
 0001:0001cc21       __ehhandler$?node_construct@?$QList@VQString@@@@AAEXPAUNode@1@ABVQString@@@Z 1001dc21 f   KrakenBuildTask.obj
 0001:0001cc40       __unwindfunclet$?node_copy@?$QList@VQString@@@@AAEXPAUNode@1@00@Z$5 1001dc40 f   KrakenBuildTask.obj
 0001:0001cc51       __ehhandler$?node_copy@?$QList@VQString@@@@AAEXPAUNode@1@00@Z 1001dc51 f   KrakenBuildTask.obj
 0001:0001cc70       __unwindfunclet$?prepare@KrakenBuildTask@U2@@EAEXXZ$0 1001dc70 f   KrakenBuildTask.obj
 0001:0001cc78       __unwindfunclet$?prepare@KrakenBuildTask@U2@@EAEXXZ$1 1001dc78 f   KrakenBuildTask.obj
 0001:0001cc80       __unwindfunclet$?prepare@KrakenBuildTask@U2@@EAEXXZ$2 1001dc80 f   KrakenBuildTask.obj
 0001:0001cc88       __unwindfunclet$?prepare@KrakenBuildTask@U2@@EAEXXZ$3 1001dc88 f   KrakenBuildTask.obj
 0001:0001cc93       __unwindfunclet$?prepare@KrakenBuildTask@U2@@EAEXXZ$4 1001dc93 f   KrakenBuildTask.obj
 0001:0001ccad       __unwindfunclet$?prepare@KrakenBuildTask@U2@@EAEXXZ$5 1001dcad f   KrakenBuildTask.obj
 0001:0001ccb8       __unwindfunclet$?prepare@KrakenBuildTask@U2@@EAEXXZ$6 1001dcb8 f   KrakenBuildTask.obj
 0001:0001ccd2       __unwindfunclet$?prepare@KrakenBuildTask@U2@@EAEXXZ$7 1001dcd2 f   KrakenBuildTask.obj
 0001:0001cceb       __unwindfunclet$?prepare@KrakenBuildTask@U2@@EAEXXZ$8 1001dceb f   KrakenBuildTask.obj
 0001:0001cd04       __unwindfunclet$?prepare@KrakenBuildTask@U2@@EAEXXZ$9 1001dd04 f   KrakenBuildTask.obj
 0001:0001cd0f       __unwindfunclet$?prepare@KrakenBuildTask@U2@@EAEXXZ$10 1001dd0f f   KrakenBuildTask.obj
 0001:0001cd29       __unwindfunclet$?prepare@KrakenBuildTask@U2@@EAEXXZ$11 1001dd29 f   KrakenBuildTask.obj
 0001:0001cd34       __unwindfunclet$?prepare@KrakenBuildTask@U2@@EAEXXZ$12 1001dd34 f   KrakenBuildTask.obj
 0001:0001cd4e       __unwindfunclet$?prepare@KrakenBuildTask@U2@@EAEXXZ$13 1001dd4e f   KrakenBuildTask.obj
 0001:0001cd67       __unwindfunclet$?prepare@KrakenBuildTask@U2@@EAEXXZ$14 1001dd67 f   KrakenBuildTask.obj
 0001:0001cd85       __unwindfunclet$?prepare@KrakenBuildTask@U2@@EAEXXZ$15 1001dd85 f   KrakenBuildTask.obj
 0001:0001cd90       __unwindfunclet$?prepare@KrakenBuildTask@U2@@EAEXXZ$16 1001dd90 f   KrakenBuildTask.obj
 0001:0001cdaf       __unwindfunclet$?prepare@KrakenBuildTask@U2@@EAEXXZ$17 1001ddaf f   KrakenBuildTask.obj
 0001:0001cdba       __unwindfunclet$?prepare@KrakenBuildTask@U2@@EAEXXZ$18 1001ddba f   KrakenBuildTask.obj
 0001:0001cdd9       __unwindfunclet$?prepare@KrakenBuildTask@U2@@EAEXXZ$19 1001ddd9 f   KrakenBuildTask.obj
 0001:0001cdf7       __unwindfunclet$?prepare@KrakenBuildTask@U2@@EAEXXZ$20 1001ddf7 f   KrakenBuildTask.obj
 0001:0001ce15       __unwindfunclet$?prepare@KrakenBuildTask@U2@@EAEXXZ$21 1001de15 f   KrakenBuildTask.obj
 0001:0001ce20       __unwindfunclet$?prepare@KrakenBuildTask@U2@@EAEXXZ$22 1001de20 f   KrakenBuildTask.obj
 0001:0001ce3f       __unwindfunclet$?prepare@KrakenBuildTask@U2@@EAEXXZ$23 1001de3f f   KrakenBuildTask.obj
 0001:0001ce4a       __unwindfunclet$?prepare@KrakenBuildTask@U2@@EAEXXZ$24 1001de4a f   KrakenBuildTask.obj
 0001:0001ce69       __unwindfunclet$?prepare@KrakenBuildTask@U2@@EAEXXZ$25 1001de69 f   KrakenBuildTask.obj
 0001:0001ce87       __unwindfunclet$?prepare@KrakenBuildTask@U2@@EAEXXZ$26 1001de87 f   KrakenBuildTask.obj
 0001:0001cea5       __unwindfunclet$?prepare@KrakenBuildTask@U2@@EAEXXZ$33 1001dea5 f   KrakenBuildTask.obj
 0001:0001ceb0       __unwindfunclet$?prepare@KrakenBuildTask@U2@@EAEXXZ$34 1001deb0 f   KrakenBuildTask.obj
 0001:0001cecf       __unwindfunclet$?prepare@KrakenBuildTask@U2@@EAEXXZ$27 1001decf f   KrakenBuildTask.obj
 0001:0001ced8       __unwindfunclet$?prepare@KrakenBuildTask@U2@@EAEXXZ$28 1001ded8 f   KrakenBuildTask.obj
 0001:0001cee1       __unwindfunclet$?prepare@KrakenBuildTask@U2@@EAEXXZ$29 1001dee1 f   KrakenBuildTask.obj
 0001:0001ceea       __unwindfunclet$?prepare@KrakenBuildTask@U2@@EAEXXZ$30 1001deea f   KrakenBuildTask.obj
 0001:0001cef3       __unwindfunclet$?prepare@KrakenBuildTask@U2@@EAEXXZ$31 1001def3 f   KrakenBuildTask.obj
 0001:0001cefc       __unwindfunclet$?prepare@KrakenBuildTask@U2@@EAEXXZ$32 1001defc f   KrakenBuildTask.obj
 0001:0001cf05       __ehhandler$?prepare@KrakenBuildTask@U2@@EAEXXZ 1001df05 f   KrakenBuildTask.obj
 0001:0001cf20       __unwindfunclet$?prepareTaxonomyData@KrakenBuildTask@U2@@AAE?AV?$QList@PAVTask@U2@@@@XZ$0 1001df20 f   KrakenBuildTask.obj
 0001:0001cf2e       __unwindfunclet$?prepareTaxonomyData@KrakenBuildTask@U2@@AAE?AV?$QList@PAVTask@U2@@@@XZ$1 1001df2e f   KrakenBuildTask.obj
 0001:0001cf36       __unwindfunclet$?prepareTaxonomyData@KrakenBuildTask@U2@@AAE?AV?$QList@PAVTask@U2@@@@XZ$2 1001df36 f   KrakenBuildTask.obj
 0001:0001cf3e       __unwindfunclet$?prepareTaxonomyData@KrakenBuildTask@U2@@AAE?AV?$QList@PAVTask@U2@@@@XZ$3 1001df3e f   KrakenBuildTask.obj
 0001:0001cf47       __unwindfunclet$?prepareTaxonomyData@KrakenBuildTask@U2@@AAE?AV?$QList@PAVTask@U2@@@@XZ$5 1001df47 f   KrakenBuildTask.obj
 0001:0001cf60       __unwindfunclet$?prepareTaxonomyData@KrakenBuildTask@U2@@AAE?AV?$QList@PAVTask@U2@@@@XZ$7 1001df60 f   KrakenBuildTask.obj
 0001:0001cf69       __unwindfunclet$?prepareTaxonomyData@KrakenBuildTask@U2@@AAE?AV?$QList@PAVTask@U2@@@@XZ$8 1001df69 f   KrakenBuildTask.obj
 0001:0001cf72       __unwindfunclet$?prepareTaxonomyData@KrakenBuildTask@U2@@AAE?AV?$QList@PAVTask@U2@@@@XZ$9 1001df72 f   KrakenBuildTask.obj
 0001:0001cf7a       __unwindfunclet$?prepareTaxonomyData@KrakenBuildTask@U2@@AAE?AV?$QList@PAVTask@U2@@@@XZ$10 1001df7a f   KrakenBuildTask.obj
 0001:0001cf82       __unwindfunclet$?prepareTaxonomyData@KrakenBuildTask@U2@@AAE?AV?$QList@PAVTask@U2@@@@XZ$11 1001df82 f   KrakenBuildTask.obj
 0001:0001cf8b       __unwindfunclet$?prepareTaxonomyData@KrakenBuildTask@U2@@AAE?AV?$QList@PAVTask@U2@@@@XZ$12 1001df8b f   KrakenBuildTask.obj
 0001:0001cf94       __unwindfunclet$?prepareTaxonomyData@KrakenBuildTask@U2@@AAE?AV?$QList@PAVTask@U2@@@@XZ$13 1001df94 f   KrakenBuildTask.obj
 0001:0001cf9d       __unwindfunclet$?prepareTaxonomyData@KrakenBuildTask@U2@@AAE?AV?$QList@PAVTask@U2@@@@XZ$14 1001df9d f   KrakenBuildTask.obj
 0001:0001cfa6       __unwindfunclet$?prepareTaxonomyData@KrakenBuildTask@U2@@AAE?AV?$QList@PAVTask@U2@@@@XZ$19 1001dfa6 f   KrakenBuildTask.obj
 0001:0001cfb1       __unwindfunclet$?prepareTaxonomyData@KrakenBuildTask@U2@@AAE?AV?$QList@PAVTask@U2@@@@XZ$20 1001dfb1 f   KrakenBuildTask.obj
 0001:0001cfcb       __unwindfunclet$?prepareTaxonomyData@KrakenBuildTask@U2@@AAE?AV?$QList@PAVTask@U2@@@@XZ$21 1001dfcb f   KrakenBuildTask.obj
 0001:0001cfe5       __unwindfunclet$?prepareTaxonomyData@KrakenBuildTask@U2@@AAE?AV?$QList@PAVTask@U2@@@@XZ$22 1001dfe5 f   KrakenBuildTask.obj
 0001:0001cfff       __unwindfunclet$?prepareTaxonomyData@KrakenBuildTask@U2@@AAE?AV?$QList@PAVTask@U2@@@@XZ$23 1001dfff f   KrakenBuildTask.obj
 0001:0001d019       __unwindfunclet$?prepareTaxonomyData@KrakenBuildTask@U2@@AAE?AV?$QList@PAVTask@U2@@@@XZ$15 1001e019 f   KrakenBuildTask.obj
 0001:0001d022       __unwindfunclet$?prepareTaxonomyData@KrakenBuildTask@U2@@AAE?AV?$QList@PAVTask@U2@@@@XZ$16 1001e022 f   KrakenBuildTask.obj
 0001:0001d02b       __unwindfunclet$?prepareTaxonomyData@KrakenBuildTask@U2@@AAE?AV?$QList@PAVTask@U2@@@@XZ$17 1001e02b f   KrakenBuildTask.obj
 0001:0001d034       __unwindfunclet$?prepareTaxonomyData@KrakenBuildTask@U2@@AAE?AV?$QList@PAVTask@U2@@@@XZ$18 1001e034 f   KrakenBuildTask.obj
 0001:0001d03d       __unwindfunclet$?prepareTaxonomyData@KrakenBuildTask@U2@@AAE?AV?$QList@PAVTask@U2@@@@XZ$6 1001e03d f   KrakenBuildTask.obj
 0001:0001d046       __ehhandler$?prepareTaxonomyData@KrakenBuildTask@U2@@AAE?AV?$QList@PAVTask@U2@@@@XZ 1001e046 f   KrakenBuildTask.obj
 0001:0001d070       __unwindfunclet$??__EalgoLog@U2@@YAXXZ$0 1001e070 f   KrakenBuildValidator.obj
 0001:0001d079       __ehhandler$??__EalgoLog@U2@@YAXXZ 1001e079 f   KrakenBuildValidator.obj
 0001:0001d0a0       __unwindfunclet$??__EcmdLog@U2@@YAXXZ$0 1001e0a0 f   KrakenBuildValidator.obj
 0001:0001d0a9       __ehhandler$??__EcmdLog@U2@@YAXXZ 1001e0a9 f   KrakenBuildValidator.obj
 0001:0001d0d0       __unwindfunclet$??__EcoreLog@U2@@YAXXZ$0 1001e0d0 f   KrakenBuildValidator.obj
 0001:0001d0d9       __ehhandler$??__EcoreLog@U2@@YAXXZ 1001e0d9 f   KrakenBuildValidator.obj
 0001:0001d100       __unwindfunclet$??__EioLog@U2@@YAXXZ$0 1001e100 f   KrakenBuildValidator.obj
 0001:0001d109       __ehhandler$??__EioLog@U2@@YAXXZ 1001e109 f   KrakenBuildValidator.obj
 0001:0001d130       __unwindfunclet$??__EperfLog@U2@@YAXXZ$0 1001e130 f   KrakenBuildValidator.obj
 0001:0001d139       __ehhandler$??__EperfLog@U2@@YAXXZ 1001e139 f   KrakenBuildValidator.obj
 0001:0001d160       __unwindfunclet$??__EscriptLog@U2@@YAXXZ$0 1001e160 f   KrakenBuildValidator.obj
 0001:0001d169       __ehhandler$??__EscriptLog@U2@@YAXXZ 1001e169 f   KrakenBuildValidator.obj
 0001:0001d190       __unwindfunclet$??__EtaskLog@U2@@YAXXZ$0 1001e190 f   KrakenBuildValidator.obj
 0001:0001d199       __ehhandler$??__EtaskLog@U2@@YAXXZ 1001e199 f   KrakenBuildValidator.obj
 0001:0001d1c0       __unwindfunclet$??__EuiLog@U2@@YAXXZ$0 1001e1c0 f   KrakenBuildValidator.obj
 0001:0001d1c9       __ehhandler$??__EuiLog@U2@@YAXXZ 1001e1c9 f   KrakenBuildValidator.obj
 0001:0001d1f0       __unwindfunclet$??__EuserActLog@U2@@YAXXZ$0 1001e1f0 f   KrakenBuildValidator.obj
 0001:0001d1f9       __ehhandler$??__EuserActLog@U2@@YAXXZ 1001e1f9 f   KrakenBuildValidator.obj
 0001:0001d220       __unwindfunclet$?append@?$QList@VWorkflowNotification@U2@@@@QAEXABVWorkflowNotification@U2@@@Z$6 1001e220 f   KrakenBuildValidator.obj
 0001:0001d22b       __ehhandler$?append@?$QList@VWorkflowNotification@U2@@@@QAEXABVWorkflowNotification@U2@@@Z 1001e22b f   KrakenBuildValidator.obj
 0001:0001d250       __ehhandler$?detach_helper_grow@?$QList@VWorkflowNotification@U2@@@@AAEPAUNode@1@HH@Z 1001e250 f   KrakenBuildValidator.obj
 0001:0001d270       __unwindfunclet$?node_construct@?$QList@VWorkflowNotification@U2@@@@AAEXPAUNode@1@ABVWorkflowNotification@U2@@@Z$0 1001e270 f   KrakenBuildValidator.obj
 0001:0001d27b       __ehhandler$?node_construct@?$QList@VWorkflowNotification@U2@@@@AAEXPAUNode@1@ABVWorkflowNotification@U2@@@Z 1001e27b f   KrakenBuildValidator.obj
 0001:0001d2a0       __unwindfunclet$?node_copy@?$QList@VWorkflowNotification@U2@@@@AAEXPAUNode@1@00@Z$4 1001e2a0 f   KrakenBuildValidator.obj
 0001:0001d2ab       __ehhandler$?node_copy@?$QList@VWorkflowNotification@U2@@@@AAEXPAUNode@1@00@Z 1001e2ab f   KrakenBuildValidator.obj
 0001:0001d2d0       __unwindfunclet$?validateMinimizerLength@KrakenBuildValidator@Workflow@U2@@ABE_NPBVActor@23@AAV?$QList@VWorkflowNotification@U2@@@@@Z$0 1001e2d0 f   KrakenBuildValidator.obj
 0001:0001d2d9       __unwindfunclet$?validateMinimizerLength@KrakenBuildValidator@Workflow@U2@@ABE_NPBVActor@23@AAV?$QList@VWorkflowNotification@U2@@@@@Z$1 1001e2d9 f   KrakenBuildValidator.obj
 0001:0001d2e2       __unwindfunclet$?validateMinimizerLength@KrakenBuildValidator@Workflow@U2@@ABE_NPBVActor@23@AAV?$QList@VWorkflowNotification@U2@@@@@Z$2 1001e2e2 f   KrakenBuildValidator.obj
 0001:0001d2eb       __ehhandler$?validateMinimizerLength@KrakenBuildValidator@Workflow@U2@@ABE_NPBVActor@23@AAV?$QList@VWorkflowNotification@U2@@@@@Z 1001e2eb f   KrakenBuildValidator.obj
 0001:0001d310       __unwindfunclet$?validateTaxonomy@KrakenBuildValidator@Workflow@U2@@ABE_NPBVActor@23@AAV?$QList@VWorkflowNotification@U2@@@@@Z$3 1001e310 f   KrakenBuildValidator.obj
 0001:0001d319       __unwindfunclet$?validateTaxonomy@KrakenBuildValidator@Workflow@U2@@ABE_NPBVActor@23@AAV?$QList@VWorkflowNotification@U2@@@@@Z$4 1001e319 f   KrakenBuildValidator.obj
 0001:0001d321       __unwindfunclet$?validateTaxonomy@KrakenBuildValidator@Workflow@U2@@ABE_NPBVActor@23@AAV?$QList@VWorkflowNotification@U2@@@@@Z$5 1001e321 f   KrakenBuildValidator.obj
 0001:0001d329       __unwindfunclet$?validateTaxonomy@KrakenBuildValidator@Workflow@U2@@ABE_NPBVActor@23@AAV?$QList@VWorkflowNotification@U2@@@@@Z$6 1001e329 f   KrakenBuildValidator.obj
 0001:0001d331       __unwindfunclet$?validateTaxonomy@KrakenBuildValidator@Workflow@U2@@ABE_NPBVActor@23@AAV?$QList@VWorkflowNotification@U2@@@@@Z$8 1001e331 f   KrakenBuildValidator.obj
 0001:0001d33a       __unwindfunclet$?validateTaxonomy@KrakenBuildValidator@Workflow@U2@@ABE_NPBVActor@23@AAV?$QList@VWorkflowNotification@U2@@@@@Z$9 1001e33a f   KrakenBuildValidator.obj
 0001:0001d343       __unwindfunclet$?validateTaxonomy@KrakenBuildValidator@Workflow@U2@@ABE_NPBVActor@23@AAV?$QList@VWorkflowNotification@U2@@@@@Z$10 1001e343 f   KrakenBuildValidator.obj
 0001:0001d34c       __unwindfunclet$?validateTaxonomy@KrakenBuildValidator@Workflow@U2@@ABE_NPBVActor@23@AAV?$QList@VWorkflowNotification@U2@@@@@Z$0 1001e34c f   KrakenBuildValidator.obj
 0001:0001d355       __unwindfunclet$?validateTaxonomy@KrakenBuildValidator@Workflow@U2@@ABE_NPBVActor@23@AAV?$QList@VWorkflowNotification@U2@@@@@Z$1 1001e355 f   KrakenBuildValidator.obj
 0001:0001d35e       __unwindfunclet$?validateTaxonomy@KrakenBuildValidator@Workflow@U2@@ABE_NPBVActor@23@AAV?$QList@VWorkflowNotification@U2@@@@@Z$2 1001e35e f   KrakenBuildValidator.obj
 0001:0001d367       __ehhandler$?validateTaxonomy@KrakenBuildValidator@Workflow@U2@@ABE_NPBVActor@23@AAV?$QList@VWorkflowNotification@U2@@@@@Z 1001e367 f   KrakenBuildValidator.obj
 0001:0001d390       __unwindfunclet$??$getAttributeValue@H@Attribute@U2@@QBEHPAVWorkflowContext@Workflow@1@@Z$0 1001e390 f   KrakenBuildWorker.obj
 0001:0001d399       __unwindfunclet$??$getAttributeValue@H@Attribute@U2@@QBEHPAVWorkflowContext@Workflow@1@@Z$1 1001e399 f   KrakenBuildWorker.obj
 0001:0001d3a1       __unwindfunclet$??$getAttributeValue@H@Attribute@U2@@QBEHPAVWorkflowContext@Workflow@1@@Z$2 1001e3a1 f   KrakenBuildWorker.obj
 0001:0001d3a9       __unwindfunclet$??$getAttributeValue@H@Attribute@U2@@QBEHPAVWorkflowContext@Workflow@1@@Z$3 1001e3a9 f   KrakenBuildWorker.obj
 0001:0001d3b1       __unwindfunclet$??$getAttributeValue@H@Attribute@U2@@QBEHPAVWorkflowContext@Workflow@1@@Z$4 1001e3b1 f   KrakenBuildWorker.obj
 0001:0001d3ba       __unwindfunclet$??$getAttributeValue@H@Attribute@U2@@QBEHPAVWorkflowContext@Workflow@1@@Z$5 1001e3ba f   KrakenBuildWorker.obj
 0001:0001d3c3       __unwindfunclet$??$getAttributeValue@H@Attribute@U2@@QBEHPAVWorkflowContext@Workflow@1@@Z$6 1001e3c3 f   KrakenBuildWorker.obj
 0001:0001d3cc       __unwindfunclet$??$getAttributeValue@H@Attribute@U2@@QBEHPAVWorkflowContext@Workflow@1@@Z$7 1001e3cc f   KrakenBuildWorker.obj
 0001:0001d3d5       __unwindfunclet$??$getAttributeValue@H@Attribute@U2@@QBEHPAVWorkflowContext@Workflow@1@@Z$8 1001e3d5 f   KrakenBuildWorker.obj
 0001:0001d3de       __unwindfunclet$??$getAttributeValue@H@Attribute@U2@@QBEHPAVWorkflowContext@Workflow@1@@Z$9 1001e3de f   KrakenBuildWorker.obj
 0001:0001d3e7       __unwindfunclet$??$getAttributeValue@H@Attribute@U2@@QBEHPAVWorkflowContext@Workflow@1@@Z$10 1001e3e7 f   KrakenBuildWorker.obj
 0001:0001d3f0       __unwindfunclet$??$getAttributeValue@H@Attribute@U2@@QBEHPAVWorkflowContext@Workflow@1@@Z$11 1001e3f0 f   KrakenBuildWorker.obj
 0001:0001d3f9       __ehhandler$??$getAttributeValue@H@Attribute@U2@@QBEHPAVWorkflowContext@Workflow@1@@Z 1001e3f9 f   KrakenBuildWorker.obj
 0001:0001d420       __unwindfunclet$??$getAttributeValue@VQString@@@Attribute@U2@@QBE?AVQString@@PAVWorkflowContext@Workflow@1@@Z$0 1001e420 f   KrakenBuildWorker.obj
 0001:0001d43a       __unwindfunclet$??$getAttributeValue@VQString@@@Attribute@U2@@QBE?AVQString@@PAVWorkflowContext@Workflow@1@@Z$1 1001e43a f   KrakenBuildWorker.obj
 0001:0001d443       __unwindfunclet$??$getAttributeValue@VQString@@@Attribute@U2@@QBE?AVQString@@PAVWorkflowContext@Workflow@1@@Z$2 1001e443 f   KrakenBuildWorker.obj
 0001:0001d44b       __unwindfunclet$??$getAttributeValue@VQString@@@Attribute@U2@@QBE?AVQString@@PAVWorkflowContext@Workflow@1@@Z$3 1001e44b f   KrakenBuildWorker.obj
 0001:0001d453       __unwindfunclet$??$getAttributeValue@VQString@@@Attribute@U2@@QBE?AVQString@@PAVWorkflowContext@Workflow@1@@Z$4 1001e453 f   KrakenBuildWorker.obj
 0001:0001d45b       __unwindfunclet$??$getAttributeValue@VQString@@@Attribute@U2@@QBE?AVQString@@PAVWorkflowContext@Workflow@1@@Z$5 1001e45b f   KrakenBuildWorker.obj
 0001:0001d464       __unwindfunclet$??$getAttributeValue@VQString@@@Attribute@U2@@QBE?AVQString@@PAVWorkflowContext@Workflow@1@@Z$6 1001e464 f   KrakenBuildWorker.obj
 0001:0001d46d       __unwindfunclet$??$getAttributeValue@VQString@@@Attribute@U2@@QBE?AVQString@@PAVWorkflowContext@Workflow@1@@Z$7 1001e46d f   KrakenBuildWorker.obj
 0001:0001d476       __unwindfunclet$??$getAttributeValue@VQString@@@Attribute@U2@@QBE?AVQString@@PAVWorkflowContext@Workflow@1@@Z$8 1001e476 f   KrakenBuildWorker.obj
 0001:0001d47f       __unwindfunclet$??$getAttributeValue@VQString@@@Attribute@U2@@QBE?AVQString@@PAVWorkflowContext@Workflow@1@@Z$9 1001e47f f   KrakenBuildWorker.obj
 0001:0001d488       __unwindfunclet$??$getAttributeValue@VQString@@@Attribute@U2@@QBE?AVQString@@PAVWorkflowContext@Workflow@1@@Z$10 1001e488 f   KrakenBuildWorker.obj
 0001:0001d491       __unwindfunclet$??$getAttributeValue@VQString@@@Attribute@U2@@QBE?AVQString@@PAVWorkflowContext@Workflow@1@@Z$11 1001e491 f   KrakenBuildWorker.obj
 0001:0001d49a       __unwindfunclet$??$getAttributeValue@VQString@@@Attribute@U2@@QBE?AVQString@@PAVWorkflowContext@Workflow@1@@Z$12 1001e49a f   KrakenBuildWorker.obj
 0001:0001d4a3       __ehhandler$??$getAttributeValue@VQString@@@Attribute@U2@@QBE?AVQString@@PAVWorkflowContext@Workflow@1@@Z 1001e4a3 f   KrakenBuildWorker.obj
 0001:0001d4d0       __unwindfunclet$??$getValue@VQString@@@BaseWorker@LocalWorkflow@U2@@IBE?AVQString@@ABV3@@Z$0 1001e4d0 f   KrakenBuildWorker.obj
 0001:0001d4ea       __unwindfunclet$??$getValue@VQString@@@BaseWorker@LocalWorkflow@U2@@IBE?AVQString@@ABV3@@Z$1 1001e4ea f   KrakenBuildWorker.obj
 0001:0001d4f3       __ehhandler$??$getValue@VQString@@@BaseWorker@LocalWorkflow@U2@@IBE?AVQString@@ABV3@@Z 1001e4f3 f   KrakenBuildWorker.obj
 0001:0001d510       __unwindfunclet$??$qRegisterMetaType@V?$QList@VDataset@U2@@@@@@YAHPBDPAV?$QList@VDataset@U2@@@@W4DefinedType@?$MetaTypeDefinedHelper@V?$QList@VDataset@U2@@@@$00@QtPrivate@@@Z$0 1001e510 f   KrakenBuildWorker.obj
 0001:0001d519       __ehhandler$??$qRegisterMetaType@V?$QList@VDataset@U2@@@@@@YAHPBDPAV?$QList@VDataset@U2@@@@W4DefinedType@?$MetaTypeDefinedHelper@V?$QList@VDataset@U2@@@@$00@QtPrivate@@@Z 1001e519 f   KrakenBuildWorker.obj
 0001:0001d540       __ehhandler$??0?$QList@PAVURLContainer@U2@@@@QAE@ABV0@@Z 1001e540 f   KrakenBuildWorker.obj
 0001:0001d560       __ehhandler$??0?$QList@VDataset@U2@@@@QAE@ABV0@@Z 1001e560 f   KrakenBuildWorker.obj
 0001:0001d580       __ehhandler$??0?$QList@VDescriptor@U2@@@@QAE@ABV0@@Z 1001e580 f   KrakenBuildWorker.obj
 0001:0001d5a0       __unwindfunclet$??A?$QMap@VQString@@VQScriptValue@@@@QAEAAVQScriptValue@@ABVQString@@@Z$0 1001e5a0 f   KrakenBuildWorker.obj
 0001:0001d5a9       __ehhandler$??A?$QMap@VQString@@VQScriptValue@@@@QAEAAVQScriptValue@@ABVQString@@@Z 1001e5a9 f   KrakenBuildWorker.obj
 0001:0001d5d0       __unwindfunclet$??A?$QMap@VQString@@VQVariant@@@@QAEAAVQVariant@@ABVQString@@@Z$0 1001e5d0 f   KrakenBuildWorker.obj
 0001:0001d5d9       __ehhandler$??A?$QMap@VQString@@VQVariant@@@@QAEAAVQVariant@@ABVQString@@@Z 1001e5d9 f   KrakenBuildWorker.obj
 0001:0001d600       __unwindfunclet$??__EalgoLog@U2@@YAXXZ$0 1001e600 f   KrakenBuildWorker.obj
 0001:0001d609       __ehhandler$??__EalgoLog@U2@@YAXXZ 1001e609 f   KrakenBuildWorker.obj
 0001:0001d630       __unwindfunclet$??__EcmdLog@U2@@YAXXZ$0 1001e630 f   KrakenBuildWorker.obj
 0001:0001d639       __ehhandler$??__EcmdLog@U2@@YAXXZ 1001e639 f   KrakenBuildWorker.obj
 0001:0001d660       __unwindfunclet$??__EcoreLog@U2@@YAXXZ$0 1001e660 f   KrakenBuildWorker.obj
 0001:0001d669       __ehhandler$??__EcoreLog@U2@@YAXXZ 1001e669 f   KrakenBuildWorker.obj
 0001:0001d690       __unwindfunclet$??__EioLog@U2@@YAXXZ$0 1001e690 f   KrakenBuildWorker.obj
 0001:0001d699       __ehhandler$??__EioLog@U2@@YAXXZ 1001e699 f   KrakenBuildWorker.obj
 0001:0001d6c0       __unwindfunclet$??__EperfLog@U2@@YAXXZ$0 1001e6c0 f   KrakenBuildWorker.obj
 0001:0001d6c9       __ehhandler$??__EperfLog@U2@@YAXXZ 1001e6c9 f   KrakenBuildWorker.obj
 0001:0001d6f0       __unwindfunclet$??__EscriptLog@U2@@YAXXZ$0 1001e6f0 f   KrakenBuildWorker.obj
 0001:0001d6f9       __ehhandler$??__EscriptLog@U2@@YAXXZ 1001e6f9 f   KrakenBuildWorker.obj
 0001:0001d720       __unwindfunclet$??__EtaskLog@U2@@YAXXZ$0 1001e720 f   KrakenBuildWorker.obj
 0001:0001d729       __ehhandler$??__EtaskLog@U2@@YAXXZ 1001e729 f   KrakenBuildWorker.obj
 0001:0001d750       __unwindfunclet$??__EuiLog@U2@@YAXXZ$0 1001e750 f   KrakenBuildWorker.obj
 0001:0001d759       __ehhandler$??__EuiLog@U2@@YAXXZ 1001e759 f   KrakenBuildWorker.obj
 0001:0001d780       __unwindfunclet$??__EuserActLog@U2@@YAXXZ$0 1001e780 f   KrakenBuildWorker.obj
 0001:0001d789       __ehhandler$??__EuserActLog@U2@@YAXXZ 1001e789 f   KrakenBuildWorker.obj
 0001:0001d7b0       __unwindfunclet$?Construct@?$QMetaTypeFunctionHelper@V?$QList@VDataset@U2@@@@$00@QtMetaTypePrivate@@SAPAXPAXPBX@Z$0 1001e7b0 f   KrakenBuildWorker.obj
 0001:0001d7c1       __ehhandler$?Construct@?$QMetaTypeFunctionHelper@V?$QList@VDataset@U2@@@@$00@QtMetaTypePrivate@@SAPAXPAXPBX@Z 1001e7c1 f   KrakenBuildWorker.obj
 0001:0001d7e0       __unwindfunclet$?Create@?$QMetaTypeFunctionHelper@V?$QList@VDataset@U2@@@@$00@QtMetaTypePrivate@@SAPAXPBX@Z$0 1001e7e0 f   KrakenBuildWorker.obj
 0001:0001d7eb       __ehhandler$?Create@?$QMetaTypeFunctionHelper@V?$QList@VDataset@U2@@@@$00@QtMetaTypePrivate@@SAPAXPBX@Z 1001e7eb f   KrakenBuildWorker.obj
 0001:0001d810       __unwindfunclet$?append@?$QList@VDescriptor@U2@@@@QAEXABVDescriptor@U2@@@Z$6 1001e810 f   KrakenBuildWorker.obj
 0001:0001d81b       __ehhandler$?append@?$QList@VDescriptor@U2@@@@QAEXABVDescriptor@U2@@@Z 1001e81b f   KrakenBuildWorker.obj
 0001:0001d840       __unwindfunclet$?createNode@?$QMapData@VQString@@VQScriptValue@@@@QAEPAU?$QMapNode@VQString@@VQScriptValue@@@@ABVQString@@ABVQScriptValue@@PAU2@_N@Z$4 1001e840 f   KrakenBuildWorker.obj
 0001:0001d854       __unwindfunclet$?createNode@?$QMapData@VQString@@VQScriptValue@@@@QAEPAU?$QMapNode@VQString@@VQScriptValue@@@@ABVQString@@ABVQScriptValue@@PAU2@_N@Z$5 1001e854 f   KrakenBuildWorker.obj
 0001:0001d868       __ehhandler$?createNode@?$QMapData@VQString@@VQScriptValue@@@@QAEPAU?$QMapNode@VQString@@VQScriptValue@@@@ABVQString@@ABVQScriptValue@@PAU2@_N@Z 1001e868 f   KrakenBuildWorker.obj
 0001:0001d890       __unwindfunclet$?createNode@?$QMapData@VQString@@VQVariant@@@@QAEPAU?$QMapNode@VQString@@VQVariant@@@@ABVQString@@ABVQVariant@@PAU2@_N@Z$4 1001e890 f   KrakenBuildWorker.obj
 0001:0001d8a4       __unwindfunclet$?createNode@?$QMapData@VQString@@VQVariant@@@@QAEPAU?$QMapNode@VQString@@VQVariant@@@@ABVQString@@ABVQVariant@@PAU2@_N@Z$5 1001e8a4 f   KrakenBuildWorker.obj
 0001:0001d8b8       __ehhandler$?createNode@?$QMapData@VQString@@VQVariant@@@@QAEPAU?$QMapNode@VQString@@VQVariant@@@@ABVQString@@ABVQVariant@@PAU2@_N@Z 1001e8b8 f   KrakenBuildWorker.obj
 0001:0001d8e0       __ehhandler$?detach_helper@?$QList@VDescriptor@U2@@@@AAEXH@Z 1001e8e0 f   KrakenBuildWorker.obj
 0001:0001d900       __ehhandler$?detach_helper_grow@?$QList@VDescriptor@U2@@@@AAEPAUNode@1@HH@Z 1001e900 f   KrakenBuildWorker.obj
 0001:0001d920       __unwindfunclet$?getSettings@KrakenBuildWorker@LocalWorkflow@U2@@AAE?AUKrakenBuildTaskSettings@3@XZ$0 1001e920 f   KrakenBuildWorker.obj
 0001:0001d939       __unwindfunclet$?getSettings@KrakenBuildWorker@LocalWorkflow@U2@@AAE?AUKrakenBuildTaskSettings@3@XZ$1 1001e939 f   KrakenBuildWorker.obj
 0001:0001d942       __unwindfunclet$?getSettings@KrakenBuildWorker@LocalWorkflow@U2@@AAE?AUKrakenBuildTaskSettings@3@XZ$2 1001e942 f   KrakenBuildWorker.obj
 0001:0001d94b       __unwindfunclet$?getSettings@KrakenBuildWorker@LocalWorkflow@U2@@AAE?AUKrakenBuildTaskSettings@3@XZ$3 1001e94b f   KrakenBuildWorker.obj
 0001:0001d953       __unwindfunclet$?getSettings@KrakenBuildWorker@LocalWorkflow@U2@@AAE?AUKrakenBuildTaskSettings@3@XZ$4 1001e953 f   KrakenBuildWorker.obj
 0001:0001d95b       __unwindfunclet$?getSettings@KrakenBuildWorker@LocalWorkflow@U2@@AAE?AUKrakenBuildTaskSettings@3@XZ$5 1001e95b f   KrakenBuildWorker.obj
 0001:0001d963       __unwindfunclet$?getSettings@KrakenBuildWorker@LocalWorkflow@U2@@AAE?AUKrakenBuildTaskSettings@3@XZ$6 1001e963 f   KrakenBuildWorker.obj
 0001:0001d96c       __unwindfunclet$?getSettings@KrakenBuildWorker@LocalWorkflow@U2@@AAE?AUKrakenBuildTaskSettings@3@XZ$7 1001e96c f   KrakenBuildWorker.obj
 0001:0001d975       __ehhandler$?getSettings@KrakenBuildWorker@LocalWorkflow@U2@@AAE?AUKrakenBuildTaskSettings@3@XZ 1001e975 f   KrakenBuildWorker.obj
 0001:0001d990       __unwindfunclet$?init@KrakenBuildWorker@LocalWorkflow@U2@@UAEXXZ$0 1001e990 f   KrakenBuildWorker.obj
 0001:0001d999       __unwindfunclet$?init@KrakenBuildWorker@LocalWorkflow@U2@@UAEXXZ$1 1001e999 f   KrakenBuildWorker.obj
 0001:0001d9a2       __unwindfunclet$?init@KrakenBuildWorker@LocalWorkflow@U2@@UAEXXZ$2 1001e9a2 f   KrakenBuildWorker.obj
 0001:0001d9ab       __unwindfunclet$?init@KrakenBuildWorker@LocalWorkflow@U2@@UAEXXZ$3 1001e9ab f   KrakenBuildWorker.obj
 0001:0001d9b4       __unwindfunclet$?init@KrakenBuildWorker@LocalWorkflow@U2@@UAEXXZ$4 1001e9b4 f   KrakenBuildWorker.obj
 0001:0001d9bd       __unwindfunclet$?init@KrakenBuildWorker@LocalWorkflow@U2@@UAEXXZ$5 1001e9bd f   KrakenBuildWorker.obj
 0001:0001d9c6       __unwindfunclet$?init@KrakenBuildWorker@LocalWorkflow@U2@@UAEXXZ$6 1001e9c6 f   KrakenBuildWorker.obj
 0001:0001d9cf       __ehhandler$?init@KrakenBuildWorker@LocalWorkflow@U2@@UAEXXZ 1001e9cf f   KrakenBuildWorker.obj
 0001:0001d9f0       __unwindfunclet$?metaType@?$QVariantValueHelper@V?$QList@VDataset@U2@@@@@QtPrivate@@SA?AV?$QList@VDataset@U2@@@@ABVQVariant@@@Z$0 1001e9f0 f   KrakenBuildWorker.obj
 0001:0001da09       __unwindfunclet$?metaType@?$QVariantValueHelper@V?$QList@VDataset@U2@@@@@QtPrivate@@SA?AV?$QList@VDataset@U2@@@@ABVQVariant@@@Z$1 1001ea09 f   KrakenBuildWorker.obj
 0001:0001da11       __ehhandler$?metaType@?$QVariantValueHelper@V?$QList@VDataset@U2@@@@@QtPrivate@@SA?AV?$QList@VDataset@U2@@@@ABVQVariant@@@Z 1001ea11 f   KrakenBuildWorker.obj
 0001:0001da30       __unwindfunclet$?metaType@?$QVariantValueHelper@VQString@@@QtPrivate@@SA?AVQString@@ABVQVariant@@@Z$0 1001ea30 f   KrakenBuildWorker.obj
 0001:0001da4a       __unwindfunclet$?metaType@?$QVariantValueHelper@VQString@@@QtPrivate@@SA?AVQString@@ABVQVariant@@@Z$1 1001ea4a f   KrakenBuildWorker.obj
 0001:0001da53       __ehhandler$?metaType@?$QVariantValueHelper@VQString@@@QtPrivate@@SA?AVQString@@ABVQVariant@@@Z 1001ea53 f   KrakenBuildWorker.obj
 0001:0001da70       __unwindfunclet$?node_construct@?$QList@VDescriptor@U2@@@@AAEXPAUNode@1@ABVDescriptor@U2@@@Z$0 1001ea70 f   KrakenBuildWorker.obj
 0001:0001da7b       __ehhandler$?node_construct@?$QList@VDescriptor@U2@@@@AAEXPAUNode@1@ABVDescriptor@U2@@@Z 1001ea7b f   KrakenBuildWorker.obj
 0001:0001daa0       __unwindfunclet$?node_copy@?$QList@VDataset@U2@@@@AAEXPAUNode@1@00@Z$4 1001eaa0 f   KrakenBuildWorker.obj
 0001:0001daab       __ehhandler$?node_copy@?$QList@VDataset@U2@@@@AAEXPAUNode@1@00@Z 1001eaab f   KrakenBuildWorker.obj
 0001:0001dad0       __unwindfunclet$?node_copy@?$QList@VDescriptor@U2@@@@AAEXPAUNode@1@00@Z$4 1001ead0 f   KrakenBuildWorker.obj
 0001:0001dadb       __ehhandler$?node_copy@?$QList@VDescriptor@U2@@@@AAEXPAUNode@1@00@Z 1001eadb f   KrakenBuildWorker.obj
 0001:0001db00       __unwindfunclet$?qt_metatype_id@?$QMetaTypeId@V?$QList@VDataset@U2@@@@@@SAHXZ$0 1001eb00 f   KrakenBuildWorker.obj
 0001:0001db09       __ehhandler$?qt_metatype_id@?$QMetaTypeId@V?$QList@VDataset@U2@@@@@@SAHXZ 1001eb09 f   KrakenBuildWorker.obj
 0001:0001db30       __unwindfunclet$?sl_taskFinished@KrakenBuildWorker@LocalWorkflow@U2@@AAEXPAVTask@3@@Z$0 1001eb30 f   KrakenBuildWorker.obj
 0001:0001db39       __unwindfunclet$?sl_taskFinished@KrakenBuildWorker@LocalWorkflow@U2@@AAEXPAVTask@3@@Z$1 1001eb39 f   KrakenBuildWorker.obj
 0001:0001db42       __unwindfunclet$?sl_taskFinished@KrakenBuildWorker@LocalWorkflow@U2@@AAEXPAVTask@3@@Z$2 1001eb42 f   KrakenBuildWorker.obj
 0001:0001db4b       __unwindfunclet$?sl_taskFinished@KrakenBuildWorker@LocalWorkflow@U2@@AAEXPAVTask@3@@Z$3 1001eb4b f   KrakenBuildWorker.obj
 0001:0001db54       __unwindfunclet$?sl_taskFinished@KrakenBuildWorker@LocalWorkflow@U2@@AAEXPAVTask@3@@Z$4 1001eb54 f   KrakenBuildWorker.obj
 0001:0001db5d       __unwindfunclet$?sl_taskFinished@KrakenBuildWorker@LocalWorkflow@U2@@AAEXPAVTask@3@@Z$5 1001eb5d f   KrakenBuildWorker.obj
 0001:0001db66       __unwindfunclet$?sl_taskFinished@KrakenBuildWorker@LocalWorkflow@U2@@AAEXPAVTask@3@@Z$6 1001eb66 f   KrakenBuildWorker.obj
 0001:0001db6e       __unwindfunclet$?sl_taskFinished@KrakenBuildWorker@LocalWorkflow@U2@@AAEXPAVTask@3@@Z$7 1001eb6e f   KrakenBuildWorker.obj
 0001:0001db77       __unwindfunclet$?sl_taskFinished@KrakenBuildWorker@LocalWorkflow@U2@@AAEXPAVTask@3@@Z$8 1001eb77 f   KrakenBuildWorker.obj
 0001:0001db80       __unwindfunclet$?sl_taskFinished@KrakenBuildWorker@LocalWorkflow@U2@@AAEXPAVTask@3@@Z$9 1001eb80 f   KrakenBuildWorker.obj
 0001:0001db89       __unwindfunclet$?sl_taskFinished@KrakenBuildWorker@LocalWorkflow@U2@@AAEXPAVTask@3@@Z$10 1001eb89 f   KrakenBuildWorker.obj
 0001:0001db92       __unwindfunclet$?sl_taskFinished@KrakenBuildWorker@LocalWorkflow@U2@@AAEXPAVTask@3@@Z$12 1001eb92 f   KrakenBuildWorker.obj
 0001:0001db9b       __unwindfunclet$?sl_taskFinished@KrakenBuildWorker@LocalWorkflow@U2@@AAEXPAVTask@3@@Z$13 1001eb9b f   KrakenBuildWorker.obj
 0001:0001dba4       __ehhandler$?sl_taskFinished@KrakenBuildWorker@LocalWorkflow@U2@@AAEXPAVTask@3@@Z 1001eba4 f   KrakenBuildWorker.obj
 0001:0001dbc0       __unwindfunclet$?tick@KrakenBuildWorker@LocalWorkflow@U2@@UAEPAVTask@3@XZ$0 1001ebc0 f   KrakenBuildWorker.obj
 0001:0001dbc8       __unwindfunclet$?tick@KrakenBuildWorker@LocalWorkflow@U2@@UAEPAVTask@3@XZ$1 1001ebc8 f   KrakenBuildWorker.obj
 0001:0001dbd3       __unwindfunclet$?tick@KrakenBuildWorker@LocalWorkflow@U2@@UAEPAVTask@3@XZ$2 1001ebd3 f   KrakenBuildWorker.obj
 0001:0001dbdb       __unwindfunclet$?tick@KrakenBuildWorker@LocalWorkflow@U2@@UAEPAVTask@3@XZ$3 1001ebdb f   KrakenBuildWorker.obj
 0001:0001dbe6       __unwindfunclet$?tick@KrakenBuildWorker@LocalWorkflow@U2@@UAEPAVTask@3@XZ$5 1001ebe6 f   KrakenBuildWorker.obj
 0001:0001dbef       __unwindfunclet$?tick@KrakenBuildWorker@LocalWorkflow@U2@@UAEPAVTask@3@XZ$6 1001ebef f   KrakenBuildWorker.obj
 0001:0001dbf8       __unwindfunclet$?tick@KrakenBuildWorker@LocalWorkflow@U2@@UAEPAVTask@3@XZ$7 1001ebf8 f   KrakenBuildWorker.obj
 0001:0001dc01       __ehhandler$?tick@KrakenBuildWorker@LocalWorkflow@U2@@UAEPAVTask@3@XZ 1001ec01 f   KrakenBuildWorker.obj
 0001:0001dc20       __unwindfunclet$?uniqueKeys@?$QMap@VDescriptor@U2@@VQVariant@@@@QBE?AV?$QList@VDescriptor@U2@@@@XZ$1 1001ec20 f   KrakenBuildWorker.obj
 0001:0001dc39       __ehhandler$?uniqueKeys@?$QMap@VDescriptor@U2@@VQVariant@@@@QBE?AV?$QList@VDescriptor@U2@@@@XZ 1001ec39 f   KrakenBuildWorker.obj
 0001:0001dc60       __unwindfunclet$??A?$QMap@VDescriptor@U2@@V?$QExplicitlySharedDataPointer@VDataType@U2@@@@@@QAEAAV?$QExplicitlySharedDataPointer@VDataType@U2@@@@ABVDescriptor@U2@@@Z$0 1001ec60 f   KrakenBuildWorkerFactory.obj
 0001:0001dc68       __ehhandler$??A?$QMap@VDescriptor@U2@@V?$QExplicitlySharedDataPointer@VDataType@U2@@@@@@QAEAAV?$QExplicitlySharedDataPointer@VDataType@U2@@@@ABVDescriptor@U2@@@Z 1001ec68 f   KrakenBuildWorkerFactory.obj
 0001:0001dc90       __unwindfunclet$??__EalgoLog@U2@@YAXXZ$0 1001ec90 f   KrakenBuildWorkerFactory.obj
 0001:0001dc99       __ehhandler$??__EalgoLog@U2@@YAXXZ 1001ec99 f   KrakenBuildWorkerFactory.obj
 0001:0001dcc0       __unwindfunclet$??__EcmdLog@U2@@YAXXZ$0 1001ecc0 f   KrakenBuildWorkerFactory.obj
 0001:0001dcc9       __ehhandler$??__EcmdLog@U2@@YAXXZ 1001ecc9 f   KrakenBuildWorkerFactory.obj
 0001:0001dcf0       __unwindfunclet$??__EcoreLog@U2@@YAXXZ$0 1001ecf0 f   KrakenBuildWorkerFactory.obj
 0001:0001dcf9       __ehhandler$??__EcoreLog@U2@@YAXXZ 1001ecf9 f   KrakenBuildWorkerFactory.obj
 0001:0001dd20       __unwindfunclet$??__EioLog@U2@@YAXXZ$0 1001ed20 f   KrakenBuildWorkerFactory.obj
 0001:0001dd29       __ehhandler$??__EioLog@U2@@YAXXZ 1001ed29 f   KrakenBuildWorkerFactory.obj
 0001:0001dd50       __unwindfunclet$??__EperfLog@U2@@YAXXZ$0 1001ed50 f   KrakenBuildWorkerFactory.obj
 0001:0001dd59       __ehhandler$??__EperfLog@U2@@YAXXZ 1001ed59 f   KrakenBuildWorkerFactory.obj
 0001:0001dd80       __unwindfunclet$??__EscriptLog@U2@@YAXXZ$0 1001ed80 f   KrakenBuildWorkerFactory.obj
 0001:0001dd89       __ehhandler$??__EscriptLog@U2@@YAXXZ 1001ed89 f   KrakenBuildWorkerFactory.obj
 0001:0001ddb0       __unwindfunclet$??__EtaskLog@U2@@YAXXZ$0 1001edb0 f   KrakenBuildWorkerFactory.obj
 0001:0001ddb9       __ehhandler$??__EtaskLog@U2@@YAXXZ 1001edb9 f   KrakenBuildWorkerFactory.obj
 0001:0001dde0       __unwindfunclet$??__EuiLog@U2@@YAXXZ$0 1001ede0 f   KrakenBuildWorkerFactory.obj
 0001:0001dde9       __ehhandler$??__EuiLog@U2@@YAXXZ 1001ede9 f   KrakenBuildWorkerFactory.obj
 0001:0001de10       __unwindfunclet$??__EuserActLog@U2@@YAXXZ$0 1001ee10 f   KrakenBuildWorkerFactory.obj
 0001:0001de19       __ehhandler$??__EuserActLog@U2@@YAXXZ 1001ee19 f   KrakenBuildWorkerFactory.obj
 0001:0001de40       __ehhandler$?append@?$QList@PAVAttribute@U2@@@@QAEXABQAVAttribute@U2@@@Z 1001ee40 f   KrakenBuildWorkerFactory.obj
 0001:0001de60       __ehhandler$?append@?$QList@PAVPortDescriptor@Workflow@U2@@@@QAEXABQAVPortDescriptor@Workflow@U2@@@Z 1001ee60 f   KrakenBuildWorkerFactory.obj
 0001:0001de80       __unwindfunclet$?createNode@?$QMapData@VDescriptor@U2@@V?$QExplicitlySharedDataPointer@VDataType@U2@@@@@@QAEPAU?$QMapNode@VDescriptor@U2@@V?$QExplicitlySharedDataPointer@VDataType@U2@@@@@@ABVDescriptor@U2@@ABV?$QExplicitlySharedDataPointer@VDataType@U2@@@@PAU2@_N@Z$4 1001ee80 f   KrakenBuildWorkerFactory.obj
 0001:0001de94       __ehhandler$?createNode@?$QMapData@VDescriptor@U2@@V?$QExplicitlySharedDataPointer@VDataType@U2@@@@@@QAEPAU?$QMapNode@VDescriptor@U2@@V?$QExplicitlySharedDataPointer@VDataType@U2@@@@@@ABVDescriptor@U2@@ABV?$QExplicitlySharedDataPointer@VDataType@U2@@@@PAU2@_N@Z 1001ee94 f   KrakenBuildWorkerFactory.obj
 0001:0001deb0       __unwindfunclet$?createNode@?$QMapData@VQString@@PAVPropertyDelegate@U2@@@@QAEPAU?$QMapNode@VQString@@PAVPropertyDelegate@U2@@@@ABVQString@@ABQAVPropertyDelegate@U2@@PAU2@_N@Z$4 1001eeb0 f   KrakenBuildWorkerFactory.obj
 0001:0001dec4       __ehhandler$?createNode@?$QMapData@VQString@@PAVPropertyDelegate@U2@@@@QAEPAU?$QMapNode@VQString@@PAVPropertyDelegate@U2@@@@ABVQString@@ABQAVPropertyDelegate@U2@@PAU2@_N@Z 1001eec4 f   KrakenBuildWorkerFactory.obj
 0001:0001dee0       __unwindfunclet$?createWorker@KrakenBuildWorkerFactory@LocalWorkflow@U2@@UAEPAVWorker@Workflow@3@PAVActor@53@@Z$0 1001eee0 f   KrakenBuildWorkerFactory.obj
 0001:0001deeb       __ehhandler$?createWorker@KrakenBuildWorkerFactory@LocalWorkflow@U2@@UAEPAVWorker@Workflow@3@PAVActor@53@@Z 1001eeeb f   KrakenBuildWorkerFactory.obj
 0001:0001df10       __ehhandler$?detach_helper_grow@?$QList@PAVAttribute@U2@@@@AAEPAUNode@1@HH@Z 1001ef10 f   KrakenBuildWorkerFactory.obj
 0001:0001df30       __ehhandler$?detach_helper_grow@?$QList@PAVPortDescriptor@Workflow@U2@@@@AAEPAUNode@1@HH@Z 1001ef30 f   KrakenBuildWorkerFactory.obj
 0001:0001df60       __unwindfunclet$?init@KrakenBuildWorkerFactory@LocalWorkflow@U2@@SAXXZ$0 1001ef60 f   KrakenBuildWorkerFactory.obj
 0001:0001df6b       __unwindfunclet$?init@KrakenBuildWorkerFactory@LocalWorkflow@U2@@SAXXZ$1 1001ef6b f   KrakenBuildWorkerFactory.obj
 0001:0001df74       __unwindfunclet$?init@KrakenBuildWorkerFactory@LocalWorkflow@U2@@SAXXZ$2 1001ef74 f   KrakenBuildWorkerFactory.obj
 0001:0001df7d       __unwindfunclet$?init@KrakenBuildWorkerFactory@LocalWorkflow@U2@@SAXXZ$3 1001ef7d f   KrakenBuildWorkerFactory.obj
 0001:0001df86       __unwindfunclet$?init@KrakenBuildWorkerFactory@LocalWorkflow@U2@@SAXXZ$4 1001ef86 f   KrakenBuildWorkerFactory.obj
 0001:0001df8f       __unwindfunclet$?init@KrakenBuildWorkerFactory@LocalWorkflow@U2@@SAXXZ$5 1001ef8f f   KrakenBuildWorkerFactory.obj
 0001:0001df98       __unwindfunclet$?init@KrakenBuildWorkerFactory@LocalWorkflow@U2@@SAXXZ$6 1001ef98 f   KrakenBuildWorkerFactory.obj
 0001:0001dfa0       __unwindfunclet$?init@KrakenBuildWorkerFactory@LocalWorkflow@U2@@SAXXZ$7 1001efa0 f   KrakenBuildWorkerFactory.obj
 0001:0001dfa8       __unwindfunclet$?init@KrakenBuildWorkerFactory@LocalWorkflow@U2@@SAXXZ$8 1001efa8 f   KrakenBuildWorkerFactory.obj
 0001:0001dfb1       __unwindfunclet$?init@KrakenBuildWorkerFactory@LocalWorkflow@U2@@SAXXZ$9 1001efb1 f   KrakenBuildWorkerFactory.obj
 0001:0001dfba       __unwindfunclet$?init@KrakenBuildWorkerFactory@LocalWorkflow@U2@@SAXXZ$10 1001efba f   KrakenBuildWorkerFactory.obj
 0001:0001dfc6       __unwindfunclet$?init@KrakenBuildWorkerFactory@LocalWorkflow@U2@@SAXXZ$11 1001efc6 f   KrakenBuildWorkerFactory.obj
 0001:0001dfd1       __unwindfunclet$?init@KrakenBuildWorkerFactory@LocalWorkflow@U2@@SAXXZ$12 1001efd1 f   KrakenBuildWorkerFactory.obj
 0001:0001dfdc       __unwindfunclet$?init@KrakenBuildWorkerFactory@LocalWorkflow@U2@@SAXXZ$13 1001efdc f   KrakenBuildWorkerFactory.obj
 0001:0001dff6       __unwindfunclet$?init@KrakenBuildWorkerFactory@LocalWorkflow@U2@@SAXXZ$14 1001eff6 f   KrakenBuildWorkerFactory.obj
 0001:0001e013       __unwindfunclet$?init@KrakenBuildWorkerFactory@LocalWorkflow@U2@@SAXXZ$16 1001f013 f   KrakenBuildWorkerFactory.obj
 0001:0001e01b       __unwindfunclet$?init@KrakenBuildWorkerFactory@LocalWorkflow@U2@@SAXXZ$17 1001f01b f   KrakenBuildWorkerFactory.obj
 0001:0001e024       __unwindfunclet$?init@KrakenBuildWorkerFactory@LocalWorkflow@U2@@SAXXZ$18 1001f024 f   KrakenBuildWorkerFactory.obj
 0001:0001e02d       __unwindfunclet$?init@KrakenBuildWorkerFactory@LocalWorkflow@U2@@SAXXZ$19 1001f02d f   KrakenBuildWorkerFactory.obj
 0001:0001e039       __unwindfunclet$?init@KrakenBuildWorkerFactory@LocalWorkflow@U2@@SAXXZ$20 1001f039 f   KrakenBuildWorkerFactory.obj
 0001:0001e042       __unwindfunclet$?init@KrakenBuildWorkerFactory@LocalWorkflow@U2@@SAXXZ$21 1001f042 f   KrakenBuildWorkerFactory.obj
 0001:0001e04b       __unwindfunclet$?init@KrakenBuildWorkerFactory@LocalWorkflow@U2@@SAXXZ$22 1001f04b f   KrakenBuildWorkerFactory.obj
 0001:0001e057       __unwindfunclet$?init@KrakenBuildWorkerFactory@LocalWorkflow@U2@@SAXXZ$23 1001f057 f   KrakenBuildWorkerFactory.obj
 0001:0001e063       __unwindfunclet$?init@KrakenBuildWorkerFactory@LocalWorkflow@U2@@SAXXZ$24 1001f063 f   KrakenBuildWorkerFactory.obj
 0001:0001e06f       __unwindfunclet$?init@KrakenBuildWorkerFactory@LocalWorkflow@U2@@SAXXZ$25 1001f06f f   KrakenBuildWorkerFactory.obj
 0001:0001e07b       __unwindfunclet$?init@KrakenBuildWorkerFactory@LocalWorkflow@U2@@SAXXZ$26 1001f07b f   KrakenBuildWorkerFactory.obj
 0001:0001e087       __unwindfunclet$?init@KrakenBuildWorkerFactory@LocalWorkflow@U2@@SAXXZ$27 1001f087 f   KrakenBuildWorkerFactory.obj
 0001:0001e093       __unwindfunclet$?init@KrakenBuildWorkerFactory@LocalWorkflow@U2@@SAXXZ$28 1001f093 f   KrakenBuildWorkerFactory.obj
 0001:0001e09f       __unwindfunclet$?init@KrakenBuildWorkerFactory@LocalWorkflow@U2@@SAXXZ$29 1001f09f f   KrakenBuildWorkerFactory.obj
 0001:0001e0ab       __unwindfunclet$?init@KrakenBuildWorkerFactory@LocalWorkflow@U2@@SAXXZ$30 1001f0ab f   KrakenBuildWorkerFactory.obj
 0001:0001e0b7       __unwindfunclet$?init@KrakenBuildWorkerFactory@LocalWorkflow@U2@@SAXXZ$31 1001f0b7 f   KrakenBuildWorkerFactory.obj
 0001:0001e0c3       __unwindfunclet$?init@KrakenBuildWorkerFactory@LocalWorkflow@U2@@SAXXZ$32 1001f0c3 f   KrakenBuildWorkerFactory.obj
 0001:0001e0cf       __unwindfunclet$?init@KrakenBuildWorkerFactory@LocalWorkflow@U2@@SAXXZ$33 1001f0cf f   KrakenBuildWorkerFactory.obj
 0001:0001e0db       __unwindfunclet$?init@KrakenBuildWorkerFactory@LocalWorkflow@U2@@SAXXZ$34 1001f0db f   KrakenBuildWorkerFactory.obj
 0001:0001e0e7       __unwindfunclet$?init@KrakenBuildWorkerFactory@LocalWorkflow@U2@@SAXXZ$35 1001f0e7 f   KrakenBuildWorkerFactory.obj
 0001:0001e0f3       __unwindfunclet$?init@KrakenBuildWorkerFactory@LocalWorkflow@U2@@SAXXZ$36 1001f0f3 f   KrakenBuildWorkerFactory.obj
 0001:0001e0ff       __unwindfunclet$?init@KrakenBuildWorkerFactory@LocalWorkflow@U2@@SAXXZ$37 1001f0ff f   KrakenBuildWorkerFactory.obj
 0001:0001e10b       __unwindfunclet$?init@KrakenBuildWorkerFactory@LocalWorkflow@U2@@SAXXZ$38 1001f10b f   KrakenBuildWorkerFactory.obj
 0001:0001e117       __unwindfunclet$?init@KrakenBuildWorkerFactory@LocalWorkflow@U2@@SAXXZ$39 1001f117 f   KrakenBuildWorkerFactory.obj
 0001:0001e123       __unwindfunclet$?init@KrakenBuildWorkerFactory@LocalWorkflow@U2@@SAXXZ$40 1001f123 f   KrakenBuildWorkerFactory.obj
 0001:0001e12f       __unwindfunclet$?init@KrakenBuildWorkerFactory@LocalWorkflow@U2@@SAXXZ$41 1001f12f f   KrakenBuildWorkerFactory.obj
 0001:0001e13b       __unwindfunclet$?init@KrakenBuildWorkerFactory@LocalWorkflow@U2@@SAXXZ$42 1001f13b f   KrakenBuildWorkerFactory.obj
 0001:0001e147       __unwindfunclet$?init@KrakenBuildWorkerFactory@LocalWorkflow@U2@@SAXXZ$43 1001f147 f   KrakenBuildWorkerFactory.obj
 0001:0001e153       __unwindfunclet$?init@KrakenBuildWorkerFactory@LocalWorkflow@U2@@SAXXZ$44 1001f153 f   KrakenBuildWorkerFactory.obj
 0001:0001e15f       __unwindfunclet$?init@KrakenBuildWorkerFactory@LocalWorkflow@U2@@SAXXZ$45 1001f15f f   KrakenBuildWorkerFactory.obj
 0001:0001e16b       __unwindfunclet$?init@KrakenBuildWorkerFactory@LocalWorkflow@U2@@SAXXZ$46 1001f16b f   KrakenBuildWorkerFactory.obj
 0001:0001e177       __unwindfunclet$?init@KrakenBuildWorkerFactory@LocalWorkflow@U2@@SAXXZ$47 1001f177 f   KrakenBuildWorkerFactory.obj
 0001:0001e183       __unwindfunclet$?init@KrakenBuildWorkerFactory@LocalWorkflow@U2@@SAXXZ$48 1001f183 f   KrakenBuildWorkerFactory.obj
 0001:0001e18f       __unwindfunclet$?init@KrakenBuildWorkerFactory@LocalWorkflow@U2@@SAXXZ$49 1001f18f f   KrakenBuildWorkerFactory.obj
 0001:0001e19b       __unwindfunclet$?init@KrakenBuildWorkerFactory@LocalWorkflow@U2@@SAXXZ$50 1001f19b f   KrakenBuildWorkerFactory.obj
 0001:0001e1a7       __unwindfunclet$?init@KrakenBuildWorkerFactory@LocalWorkflow@U2@@SAXXZ$51 1001f1a7 f   KrakenBuildWorkerFactory.obj
 0001:0001e1b3       __unwindfunclet$?init@KrakenBuildWorkerFactory@LocalWorkflow@U2@@SAXXZ$52 1001f1b3 f   KrakenBuildWorkerFactory.obj
 0001:0001e1bf       __unwindfunclet$?init@KrakenBuildWorkerFactory@LocalWorkflow@U2@@SAXXZ$53 1001f1bf f   KrakenBuildWorkerFactory.obj
 0001:0001e1cb       __unwindfunclet$?init@KrakenBuildWorkerFactory@LocalWorkflow@U2@@SAXXZ$54 1001f1cb f   KrakenBuildWorkerFactory.obj
 0001:0001e1d7       __unwindfunclet$?init@KrakenBuildWorkerFactory@LocalWorkflow@U2@@SAXXZ$55 1001f1d7 f   KrakenBuildWorkerFactory.obj
 0001:0001e1e3       __unwindfunclet$?init@KrakenBuildWorkerFactory@LocalWorkflow@U2@@SAXXZ$56 1001f1e3 f   KrakenBuildWorkerFactory.obj
 0001:0001e1ee       __unwindfunclet$?init@KrakenBuildWorkerFactory@LocalWorkflow@U2@@SAXXZ$57 1001f1ee f   KrakenBuildWorkerFactory.obj
 0001:0001e208       __unwindfunclet$?init@KrakenBuildWorkerFactory@LocalWorkflow@U2@@SAXXZ$59 1001f208 f   KrakenBuildWorkerFactory.obj
 0001:0001e213       __unwindfunclet$?init@KrakenBuildWorkerFactory@LocalWorkflow@U2@@SAXXZ$60 1001f213 f   KrakenBuildWorkerFactory.obj
 0001:0001e22d       __unwindfunclet$?init@KrakenBuildWorkerFactory@LocalWorkflow@U2@@SAXXZ$62 1001f22d f   KrakenBuildWorkerFactory.obj
 0001:0001e238       __unwindfunclet$?init@KrakenBuildWorkerFactory@LocalWorkflow@U2@@SAXXZ$63 1001f238 f   KrakenBuildWorkerFactory.obj
 0001:0001e252       __unwindfunclet$?init@KrakenBuildWorkerFactory@LocalWorkflow@U2@@SAXXZ$65 1001f252 f   KrakenBuildWorkerFactory.obj
 0001:0001e25d       __unwindfunclet$?init@KrakenBuildWorkerFactory@LocalWorkflow@U2@@SAXXZ$66 1001f25d f   KrakenBuildWorkerFactory.obj
 0001:0001e277       __unwindfunclet$?init@KrakenBuildWorkerFactory@LocalWorkflow@U2@@SAXXZ$68 1001f277 f   KrakenBuildWorkerFactory.obj
 0001:0001e282       __unwindfunclet$?init@KrakenBuildWorkerFactory@LocalWorkflow@U2@@SAXXZ$69 1001f282 f   KrakenBuildWorkerFactory.obj
 0001:0001e29c       __unwindfunclet$?init@KrakenBuildWorkerFactory@LocalWorkflow@U2@@SAXXZ$71 1001f29c f   KrakenBuildWorkerFactory.obj
 0001:0001e2a7       __unwindfunclet$?init@KrakenBuildWorkerFactory@LocalWorkflow@U2@@SAXXZ$72 1001f2a7 f   KrakenBuildWorkerFactory.obj
 0001:0001e2c6       __unwindfunclet$?init@KrakenBuildWorkerFactory@LocalWorkflow@U2@@SAXXZ$74 1001f2c6 f   KrakenBuildWorkerFactory.obj
 0001:0001e2d1       __unwindfunclet$?init@KrakenBuildWorkerFactory@LocalWorkflow@U2@@SAXXZ$75 1001f2d1 f   KrakenBuildWorkerFactory.obj
 0001:0001e2f0       __unwindfunclet$?init@KrakenBuildWorkerFactory@LocalWorkflow@U2@@SAXXZ$77 1001f2f0 f   KrakenBuildWorkerFactory.obj
 0001:0001e2fb       __unwindfunclet$?init@KrakenBuildWorkerFactory@LocalWorkflow@U2@@SAXXZ$78 1001f2fb f   KrakenBuildWorkerFactory.obj
 0001:0001e31a       __unwindfunclet$?init@KrakenBuildWorkerFactory@LocalWorkflow@U2@@SAXXZ$80 1001f31a f   KrakenBuildWorkerFactory.obj
 0001:0001e325       __unwindfunclet$?init@KrakenBuildWorkerFactory@LocalWorkflow@U2@@SAXXZ$81 1001f325 f   KrakenBuildWorkerFactory.obj
 0001:0001e344       __unwindfunclet$?init@KrakenBuildWorkerFactory@LocalWorkflow@U2@@SAXXZ$83 1001f344 f   KrakenBuildWorkerFactory.obj
 0001:0001e34f       __unwindfunclet$?init@KrakenBuildWorkerFactory@LocalWorkflow@U2@@SAXXZ$84 1001f34f f   KrakenBuildWorkerFactory.obj
 0001:0001e36e       __unwindfunclet$?init@KrakenBuildWorkerFactory@LocalWorkflow@U2@@SAXXZ$86 1001f36e f   KrakenBuildWorkerFactory.obj
 0001:0001e379       __unwindfunclet$?init@KrakenBuildWorkerFactory@LocalWorkflow@U2@@SAXXZ$87 1001f379 f   KrakenBuildWorkerFactory.obj
 0001:0001e398       __unwindfunclet$?init@KrakenBuildWorkerFactory@LocalWorkflow@U2@@SAXXZ$89 1001f398 f   KrakenBuildWorkerFactory.obj
 0001:0001e3a3       __unwindfunclet$?init@KrakenBuildWorkerFactory@LocalWorkflow@U2@@SAXXZ$90 1001f3a3 f   KrakenBuildWorkerFactory.obj
 0001:0001e3c2       __unwindfunclet$?init@KrakenBuildWorkerFactory@LocalWorkflow@U2@@SAXXZ$92 1001f3c2 f   KrakenBuildWorkerFactory.obj
 0001:0001e3cd       __unwindfunclet$?init@KrakenBuildWorkerFactory@LocalWorkflow@U2@@SAXXZ$93 1001f3cd f   KrakenBuildWorkerFactory.obj
 0001:0001e3ec       __unwindfunclet$?init@KrakenBuildWorkerFactory@LocalWorkflow@U2@@SAXXZ$95 1001f3ec f   KrakenBuildWorkerFactory.obj
 0001:0001e3f7       __unwindfunclet$?init@KrakenBuildWorkerFactory@LocalWorkflow@U2@@SAXXZ$96 1001f3f7 f   KrakenBuildWorkerFactory.obj
 0001:0001e416       __unwindfunclet$?init@KrakenBuildWorkerFactory@LocalWorkflow@U2@@SAXXZ$97 1001f416 f   KrakenBuildWorkerFactory.obj
 0001:0001e421       __unwindfunclet$?init@KrakenBuildWorkerFactory@LocalWorkflow@U2@@SAXXZ$98 1001f421 f   KrakenBuildWorkerFactory.obj
 0001:0001e440       __unwindfunclet$?init@KrakenBuildWorkerFactory@LocalWorkflow@U2@@SAXXZ$99 1001f440 f   KrakenBuildWorkerFactory.obj
 0001:0001e44b       __unwindfunclet$?init@KrakenBuildWorkerFactory@LocalWorkflow@U2@@SAXXZ$100 1001f44b f   KrakenBuildWorkerFactory.obj
 0001:0001e46a       __unwindfunclet$?init@KrakenBuildWorkerFactory@LocalWorkflow@U2@@SAXXZ$101 1001f46a f   KrakenBuildWorkerFactory.obj
 0001:0001e475       __unwindfunclet$?init@KrakenBuildWorkerFactory@LocalWorkflow@U2@@SAXXZ$102 1001f475 f   KrakenBuildWorkerFactory.obj
 0001:0001e494       __unwindfunclet$?init@KrakenBuildWorkerFactory@LocalWorkflow@U2@@SAXXZ$103 1001f494 f   KrakenBuildWorkerFactory.obj
 0001:0001e49f       __unwindfunclet$?init@KrakenBuildWorkerFactory@LocalWorkflow@U2@@SAXXZ$104 1001f49f f   KrakenBuildWorkerFactory.obj
 0001:0001e4be       __unwindfunclet$?init@KrakenBuildWorkerFactory@LocalWorkflow@U2@@SAXXZ$105 1001f4be f   KrakenBuildWorkerFactory.obj
 0001:0001e4c9       __unwindfunclet$?init@KrakenBuildWorkerFactory@LocalWorkflow@U2@@SAXXZ$106 1001f4c9 f   KrakenBuildWorkerFactory.obj
 0001:0001e4e8       __unwindfunclet$?init@KrakenBuildWorkerFactory@LocalWorkflow@U2@@SAXXZ$107 1001f4e8 f   KrakenBuildWorkerFactory.obj
 0001:0001e4f3       __unwindfunclet$?init@KrakenBuildWorkerFactory@LocalWorkflow@U2@@SAXXZ$108 1001f4f3 f   KrakenBuildWorkerFactory.obj
 0001:0001e512       __unwindfunclet$?init@KrakenBuildWorkerFactory@LocalWorkflow@U2@@SAXXZ$109 1001f512 f   KrakenBuildWorkerFactory.obj
 0001:0001e51a       __unwindfunclet$?init@KrakenBuildWorkerFactory@LocalWorkflow@U2@@SAXXZ$110 1001f51a f   KrakenBuildWorkerFactory.obj
 0001:0001e522       __unwindfunclet$?init@KrakenBuildWorkerFactory@LocalWorkflow@U2@@SAXXZ$111 1001f522 f   KrakenBuildWorkerFactory.obj
 0001:0001e52b       __unwindfunclet$?init@KrakenBuildWorkerFactory@LocalWorkflow@U2@@SAXXZ$112 1001f52b f   KrakenBuildWorkerFactory.obj
 0001:0001e534       __unwindfunclet$?init@KrakenBuildWorkerFactory@LocalWorkflow@U2@@SAXXZ$113 1001f534 f   KrakenBuildWorkerFactory.obj
 0001:0001e53d       __unwindfunclet$?init@KrakenBuildWorkerFactory@LocalWorkflow@U2@@SAXXZ$114 1001f53d f   KrakenBuildWorkerFactory.obj
 0001:0001e546       __unwindfunclet$?init@KrakenBuildWorkerFactory@LocalWorkflow@U2@@SAXXZ$115 1001f546 f   KrakenBuildWorkerFactory.obj
 0001:0001e551       __unwindfunclet$?init@KrakenBuildWorkerFactory@LocalWorkflow@U2@@SAXXZ$116 1001f551 f   KrakenBuildWorkerFactory.obj
 0001:0001e55c       __unwindfunclet$?init@KrakenBuildWorkerFactory@LocalWorkflow@U2@@SAXXZ$117 1001f55c f   KrakenBuildWorkerFactory.obj
 0001:0001e57b       __unwindfunclet$?init@KrakenBuildWorkerFactory@LocalWorkflow@U2@@SAXXZ$118 1001f57b f   KrakenBuildWorkerFactory.obj
 0001:0001e59a       __unwindfunclet$?init@KrakenBuildWorkerFactory@LocalWorkflow@U2@@SAXXZ$119 1001f59a f   KrakenBuildWorkerFactory.obj
 0001:0001e5b9       __unwindfunclet$?init@KrakenBuildWorkerFactory@LocalWorkflow@U2@@SAXXZ$120 1001f5b9 f   KrakenBuildWorkerFactory.obj
 0001:0001e5c4       __unwindfunclet$?init@KrakenBuildWorkerFactory@LocalWorkflow@U2@@SAXXZ$121 1001f5c4 f   KrakenBuildWorkerFactory.obj
 0001:0001e5e3       __unwindfunclet$?init@KrakenBuildWorkerFactory@LocalWorkflow@U2@@SAXXZ$122 1001f5e3 f   KrakenBuildWorkerFactory.obj
 0001:0001e602       __unwindfunclet$?init@KrakenBuildWorkerFactory@LocalWorkflow@U2@@SAXXZ$123 1001f602 f   KrakenBuildWorkerFactory.obj
 0001:0001e621       __unwindfunclet$?init@KrakenBuildWorkerFactory@LocalWorkflow@U2@@SAXXZ$124 1001f621 f   KrakenBuildWorkerFactory.obj
 0001:0001e62c       __unwindfunclet$?init@KrakenBuildWorkerFactory@LocalWorkflow@U2@@SAXXZ$125 1001f62c f   KrakenBuildWorkerFactory.obj
 0001:0001e634       __unwindfunclet$?init@KrakenBuildWorkerFactory@LocalWorkflow@U2@@SAXXZ$126 1001f634 f   KrakenBuildWorkerFactory.obj
 0001:0001e63d       __unwindfunclet$?init@KrakenBuildWorkerFactory@LocalWorkflow@U2@@SAXXZ$127 1001f63d f   KrakenBuildWorkerFactory.obj
 0001:0001e646       __unwindfunclet$?init@KrakenBuildWorkerFactory@LocalWorkflow@U2@@SAXXZ$128 1001f646 f   KrakenBuildWorkerFactory.obj
 0001:0001e652       __unwindfunclet$?init@KrakenBuildWorkerFactory@LocalWorkflow@U2@@SAXXZ$129 1001f652 f   KrakenBuildWorkerFactory.obj
 0001:0001e65b       __unwindfunclet$?init@KrakenBuildWorkerFactory@LocalWorkflow@U2@@SAXXZ$130 1001f65b f   KrakenBuildWorkerFactory.obj
 0001:0001e667       __unwindfunclet$?init@KrakenBuildWorkerFactory@LocalWorkflow@U2@@SAXXZ$131 1001f667 f   KrakenBuildWorkerFactory.obj
 0001:0001e670       __unwindfunclet$?init@KrakenBuildWorkerFactory@LocalWorkflow@U2@@SAXXZ$132 1001f670 f   KrakenBuildWorkerFactory.obj
 0001:0001e67b       __unwindfunclet$?init@KrakenBuildWorkerFactory@LocalWorkflow@U2@@SAXXZ$133 1001f67b f   KrakenBuildWorkerFactory.obj
 0001:0001e683       __unwindfunclet$?init@KrakenBuildWorkerFactory@LocalWorkflow@U2@@SAXXZ$134 1001f683 f   KrakenBuildWorkerFactory.obj
 0001:0001e68c       __unwindfunclet$?init@KrakenBuildWorkerFactory@LocalWorkflow@U2@@SAXXZ$135 1001f68c f   KrakenBuildWorkerFactory.obj
 0001:0001e695       __unwindfunclet$?init@KrakenBuildWorkerFactory@LocalWorkflow@U2@@SAXXZ$136 1001f695 f   KrakenBuildWorkerFactory.obj
 0001:0001e6a1       __unwindfunclet$?init@KrakenBuildWorkerFactory@LocalWorkflow@U2@@SAXXZ$137 1001f6a1 f   KrakenBuildWorkerFactory.obj
 0001:0001e6aa       __unwindfunclet$?init@KrakenBuildWorkerFactory@LocalWorkflow@U2@@SAXXZ$138 1001f6aa f   KrakenBuildWorkerFactory.obj
 0001:0001e6b5       __unwindfunclet$?init@KrakenBuildWorkerFactory@LocalWorkflow@U2@@SAXXZ$139 1001f6b5 f   KrakenBuildWorkerFactory.obj
 0001:0001e6bd       __unwindfunclet$?init@KrakenBuildWorkerFactory@LocalWorkflow@U2@@SAXXZ$140 1001f6bd f   KrakenBuildWorkerFactory.obj
 0001:0001e6c6       __unwindfunclet$?init@KrakenBuildWorkerFactory@LocalWorkflow@U2@@SAXXZ$141 1001f6c6 f   KrakenBuildWorkerFactory.obj
 0001:0001e6cf       __unwindfunclet$?init@KrakenBuildWorkerFactory@LocalWorkflow@U2@@SAXXZ$142 1001f6cf f   KrakenBuildWorkerFactory.obj
 0001:0001e6db       __unwindfunclet$?init@KrakenBuildWorkerFactory@LocalWorkflow@U2@@SAXXZ$143 1001f6db f   KrakenBuildWorkerFactory.obj
 0001:0001e6e4       __unwindfunclet$?init@KrakenBuildWorkerFactory@LocalWorkflow@U2@@SAXXZ$144 1001f6e4 f   KrakenBuildWorkerFactory.obj
 0001:0001e6ef       __unwindfunclet$?init@KrakenBuildWorkerFactory@LocalWorkflow@U2@@SAXXZ$145 1001f6ef f   KrakenBuildWorkerFactory.obj
 0001:0001e6f7       __unwindfunclet$?init@KrakenBuildWorkerFactory@LocalWorkflow@U2@@SAXXZ$146 1001f6f7 f   KrakenBuildWorkerFactory.obj
 0001:0001e700       __unwindfunclet$?init@KrakenBuildWorkerFactory@LocalWorkflow@U2@@SAXXZ$147 1001f700 f   KrakenBuildWorkerFactory.obj
 0001:0001e709       __unwindfunclet$?init@KrakenBuildWorkerFactory@LocalWorkflow@U2@@SAXXZ$148 1001f709 f   KrakenBuildWorkerFactory.obj
 0001:0001e715       __unwindfunclet$?init@KrakenBuildWorkerFactory@LocalWorkflow@U2@@SAXXZ$149 1001f715 f   KrakenBuildWorkerFactory.obj
 0001:0001e71e       __unwindfunclet$?init@KrakenBuildWorkerFactory@LocalWorkflow@U2@@SAXXZ$150 1001f71e f   KrakenBuildWorkerFactory.obj
 0001:0001e72a       __unwindfunclet$?init@KrakenBuildWorkerFactory@LocalWorkflow@U2@@SAXXZ$151 1001f72a f   KrakenBuildWorkerFactory.obj
 0001:0001e733       __unwindfunclet$?init@KrakenBuildWorkerFactory@LocalWorkflow@U2@@SAXXZ$152 1001f733 f   KrakenBuildWorkerFactory.obj
 0001:0001e73c       __unwindfunclet$?init@KrakenBuildWorkerFactory@LocalWorkflow@U2@@SAXXZ$153 1001f73c f   KrakenBuildWorkerFactory.obj
 0001:0001e745       __unwindfunclet$?init@KrakenBuildWorkerFactory@LocalWorkflow@U2@@SAXXZ$154 1001f745 f   KrakenBuildWorkerFactory.obj
 0001:0001e74e       __unwindfunclet$?init@KrakenBuildWorkerFactory@LocalWorkflow@U2@@SAXXZ$155 1001f74e f   KrakenBuildWorkerFactory.obj
 0001:0001e75a       __unwindfunclet$?init@KrakenBuildWorkerFactory@LocalWorkflow@U2@@SAXXZ$156 1001f75a f   KrakenBuildWorkerFactory.obj
 0001:0001e763       __unwindfunclet$?init@KrakenBuildWorkerFactory@LocalWorkflow@U2@@SAXXZ$157 1001f763 f   KrakenBuildWorkerFactory.obj
 0001:0001e76e       __unwindfunclet$?init@KrakenBuildWorkerFactory@LocalWorkflow@U2@@SAXXZ$158 1001f76e f   KrakenBuildWorkerFactory.obj
 0001:0001e776       __unwindfunclet$?init@KrakenBuildWorkerFactory@LocalWorkflow@U2@@SAXXZ$159 1001f776 f   KrakenBuildWorkerFactory.obj
 0001:0001e77f       __unwindfunclet$?init@KrakenBuildWorkerFactory@LocalWorkflow@U2@@SAXXZ$160 1001f77f f   KrakenBuildWorkerFactory.obj
 0001:0001e788       __unwindfunclet$?init@KrakenBuildWorkerFactory@LocalWorkflow@U2@@SAXXZ$161 1001f788 f   KrakenBuildWorkerFactory.obj
 0001:0001e794       __unwindfunclet$?init@KrakenBuildWorkerFactory@LocalWorkflow@U2@@SAXXZ$162 1001f794 f   KrakenBuildWorkerFactory.obj
 0001:0001e79d       __unwindfunclet$?init@KrakenBuildWorkerFactory@LocalWorkflow@U2@@SAXXZ$163 1001f79d f   KrakenBuildWorkerFactory.obj
 0001:0001e7a8       __unwindfunclet$?init@KrakenBuildWorkerFactory@LocalWorkflow@U2@@SAXXZ$164 1001f7a8 f   KrakenBuildWorkerFactory.obj
 0001:0001e7b3       __unwindfunclet$?init@KrakenBuildWorkerFactory@LocalWorkflow@U2@@SAXXZ$165 1001f7b3 f   KrakenBuildWorkerFactory.obj
 0001:0001e7be       __unwindfunclet$?init@KrakenBuildWorkerFactory@LocalWorkflow@U2@@SAXXZ$166 1001f7be f   KrakenBuildWorkerFactory.obj
 0001:0001e7c6       __unwindfunclet$?init@KrakenBuildWorkerFactory@LocalWorkflow@U2@@SAXXZ$167 1001f7c6 f   KrakenBuildWorkerFactory.obj
 0001:0001e7cf       __unwindfunclet$?init@KrakenBuildWorkerFactory@LocalWorkflow@U2@@SAXXZ$168 1001f7cf f   KrakenBuildWorkerFactory.obj
 0001:0001e7d8       __unwindfunclet$?init@KrakenBuildWorkerFactory@LocalWorkflow@U2@@SAXXZ$169 1001f7d8 f   KrakenBuildWorkerFactory.obj
 0001:0001e7e4       __unwindfunclet$?init@KrakenBuildWorkerFactory@LocalWorkflow@U2@@SAXXZ$170 1001f7e4 f   KrakenBuildWorkerFactory.obj
 0001:0001e7ed       __unwindfunclet$?init@KrakenBuildWorkerFactory@LocalWorkflow@U2@@SAXXZ$171 1001f7ed f   KrakenBuildWorkerFactory.obj
 0001:0001e7f9       __unwindfunclet$?init@KrakenBuildWorkerFactory@LocalWorkflow@U2@@SAXXZ$172 1001f7f9 f   KrakenBuildWorkerFactory.obj
 0001:0001e802       __unwindfunclet$?init@KrakenBuildWorkerFactory@LocalWorkflow@U2@@SAXXZ$173 1001f802 f   KrakenBuildWorkerFactory.obj
 0001:0001e80b       __unwindfunclet$?init@KrakenBuildWorkerFactory@LocalWorkflow@U2@@SAXXZ$174 1001f80b f   KrakenBuildWorkerFactory.obj
 0001:0001e814       __unwindfunclet$?init@KrakenBuildWorkerFactory@LocalWorkflow@U2@@SAXXZ$175 1001f814 f   KrakenBuildWorkerFactory.obj
 0001:0001e81d       __unwindfunclet$?init@KrakenBuildWorkerFactory@LocalWorkflow@U2@@SAXXZ$176 1001f81d f   KrakenBuildWorkerFactory.obj
 0001:0001e828       __unwindfunclet$?init@KrakenBuildWorkerFactory@LocalWorkflow@U2@@SAXXZ$177 1001f828 f   KrakenBuildWorkerFactory.obj
 0001:0001e830       __unwindfunclet$?init@KrakenBuildWorkerFactory@LocalWorkflow@U2@@SAXXZ$178 1001f830 f   KrakenBuildWorkerFactory.obj
 0001:0001e839       __unwindfunclet$?init@KrakenBuildWorkerFactory@LocalWorkflow@U2@@SAXXZ$179 1001f839 f   KrakenBuildWorkerFactory.obj
 0001:0001e842       __unwindfunclet$?init@KrakenBuildWorkerFactory@LocalWorkflow@U2@@SAXXZ$180 1001f842 f   KrakenBuildWorkerFactory.obj
 0001:0001e84b       __unwindfunclet$?init@KrakenBuildWorkerFactory@LocalWorkflow@U2@@SAXXZ$181 1001f84b f   KrakenBuildWorkerFactory.obj
 0001:0001e854       __unwindfunclet$?init@KrakenBuildWorkerFactory@LocalWorkflow@U2@@SAXXZ$182 1001f854 f   KrakenBuildWorkerFactory.obj
 0001:0001e85f       __unwindfunclet$?init@KrakenBuildWorkerFactory@LocalWorkflow@U2@@SAXXZ$183 1001f85f f   KrakenBuildWorkerFactory.obj
 0001:0001e868       __unwindfunclet$?init@KrakenBuildWorkerFactory@LocalWorkflow@U2@@SAXXZ$184 1001f868 f   KrakenBuildWorkerFactory.obj
 0001:0001e871       __unwindfunclet$?init@KrakenBuildWorkerFactory@LocalWorkflow@U2@@SAXXZ$185 1001f871 f   KrakenBuildWorkerFactory.obj
 0001:0001e87d       __unwindfunclet$?init@KrakenBuildWorkerFactory@LocalWorkflow@U2@@SAXXZ$186 1001f87d f   KrakenBuildWorkerFactory.obj
 0001:0001e888       __unwindfunclet$?init@KrakenBuildWorkerFactory@LocalWorkflow@U2@@SAXXZ$187 1001f888 f   KrakenBuildWorkerFactory.obj
 0001:0001e893       __unwindfunclet$?init@KrakenBuildWorkerFactory@LocalWorkflow@U2@@SAXXZ$188 1001f893 f   KrakenBuildWorkerFactory.obj
 0001:0001e89e       __unwindfunclet$?init@KrakenBuildWorkerFactory@LocalWorkflow@U2@@SAXXZ$189 1001f89e f   KrakenBuildWorkerFactory.obj
 0001:0001e8a7       __unwindfunclet$?init@KrakenBuildWorkerFactory@LocalWorkflow@U2@@SAXXZ$190 1001f8a7 f   KrakenBuildWorkerFactory.obj
 0001:0001e8b0       __unwindfunclet$?init@KrakenBuildWorkerFactory@LocalWorkflow@U2@@SAXXZ$191 1001f8b0 f   KrakenBuildWorkerFactory.obj
 0001:0001e8bb       __ehhandler$?init@KrakenBuildWorkerFactory@LocalWorkflow@U2@@SAXXZ 1001f8bb f   KrakenBuildWorkerFactory.obj
 0001:0001e8e0       __unwindfunclet$??__EalgoLog@U2@@YAXXZ$0 1001f8e0 f   KrakenClassifyLogParser.obj
 0001:0001e8e9       __ehhandler$??__EalgoLog@U2@@YAXXZ 1001f8e9 f   KrakenClassifyLogParser.obj
 0001:0001e910       __unwindfunclet$??__EcmdLog@U2@@YAXXZ$0 1001f910 f   KrakenClassifyLogParser.obj
 0001:0001e919       __ehhandler$??__EcmdLog@U2@@YAXXZ 1001f919 f   KrakenClassifyLogParser.obj
 0001:0001e940       __unwindfunclet$??__EcoreLog@U2@@YAXXZ$0 1001f940 f   KrakenClassifyLogParser.obj
 0001:0001e949       __ehhandler$??__EcoreLog@U2@@YAXXZ 1001f949 f   KrakenClassifyLogParser.obj
 0001:0001e970       __unwindfunclet$??__EioLog@U2@@YAXXZ$0 1001f970 f   KrakenClassifyLogParser.obj
 0001:0001e979       __ehhandler$??__EioLog@U2@@YAXXZ 1001f979 f   KrakenClassifyLogParser.obj
 0001:0001e9a0       __unwindfunclet$??__EperfLog@U2@@YAXXZ$0 1001f9a0 f   KrakenClassifyLogParser.obj
 0001:0001e9a9       __ehhandler$??__EperfLog@U2@@YAXXZ 1001f9a9 f   KrakenClassifyLogParser.obj
 0001:0001e9d0       __unwindfunclet$??__EscriptLog@U2@@YAXXZ$0 1001f9d0 f   KrakenClassifyLogParser.obj
 0001:0001e9d9       __ehhandler$??__EscriptLog@U2@@YAXXZ 1001f9d9 f   KrakenClassifyLogParser.obj
 0001:0001ea00       __unwindfunclet$??__EtaskLog@U2@@YAXXZ$0 1001fa00 f   KrakenClassifyLogParser.obj
 0001:0001ea09       __ehhandler$??__EtaskLog@U2@@YAXXZ 1001fa09 f   KrakenClassifyLogParser.obj
 0001:0001ea30       __unwindfunclet$??__EuiLog@U2@@YAXXZ$0 1001fa30 f   KrakenClassifyLogParser.obj
 0001:0001ea39       __ehhandler$??__EuiLog@U2@@YAXXZ 1001fa39 f   KrakenClassifyLogParser.obj
 0001:0001ea60       __unwindfunclet$??__EuserActLog@U2@@YAXXZ$0 1001fa60 f   KrakenClassifyLogParser.obj
 0001:0001ea69       __ehhandler$??__EuserActLog@U2@@YAXXZ 1001fa69 f   KrakenClassifyLogParser.obj
 0001:0001ea90       __unwindfunclet$?initWellKnownErrors@KrakenClassifyLogParser@U2@@CA?AVQStringList@@XZ$0 1001fa90 f   KrakenClassifyLogParser.obj
 0001:0001eaa9       __unwindfunclet$?initWellKnownErrors@KrakenClassifyLogParser@U2@@CA?AVQStringList@@XZ$1 1001faa9 f   KrakenClassifyLogParser.obj
 0001:0001eab2       __unwindfunclet$?initWellKnownErrors@KrakenClassifyLogParser@U2@@CA?AVQStringList@@XZ$2 1001fab2 f   KrakenClassifyLogParser.obj
 0001:0001eabb       __unwindfunclet$?initWellKnownErrors@KrakenClassifyLogParser@U2@@CA?AVQStringList@@XZ$3 1001fabb f   KrakenClassifyLogParser.obj
 0001:0001eac4       __unwindfunclet$?initWellKnownErrors@KrakenClassifyLogParser@U2@@CA?AVQStringList@@XZ$4 1001fac4 f   KrakenClassifyLogParser.obj
 0001:0001eacd       __unwindfunclet$?initWellKnownErrors@KrakenClassifyLogParser@U2@@CA?AVQStringList@@XZ$5 1001facd f   KrakenClassifyLogParser.obj
 0001:0001ead6       __unwindfunclet$?initWellKnownErrors@KrakenClassifyLogParser@U2@@CA?AVQStringList@@XZ$6 1001fad6 f   KrakenClassifyLogParser.obj
 0001:0001eadf       __unwindfunclet$?initWellKnownErrors@KrakenClassifyLogParser@U2@@CA?AVQStringList@@XZ$7 1001fadf f   KrakenClassifyLogParser.obj
 0001:0001eae8       __unwindfunclet$?initWellKnownErrors@KrakenClassifyLogParser@U2@@CA?AVQStringList@@XZ$8 1001fae8 f   KrakenClassifyLogParser.obj
 0001:0001eaf1       __ehhandler$?initWellKnownErrors@KrakenClassifyLogParser@U2@@CA?AVQStringList@@XZ 1001faf1 f   KrakenClassifyLogParser.obj
 0001:0001eb10       __unwindfunclet$?isError@KrakenClassifyLogParser@U2@@EBE_NABVQString@@@Z$0 1001fb10 f   KrakenClassifyLogParser.obj
 0001:0001eb18       __ehhandler$?isError@KrakenClassifyLogParser@U2@@EBE_NABVQString@@@Z 1001fb18 f   KrakenClassifyLogParser.obj
 0001:0001eb40       __unwindfunclet$??__EalgoLog@U2@@YAXXZ$0 1001fb40 f   KrakenClassifyPrompter.obj
 0001:0001eb49       __ehhandler$??__EalgoLog@U2@@YAXXZ 1001fb49 f   KrakenClassifyPrompter.obj
 0001:0001eb70       __unwindfunclet$??__EcmdLog@U2@@YAXXZ$0 1001fb70 f   KrakenClassifyPrompter.obj
 0001:0001eb79       __ehhandler$??__EcmdLog@U2@@YAXXZ 1001fb79 f   KrakenClassifyPrompter.obj
 0001:0001eba0       __unwindfunclet$??__EcoreLog@U2@@YAXXZ$0 1001fba0 f   KrakenClassifyPrompter.obj
 0001:0001eba9       __ehhandler$??__EcoreLog@U2@@YAXXZ 1001fba9 f   KrakenClassifyPrompter.obj
 0001:0001ebd0       __unwindfunclet$??__EioLog@U2@@YAXXZ$0 1001fbd0 f   KrakenClassifyPrompter.obj
 0001:0001ebd9       __ehhandler$??__EioLog@U2@@YAXXZ 1001fbd9 f   KrakenClassifyPrompter.obj
 0001:0001ec00       __unwindfunclet$??__EperfLog@U2@@YAXXZ$0 1001fc00 f   KrakenClassifyPrompter.obj
 0001:0001ec09       __ehhandler$??__EperfLog@U2@@YAXXZ 1001fc09 f   KrakenClassifyPrompter.obj
 0001:0001ec30       __unwindfunclet$??__EscriptLog@U2@@YAXXZ$0 1001fc30 f   KrakenClassifyPrompter.obj
 0001:0001ec39       __ehhandler$??__EscriptLog@U2@@YAXXZ 1001fc39 f   KrakenClassifyPrompter.obj
 0001:0001ec60       __unwindfunclet$??__EtaskLog@U2@@YAXXZ$0 1001fc60 f   KrakenClassifyPrompter.obj
 0001:0001ec69       __ehhandler$??__EtaskLog@U2@@YAXXZ 1001fc69 f   KrakenClassifyPrompter.obj
 0001:0001ec90       __unwindfunclet$??__EuiLog@U2@@YAXXZ$0 1001fc90 f   KrakenClassifyPrompter.obj
 0001:0001ec99       __ehhandler$??__EuiLog@U2@@YAXXZ 1001fc99 f   KrakenClassifyPrompter.obj
 0001:0001ecc0       __unwindfunclet$??__EuserActLog@U2@@YAXXZ$0 1001fcc0 f   KrakenClassifyPrompter.obj
 0001:0001ecc9       __ehhandler$??__EuserActLog@U2@@YAXXZ 1001fcc9 f   KrakenClassifyPrompter.obj
 0001:0001ecf0       __unwindfunclet$?composeRichDoc@KrakenClassifyPrompter@LocalWorkflow@U2@@EAE?AVQString@@XZ$0 1001fcf0 f   KrakenClassifyPrompter.obj
 0001:0001ecf9       __unwindfunclet$?composeRichDoc@KrakenClassifyPrompter@LocalWorkflow@U2@@EAE?AVQString@@XZ$1 1001fcf9 f   KrakenClassifyPrompter.obj
 0001:0001ed02       __unwindfunclet$?composeRichDoc@KrakenClassifyPrompter@LocalWorkflow@U2@@EAE?AVQString@@XZ$2 1001fd02 f   KrakenClassifyPrompter.obj
 0001:0001ed0b       __unwindfunclet$?composeRichDoc@KrakenClassifyPrompter@LocalWorkflow@U2@@EAE?AVQString@@XZ$3 1001fd0b f   KrakenClassifyPrompter.obj
 0001:0001ed14       __unwindfunclet$?composeRichDoc@KrakenClassifyPrompter@LocalWorkflow@U2@@EAE?AVQString@@XZ$4 1001fd14 f   KrakenClassifyPrompter.obj
 0001:0001ed1d       __unwindfunclet$?composeRichDoc@KrakenClassifyPrompter@LocalWorkflow@U2@@EAE?AVQString@@XZ$5 1001fd1d f   KrakenClassifyPrompter.obj
 0001:0001ed26       __unwindfunclet$?composeRichDoc@KrakenClassifyPrompter@LocalWorkflow@U2@@EAE?AVQString@@XZ$6 1001fd26 f   KrakenClassifyPrompter.obj
 0001:0001ed2f       __unwindfunclet$?composeRichDoc@KrakenClassifyPrompter@LocalWorkflow@U2@@EAE?AVQString@@XZ$7 1001fd2f f   KrakenClassifyPrompter.obj
 0001:0001ed38       __unwindfunclet$?composeRichDoc@KrakenClassifyPrompter@LocalWorkflow@U2@@EAE?AVQString@@XZ$8 1001fd38 f   KrakenClassifyPrompter.obj
 0001:0001ed41       __unwindfunclet$?composeRichDoc@KrakenClassifyPrompter@LocalWorkflow@U2@@EAE?AVQString@@XZ$9 1001fd41 f   KrakenClassifyPrompter.obj
 0001:0001ed5b       __unwindfunclet$?composeRichDoc@KrakenClassifyPrompter@LocalWorkflow@U2@@EAE?AVQString@@XZ$10 1001fd5b f   KrakenClassifyPrompter.obj
 0001:0001ed64       __unwindfunclet$?composeRichDoc@KrakenClassifyPrompter@LocalWorkflow@U2@@EAE?AVQString@@XZ$11 1001fd64 f   KrakenClassifyPrompter.obj
 0001:0001ed6d       __ehhandler$?composeRichDoc@KrakenClassifyPrompter@LocalWorkflow@U2@@EAE?AVQString@@XZ 1001fd6d f   KrakenClassifyPrompter.obj
 0001:0001ed90       __unwindfunclet$?createDescription@?$PrompterBase@VKrakenClassifyPrompter@LocalWorkflow@U2@@@U2@@UAEPAVActorDocument@Workflow@2@PAVActor@42@@Z$0 1001fd90 f   KrakenClassifyPrompter.obj
 0001:0001ed9b       __unwindfunclet$?createDescription@?$PrompterBase@VKrakenClassifyPrompter@LocalWorkflow@U2@@@U2@@UAEPAVActorDocument@Workflow@2@PAVActor@42@@Z$3 1001fd9b f   KrakenClassifyPrompter.obj
 0001:0001eda3       __unwindfunclet$?createDescription@?$PrompterBase@VKrakenClassifyPrompter@LocalWorkflow@U2@@@U2@@UAEPAVActorDocument@Workflow@2@PAVActor@42@@Z$4 1001fda3 f   KrakenClassifyPrompter.obj
 0001:0001edab       __unwindfunclet$?createDescription@?$PrompterBase@VKrakenClassifyPrompter@LocalWorkflow@U2@@@U2@@UAEPAVActorDocument@Workflow@2@PAVActor@42@@Z$6 1001fdab f   KrakenClassifyPrompter.obj
 0001:0001edb3       __unwindfunclet$?createDescription@?$PrompterBase@VKrakenClassifyPrompter@LocalWorkflow@U2@@@U2@@UAEPAVActorDocument@Workflow@2@PAVActor@42@@Z$7 1001fdb3 f   KrakenClassifyPrompter.obj
 0001:0001edbb       __ehhandler$?createDescription@?$PrompterBase@VKrakenClassifyPrompter@LocalWorkflow@U2@@@U2@@UAEPAVActorDocument@Workflow@2@PAVActor@42@@Z 1001fdbb f   KrakenClassifyPrompter.obj
 0001:0001ede0       __unwindfunclet$??0KrakenClassifyTask@U2@@QAE@ABUKrakenClassifyTaskSettings@1@@Z$0 1001fde0 f   KrakenClassifyTask.obj
 0001:0001ede9       __unwindfunclet$??0KrakenClassifyTask@U2@@QAE@ABUKrakenClassifyTaskSettings@1@@Z$1 1001fde9 f   KrakenClassifyTask.obj
 0001:0001edf2       __unwindfunclet$??0KrakenClassifyTask@U2@@QAE@ABUKrakenClassifyTaskSettings@1@@Z$2 1001fdf2 f   KrakenClassifyTask.obj
 0001:0001ee00       __unwindfunclet$??0KrakenClassifyTask@U2@@QAE@ABUKrakenClassifyTaskSettings@1@@Z$3 1001fe00 f   KrakenClassifyTask.obj
 0001:0001ee0e       __unwindfunclet$??0KrakenClassifyTask@U2@@QAE@ABUKrakenClassifyTaskSettings@1@@Z$4 1001fe0e f   KrakenClassifyTask.obj
 0001:0001ee1c       __unwindfunclet$??0KrakenClassifyTask@U2@@QAE@ABUKrakenClassifyTaskSettings@1@@Z$5 1001fe1c f   KrakenClassifyTask.obj
 0001:0001ee25       __unwindfunclet$??0KrakenClassifyTask@U2@@QAE@ABUKrakenClassifyTaskSettings@1@@Z$6 1001fe25 f   KrakenClassifyTask.obj
 0001:0001ee2e       __unwindfunclet$??0KrakenClassifyTask@U2@@QAE@ABUKrakenClassifyTaskSettings@1@@Z$7 1001fe2e f   KrakenClassifyTask.obj
 0001:0001ee37       __unwindfunclet$??0KrakenClassifyTask@U2@@QAE@ABUKrakenClassifyTaskSettings@1@@Z$8 1001fe37 f   KrakenClassifyTask.obj
 0001:0001ee40       __unwindfunclet$??0KrakenClassifyTask@U2@@QAE@ABUKrakenClassifyTaskSettings@1@@Z$10 1001fe40 f   KrakenClassifyTask.obj
 0001:0001ee49       __unwindfunclet$??0KrakenClassifyTask@U2@@QAE@ABUKrakenClassifyTaskSettings@1@@Z$11 1001fe49 f   KrakenClassifyTask.obj
 0001:0001ee52       __ehhandler$??0KrakenClassifyTask@U2@@QAE@ABUKrakenClassifyTaskSettings@1@@Z 1001fe52 f   KrakenClassifyTask.obj
 0001:0001ee70       __unwindfunclet$??0KrakenClassifyTaskSettings@U2@@QAE@ABU01@@Z$0 1001fe70 f   KrakenClassifyTask.obj
 0001:0001ee79       __unwindfunclet$??0KrakenClassifyTaskSettings@U2@@QAE@ABU01@@Z$1 1001fe79 f   KrakenClassifyTask.obj
 0001:0001ee85       __unwindfunclet$??0KrakenClassifyTaskSettings@U2@@QAE@ABU01@@Z$2 1001fe85 f   KrakenClassifyTask.obj
 0001:0001ee91       __ehhandler$??0KrakenClassifyTaskSettings@U2@@QAE@ABU01@@Z 1001fe91 f   KrakenClassifyTask.obj
 0001:0001eeb0       __unwindfunclet$??0KrakenClassifyTaskSettings@U2@@QAE@XZ$0 1001feb0 f   KrakenClassifyTask.obj
 0001:0001eeb9       __unwindfunclet$??0KrakenClassifyTaskSettings@U2@@QAE@XZ$1 1001feb9 f   KrakenClassifyTask.obj
 0001:0001eec5       __unwindfunclet$??0KrakenClassifyTaskSettings@U2@@QAE@XZ$2 1001fec5 f   KrakenClassifyTask.obj
 0001:0001eed1       __ehhandler$??0KrakenClassifyTaskSettings@U2@@QAE@XZ 1001fed1 f   KrakenClassifyTask.obj
 0001:0001eef0       __unwindfunclet$??1KrakenClassifyTask@U2@@UAE@XZ$0 1001fef0 f   KrakenClassifyTask.obj
 0001:0001eef9       __unwindfunclet$??1KrakenClassifyTask@U2@@UAE@XZ$1 1001fef9 f   KrakenClassifyTask.obj
 0001:0001ef07       __unwindfunclet$??1KrakenClassifyTask@U2@@UAE@XZ$3 1001ff07 f   KrakenClassifyTask.obj
 0001:0001ef10       __unwindfunclet$??1KrakenClassifyTask@U2@@UAE@XZ$4 1001ff10 f   KrakenClassifyTask.obj
 0001:0001ef1c       __unwindfunclet$??1KrakenClassifyTask@U2@@UAE@XZ$5 1001ff1c f   KrakenClassifyTask.obj
 0001:0001ef28       __ehhandler$??1KrakenClassifyTask@U2@@UAE@XZ 1001ff28 f   KrakenClassifyTask.obj
 0001:0001ef50       __unwindfunclet$??1KrakenClassifyTaskSettings@U2@@QAE@XZ$0 1001ff50 f   KrakenClassifyTask.obj
 0001:0001ef59       __unwindfunclet$??1KrakenClassifyTaskSettings@U2@@QAE@XZ$1 1001ff59 f   KrakenClassifyTask.obj
 0001:0001ef65       __unwindfunclet$??1KrakenClassifyTaskSettings@U2@@QAE@XZ$2 1001ff65 f   KrakenClassifyTask.obj
 0001:0001ef71       __ehhandler$??1KrakenClassifyTaskSettings@U2@@QAE@XZ 1001ff71 f   KrakenClassifyTask.obj
 0001:0001ef90       __unwindfunclet$??__EalgoLog@U2@@YAXXZ$0 1001ff90 f   KrakenClassifyTask.obj
 0001:0001ef99       __ehhandler$??__EalgoLog@U2@@YAXXZ 1001ff99 f   KrakenClassifyTask.obj
 0001:0001efc0       __unwindfunclet$??__EcmdLog@U2@@YAXXZ$0 1001ffc0 f   KrakenClassifyTask.obj
 0001:0001efc9       __ehhandler$??__EcmdLog@U2@@YAXXZ 1001ffc9 f   KrakenClassifyTask.obj
 0001:0001eff0       __unwindfunclet$??__EcoreLog@U2@@YAXXZ$0 1001fff0 f   KrakenClassifyTask.obj
 0001:0001eff9       __ehhandler$??__EcoreLog@U2@@YAXXZ 1001fff9 f   KrakenClassifyTask.obj
 0001:0001f020       __unwindfunclet$??__EioLog@U2@@YAXXZ$0 10020020 f   KrakenClassifyTask.obj
 0001:0001f029       __ehhandler$??__EioLog@U2@@YAXXZ 10020029 f   KrakenClassifyTask.obj
 0001:0001f050       __unwindfunclet$??__EperfLog@U2@@YAXXZ$0 10020050 f   KrakenClassifyTask.obj
 0001:0001f059       __ehhandler$??__EperfLog@U2@@YAXXZ 10020059 f   KrakenClassifyTask.obj
 0001:0001f080       __unwindfunclet$??__EscriptLog@U2@@YAXXZ$0 10020080 f   KrakenClassifyTask.obj
 0001:0001f089       __ehhandler$??__EscriptLog@U2@@YAXXZ 10020089 f   KrakenClassifyTask.obj
 0001:0001f0b0       __unwindfunclet$??__EtaskLog@U2@@YAXXZ$0 100200b0 f   KrakenClassifyTask.obj
 0001:0001f0b9       __ehhandler$??__EtaskLog@U2@@YAXXZ 100200b9 f   KrakenClassifyTask.obj
 0001:0001f0e0       __unwindfunclet$??__EuiLog@U2@@YAXXZ$0 100200e0 f   KrakenClassifyTask.obj
 0001:0001f0e9       __ehhandler$??__EuiLog@U2@@YAXXZ 100200e9 f   KrakenClassifyTask.obj
 0001:0001f110       __unwindfunclet$??__EuserActLog@U2@@YAXXZ$0 10020110 f   KrakenClassifyTask.obj
 0001:0001f119       __ehhandler$??__EuserActLog@U2@@YAXXZ 10020119 f   KrakenClassifyTask.obj
 0001:0001f140       __unwindfunclet$?createNode@?$QMapData@VQString@@I@@QAEPAU?$QMapNode@VQString@@I@@ABVQString@@ABIPAU2@_N@Z$4 10020140 f   KrakenClassifyTask.obj
 0001:0001f154       __ehhandler$?createNode@?$QMapData@VQString@@I@@QAEPAU?$QMapNode@VQString@@I@@ABVQString@@ABIPAU2@_N@Z 10020154 f   KrakenClassifyTask.obj
 0001:0001f170       __ehhandler$?detach_helper@?$QList@VQByteArray@@@@AAEXH@Z 10020170 f   KrakenClassifyTask.obj
 0001:0001f190       __unwindfunclet$?getArguments@KrakenClassifyTask@U2@@AAE?AVQStringList@@XZ$0 10020190 f   KrakenClassifyTask.obj
 0001:0001f1a9       __unwindfunclet$?getArguments@KrakenClassifyTask@U2@@AAE?AVQStringList@@XZ$1 100201a9 f   KrakenClassifyTask.obj
 0001:0001f1b2       __unwindfunclet$?getArguments@KrakenClassifyTask@U2@@AAE?AVQStringList@@XZ$2 100201b2 f   KrakenClassifyTask.obj
 0001:0001f1bb       __unwindfunclet$?getArguments@KrakenClassifyTask@U2@@AAE?AVQStringList@@XZ$3 100201bb f   KrakenClassifyTask.obj
 0001:0001f1c4       __unwindfunclet$?getArguments@KrakenClassifyTask@U2@@AAE?AVQStringList@@XZ$4 100201c4 f   KrakenClassifyTask.obj
 0001:0001f1cd       __unwindfunclet$?getArguments@KrakenClassifyTask@U2@@AAE?AVQStringList@@XZ$5 100201cd f   KrakenClassifyTask.obj
 0001:0001f1d6       __unwindfunclet$?getArguments@KrakenClassifyTask@U2@@AAE?AVQStringList@@XZ$6 100201d6 f   KrakenClassifyTask.obj
 0001:0001f1df       __unwindfunclet$?getArguments@KrakenClassifyTask@U2@@AAE?AVQStringList@@XZ$7 100201df f   KrakenClassifyTask.obj
 0001:0001f1e8       __unwindfunclet$?getArguments@KrakenClassifyTask@U2@@AAE?AVQStringList@@XZ$8 100201e8 f   KrakenClassifyTask.obj
 0001:0001f1f1       __unwindfunclet$?getArguments@KrakenClassifyTask@U2@@AAE?AVQStringList@@XZ$9 100201f1 f   KrakenClassifyTask.obj
 0001:0001f1fa       __unwindfunclet$?getArguments@KrakenClassifyTask@U2@@AAE?AVQStringList@@XZ$10 100201fa f   KrakenClassifyTask.obj
 0001:0001f203       __ehhandler$?getArguments@KrakenClassifyTask@U2@@AAE?AVQStringList@@XZ 10020203 f   KrakenClassifyTask.obj
 0001:0001f220       __unwindfunclet$?node_copy@?$QList@VQByteArray@@@@AAEXPAUNode@1@00@Z$5 10020220 f   KrakenClassifyTask.obj
 0001:0001f231       __ehhandler$?node_copy@?$QList@VQByteArray@@@@AAEXPAUNode@1@00@Z 10020231 f   KrakenClassifyTask.obj
 0001:0001f250       __unwindfunclet$?prepare@KrakenClassifyTask@U2@@EAEXXZ$0 10020250 f   KrakenClassifyTask.obj
 0001:0001f25b       __unwindfunclet$?prepare@KrakenClassifyTask@U2@@EAEXXZ$1 1002025b f   KrakenClassifyTask.obj
 0001:0001f275       __unwindfunclet$?prepare@KrakenClassifyTask@U2@@EAEXXZ$2 10020275 f   KrakenClassifyTask.obj
 0001:0001f280       __unwindfunclet$?prepare@KrakenClassifyTask@U2@@EAEXXZ$3 10020280 f   KrakenClassifyTask.obj
 0001:0001f29a       __unwindfunclet$?prepare@KrakenClassifyTask@U2@@EAEXXZ$4 1002029a f   KrakenClassifyTask.obj
 0001:0001f2b3       __unwindfunclet$?prepare@KrakenClassifyTask@U2@@EAEXXZ$5 100202b3 f   KrakenClassifyTask.obj
 0001:0001f2cc       __ehhandler$?prepare@KrakenClassifyTask@U2@@EAEXXZ 100202cc f   KrakenClassifyTask.obj
 0001:0001f2f0       __unwindfunclet$?run@KrakenClassifyTask@U2@@EAEXXZ$0 100202f0 f   KrakenClassifyTask.obj
 0001:0001f2f9       __unwindfunclet$?run@KrakenClassifyTask@U2@@EAEXXZ$1 100202f9 f   KrakenClassifyTask.obj
 0001:0001f302       __unwindfunclet$?run@KrakenClassifyTask@U2@@EAEXXZ$2 10020302 f   KrakenClassifyTask.obj
 0001:0001f30b       __unwindfunclet$?run@KrakenClassifyTask@U2@@EAEXXZ$3 1002030b f   KrakenClassifyTask.obj
 0001:0001f314       __unwindfunclet$?run@KrakenClassifyTask@U2@@EAEXXZ$4 10020314 f   KrakenClassifyTask.obj
 0001:0001f31d       __unwindfunclet$?run@KrakenClassifyTask@U2@@EAEXXZ$5 1002031d f   KrakenClassifyTask.obj
 0001:0001f325       __unwindfunclet$?run@KrakenClassifyTask@U2@@EAEXXZ$6 10020325 f   KrakenClassifyTask.obj
 0001:0001f32e       __unwindfunclet$?run@KrakenClassifyTask@U2@@EAEXXZ$7 1002032e f   KrakenClassifyTask.obj
 0001:0001f337       __unwindfunclet$?run@KrakenClassifyTask@U2@@EAEXXZ$8 10020337 f   KrakenClassifyTask.obj
 0001:0001f340       __unwindfunclet$?run@KrakenClassifyTask@U2@@EAEXXZ$9 10020340 f   KrakenClassifyTask.obj
 0001:0001f349       __unwindfunclet$?run@KrakenClassifyTask@U2@@EAEXXZ$10 10020349 f   KrakenClassifyTask.obj
 0001:0001f352       __unwindfunclet$?run@KrakenClassifyTask@U2@@EAEXXZ$11 10020352 f   KrakenClassifyTask.obj
 0001:0001f35b       __unwindfunclet$?run@KrakenClassifyTask@U2@@EAEXXZ$12 1002035b f   KrakenClassifyTask.obj
 0001:0001f364       __unwindfunclet$?run@KrakenClassifyTask@U2@@EAEXXZ$13 10020364 f   KrakenClassifyTask.obj
 0001:0001f36d       __unwindfunclet$?run@KrakenClassifyTask@U2@@EAEXXZ$14 1002036d f   KrakenClassifyTask.obj
 0001:0001f376       __ehhandler$?run@KrakenClassifyTask@U2@@EAEXXZ 10020376 f   KrakenClassifyTask.obj
 0001:0001f3a0       __unwindfunclet$??__EalgoLog@U2@@YAXXZ$0 100203a0 f   KrakenClassifyValidator.obj
 0001:0001f3a9       __ehhandler$??__EalgoLog@U2@@YAXXZ 100203a9 f   KrakenClassifyValidator.obj
 0001:0001f3d0       __unwindfunclet$??__EcmdLog@U2@@YAXXZ$0 100203d0 f   KrakenClassifyValidator.obj
 0001:0001f3d9       __ehhandler$??__EcmdLog@U2@@YAXXZ 100203d9 f   KrakenClassifyValidator.obj
 0001:0001f400       __unwindfunclet$??__EcoreLog@U2@@YAXXZ$0 10020400 f   KrakenClassifyValidator.obj
 0001:0001f409       __ehhandler$??__EcoreLog@U2@@YAXXZ 10020409 f   KrakenClassifyValidator.obj
 0001:0001f430       __unwindfunclet$??__EioLog@U2@@YAXXZ$0 10020430 f   KrakenClassifyValidator.obj
 0001:0001f439       __ehhandler$??__EioLog@U2@@YAXXZ 10020439 f   KrakenClassifyValidator.obj
 0001:0001f460       __unwindfunclet$??__EperfLog@U2@@YAXXZ$0 10020460 f   KrakenClassifyValidator.obj
 0001:0001f469       __ehhandler$??__EperfLog@U2@@YAXXZ 10020469 f   KrakenClassifyValidator.obj
 0001:0001f490       __unwindfunclet$??__EscriptLog@U2@@YAXXZ$0 10020490 f   KrakenClassifyValidator.obj
 0001:0001f499       __ehhandler$??__EscriptLog@U2@@YAXXZ 10020499 f   KrakenClassifyValidator.obj
 0001:0001f4c0       __unwindfunclet$??__EtaskLog@U2@@YAXXZ$0 100204c0 f   KrakenClassifyValidator.obj
 0001:0001f4c9       __ehhandler$??__EtaskLog@U2@@YAXXZ 100204c9 f   KrakenClassifyValidator.obj
 0001:0001f4f0       __unwindfunclet$??__EuiLog@U2@@YAXXZ$0 100204f0 f   KrakenClassifyValidator.obj
 0001:0001f4f9       __ehhandler$??__EuiLog@U2@@YAXXZ 100204f9 f   KrakenClassifyValidator.obj
 0001:0001f520       __unwindfunclet$??__EuserActLog@U2@@YAXXZ$0 10020520 f   KrakenClassifyValidator.obj
 0001:0001f529       __ehhandler$??__EuserActLog@U2@@YAXXZ 10020529 f   KrakenClassifyValidator.obj
 0001:0001f550       __unwindfunclet$?validateDatabase@KrakenClassifyValidator@Workflow@U2@@ABE_NPBVActor@23@AAV?$QList@VWorkflowNotification@U2@@@@@Z$0 10020550 f   KrakenClassifyValidator.obj
 0001:0001f559       __unwindfunclet$?validateDatabase@KrakenClassifyValidator@Workflow@U2@@ABE_NPBVActor@23@AAV?$QList@VWorkflowNotification@U2@@@@@Z$1 10020559 f   KrakenClassifyValidator.obj
 0001:0001f562       __unwindfunclet$?validateDatabase@KrakenClassifyValidator@Workflow@U2@@ABE_NPBVActor@23@AAV?$QList@VWorkflowNotification@U2@@@@@Z$2 10020562 f   KrakenClassifyValidator.obj
 0001:0001f56b       __unwindfunclet$?validateDatabase@KrakenClassifyValidator@Workflow@U2@@ABE_NPBVActor@23@AAV?$QList@VWorkflowNotification@U2@@@@@Z$3 1002056b f   KrakenClassifyValidator.obj
 0001:0001f574       __unwindfunclet$?validateDatabase@KrakenClassifyValidator@Workflow@U2@@ABE_NPBVActor@23@AAV?$QList@VWorkflowNotification@U2@@@@@Z$4 10020574 f   KrakenClassifyValidator.obj
 0001:0001f57d       __unwindfunclet$?validateDatabase@KrakenClassifyValidator@Workflow@U2@@ABE_NPBVActor@23@AAV?$QList@VWorkflowNotification@U2@@@@@Z$5 1002057d f   KrakenClassifyValidator.obj
 0001:0001f586       __unwindfunclet$?validateDatabase@KrakenClassifyValidator@Workflow@U2@@ABE_NPBVActor@23@AAV?$QList@VWorkflowNotification@U2@@@@@Z$6 10020586 f   KrakenClassifyValidator.obj
 0001:0001f58f       __unwindfunclet$?validateDatabase@KrakenClassifyValidator@Workflow@U2@@ABE_NPBVActor@23@AAV?$QList@VWorkflowNotification@U2@@@@@Z$7 1002058f f   KrakenClassifyValidator.obj
 0001:0001f598       __unwindfunclet$?validateDatabase@KrakenClassifyValidator@Workflow@U2@@ABE_NPBVActor@23@AAV?$QList@VWorkflowNotification@U2@@@@@Z$8 10020598 f   KrakenClassifyValidator.obj
 0001:0001f5a1       __unwindfunclet$?validateDatabase@KrakenClassifyValidator@Workflow@U2@@ABE_NPBVActor@23@AAV?$QList@VWorkflowNotification@U2@@@@@Z$9 100205a1 f   KrakenClassifyValidator.obj
 0001:0001f5aa       __unwindfunclet$?validateDatabase@KrakenClassifyValidator@Workflow@U2@@ABE_NPBVActor@23@AAV?$QList@VWorkflowNotification@U2@@@@@Z$10 100205aa f   KrakenClassifyValidator.obj
 0001:0001f5b2       __unwindfunclet$?validateDatabase@KrakenClassifyValidator@Workflow@U2@@ABE_NPBVActor@23@AAV?$QList@VWorkflowNotification@U2@@@@@Z$11 100205b2 f   KrakenClassifyValidator.obj
 0001:0001f5ba       __unwindfunclet$?validateDatabase@KrakenClassifyValidator@Workflow@U2@@ABE_NPBVActor@23@AAV?$QList@VWorkflowNotification@U2@@@@@Z$12 100205ba f   KrakenClassifyValidator.obj
 0001:0001f5c2       __unwindfunclet$?validateDatabase@KrakenClassifyValidator@Workflow@U2@@ABE_NPBVActor@23@AAV?$QList@VWorkflowNotification@U2@@@@@Z$13 100205c2 f   KrakenClassifyValidator.obj
 0001:0001f5ca       __unwindfunclet$?validateDatabase@KrakenClassifyValidator@Workflow@U2@@ABE_NPBVActor@23@AAV?$QList@VWorkflowNotification@U2@@@@@Z$14 100205ca f   KrakenClassifyValidator.obj
 0001:0001f5d3       __unwindfunclet$?validateDatabase@KrakenClassifyValidator@Workflow@U2@@ABE_NPBVActor@23@AAV?$QList@VWorkflowNotification@U2@@@@@Z$15 100205d3 f   KrakenClassifyValidator.obj
 0001:0001f5dc       __unwindfunclet$?validateDatabase@KrakenClassifyValidator@Workflow@U2@@ABE_NPBVActor@23@AAV?$QList@VWorkflowNotification@U2@@@@@Z$16 100205dc f   KrakenClassifyValidator.obj
 0001:0001f5e5       __unwindfunclet$?validateDatabase@KrakenClassifyValidator@Workflow@U2@@ABE_NPBVActor@23@AAV?$QList@VWorkflowNotification@U2@@@@@Z$17 100205e5 f   KrakenClassifyValidator.obj
 0001:0001f5ed       __unwindfunclet$?validateDatabase@KrakenClassifyValidator@Workflow@U2@@ABE_NPBVActor@23@AAV?$QList@VWorkflowNotification@U2@@@@@Z$18 100205ed f   KrakenClassifyValidator.obj
 0001:0001f5f6       __unwindfunclet$?validateDatabase@KrakenClassifyValidator@Workflow@U2@@ABE_NPBVActor@23@AAV?$QList@VWorkflowNotification@U2@@@@@Z$19 100205f6 f   KrakenClassifyValidator.obj
 0001:0001f5ff       __unwindfunclet$?validateDatabase@KrakenClassifyValidator@Workflow@U2@@ABE_NPBVActor@23@AAV?$QList@VWorkflowNotification@U2@@@@@Z$20 100205ff f   KrakenClassifyValidator.obj
 0001:0001f608       __unwindfunclet$?validateDatabase@KrakenClassifyValidator@Workflow@U2@@ABE_NPBVActor@23@AAV?$QList@VWorkflowNotification@U2@@@@@Z$21 10020608 f   KrakenClassifyValidator.obj
 0001:0001f611       __unwindfunclet$?validateDatabase@KrakenClassifyValidator@Workflow@U2@@ABE_NPBVActor@23@AAV?$QList@VWorkflowNotification@U2@@@@@Z$22 10020611 f   KrakenClassifyValidator.obj
 0001:0001f61a       __unwindfunclet$?validateDatabase@KrakenClassifyValidator@Workflow@U2@@ABE_NPBVActor@23@AAV?$QList@VWorkflowNotification@U2@@@@@Z$23 1002061a f   KrakenClassifyValidator.obj
 0001:0001f623       __ehhandler$?validateDatabase@KrakenClassifyValidator@Workflow@U2@@ABE_NPBVActor@23@AAV?$QList@VWorkflowNotification@U2@@@@@Z 10020623 f   KrakenClassifyValidator.obj
 0001:0001f640       __unwindfunclet$??$qRegisterMetaType@V?$QMap@VQString@@I@@@@YAHPBDPAV?$QMap@VQString@@I@@W4DefinedType@?$MetaTypeDefinedHelper@V?$QMap@VQString@@I@@$00@QtPrivate@@@Z$0 10020640 f   KrakenClassifyWorker.obj
 0001:0001f649       __ehhandler$??$qRegisterMetaType@V?$QMap@VQString@@I@@@@YAHPBDPAV?$QMap@VQString@@I@@W4DefinedType@?$MetaTypeDefinedHelper@V?$QMap@VQString@@I@@$00@QtPrivate@@@Z 10020649 f   KrakenClassifyWorker.obj
 0001:0001f670       __unwindfunclet$??$qRegisterMetaType@VQAssociativeIterableImpl@QtMetaTypePrivate@@@@YAHPBDPAVQAssociativeIterableImpl@QtMetaTypePrivate@@W4DefinedType@?$MetaTypeDefinedHelper@VQAssociativeIterableImpl@QtMetaTypePrivate@@$00@QtPrivate@@@Z$0 10020670 f   KrakenClassifyWorker.obj
 0001:0001f679       __ehhandler$??$qRegisterMetaType@VQAssociativeIterableImpl@QtMetaTypePrivate@@@@YAHPBDPAVQAssociativeIterableImpl@QtMetaTypePrivate@@W4DefinedType@?$MetaTypeDefinedHelper@VQAssociativeIterableImpl@QtMetaTypePrivate@@$00@QtPrivate@@@Z 10020679 f   KrakenClassifyWorker.obj
 0001:0001f6a0       __unwindfunclet$??__EalgoLog@U2@@YAXXZ$0 100206a0 f   KrakenClassifyWorker.obj
 0001:0001f6a9       __ehhandler$??__EalgoLog@U2@@YAXXZ 100206a9 f   KrakenClassifyWorker.obj
 0001:0001f6d0       __unwindfunclet$??__EcmdLog@U2@@YAXXZ$0 100206d0 f   KrakenClassifyWorker.obj
 0001:0001f6d9       __ehhandler$??__EcmdLog@U2@@YAXXZ 100206d9 f   KrakenClassifyWorker.obj
 0001:0001f700       __unwindfunclet$??__EcoreLog@U2@@YAXXZ$0 10020700 f   KrakenClassifyWorker.obj
 0001:0001f709       __ehhandler$??__EcoreLog@U2@@YAXXZ 10020709 f   KrakenClassifyWorker.obj
 0001:0001f730       __unwindfunclet$??__EioLog@U2@@YAXXZ$0 10020730 f   KrakenClassifyWorker.obj
 0001:0001f739       __ehhandler$??__EioLog@U2@@YAXXZ 10020739 f   KrakenClassifyWorker.obj
 0001:0001f760       __unwindfunclet$??__EperfLog@U2@@YAXXZ$0 10020760 f   KrakenClassifyWorker.obj
 0001:0001f769       __ehhandler$??__EperfLog@U2@@YAXXZ 10020769 f   KrakenClassifyWorker.obj
 0001:0001f790       __unwindfunclet$??__EscriptLog@U2@@YAXXZ$0 10020790 f   KrakenClassifyWorker.obj
 0001:0001f799       __ehhandler$??__EscriptLog@U2@@YAXXZ 10020799 f   KrakenClassifyWorker.obj
 0001:0001f7c0       __unwindfunclet$??__EtaskLog@U2@@YAXXZ$0 100207c0 f   KrakenClassifyWorker.obj
 0001:0001f7c9       __ehhandler$??__EtaskLog@U2@@YAXXZ 100207c9 f   KrakenClassifyWorker.obj
 0001:0001f7f0       __unwindfunclet$??__EuiLog@U2@@YAXXZ$0 100207f0 f   KrakenClassifyWorker.obj
 0001:0001f7f9       __ehhandler$??__EuiLog@U2@@YAXXZ 100207f9 f   KrakenClassifyWorker.obj
 0001:0001f820       __unwindfunclet$??__EuserActLog@U2@@YAXXZ$0 10020820 f   KrakenClassifyWorker.obj
 0001:0001f829       __ehhandler$??__EuserActLog@U2@@YAXXZ 10020829 f   KrakenClassifyWorker.obj
 0001:0001f850       __unwindfunclet$?Construct@?$QMetaTypeFunctionHelper@V?$QMap@VQString@@I@@$00@QtMetaTypePrivate@@SAPAXPAXPBX@Z$0 10020850 f   KrakenClassifyWorker.obj
 0001:0001f861       __ehhandler$?Construct@?$QMetaTypeFunctionHelper@V?$QMap@VQString@@I@@$00@QtMetaTypePrivate@@SAPAXPAXPBX@Z 10020861 f   KrakenClassifyWorker.obj
 0001:0001f880       __unwindfunclet$?Create@?$QMetaTypeFunctionHelper@V?$QMap@VQString@@I@@$00@QtMetaTypePrivate@@SAPAXPBX@Z$0 10020880 f   KrakenClassifyWorker.obj
 0001:0001f88b       __ehhandler$?Create@?$QMetaTypeFunctionHelper@V?$QMap@VQString@@I@@$00@QtMetaTypePrivate@@SAPAXPBX@Z 1002088b f   KrakenClassifyWorker.obj
 0001:0001f8b0       __unwindfunclet$?getSettings@KrakenClassifyWorker@LocalWorkflow@U2@@AAE?AUKrakenClassifyTaskSettings@3@AAVU2OpStatus@3@@Z$0 100208b0 f   KrakenClassifyWorker.obj
 0001:0001f8c9       __unwindfunclet$?getSettings@KrakenClassifyWorker@LocalWorkflow@U2@@AAE?AUKrakenClassifyTaskSettings@3@AAVU2OpStatus@3@@Z$1 100208c9 f   KrakenClassifyWorker.obj
 0001:0001f8d2       __unwindfunclet$?getSettings@KrakenClassifyWorker@LocalWorkflow@U2@@AAE?AUKrakenClassifyTaskSettings@3@AAVU2OpStatus@3@@Z$2 100208d2 f   KrakenClassifyWorker.obj
 0001:0001f8db       __unwindfunclet$?getSettings@KrakenClassifyWorker@LocalWorkflow@U2@@AAE?AUKrakenClassifyTaskSettings@3@AAVU2OpStatus@3@@Z$3 100208db f   KrakenClassifyWorker.obj
 0001:0001f8e4       __unwindfunclet$?getSettings@KrakenClassifyWorker@LocalWorkflow@U2@@AAE?AUKrakenClassifyTaskSettings@3@AAVU2OpStatus@3@@Z$4 100208e4 f   KrakenClassifyWorker.obj
 0001:0001f8ec       __unwindfunclet$?getSettings@KrakenClassifyWorker@LocalWorkflow@U2@@AAE?AUKrakenClassifyTaskSettings@3@AAVU2OpStatus@3@@Z$5 100208ec f   KrakenClassifyWorker.obj
 0001:0001f8f5       __unwindfunclet$?getSettings@KrakenClassifyWorker@LocalWorkflow@U2@@AAE?AUKrakenClassifyTaskSettings@3@AAVU2OpStatus@3@@Z$6 100208f5 f   KrakenClassifyWorker.obj
 0001:0001f8fe       __unwindfunclet$?getSettings@KrakenClassifyWorker@LocalWorkflow@U2@@AAE?AUKrakenClassifyTaskSettings@3@AAVU2OpStatus@3@@Z$7 100208fe f   KrakenClassifyWorker.obj
 0001:0001f906       __unwindfunclet$?getSettings@KrakenClassifyWorker@LocalWorkflow@U2@@AAE?AUKrakenClassifyTaskSettings@3@AAVU2OpStatus@3@@Z$8 10020906 f   KrakenClassifyWorker.obj
 0001:0001f90f       __unwindfunclet$?getSettings@KrakenClassifyWorker@LocalWorkflow@U2@@AAE?AUKrakenClassifyTaskSettings@3@AAVU2OpStatus@3@@Z$9 1002090f f   KrakenClassifyWorker.obj
 0001:0001f918       __unwindfunclet$?getSettings@KrakenClassifyWorker@LocalWorkflow@U2@@AAE?AUKrakenClassifyTaskSettings@3@AAVU2OpStatus@3@@Z$10 10020918 f   KrakenClassifyWorker.obj
 0001:0001f921       __unwindfunclet$?getSettings@KrakenClassifyWorker@LocalWorkflow@U2@@AAE?AUKrakenClassifyTaskSettings@3@AAVU2OpStatus@3@@Z$11 10020921 f   KrakenClassifyWorker.obj
 0001:0001f92a       __unwindfunclet$?getSettings@KrakenClassifyWorker@LocalWorkflow@U2@@AAE?AUKrakenClassifyTaskSettings@3@AAVU2OpStatus@3@@Z$12 1002092a f   KrakenClassifyWorker.obj
 0001:0001f933       __unwindfunclet$?getSettings@KrakenClassifyWorker@LocalWorkflow@U2@@AAE?AUKrakenClassifyTaskSettings@3@AAVU2OpStatus@3@@Z$13 10020933 f   KrakenClassifyWorker.obj
 0001:0001f93c       __unwindfunclet$?getSettings@KrakenClassifyWorker@LocalWorkflow@U2@@AAE?AUKrakenClassifyTaskSettings@3@AAVU2OpStatus@3@@Z$14 1002093c f   KrakenClassifyWorker.obj
 0001:0001f945       __unwindfunclet$?getSettings@KrakenClassifyWorker@LocalWorkflow@U2@@AAE?AUKrakenClassifyTaskSettings@3@AAVU2OpStatus@3@@Z$15 10020945 f   KrakenClassifyWorker.obj
 0001:0001f94e       __unwindfunclet$?getSettings@KrakenClassifyWorker@LocalWorkflow@U2@@AAE?AUKrakenClassifyTaskSettings@3@AAVU2OpStatus@3@@Z$16 1002094e f   KrakenClassifyWorker.obj
 0001:0001f957       __unwindfunclet$?getSettings@KrakenClassifyWorker@LocalWorkflow@U2@@AAE?AUKrakenClassifyTaskSettings@3@AAVU2OpStatus@3@@Z$17 10020957 f   KrakenClassifyWorker.obj
 0001:0001f960       __unwindfunclet$?getSettings@KrakenClassifyWorker@LocalWorkflow@U2@@AAE?AUKrakenClassifyTaskSettings@3@AAVU2OpStatus@3@@Z$18 10020960 f   KrakenClassifyWorker.obj
 0001:0001f969       __unwindfunclet$?getSettings@KrakenClassifyWorker@LocalWorkflow@U2@@AAE?AUKrakenClassifyTaskSettings@3@AAVU2OpStatus@3@@Z$19 10020969 f   KrakenClassifyWorker.obj
 0001:0001f983       __unwindfunclet$?getSettings@KrakenClassifyWorker@LocalWorkflow@U2@@AAE?AUKrakenClassifyTaskSettings@3@AAVU2OpStatus@3@@Z$20 10020983 f   KrakenClassifyWorker.obj
 0001:0001f99d       __unwindfunclet$?getSettings@KrakenClassifyWorker@LocalWorkflow@U2@@AAE?AUKrakenClassifyTaskSettings@3@AAVU2OpStatus@3@@Z$21 1002099d f   KrakenClassifyWorker.obj
 0001:0001f9b7       __unwindfunclet$?getSettings@KrakenClassifyWorker@LocalWorkflow@U2@@AAE?AUKrakenClassifyTaskSettings@3@AAVU2OpStatus@3@@Z$22 100209b7 f   KrakenClassifyWorker.obj
 0001:0001f9d1       __unwindfunclet$?getSettings@KrakenClassifyWorker@LocalWorkflow@U2@@AAE?AUKrakenClassifyTaskSettings@3@AAVU2OpStatus@3@@Z$23 100209d1 f   KrakenClassifyWorker.obj
 0001:0001f9ea       __unwindfunclet$?getSettings@KrakenClassifyWorker@LocalWorkflow@U2@@AAE?AUKrakenClassifyTaskSettings@3@AAVU2OpStatus@3@@Z$24 100209ea f   KrakenClassifyWorker.obj
 0001:0001fa04       __unwindfunclet$?getSettings@KrakenClassifyWorker@LocalWorkflow@U2@@AAE?AUKrakenClassifyTaskSettings@3@AAVU2OpStatus@3@@Z$25 10020a04 f   KrakenClassifyWorker.obj
 0001:0001fa0d       __unwindfunclet$?getSettings@KrakenClassifyWorker@LocalWorkflow@U2@@AAE?AUKrakenClassifyTaskSettings@3@AAVU2OpStatus@3@@Z$26 10020a0d f   KrakenClassifyWorker.obj
 0001:0001fa16       __unwindfunclet$?getSettings@KrakenClassifyWorker@LocalWorkflow@U2@@AAE?AUKrakenClassifyTaskSettings@3@AAVU2OpStatus@3@@Z$27 10020a16 f   KrakenClassifyWorker.obj
 0001:0001fa1f       __unwindfunclet$?getSettings@KrakenClassifyWorker@LocalWorkflow@U2@@AAE?AUKrakenClassifyTaskSettings@3@AAVU2OpStatus@3@@Z$28 10020a1f f   KrakenClassifyWorker.obj
 0001:0001fa27       __unwindfunclet$?getSettings@KrakenClassifyWorker@LocalWorkflow@U2@@AAE?AUKrakenClassifyTaskSettings@3@AAVU2OpStatus@3@@Z$29 10020a27 f   KrakenClassifyWorker.obj
 0001:0001fa30       __ehhandler$?getSettings@KrakenClassifyWorker@LocalWorkflow@U2@@AAE?AUKrakenClassifyTaskSettings@3@AAVU2OpStatus@3@@Z 10020a30 f   KrakenClassifyWorker.obj
 0001:0001fa50       __unwindfunclet$?init@KrakenClassifyWorker@LocalWorkflow@U2@@UAEXXZ$0 10020a50 f   KrakenClassifyWorker.obj
 0001:0001fa59       __unwindfunclet$?init@KrakenClassifyWorker@LocalWorkflow@U2@@UAEXXZ$1 10020a59 f   KrakenClassifyWorker.obj
 0001:0001fa62       __unwindfunclet$?init@KrakenClassifyWorker@LocalWorkflow@U2@@UAEXXZ$2 10020a62 f   KrakenClassifyWorker.obj
 0001:0001fa6b       __unwindfunclet$?init@KrakenClassifyWorker@LocalWorkflow@U2@@UAEXXZ$3 10020a6b f   KrakenClassifyWorker.obj
 0001:0001fa74       __unwindfunclet$?init@KrakenClassifyWorker@LocalWorkflow@U2@@UAEXXZ$4 10020a74 f   KrakenClassifyWorker.obj
 0001:0001fa7d       __unwindfunclet$?init@KrakenClassifyWorker@LocalWorkflow@U2@@UAEXXZ$5 10020a7d f   KrakenClassifyWorker.obj
 0001:0001fa86       __unwindfunclet$?init@KrakenClassifyWorker@LocalWorkflow@U2@@UAEXXZ$6 10020a86 f   KrakenClassifyWorker.obj
 0001:0001fa8f       __unwindfunclet$?init@KrakenClassifyWorker@LocalWorkflow@U2@@UAEXXZ$7 10020a8f f   KrakenClassifyWorker.obj
 0001:0001fa98       __unwindfunclet$?init@KrakenClassifyWorker@LocalWorkflow@U2@@UAEXXZ$8 10020a98 f   KrakenClassifyWorker.obj
 0001:0001faa1       __unwindfunclet$?init@KrakenClassifyWorker@LocalWorkflow@U2@@UAEXXZ$9 10020aa1 f   KrakenClassifyWorker.obj
 0001:0001faaa       __unwindfunclet$?init@KrakenClassifyWorker@LocalWorkflow@U2@@UAEXXZ$10 10020aaa f   KrakenClassifyWorker.obj
 0001:0001fab3       __unwindfunclet$?init@KrakenClassifyWorker@LocalWorkflow@U2@@UAEXXZ$11 10020ab3 f   KrakenClassifyWorker.obj
 0001:0001fabc       __unwindfunclet$?init@KrakenClassifyWorker@LocalWorkflow@U2@@UAEXXZ$12 10020abc f   KrakenClassifyWorker.obj
 0001:0001fac5       __unwindfunclet$?init@KrakenClassifyWorker@LocalWorkflow@U2@@UAEXXZ$13 10020ac5 f   KrakenClassifyWorker.obj
 0001:0001face       __unwindfunclet$?init@KrakenClassifyWorker@LocalWorkflow@U2@@UAEXXZ$14 10020ace f   KrakenClassifyWorker.obj
 0001:0001fad7       __ehhandler$?init@KrakenClassifyWorker@LocalWorkflow@U2@@UAEXXZ 10020ad7 f   KrakenClassifyWorker.obj
 0001:0001fb00       __unwindfunclet$?qt_metatype_id@?$QMetaTypeId@V?$QMap@VQString@@I@@@@SAHXZ$0 10020b00 f   KrakenClassifyWorker.obj
 0001:0001fb09       __ehhandler$?qt_metatype_id@?$QMetaTypeId@V?$QMap@VQString@@I@@@@SAHXZ 10020b09 f   KrakenClassifyWorker.obj
 0001:0001fb30       __unwindfunclet$?qt_metatype_id@?$QMetaTypeId@VQAssociativeIterableImpl@QtMetaTypePrivate@@@@SAHXZ$0 10020b30 f   KrakenClassifyWorker.obj
 0001:0001fb39       __ehhandler$?qt_metatype_id@?$QMetaTypeId@VQAssociativeIterableImpl@QtMetaTypePrivate@@@@SAHXZ 10020b39 f   KrakenClassifyWorker.obj
 0001:0001fb60       __unwindfunclet$?sl_taskFinished@KrakenClassifyWorker@LocalWorkflow@U2@@AAEXPAVTask@3@@Z$0 10020b60 f   KrakenClassifyWorker.obj
 0001:0001fb69       __unwindfunclet$?sl_taskFinished@KrakenClassifyWorker@LocalWorkflow@U2@@AAEXPAVTask@3@@Z$1 10020b69 f   KrakenClassifyWorker.obj
 0001:0001fb71       __unwindfunclet$?sl_taskFinished@KrakenClassifyWorker@LocalWorkflow@U2@@AAEXPAVTask@3@@Z$2 10020b71 f   KrakenClassifyWorker.obj
 0001:0001fb7a       __unwindfunclet$?sl_taskFinished@KrakenClassifyWorker@LocalWorkflow@U2@@AAEXPAVTask@3@@Z$3 10020b7a f   KrakenClassifyWorker.obj
 0001:0001fb83       __unwindfunclet$?sl_taskFinished@KrakenClassifyWorker@LocalWorkflow@U2@@AAEXPAVTask@3@@Z$5 10020b83 f   KrakenClassifyWorker.obj
 0001:0001fb8c       __unwindfunclet$?sl_taskFinished@KrakenClassifyWorker@LocalWorkflow@U2@@AAEXPAVTask@3@@Z$6 10020b8c f   KrakenClassifyWorker.obj
 0001:0001fb95       __unwindfunclet$?sl_taskFinished@KrakenClassifyWorker@LocalWorkflow@U2@@AAEXPAVTask@3@@Z$7 10020b95 f   KrakenClassifyWorker.obj
 0001:0001fb9e       __unwindfunclet$?sl_taskFinished@KrakenClassifyWorker@LocalWorkflow@U2@@AAEXPAVTask@3@@Z$8 10020b9e f   KrakenClassifyWorker.obj
 0001:0001fba7       __unwindfunclet$?sl_taskFinished@KrakenClassifyWorker@LocalWorkflow@U2@@AAEXPAVTask@3@@Z$9 10020ba7 f   KrakenClassifyWorker.obj
 0001:0001fbb0       __unwindfunclet$?sl_taskFinished@KrakenClassifyWorker@LocalWorkflow@U2@@AAEXPAVTask@3@@Z$10 10020bb0 f   KrakenClassifyWorker.obj
 0001:0001fbb9       __unwindfunclet$?sl_taskFinished@KrakenClassifyWorker@LocalWorkflow@U2@@AAEXPAVTask@3@@Z$11 10020bb9 f   KrakenClassifyWorker.obj
 0001:0001fbc2       __unwindfunclet$?sl_taskFinished@KrakenClassifyWorker@LocalWorkflow@U2@@AAEXPAVTask@3@@Z$12 10020bc2 f   KrakenClassifyWorker.obj
 0001:0001fbcb       __ehhandler$?sl_taskFinished@KrakenClassifyWorker@LocalWorkflow@U2@@AAEXPAVTask@3@@Z 10020bcb f   KrakenClassifyWorker.obj
 0001:0001fbf0       __unwindfunclet$?tick@KrakenClassifyWorker@LocalWorkflow@U2@@UAEPAVTask@3@XZ$0 10020bf0 f   KrakenClassifyWorker.obj
 0001:0001fbf9       __unwindfunclet$?tick@KrakenClassifyWorker@LocalWorkflow@U2@@UAEPAVTask@3@XZ$1 10020bf9 f   KrakenClassifyWorker.obj
 0001:0001fc01       __unwindfunclet$?tick@KrakenClassifyWorker@LocalWorkflow@U2@@UAEPAVTask@3@XZ$2 10020c01 f   KrakenClassifyWorker.obj
 0001:0001fc0c       __unwindfunclet$?tick@KrakenClassifyWorker@LocalWorkflow@U2@@UAEPAVTask@3@XZ$3 10020c0c f   KrakenClassifyWorker.obj
 0001:0001fc26       __unwindfunclet$?tick@KrakenClassifyWorker@LocalWorkflow@U2@@UAEPAVTask@3@XZ$4 10020c26 f   KrakenClassifyWorker.obj
 0001:0001fc31       __unwindfunclet$?tick@KrakenClassifyWorker@LocalWorkflow@U2@@UAEPAVTask@3@XZ$5 10020c31 f   KrakenClassifyWorker.obj
 0001:0001fc39       __unwindfunclet$?tick@KrakenClassifyWorker@LocalWorkflow@U2@@UAEPAVTask@3@XZ$6 10020c39 f   KrakenClassifyWorker.obj
 0001:0001fc44       __unwindfunclet$?tick@KrakenClassifyWorker@LocalWorkflow@U2@@UAEPAVTask@3@XZ$8 10020c44 f   KrakenClassifyWorker.obj
 0001:0001fc4d       __unwindfunclet$?tick@KrakenClassifyWorker@LocalWorkflow@U2@@UAEPAVTask@3@XZ$9 10020c4d f   KrakenClassifyWorker.obj
 0001:0001fc56       __unwindfunclet$?tick@KrakenClassifyWorker@LocalWorkflow@U2@@UAEPAVTask@3@XZ$10 10020c56 f   KrakenClassifyWorker.obj
 0001:0001fc5f       __ehhandler$?tick@KrakenClassifyWorker@LocalWorkflow@U2@@UAEPAVTask@3@XZ 10020c5f f   KrakenClassifyWorker.obj
 0001:0001fc80       __unwindfunclet$??__EalgoLog@U2@@YAXXZ$0 10020c80 f   KrakenClassifyWorkerFactory.obj
 0001:0001fc89       __ehhandler$??__EalgoLog@U2@@YAXXZ 10020c89 f   KrakenClassifyWorkerFactory.obj
 0001:0001fcb0       __unwindfunclet$??__EcmdLog@U2@@YAXXZ$0 10020cb0 f   KrakenClassifyWorkerFactory.obj
 0001:0001fcb9       __ehhandler$??__EcmdLog@U2@@YAXXZ 10020cb9 f   KrakenClassifyWorkerFactory.obj
 0001:0001fce0       __unwindfunclet$??__EcoreLog@U2@@YAXXZ$0 10020ce0 f   KrakenClassifyWorkerFactory.obj
 0001:0001fce9       __ehhandler$??__EcoreLog@U2@@YAXXZ 10020ce9 f   KrakenClassifyWorkerFactory.obj
 0001:0001fd10       __unwindfunclet$??__EioLog@U2@@YAXXZ$0 10020d10 f   KrakenClassifyWorkerFactory.obj
 0001:0001fd19       __ehhandler$??__EioLog@U2@@YAXXZ 10020d19 f   KrakenClassifyWorkerFactory.obj
 0001:0001fd40       __unwindfunclet$??__EperfLog@U2@@YAXXZ$0 10020d40 f   KrakenClassifyWorkerFactory.obj
 0001:0001fd49       __ehhandler$??__EperfLog@U2@@YAXXZ 10020d49 f   KrakenClassifyWorkerFactory.obj
 0001:0001fd70       __unwindfunclet$??__EscriptLog@U2@@YAXXZ$0 10020d70 f   KrakenClassifyWorkerFactory.obj
 0001:0001fd79       __ehhandler$??__EscriptLog@U2@@YAXXZ 10020d79 f   KrakenClassifyWorkerFactory.obj
 0001:0001fda0       __unwindfunclet$??__EtaskLog@U2@@YAXXZ$0 10020da0 f   KrakenClassifyWorkerFactory.obj
 0001:0001fda9       __ehhandler$??__EtaskLog@U2@@YAXXZ 10020da9 f   KrakenClassifyWorkerFactory.obj
 0001:0001fdd0       __unwindfunclet$??__EuiLog@U2@@YAXXZ$0 10020dd0 f   KrakenClassifyWorkerFactory.obj
 0001:0001fdd9       __ehhandler$??__EuiLog@U2@@YAXXZ 10020dd9 f   KrakenClassifyWorkerFactory.obj
 0001:0001fe00       __unwindfunclet$??__EuserActLog@U2@@YAXXZ$0 10020e00 f   KrakenClassifyWorkerFactory.obj
 0001:0001fe09       __ehhandler$??__EuserActLog@U2@@YAXXZ 10020e09 f   KrakenClassifyWorkerFactory.obj
 0001:0001fe30       __unwindfunclet$?append@?$QList@VQVariant@@@@QAEXABVQVariant@@@Z$6 10020e30 f   KrakenClassifyWorkerFactory.obj
 0001:0001fe3b       __ehhandler$?append@?$QList@VQVariant@@@@QAEXABVQVariant@@@Z 10020e3b f   KrakenClassifyWorkerFactory.obj
 0001:0001fe60       __unwindfunclet$?createWorker@KrakenClassifyWorkerFactory@LocalWorkflow@U2@@UAEPAVWorker@Workflow@3@PAVActor@53@@Z$0 10020e60 f   KrakenClassifyWorkerFactory.obj
 0001:0001fe6b       __ehhandler$?createWorker@KrakenClassifyWorkerFactory@LocalWorkflow@U2@@UAEPAVWorker@Workflow@3@PAVActor@53@@Z 10020e6b f   KrakenClassifyWorkerFactory.obj
 0001:0001fe90       __ehhandler$?detach_helper_grow@?$QList@VQVariant@@@@AAEPAUNode@1@HH@Z 10020e90 f   KrakenClassifyWorkerFactory.obj
 0001:0001feb0       __unwindfunclet$?init@KrakenClassifyWorkerFactory@LocalWorkflow@U2@@SAXXZ$0 10020eb0 f   KrakenClassifyWorkerFactory.obj
 0001:0001feb8       __unwindfunclet$?init@KrakenClassifyWorkerFactory@LocalWorkflow@U2@@SAXXZ$1 10020eb8 f   KrakenClassifyWorkerFactory.obj
 0001:0001fec1       __unwindfunclet$?init@KrakenClassifyWorkerFactory@LocalWorkflow@U2@@SAXXZ$2 10020ec1 f   KrakenClassifyWorkerFactory.obj
 0001:0001feca       __unwindfunclet$?init@KrakenClassifyWorkerFactory@LocalWorkflow@U2@@SAXXZ$3 10020eca f   KrakenClassifyWorkerFactory.obj
 0001:0001fed3       __unwindfunclet$?init@KrakenClassifyWorkerFactory@LocalWorkflow@U2@@SAXXZ$4 10020ed3 f   KrakenClassifyWorkerFactory.obj
 0001:0001fedc       __unwindfunclet$?init@KrakenClassifyWorkerFactory@LocalWorkflow@U2@@SAXXZ$5 10020edc f   KrakenClassifyWorkerFactory.obj
 0001:0001fee5       __unwindfunclet$?init@KrakenClassifyWorkerFactory@LocalWorkflow@U2@@SAXXZ$6 10020ee5 f   KrakenClassifyWorkerFactory.obj
 0001:0001fef1       __unwindfunclet$?init@KrakenClassifyWorkerFactory@LocalWorkflow@U2@@SAXXZ$7 10020ef1 f   KrakenClassifyWorkerFactory.obj
 0001:0001fef9       __unwindfunclet$?init@KrakenClassifyWorkerFactory@LocalWorkflow@U2@@SAXXZ$8 10020ef9 f   KrakenClassifyWorkerFactory.obj
 0001:0001ff01       __unwindfunclet$?init@KrakenClassifyWorkerFactory@LocalWorkflow@U2@@SAXXZ$9 10020f01 f   KrakenClassifyWorkerFactory.obj
 0001:0001ff09       __unwindfunclet$?init@KrakenClassifyWorkerFactory@LocalWorkflow@U2@@SAXXZ$10 10020f09 f   KrakenClassifyWorkerFactory.obj
 0001:0001ff11       __unwindfunclet$?init@KrakenClassifyWorkerFactory@LocalWorkflow@U2@@SAXXZ$11 10020f11 f   KrakenClassifyWorkerFactory.obj
 0001:0001ff19       __unwindfunclet$?init@KrakenClassifyWorkerFactory@LocalWorkflow@U2@@SAXXZ$12 10020f19 f   KrakenClassifyWorkerFactory.obj
 0001:0001ff22       __unwindfunclet$?init@KrakenClassifyWorkerFactory@LocalWorkflow@U2@@SAXXZ$13 10020f22 f   KrakenClassifyWorkerFactory.obj
 0001:0001ff2b       __unwindfunclet$?init@KrakenClassifyWorkerFactory@LocalWorkflow@U2@@SAXXZ$14 10020f2b f   KrakenClassifyWorkerFactory.obj
 0001:0001ff34       __unwindfunclet$?init@KrakenClassifyWorkerFactory@LocalWorkflow@U2@@SAXXZ$15 10020f34 f   KrakenClassifyWorkerFactory.obj
 0001:0001ff40       __unwindfunclet$?init@KrakenClassifyWorkerFactory@LocalWorkflow@U2@@SAXXZ$16 10020f40 f   KrakenClassifyWorkerFactory.obj
 0001:0001ff49       __unwindfunclet$?init@KrakenClassifyWorkerFactory@LocalWorkflow@U2@@SAXXZ$17 10020f49 f   KrakenClassifyWorkerFactory.obj
 0001:0001ff52       __unwindfunclet$?init@KrakenClassifyWorkerFactory@LocalWorkflow@U2@@SAXXZ$18 10020f52 f   KrakenClassifyWorkerFactory.obj
 0001:0001ff5e       __unwindfunclet$?init@KrakenClassifyWorkerFactory@LocalWorkflow@U2@@SAXXZ$19 10020f5e f   KrakenClassifyWorkerFactory.obj
 0001:0001ff69       __unwindfunclet$?init@KrakenClassifyWorkerFactory@LocalWorkflow@U2@@SAXXZ$20 10020f69 f   KrakenClassifyWorkerFactory.obj
 0001:0001ff74       __unwindfunclet$?init@KrakenClassifyWorkerFactory@LocalWorkflow@U2@@SAXXZ$21 10020f74 f   KrakenClassifyWorkerFactory.obj
 0001:0001ff8e       __unwindfunclet$?init@KrakenClassifyWorkerFactory@LocalWorkflow@U2@@SAXXZ$22 10020f8e f   KrakenClassifyWorkerFactory.obj
 0001:0001ffab       __unwindfunclet$?init@KrakenClassifyWorkerFactory@LocalWorkflow@U2@@SAXXZ$24 10020fab f   KrakenClassifyWorkerFactory.obj
 0001:0001ffb6       __unwindfunclet$?init@KrakenClassifyWorkerFactory@LocalWorkflow@U2@@SAXXZ$25 10020fb6 f   KrakenClassifyWorkerFactory.obj
 0001:0001ffc1       __unwindfunclet$?init@KrakenClassifyWorkerFactory@LocalWorkflow@U2@@SAXXZ$26 10020fc1 f   KrakenClassifyWorkerFactory.obj
 0001:0001ffdb       __unwindfunclet$?init@KrakenClassifyWorkerFactory@LocalWorkflow@U2@@SAXXZ$27 10020fdb f   KrakenClassifyWorkerFactory.obj
 0001:0001fff8       __unwindfunclet$?init@KrakenClassifyWorkerFactory@LocalWorkflow@U2@@SAXXZ$29 10020ff8 f   KrakenClassifyWorkerFactory.obj
 0001:00020000       __unwindfunclet$?init@KrakenClassifyWorkerFactory@LocalWorkflow@U2@@SAXXZ$30 10021000 f   KrakenClassifyWorkerFactory.obj
 0001:00020009       __unwindfunclet$?init@KrakenClassifyWorkerFactory@LocalWorkflow@U2@@SAXXZ$31 10021009 f   KrakenClassifyWorkerFactory.obj
 0001:00020012       __unwindfunclet$?init@KrakenClassifyWorkerFactory@LocalWorkflow@U2@@SAXXZ$32 10021012 f   KrakenClassifyWorkerFactory.obj
 0001:0002001e       __unwindfunclet$?init@KrakenClassifyWorkerFactory@LocalWorkflow@U2@@SAXXZ$33 1002101e f   KrakenClassifyWorkerFactory.obj
 0001:00020027       __unwindfunclet$?init@KrakenClassifyWorkerFactory@LocalWorkflow@U2@@SAXXZ$34 10021027 f   KrakenClassifyWorkerFactory.obj
 0001:00020030       __unwindfunclet$?init@KrakenClassifyWorkerFactory@LocalWorkflow@U2@@SAXXZ$35 10021030 f   KrakenClassifyWorkerFactory.obj
 0001:0002003c       __unwindfunclet$?init@KrakenClassifyWorkerFactory@LocalWorkflow@U2@@SAXXZ$36 1002103c f   KrakenClassifyWorkerFactory.obj
 0001:00020045       __unwindfunclet$?init@KrakenClassifyWorkerFactory@LocalWorkflow@U2@@SAXXZ$37 10021045 f   KrakenClassifyWorkerFactory.obj
 0001:0002004e       __unwindfunclet$?init@KrakenClassifyWorkerFactory@LocalWorkflow@U2@@SAXXZ$38 1002104e f   KrakenClassifyWorkerFactory.obj
 0001:0002005a       __unwindfunclet$?init@KrakenClassifyWorkerFactory@LocalWorkflow@U2@@SAXXZ$39 1002105a f   KrakenClassifyWorkerFactory.obj
 0001:00020063       __unwindfunclet$?init@KrakenClassifyWorkerFactory@LocalWorkflow@U2@@SAXXZ$40 10021063 f   KrakenClassifyWorkerFactory.obj
 0001:0002006c       __unwindfunclet$?init@KrakenClassifyWorkerFactory@LocalWorkflow@U2@@SAXXZ$41 1002106c f   KrakenClassifyWorkerFactory.obj
 0001:00020078       __unwindfunclet$?init@KrakenClassifyWorkerFactory@LocalWorkflow@U2@@SAXXZ$42 10021078 f   KrakenClassifyWorkerFactory.obj
 0001:00020084       __unwindfunclet$?init@KrakenClassifyWorkerFactory@LocalWorkflow@U2@@SAXXZ$43 10021084 f   KrakenClassifyWorkerFactory.obj
 0001:00020090       __unwindfunclet$?init@KrakenClassifyWorkerFactory@LocalWorkflow@U2@@SAXXZ$44 10021090 f   KrakenClassifyWorkerFactory.obj
 0001:0002009c       __unwindfunclet$?init@KrakenClassifyWorkerFactory@LocalWorkflow@U2@@SAXXZ$45 1002109c f   KrakenClassifyWorkerFactory.obj
 0001:000200a8       __unwindfunclet$?init@KrakenClassifyWorkerFactory@LocalWorkflow@U2@@SAXXZ$46 100210a8 f   KrakenClassifyWorkerFactory.obj
 0001:000200b4       __unwindfunclet$?init@KrakenClassifyWorkerFactory@LocalWorkflow@U2@@SAXXZ$47 100210b4 f   KrakenClassifyWorkerFactory.obj
 0001:000200c0       __unwindfunclet$?init@KrakenClassifyWorkerFactory@LocalWorkflow@U2@@SAXXZ$48 100210c0 f   KrakenClassifyWorkerFactory.obj
 0001:000200c9       __unwindfunclet$?init@KrakenClassifyWorkerFactory@LocalWorkflow@U2@@SAXXZ$49 100210c9 f   KrakenClassifyWorkerFactory.obj
 0001:000200d5       __unwindfunclet$?init@KrakenClassifyWorkerFactory@LocalWorkflow@U2@@SAXXZ$50 100210d5 f   KrakenClassifyWorkerFactory.obj
 0001:000200e1       __unwindfunclet$?init@KrakenClassifyWorkerFactory@LocalWorkflow@U2@@SAXXZ$51 100210e1 f   KrakenClassifyWorkerFactory.obj
 0001:000200ea       __unwindfunclet$?init@KrakenClassifyWorkerFactory@LocalWorkflow@U2@@SAXXZ$52 100210ea f   KrakenClassifyWorkerFactory.obj
 0001:000200f6       __unwindfunclet$?init@KrakenClassifyWorkerFactory@LocalWorkflow@U2@@SAXXZ$53 100210f6 f   KrakenClassifyWorkerFactory.obj
 0001:00020101       __unwindfunclet$?init@KrakenClassifyWorkerFactory@LocalWorkflow@U2@@SAXXZ$54 10021101 f   KrakenClassifyWorkerFactory.obj
 0001:0002011b       __unwindfunclet$?init@KrakenClassifyWorkerFactory@LocalWorkflow@U2@@SAXXZ$56 1002111b f   KrakenClassifyWorkerFactory.obj
 0001:00020126       __unwindfunclet$?init@KrakenClassifyWorkerFactory@LocalWorkflow@U2@@SAXXZ$57 10021126 f   KrakenClassifyWorkerFactory.obj
 0001:00020140       __unwindfunclet$?init@KrakenClassifyWorkerFactory@LocalWorkflow@U2@@SAXXZ$58 10021140 f   KrakenClassifyWorkerFactory.obj
 0001:00020159       __unwindfunclet$?init@KrakenClassifyWorkerFactory@LocalWorkflow@U2@@SAXXZ$59 10021159 f   KrakenClassifyWorkerFactory.obj
 0001:00020162       __unwindfunclet$?init@KrakenClassifyWorkerFactory@LocalWorkflow@U2@@SAXXZ$60 10021162 f   KrakenClassifyWorkerFactory.obj
 0001:0002016b       __unwindfunclet$?init@KrakenClassifyWorkerFactory@LocalWorkflow@U2@@SAXXZ$61 1002116b f   KrakenClassifyWorkerFactory.obj
 0001:00020176       __unwindfunclet$?init@KrakenClassifyWorkerFactory@LocalWorkflow@U2@@SAXXZ$62 10021176 f   KrakenClassifyWorkerFactory.obj
 0001:00020195       __unwindfunclet$?init@KrakenClassifyWorkerFactory@LocalWorkflow@U2@@SAXXZ$64 10021195 f   KrakenClassifyWorkerFactory.obj
 0001:000201a0       __unwindfunclet$?init@KrakenClassifyWorkerFactory@LocalWorkflow@U2@@SAXXZ$65 100211a0 f   KrakenClassifyWorkerFactory.obj
 0001:000201bf       __unwindfunclet$?init@KrakenClassifyWorkerFactory@LocalWorkflow@U2@@SAXXZ$67 100211bf f   KrakenClassifyWorkerFactory.obj
 0001:000201ca       __unwindfunclet$?init@KrakenClassifyWorkerFactory@LocalWorkflow@U2@@SAXXZ$68 100211ca f   KrakenClassifyWorkerFactory.obj
 0001:000201e9       __unwindfunclet$?init@KrakenClassifyWorkerFactory@LocalWorkflow@U2@@SAXXZ$70 100211e9 f   KrakenClassifyWorkerFactory.obj
 0001:000201f4       __unwindfunclet$?init@KrakenClassifyWorkerFactory@LocalWorkflow@U2@@SAXXZ$71 100211f4 f   KrakenClassifyWorkerFactory.obj
 0001:00020213       __unwindfunclet$?init@KrakenClassifyWorkerFactory@LocalWorkflow@U2@@SAXXZ$73 10021213 f   KrakenClassifyWorkerFactory.obj
 0001:0002021e       __unwindfunclet$?init@KrakenClassifyWorkerFactory@LocalWorkflow@U2@@SAXXZ$74 1002121e f   KrakenClassifyWorkerFactory.obj
 0001:0002023d       __unwindfunclet$?init@KrakenClassifyWorkerFactory@LocalWorkflow@U2@@SAXXZ$76 1002123d f   KrakenClassifyWorkerFactory.obj
 0001:00020248       __unwindfunclet$?init@KrakenClassifyWorkerFactory@LocalWorkflow@U2@@SAXXZ$77 10021248 f   KrakenClassifyWorkerFactory.obj
 0001:00020267       __unwindfunclet$?init@KrakenClassifyWorkerFactory@LocalWorkflow@U2@@SAXXZ$79 10021267 f   KrakenClassifyWorkerFactory.obj
 0001:00020272       __unwindfunclet$?init@KrakenClassifyWorkerFactory@LocalWorkflow@U2@@SAXXZ$80 10021272 f   KrakenClassifyWorkerFactory.obj
 0001:00020291       __unwindfunclet$?init@KrakenClassifyWorkerFactory@LocalWorkflow@U2@@SAXXZ$82 10021291 f   KrakenClassifyWorkerFactory.obj
 0001:0002029c       __unwindfunclet$?init@KrakenClassifyWorkerFactory@LocalWorkflow@U2@@SAXXZ$83 1002129c f   KrakenClassifyWorkerFactory.obj
 0001:000202bb       __unwindfunclet$?init@KrakenClassifyWorkerFactory@LocalWorkflow@U2@@SAXXZ$84 100212bb f   KrakenClassifyWorkerFactory.obj
 0001:000202c6       __unwindfunclet$?init@KrakenClassifyWorkerFactory@LocalWorkflow@U2@@SAXXZ$85 100212c6 f   KrakenClassifyWorkerFactory.obj
 0001:000202ce       __unwindfunclet$?init@KrakenClassifyWorkerFactory@LocalWorkflow@U2@@SAXXZ$86 100212ce f   KrakenClassifyWorkerFactory.obj
 0001:000202d6       __unwindfunclet$?init@KrakenClassifyWorkerFactory@LocalWorkflow@U2@@SAXXZ$87 100212d6 f   KrakenClassifyWorkerFactory.obj
 0001:000202df       __unwindfunclet$?init@KrakenClassifyWorkerFactory@LocalWorkflow@U2@@SAXXZ$88 100212df f   KrakenClassifyWorkerFactory.obj
 0001:000202e8       __unwindfunclet$?init@KrakenClassifyWorkerFactory@LocalWorkflow@U2@@SAXXZ$89 100212e8 f   KrakenClassifyWorkerFactory.obj
 0001:000202f3       __unwindfunclet$?init@KrakenClassifyWorkerFactory@LocalWorkflow@U2@@SAXXZ$90 100212f3 f   KrakenClassifyWorkerFactory.obj
 0001:000202fe       __unwindfunclet$?init@KrakenClassifyWorkerFactory@LocalWorkflow@U2@@SAXXZ$91 100212fe f   KrakenClassifyWorkerFactory.obj
 0001:0002031d       __unwindfunclet$?init@KrakenClassifyWorkerFactory@LocalWorkflow@U2@@SAXXZ$92 1002131d f   KrakenClassifyWorkerFactory.obj
 0001:00020329       __unwindfunclet$?init@KrakenClassifyWorkerFactory@LocalWorkflow@U2@@SAXXZ$93 10021329 f   KrakenClassifyWorkerFactory.obj
 0001:00020332       __unwindfunclet$?init@KrakenClassifyWorkerFactory@LocalWorkflow@U2@@SAXXZ$94 10021332 f   KrakenClassifyWorkerFactory.obj
 0001:0002033a       __unwindfunclet$?init@KrakenClassifyWorkerFactory@LocalWorkflow@U2@@SAXXZ$95 1002133a f   KrakenClassifyWorkerFactory.obj
 0001:00020343       __unwindfunclet$?init@KrakenClassifyWorkerFactory@LocalWorkflow@U2@@SAXXZ$96 10021343 f   KrakenClassifyWorkerFactory.obj
 0001:0002034c       __unwindfunclet$?init@KrakenClassifyWorkerFactory@LocalWorkflow@U2@@SAXXZ$97 1002134c f   KrakenClassifyWorkerFactory.obj
 0001:00020358       __unwindfunclet$?init@KrakenClassifyWorkerFactory@LocalWorkflow@U2@@SAXXZ$98 10021358 f   KrakenClassifyWorkerFactory.obj
 0001:00020363       __unwindfunclet$?init@KrakenClassifyWorkerFactory@LocalWorkflow@U2@@SAXXZ$99 10021363 f   KrakenClassifyWorkerFactory.obj
 0001:00020382       __unwindfunclet$?init@KrakenClassifyWorkerFactory@LocalWorkflow@U2@@SAXXZ$100 10021382 f   KrakenClassifyWorkerFactory.obj
 0001:0002038d       __unwindfunclet$?init@KrakenClassifyWorkerFactory@LocalWorkflow@U2@@SAXXZ$101 1002138d f   KrakenClassifyWorkerFactory.obj
 0001:00020395       __unwindfunclet$?init@KrakenClassifyWorkerFactory@LocalWorkflow@U2@@SAXXZ$102 10021395 f   KrakenClassifyWorkerFactory.obj
 0001:0002039e       __unwindfunclet$?init@KrakenClassifyWorkerFactory@LocalWorkflow@U2@@SAXXZ$103 1002139e f   KrakenClassifyWorkerFactory.obj
 0001:000203a7       __unwindfunclet$?init@KrakenClassifyWorkerFactory@LocalWorkflow@U2@@SAXXZ$104 100213a7 f   KrakenClassifyWorkerFactory.obj
 0001:000203b0       __unwindfunclet$?init@KrakenClassifyWorkerFactory@LocalWorkflow@U2@@SAXXZ$105 100213b0 f   KrakenClassifyWorkerFactory.obj
 0001:000203b9       __unwindfunclet$?init@KrakenClassifyWorkerFactory@LocalWorkflow@U2@@SAXXZ$106 100213b9 f   KrakenClassifyWorkerFactory.obj
 0001:000203c4       __unwindfunclet$?init@KrakenClassifyWorkerFactory@LocalWorkflow@U2@@SAXXZ$107 100213c4 f   KrakenClassifyWorkerFactory.obj
 0001:000203cf       __unwindfunclet$?init@KrakenClassifyWorkerFactory@LocalWorkflow@U2@@SAXXZ$108 100213cf f   KrakenClassifyWorkerFactory.obj
 0001:000203d8       __unwindfunclet$?init@KrakenClassifyWorkerFactory@LocalWorkflow@U2@@SAXXZ$109 100213d8 f   KrakenClassifyWorkerFactory.obj
 0001:000203e1       __unwindfunclet$?init@KrakenClassifyWorkerFactory@LocalWorkflow@U2@@SAXXZ$110 100213e1 f   KrakenClassifyWorkerFactory.obj
 0001:000203ed       __unwindfunclet$?init@KrakenClassifyWorkerFactory@LocalWorkflow@U2@@SAXXZ$111 100213ed f   KrakenClassifyWorkerFactory.obj
 0001:000203f8       __unwindfunclet$?init@KrakenClassifyWorkerFactory@LocalWorkflow@U2@@SAXXZ$112 100213f8 f   KrakenClassifyWorkerFactory.obj
 0001:00020403       __unwindfunclet$?init@KrakenClassifyWorkerFactory@LocalWorkflow@U2@@SAXXZ$113 10021403 f   KrakenClassifyWorkerFactory.obj
 0001:0002040e       __unwindfunclet$?init@KrakenClassifyWorkerFactory@LocalWorkflow@U2@@SAXXZ$114 1002140e f   KrakenClassifyWorkerFactory.obj
 0001:00020417       __unwindfunclet$?init@KrakenClassifyWorkerFactory@LocalWorkflow@U2@@SAXXZ$115 10021417 f   KrakenClassifyWorkerFactory.obj
 0001:00020422       __unwindfunclet$?init@KrakenClassifyWorkerFactory@LocalWorkflow@U2@@SAXXZ$116 10021422 f   KrakenClassifyWorkerFactory.obj
 0001:0002042b       __unwindfunclet$?init@KrakenClassifyWorkerFactory@LocalWorkflow@U2@@SAXXZ$117 1002142b f   KrakenClassifyWorkerFactory.obj
 0001:00020436       __ehhandler$?init@KrakenClassifyWorkerFactory@LocalWorkflow@U2@@SAXXZ 10021436 f   KrakenClassifyWorkerFactory.obj
 0001:00020460       __unwindfunclet$?node_construct@?$QList@VQVariant@@@@AAEXPAUNode@1@ABVQVariant@@@Z$0 10021460 f   KrakenClassifyWorkerFactory.obj
 0001:0002046b       __ehhandler$?node_construct@?$QList@VQVariant@@@@AAEXPAUNode@1@ABVQVariant@@@Z 1002146b f   KrakenClassifyWorkerFactory.obj
 0001:00020490       __unwindfunclet$?node_copy@?$QList@VQVariant@@@@AAEXPAUNode@1@00@Z$4 10021490 f   KrakenClassifyWorkerFactory.obj
 0001:0002049b       __ehhandler$?node_copy@?$QList@VQVariant@@@@AAEXPAUNode@1@00@Z 1002149b f   KrakenClassifyWorkerFactory.obj
 0001:000204c0       __unwindfunclet$??0KrakenSupport@U2@@QAE@ABVQString@@0@Z$0 100214c0 f   KrakenSupport.obj
 0001:000204c9       __unwindfunclet$??0KrakenSupport@U2@@QAE@ABVQString@@0@Z$1 100214c9 f   KrakenSupport.obj
 0001:000204d2       __unwindfunclet$??0KrakenSupport@U2@@QAE@ABVQString@@0@Z$3 100214d2 f   KrakenSupport.obj
 0001:000204db       __unwindfunclet$??0KrakenSupport@U2@@QAE@ABVQString@@0@Z$4 100214db f   KrakenSupport.obj
 0001:000204e4       __unwindfunclet$??0KrakenSupport@U2@@QAE@ABVQString@@0@Z$5 100214e4 f   KrakenSupport.obj
 0001:000204ed       __unwindfunclet$??0KrakenSupport@U2@@QAE@ABVQString@@0@Z$6 100214ed f   KrakenSupport.obj
 0001:000204f6       __unwindfunclet$??0KrakenSupport@U2@@QAE@ABVQString@@0@Z$7 100214f6 f   KrakenSupport.obj
 0001:000204ff       __unwindfunclet$??0KrakenSupport@U2@@QAE@ABVQString@@0@Z$8 100214ff f   KrakenSupport.obj
 0001:00020508       __unwindfunclet$??0KrakenSupport@U2@@QAE@ABVQString@@0@Z$9 10021508 f   KrakenSupport.obj
 0001:00020511       __ehhandler$??0KrakenSupport@U2@@QAE@ABVQString@@0@Z 10021511 f   KrakenSupport.obj
 0001:00020530       __unwindfunclet$?getAdditionalPaths@KrakenSupport@U2@@UBE?AVQStringList@@XZ$0 10021530 f   KrakenSupport.obj
 0001:00020539       __unwindfunclet$?getAdditionalPaths@KrakenSupport@U2@@UBE?AVQStringList@@XZ$1 10021539 f   KrakenSupport.obj
 0001:00020542       __unwindfunclet$?getAdditionalPaths@KrakenSupport@U2@@UBE?AVQStringList@@XZ$2 10021542 f   KrakenSupport.obj
 0001:0002054b       __unwindfunclet$?getAdditionalPaths@KrakenSupport@U2@@UBE?AVQStringList@@XZ$3 1002154b f   KrakenSupport.obj
 0001:00020554       __unwindfunclet$?getAdditionalPaths@KrakenSupport@U2@@UBE?AVQStringList@@XZ$4 10021554 f   KrakenSupport.obj
 0001:0002055d       __unwindfunclet$?getAdditionalPaths@KrakenSupport@U2@@UBE?AVQStringList@@XZ$5 1002155d f   KrakenSupport.obj
 0001:00020566       __unwindfunclet$?getAdditionalPaths@KrakenSupport@U2@@UBE?AVQStringList@@XZ$6 10021566 f   KrakenSupport.obj
 0001:0002056f       __unwindfunclet$?getAdditionalPaths@KrakenSupport@U2@@UBE?AVQStringList@@XZ$7 1002156f f   KrakenSupport.obj
 0001:00020578       __unwindfunclet$?getAdditionalPaths@KrakenSupport@U2@@UBE?AVQStringList@@XZ$8 10021578 f   KrakenSupport.obj
 0001:00020580       __ehhandler$?getAdditionalPaths@KrakenSupport@U2@@UBE?AVQStringList@@XZ 10021580 f   KrakenSupport.obj
 0001:000205a0       __unwindfunclet$?initBuild@KrakenSupport@U2@@AAEXXZ$0 100215a0 f   KrakenSupport.obj
 0001:000205a9       __ehhandler$?initBuild@KrakenSupport@U2@@AAEXXZ 100215a9 f   KrakenSupport.obj
 0001:000205d0       __unwindfunclet$?initClassify@KrakenSupport@U2@@AAEXXZ$0 100215d0 f   KrakenSupport.obj
 0001:000205d9       __ehhandler$?initClassify@KrakenSupport@U2@@AAEXXZ 100215d9 f   KrakenSupport.obj
 0001:00020600       __unwindfunclet$??0KrakenSupportPlugin@U2@@QAE@XZ$0 10021600 f   KrakenSupportPlugin.obj
 0001:00020609       __unwindfunclet$??0KrakenSupportPlugin@U2@@QAE@XZ$1 10021609 f   KrakenSupportPlugin.obj
 0001:00020614       __unwindfunclet$??0KrakenSupportPlugin@U2@@QAE@XZ$2 10021614 f   KrakenSupportPlugin.obj
 0001:0002061f       __unwindfunclet$??0KrakenSupportPlugin@U2@@QAE@XZ$3 1002161f f   KrakenSupportPlugin.obj
 0001:00020628       __ehhandler$??0KrakenSupportPlugin@U2@@QAE@XZ 10021628 f   KrakenSupportPlugin.obj
 0001:00020650       __unwindfunclet$??1KrakenSupportPlugin@U2@@UAE@XZ$0 10021650 f   KrakenSupportPlugin.obj
 0001:00020659       __ehhandler$??1KrakenSupportPlugin@U2@@UAE@XZ 10021659 f   KrakenSupportPlugin.obj
 0001:00020680       __unwindfunclet$??_GKrakenSupportPlugin@U2@@UAEPAXI@Z$0 10021680 f   KrakenSupportPlugin.obj
 0001:00020689       __ehhandler$??_GKrakenSupportPlugin@U2@@UAEPAXI@Z 10021689 f   KrakenSupportPlugin.obj
 0001:000206b0       __unwindfunclet$??__EalgoLog@U2@@YAXXZ$0 100216b0 f   KrakenSupportPlugin.obj
 0001:000206b9       __ehhandler$??__EalgoLog@U2@@YAXXZ 100216b9 f   KrakenSupportPlugin.obj
 0001:000206e0       __unwindfunclet$??__EcmdLog@U2@@YAXXZ$0 100216e0 f   KrakenSupportPlugin.obj
 0001:000206e9       __ehhandler$??__EcmdLog@U2@@YAXXZ 100216e9 f   KrakenSupportPlugin.obj
 0001:00020710       __unwindfunclet$??__EcoreLog@U2@@YAXXZ$0 10021710 f   KrakenSupportPlugin.obj
 0001:00020719       __ehhandler$??__EcoreLog@U2@@YAXXZ 10021719 f   KrakenSupportPlugin.obj
 0001:00020740       __unwindfunclet$??__EioLog@U2@@YAXXZ$0 10021740 f   KrakenSupportPlugin.obj
 0001:00020749       __ehhandler$??__EioLog@U2@@YAXXZ 10021749 f   KrakenSupportPlugin.obj
 0001:00020770       __unwindfunclet$??__EperfLog@U2@@YAXXZ$0 10021770 f   KrakenSupportPlugin.obj
 0001:00020779       __ehhandler$??__EperfLog@U2@@YAXXZ 10021779 f   KrakenSupportPlugin.obj
 0001:000207a0       __unwindfunclet$??__EscriptLog@U2@@YAXXZ$0 100217a0 f   KrakenSupportPlugin.obj
 0001:000207a9       __ehhandler$??__EscriptLog@U2@@YAXXZ 100217a9 f   KrakenSupportPlugin.obj
 0001:000207d0       __unwindfunclet$??__EtaskLog@U2@@YAXXZ$0 100217d0 f   KrakenSupportPlugin.obj
 0001:000207d9       __ehhandler$??__EtaskLog@U2@@YAXXZ 100217d9 f   KrakenSupportPlugin.obj
 0001:00020800       __unwindfunclet$??__EuiLog@U2@@YAXXZ$0 10021800 f   KrakenSupportPlugin.obj
 0001:00020809       __ehhandler$??__EuiLog@U2@@YAXXZ 10021809 f   KrakenSupportPlugin.obj
 0001:00020830       __unwindfunclet$??__EuserActLog@U2@@YAXXZ$0 10021830 f   KrakenSupportPlugin.obj
 0001:00020839       __ehhandler$??__EuserActLog@U2@@YAXXZ 10021839 f   KrakenSupportPlugin.obj
 0001:00020860       __unwindfunclet$??__EalgoLog@U2@@YAXXZ$0 10021860 f   KrakenTranslateLogParser.obj
 0001:00020869       __ehhandler$??__EalgoLog@U2@@YAXXZ 10021869 f   KrakenTranslateLogParser.obj
 0001:00020890       __unwindfunclet$??__EcmdLog@U2@@YAXXZ$0 10021890 f   KrakenTranslateLogParser.obj
 0001:00020899       __ehhandler$??__EcmdLog@U2@@YAXXZ 10021899 f   KrakenTranslateLogParser.obj
 0001:000208c0       __unwindfunclet$??__EcoreLog@U2@@YAXXZ$0 100218c0 f   KrakenTranslateLogParser.obj
 0001:000208c9       __ehhandler$??__EcoreLog@U2@@YAXXZ 100218c9 f   KrakenTranslateLogParser.obj
 0001:000208f0       __unwindfunclet$??__EioLog@U2@@YAXXZ$0 100218f0 f   KrakenTranslateLogParser.obj
 0001:000208f9       __ehhandler$??__EioLog@U2@@YAXXZ 100218f9 f   KrakenTranslateLogParser.obj
 0001:00020920       __unwindfunclet$??__EperfLog@U2@@YAXXZ$0 10021920 f   KrakenTranslateLogParser.obj
 0001:00020929       __ehhandler$??__EperfLog@U2@@YAXXZ 10021929 f   KrakenTranslateLogParser.obj
 0001:00020950       __unwindfunclet$??__EscriptLog@U2@@YAXXZ$0 10021950 f   KrakenTranslateLogParser.obj
 0001:00020959       __ehhandler$??__EscriptLog@U2@@YAXXZ 10021959 f   KrakenTranslateLogParser.obj
 0001:00020980       __unwindfunclet$??__EtaskLog@U2@@YAXXZ$0 10021980 f   KrakenTranslateLogParser.obj
 0001:00020989       __ehhandler$??__EtaskLog@U2@@YAXXZ 10021989 f   KrakenTranslateLogParser.obj
 0001:000209b0       __unwindfunclet$??__EuiLog@U2@@YAXXZ$0 100219b0 f   KrakenTranslateLogParser.obj
 0001:000209b9       __ehhandler$??__EuiLog@U2@@YAXXZ 100219b9 f   KrakenTranslateLogParser.obj
 0001:000209e0       __unwindfunclet$??__EuserActLog@U2@@YAXXZ$0 100219e0 f   KrakenTranslateLogParser.obj
 0001:000209e9       __ehhandler$??__EuserActLog@U2@@YAXXZ 100219e9 f   KrakenTranslateLogParser.obj
 0001:00020a10       __unwindfunclet$?initWellKnownErrors@KrakenTranslateLogParser@U2@@CA?AVQStringList@@XZ$0 10021a10 f   KrakenTranslateLogParser.obj
 0001:00020a29       __unwindfunclet$?initWellKnownErrors@KrakenTranslateLogParser@U2@@CA?AVQStringList@@XZ$1 10021a29 f   KrakenTranslateLogParser.obj
 0001:00020a32       __unwindfunclet$?initWellKnownErrors@KrakenTranslateLogParser@U2@@CA?AVQStringList@@XZ$2 10021a32 f   KrakenTranslateLogParser.obj
 0001:00020a3b       __unwindfunclet$?initWellKnownErrors@KrakenTranslateLogParser@U2@@CA?AVQStringList@@XZ$3 10021a3b f   KrakenTranslateLogParser.obj
 0001:00020a44       __unwindfunclet$?initWellKnownErrors@KrakenTranslateLogParser@U2@@CA?AVQStringList@@XZ$4 10021a44 f   KrakenTranslateLogParser.obj
 0001:00020a4d       __unwindfunclet$?initWellKnownErrors@KrakenTranslateLogParser@U2@@CA?AVQStringList@@XZ$5 10021a4d f   KrakenTranslateLogParser.obj
 0001:00020a56       __ehhandler$?initWellKnownErrors@KrakenTranslateLogParser@U2@@CA?AVQStringList@@XZ 10021a56 f   KrakenTranslateLogParser.obj
 0001:00020a80       __unwindfunclet$?isError@KrakenTranslateLogParser@U2@@EBE_NABVQString@@@Z$0 10021a80 f   KrakenTranslateLogParser.obj
 0001:00020a88       __ehhandler$?isError@KrakenTranslateLogParser@U2@@EBE_NABVQString@@@Z 10021a88 f   KrakenTranslateLogParser.obj
 0001:00020ab0       __unwindfunclet$??__EalgoLog@U2@@YAXXZ$0 10021ab0 f   moc_KrakenBuildPrompter.obj
 0001:00020ab9       __ehhandler$??__EalgoLog@U2@@YAXXZ 10021ab9 f   moc_KrakenBuildPrompter.obj
 0001:00020ae0       __unwindfunclet$??__EcmdLog@U2@@YAXXZ$0 10021ae0 f   moc_KrakenBuildPrompter.obj
 0001:00020ae9       __ehhandler$??__EcmdLog@U2@@YAXXZ 10021ae9 f   moc_KrakenBuildPrompter.obj
 0001:00020b10       __unwindfunclet$??__EcoreLog@U2@@YAXXZ$0 10021b10 f   moc_KrakenBuildPrompter.obj
 0001:00020b19       __ehhandler$??__EcoreLog@U2@@YAXXZ 10021b19 f   moc_KrakenBuildPrompter.obj
 0001:00020b40       __unwindfunclet$??__EioLog@U2@@YAXXZ$0 10021b40 f   moc_KrakenBuildPrompter.obj
 0001:00020b49       __ehhandler$??__EioLog@U2@@YAXXZ 10021b49 f   moc_KrakenBuildPrompter.obj
 0001:00020b70       __unwindfunclet$??__EperfLog@U2@@YAXXZ$0 10021b70 f   moc_KrakenBuildPrompter.obj
 0001:00020b79       __ehhandler$??__EperfLog@U2@@YAXXZ 10021b79 f   moc_KrakenBuildPrompter.obj
 0001:00020ba0       __unwindfunclet$??__EscriptLog@U2@@YAXXZ$0 10021ba0 f   moc_KrakenBuildPrompter.obj
 0001:00020ba9       __ehhandler$??__EscriptLog@U2@@YAXXZ 10021ba9 f   moc_KrakenBuildPrompter.obj
 0001:00020bd0       __unwindfunclet$??__EtaskLog@U2@@YAXXZ$0 10021bd0 f   moc_KrakenBuildPrompter.obj
 0001:00020bd9       __ehhandler$??__EtaskLog@U2@@YAXXZ 10021bd9 f   moc_KrakenBuildPrompter.obj
 0001:00020c00       __unwindfunclet$??__EuiLog@U2@@YAXXZ$0 10021c00 f   moc_KrakenBuildPrompter.obj
 0001:00020c09       __ehhandler$??__EuiLog@U2@@YAXXZ 10021c09 f   moc_KrakenBuildPrompter.obj
 0001:00020c30       __unwindfunclet$??__EuserActLog@U2@@YAXXZ$0 10021c30 f   moc_KrakenBuildPrompter.obj
 0001:00020c39       __ehhandler$??__EuserActLog@U2@@YAXXZ 10021c39 f   moc_KrakenBuildPrompter.obj
 0001:00020c60       __unwindfunclet$??__EalgoLog@U2@@YAXXZ$0 10021c60 f   moc_KrakenBuildTask.obj
 0001:00020c69       __ehhandler$??__EalgoLog@U2@@YAXXZ 10021c69 f   moc_KrakenBuildTask.obj
 0001:00020c90       __unwindfunclet$??__EcmdLog@U2@@YAXXZ$0 10021c90 f   moc_KrakenBuildTask.obj
 0001:00020c99       __ehhandler$??__EcmdLog@U2@@YAXXZ 10021c99 f   moc_KrakenBuildTask.obj
 0001:00020cc0       __unwindfunclet$??__EcoreLog@U2@@YAXXZ$0 10021cc0 f   moc_KrakenBuildTask.obj
 0001:00020cc9       __ehhandler$??__EcoreLog@U2@@YAXXZ 10021cc9 f   moc_KrakenBuildTask.obj
 0001:00020cf0       __unwindfunclet$??__EioLog@U2@@YAXXZ$0 10021cf0 f   moc_KrakenBuildTask.obj
 0001:00020cf9       __ehhandler$??__EioLog@U2@@YAXXZ 10021cf9 f   moc_KrakenBuildTask.obj
 0001:00020d20       __unwindfunclet$??__EperfLog@U2@@YAXXZ$0 10021d20 f   moc_KrakenBuildTask.obj
 0001:00020d29       __ehhandler$??__EperfLog@U2@@YAXXZ 10021d29 f   moc_KrakenBuildTask.obj
 0001:00020d50       __unwindfunclet$??__EscriptLog@U2@@YAXXZ$0 10021d50 f   moc_KrakenBuildTask.obj
 0001:00020d59       __ehhandler$??__EscriptLog@U2@@YAXXZ 10021d59 f   moc_KrakenBuildTask.obj
 0001:00020d80       __unwindfunclet$??__EtaskLog@U2@@YAXXZ$0 10021d80 f   moc_KrakenBuildTask.obj
 0001:00020d89       __ehhandler$??__EtaskLog@U2@@YAXXZ 10021d89 f   moc_KrakenBuildTask.obj
 0001:00020db0       __unwindfunclet$??__EuiLog@U2@@YAXXZ$0 10021db0 f   moc_KrakenBuildTask.obj
 0001:00020db9       __ehhandler$??__EuiLog@U2@@YAXXZ 10021db9 f   moc_KrakenBuildTask.obj
 0001:00020de0       __unwindfunclet$??__EuserActLog@U2@@YAXXZ$0 10021de0 f   moc_KrakenBuildTask.obj
 0001:00020de9       __ehhandler$??__EuserActLog@U2@@YAXXZ 10021de9 f   moc_KrakenBuildTask.obj
 0001:00020e10       __unwindfunclet$??__EalgoLog@U2@@YAXXZ$0 10021e10 f   moc_KrakenBuildWorker.obj
 0001:00020e19       __ehhandler$??__EalgoLog@U2@@YAXXZ 10021e19 f   moc_KrakenBuildWorker.obj
 0001:00020e40       __unwindfunclet$??__EcmdLog@U2@@YAXXZ$0 10021e40 f   moc_KrakenBuildWorker.obj
 0001:00020e49       __ehhandler$??__EcmdLog@U2@@YAXXZ 10021e49 f   moc_KrakenBuildWorker.obj
 0001:00020e70       __unwindfunclet$??__EcoreLog@U2@@YAXXZ$0 10021e70 f   moc_KrakenBuildWorker.obj
 0001:00020e79       __ehhandler$??__EcoreLog@U2@@YAXXZ 10021e79 f   moc_KrakenBuildWorker.obj
 0001:00020ea0       __unwindfunclet$??__EioLog@U2@@YAXXZ$0 10021ea0 f   moc_KrakenBuildWorker.obj
 0001:00020ea9       __ehhandler$??__EioLog@U2@@YAXXZ 10021ea9 f   moc_KrakenBuildWorker.obj
 0001:00020ed0       __unwindfunclet$??__EperfLog@U2@@YAXXZ$0 10021ed0 f   moc_KrakenBuildWorker.obj
 0001:00020ed9       __ehhandler$??__EperfLog@U2@@YAXXZ 10021ed9 f   moc_KrakenBuildWorker.obj
 0001:00020f00       __unwindfunclet$??__EscriptLog@U2@@YAXXZ$0 10021f00 f   moc_KrakenBuildWorker.obj
 0001:00020f09       __ehhandler$??__EscriptLog@U2@@YAXXZ 10021f09 f   moc_KrakenBuildWorker.obj
 0001:00020f30       __unwindfunclet$??__EtaskLog@U2@@YAXXZ$0 10021f30 f   moc_KrakenBuildWorker.obj
 0001:00020f39       __ehhandler$??__EtaskLog@U2@@YAXXZ 10021f39 f   moc_KrakenBuildWorker.obj
 0001:00020f60       __unwindfunclet$??__EuiLog@U2@@YAXXZ$0 10021f60 f   moc_KrakenBuildWorker.obj
 0001:00020f69       __ehhandler$??__EuiLog@U2@@YAXXZ 10021f69 f   moc_KrakenBuildWorker.obj
 0001:00020f90       __unwindfunclet$??__EuserActLog@U2@@YAXXZ$0 10021f90 f   moc_KrakenBuildWorker.obj
 0001:00020f99       __ehhandler$??__EuserActLog@U2@@YAXXZ 10021f99 f   moc_KrakenBuildWorker.obj
 0001:00020fc0       __unwindfunclet$?qt_metatype_id@?$QMetaTypeIdQObject@PAVTask@U2@@$00@@SAHXZ$0 10021fc0 f   moc_KrakenBuildWorker.obj
 0001:00020fc9       __ehhandler$?qt_metatype_id@?$QMetaTypeIdQObject@PAVTask@U2@@$00@@SAHXZ 10021fc9 f   moc_KrakenBuildWorker.obj
 0001:00020ff0       __unwindfunclet$??__EalgoLog@U2@@YAXXZ$0 10021ff0 f   moc_KrakenClassifyPrompter.obj
 0001:00020ff9       __ehhandler$??__EalgoLog@U2@@YAXXZ 10021ff9 f   moc_KrakenClassifyPrompter.obj
 0001:00021020       __unwindfunclet$??__EcmdLog@U2@@YAXXZ$0 10022020 f   moc_KrakenClassifyPrompter.obj
 0001:00021029       __ehhandler$??__EcmdLog@U2@@YAXXZ 10022029 f   moc_KrakenClassifyPrompter.obj
 0001:00021050       __unwindfunclet$??__EcoreLog@U2@@YAXXZ$0 10022050 f   moc_KrakenClassifyPrompter.obj
 0001:00021059       __ehhandler$??__EcoreLog@U2@@YAXXZ 10022059 f   moc_KrakenClassifyPrompter.obj
 0001:00021080       __unwindfunclet$??__EioLog@U2@@YAXXZ$0 10022080 f   moc_KrakenClassifyPrompter.obj
 0001:00021089       __ehhandler$??__EioLog@U2@@YAXXZ 10022089 f   moc_KrakenClassifyPrompter.obj
 0001:000210b0       __unwindfunclet$??__EperfLog@U2@@YAXXZ$0 100220b0 f   moc_KrakenClassifyPrompter.obj
 0001:000210b9       __ehhandler$??__EperfLog@U2@@YAXXZ 100220b9 f   moc_KrakenClassifyPrompter.obj
 0001:000210e0       __unwindfunclet$??__EscriptLog@U2@@YAXXZ$0 100220e0 f   moc_KrakenClassifyPrompter.obj
 0001:000210e9       __ehhandler$??__EscriptLog@U2@@YAXXZ 100220e9 f   moc_KrakenClassifyPrompter.obj
 0001:00021110       __unwindfunclet$??__EtaskLog@U2@@YAXXZ$0 10022110 f   moc_KrakenClassifyPrompter.obj
 0001:00021119       __ehhandler$??__EtaskLog@U2@@YAXXZ 10022119 f   moc_KrakenClassifyPrompter.obj
 0001:00021140       __unwindfunclet$??__EuiLog@U2@@YAXXZ$0 10022140 f   moc_KrakenClassifyPrompter.obj
 0001:00021149       __ehhandler$??__EuiLog@U2@@YAXXZ 10022149 f   moc_KrakenClassifyPrompter.obj
 0001:00021170       __unwindfunclet$??__EuserActLog@U2@@YAXXZ$0 10022170 f   moc_KrakenClassifyPrompter.obj
 0001:00021179       __ehhandler$??__EuserActLog@U2@@YAXXZ 10022179 f   moc_KrakenClassifyPrompter.obj
 0001:000211a0       __unwindfunclet$??__EalgoLog@U2@@YAXXZ$0 100221a0 f   moc_KrakenClassifyTask.obj
 0001:000211a9       __ehhandler$??__EalgoLog@U2@@YAXXZ 100221a9 f   moc_KrakenClassifyTask.obj
 0001:000211d0       __unwindfunclet$??__EcmdLog@U2@@YAXXZ$0 100221d0 f   moc_KrakenClassifyTask.obj
 0001:000211d9       __ehhandler$??__EcmdLog@U2@@YAXXZ 100221d9 f   moc_KrakenClassifyTask.obj
 0001:00021200       __unwindfunclet$??__EcoreLog@U2@@YAXXZ$0 10022200 f   moc_KrakenClassifyTask.obj
 0001:00021209       __ehhandler$??__EcoreLog@U2@@YAXXZ 10022209 f   moc_KrakenClassifyTask.obj
 0001:00021230       __unwindfunclet$??__EioLog@U2@@YAXXZ$0 10022230 f   moc_KrakenClassifyTask.obj
 0001:00021239       __ehhandler$??__EioLog@U2@@YAXXZ 10022239 f   moc_KrakenClassifyTask.obj
 0001:00021260       __unwindfunclet$??__EperfLog@U2@@YAXXZ$0 10022260 f   moc_KrakenClassifyTask.obj
 0001:00021269       __ehhandler$??__EperfLog@U2@@YAXXZ 10022269 f   moc_KrakenClassifyTask.obj
 0001:00021290       __unwindfunclet$??__EscriptLog@U2@@YAXXZ$0 10022290 f   moc_KrakenClassifyTask.obj
 0001:00021299       __ehhandler$??__EscriptLog@U2@@YAXXZ 10022299 f   moc_KrakenClassifyTask.obj
 0001:000212c0       __unwindfunclet$??__EtaskLog@U2@@YAXXZ$0 100222c0 f   moc_KrakenClassifyTask.obj
 0001:000212c9       __ehhandler$??__EtaskLog@U2@@YAXXZ 100222c9 f   moc_KrakenClassifyTask.obj
 0001:000212f0       __unwindfunclet$??__EuiLog@U2@@YAXXZ$0 100222f0 f   moc_KrakenClassifyTask.obj
 0001:000212f9       __ehhandler$??__EuiLog@U2@@YAXXZ 100222f9 f   moc_KrakenClassifyTask.obj
 0001:00021320       __unwindfunclet$??__EuserActLog@U2@@YAXXZ$0 10022320 f   moc_KrakenClassifyTask.obj
 0001:00021329       __ehhandler$??__EuserActLog@U2@@YAXXZ 10022329 f   moc_KrakenClassifyTask.obj
 0001:00021350       __unwindfunclet$??__EalgoLog@U2@@YAXXZ$0 10022350 f   moc_KrakenClassifyWorker.obj
 0001:00021359       __ehhandler$??__EalgoLog@U2@@YAXXZ 10022359 f   moc_KrakenClassifyWorker.obj
 0001:00021380       __unwindfunclet$??__EcmdLog@U2@@YAXXZ$0 10022380 f   moc_KrakenClassifyWorker.obj
 0001:00021389       __ehhandler$??__EcmdLog@U2@@YAXXZ 10022389 f   moc_KrakenClassifyWorker.obj
 0001:000213b0       __unwindfunclet$??__EcoreLog@U2@@YAXXZ$0 100223b0 f   moc_KrakenClassifyWorker.obj
 0001:000213b9       __ehhandler$??__EcoreLog@U2@@YAXXZ 100223b9 f   moc_KrakenClassifyWorker.obj
 0001:000213e0       __unwindfunclet$??__EioLog@U2@@YAXXZ$0 100223e0 f   moc_KrakenClassifyWorker.obj
 0001:000213e9       __ehhandler$??__EioLog@U2@@YAXXZ 100223e9 f   moc_KrakenClassifyWorker.obj
 0001:00021410       __unwindfunclet$??__EperfLog@U2@@YAXXZ$0 10022410 f   moc_KrakenClassifyWorker.obj
 0001:00021419       __ehhandler$??__EperfLog@U2@@YAXXZ 10022419 f   moc_KrakenClassifyWorker.obj
 0001:00021440       __unwindfunclet$??__EscriptLog@U2@@YAXXZ$0 10022440 f   moc_KrakenClassifyWorker.obj
 0001:00021449       __ehhandler$??__EscriptLog@U2@@YAXXZ 10022449 f   moc_KrakenClassifyWorker.obj
 0001:00021470       __unwindfunclet$??__EtaskLog@U2@@YAXXZ$0 10022470 f   moc_KrakenClassifyWorker.obj
 0001:00021479       __ehhandler$??__EtaskLog@U2@@YAXXZ 10022479 f   moc_KrakenClassifyWorker.obj
 0001:000214a0       __unwindfunclet$??__EuiLog@U2@@YAXXZ$0 100224a0 f   moc_KrakenClassifyWorker.obj
 0001:000214a9       __ehhandler$??__EuiLog@U2@@YAXXZ 100224a9 f   moc_KrakenClassifyWorker.obj
 0001:000214d0       __unwindfunclet$??__EuserActLog@U2@@YAXXZ$0 100224d0 f   moc_KrakenClassifyWorker.obj
 0001:000214d9       __ehhandler$??__EuserActLog@U2@@YAXXZ 100224d9 f   moc_KrakenClassifyWorker.obj
 0001:00021500       ??__F?_Generic_object@?$_Error_objects@H@std@@2V_Generic_error_category@2@A@@YAXXZ 10022500 f   DatabaseSizeRelation.obj
 0001:00021510       ??__F?_Iostream_object@?$_Error_objects@H@std@@2V_Iostream_error_category@2@A@@YAXXZ 10022510 f   DatabaseSizeRelation.obj
 0001:00021520       ??__F?_System_object@?$_Error_objects@H@std@@2V_System_error_category@2@A@@YAXXZ 10022520 f   DatabaseSizeRelation.obj
 0001:00021530       ??__FalgoLog@U2@@YAXXZ     10022530 f   DatabaseSizeRelation.obj
 0001:00021540       ??__FcmdLog@U2@@YAXXZ      10022540 f   DatabaseSizeRelation.obj
 0001:00021550       ??__FcoreLog@U2@@YAXXZ     10022550 f   DatabaseSizeRelation.obj
 0001:00021560       ??__FioLog@U2@@YAXXZ       10022560 f   DatabaseSizeRelation.obj
 0001:00021570       ??__FperfLog@U2@@YAXXZ     10022570 f   DatabaseSizeRelation.obj
 0001:00021580       ??__FscriptLog@U2@@YAXXZ   10022580 f   DatabaseSizeRelation.obj
 0001:00021590       ??__FtaskLog@U2@@YAXXZ     10022590 f   DatabaseSizeRelation.obj
 0001:000215a0       ??__FuiLog@U2@@YAXXZ       100225a0 f   DatabaseSizeRelation.obj
 0001:000215b0       ??__FuserActLog@U2@@YAXXZ  100225b0 f   DatabaseSizeRelation.obj
 0001:000215c0       ??__F?_Generic_object@?$_Error_objects@H@std@@2V_Generic_error_category@2@A@@YAXXZ 100225c0 f   KrakenBuildPrompter.obj
 0001:000215d0       ??__F?_Iostream_object@?$_Error_objects@H@std@@2V_Iostream_error_category@2@A@@YAXXZ 100225d0 f   KrakenBuildPrompter.obj
 0001:000215e0       ??__F?_System_object@?$_Error_objects@H@std@@2V_System_error_category@2@A@@YAXXZ 100225e0 f   KrakenBuildPrompter.obj
 0001:000215f0       ??__FalgoLog@U2@@YAXXZ     100225f0 f   KrakenBuildPrompter.obj
 0001:00021600       ??__FcmdLog@U2@@YAXXZ      10022600 f   KrakenBuildPrompter.obj
 0001:00021610       ??__FcoreLog@U2@@YAXXZ     10022610 f   KrakenBuildPrompter.obj
 0001:00021620       ??__FioLog@U2@@YAXXZ       10022620 f   KrakenBuildPrompter.obj
 0001:00021630       ??__FperfLog@U2@@YAXXZ     10022630 f   KrakenBuildPrompter.obj
 0001:00021640       ??__FscriptLog@U2@@YAXXZ   10022640 f   KrakenBuildPrompter.obj
 0001:00021650       ??__FtaskLog@U2@@YAXXZ     10022650 f   KrakenBuildPrompter.obj
 0001:00021660       ??__FuiLog@U2@@YAXXZ       10022660 f   KrakenBuildPrompter.obj
 0001:00021670       ??__FuserActLog@U2@@YAXXZ  10022670 f   KrakenBuildPrompter.obj
 0001:00021680       ??__F?BUILD@KrakenBuildTaskSettings@U2@@2VQString@@B@@YAXXZ 10022680 f   KrakenBuildTask.obj
 0001:00021690       ??__F?SHRINK@KrakenBuildTaskSettings@U2@@2VQString@@B@@YAXXZ 10022690 f   KrakenBuildTask.obj
 0001:000216a0       ??__F?_Generic_object@?$_Error_objects@H@std@@2V_Generic_error_category@2@A@@YAXXZ 100226a0 f   KrakenBuildTask.obj
 0001:000216b0       ??__F?_Iostream_object@?$_Error_objects@H@std@@2V_Iostream_error_category@2@A@@YAXXZ 100226b0 f   KrakenBuildTask.obj
 0001:000216c0       ??__F?_System_object@?$_Error_objects@H@std@@2V_System_error_category@2@A@@YAXXZ 100226c0 f   KrakenBuildTask.obj
 0001:000216d0       ??__FTAXONOMY_FILES_TO_COPY@?1??prepareTaxonomyData@KrakenBuildTask@U2@@AAE?AV?$QList@PAVTask@U2@@@@XZ@YAXXZ 100226d0 f   KrakenBuildTask.obj
 0001:000216e0       ??__FalgoLog@U2@@YAXXZ     100226e0 f   KrakenBuildTask.obj
 0001:000216f0       ??__FcmdLog@U2@@YAXXZ      100226f0 f   KrakenBuildTask.obj
 0001:00021700       ??__FcoreLog@U2@@YAXXZ     10022700 f   KrakenBuildTask.obj
 0001:00021710       ??__Fcvar@?1???0KrakenBuildTask@U2@@QAE@ABUKrakenBuildTaskSettings@1@@Z@YAXXZ 10022710 f   KrakenBuildTask.obj
 0001:00021720       ??__FioLog@U2@@YAXXZ       10022720 f   KrakenBuildTask.obj
 0001:00021730       ??__FperfLog@U2@@YAXXZ     10022730 f   KrakenBuildTask.obj
 0001:00021740       ??__FscriptLog@U2@@YAXXZ   10022740 f   KrakenBuildTask.obj
 0001:00021750       ??__FtaskLog@U2@@YAXXZ     10022750 f   KrakenBuildTask.obj
 0001:00021760       ??__FuiLog@U2@@YAXXZ       10022760 f   KrakenBuildTask.obj
 0001:00021770       ??__FuserActLog@U2@@YAXXZ  10022770 f   KrakenBuildTask.obj
 0001:00021780       ??__F?_Generic_object@?$_Error_objects@H@std@@2V_Generic_error_category@2@A@@YAXXZ 10022780 f   KrakenBuildValidator.obj
 0001:00021790       ??__F?_Iostream_object@?$_Error_objects@H@std@@2V_Iostream_error_category@2@A@@YAXXZ 10022790 f   KrakenBuildValidator.obj
 0001:000217a0       ??__F?_System_object@?$_Error_objects@H@std@@2V_System_error_category@2@A@@YAXXZ 100227a0 f   KrakenBuildValidator.obj
 0001:000217b0       ??__FalgoLog@U2@@YAXXZ     100227b0 f   KrakenBuildValidator.obj
 0001:000217c0       ??__FcmdLog@U2@@YAXXZ      100227c0 f   KrakenBuildValidator.obj
 0001:000217d0       ??__FcoreLog@U2@@YAXXZ     100227d0 f   KrakenBuildValidator.obj
 0001:000217e0       ??__FioLog@U2@@YAXXZ       100227e0 f   KrakenBuildValidator.obj
 0001:000217f0       ??__FperfLog@U2@@YAXXZ     100227f0 f   KrakenBuildValidator.obj
 0001:00021800       ??__FscriptLog@U2@@YAXXZ   10022800 f   KrakenBuildValidator.obj
 0001:00021810       ??__FtaskLog@U2@@YAXXZ     10022810 f   KrakenBuildValidator.obj
 0001:00021820       ??__FuiLog@U2@@YAXXZ       10022820 f   KrakenBuildValidator.obj
 0001:00021830       ??__FuserActLog@U2@@YAXXZ  10022830 f   KrakenBuildValidator.obj
 0001:00021840       ??__F?_Generic_object@?$_Error_objects@H@std@@2V_Generic_error_category@2@A@@YAXXZ 10022840 f   KrakenBuildWorker.obj
 0001:00021850       ??__F?_Iostream_object@?$_Error_objects@H@std@@2V_Iostream_error_category@2@A@@YAXXZ 10022850 f   KrakenBuildWorker.obj
 0001:00021860       ??__F?_System_object@?$_Error_objects@H@std@@2V_System_error_category@2@A@@YAXXZ 10022860 f   KrakenBuildWorker.obj
 0001:00021870       ??__FalgoLog@U2@@YAXXZ     10022870 f   KrakenBuildWorker.obj
 0001:00021880       ??__FcmdLog@U2@@YAXXZ      10022880 f   KrakenBuildWorker.obj
 0001:00021890       ??__FcoreLog@U2@@YAXXZ     10022890 f   KrakenBuildWorker.obj
 0001:000218a0       ??__FioLog@U2@@YAXXZ       100228a0 f   KrakenBuildWorker.obj
 0001:000218b0       ??__FperfLog@U2@@YAXXZ     100228b0 f   KrakenBuildWorker.obj
 0001:000218c0       ??__FscriptLog@U2@@YAXXZ   100228c0 f   KrakenBuildWorker.obj
 0001:000218d0       ??__FtaskLog@U2@@YAXXZ     100228d0 f   KrakenBuildWorker.obj
 0001:000218e0       ??__FuiLog@U2@@YAXXZ       100228e0 f   KrakenBuildWorker.obj
 0001:000218f0       ??__FuserActLog@U2@@YAXXZ  100228f0 f   KrakenBuildWorker.obj
 0001:00021900       ??__F?ACTOR_ID@KrakenBuildWorkerFactory@LocalWorkflow@U2@@2VQString@@B@@YAXXZ 10022900 f   KrakenBuildWorkerFactory.obj
 0001:00021910       ??__F?CLEAN_ATTR_ID@KrakenBuildWorkerFactory@LocalWorkflow@U2@@2VQString@@B@@YAXXZ 10022910 f   KrakenBuildWorkerFactory.obj
 0001:00021920       ??__F?GENOMIC_LIBRARY_ATTR_ID@KrakenBuildWorkerFactory@LocalWorkflow@U2@@2VQString@@B@@YAXXZ 10022920 f   KrakenBuildWorkerFactory.obj
 0001:00021930       ??__F?INPUT_DATABASE_NAME_ATTR_ID@KrakenBuildWorkerFactory@LocalWorkflow@U2@@2VQString@@B@@YAXXZ 10022930 f   KrakenBuildWorkerFactory.obj
 0001:00021940       ??__F?JELLYFISH_HASH_SIZE_ATTR_ID@KrakenBuildWorkerFactory@LocalWorkflow@U2@@2VQString@@B@@YAXXZ 10022940 f   KrakenBuildWorkerFactory.obj
 0001:00021950       ??__F?K_MER_LENGTH_ATTR_ID@KrakenBuildWorkerFactory@LocalWorkflow@U2@@2VQString@@B@@YAXXZ 10022950 f   KrakenBuildWorkerFactory.obj
 0001:00021960       ??__F?MAXIMUM_DATABASE_SIZE_ATTR_ID@KrakenBuildWorkerFactory@LocalWorkflow@U2@@2VQString@@B@@YAXXZ 10022960 f   KrakenBuildWorkerFactory.obj
 0001:00021970       ??__F?MINIMIZER_LENGTH_ATTR_ID@KrakenBuildWorkerFactory@LocalWorkflow@U2@@2VQString@@B@@YAXXZ 10022970 f   KrakenBuildWorkerFactory.obj
 0001:00021980       ??__F?MODE_ATTR_ID@KrakenBuildWorkerFactory@LocalWorkflow@U2@@2VQString@@B@@YAXXZ 10022980 f   KrakenBuildWorkerFactory.obj
 0001:00021990       ??__F?NEW_DATABASE_NAME_ATTR_ID@KrakenBuildWorkerFactory@LocalWorkflow@U2@@2VQString@@B@@YAXXZ 10022990 f   KrakenBuildWorkerFactory.obj
 0001:000219a0       ??__F?NUMBER_OF_K_MERS_ATTR_ID@KrakenBuildWorkerFactory@LocalWorkflow@U2@@2VQString@@B@@YAXXZ 100229a0 f   KrakenBuildWorkerFactory.obj
 0001:000219b0       ??__F?OUTPUT_PORT_ID@KrakenBuildWorkerFactory@LocalWorkflow@U2@@2VQString@@B@@YAXXZ 100229b0 f   KrakenBuildWorkerFactory.obj
 0001:000219c0       ??__F?SHRINK_BLOCK_OFFSET_ATTR_ID@KrakenBuildWorkerFactory@LocalWorkflow@U2@@2VQString@@B@@YAXXZ 100229c0 f   KrakenBuildWorkerFactory.obj
 0001:000219d0       ??__F?THREADS_NUMBER_ATTR_ID@KrakenBuildWorkerFactory@LocalWorkflow@U2@@2VQString@@B@@YAXXZ 100229d0 f   KrakenBuildWorkerFactory.obj
 0001:000219e0       ??__F?WORK_ON_DISK_ATTR_ID@KrakenBuildWorkerFactory@LocalWorkflow@U2@@2VQString@@B@@YAXXZ 100229e0 f   KrakenBuildWorkerFactory.obj
 0001:000219f0       ??__F?_Generic_object@?$_Error_objects@H@std@@2V_Generic_error_category@2@A@@YAXXZ 100229f0 f   KrakenBuildWorkerFactory.obj
 0001:00021a00       ??__F?_Iostream_object@?$_Error_objects@H@std@@2V_Iostream_error_category@2@A@@YAXXZ 10022a00 f   KrakenBuildWorkerFactory.obj
 0001:00021a10       ??__F?_System_object@?$_Error_objects@H@std@@2V_System_error_category@2@A@@YAXXZ 10022a10 f   KrakenBuildWorkerFactory.obj
 0001:00021a20       ??__FalgoLog@U2@@YAXXZ     10022a20 f   KrakenBuildWorkerFactory.obj
 0001:00021a30       ??__FcmdLog@U2@@YAXXZ      10022a30 f   KrakenBuildWorkerFactory.obj
 0001:00021a40       ??__FcoreLog@U2@@YAXXZ     10022a40 f   KrakenBuildWorkerFactory.obj
 0001:00021a50       ??__FioLog@U2@@YAXXZ       10022a50 f   KrakenBuildWorkerFactory.obj
 0001:00021a60       ??__FperfLog@U2@@YAXXZ     10022a60 f   KrakenBuildWorkerFactory.obj
 0001:00021a70       ??__FscriptLog@U2@@YAXXZ   10022a70 f   KrakenBuildWorkerFactory.obj
 0001:00021a80       ??__FtaskLog@U2@@YAXXZ     10022a80 f   KrakenBuildWorkerFactory.obj
 0001:00021a90       ??__FuiLog@U2@@YAXXZ       10022a90 f   KrakenBuildWorkerFactory.obj
 0001:00021aa0       ??__FuserActLog@U2@@YAXXZ  10022aa0 f   KrakenBuildWorkerFactory.obj
 0001:00021ab0       ??__F?_Generic_object@?$_Error_objects@H@std@@2V_Generic_error_category@2@A@@YAXXZ 10022ab0 f   KrakenClassifyLogParser.obj
 0001:00021ac0       ??__F?_Iostream_object@?$_Error_objects@H@std@@2V_Iostream_error_category@2@A@@YAXXZ 10022ac0 f   KrakenClassifyLogParser.obj
 0001:00021ad0       ??__F?_System_object@?$_Error_objects@H@std@@2V_System_error_category@2@A@@YAXXZ 10022ad0 f   KrakenClassifyLogParser.obj
 0001:00021ae0       ??__F?wellKnownErrors@KrakenClassifyLogParser@U2@@0VQStringList@@B@@YAXXZ 10022ae0 f   KrakenClassifyLogParser.obj
 0001:00021af0       ??__FalgoLog@U2@@YAXXZ     10022af0 f   KrakenClassifyLogParser.obj
 0001:00021b00       ??__FcmdLog@U2@@YAXXZ      10022b00 f   KrakenClassifyLogParser.obj
 0001:00021b10       ??__FcoreLog@U2@@YAXXZ     10022b10 f   KrakenClassifyLogParser.obj
 0001:00021b20       ??__FioLog@U2@@YAXXZ       10022b20 f   KrakenClassifyLogParser.obj
 0001:00021b30       ??__FperfLog@U2@@YAXXZ     10022b30 f   KrakenClassifyLogParser.obj
 0001:00021b40       ??__FscriptLog@U2@@YAXXZ   10022b40 f   KrakenClassifyLogParser.obj
 0001:00021b50       ??__FtaskLog@U2@@YAXXZ     10022b50 f   KrakenClassifyLogParser.obj
 0001:00021b60       ??__FuiLog@U2@@YAXXZ       10022b60 f   KrakenClassifyLogParser.obj
 0001:00021b70       ??__FuserActLog@U2@@YAXXZ  10022b70 f   KrakenClassifyLogParser.obj
 0001:00021b80       ??__F?_Generic_object@?$_Error_objects@H@std@@2V_Generic_error_category@2@A@@YAXXZ 10022b80 f   KrakenClassifyPrompter.obj
 0001:00021b90       ??__F?_Iostream_object@?$_Error_objects@H@std@@2V_Iostream_error_category@2@A@@YAXXZ 10022b90 f   KrakenClassifyPrompter.obj
 0001:00021ba0       ??__F?_System_object@?$_Error_objects@H@std@@2V_System_error_category@2@A@@YAXXZ 10022ba0 f   KrakenClassifyPrompter.obj
 0001:00021bb0       ??__FalgoLog@U2@@YAXXZ     10022bb0 f   KrakenClassifyPrompter.obj
 0001:00021bc0       ??__FcmdLog@U2@@YAXXZ      10022bc0 f   KrakenClassifyPrompter.obj
 0001:00021bd0       ??__FcoreLog@U2@@YAXXZ     10022bd0 f   KrakenClassifyPrompter.obj
 0001:00021be0       ??__FioLog@U2@@YAXXZ       10022be0 f   KrakenClassifyPrompter.obj
 0001:00021bf0       ??__FperfLog@U2@@YAXXZ     10022bf0 f   KrakenClassifyPrompter.obj
 0001:00021c00       ??__FscriptLog@U2@@YAXXZ   10022c00 f   KrakenClassifyPrompter.obj
 0001:00021c10       ??__FtaskLog@U2@@YAXXZ     10022c10 f   KrakenClassifyPrompter.obj
 0001:00021c20       ??__FuiLog@U2@@YAXXZ       10022c20 f   KrakenClassifyPrompter.obj
 0001:00021c30       ??__FuserActLog@U2@@YAXXZ  10022c30 f   KrakenClassifyPrompter.obj
 0001:00021c40       ??__F?PAIRED_END@KrakenClassifyTaskSettings@U2@@2VQString@@B@@YAXXZ 10022c40 f   KrakenClassifyTask.obj
 0001:00021c50       ??__F?SINGLE_END@KrakenClassifyTaskSettings@U2@@2VQString@@B@@YAXXZ 10022c50 f   KrakenClassifyTask.obj
 0001:00021c60       ??__F?_Generic_object@?$_Error_objects@H@std@@2V_Generic_error_category@2@A@@YAXXZ 10022c60 f   KrakenClassifyTask.obj
 0001:00021c70       ??__F?_Iostream_object@?$_Error_objects@H@std@@2V_Iostream_error_category@2@A@@YAXXZ 10022c70 f   KrakenClassifyTask.obj
 0001:00021c80       ??__F?_System_object@?$_Error_objects@H@std@@2V_System_error_category@2@A@@YAXXZ 10022c80 f   KrakenClassifyTask.obj
 0001:00021c90       ??__FalgoLog@U2@@YAXXZ     10022c90 f   KrakenClassifyTask.obj
 0001:00021ca0       ??__FcmdLog@U2@@YAXXZ      10022ca0 f   KrakenClassifyTask.obj
 0001:00021cb0       ??__FcoreLog@U2@@YAXXZ     10022cb0 f   KrakenClassifyTask.obj
 0001:00021cc0       ??__Fcvar@?1???0KrakenClassifyTask@U2@@QAE@ABUKrakenClassifyTaskSettings@1@@Z@YAXXZ 10022cc0 f   KrakenClassifyTask.obj
 0001:00021cd0       ??__FioLog@U2@@YAXXZ       10022cd0 f   KrakenClassifyTask.obj
 0001:00021ce0       ??__FperfLog@U2@@YAXXZ     10022ce0 f   KrakenClassifyTask.obj
 0001:00021cf0       ??__FscriptLog@U2@@YAXXZ   10022cf0 f   KrakenClassifyTask.obj
 0001:00021d00       ??__FtaskLog@U2@@YAXXZ     10022d00 f   KrakenClassifyTask.obj
 0001:00021d10       ??__FuiLog@U2@@YAXXZ       10022d10 f   KrakenClassifyTask.obj
 0001:00021d20       ??__FuserActLog@U2@@YAXXZ  10022d20 f   KrakenClassifyTask.obj
 0001:00021d30       ??__F?_Generic_object@?$_Error_objects@H@std@@2V_Generic_error_category@2@A@@YAXXZ 10022d30 f   KrakenClassifyValidator.obj
 0001:00021d40       ??__F?_Iostream_object@?$_Error_objects@H@std@@2V_Iostream_error_category@2@A@@YAXXZ 10022d40 f   KrakenClassifyValidator.obj
 0001:00021d50       ??__F?_System_object@?$_Error_objects@H@std@@2V_System_error_category@2@A@@YAXXZ 10022d50 f   KrakenClassifyValidator.obj
 0001:00021d60       ??__FalgoLog@U2@@YAXXZ     10022d60 f   KrakenClassifyValidator.obj
 0001:00021d70       ??__FcmdLog@U2@@YAXXZ      10022d70 f   KrakenClassifyValidator.obj
 0001:00021d80       ??__FcoreLog@U2@@YAXXZ     10022d80 f   KrakenClassifyValidator.obj
 0001:00021d90       ??__FioLog@U2@@YAXXZ       10022d90 f   KrakenClassifyValidator.obj
 0001:00021da0       ??__FperfLog@U2@@YAXXZ     10022da0 f   KrakenClassifyValidator.obj
 0001:00021db0       ??__FscriptLog@U2@@YAXXZ   10022db0 f   KrakenClassifyValidator.obj
 0001:00021dc0       ??__FtaskLog@U2@@YAXXZ     10022dc0 f   KrakenClassifyValidator.obj
 0001:00021dd0       ??__FuiLog@U2@@YAXXZ       10022dd0 f   KrakenClassifyValidator.obj
 0001:00021de0       ??__FuserActLog@U2@@YAXXZ  10022de0 f   KrakenClassifyValidator.obj
 0001:00021df0       ??__F?KRAKEN_DIR@KrakenClassifyWorker@LocalWorkflow@U2@@0VQString@@B@@YAXXZ 10022df0 f   KrakenClassifyWorker.obj
 0001:00021e00       ??__F?_Generic_object@?$_Error_objects@H@std@@2V_Generic_error_category@2@A@@YAXXZ 10022e00 f   KrakenClassifyWorker.obj
 0001:00021e10       ??__F?_Iostream_object@?$_Error_objects@H@std@@2V_Iostream_error_category@2@A@@YAXXZ 10022e10 f   KrakenClassifyWorker.obj
 0001:00021e20       ??__F?_System_object@?$_Error_objects@H@std@@2V_System_error_category@2@A@@YAXXZ 10022e20 f   KrakenClassifyWorker.obj
 0001:00021e30       ??__FalgoLog@U2@@YAXXZ     10022e30 f   KrakenClassifyWorker.obj
 0001:00021e40       ??__FcmdLog@U2@@YAXXZ      10022e40 f   KrakenClassifyWorker.obj
 0001:00021e50       ??__FcoreLog@U2@@YAXXZ     10022e50 f   KrakenClassifyWorker.obj
 0001:00021e80       ??__FioLog@U2@@YAXXZ       10022e80 f   KrakenClassifyWorker.obj
 0001:00021e90       ??__FperfLog@U2@@YAXXZ     10022e90 f   KrakenClassifyWorker.obj
 0001:00021ea0       ??__FscriptLog@U2@@YAXXZ   10022ea0 f   KrakenClassifyWorker.obj
 0001:00021eb0       ??__FtaskLog@U2@@YAXXZ     10022eb0 f   KrakenClassifyWorker.obj
 0001:00021ec0       ??__FuiLog@U2@@YAXXZ       10022ec0 f   KrakenClassifyWorker.obj
 0001:00021ed0       ??__FuserActLog@U2@@YAXXZ  10022ed0 f   KrakenClassifyWorker.obj
 0001:00021ee0       ??__F?ACTOR_ID@KrakenClassifyWorkerFactory@LocalWorkflow@U2@@2VQString@@B@@YAXXZ 10022ee0 f   KrakenClassifyWorkerFactory.obj
 0001:00021ef0       ??__F?DATABASE_ATTR_ID@KrakenClassifyWorkerFactory@LocalWorkflow@U2@@2VQString@@B@@YAXXZ 10022ef0 f   KrakenClassifyWorkerFactory.obj
 0001:00021f00       ??__F?INPUT_DATA_ATTR_ID@KrakenClassifyWorkerFactory@LocalWorkflow@U2@@2VQString@@B@@YAXXZ 10022f00 f   KrakenClassifyWorkerFactory.obj
 0001:00021f10       ??__F?INPUT_PORT_ID@KrakenClassifyWorkerFactory@LocalWorkflow@U2@@2VQString@@B@@YAXXZ 10022f10 f   KrakenClassifyWorkerFactory.obj
 0001:00021f20       ??__F?INPUT_SLOT@KrakenClassifyWorkerFactory@LocalWorkflow@U2@@2VQString@@B@@YAXXZ 10022f20 f   KrakenClassifyWorkerFactory.obj
 0001:00021f30       ??__F?MIN_HITS_NUMBER_ATTR_ID@KrakenClassifyWorkerFactory@LocalWorkflow@U2@@2VQString@@B@@YAXXZ 10022f30 f   KrakenClassifyWorkerFactory.obj
 0001:00021f40       ??__F?OUTPUT_PORT_ID@KrakenClassifyWorkerFactory@LocalWorkflow@U2@@2VQString@@B@@YAXXZ 10022f40 f   KrakenClassifyWorkerFactory.obj
 0001:00021f50       ??__F?OUTPUT_URL_ATTR_ID@KrakenClassifyWorkerFactory@LocalWorkflow@U2@@2VQString@@B@@YAXXZ 10022f50 f   KrakenClassifyWorkerFactory.obj
 0001:00021f60       ??__F?PAIRED_END_TEXT@KrakenClassifyWorkerFactory@LocalWorkflow@U2@@2VQString@@B@@YAXXZ 10022f60 f   KrakenClassifyWorkerFactory.obj
 0001:00021f70       ??__F?PAIRED_INPUT_SLOT@KrakenClassifyWorkerFactory@LocalWorkflow@U2@@2VQString@@B@@YAXXZ 10022f70 f   KrakenClassifyWorkerFactory.obj
 0001:00021f80       ??__F?PRELOAD_DATABASE_ATTR_ID@KrakenClassifyWorkerFactory@LocalWorkflow@U2@@2VQString@@B@@YAXXZ 10022f80 f   KrakenClassifyWorkerFactory.obj
 0001:00021f90       ??__F?QUICK_OPERATION_ATTR_ID@KrakenClassifyWorkerFactory@LocalWorkflow@U2@@2VQString@@B@@YAXXZ 10022f90 f   KrakenClassifyWorkerFactory.obj
 0001:00021fa0       ??__F?SINGLE_END_TEXT@KrakenClassifyWorkerFactory@LocalWorkflow@U2@@2VQString@@B@@YAXXZ 10022fa0 f   KrakenClassifyWorkerFactory.obj
 0001:00021fb0       ??__F?THREADS_NUMBER_ATTR_ID@KrakenClassifyWorkerFactory@LocalWorkflow@U2@@2VQString@@B@@YAXXZ 10022fb0 f   KrakenClassifyWorkerFactory.obj
 0001:00021fc0       ??__F?WORKFLOW_CLASSIFY_TOOL_KRAKEN@KrakenClassifyWorkerFactory@LocalWorkflow@U2@@2VQString@@B@@YAXXZ 10022fc0 f   KrakenClassifyWorkerFactory.obj
 0001:00021fd0       ??__F?_Generic_object@?$_Error_objects@H@std@@2V_Generic_error_category@2@A@@YAXXZ 10022fd0 f   KrakenClassifyWorkerFactory.obj
 0001:00021fe0       ??__F?_Iostream_object@?$_Error_objects@H@std@@2V_Iostream_error_category@2@A@@YAXXZ 10022fe0 f   KrakenClassifyWorkerFactory.obj
 0001:00021ff0       ??__F?_System_object@?$_Error_objects@H@std@@2V_System_error_category@2@A@@YAXXZ 10022ff0 f   KrakenClassifyWorkerFactory.obj
 0001:00022000       ??__FalgoLog@U2@@YAXXZ     10023000 f   KrakenClassifyWorkerFactory.obj
 0001:00022010       ??__FcmdLog@U2@@YAXXZ      10023010 f   KrakenClassifyWorkerFactory.obj
 0001:00022020       ??__FcoreLog@U2@@YAXXZ     10023020 f   KrakenClassifyWorkerFactory.obj
 0001:00022030       ??__FioLog@U2@@YAXXZ       10023030 f   KrakenClassifyWorkerFactory.obj
 0001:00022040       ??__FperfLog@U2@@YAXXZ     10023040 f   KrakenClassifyWorkerFactory.obj
 0001:00022050       ??__FscriptLog@U2@@YAXXZ   10023050 f   KrakenClassifyWorkerFactory.obj
 0001:00022060       ??__FtaskLog@U2@@YAXXZ     10023060 f   KrakenClassifyWorkerFactory.obj
 0001:00022070       ??__FuiLog@U2@@YAXXZ       10023070 f   KrakenClassifyWorkerFactory.obj
 0001:00022080       ??__FuserActLog@U2@@YAXXZ  10023080 f   KrakenClassifyWorkerFactory.obj
 0001:00022090       ??__F?BUILD_TOOL@KrakenSupport@U2@@2VQString@@B@@YAXXZ 10023090 f   KrakenSupport.obj
 0001:000220a0       ??__F?BUILD_TOOL_ID@KrakenSupport@U2@@2VQString@@B@@YAXXZ 100230a0 f   KrakenSupport.obj
 0001:000220b0       ??__F?CLASSIFY_TOOL@KrakenSupport@U2@@2VQString@@B@@YAXXZ 100230b0 f   KrakenSupport.obj
 0001:000220c0       ??__F?CLASSIFY_TOOL_ID@KrakenSupport@U2@@2VQString@@B@@YAXXZ 100230c0 f   KrakenSupport.obj
 0001:000220d0       ??__F?GROUP_NAME@KrakenSupport@U2@@2VQString@@B@@YAXXZ 100230d0 f   KrakenSupport.obj
 0001:000220e0       ??__F?_Generic_object@?$_Error_objects@H@std@@2V_Generic_error_category@2@A@@YAXXZ 100230e0 f   KrakenSupport.obj
 0001:000220f0       ??__F?_Iostream_object@?$_Error_objects@H@std@@2V_Iostream_error_category@2@A@@YAXXZ 100230f0 f   KrakenSupport.obj
 0001:00022100       ??__F?_System_object@?$_Error_objects@H@std@@2V_System_error_category@2@A@@YAXXZ 10023100 f   KrakenSupport.obj
 0001:00022110       ??__F?PLUGIN_DESCRIPRION@KrakenSupportPlugin@U2@@2VQString@@B@@YAXXZ 10023110 f   KrakenSupportPlugin.obj
 0001:00022120       ??__F?PLUGIN_NAME@KrakenSupportPlugin@U2@@2VQString@@B@@YAXXZ 10023120 f   KrakenSupportPlugin.obj
 0001:00022130       ??__F?_Generic_object@?$_Error_objects@H@std@@2V_Generic_error_category@2@A@@YAXXZ 10023130 f   KrakenSupportPlugin.obj
 0001:00022140       ??__F?_Iostream_object@?$_Error_objects@H@std@@2V_Iostream_error_category@2@A@@YAXXZ 10023140 f   KrakenSupportPlugin.obj
 0001:00022150       ??__F?_System_object@?$_Error_objects@H@std@@2V_System_error_category@2@A@@YAXXZ 10023150 f   KrakenSupportPlugin.obj
 0001:00022160       ??__FalgoLog@U2@@YAXXZ     10023160 f   KrakenSupportPlugin.obj
 0001:00022170       ??__FcmdLog@U2@@YAXXZ      10023170 f   KrakenSupportPlugin.obj
 0001:00022180       ??__FcoreLog@U2@@YAXXZ     10023180 f   KrakenSupportPlugin.obj
 0001:00022190       ??__FioLog@U2@@YAXXZ       10023190 f   KrakenSupportPlugin.obj
 0001:000221a0       ??__FperfLog@U2@@YAXXZ     100231a0 f   KrakenSupportPlugin.obj
 0001:000221b0       ??__FscriptLog@U2@@YAXXZ   100231b0 f   KrakenSupportPlugin.obj
 0001:000221c0       ??__FtaskLog@U2@@YAXXZ     100231c0 f   KrakenSupportPlugin.obj
 0001:000221d0       ??__FuiLog@U2@@YAXXZ       100231d0 f   KrakenSupportPlugin.obj
 0001:000221e0       ??__FuserActLog@U2@@YAXXZ  100231e0 f   KrakenSupportPlugin.obj
 0001:000221f0       ??__F?_Generic_object@?$_Error_objects@H@std@@2V_Generic_error_category@2@A@@YAXXZ 100231f0 f   KrakenTranslateLogParser.obj
 0001:00022200       ??__F?_Iostream_object@?$_Error_objects@H@std@@2V_Iostream_error_category@2@A@@YAXXZ 10023200 f   KrakenTranslateLogParser.obj
 0001:00022210       ??__F?_System_object@?$_Error_objects@H@std@@2V_System_error_category@2@A@@YAXXZ 10023210 f   KrakenTranslateLogParser.obj
 0001:00022220       ??__F?wellKnownErrors@KrakenTranslateLogParser@U2@@0VQStringList@@B@@YAXXZ 10023220 f   KrakenTranslateLogParser.obj
 0001:00022230       ??__FalgoLog@U2@@YAXXZ     10023230 f   KrakenTranslateLogParser.obj
 0001:00022240       ??__FcmdLog@U2@@YAXXZ      10023240 f   KrakenTranslateLogParser.obj
 0001:00022250       ??__FcoreLog@U2@@YAXXZ     10023250 f   KrakenTranslateLogParser.obj
 0001:00022260       ??__FioLog@U2@@YAXXZ       10023260 f   KrakenTranslateLogParser.obj
 0001:00022270       ??__FperfLog@U2@@YAXXZ     10023270 f   KrakenTranslateLogParser.obj
 0001:00022280       ??__FscriptLog@U2@@YAXXZ   10023280 f   KrakenTranslateLogParser.obj
 0001:00022290       ??__FtaskLog@U2@@YAXXZ     10023290 f   KrakenTranslateLogParser.obj
 0001:000222a0       ??__FuiLog@U2@@YAXXZ       100232a0 f   KrakenTranslateLogParser.obj
 0001:000222b0       ??__FuserActLog@U2@@YAXXZ  100232b0 f   KrakenTranslateLogParser.obj
 0001:000222c0       ??__F?_Generic_object@?$_Error_objects@H@std@@2V_Generic_error_category@2@A@@YAXXZ 100232c0 f   moc_KrakenBuildPrompter.obj
 0001:000222d0       ??__F?_Iostream_object@?$_Error_objects@H@std@@2V_Iostream_error_category@2@A@@YAXXZ 100232d0 f   moc_KrakenBuildPrompter.obj
 0001:000222e0       ??__F?_System_object@?$_Error_objects@H@std@@2V_System_error_category@2@A@@YAXXZ 100232e0 f   moc_KrakenBuildPrompter.obj
 0001:000222f0       ??__FalgoLog@U2@@YAXXZ     100232f0 f   moc_KrakenBuildPrompter.obj
 0001:00022300       ??__FcmdLog@U2@@YAXXZ      10023300 f   moc_KrakenBuildPrompter.obj
 0001:00022310       ??__FcoreLog@U2@@YAXXZ     10023310 f   moc_KrakenBuildPrompter.obj
 0001:00022320       ??__FioLog@U2@@YAXXZ       10023320 f   moc_KrakenBuildPrompter.obj
 0001:00022330       ??__FperfLog@U2@@YAXXZ     10023330 f   moc_KrakenBuildPrompter.obj
 0001:00022340       ??__FscriptLog@U2@@YAXXZ   10023340 f   moc_KrakenBuildPrompter.obj
 0001:00022350       ??__FtaskLog@U2@@YAXXZ     10023350 f   moc_KrakenBuildPrompter.obj
 0001:00022360       ??__FuiLog@U2@@YAXXZ       10023360 f   moc_KrakenBuildPrompter.obj
 0001:00022370       ??__FuserActLog@U2@@YAXXZ  10023370 f   moc_KrakenBuildPrompter.obj
 0001:00022380       ??__F?_Generic_object@?$_Error_objects@H@std@@2V_Generic_error_category@2@A@@YAXXZ 10023380 f   moc_KrakenBuildTask.obj
 0001:00022390       ??__F?_Iostream_object@?$_Error_objects@H@std@@2V_Iostream_error_category@2@A@@YAXXZ 10023390 f   moc_KrakenBuildTask.obj
 0001:000223a0       ??__F?_System_object@?$_Error_objects@H@std@@2V_System_error_category@2@A@@YAXXZ 100233a0 f   moc_KrakenBuildTask.obj
 0001:000223b0       ??__FalgoLog@U2@@YAXXZ     100233b0 f   moc_KrakenBuildTask.obj
 0001:000223c0       ??__FcmdLog@U2@@YAXXZ      100233c0 f   moc_KrakenBuildTask.obj
 0001:000223d0       ??__FcoreLog@U2@@YAXXZ     100233d0 f   moc_KrakenBuildTask.obj
 0001:000223e0       ??__FioLog@U2@@YAXXZ       100233e0 f   moc_KrakenBuildTask.obj
 0001:000223f0       ??__FperfLog@U2@@YAXXZ     100233f0 f   moc_KrakenBuildTask.obj
 0001:00022400       ??__FscriptLog@U2@@YAXXZ   10023400 f   moc_KrakenBuildTask.obj
 0001:00022410       ??__FtaskLog@U2@@YAXXZ     10023410 f   moc_KrakenBuildTask.obj
 0001:00022420       ??__FuiLog@U2@@YAXXZ       10023420 f   moc_KrakenBuildTask.obj
 0001:00022430       ??__FuserActLog@U2@@YAXXZ  10023430 f   moc_KrakenBuildTask.obj
 0001:00022440       ??__F?_Generic_object@?$_Error_objects@H@std@@2V_Generic_error_category@2@A@@YAXXZ 10023440 f   moc_KrakenBuildWorker.obj
 0001:00022450       ??__F?_Iostream_object@?$_Error_objects@H@std@@2V_Iostream_error_category@2@A@@YAXXZ 10023450 f   moc_KrakenBuildWorker.obj
 0001:00022460       ??__F?_System_object@?$_Error_objects@H@std@@2V_System_error_category@2@A@@YAXXZ 10023460 f   moc_KrakenBuildWorker.obj
 0001:00022470       ??__FalgoLog@U2@@YAXXZ     10023470 f   moc_KrakenBuildWorker.obj
 0001:00022480       ??__FcmdLog@U2@@YAXXZ      10023480 f   moc_KrakenBuildWorker.obj
 0001:00022490       ??__FcoreLog@U2@@YAXXZ     10023490 f   moc_KrakenBuildWorker.obj
 0001:000224a0       ??__FioLog@U2@@YAXXZ       100234a0 f   moc_KrakenBuildWorker.obj
 0001:000224b0       ??__FperfLog@U2@@YAXXZ     100234b0 f   moc_KrakenBuildWorker.obj
 0001:000224c0       ??__FscriptLog@U2@@YAXXZ   100234c0 f   moc_KrakenBuildWorker.obj
 0001:000224d0       ??__FtaskLog@U2@@YAXXZ     100234d0 f   moc_KrakenBuildWorker.obj
 0001:000224e0       ??__FuiLog@U2@@YAXXZ       100234e0 f   moc_KrakenBuildWorker.obj
 0001:000224f0       ??__FuserActLog@U2@@YAXXZ  100234f0 f   moc_KrakenBuildWorker.obj
 0001:00022500       ??__F?_Generic_object@?$_Error_objects@H@std@@2V_Generic_error_category@2@A@@YAXXZ 10023500 f   moc_KrakenClassifyPrompter.obj
 0001:00022510       ??__F?_Iostream_object@?$_Error_objects@H@std@@2V_Iostream_error_category@2@A@@YAXXZ 10023510 f   moc_KrakenClassifyPrompter.obj
 0001:00022520       ??__F?_System_object@?$_Error_objects@H@std@@2V_System_error_category@2@A@@YAXXZ 10023520 f   moc_KrakenClassifyPrompter.obj
 0001:00022530       ??__FalgoLog@U2@@YAXXZ     10023530 f   moc_KrakenClassifyPrompter.obj
 0001:00022540       ??__FcmdLog@U2@@YAXXZ      10023540 f   moc_KrakenClassifyPrompter.obj
 0001:00022550       ??__FcoreLog@U2@@YAXXZ     10023550 f   moc_KrakenClassifyPrompter.obj
 0001:00022560       ??__FioLog@U2@@YAXXZ       10023560 f   moc_KrakenClassifyPrompter.obj
 0001:00022570       ??__FperfLog@U2@@YAXXZ     10023570 f   moc_KrakenClassifyPrompter.obj
 0001:00022580       ??__FscriptLog@U2@@YAXXZ   10023580 f   moc_KrakenClassifyPrompter.obj
 0001:00022590       ??__FtaskLog@U2@@YAXXZ     10023590 f   moc_KrakenClassifyPrompter.obj
 0001:000225a0       ??__FuiLog@U2@@YAXXZ       100235a0 f   moc_KrakenClassifyPrompter.obj
 0001:000225b0       ??__FuserActLog@U2@@YAXXZ  100235b0 f   moc_KrakenClassifyPrompter.obj
 0001:000225c0       ??__F?_Generic_object@?$_Error_objects@H@std@@2V_Generic_error_category@2@A@@YAXXZ 100235c0 f   moc_KrakenClassifyTask.obj
 0001:000225d0       ??__F?_Iostream_object@?$_Error_objects@H@std@@2V_Iostream_error_category@2@A@@YAXXZ 100235d0 f   moc_KrakenClassifyTask.obj
 0001:000225e0       ??__F?_System_object@?$_Error_objects@H@std@@2V_System_error_category@2@A@@YAXXZ 100235e0 f   moc_KrakenClassifyTask.obj
 0001:000225f0       ??__FalgoLog@U2@@YAXXZ     100235f0 f   moc_KrakenClassifyTask.obj
 0001:00022600       ??__FcmdLog@U2@@YAXXZ      10023600 f   moc_KrakenClassifyTask.obj
 0001:00022610       ??__FcoreLog@U2@@YAXXZ     10023610 f   moc_KrakenClassifyTask.obj
 0001:00022620       ??__FioLog@U2@@YAXXZ       10023620 f   moc_KrakenClassifyTask.obj
 0001:00022630       ??__FperfLog@U2@@YAXXZ     10023630 f   moc_KrakenClassifyTask.obj
 0001:00022640       ??__FscriptLog@U2@@YAXXZ   10023640 f   moc_KrakenClassifyTask.obj
 0001:00022650       ??__FtaskLog@U2@@YAXXZ     10023650 f   moc_KrakenClassifyTask.obj
 0001:00022660       ??__FuiLog@U2@@YAXXZ       10023660 f   moc_KrakenClassifyTask.obj
 0001:00022670       ??__FuserActLog@U2@@YAXXZ  10023670 f   moc_KrakenClassifyTask.obj
 0001:00022680       ??__F?_Generic_object@?$_Error_objects@H@std@@2V_Generic_error_category@2@A@@YAXXZ 10023680 f   moc_KrakenClassifyWorker.obj
 0001:00022690       ??__F?_Iostream_object@?$_Error_objects@H@std@@2V_Iostream_error_category@2@A@@YAXXZ 10023690 f   moc_KrakenClassifyWorker.obj
 0001:000226a0       ??__F?_System_object@?$_Error_objects@H@std@@2V_System_error_category@2@A@@YAXXZ 100236a0 f   moc_KrakenClassifyWorker.obj
 0001:000226b0       ??__FalgoLog@U2@@YAXXZ     100236b0 f   moc_KrakenClassifyWorker.obj
 0001:000226c0       ??__FcmdLog@U2@@YAXXZ      100236c0 f   moc_KrakenClassifyWorker.obj
 0001:000226d0       ??__FcoreLog@U2@@YAXXZ     100236d0 f   moc_KrakenClassifyWorker.obj
 0001:000226e0       ??__FioLog@U2@@YAXXZ       100236e0 f   moc_KrakenClassifyWorker.obj
 0001:000226f0       ??__FperfLog@U2@@YAXXZ     100236f0 f   moc_KrakenClassifyWorker.obj
 0001:00022700       ??__FscriptLog@U2@@YAXXZ   10023700 f   moc_KrakenClassifyWorker.obj
 0001:00022710       ??__FtaskLog@U2@@YAXXZ     10023710 f   moc_KrakenClassifyWorker.obj
 0001:00022720       ??__FuiLog@U2@@YAXXZ       10023720 f   moc_KrakenClassifyWorker.obj
 0001:00022730       ??__FuserActLog@U2@@YAXXZ  10023730 f   moc_KrakenClassifyWorker.obj
 0001:00022740       ??__F?_Generic_object@?$_Error_objects@H@std@@2V_Generic_error_category@2@A@@YAXXZ 10023740 f   moc_KrakenSupport.obj
 0001:00022750       ??__F?_Iostream_object@?$_Error_objects@H@std@@2V_Iostream_error_category@2@A@@YAXXZ 10023750 f   moc_KrakenSupport.obj
 0001:00022760       ??__F?_System_object@?$_Error_objects@H@std@@2V_System_error_category@2@A@@YAXXZ 10023760 f   moc_KrakenSupport.obj
 0001:00022770       ??__F?_Generic_object@?$_Error_objects@H@std@@2V_Generic_error_category@2@A@@YAXXZ 10023770 f   moc_KrakenSupportPlugin.obj
 0001:00022780       ??__F?_Iostream_object@?$_Error_objects@H@std@@2V_Iostream_error_category@2@A@@YAXXZ 10023780 f   moc_KrakenSupportPlugin.obj
 0001:00022790       ??__F?_System_object@?$_Error_objects@H@std@@2V_System_error_category@2@A@@YAXXZ 10023790 f   moc_KrakenSupportPlugin.obj
 0002:000008c0       _algoLog$initializer$      100248c0     DatabaseSizeRelation.obj
 0002:000008c4       _cmdLog$initializer$       100248c4     DatabaseSizeRelation.obj
 0002:000008c8       _coreLog$initializer$      100248c8     DatabaseSizeRelation.obj
 0002:000008cc       _ioLog$initializer$        100248cc     DatabaseSizeRelation.obj
 0002:000008d0       _perfLog$initializer$      100248d0     DatabaseSizeRelation.obj
 0002:000008d4       _scriptLog$initializer$    100248d4     DatabaseSizeRelation.obj
 0002:000008d8       _taskLog$initializer$      100248d8     DatabaseSizeRelation.obj
 0002:000008dc       _uiLog$initializer$        100248dc     DatabaseSizeRelation.obj
 0002:000008e0       _userActLog$initializer$   100248e0     DatabaseSizeRelation.obj
 0002:000008e4       ?_Generic_object$initializer$@?$_Error_objects@H@std@@2P6AXXZA 100248e4     DatabaseSizeRelation.obj
 0002:000008e8       ?_Iostream_object$initializer$@?$_Error_objects@H@std@@2P6AXXZA 100248e8     DatabaseSizeRelation.obj
 0002:000008ec       ?_System_object$initializer$@?$_Error_objects@H@std@@2P6AXXZA 100248ec     DatabaseSizeRelation.obj
 0002:000008f0       _algoLog$initializer$      100248f0     KrakenBuildPrompter.obj
 0002:000008f4       _cmdLog$initializer$       100248f4     KrakenBuildPrompter.obj
 0002:000008f8       _coreLog$initializer$      100248f8     KrakenBuildPrompter.obj
 0002:000008fc       _ioLog$initializer$        100248fc     KrakenBuildPrompter.obj
 0002:00000900       _perfLog$initializer$      10024900     KrakenBuildPrompter.obj
 0002:00000904       _scriptLog$initializer$    10024904     KrakenBuildPrompter.obj
 0002:00000908       _taskLog$initializer$      10024908     KrakenBuildPrompter.obj
 0002:0000090c       _uiLog$initializer$        1002490c     KrakenBuildPrompter.obj
 0002:00000910       _userActLog$initializer$   10024910     KrakenBuildPrompter.obj
 0002:00000914       _algoLog$initializer$      10024914     KrakenBuildTask.obj
 0002:00000918       _cmdLog$initializer$       10024918     KrakenBuildTask.obj
 0002:0000091c       _coreLog$initializer$      1002491c     KrakenBuildTask.obj
 0002:00000920       _ioLog$initializer$        10024920     KrakenBuildTask.obj
 0002:00000924       _perfLog$initializer$      10024924     KrakenBuildTask.obj
 0002:00000928       _scriptLog$initializer$    10024928     KrakenBuildTask.obj
 0002:0000092c       _taskLog$initializer$      1002492c     KrakenBuildTask.obj
 0002:00000930       _uiLog$initializer$        10024930     KrakenBuildTask.obj
 0002:00000934       _userActLog$initializer$   10024934     KrakenBuildTask.obj
 0002:00000938       ?BUILD$initializer$@KrakenBuildTaskSettings@U2@@2P6AXXZA 10024938     KrakenBuildTask.obj
 0002:0000093c       ?SHRINK$initializer$@KrakenBuildTaskSettings@U2@@2P6AXXZA 1002493c     KrakenBuildTask.obj
 0002:00000940       _algoLog$initializer$      10024940     KrakenBuildValidator.obj
 0002:00000944       _cmdLog$initializer$       10024944     KrakenBuildValidator.obj
 0002:00000948       _coreLog$initializer$      10024948     KrakenBuildValidator.obj
 0002:0000094c       _ioLog$initializer$        1002494c     KrakenBuildValidator.obj
 0002:00000950       _perfLog$initializer$      10024950     KrakenBuildValidator.obj
 0002:00000954       _scriptLog$initializer$    10024954     KrakenBuildValidator.obj
 0002:00000958       _taskLog$initializer$      10024958     KrakenBuildValidator.obj
 0002:0000095c       _uiLog$initializer$        1002495c     KrakenBuildValidator.obj
 0002:00000960       _userActLog$initializer$   10024960     KrakenBuildValidator.obj
 0002:00000964       _algoLog$initializer$      10024964     KrakenBuildWorker.obj
 0002:00000968       _cmdLog$initializer$       10024968     KrakenBuildWorker.obj
 0002:0000096c       _coreLog$initializer$      1002496c     KrakenBuildWorker.obj
 0002:00000970       _ioLog$initializer$        10024970     KrakenBuildWorker.obj
 0002:00000974       _perfLog$initializer$      10024974     KrakenBuildWorker.obj
 0002:00000978       _scriptLog$initializer$    10024978     KrakenBuildWorker.obj
 0002:0000097c       _taskLog$initializer$      1002497c     KrakenBuildWorker.obj
 0002:00000980       _uiLog$initializer$        10024980     KrakenBuildWorker.obj
 0002:00000984       _userActLog$initializer$   10024984     KrakenBuildWorker.obj
 0002:00000988       _algoLog$initializer$      10024988     KrakenBuildWorkerFactory.obj
 0002:0000098c       _cmdLog$initializer$       1002498c     KrakenBuildWorkerFactory.obj
 0002:00000990       _coreLog$initializer$      10024990     KrakenBuildWorkerFactory.obj
 0002:00000994       _ioLog$initializer$        10024994     KrakenBuildWorkerFactory.obj
 0002:00000998       _perfLog$initializer$      10024998     KrakenBuildWorkerFactory.obj
 0002:0000099c       _scriptLog$initializer$    1002499c     KrakenBuildWorkerFactory.obj
 0002:000009a0       _taskLog$initializer$      100249a0     KrakenBuildWorkerFactory.obj
 0002:000009a4       _uiLog$initializer$        100249a4     KrakenBuildWorkerFactory.obj
 0002:000009a8       _userActLog$initializer$   100249a8     KrakenBuildWorkerFactory.obj
 0002:000009ac       ?ACTOR_ID$initializer$@KrakenBuildWorkerFactory@LocalWorkflow@U2@@2P6AXXZA 100249ac     KrakenBuildWorkerFactory.obj
 0002:000009b0       ?OUTPUT_PORT_ID$initializer$@KrakenBuildWorkerFactory@LocalWorkflow@U2@@2P6AXXZA 100249b0     KrakenBuildWorkerFactory.obj
 0002:000009b4       ?MODE_ATTR_ID$initializer$@KrakenBuildWorkerFactory@LocalWorkflow@U2@@2P6AXXZA 100249b4     KrakenBuildWorkerFactory.obj
 0002:000009b8       ?INPUT_DATABASE_NAME_ATTR_ID$initializer$@KrakenBuildWorkerFactory@LocalWorkflow@U2@@2P6AXXZA 100249b8     KrakenBuildWorkerFactory.obj
 0002:000009bc       ?NEW_DATABASE_NAME_ATTR_ID$initializer$@KrakenBuildWorkerFactory@LocalWorkflow@U2@@2P6AXXZA 100249bc     KrakenBuildWorkerFactory.obj
 0002:000009c0       ?GENOMIC_LIBRARY_ATTR_ID$initializer$@KrakenBuildWorkerFactory@LocalWorkflow@U2@@2P6AXXZA 100249c0     KrakenBuildWorkerFactory.obj
 0002:000009c4       ?NUMBER_OF_K_MERS_ATTR_ID$initializer$@KrakenBuildWorkerFactory@LocalWorkflow@U2@@2P6AXXZA 100249c4     KrakenBuildWorkerFactory.obj
 0002:000009c8       ?K_MER_LENGTH_ATTR_ID$initializer$@KrakenBuildWorkerFactory@LocalWorkflow@U2@@2P6AXXZA 100249c8     KrakenBuildWorkerFactory.obj
 0002:000009cc       ?MINIMIZER_LENGTH_ATTR_ID$initializer$@KrakenBuildWorkerFactory@LocalWorkflow@U2@@2P6AXXZA 100249cc     KrakenBuildWorkerFactory.obj
 0002:000009d0       ?MAXIMUM_DATABASE_SIZE_ATTR_ID$initializer$@KrakenBuildWorkerFactory@LocalWorkflow@U2@@2P6AXXZA 100249d0     KrakenBuildWorkerFactory.obj
 0002:000009d4       ?SHRINK_BLOCK_OFFSET_ATTR_ID$initializer$@KrakenBuildWorkerFactory@LocalWorkflow@U2@@2P6AXXZA 100249d4     KrakenBuildWorkerFactory.obj
 0002:000009d8       ?CLEAN_ATTR_ID$initializer$@KrakenBuildWorkerFactory@LocalWorkflow@U2@@2P6AXXZA 100249d8     KrakenBuildWorkerFactory.obj
 0002:000009dc       ?WORK_ON_DISK_ATTR_ID$initializer$@KrakenBuildWorkerFactory@LocalWorkflow@U2@@2P6AXXZA 100249dc     KrakenBuildWorkerFactory.obj
 0002:000009e0       ?JELLYFISH_HASH_SIZE_ATTR_ID$initializer$@KrakenBuildWorkerFactory@LocalWorkflow@U2@@2P6AXXZA 100249e0     KrakenBuildWorkerFactory.obj
 0002:000009e4       ?THREADS_NUMBER_ATTR_ID$initializer$@KrakenBuildWorkerFactory@LocalWorkflow@U2@@2P6AXXZA 100249e4     KrakenBuildWorkerFactory.obj
 0002:000009e8       _algoLog$initializer$      100249e8     KrakenClassifyLogParser.obj
 0002:000009ec       _cmdLog$initializer$       100249ec     KrakenClassifyLogParser.obj
 0002:000009f0       _coreLog$initializer$      100249f0     KrakenClassifyLogParser.obj
 0002:000009f4       _ioLog$initializer$        100249f4     KrakenClassifyLogParser.obj
 0002:000009f8       _perfLog$initializer$      100249f8     KrakenClassifyLogParser.obj
 0002:000009fc       _scriptLog$initializer$    100249fc     KrakenClassifyLogParser.obj
 0002:00000a00       _taskLog$initializer$      10024a00     KrakenClassifyLogParser.obj
 0002:00000a04       _uiLog$initializer$        10024a04     KrakenClassifyLogParser.obj
 0002:00000a08       _userActLog$initializer$   10024a08     KrakenClassifyLogParser.obj
 0002:00000a0c       ?wellKnownErrors$initializer$@KrakenClassifyLogParser@U2@@0P6AXXZA 10024a0c     KrakenClassifyLogParser.obj
 0002:00000a10       _algoLog$initializer$      10024a10     KrakenClassifyPrompter.obj
 0002:00000a14       _cmdLog$initializer$       10024a14     KrakenClassifyPrompter.obj
 0002:00000a18       _coreLog$initializer$      10024a18     KrakenClassifyPrompter.obj
 0002:00000a1c       _ioLog$initializer$        10024a1c     KrakenClassifyPrompter.obj
 0002:00000a20       _perfLog$initializer$      10024a20     KrakenClassifyPrompter.obj
 0002:00000a24       _scriptLog$initializer$    10024a24     KrakenClassifyPrompter.obj
 0002:00000a28       _taskLog$initializer$      10024a28     KrakenClassifyPrompter.obj
 0002:00000a2c       _uiLog$initializer$        10024a2c     KrakenClassifyPrompter.obj
 0002:00000a30       _userActLog$initializer$   10024a30     KrakenClassifyPrompter.obj
 0002:00000a34       _algoLog$initializer$      10024a34     KrakenClassifyTask.obj
 0002:00000a38       _cmdLog$initializer$       10024a38     KrakenClassifyTask.obj
 0002:00000a3c       _coreLog$initializer$      10024a3c     KrakenClassifyTask.obj
 0002:00000a40       _ioLog$initializer$        10024a40     KrakenClassifyTask.obj
 0002:00000a44       _perfLog$initializer$      10024a44     KrakenClassifyTask.obj
 0002:00000a48       _scriptLog$initializer$    10024a48     KrakenClassifyTask.obj
 0002:00000a4c       _taskLog$initializer$      10024a4c     KrakenClassifyTask.obj
 0002:00000a50       _uiLog$initializer$        10024a50     KrakenClassifyTask.obj
 0002:00000a54       _userActLog$initializer$   10024a54     KrakenClassifyTask.obj
 0002:00000a58       ?SINGLE_END$initializer$@KrakenClassifyTaskSettings@U2@@2P6AXXZA 10024a58     KrakenClassifyTask.obj
 0002:00000a5c       ?PAIRED_END$initializer$@KrakenClassifyTaskSettings@U2@@2P6AXXZA 10024a5c     KrakenClassifyTask.obj
 0002:00000a60       _algoLog$initializer$      10024a60     KrakenClassifyValidator.obj
 0002:00000a64       _cmdLog$initializer$       10024a64     KrakenClassifyValidator.obj
 0002:00000a68       _coreLog$initializer$      10024a68     KrakenClassifyValidator.obj
 0002:00000a6c       _ioLog$initializer$        10024a6c     KrakenClassifyValidator.obj
 0002:00000a70       _perfLog$initializer$      10024a70     KrakenClassifyValidator.obj
 0002:00000a74       _scriptLog$initializer$    10024a74     KrakenClassifyValidator.obj
 0002:00000a78       _taskLog$initializer$      10024a78     KrakenClassifyValidator.obj
 0002:00000a7c       _uiLog$initializer$        10024a7c     KrakenClassifyValidator.obj
 0002:00000a80       _userActLog$initializer$   10024a80     KrakenClassifyValidator.obj
 0002:00000a84       _algoLog$initializer$      10024a84     KrakenClassifyWorker.obj
 0002:00000a88       _cmdLog$initializer$       10024a88     KrakenClassifyWorker.obj
 0002:00000a8c       _coreLog$initializer$      10024a8c     KrakenClassifyWorker.obj
 0002:00000a90       _ioLog$initializer$        10024a90     KrakenClassifyWorker.obj
 0002:00000a94       _perfLog$initializer$      10024a94     KrakenClassifyWorker.obj
 0002:00000a98       _scriptLog$initializer$    10024a98     KrakenClassifyWorker.obj
 0002:00000a9c       _taskLog$initializer$      10024a9c     KrakenClassifyWorker.obj
 0002:00000aa0       _uiLog$initializer$        10024aa0     KrakenClassifyWorker.obj
 0002:00000aa4       _userActLog$initializer$   10024aa4     KrakenClassifyWorker.obj
 0002:00000aa8       ?KRAKEN_DIR$initializer$@KrakenClassifyWorker@LocalWorkflow@U2@@0P6AXXZA 10024aa8     KrakenClassifyWorker.obj
 0002:00000aac       _algoLog$initializer$      10024aac     KrakenClassifyWorkerFactory.obj
 0002:00000ab0       _cmdLog$initializer$       10024ab0     KrakenClassifyWorkerFactory.obj
 0002:00000ab4       _coreLog$initializer$      10024ab4     KrakenClassifyWorkerFactory.obj
 0002:00000ab8       _ioLog$initializer$        10024ab8     KrakenClassifyWorkerFactory.obj
 0002:00000abc       _perfLog$initializer$      10024abc     KrakenClassifyWorkerFactory.obj
 0002:00000ac0       _scriptLog$initializer$    10024ac0     KrakenClassifyWorkerFactory.obj
 0002:00000ac4       _taskLog$initializer$      10024ac4     KrakenClassifyWorkerFactory.obj
 0002:00000ac8       _uiLog$initializer$        10024ac8     KrakenClassifyWorkerFactory.obj
 0002:00000acc       _userActLog$initializer$   10024acc     KrakenClassifyWorkerFactory.obj
 0002:00000ad0       ?ACTOR_ID$initializer$@KrakenClassifyWorkerFactory@LocalWorkflow@U2@@2P6AXXZA 10024ad0     KrakenClassifyWorkerFactory.obj
 0002:00000ad4       ?INPUT_PORT_ID$initializer$@KrakenClassifyWorkerFactory@LocalWorkflow@U2@@2P6AXXZA 10024ad4     KrakenClassifyWorkerFactory.obj
 0002:00000ad8       ?OUTPUT_PORT_ID$initializer$@KrakenClassifyWorkerFactory@LocalWorkflow@U2@@2P6AXXZA 10024ad8     KrakenClassifyWorkerFactory.obj
 0002:00000adc       ?INPUT_SLOT$initializer$@KrakenClassifyWorkerFactory@LocalWorkflow@U2@@2P6AXXZA 10024adc     KrakenClassifyWorkerFactory.obj
 0002:00000ae0       ?PAIRED_INPUT_SLOT$initializer$@KrakenClassifyWorkerFactory@LocalWorkflow@U2@@2P6AXXZA 10024ae0     KrakenClassifyWorkerFactory.obj
 0002:00000ae4       ?INPUT_DATA_ATTR_ID$initializer$@KrakenClassifyWorkerFactory@LocalWorkflow@U2@@2P6AXXZA 10024ae4     KrakenClassifyWorkerFactory.obj
 0002:00000ae8       ?DATABASE_ATTR_ID$initializer$@KrakenClassifyWorkerFactory@LocalWorkflow@U2@@2P6AXXZA 10024ae8     KrakenClassifyWorkerFactory.obj
 0002:00000aec       ?OUTPUT_URL_ATTR_ID$initializer$@KrakenClassifyWorkerFactory@LocalWorkflow@U2@@2P6AXXZA 10024aec     KrakenClassifyWorkerFactory.obj
 0002:00000af0       ?QUICK_OPERATION_ATTR_ID$initializer$@KrakenClassifyWorkerFactory@LocalWorkflow@U2@@2P6AXXZA 10024af0     KrakenClassifyWorkerFactory.obj
 0002:00000af4       ?MIN_HITS_NUMBER_ATTR_ID$initializer$@KrakenClassifyWorkerFactory@LocalWorkflow@U2@@2P6AXXZA 10024af4     KrakenClassifyWorkerFactory.obj
 0002:00000af8       ?THREADS_NUMBER_ATTR_ID$initializer$@KrakenClassifyWorkerFactory@LocalWorkflow@U2@@2P6AXXZA 10024af8     KrakenClassifyWorkerFactory.obj
 0002:00000afc       ?PRELOAD_DATABASE_ATTR_ID$initializer$@KrakenClassifyWorkerFactory@LocalWorkflow@U2@@2P6AXXZA 10024afc     KrakenClassifyWorkerFactory.obj
 0002:00000b00       ?SINGLE_END_TEXT$initializer$@KrakenClassifyWorkerFactory@LocalWorkflow@U2@@2P6AXXZA 10024b00     KrakenClassifyWorkerFactory.obj
 0002:00000b04       ?PAIRED_END_TEXT$initializer$@KrakenClassifyWorkerFactory@LocalWorkflow@U2@@2P6AXXZA 10024b04     KrakenClassifyWorkerFactory.obj
 0002:00000b08       ?WORKFLOW_CLASSIFY_TOOL_KRAKEN$initializer$@KrakenClassifyWorkerFactory@LocalWorkflow@U2@@2P6AXXZA 10024b08     KrakenClassifyWorkerFactory.obj
 0002:00000b0c       ?BUILD_TOOL$initializer$@KrakenSupport@U2@@2P6AXXZA 10024b0c     KrakenSupport.obj
 0002:00000b10       ?BUILD_TOOL_ID$initializer$@KrakenSupport@U2@@2P6AXXZA 10024b10     KrakenSupport.obj
 0002:00000b14       ?CLASSIFY_TOOL$initializer$@KrakenSupport@U2@@2P6AXXZA 10024b14     KrakenSupport.obj
 0002:00000b18       ?CLASSIFY_TOOL_ID$initializer$@KrakenSupport@U2@@2P6AXXZA 10024b18     KrakenSupport.obj
 0002:00000b1c       ?GROUP_NAME$initializer$@KrakenSupport@U2@@2P6AXXZA 10024b1c     KrakenSupport.obj
 0002:00000b20       _algoLog$initializer$      10024b20     KrakenSupportPlugin.obj
 0002:00000b24       _cmdLog$initializer$       10024b24     KrakenSupportPlugin.obj
 0002:00000b28       _coreLog$initializer$      10024b28     KrakenSupportPlugin.obj
 0002:00000b2c       _ioLog$initializer$        10024b2c     KrakenSupportPlugin.obj
 0002:00000b30       _perfLog$initializer$      10024b30     KrakenSupportPlugin.obj
 0002:00000b34       _scriptLog$initializer$    10024b34     KrakenSupportPlugin.obj
 0002:00000b38       _taskLog$initializer$      10024b38     KrakenSupportPlugin.obj
 0002:00000b3c       _uiLog$initializer$        10024b3c     KrakenSupportPlugin.obj
 0002:00000b40       _userActLog$initializer$   10024b40     KrakenSupportPlugin.obj
 0002:00000b44       ?PLUGIN_NAME$initializer$@KrakenSupportPlugin@U2@@2P6AXXZA 10024b44     KrakenSupportPlugin.obj
 0002:00000b48       ?PLUGIN_DESCRIPRION$initializer$@KrakenSupportPlugin@U2@@2P6AXXZA 10024b48     KrakenSupportPlugin.obj
 0002:00000b4c       _algoLog$initializer$      10024b4c     KrakenTranslateLogParser.obj
 0002:00000b50       _cmdLog$initializer$       10024b50     KrakenTranslateLogParser.obj
 0002:00000b54       _coreLog$initializer$      10024b54     KrakenTranslateLogParser.obj
 0002:00000b58       _ioLog$initializer$        10024b58     KrakenTranslateLogParser.obj
 0002:00000b5c       _perfLog$initializer$      10024b5c     KrakenTranslateLogParser.obj
 0002:00000b60       _scriptLog$initializer$    10024b60     KrakenTranslateLogParser.obj
 0002:00000b64       _taskLog$initializer$      10024b64     KrakenTranslateLogParser.obj
 0002:00000b68       _uiLog$initializer$        10024b68     KrakenTranslateLogParser.obj
 0002:00000b6c       _userActLog$initializer$   10024b6c     KrakenTranslateLogParser.obj
 0002:00000b70       ?wellKnownErrors$initializer$@KrakenTranslateLogParser@U2@@0P6AXXZA 10024b70     KrakenTranslateLogParser.obj
 0002:00000b74       _algoLog$initializer$      10024b74     moc_KrakenBuildPrompter.obj
 0002:00000b78       _cmdLog$initializer$       10024b78     moc_KrakenBuildPrompter.obj
 0002:00000b7c       _coreLog$initializer$      10024b7c     moc_KrakenBuildPrompter.obj
 0002:00000b80       _ioLog$initializer$        10024b80     moc_KrakenBuildPrompter.obj
 0002:00000b84       _perfLog$initializer$      10024b84     moc_KrakenBuildPrompter.obj
 0002:00000b88       _scriptLog$initializer$    10024b88     moc_KrakenBuildPrompter.obj
 0002:00000b8c       _taskLog$initializer$      10024b8c     moc_KrakenBuildPrompter.obj
 0002:00000b90       _uiLog$initializer$        10024b90     moc_KrakenBuildPrompter.obj
 0002:00000b94       _userActLog$initializer$   10024b94     moc_KrakenBuildPrompter.obj
 0002:00000b98       ?staticMetaObject$initializer$@KrakenBuildPrompter@LocalWorkflow@U2@@2P6AXXZA 10024b98     moc_KrakenBuildPrompter.obj
 0002:00000b9c       _algoLog$initializer$      10024b9c     moc_KrakenBuildTask.obj
 0002:00000ba0       _cmdLog$initializer$       10024ba0     moc_KrakenBuildTask.obj
 0002:00000ba4       _coreLog$initializer$      10024ba4     moc_KrakenBuildTask.obj
 0002:00000ba8       _ioLog$initializer$        10024ba8     moc_KrakenBuildTask.obj
 0002:00000bac       _perfLog$initializer$      10024bac     moc_KrakenBuildTask.obj
 0002:00000bb0       _scriptLog$initializer$    10024bb0     moc_KrakenBuildTask.obj
 0002:00000bb4       _taskLog$initializer$      10024bb4     moc_KrakenBuildTask.obj
 0002:00000bb8       _uiLog$initializer$        10024bb8     moc_KrakenBuildTask.obj
 0002:00000bbc       _userActLog$initializer$   10024bbc     moc_KrakenBuildTask.obj
 0002:00000bc0       ?staticMetaObject$initializer$@KrakenBuildTask@U2@@2P6AXXZA 10024bc0     moc_KrakenBuildTask.obj
 0002:00000bc4       _algoLog$initializer$      10024bc4     moc_KrakenBuildWorker.obj
 0002:00000bc8       _cmdLog$initializer$       10024bc8     moc_KrakenBuildWorker.obj
 0002:00000bcc       _coreLog$initializer$      10024bcc     moc_KrakenBuildWorker.obj
 0002:00000bd0       _ioLog$initializer$        10024bd0     moc_KrakenBuildWorker.obj
 0002:00000bd4       _perfLog$initializer$      10024bd4     moc_KrakenBuildWorker.obj
 0002:00000bd8       _scriptLog$initializer$    10024bd8     moc_KrakenBuildWorker.obj
 0002:00000bdc       _taskLog$initializer$      10024bdc     moc_KrakenBuildWorker.obj
 0002:00000be0       _uiLog$initializer$        10024be0     moc_KrakenBuildWorker.obj
 0002:00000be4       _userActLog$initializer$   10024be4     moc_KrakenBuildWorker.obj
 0002:00000be8       ?staticMetaObject$initializer$@KrakenBuildWorker@LocalWorkflow@U2@@2P6AXXZA 10024be8     moc_KrakenBuildWorker.obj
 0002:00000bec       _algoLog$initializer$      10024bec     moc_KrakenClassifyPrompter.obj
 0002:00000bf0       _cmdLog$initializer$       10024bf0     moc_KrakenClassifyPrompter.obj
 0002:00000bf4       _coreLog$initializer$      10024bf4     moc_KrakenClassifyPrompter.obj
 0002:00000bf8       _ioLog$initializer$        10024bf8     moc_KrakenClassifyPrompter.obj
 0002:00000bfc       _perfLog$initializer$      10024bfc     moc_KrakenClassifyPrompter.obj
 0002:00000c00       _scriptLog$initializer$    10024c00     moc_KrakenClassifyPrompter.obj
 0002:00000c04       _taskLog$initializer$      10024c04     moc_KrakenClassifyPrompter.obj
 0002:00000c08       _uiLog$initializer$        10024c08     moc_KrakenClassifyPrompter.obj
 0002:00000c0c       _userActLog$initializer$   10024c0c     moc_KrakenClassifyPrompter.obj
 0002:00000c10       ?staticMetaObject$initializer$@KrakenClassifyPrompter@LocalWorkflow@U2@@2P6AXXZA 10024c10     moc_KrakenClassifyPrompter.obj
 0002:00000c14       _algoLog$initializer$      10024c14     moc_KrakenClassifyTask.obj
 0002:00000c18       _cmdLog$initializer$       10024c18     moc_KrakenClassifyTask.obj
 0002:00000c1c       _coreLog$initializer$      10024c1c     moc_KrakenClassifyTask.obj
 0002:00000c20       _ioLog$initializer$        10024c20     moc_KrakenClassifyTask.obj
 0002:00000c24       _perfLog$initializer$      10024c24     moc_KrakenClassifyTask.obj
 0002:00000c28       _scriptLog$initializer$    10024c28     moc_KrakenClassifyTask.obj
 0002:00000c2c       _taskLog$initializer$      10024c2c     moc_KrakenClassifyTask.obj
 0002:00000c30       _uiLog$initializer$        10024c30     moc_KrakenClassifyTask.obj
 0002:00000c34       _userActLog$initializer$   10024c34     moc_KrakenClassifyTask.obj
 0002:00000c38       ?staticMetaObject$initializer$@KrakenClassifyTask@U2@@2P6AXXZA 10024c38     moc_KrakenClassifyTask.obj
 0002:00000c3c       _algoLog$initializer$      10024c3c     moc_KrakenClassifyWorker.obj
 0002:00000c40       _cmdLog$initializer$       10024c40     moc_KrakenClassifyWorker.obj
 0002:00000c44       _coreLog$initializer$      10024c44     moc_KrakenClassifyWorker.obj
 0002:00000c48       _ioLog$initializer$        10024c48     moc_KrakenClassifyWorker.obj
 0002:00000c4c       _perfLog$initializer$      10024c4c     moc_KrakenClassifyWorker.obj
 0002:00000c50       _scriptLog$initializer$    10024c50     moc_KrakenClassifyWorker.obj
 0002:00000c54       _taskLog$initializer$      10024c54     moc_KrakenClassifyWorker.obj
 0002:00000c58       _uiLog$initializer$        10024c58     moc_KrakenClassifyWorker.obj
 0002:00000c5c       _userActLog$initializer$   10024c5c     moc_KrakenClassifyWorker.obj
 0002:00000c60       ?staticMetaObject$initializer$@KrakenClassifyWorker@LocalWorkflow@U2@@2P6AXXZA 10024c60     moc_KrakenClassifyWorker.obj
 0002:00000c64       ?staticMetaObject$initializer$@KrakenSupport@U2@@2P6AXXZA 10024c64     moc_KrakenSupport.obj
 0002:00000c68       ?staticMetaObject$initializer$@KrakenSupportPlugin@U2@@2P6AXXZA 10024c68     moc_KrakenSupportPlugin.obj
 0002:00000c74       _pcinit                    10024c74     MSVCRT:crtdll.obj
 0002:00000c78       _pinit                     10024c78     MSVCRT:atonexit.obj
 0002:00003b28       _qt_meta_stringdata_U2__LocalWorkflow__KrakenBuildPrompter 10027b28     moc_KrakenBuildPrompter.obj
 0002:00003b60       _qt_meta_data_U2__LocalWorkflow__KrakenBuildPrompter 10027b60     moc_KrakenBuildPrompter.obj
 0002:00003b9c       _qt_meta_stringdata_U2__KrakenBuildTask 10027b9c     moc_KrakenBuildTask.obj
 0002:00003bc0       _qt_meta_data_U2__KrakenBuildTask 10027bc0     moc_KrakenBuildTask.obj
 0002:00003c00       _qt_meta_stringdata_U2__LocalWorkflow__KrakenBuildWorker 10027c00     moc_KrakenBuildWorker.obj
 0002:00003c98       _qt_meta_data_U2__LocalWorkflow__KrakenBuildWorker 10027c98     moc_KrakenBuildWorker.obj
 0002:00003cf4       _qt_meta_stringdata_U2__LocalWorkflow__KrakenClassifyPrompter 10027cf4     moc_KrakenClassifyPrompter.obj
 0002:00003d30       _qt_meta_data_U2__LocalWorkflow__KrakenClassifyPrompter 10027d30     moc_KrakenClassifyPrompter.obj
 0002:00003d6c       _qt_meta_stringdata_U2__KrakenClassifyTask 10027d6c     moc_KrakenClassifyTask.obj
 0002:00003d94       _qt_meta_data_U2__KrakenClassifyTask 10027d94     moc_KrakenClassifyTask.obj
 0002:00003dd0       _qt_meta_stringdata_U2__LocalWorkflow__KrakenClassifyWorker 10027dd0     moc_KrakenClassifyWorker.obj
 0002:00003e68       _qt_meta_data_U2__LocalWorkflow__KrakenClassifyWorker 10027e68     moc_KrakenClassifyWorker.obj
 0002:00003ec4       _qt_meta_data_U2__KrakenSupport 10027ec4     moc_KrakenSupport.obj
 0002:00003f00       _qt_meta_stringdata_U2__KrakenSupport 10027f00     moc_KrakenSupport.obj
 0002:00003f24       _qt_meta_stringdata_U2__KrakenSupportPlugin 10027f24     moc_KrakenSupportPlugin.obj
 0002:00003f4c       _qt_meta_data_U2__KrakenSupportPlugin 10027f4c     moc_KrakenSupportPlugin.obj
 0002:00003f98       _GS_ExceptionPointers      10027f98     MSVCRT:gs_report.obj
 0002:00005a88       __catchsym$?_Copy@?$basic_string@DU?$char_traits@D@std@@V?$allocator@D@2@@std@@QAEXII@Z$5 10029a88     DatabaseSizeRelation.obj
 0002:00005a98       __catchsym$?_Copy@?$basic_string@DU?$char_traits@D@std@@V?$allocator@D@2@@std@@QAEXII@Z$4 10029a98     DatabaseSizeRelation.obj
 0002:00005aa8       __unwindtable$?_Copy@?$basic_string@DU?$char_traits@D@std@@V?$allocator@D@2@@std@@QAEXII@Z 10029aa8     DatabaseSizeRelation.obj
 0002:00005ac8       __ehfuncinfo$?_Copy@?$basic_string@DU?$char_traits@D@std@@V?$allocator@D@2@@std@@QAEXII@Z 10029ac8     DatabaseSizeRelation.obj
 0002:00005aec       __tryblocktable$?_Copy@?$basic_string@DU?$char_traits@D@std@@V?$allocator@D@2@@std@@QAEXII@Z 10029aec     DatabaseSizeRelation.obj
 0002:00005b14       __unwindtable$??H@YA?BVQString@@ABV0@PBD@Z 10029b14     DatabaseSizeRelation.obj
 0002:00005b24       __ehfuncinfo$??H@YA?BVQString@@ABV0@PBD@Z 10029b24     DatabaseSizeRelation.obj
 0002:00005b48       __unwindtable$??__EalgoLog@U2@@YAXXZ 10029b48     DatabaseSizeRelation.obj
 0002:00005b50       __ehfuncinfo$??__EalgoLog@U2@@YAXXZ 10029b50     DatabaseSizeRelation.obj
 0002:00005b74       __unwindtable$??__EcmdLog@U2@@YAXXZ 10029b74     DatabaseSizeRelation.obj
 0002:00005b7c       __ehfuncinfo$??__EcmdLog@U2@@YAXXZ 10029b7c     DatabaseSizeRelation.obj
 0002:00005ba0       __unwindtable$??__EcoreLog@U2@@YAXXZ 10029ba0     DatabaseSizeRelation.obj
 0002:00005ba8       __ehfuncinfo$??__EcoreLog@U2@@YAXXZ 10029ba8     DatabaseSizeRelation.obj
 0002:00005bcc       __unwindtable$??__EioLog@U2@@YAXXZ 10029bcc     DatabaseSizeRelation.obj
 0002:00005bd4       __ehfuncinfo$??__EioLog@U2@@YAXXZ 10029bd4     DatabaseSizeRelation.obj
 0002:00005bf8       __unwindtable$??__EperfLog@U2@@YAXXZ 10029bf8     DatabaseSizeRelation.obj
 0002:00005c00       __ehfuncinfo$??__EperfLog@U2@@YAXXZ 10029c00     DatabaseSizeRelation.obj
 0002:00005c24       __unwindtable$??__EscriptLog@U2@@YAXXZ 10029c24     DatabaseSizeRelation.obj
 0002:00005c2c       __ehfuncinfo$??__EscriptLog@U2@@YAXXZ 10029c2c     DatabaseSizeRelation.obj
 0002:00005c50       __unwindtable$??__EtaskLog@U2@@YAXXZ 10029c50     DatabaseSizeRelation.obj
 0002:00005c58       __ehfuncinfo$??__EtaskLog@U2@@YAXXZ 10029c58     DatabaseSizeRelation.obj
 0002:00005c7c       __unwindtable$??__EuiLog@U2@@YAXXZ 10029c7c     DatabaseSizeRelation.obj
 0002:00005c84       __ehfuncinfo$??__EuiLog@U2@@YAXXZ 10029c84     DatabaseSizeRelation.obj
 0002:00005ca8       __unwindtable$??__EuserActLog@U2@@YAXXZ 10029ca8     DatabaseSizeRelation.obj
 0002:00005cb0       __ehfuncinfo$??__EuserActLog@U2@@YAXXZ 10029cb0     DatabaseSizeRelation.obj
 0002:00005cd4       __unwindtable$??0DatabaseSizeRelation@LocalWorkflow@U2@@QAE@ABVQString@@@Z 10029cd4     DatabaseSizeRelation.obj
 0002:00005cec       __ehfuncinfo$??0DatabaseSizeRelation@LocalWorkflow@U2@@QAE@ABVQString@@@Z 10029cec     DatabaseSizeRelation.obj
 0002:00005d10       __ehfuncinfo$?getAffectResult@DatabaseSizeRelation@LocalWorkflow@U2@@UBE?AVQVariant@@ABV4@0PAVDelegateTags@3@1@Z 10029d10     DatabaseSizeRelation.obj
 0002:00005d34       __unwindtable$?getAffectResult@DatabaseSizeRelation@LocalWorkflow@U2@@UBE?AVQVariant@@ABV4@0PAVDelegateTags@3@1@Z 10029d34     DatabaseSizeRelation.obj
 0002:00005d5c       __unwindtable$?clone@DatabaseSizeRelation@LocalWorkflow@U2@@UBEPAV123@XZ 10029d5c     DatabaseSizeRelation.obj
 0002:00005d64       __ehfuncinfo$?clone@DatabaseSizeRelation@LocalWorkflow@U2@@UBEPAV123@XZ 10029d64     DatabaseSizeRelation.obj
 0002:00005d88       __unwindtable$??__EalgoLog@U2@@YAXXZ 10029d88     KrakenBuildPrompter.obj
 0002:00005d90       __ehfuncinfo$??__EalgoLog@U2@@YAXXZ 10029d90     KrakenBuildPrompter.obj
 0002:00005db4       __unwindtable$??__EcmdLog@U2@@YAXXZ 10029db4     KrakenBuildPrompter.obj
 0002:00005dbc       __ehfuncinfo$??__EcmdLog@U2@@YAXXZ 10029dbc     KrakenBuildPrompter.obj
 0002:00005de0       __unwindtable$??__EcoreLog@U2@@YAXXZ 10029de0     KrakenBuildPrompter.obj
 0002:00005de8       __ehfuncinfo$??__EcoreLog@U2@@YAXXZ 10029de8     KrakenBuildPrompter.obj
 0002:00005e0c       __unwindtable$??__EioLog@U2@@YAXXZ 10029e0c     KrakenBuildPrompter.obj
 0002:00005e14       __ehfuncinfo$??__EioLog@U2@@YAXXZ 10029e14     KrakenBuildPrompter.obj
 0002:00005e38       __unwindtable$??__EperfLog@U2@@YAXXZ 10029e38     KrakenBuildPrompter.obj
 0002:00005e40       __ehfuncinfo$??__EperfLog@U2@@YAXXZ 10029e40     KrakenBuildPrompter.obj
 0002:00005e64       __unwindtable$??__EscriptLog@U2@@YAXXZ 10029e64     KrakenBuildPrompter.obj
 0002:00005e6c       __ehfuncinfo$??__EscriptLog@U2@@YAXXZ 10029e6c     KrakenBuildPrompter.obj
 0002:00005e90       __unwindtable$??__EtaskLog@U2@@YAXXZ 10029e90     KrakenBuildPrompter.obj
 0002:00005e98       __ehfuncinfo$??__EtaskLog@U2@@YAXXZ 10029e98     KrakenBuildPrompter.obj
 0002:00005ebc       __unwindtable$??__EuiLog@U2@@YAXXZ 10029ebc     KrakenBuildPrompter.obj
 0002:00005ec4       __ehfuncinfo$??__EuiLog@U2@@YAXXZ 10029ec4     KrakenBuildPrompter.obj
 0002:00005ee8       __unwindtable$??__EuserActLog@U2@@YAXXZ 10029ee8     KrakenBuildPrompter.obj
 0002:00005ef0       __ehfuncinfo$??__EuserActLog@U2@@YAXXZ 10029ef0     KrakenBuildPrompter.obj
 0002:00005f14       __ehfuncinfo$?createDescription@?$PrompterBase@VKrakenBuildPrompter@LocalWorkflow@U2@@@U2@@UAEPAVActorDocument@Workflow@2@PAVActor@42@@Z 10029f14     KrakenBuildPrompter.obj
 0002:00005f38       __unwindtable$?createDescription@?$PrompterBase@VKrakenBuildPrompter@LocalWorkflow@U2@@@U2@@UAEPAVActorDocument@Workflow@2@PAVActor@42@@Z 10029f38     KrakenBuildPrompter.obj
 0002:00005f70       __ehfuncinfo$?composeRichDoc@KrakenBuildPrompter@LocalWorkflow@U2@@EAE?AVQString@@XZ 10029f70     KrakenBuildPrompter.obj
 0002:00005f94       __unwindtable$?composeRichDoc@KrakenBuildPrompter@LocalWorkflow@U2@@EAE?AVQString@@XZ 10029f94     KrakenBuildPrompter.obj
 0002:0000606c       __catchsym$??0?$QList@PAVPort@Workflow@U2@@@@QAE@ABV0@@Z$2 1002a06c     KrakenBuildPrompter.obj
 0002:0000607c       __unwindtable$??0?$QList@PAVPort@Workflow@U2@@@@QAE@ABV0@@Z 1002a07c     KrakenBuildPrompter.obj
 0002:0000608c       __tryblocktable$??0?$QList@PAVPort@Workflow@U2@@@@QAE@ABV0@@Z 1002a08c     KrakenBuildPrompter.obj
 0002:000060a0       __ehfuncinfo$??0?$QList@PAVPort@Workflow@U2@@@@QAE@ABV0@@Z 1002a0a0     KrakenBuildPrompter.obj
 0002:000060c4       __unwindtable$??H@YA?BVQString@@ABV0@0@Z 1002a0c4     KrakenBuildTask.obj
 0002:000060cc       __ehfuncinfo$??H@YA?BVQString@@ABV0@0@Z 1002a0cc     KrakenBuildTask.obj
 0002:000060f0       __catchsym$??0?$QList@VQString@@@@QAE@ABV0@@Z$2 1002a0f0     KrakenBuildTask.obj
 0002:00006100       __unwindtable$??0?$QList@VQString@@@@QAE@ABV0@@Z 1002a100     KrakenBuildTask.obj
 0002:00006110       __tryblocktable$??0?$QList@VQString@@@@QAE@ABV0@@Z 1002a110     KrakenBuildTask.obj
 0002:00006124       __ehfuncinfo$??0?$QList@VQString@@@@QAE@ABV0@@Z 1002a124     KrakenBuildTask.obj
 0002:00006148       __catchsym$?append@?$QList@VQString@@@@QAEXABVQString@@@Z$13 1002a148     KrakenBuildTask.obj
 0002:00006158       __catchsym$?append@?$QList@VQString@@@@QAEXABVQString@@@Z$12 1002a158     KrakenBuildTask.obj
 0002:00006168       __ehfuncinfo$?append@?$QList@VQString@@@@QAEXABVQString@@@Z 1002a168     KrakenBuildTask.obj
 0002:0000618c       __tryblocktable$?append@?$QList@VQString@@@@QAEXABVQString@@@Z 1002a18c     KrakenBuildTask.obj
 0002:000061b4       __unwindtable$?append@?$QList@VQString@@@@QAEXABVQString@@@Z 1002a1b4     KrakenBuildTask.obj
 0002:00006214       __catchsym$?detach_helper_grow@?$QList@VQString@@@@AAEPAUNode@1@HH@Z$5 1002a214     KrakenBuildTask.obj
 0002:00006224       __catchsym$?detach_helper_grow@?$QList@VQString@@@@AAEPAUNode@1@HH@Z$4 1002a224     KrakenBuildTask.obj
 0002:00006234       __unwindtable$?detach_helper_grow@?$QList@VQString@@@@AAEPAUNode@1@HH@Z 1002a234     KrakenBuildTask.obj
 0002:00006254       __ehfuncinfo$?detach_helper_grow@?$QList@VQString@@@@AAEPAUNode@1@HH@Z 1002a254     KrakenBuildTask.obj
 0002:00006278       __tryblocktable$?detach_helper_grow@?$QList@VQString@@@@AAEPAUNode@1@HH@Z 1002a278     KrakenBuildTask.obj
 0002:000062a0       __unwindtable$?node_construct@?$QList@VQString@@@@AAEXPAUNode@1@ABVQString@@@Z 1002a2a0     KrakenBuildTask.obj
 0002:000062b0       __ehfuncinfo$?node_construct@?$QList@VQString@@@@AAEXPAUNode@1@ABVQString@@@Z 1002a2b0     KrakenBuildTask.obj
 0002:000062d4       __catchsym$?node_copy@?$QList@VQString@@@@AAEXPAUNode@1@00@Z$6 1002a2d4     KrakenBuildTask.obj
 0002:000062e4       __tryblocktable$?node_copy@?$QList@VQString@@@@AAEXPAUNode@1@00@Z 1002a2e4     KrakenBuildTask.obj
 0002:000062f8       __ehfuncinfo$?node_copy@?$QList@VQString@@@@AAEXPAUNode@1@00@Z 1002a2f8     KrakenBuildTask.obj
 0002:0000631c       __unwindtable$?node_copy@?$QList@VQString@@@@AAEXPAUNode@1@00@Z 1002a31c     KrakenBuildTask.obj
 0002:0000634c       __unwindtable$??__EalgoLog@U2@@YAXXZ 1002a34c     KrakenBuildTask.obj
 0002:00006354       __ehfuncinfo$??__EalgoLog@U2@@YAXXZ 1002a354     KrakenBuildTask.obj
 0002:00006378       __unwindtable$??__EcmdLog@U2@@YAXXZ 1002a378     KrakenBuildTask.obj
 0002:00006380       __ehfuncinfo$??__EcmdLog@U2@@YAXXZ 1002a380     KrakenBuildTask.obj
 0002:000063a4       __unwindtable$??__EcoreLog@U2@@YAXXZ 1002a3a4     KrakenBuildTask.obj
 0002:000063ac       __ehfuncinfo$??__EcoreLog@U2@@YAXXZ 1002a3ac     KrakenBuildTask.obj
 0002:000063d0       __unwindtable$??__EioLog@U2@@YAXXZ 1002a3d0     KrakenBuildTask.obj
 0002:000063d8       __ehfuncinfo$??__EioLog@U2@@YAXXZ 1002a3d8     KrakenBuildTask.obj
 0002:000063fc       __unwindtable$??__EperfLog@U2@@YAXXZ 1002a3fc     KrakenBuildTask.obj
 0002:00006404       __ehfuncinfo$??__EperfLog@U2@@YAXXZ 1002a404     KrakenBuildTask.obj
 0002:00006428       __unwindtable$??__EscriptLog@U2@@YAXXZ 1002a428     KrakenBuildTask.obj
 0002:00006430       __ehfuncinfo$??__EscriptLog@U2@@YAXXZ 1002a430     KrakenBuildTask.obj
 0002:00006454       __unwindtable$??__EtaskLog@U2@@YAXXZ 1002a454     KrakenBuildTask.obj
 0002:0000645c       __ehfuncinfo$??__EtaskLog@U2@@YAXXZ 1002a45c     KrakenBuildTask.obj
 0002:00006480       __unwindtable$??__EuiLog@U2@@YAXXZ 1002a480     KrakenBuildTask.obj
 0002:00006488       __ehfuncinfo$??__EuiLog@U2@@YAXXZ 1002a488     KrakenBuildTask.obj
 0002:000064ac       __unwindtable$??__EuserActLog@U2@@YAXXZ 1002a4ac     KrakenBuildTask.obj
 0002:000064b4       __ehfuncinfo$??__EuserActLog@U2@@YAXXZ 1002a4b4     KrakenBuildTask.obj
 0002:000064d8       __catchsym$??0?$QList@PAVTask@U2@@@@QAE@ABV0@@Z$2 1002a4d8     KrakenBuildTask.obj
 0002:000064e8       __unwindtable$??0?$QList@PAVTask@U2@@@@QAE@ABV0@@Z 1002a4e8     KrakenBuildTask.obj
 0002:000064f8       __tryblocktable$??0?$QList@PAVTask@U2@@@@QAE@ABV0@@Z 1002a4f8     KrakenBuildTask.obj
 0002:0000650c       __ehfuncinfo$??0?$QList@PAVTask@U2@@@@QAE@ABV0@@Z 1002a50c     KrakenBuildTask.obj
 0002:00006530       __catchsym$?append@?$QList@PAVTask@U2@@@@QAEXABQAVTask@U2@@@Z$6 1002a530     KrakenBuildTask.obj
 0002:00006540       __tryblocktable$?append@?$QList@PAVTask@U2@@@@QAEXABQAVTask@U2@@@Z 1002a540     KrakenBuildTask.obj
 0002:00006554       __ehfuncinfo$?append@?$QList@PAVTask@U2@@@@QAEXABQAVTask@U2@@@Z 1002a554     KrakenBuildTask.obj
 0002:00006578       __unwindtable$?append@?$QList@PAVTask@U2@@@@QAEXABQAVTask@U2@@@Z 1002a578     KrakenBuildTask.obj
 0002:000065a8       __catchsym$??Y?$QList@PAVTask@U2@@@@QAEAAV0@ABV0@@Z$2 1002a5a8     KrakenBuildTask.obj
 0002:000065b8       __unwindtable$??Y?$QList@PAVTask@U2@@@@QAEAAV0@ABV0@@Z 1002a5b8     KrakenBuildTask.obj
 0002:000065c8       __tryblocktable$??Y?$QList@PAVTask@U2@@@@QAEAAV0@ABV0@@Z 1002a5c8     KrakenBuildTask.obj
 0002:000065dc       __ehfuncinfo$??Y?$QList@PAVTask@U2@@@@QAEAAV0@ABV0@@Z 1002a5dc     KrakenBuildTask.obj
 0002:00006600       __catchsym$?detach_helper_grow@?$QList@PAVTask@U2@@@@AAEPAUNode@1@HH@Z$5 1002a600     KrakenBuildTask.obj
 0002:00006610       __catchsym$?detach_helper_grow@?$QList@PAVTask@U2@@@@AAEPAUNode@1@HH@Z$4 1002a610     KrakenBuildTask.obj
 0002:00006620       __unwindtable$?detach_helper_grow@?$QList@PAVTask@U2@@@@AAEPAUNode@1@HH@Z 1002a620     KrakenBuildTask.obj
 0002:00006640       __ehfuncinfo$?detach_helper_grow@?$QList@PAVTask@U2@@@@AAEPAUNode@1@HH@Z 1002a640     KrakenBuildTask.obj
 0002:00006664       __tryblocktable$?detach_helper_grow@?$QList@PAVTask@U2@@@@AAEPAUNode@1@HH@Z 1002a664     KrakenBuildTask.obj
 0002:0000668c       __unwindtable$??0KrakenBuildTaskSettings@U2@@QAE@XZ 1002a68c     KrakenBuildTask.obj
 0002:0000669c       __ehfuncinfo$??0KrakenBuildTaskSettings@U2@@QAE@XZ 1002a69c     KrakenBuildTask.obj
 0002:000066c0       __unwindtable$??1KrakenBuildTaskSettings@U2@@QAE@XZ 1002a6c0     KrakenBuildTask.obj
 0002:000066d8       __ehfuncinfo$??1KrakenBuildTaskSettings@U2@@QAE@XZ 1002a6d8     KrakenBuildTask.obj
 0002:000066fc       __unwindtable$??0KrakenBuildTaskSettings@U2@@QAE@ABU01@@Z 1002a6fc     KrakenBuildTask.obj
 0002:00006714       __ehfuncinfo$??0KrakenBuildTaskSettings@U2@@QAE@ABU01@@Z 1002a714     KrakenBuildTask.obj
 0002:00006738       __ehfuncinfo$??0KrakenBuildTask@U2@@QAE@ABUKrakenBuildTaskSettings@1@@Z 1002a738     KrakenBuildTask.obj
 0002:0000675c       __unwindtable$??0KrakenBuildTask@U2@@QAE@ABUKrakenBuildTaskSettings@1@@Z 1002a75c     KrakenBuildTask.obj
 0002:000067bc       __ehfuncinfo$?prepare@KrakenBuildTask@U2@@EAEXXZ 1002a7bc     KrakenBuildTask.obj
 0002:000067e0       __unwindtable$?prepare@KrakenBuildTask@U2@@EAEXXZ 1002a7e0     KrakenBuildTask.obj
 0002:00006980       __ehfuncinfo$?checkSettings@KrakenBuildTask@U2@@AAEXXZ 1002a980     KrakenBuildTask.obj
 0002:000069a4       __unwindtable$?checkSettings@KrakenBuildTask@U2@@AAEXXZ 1002a9a4     KrakenBuildTask.obj
 0002:00006a44       __unwindtable$?checkTaxonomy@KrakenBuildTask@U2@@AAEXXZ 1002aa44     KrakenBuildTask.obj
 0002:00006a4c       __ehfuncinfo$?checkTaxonomy@KrakenBuildTask@U2@@AAEXXZ 1002aa4c     KrakenBuildTask.obj
 0002:00006a70       __ehfuncinfo$?prepareTaxonomyData@KrakenBuildTask@U2@@AAE?AV?$QList@PAVTask@U2@@@@XZ 1002aa70     KrakenBuildTask.obj
 0002:00006a94       __unwindtable$?prepareTaxonomyData@KrakenBuildTask@U2@@AAE?AV?$QList@PAVTask@U2@@@@XZ 1002aa94     KrakenBuildTask.obj
 0002:00006b7c       __unwindtable$?getAddToLibraryArguments@KrakenBuildTask@U2@@ABE?AVQStringList@@ABVQString@@@Z 1002ab7c     KrakenBuildTask.obj
 0002:00006b94       __ehfuncinfo$?getAddToLibraryArguments@KrakenBuildTask@U2@@ABE?AVQStringList@@ABVQString@@@Z 1002ab94     KrakenBuildTask.obj
 0002:00006bb8       __ehfuncinfo$?getBuildArguments@KrakenBuildTask@U2@@ABE?AVQStringList@@XZ 1002abb8     KrakenBuildTask.obj
 0002:00006bdc       __unwindtable$?getBuildArguments@KrakenBuildTask@U2@@ABE?AVQStringList@@XZ 1002abdc     KrakenBuildTask.obj
 0002:00006c4c       __unwindtable$?getCleanArguments@KrakenBuildTask@U2@@ABE?AVQStringList@@XZ 1002ac4c     KrakenBuildTask.obj
 0002:00006c64       __ehfuncinfo$?getCleanArguments@KrakenBuildTask@U2@@ABE?AVQStringList@@XZ 1002ac64     KrakenBuildTask.obj
 0002:00006c88       __ehfuncinfo$?getShrinkArguments@KrakenBuildTask@U2@@ABE?AVQStringList@@XZ 1002ac88     KrakenBuildTask.obj
 0002:00006cac       __unwindtable$?getShrinkArguments@KrakenBuildTask@U2@@ABE?AVQStringList@@XZ 1002acac     KrakenBuildTask.obj
 0002:00006d1c       __unwindtable$??1KrakenBuildTask@U2@@UAE@XZ 1002ad1c     KrakenBuildTask.obj
 0002:00006d3c       __ehfuncinfo$??1KrakenBuildTask@U2@@UAE@XZ 1002ad3c     KrakenBuildTask.obj
 0002:00006d60       __unwindtable$??_GKrakenBuildTask@U2@@UAEPAXI@Z 1002ad60     KrakenBuildTask.obj
 0002:00006d80       __ehfuncinfo$??_GKrakenBuildTask@U2@@UAEPAXI@Z 1002ad80     KrakenBuildTask.obj
 0002:00006da4       __unwindtable$??__EalgoLog@U2@@YAXXZ 1002ada4     KrakenBuildValidator.obj
 0002:00006dac       __ehfuncinfo$??__EalgoLog@U2@@YAXXZ 1002adac     KrakenBuildValidator.obj
 0002:00006dd0       __unwindtable$??__EcmdLog@U2@@YAXXZ 1002add0     KrakenBuildValidator.obj
 0002:00006dd8       __ehfuncinfo$??__EcmdLog@U2@@YAXXZ 1002add8     KrakenBuildValidator.obj
 0002:00006dfc       __unwindtable$??__EcoreLog@U2@@YAXXZ 1002adfc     KrakenBuildValidator.obj
 0002:00006e04       __ehfuncinfo$??__EcoreLog@U2@@YAXXZ 1002ae04     KrakenBuildValidator.obj
 0002:00006e28       __unwindtable$??__EioLog@U2@@YAXXZ 1002ae28     KrakenBuildValidator.obj
 0002:00006e30       __ehfuncinfo$??__EioLog@U2@@YAXXZ 1002ae30     KrakenBuildValidator.obj
 0002:00006e54       __unwindtable$??__EperfLog@U2@@YAXXZ 1002ae54     KrakenBuildValidator.obj
 0002:00006e5c       __ehfuncinfo$??__EperfLog@U2@@YAXXZ 1002ae5c     KrakenBuildValidator.obj
 0002:00006e80       __unwindtable$??__EscriptLog@U2@@YAXXZ 1002ae80     KrakenBuildValidator.obj
 0002:00006e88       __ehfuncinfo$??__EscriptLog@U2@@YAXXZ 1002ae88     KrakenBuildValidator.obj
 0002:00006eac       __unwindtable$??__EtaskLog@U2@@YAXXZ 1002aeac     KrakenBuildValidator.obj
 0002:00006eb4       __ehfuncinfo$??__EtaskLog@U2@@YAXXZ 1002aeb4     KrakenBuildValidator.obj
 0002:00006ed8       __unwindtable$??__EuiLog@U2@@YAXXZ 1002aed8     KrakenBuildValidator.obj
 0002:00006ee0       __ehfuncinfo$??__EuiLog@U2@@YAXXZ 1002aee0     KrakenBuildValidator.obj
 0002:00006f04       __unwindtable$??__EuserActLog@U2@@YAXXZ 1002af04     KrakenBuildValidator.obj
 0002:00006f0c       __ehfuncinfo$??__EuserActLog@U2@@YAXXZ 1002af0c     KrakenBuildValidator.obj
 0002:00006f30       __unwindtable$?validateMinimizerLength@KrakenBuildValidator@Workflow@U2@@ABE_NPBVActor@23@AAV?$QList@VWorkflowNotification@U2@@@@@Z 1002af30     KrakenBuildValidator.obj
 0002:00006f48       __ehfuncinfo$?validateMinimizerLength@KrakenBuildValidator@Workflow@U2@@ABE_NPBVActor@23@AAV?$QList@VWorkflowNotification@U2@@@@@Z 1002af48     KrakenBuildValidator.obj
 0002:00006f6c       __ehfuncinfo$?validateTaxonomy@KrakenBuildValidator@Workflow@U2@@ABE_NPBVActor@23@AAV?$QList@VWorkflowNotification@U2@@@@@Z 1002af6c     KrakenBuildValidator.obj
 0002:00006f90       __unwindtable$?validateTaxonomy@KrakenBuildValidator@Workflow@U2@@ABE_NPBVActor@23@AAV?$QList@VWorkflowNotification@U2@@@@@Z 1002af90     KrakenBuildValidator.obj
 0002:00006fe8       __catchsym$?append@?$QList@VWorkflowNotification@U2@@@@QAEXABVWorkflowNotification@U2@@@Z$11 1002afe8     KrakenBuildValidator.obj
 0002:00006ff8       __catchsym$?append@?$QList@VWorkflowNotification@U2@@@@QAEXABVWorkflowNotification@U2@@@Z$10 1002aff8     KrakenBuildValidator.obj
 0002:00007008       __ehfuncinfo$?append@?$QList@VWorkflowNotification@U2@@@@QAEXABVWorkflowNotification@U2@@@Z 1002b008     KrakenBuildValidator.obj
 0002:0000702c       __tryblocktable$?append@?$QList@VWorkflowNotification@U2@@@@QAEXABVWorkflowNotification@U2@@@Z 1002b02c     KrakenBuildValidator.obj
 0002:00007054       __unwindtable$?append@?$QList@VWorkflowNotification@U2@@@@QAEXABVWorkflowNotification@U2@@@Z 1002b054     KrakenBuildValidator.obj
 0002:000070a4       __catchsym$?detach_helper_grow@?$QList@VWorkflowNotification@U2@@@@AAEPAUNode@1@HH@Z$5 1002b0a4     KrakenBuildValidator.obj
 0002:000070b4       __catchsym$?detach_helper_grow@?$QList@VWorkflowNotification@U2@@@@AAEPAUNode@1@HH@Z$4 1002b0b4     KrakenBuildValidator.obj
 0002:000070c4       __unwindtable$?detach_helper_grow@?$QList@VWorkflowNotification@U2@@@@AAEPAUNode@1@HH@Z 1002b0c4     KrakenBuildValidator.obj
 0002:000070e4       __ehfuncinfo$?detach_helper_grow@?$QList@VWorkflowNotification@U2@@@@AAEPAUNode@1@HH@Z 1002b0e4     KrakenBuildValidator.obj
 0002:00007108       __tryblocktable$?detach_helper_grow@?$QList@VWorkflowNotification@U2@@@@AAEPAUNode@1@HH@Z 1002b108     KrakenBuildValidator.obj
 0002:00007130       __unwindtable$?node_construct@?$QList@VWorkflowNotification@U2@@@@AAEXPAUNode@1@ABVWorkflowNotification@U2@@@Z 1002b130     KrakenBuildValidator.obj
 0002:00007140       __ehfuncinfo$?node_construct@?$QList@VWorkflowNotification@U2@@@@AAEXPAUNode@1@ABVWorkflowNotification@U2@@@Z 1002b140     KrakenBuildValidator.obj
 0002:00007164       __catchsym$?node_copy@?$QList@VWorkflowNotification@U2@@@@AAEXPAUNode@1@00@Z$6 1002b164     KrakenBuildValidator.obj
 0002:00007174       __tryblocktable$?node_copy@?$QList@VWorkflowNotification@U2@@@@AAEXPAUNode@1@00@Z 1002b174     KrakenBuildValidator.obj
 0002:00007188       __ehfuncinfo$?node_copy@?$QList@VWorkflowNotification@U2@@@@AAEXPAUNode@1@00@Z 1002b188     KrakenBuildValidator.obj
 0002:000071ac       __unwindtable$?node_copy@?$QList@VWorkflowNotification@U2@@@@AAEXPAUNode@1@00@Z 1002b1ac     KrakenBuildValidator.obj
 0002:000071dc       __unwindtable$??A?$QMap@VQString@@VQVariant@@@@QAEAAVQVariant@@ABVQString@@@Z 1002b1dc     KrakenBuildWorker.obj
 0002:000071e4       __ehfuncinfo$??A?$QMap@VQString@@VQVariant@@@@QAEAAVQVariant@@ABVQString@@@Z 1002b1e4     KrakenBuildWorker.obj
 0002:00007208       __catchsym$??0?$QList@VDescriptor@U2@@@@QAE@ABV0@@Z$2 1002b208     KrakenBuildWorker.obj
 0002:00007218       __unwindtable$??0?$QList@VDescriptor@U2@@@@QAE@ABV0@@Z 1002b218     KrakenBuildWorker.obj
 0002:00007228       __tryblocktable$??0?$QList@VDescriptor@U2@@@@QAE@ABV0@@Z 1002b228     KrakenBuildWorker.obj
 0002:0000723c       __ehfuncinfo$??0?$QList@VDescriptor@U2@@@@QAE@ABV0@@Z 1002b23c     KrakenBuildWorker.obj
 0002:00007260       __catchsym$?append@?$QList@VDescriptor@U2@@@@QAEXABVDescriptor@U2@@@Z$9 1002b260     KrakenBuildWorker.obj
 0002:00007270       __catchsym$?append@?$QList@VDescriptor@U2@@@@QAEXABVDescriptor@U2@@@Z$8 1002b270     KrakenBuildWorker.obj
 0002:00007280       __ehfuncinfo$?append@?$QList@VDescriptor@U2@@@@QAEXABVDescriptor@U2@@@Z 1002b280     KrakenBuildWorker.obj
 0002:000072a4       __tryblocktable$?append@?$QList@VDescriptor@U2@@@@QAEXABVDescriptor@U2@@@Z 1002b2a4     KrakenBuildWorker.obj
 0002:000072cc       __unwindtable$?append@?$QList@VDescriptor@U2@@@@QAEXABVDescriptor@U2@@@Z 1002b2cc     KrakenBuildWorker.obj
 0002:0000730c       __catchsym$?detach_helper_grow@?$QList@VDescriptor@U2@@@@AAEPAUNode@1@HH@Z$5 1002b30c     KrakenBuildWorker.obj
 0002:0000731c       __catchsym$?detach_helper_grow@?$QList@VDescriptor@U2@@@@AAEPAUNode@1@HH@Z$4 1002b31c     KrakenBuildWorker.obj
 0002:0000732c       __unwindtable$?detach_helper_grow@?$QList@VDescriptor@U2@@@@AAEPAUNode@1@HH@Z 1002b32c     KrakenBuildWorker.obj
 0002:0000734c       __ehfuncinfo$?detach_helper_grow@?$QList@VDescriptor@U2@@@@AAEPAUNode@1@HH@Z 1002b34c     KrakenBuildWorker.obj
 0002:00007370       __tryblocktable$?detach_helper_grow@?$QList@VDescriptor@U2@@@@AAEPAUNode@1@HH@Z 1002b370     KrakenBuildWorker.obj
 0002:00007398       __catchsym$?detach_helper@?$QList@VDescriptor@U2@@@@AAEXH@Z$2 1002b398     KrakenBuildWorker.obj
 0002:000073a8       __unwindtable$?detach_helper@?$QList@VDescriptor@U2@@@@AAEXH@Z 1002b3a8     KrakenBuildWorker.obj
 0002:000073b8       __tryblocktable$?detach_helper@?$QList@VDescriptor@U2@@@@AAEXH@Z 1002b3b8     KrakenBuildWorker.obj
 0002:000073cc       __ehfuncinfo$?detach_helper@?$QList@VDescriptor@U2@@@@AAEXH@Z 1002b3cc     KrakenBuildWorker.obj
 0002:000073f0       __unwindtable$?node_construct@?$QList@VDescriptor@U2@@@@AAEXPAUNode@1@ABVDescriptor@U2@@@Z 1002b3f0     KrakenBuildWorker.obj
 0002:00007400       __ehfuncinfo$?node_construct@?$QList@VDescriptor@U2@@@@AAEXPAUNode@1@ABVDescriptor@U2@@@Z 1002b400     KrakenBuildWorker.obj
 0002:00007424       __catchsym$?node_copy@?$QList@VDescriptor@U2@@@@AAEXPAUNode@1@00@Z$6 1002b424     KrakenBuildWorker.obj
 0002:00007434       __tryblocktable$?node_copy@?$QList@VDescriptor@U2@@@@AAEXPAUNode@1@00@Z 1002b434     KrakenBuildWorker.obj
 0002:00007448       __ehfuncinfo$?node_copy@?$QList@VDescriptor@U2@@@@AAEXPAUNode@1@00@Z 1002b448     KrakenBuildWorker.obj
 0002:0000746c       __unwindtable$?node_copy@?$QList@VDescriptor@U2@@@@AAEXPAUNode@1@00@Z 1002b46c     KrakenBuildWorker.obj
 0002:0000749c       __catchsym$??0?$QList@PAVURLContainer@U2@@@@QAE@ABV0@@Z$2 1002b49c     KrakenBuildWorker.obj
 0002:000074ac       __unwindtable$??0?$QList@PAVURLContainer@U2@@@@QAE@ABV0@@Z 1002b4ac     KrakenBuildWorker.obj
 0002:000074bc       __tryblocktable$??0?$QList@PAVURLContainer@U2@@@@QAE@ABV0@@Z 1002b4bc     KrakenBuildWorker.obj
 0002:000074d0       __ehfuncinfo$??0?$QList@PAVURLContainer@U2@@@@QAE@ABV0@@Z 1002b4d0     KrakenBuildWorker.obj
 0002:000074f4       __catchsym$??0?$QList@VDataset@U2@@@@QAE@ABV0@@Z$2 1002b4f4     KrakenBuildWorker.obj
 0002:00007504       __unwindtable$??0?$QList@VDataset@U2@@@@QAE@ABV0@@Z 1002b504     KrakenBuildWorker.obj
 0002:00007514       __tryblocktable$??0?$QList@VDataset@U2@@@@QAE@ABV0@@Z 1002b514     KrakenBuildWorker.obj
 0002:00007528       __ehfuncinfo$??0?$QList@VDataset@U2@@@@QAE@ABV0@@Z 1002b528     KrakenBuildWorker.obj
 0002:0000754c       __catchsym$?node_copy@?$QList@VDataset@U2@@@@AAEXPAUNode@1@00@Z$6 1002b54c     KrakenBuildWorker.obj
 0002:0000755c       __tryblocktable$?node_copy@?$QList@VDataset@U2@@@@AAEXPAUNode@1@00@Z 1002b55c     KrakenBuildWorker.obj
 0002:00007570       __ehfuncinfo$?node_copy@?$QList@VDataset@U2@@@@AAEXPAUNode@1@00@Z 1002b570     KrakenBuildWorker.obj
 0002:00007594       __unwindtable$?node_copy@?$QList@VDataset@U2@@@@AAEXPAUNode@1@00@Z 1002b594     KrakenBuildWorker.obj
 0002:000075c4       __unwindtable$?qt_metatype_id@?$QMetaTypeId@V?$QList@VDataset@U2@@@@@@SAHXZ 1002b5c4     KrakenBuildWorker.obj
 0002:000075cc       __ehfuncinfo$?qt_metatype_id@?$QMetaTypeId@V?$QList@VDataset@U2@@@@@@SAHXZ 1002b5cc     KrakenBuildWorker.obj
 0002:000075f0       __unwindtable$??$qRegisterMetaType@V?$QList@VDataset@U2@@@@@@YAHPBDPAV?$QList@VDataset@U2@@@@W4DefinedType@?$MetaTypeDefinedHelper@V?$QList@VDataset@U2@@@@$00@QtPrivate@@@Z 1002b5f0     KrakenBuildWorker.obj
 0002:000075f8       __ehfuncinfo$??$qRegisterMetaType@V?$QList@VDataset@U2@@@@@@YAHPBDPAV?$QList@VDataset@U2@@@@W4DefinedType@?$MetaTypeDefinedHelper@V?$QList@VDataset@U2@@@@$00@QtPrivate@@@Z 1002b5f8     KrakenBuildWorker.obj
 0002:0000761c       __unwindtable$??__EalgoLog@U2@@YAXXZ 1002b61c     KrakenBuildWorker.obj
 0002:00007624       __ehfuncinfo$??__EalgoLog@U2@@YAXXZ 1002b624     KrakenBuildWorker.obj
 0002:00007648       __unwindtable$??__EcmdLog@U2@@YAXXZ 1002b648     KrakenBuildWorker.obj
 0002:00007650       __ehfuncinfo$??__EcmdLog@U2@@YAXXZ 1002b650     KrakenBuildWorker.obj
 0002:00007674       __unwindtable$??__EcoreLog@U2@@YAXXZ 1002b674     KrakenBuildWorker.obj
 0002:0000767c       __ehfuncinfo$??__EcoreLog@U2@@YAXXZ 1002b67c     KrakenBuildWorker.obj
 0002:000076a0       __unwindtable$??__EioLog@U2@@YAXXZ 1002b6a0     KrakenBuildWorker.obj
 0002:000076a8       __ehfuncinfo$??__EioLog@U2@@YAXXZ 1002b6a8     KrakenBuildWorker.obj
 0002:000076cc       __unwindtable$??__EperfLog@U2@@YAXXZ 1002b6cc     KrakenBuildWorker.obj
 0002:000076d4       __ehfuncinfo$??__EperfLog@U2@@YAXXZ 1002b6d4     KrakenBuildWorker.obj
 0002:000076f8       __unwindtable$??__EscriptLog@U2@@YAXXZ 1002b6f8     KrakenBuildWorker.obj
 0002:00007700       __ehfuncinfo$??__EscriptLog@U2@@YAXXZ 1002b700     KrakenBuildWorker.obj
 0002:00007724       __unwindtable$??__EtaskLog@U2@@YAXXZ 1002b724     KrakenBuildWorker.obj
 0002:0000772c       __ehfuncinfo$??__EtaskLog@U2@@YAXXZ 1002b72c     KrakenBuildWorker.obj
 0002:00007750       __unwindtable$??__EuiLog@U2@@YAXXZ 1002b750     KrakenBuildWorker.obj
 0002:00007758       __ehfuncinfo$??__EuiLog@U2@@YAXXZ 1002b758     KrakenBuildWorker.obj
 0002:0000777c       __unwindtable$??__EuserActLog@U2@@YAXXZ 1002b77c     KrakenBuildWorker.obj
 0002:00007784       __ehfuncinfo$??__EuserActLog@U2@@YAXXZ 1002b784     KrakenBuildWorker.obj
 0002:000077a8       __unwindtable$??A?$QMap@VQString@@VQScriptValue@@@@QAEAAVQScriptValue@@ABVQString@@@Z 1002b7a8     KrakenBuildWorker.obj
 0002:000077b0       __ehfuncinfo$??A?$QMap@VQString@@VQScriptValue@@@@QAEAAVQScriptValue@@ABVQString@@@Z 1002b7b0     KrakenBuildWorker.obj
 0002:000077d4       __unwindtable$?uniqueKeys@?$QMap@VDescriptor@U2@@VQVariant@@@@QBE?AV?$QList@VDescriptor@U2@@@@XZ 1002b7d4     KrakenBuildWorker.obj
 0002:000077dc       __ehfuncinfo$?uniqueKeys@?$QMap@VDescriptor@U2@@VQVariant@@@@QBE?AV?$QList@VDescriptor@U2@@@@XZ 1002b7dc     KrakenBuildWorker.obj
 0002:00007800       __ehfuncinfo$??$getAttributeValue@VQString@@@Attribute@U2@@QBE?AVQString@@PAVWorkflowContext@Workflow@1@@Z 1002b800     KrakenBuildWorker.obj
 0002:00007824       __unwindtable$??$getAttributeValue@VQString@@@Attribute@U2@@QBE?AVQString@@PAVWorkflowContext@Workflow@1@@Z 1002b824     KrakenBuildWorker.obj
 0002:00007894       __ehfuncinfo$??$getAttributeValue@H@Attribute@U2@@QBEHPAVWorkflowContext@Workflow@1@@Z 1002b894     KrakenBuildWorker.obj
 0002:000078b8       __unwindtable$??$getAttributeValue@H@Attribute@U2@@QBEHPAVWorkflowContext@Workflow@1@@Z 1002b8b8     KrakenBuildWorker.obj
 0002:00007920       __unwindtable$??$getValue@VQString@@@BaseWorker@LocalWorkflow@U2@@IBE?AVQString@@ABV3@@Z 1002b920     KrakenBuildWorker.obj
 0002:00007930       __ehfuncinfo$??$getValue@VQString@@@BaseWorker@LocalWorkflow@U2@@IBE?AVQString@@ABV3@@Z 1002b930     KrakenBuildWorker.obj
 0002:00007954       __ehfuncinfo$?init@KrakenBuildWorker@LocalWorkflow@U2@@UAEXXZ 1002b954     KrakenBuildWorker.obj
 0002:00007978       __unwindtable$?init@KrakenBuildWorker@LocalWorkflow@U2@@UAEXXZ 1002b978     KrakenBuildWorker.obj
 0002:000079b0       __ehfuncinfo$?tick@KrakenBuildWorker@LocalWorkflow@U2@@UAEPAVTask@3@XZ 1002b9b0     KrakenBuildWorker.obj
 0002:000079d4       __unwindtable$?tick@KrakenBuildWorker@LocalWorkflow@U2@@UAEPAVTask@3@XZ 1002b9d4     KrakenBuildWorker.obj
 0002:00007a0c       __ehfuncinfo$?sl_taskFinished@KrakenBuildWorker@LocalWorkflow@U2@@AAEXPAVTask@3@@Z 1002ba0c     KrakenBuildWorker.obj
 0002:00007a30       __unwindtable$?sl_taskFinished@KrakenBuildWorker@LocalWorkflow@U2@@AAEXPAVTask@3@@Z 1002ba30     KrakenBuildWorker.obj
 0002:00007a98       __ehfuncinfo$?getSettings@KrakenBuildWorker@LocalWorkflow@U2@@AAE?AUKrakenBuildTaskSettings@3@XZ 1002ba98     KrakenBuildWorker.obj
 0002:00007abc       __unwindtable$?getSettings@KrakenBuildWorker@LocalWorkflow@U2@@AAE?AUKrakenBuildTaskSettings@3@XZ 1002babc     KrakenBuildWorker.obj
 0002:00007b04       __catchsym$?createNode@?$QMapData@VQString@@VQVariant@@@@QAEPAU?$QMapNode@VQString@@VQVariant@@@@ABVQString@@ABVQVariant@@PAU2@_N@Z$7 1002bb04     KrakenBuildWorker.obj
 0002:00007b14       __catchsym$?createNode@?$QMapData@VQString@@VQVariant@@@@QAEPAU?$QMapNode@VQString@@VQVariant@@@@ABVQString@@ABVQVariant@@PAU2@_N@Z$6 1002bb14     KrakenBuildWorker.obj
 0002:00007b24       __ehfuncinfo$?createNode@?$QMapData@VQString@@VQVariant@@@@QAEPAU?$QMapNode@VQString@@VQVariant@@@@ABVQString@@ABVQVariant@@PAU2@_N@Z 1002bb24     KrakenBuildWorker.obj
 0002:00007b48       __tryblocktable$?createNode@?$QMapData@VQString@@VQVariant@@@@QAEPAU?$QMapNode@VQString@@VQVariant@@@@ABVQString@@ABVQVariant@@PAU2@_N@Z 1002bb48     KrakenBuildWorker.obj
 0002:00007b70       __unwindtable$?createNode@?$QMapData@VQString@@VQVariant@@@@QAEPAU?$QMapNode@VQString@@VQVariant@@@@ABVQString@@ABVQVariant@@PAU2@_N@Z 1002bb70     KrakenBuildWorker.obj
 0002:00007ba0       __catchsym$?createNode@?$QMapData@VQString@@VQScriptValue@@@@QAEPAU?$QMapNode@VQString@@VQScriptValue@@@@ABVQString@@ABVQScriptValue@@PAU2@_N@Z$7 1002bba0     KrakenBuildWorker.obj
 0002:00007bb0       __catchsym$?createNode@?$QMapData@VQString@@VQScriptValue@@@@QAEPAU?$QMapNode@VQString@@VQScriptValue@@@@ABVQString@@ABVQScriptValue@@PAU2@_N@Z$6 1002bbb0     KrakenBuildWorker.obj
 0002:00007bc0       __ehfuncinfo$?createNode@?$QMapData@VQString@@VQScriptValue@@@@QAEPAU?$QMapNode@VQString@@VQScriptValue@@@@ABVQString@@ABVQScriptValue@@PAU2@_N@Z 1002bbc0     KrakenBuildWorker.obj
 0002:00007be4       __tryblocktable$?createNode@?$QMapData@VQString@@VQScriptValue@@@@QAEPAU?$QMapNode@VQString@@VQScriptValue@@@@ABVQString@@ABVQScriptValue@@PAU2@_N@Z 1002bbe4     KrakenBuildWorker.obj
 0002:00007c0c       __unwindtable$?createNode@?$QMapData@VQString@@VQScriptValue@@@@QAEPAU?$QMapNode@VQString@@VQScriptValue@@@@ABVQString@@ABVQScriptValue@@PAU2@_N@Z 1002bc0c     KrakenBuildWorker.obj
 0002:00007c3c       __unwindtable$?metaType@?$QVariantValueHelper@VQString@@@QtPrivate@@SA?AVQString@@ABVQVariant@@@Z 1002bc3c     KrakenBuildWorker.obj
 0002:00007c4c       __ehfuncinfo$?metaType@?$QVariantValueHelper@VQString@@@QtPrivate@@SA?AVQString@@ABVQVariant@@@Z 1002bc4c     KrakenBuildWorker.obj
 0002:00007c70       __unwindtable$?Create@?$QMetaTypeFunctionHelper@V?$QList@VDataset@U2@@@@$00@QtMetaTypePrivate@@SAPAXPBX@Z 1002bc70     KrakenBuildWorker.obj
 0002:00007c78       __ehfuncinfo$?Create@?$QMetaTypeFunctionHelper@V?$QList@VDataset@U2@@@@$00@QtMetaTypePrivate@@SAPAXPBX@Z 1002bc78     KrakenBuildWorker.obj
 0002:00007c9c       __unwindtable$?Construct@?$QMetaTypeFunctionHelper@V?$QList@VDataset@U2@@@@$00@QtMetaTypePrivate@@SAPAXPAXPBX@Z 1002bc9c     KrakenBuildWorker.obj
 0002:00007ca4       __ehfuncinfo$?Construct@?$QMetaTypeFunctionHelper@V?$QList@VDataset@U2@@@@$00@QtMetaTypePrivate@@SAPAXPAXPBX@Z 1002bca4     KrakenBuildWorker.obj
 0002:00007cc8       __unwindtable$?metaType@?$QVariantValueHelper@V?$QList@VDataset@U2@@@@@QtPrivate@@SA?AV?$QList@VDataset@U2@@@@ABVQVariant@@@Z 1002bcc8     KrakenBuildWorker.obj
 0002:00007cd8       __ehfuncinfo$?metaType@?$QVariantValueHelper@V?$QList@VDataset@U2@@@@@QtPrivate@@SA?AV?$QList@VDataset@U2@@@@ABVQVariant@@@Z 1002bcd8     KrakenBuildWorker.obj
 0002:00007cfc       __unwindtable$??__EalgoLog@U2@@YAXXZ 1002bcfc     KrakenBuildWorkerFactory.obj
 0002:00007d04       __ehfuncinfo$??__EalgoLog@U2@@YAXXZ 1002bd04     KrakenBuildWorkerFactory.obj
 0002:00007d28       __unwindtable$??__EcmdLog@U2@@YAXXZ 1002bd28     KrakenBuildWorkerFactory.obj
 0002:00007d30       __ehfuncinfo$??__EcmdLog@U2@@YAXXZ 1002bd30     KrakenBuildWorkerFactory.obj
 0002:00007d54       __unwindtable$??__EcoreLog@U2@@YAXXZ 1002bd54     KrakenBuildWorkerFactory.obj
 0002:00007d5c       __ehfuncinfo$??__EcoreLog@U2@@YAXXZ 1002bd5c     KrakenBuildWorkerFactory.obj
 0002:00007d80       __unwindtable$??__EioLog@U2@@YAXXZ 1002bd80     KrakenBuildWorkerFactory.obj
 0002:00007d88       __ehfuncinfo$??__EioLog@U2@@YAXXZ 1002bd88     KrakenBuildWorkerFactory.obj
 0002:00007dac       __unwindtable$??__EperfLog@U2@@YAXXZ 1002bdac     KrakenBuildWorkerFactory.obj
 0002:00007db4       __ehfuncinfo$??__EperfLog@U2@@YAXXZ 1002bdb4     KrakenBuildWorkerFactory.obj
 0002:00007dd8       __unwindtable$??__EscriptLog@U2@@YAXXZ 1002bdd8     KrakenBuildWorkerFactory.obj
 0002:00007de0       __ehfuncinfo$??__EscriptLog@U2@@YAXXZ 1002bde0     KrakenBuildWorkerFactory.obj
 0002:00007e04       __unwindtable$??__EtaskLog@U2@@YAXXZ 1002be04     KrakenBuildWorkerFactory.obj
 0002:00007e0c       __ehfuncinfo$??__EtaskLog@U2@@YAXXZ 1002be0c     KrakenBuildWorkerFactory.obj
 0002:00007e30       __unwindtable$??__EuiLog@U2@@YAXXZ 1002be30     KrakenBuildWorkerFactory.obj
 0002:00007e38       __ehfuncinfo$??__EuiLog@U2@@YAXXZ 1002be38     KrakenBuildWorkerFactory.obj
 0002:00007e5c       __unwindtable$??__EuserActLog@U2@@YAXXZ 1002be5c     KrakenBuildWorkerFactory.obj
 0002:00007e64       __ehfuncinfo$??__EuserActLog@U2@@YAXXZ 1002be64     KrakenBuildWorkerFactory.obj
 0002:00007e88       __unwindtable$??A?$QMap@VDescriptor@U2@@V?$QExplicitlySharedDataPointer@VDataType@U2@@@@@@QAEAAV?$QExplicitlySharedDataPointer@VDataType@U2@@@@ABVDescriptor@U2@@@Z 1002be88     KrakenBuildWorkerFactory.obj
 0002:00007e90       __ehfuncinfo$??A?$QMap@VDescriptor@U2@@V?$QExplicitlySharedDataPointer@VDataType@U2@@@@@@QAEAAV?$QExplicitlySharedDataPointer@VDataType@U2@@@@ABVDescriptor@U2@@@Z 1002be90     KrakenBuildWorkerFactory.obj
 0002:00007eb4       __catchsym$?append@?$QList@PAVAttribute@U2@@@@QAEXABQAVAttribute@U2@@@Z$6 1002beb4     KrakenBuildWorkerFactory.obj
 0002:00007ec4       __tryblocktable$?append@?$QList@PAVAttribute@U2@@@@QAEXABQAVAttribute@U2@@@Z 1002bec4     KrakenBuildWorkerFactory.obj
 0002:00007ed8       __ehfuncinfo$?append@?$QList@PAVAttribute@U2@@@@QAEXABQAVAttribute@U2@@@Z 1002bed8     KrakenBuildWorkerFactory.obj
 0002:00007efc       __unwindtable$?append@?$QList@PAVAttribute@U2@@@@QAEXABQAVAttribute@U2@@@Z 1002befc     KrakenBuildWorkerFactory.obj
 0002:00007f2c       __catchsym$?detach_helper_grow@?$QList@PAVAttribute@U2@@@@AAEPAUNode@1@HH@Z$5 1002bf2c     KrakenBuildWorkerFactory.obj
 0002:00007f3c       __catchsym$?detach_helper_grow@?$QList@PAVAttribute@U2@@@@AAEPAUNode@1@HH@Z$4 1002bf3c     KrakenBuildWorkerFactory.obj
 0002:00007f4c       __unwindtable$?detach_helper_grow@?$QList@PAVAttribute@U2@@@@AAEPAUNode@1@HH@Z 1002bf4c     KrakenBuildWorkerFactory.obj
 0002:00007f6c       __ehfuncinfo$?detach_helper_grow@?$QList@PAVAttribute@U2@@@@AAEPAUNode@1@HH@Z 1002bf6c     KrakenBuildWorkerFactory.obj
 0002:00007f90       __tryblocktable$?detach_helper_grow@?$QList@PAVAttribute@U2@@@@AAEPAUNode@1@HH@Z 1002bf90     KrakenBuildWorkerFactory.obj
 0002:00007fb8       __catchsym$?append@?$QList@PAVPortDescriptor@Workflow@U2@@@@QAEXABQAVPortDescriptor@Workflow@U2@@@Z$6 1002bfb8     KrakenBuildWorkerFactory.obj
 0002:00007fc8       __tryblocktable$?append@?$QList@PAVPortDescriptor@Workflow@U2@@@@QAEXABQAVPortDescriptor@Workflow@U2@@@Z 1002bfc8     KrakenBuildWorkerFactory.obj
 0002:00007fdc       __ehfuncinfo$?append@?$QList@PAVPortDescriptor@Workflow@U2@@@@QAEXABQAVPortDescriptor@Workflow@U2@@@Z 1002bfdc     KrakenBuildWorkerFactory.obj
 0002:00008000       __unwindtable$?append@?$QList@PAVPortDescriptor@Workflow@U2@@@@QAEXABQAVPortDescriptor@Workflow@U2@@@Z 1002c000     KrakenBuildWorkerFactory.obj
 0002:00008030       __catchsym$?detach_helper_grow@?$QList@PAVPortDescriptor@Workflow@U2@@@@AAEPAUNode@1@HH@Z$5 1002c030     KrakenBuildWorkerFactory.obj
 0002:00008040       __catchsym$?detach_helper_grow@?$QList@PAVPortDescriptor@Workflow@U2@@@@AAEPAUNode@1@HH@Z$4 1002c040     KrakenBuildWorkerFactory.obj
 0002:00008050       __unwindtable$?detach_helper_grow@?$QList@PAVPortDescriptor@Workflow@U2@@@@AAEPAUNode@1@HH@Z 1002c050     KrakenBuildWorkerFactory.obj
 0002:00008070       __ehfuncinfo$?detach_helper_grow@?$QList@PAVPortDescriptor@Workflow@U2@@@@AAEPAUNode@1@HH@Z 1002c070     KrakenBuildWorkerFactory.obj
 0002:00008094       __tryblocktable$?detach_helper_grow@?$QList@PAVPortDescriptor@Workflow@U2@@@@AAEPAUNode@1@HH@Z 1002c094     KrakenBuildWorkerFactory.obj
 0002:000080bc       __unwindtable$?createWorker@KrakenBuildWorkerFactory@LocalWorkflow@U2@@UAEPAVWorker@Workflow@3@PAVActor@53@@Z 1002c0bc     KrakenBuildWorkerFactory.obj
 0002:000080c4       __ehfuncinfo$?createWorker@KrakenBuildWorkerFactory@LocalWorkflow@U2@@UAEPAVWorker@Workflow@3@PAVActor@53@@Z 1002c0c4     KrakenBuildWorkerFactory.obj
 0002:000080e8       __ehfuncinfo$?init@KrakenBuildWorkerFactory@LocalWorkflow@U2@@SAXXZ 1002c0e8     KrakenBuildWorkerFactory.obj
 0002:0000810c       __unwindtable$?init@KrakenBuildWorkerFactory@LocalWorkflow@U2@@SAXXZ 1002c10c     KrakenBuildWorkerFactory.obj
 0002:0000889c       __catchsym$?createNode@?$QMapData@VDescriptor@U2@@V?$QExplicitlySharedDataPointer@VDataType@U2@@@@@@QAEPAU?$QMapNode@VDescriptor@U2@@V?$QExplicitlySharedDataPointer@VDataType@U2@@@@@@ABVDescriptor@U2@@ABV?$QExplicitlySharedDataPointer@VDataType@U2@@@@PAU2@_N@Z$6 1002c89c     KrakenBuildWorkerFactory.obj
 0002:000088ac       __tryblocktable$?createNode@?$QMapData@VDescriptor@U2@@V?$QExplicitlySharedDataPointer@VDataType@U2@@@@@@QAEPAU?$QMapNode@VDescriptor@U2@@V?$QExplicitlySharedDataPointer@VDataType@U2@@@@@@ABVDescriptor@U2@@ABV?$QExplicitlySharedDataPointer@VDataType@U2@@@@PAU2@_N@Z 1002c8ac     KrakenBuildWorkerFactory.obj
 0002:000088c0       __ehfuncinfo$?createNode@?$QMapData@VDescriptor@U2@@V?$QExplicitlySharedDataPointer@VDataType@U2@@@@@@QAEPAU?$QMapNode@VDescriptor@U2@@V?$QExplicitlySharedDataPointer@VDataType@U2@@@@@@ABVDescriptor@U2@@ABV?$QExplicitlySharedDataPointer@VDataType@U2@@@@PAU2@_N@Z 1002c8c0     KrakenBuildWorkerFactory.obj
 0002:000088e4       __unwindtable$?createNode@?$QMapData@VDescriptor@U2@@V?$QExplicitlySharedDataPointer@VDataType@U2@@@@@@QAEPAU?$QMapNode@VDescriptor@U2@@V?$QExplicitlySharedDataPointer@VDataType@U2@@@@@@ABVDescriptor@U2@@ABV?$QExplicitlySharedDataPointer@VDataType@U2@@@@PAU2@_N@Z 1002c8e4     KrakenBuildWorkerFactory.obj
 0002:0000890c       __catchsym$?createNode@?$QMapData@VQString@@PAVPropertyDelegate@U2@@@@QAEPAU?$QMapNode@VQString@@PAVPropertyDelegate@U2@@@@ABVQString@@ABQAVPropertyDelegate@U2@@PAU2@_N@Z$5 1002c90c     KrakenBuildWorkerFactory.obj
 0002:0000891c       __tryblocktable$?createNode@?$QMapData@VQString@@PAVPropertyDelegate@U2@@@@QAEPAU?$QMapNode@VQString@@PAVPropertyDelegate@U2@@@@ABVQString@@ABQAVPropertyDelegate@U2@@PAU2@_N@Z 1002c91c     KrakenBuildWorkerFactory.obj
 0002:00008930       __ehfuncinfo$?createNode@?$QMapData@VQString@@PAVPropertyDelegate@U2@@@@QAEPAU?$QMapNode@VQString@@PAVPropertyDelegate@U2@@@@ABVQString@@ABQAVPropertyDelegate@U2@@PAU2@_N@Z 1002c930     KrakenBuildWorkerFactory.obj
 0002:00008954       __unwindtable$?createNode@?$QMapData@VQString@@PAVPropertyDelegate@U2@@@@QAEPAU?$QMapNode@VQString@@PAVPropertyDelegate@U2@@@@ABVQString@@ABQAVPropertyDelegate@U2@@PAU2@_N@Z 1002c954     KrakenBuildWorkerFactory.obj
 0002:0000897c       __unwindtable$??__EalgoLog@U2@@YAXXZ 1002c97c     KrakenClassifyLogParser.obj
 0002:00008984       __ehfuncinfo$??__EalgoLog@U2@@YAXXZ 1002c984     KrakenClassifyLogParser.obj
 0002:000089a8       __unwindtable$??__EcmdLog@U2@@YAXXZ 1002c9a8     KrakenClassifyLogParser.obj
 0002:000089b0       __ehfuncinfo$??__EcmdLog@U2@@YAXXZ 1002c9b0     KrakenClassifyLogParser.obj
 0002:000089d4       __unwindtable$??__EcoreLog@U2@@YAXXZ 1002c9d4     KrakenClassifyLogParser.obj
 0002:000089dc       __ehfuncinfo$??__EcoreLog@U2@@YAXXZ 1002c9dc     KrakenClassifyLogParser.obj
 0002:00008a00       __unwindtable$??__EioLog@U2@@YAXXZ 1002ca00     KrakenClassifyLogParser.obj
 0002:00008a08       __ehfuncinfo$??__EioLog@U2@@YAXXZ 1002ca08     KrakenClassifyLogParser.obj
 0002:00008a2c       __unwindtable$??__EperfLog@U2@@YAXXZ 1002ca2c     KrakenClassifyLogParser.obj
 0002:00008a34       __ehfuncinfo$??__EperfLog@U2@@YAXXZ 1002ca34     KrakenClassifyLogParser.obj
 0002:00008a58       __unwindtable$??__EscriptLog@U2@@YAXXZ 1002ca58     KrakenClassifyLogParser.obj
 0002:00008a60       __ehfuncinfo$??__EscriptLog@U2@@YAXXZ 1002ca60     KrakenClassifyLogParser.obj
 0002:00008a84       __unwindtable$??__EtaskLog@U2@@YAXXZ 1002ca84     KrakenClassifyLogParser.obj
 0002:00008a8c       __ehfuncinfo$??__EtaskLog@U2@@YAXXZ 1002ca8c     KrakenClassifyLogParser.obj
 0002:00008ab0       __unwindtable$??__EuiLog@U2@@YAXXZ 1002cab0     KrakenClassifyLogParser.obj
 0002:00008ab8       __ehfuncinfo$??__EuiLog@U2@@YAXXZ 1002cab8     KrakenClassifyLogParser.obj
 0002:00008adc       __unwindtable$??__EuserActLog@U2@@YAXXZ 1002cadc     KrakenClassifyLogParser.obj
 0002:00008ae4       __ehfuncinfo$??__EuserActLog@U2@@YAXXZ 1002cae4     KrakenClassifyLogParser.obj
 0002:00008b08       __unwindtable$?isError@KrakenClassifyLogParser@U2@@EBE_NABVQString@@@Z 1002cb08     KrakenClassifyLogParser.obj
 0002:00008b10       __ehfuncinfo$?isError@KrakenClassifyLogParser@U2@@EBE_NABVQString@@@Z 1002cb10     KrakenClassifyLogParser.obj
 0002:00008b34       __ehfuncinfo$?initWellKnownErrors@KrakenClassifyLogParser@U2@@CA?AVQStringList@@XZ 1002cb34     KrakenClassifyLogParser.obj
 0002:00008b58       __unwindtable$?initWellKnownErrors@KrakenClassifyLogParser@U2@@CA?AVQStringList@@XZ 1002cb58     KrakenClassifyLogParser.obj
 0002:00008ba0       __unwindtable$??__EalgoLog@U2@@YAXXZ 1002cba0     KrakenClassifyPrompter.obj
 0002:00008ba8       __ehfuncinfo$??__EalgoLog@U2@@YAXXZ 1002cba8     KrakenClassifyPrompter.obj
 0002:00008bcc       __unwindtable$??__EcmdLog@U2@@YAXXZ 1002cbcc     KrakenClassifyPrompter.obj
 0002:00008bd4       __ehfuncinfo$??__EcmdLog@U2@@YAXXZ 1002cbd4     KrakenClassifyPrompter.obj
 0002:00008bf8       __unwindtable$??__EcoreLog@U2@@YAXXZ 1002cbf8     KrakenClassifyPrompter.obj
 0002:00008c00       __ehfuncinfo$??__EcoreLog@U2@@YAXXZ 1002cc00     KrakenClassifyPrompter.obj
 0002:00008c24       __unwindtable$??__EioLog@U2@@YAXXZ 1002cc24     KrakenClassifyPrompter.obj
 0002:00008c2c       __ehfuncinfo$??__EioLog@U2@@YAXXZ 1002cc2c     KrakenClassifyPrompter.obj
 0002:00008c50       __unwindtable$??__EperfLog@U2@@YAXXZ 1002cc50     KrakenClassifyPrompter.obj
 0002:00008c58       __ehfuncinfo$??__EperfLog@U2@@YAXXZ 1002cc58     KrakenClassifyPrompter.obj
 0002:00008c7c       __unwindtable$??__EscriptLog@U2@@YAXXZ 1002cc7c     KrakenClassifyPrompter.obj
 0002:00008c84       __ehfuncinfo$??__EscriptLog@U2@@YAXXZ 1002cc84     KrakenClassifyPrompter.obj
 0002:00008ca8       __unwindtable$??__EtaskLog@U2@@YAXXZ 1002cca8     KrakenClassifyPrompter.obj
 0002:00008cb0       __ehfuncinfo$??__EtaskLog@U2@@YAXXZ 1002ccb0     KrakenClassifyPrompter.obj
 0002:00008cd4       __unwindtable$??__EuiLog@U2@@YAXXZ 1002ccd4     KrakenClassifyPrompter.obj
 0002:00008cdc       __ehfuncinfo$??__EuiLog@U2@@YAXXZ 1002ccdc     KrakenClassifyPrompter.obj
 0002:00008d00       __unwindtable$??__EuserActLog@U2@@YAXXZ 1002cd00     KrakenClassifyPrompter.obj
 0002:00008d08       __ehfuncinfo$??__EuserActLog@U2@@YAXXZ 1002cd08     KrakenClassifyPrompter.obj
 0002:00008d2c       __ehfuncinfo$?createDescription@?$PrompterBase@VKrakenClassifyPrompter@LocalWorkflow@U2@@@U2@@UAEPAVActorDocument@Workflow@2@PAVActor@42@@Z 1002cd2c     KrakenClassifyPrompter.obj
 0002:00008d50       __unwindtable$?createDescription@?$PrompterBase@VKrakenClassifyPrompter@LocalWorkflow@U2@@@U2@@UAEPAVActorDocument@Workflow@2@PAVActor@42@@Z 1002cd50     KrakenClassifyPrompter.obj
 0002:00008d88       __ehfuncinfo$?composeRichDoc@KrakenClassifyPrompter@LocalWorkflow@U2@@EAE?AVQString@@XZ 1002cd88     KrakenClassifyPrompter.obj
 0002:00008dac       __unwindtable$?composeRichDoc@KrakenClassifyPrompter@LocalWorkflow@U2@@EAE?AVQString@@XZ 1002cdac     KrakenClassifyPrompter.obj
 0002:00008e24       __catchsym$?detach_helper@?$QList@VQByteArray@@@@AAEXH@Z$2 1002ce24     KrakenClassifyTask.obj
 0002:00008e34       __unwindtable$?detach_helper@?$QList@VQByteArray@@@@AAEXH@Z 1002ce34     KrakenClassifyTask.obj
 0002:00008e44       __tryblocktable$?detach_helper@?$QList@VQByteArray@@@@AAEXH@Z 1002ce44     KrakenClassifyTask.obj
 0002:00008e58       __ehfuncinfo$?detach_helper@?$QList@VQByteArray@@@@AAEXH@Z 1002ce58     KrakenClassifyTask.obj
 0002:00008e7c       __catchsym$?node_copy@?$QList@VQByteArray@@@@AAEXPAUNode@1@00@Z$6 1002ce7c     KrakenClassifyTask.obj
 0002:00008e8c       __tryblocktable$?node_copy@?$QList@VQByteArray@@@@AAEXPAUNode@1@00@Z 1002ce8c     KrakenClassifyTask.obj
 0002:00008ea0       __ehfuncinfo$?node_copy@?$QList@VQByteArray@@@@AAEXPAUNode@1@00@Z 1002cea0     KrakenClassifyTask.obj
 0002:00008ec4       __unwindtable$?node_copy@?$QList@VQByteArray@@@@AAEXPAUNode@1@00@Z 1002cec4     KrakenClassifyTask.obj
 0002:00008ef4       __unwindtable$??__EalgoLog@U2@@YAXXZ 1002cef4     KrakenClassifyTask.obj
 0002:00008efc       __ehfuncinfo$??__EalgoLog@U2@@YAXXZ 1002cefc     KrakenClassifyTask.obj
 0002:00008f20       __unwindtable$??__EcmdLog@U2@@YAXXZ 1002cf20     KrakenClassifyTask.obj
 0002:00008f28       __ehfuncinfo$??__EcmdLog@U2@@YAXXZ 1002cf28     KrakenClassifyTask.obj
 0002:00008f4c       __unwindtable$??__EcoreLog@U2@@YAXXZ 1002cf4c     KrakenClassifyTask.obj
 0002:00008f54       __ehfuncinfo$??__EcoreLog@U2@@YAXXZ 1002cf54     KrakenClassifyTask.obj
 0002:00008f78       __unwindtable$??__EioLog@U2@@YAXXZ 1002cf78     KrakenClassifyTask.obj
 0002:00008f80       __ehfuncinfo$??__EioLog@U2@@YAXXZ 1002cf80     KrakenClassifyTask.obj
 0002:00008fa4       __unwindtable$??__EperfLog@U2@@YAXXZ 1002cfa4     KrakenClassifyTask.obj
 0002:00008fac       __ehfuncinfo$??__EperfLog@U2@@YAXXZ 1002cfac     KrakenClassifyTask.obj
 0002:00008fd0       __unwindtable$??__EscriptLog@U2@@YAXXZ 1002cfd0     KrakenClassifyTask.obj
 0002:00008fd8       __ehfuncinfo$??__EscriptLog@U2@@YAXXZ 1002cfd8     KrakenClassifyTask.obj
 0002:00008ffc       __unwindtable$??__EtaskLog@U2@@YAXXZ 1002cffc     KrakenClassifyTask.obj
 0002:00009004       __ehfuncinfo$??__EtaskLog@U2@@YAXXZ 1002d004     KrakenClassifyTask.obj
 0002:00009028       __unwindtable$??__EuiLog@U2@@YAXXZ 1002d028     KrakenClassifyTask.obj
 0002:00009030       __ehfuncinfo$??__EuiLog@U2@@YAXXZ 1002d030     KrakenClassifyTask.obj
 0002:00009054       __unwindtable$??__EuserActLog@U2@@YAXXZ 1002d054     KrakenClassifyTask.obj
 0002:0000905c       __ehfuncinfo$??__EuserActLog@U2@@YAXXZ 1002d05c     KrakenClassifyTask.obj
 0002:00009080       __unwindtable$??0KrakenClassifyTaskSettings@U2@@QAE@XZ 1002d080     KrakenClassifyTask.obj
 0002:00009098       __ehfuncinfo$??0KrakenClassifyTaskSettings@U2@@QAE@XZ 1002d098     KrakenClassifyTask.obj
 0002:000090bc       __unwindtable$??1KrakenClassifyTaskSettings@U2@@QAE@XZ 1002d0bc     KrakenClassifyTask.obj
 0002:000090d4       __ehfuncinfo$??1KrakenClassifyTaskSettings@U2@@QAE@XZ 1002d0d4     KrakenClassifyTask.obj
 0002:000090f8       __unwindtable$??0KrakenClassifyTaskSettings@U2@@QAE@ABU01@@Z 1002d0f8     KrakenClassifyTask.obj
 0002:00009110       __ehfuncinfo$??0KrakenClassifyTaskSettings@U2@@QAE@ABU01@@Z 1002d110     KrakenClassifyTask.obj
 0002:00009134       __ehfuncinfo$??0KrakenClassifyTask@U2@@QAE@ABUKrakenClassifyTaskSettings@1@@Z 1002d134     KrakenClassifyTask.obj
 0002:00009158       __unwindtable$??0KrakenClassifyTask@U2@@QAE@ABUKrakenClassifyTaskSettings@1@@Z 1002d158     KrakenClassifyTask.obj
 0002:000091c0       __ehfuncinfo$?prepare@KrakenClassifyTask@U2@@EAEXXZ 1002d1c0     KrakenClassifyTask.obj
 0002:000091e4       __unwindtable$?prepare@KrakenClassifyTask@U2@@EAEXXZ 1002d1e4     KrakenClassifyTask.obj
 0002:00009234       __ehfuncinfo$?run@KrakenClassifyTask@U2@@EAEXXZ 1002d234     KrakenClassifyTask.obj
 0002:00009258       __unwindtable$?run@KrakenClassifyTask@U2@@EAEXXZ 1002d258     KrakenClassifyTask.obj
 0002:000092d8       __ehfuncinfo$?getArguments@KrakenClassifyTask@U2@@AAE?AVQStringList@@XZ 1002d2d8     KrakenClassifyTask.obj
 0002:000092fc       __unwindtable$?getArguments@KrakenClassifyTask@U2@@AAE?AVQStringList@@XZ 1002d2fc     KrakenClassifyTask.obj
 0002:00009354       __ehfuncinfo$??1KrakenClassifyTask@U2@@UAE@XZ 1002d354     KrakenClassifyTask.obj
 0002:00009378       __unwindtable$??1KrakenClassifyTask@U2@@UAE@XZ 1002d378     KrakenClassifyTask.obj
 0002:000093a0       __catchsym$?createNode@?$QMapData@VQString@@I@@QAEPAU?$QMapNode@VQString@@I@@ABVQString@@ABIPAU2@_N@Z$5 1002d3a0     KrakenClassifyTask.obj
 0002:000093b0       __tryblocktable$?createNode@?$QMapData@VQString@@I@@QAEPAU?$QMapNode@VQString@@I@@ABVQString@@ABIPAU2@_N@Z 1002d3b0     KrakenClassifyTask.obj
 0002:000093c4       __ehfuncinfo$?createNode@?$QMapData@VQString@@I@@QAEPAU?$QMapNode@VQString@@I@@ABVQString@@ABIPAU2@_N@Z 1002d3c4     KrakenClassifyTask.obj
 0002:000093e8       __unwindtable$?createNode@?$QMapData@VQString@@I@@QAEPAU?$QMapNode@VQString@@I@@ABVQString@@ABIPAU2@_N@Z 1002d3e8     KrakenClassifyTask.obj
 0002:00009410       __unwindtable$??__EalgoLog@U2@@YAXXZ 1002d410     KrakenClassifyValidator.obj
 0002:00009418       __ehfuncinfo$??__EalgoLog@U2@@YAXXZ 1002d418     KrakenClassifyValidator.obj
 0002:0000943c       __unwindtable$??__EcmdLog@U2@@YAXXZ 1002d43c     KrakenClassifyValidator.obj
 0002:00009444       __ehfuncinfo$??__EcmdLog@U2@@YAXXZ 1002d444     KrakenClassifyValidator.obj
 0002:00009468       __unwindtable$??__EcoreLog@U2@@YAXXZ 1002d468     KrakenClassifyValidator.obj
 0002:00009470       __ehfuncinfo$??__EcoreLog@U2@@YAXXZ 1002d470     KrakenClassifyValidator.obj
 0002:00009494       __unwindtable$??__EioLog@U2@@YAXXZ 1002d494     KrakenClassifyValidator.obj
 0002:0000949c       __ehfuncinfo$??__EioLog@U2@@YAXXZ 1002d49c     KrakenClassifyValidator.obj
 0002:000094c0       __unwindtable$??__EperfLog@U2@@YAXXZ 1002d4c0     KrakenClassifyValidator.obj
 0002:000094c8       __ehfuncinfo$??__EperfLog@U2@@YAXXZ 1002d4c8     KrakenClassifyValidator.obj
 0002:000094ec       __unwindtable$??__EscriptLog@U2@@YAXXZ 1002d4ec     KrakenClassifyValidator.obj
 0002:000094f4       __ehfuncinfo$??__EscriptLog@U2@@YAXXZ 1002d4f4     KrakenClassifyValidator.obj
 0002:00009518       __unwindtable$??__EtaskLog@U2@@YAXXZ 1002d518     KrakenClassifyValidator.obj
 0002:00009520       __ehfuncinfo$??__EtaskLog@U2@@YAXXZ 1002d520     KrakenClassifyValidator.obj
 0002:00009544       __unwindtable$??__EuiLog@U2@@YAXXZ 1002d544     KrakenClassifyValidator.obj
 0002:0000954c       __ehfuncinfo$??__EuiLog@U2@@YAXXZ 1002d54c     KrakenClassifyValidator.obj
 0002:00009570       __unwindtable$??__EuserActLog@U2@@YAXXZ 1002d570     KrakenClassifyValidator.obj
 0002:00009578       __ehfuncinfo$??__EuserActLog@U2@@YAXXZ 1002d578     KrakenClassifyValidator.obj
 0002:0000959c       __ehfuncinfo$?validateDatabase@KrakenClassifyValidator@Workflow@U2@@ABE_NPBVActor@23@AAV?$QList@VWorkflowNotification@U2@@@@@Z 1002d59c     KrakenClassifyValidator.obj
 0002:000095c0       __unwindtable$?validateDatabase@KrakenClassifyValidator@Workflow@U2@@ABE_NPBVActor@23@AAV?$QList@VWorkflowNotification@U2@@@@@Z 1002d5c0     KrakenClassifyValidator.obj
 0002:000096a8       __unwindtable$?qt_metatype_id@?$QMetaTypeId@VQAssociativeIterableImpl@QtMetaTypePrivate@@@@SAHXZ 1002d6a8     KrakenClassifyWorker.obj
 0002:000096b0       __ehfuncinfo$?qt_metatype_id@?$QMetaTypeId@VQAssociativeIterableImpl@QtMetaTypePrivate@@@@SAHXZ 1002d6b0     KrakenClassifyWorker.obj
 0002:000096d4       __unwindtable$??$qRegisterMetaType@VQAssociativeIterableImpl@QtMetaTypePrivate@@@@YAHPBDPAVQAssociativeIterableImpl@QtMetaTypePrivate@@W4DefinedType@?$MetaTypeDefinedHelper@VQAssociativeIterableImpl@QtMetaTypePrivate@@$00@QtPrivate@@@Z 1002d6d4     KrakenClassifyWorker.obj
 0002:000096dc       __ehfuncinfo$??$qRegisterMetaType@VQAssociativeIterableImpl@QtMetaTypePrivate@@@@YAHPBDPAVQAssociativeIterableImpl@QtMetaTypePrivate@@W4DefinedType@?$MetaTypeDefinedHelper@VQAssociativeIterableImpl@QtMetaTypePrivate@@$00@QtPrivate@@@Z 1002d6dc     KrakenClassifyWorker.obj
 0002:00009700       __unwindtable$??__EalgoLog@U2@@YAXXZ 1002d700     KrakenClassifyWorker.obj
 0002:00009708       __ehfuncinfo$??__EalgoLog@U2@@YAXXZ 1002d708     KrakenClassifyWorker.obj
 0002:0000972c       __unwindtable$??__EcmdLog@U2@@YAXXZ 1002d72c     KrakenClassifyWorker.obj
 0002:00009734       __ehfuncinfo$??__EcmdLog@U2@@YAXXZ 1002d734     KrakenClassifyWorker.obj
 0002:00009758       __unwindtable$??__EcoreLog@U2@@YAXXZ 1002d758     KrakenClassifyWorker.obj
 0002:00009760       __ehfuncinfo$??__EcoreLog@U2@@YAXXZ 1002d760     KrakenClassifyWorker.obj
 0002:00009784       __unwindtable$??__EioLog@U2@@YAXXZ 1002d784     KrakenClassifyWorker.obj
 0002:0000978c       __ehfuncinfo$??__EioLog@U2@@YAXXZ 1002d78c     KrakenClassifyWorker.obj
 0002:000097b0       __unwindtable$??__EperfLog@U2@@YAXXZ 1002d7b0     KrakenClassifyWorker.obj
 0002:000097b8       __ehfuncinfo$??__EperfLog@U2@@YAXXZ 1002d7b8     KrakenClassifyWorker.obj
 0002:000097dc       __unwindtable$??__EscriptLog@U2@@YAXXZ 1002d7dc     KrakenClassifyWorker.obj
 0002:000097e4       __ehfuncinfo$??__EscriptLog@U2@@YAXXZ 1002d7e4     KrakenClassifyWorker.obj
 0002:00009808       __unwindtable$??__EtaskLog@U2@@YAXXZ 1002d808     KrakenClassifyWorker.obj
 0002:00009810       __ehfuncinfo$??__EtaskLog@U2@@YAXXZ 1002d810     KrakenClassifyWorker.obj
 0002:00009834       __unwindtable$??__EuiLog@U2@@YAXXZ 1002d834     KrakenClassifyWorker.obj
 0002:0000983c       __ehfuncinfo$??__EuiLog@U2@@YAXXZ 1002d83c     KrakenClassifyWorker.obj
 0002:00009860       __unwindtable$??__EuserActLog@U2@@YAXXZ 1002d860     KrakenClassifyWorker.obj
 0002:00009868       __ehfuncinfo$??__EuserActLog@U2@@YAXXZ 1002d868     KrakenClassifyWorker.obj
 0002:0000988c       __unwindtable$?qt_metatype_id@?$QMetaTypeId@V?$QMap@VQString@@I@@@@SAHXZ 1002d88c     KrakenClassifyWorker.obj
 0002:00009894       __ehfuncinfo$?qt_metatype_id@?$QMetaTypeId@V?$QMap@VQString@@I@@@@SAHXZ 1002d894     KrakenClassifyWorker.obj
 0002:000098b8       __unwindtable$??$qRegisterMetaType@V?$QMap@VQString@@I@@@@YAHPBDPAV?$QMap@VQString@@I@@W4DefinedType@?$MetaTypeDefinedHelper@V?$QMap@VQString@@I@@$00@QtPrivate@@@Z 1002d8b8     KrakenClassifyWorker.obj
 0002:000098c0       __ehfuncinfo$??$qRegisterMetaType@V?$QMap@VQString@@I@@@@YAHPBDPAV?$QMap@VQString@@I@@W4DefinedType@?$MetaTypeDefinedHelper@V?$QMap@VQString@@I@@$00@QtPrivate@@@Z 1002d8c0     KrakenClassifyWorker.obj
 0002:000098e4       __ehfuncinfo$?init@KrakenClassifyWorker@LocalWorkflow@U2@@UAEXXZ 1002d8e4     KrakenClassifyWorker.obj
 0002:00009908       __unwindtable$?init@KrakenClassifyWorker@LocalWorkflow@U2@@UAEXXZ 1002d908     KrakenClassifyWorker.obj
 0002:00009980       __ehfuncinfo$?tick@KrakenClassifyWorker@LocalWorkflow@U2@@UAEPAVTask@3@XZ 1002d980     KrakenClassifyWorker.obj
 0002:000099a4       __unwindtable$?tick@KrakenClassifyWorker@LocalWorkflow@U2@@UAEPAVTask@3@XZ 1002d9a4     KrakenClassifyWorker.obj
 0002:000099fc       __ehfuncinfo$?sl_taskFinished@KrakenClassifyWorker@LocalWorkflow@U2@@AAEXPAVTask@3@@Z 1002d9fc     KrakenClassifyWorker.obj
 0002:00009a20       __unwindtable$?sl_taskFinished@KrakenClassifyWorker@LocalWorkflow@U2@@AAEXPAVTask@3@@Z 1002da20     KrakenClassifyWorker.obj
 0002:00009a80       __ehfuncinfo$?getSettings@KrakenClassifyWorker@LocalWorkflow@U2@@AAE?AUKrakenClassifyTaskSettings@3@AAVU2OpStatus@3@@Z 1002da80     KrakenClassifyWorker.obj
 0002:00009aa4       __unwindtable$?getSettings@KrakenClassifyWorker@LocalWorkflow@U2@@AAE?AUKrakenClassifyTaskSettings@3@AAVU2OpStatus@3@@Z 1002daa4     KrakenClassifyWorker.obj
 0002:00009bac       __unwindtable$?Create@?$QMetaTypeFunctionHelper@V?$QMap@VQString@@I@@$00@QtMetaTypePrivate@@SAPAXPBX@Z 1002dbac     KrakenClassifyWorker.obj
 0002:00009bb4       __ehfuncinfo$?Create@?$QMetaTypeFunctionHelper@V?$QMap@VQString@@I@@$00@QtMetaTypePrivate@@SAPAXPBX@Z 1002dbb4     KrakenClassifyWorker.obj
 0002:00009bd8       __unwindtable$?Construct@?$QMetaTypeFunctionHelper@V?$QMap@VQString@@I@@$00@QtMetaTypePrivate@@SAPAXPAXPBX@Z 1002dbd8     KrakenClassifyWorker.obj
 0002:00009be0       __ehfuncinfo$?Construct@?$QMetaTypeFunctionHelper@V?$QMap@VQString@@I@@$00@QtMetaTypePrivate@@SAPAXPAXPBX@Z 1002dbe0     KrakenClassifyWorker.obj
 0002:00009c04       __catchsym$?append@?$QList@VQVariant@@@@QAEXABVQVariant@@@Z$11 1002dc04     KrakenClassifyWorkerFactory.obj
 0002:00009c14       __catchsym$?append@?$QList@VQVariant@@@@QAEXABVQVariant@@@Z$10 1002dc14     KrakenClassifyWorkerFactory.obj
 0002:00009c24       __ehfuncinfo$?append@?$QList@VQVariant@@@@QAEXABVQVariant@@@Z 1002dc24     KrakenClassifyWorkerFactory.obj
 0002:00009c48       __tryblocktable$?append@?$QList@VQVariant@@@@QAEXABVQVariant@@@Z 1002dc48     KrakenClassifyWorkerFactory.obj
 0002:00009c70       __unwindtable$?append@?$QList@VQVariant@@@@QAEXABVQVariant@@@Z 1002dc70     KrakenClassifyWorkerFactory.obj
 0002:00009cc0       __catchsym$?detach_helper_grow@?$QList@VQVariant@@@@AAEPAUNode@1@HH@Z$5 1002dcc0     KrakenClassifyWorkerFactory.obj
 0002:00009cd0       __catchsym$?detach_helper_grow@?$QList@VQVariant@@@@AAEPAUNode@1@HH@Z$4 1002dcd0     KrakenClassifyWorkerFactory.obj
 0002:00009ce0       __unwindtable$?detach_helper_grow@?$QList@VQVariant@@@@AAEPAUNode@1@HH@Z 1002dce0     KrakenClassifyWorkerFactory.obj
 0002:00009d00       __ehfuncinfo$?detach_helper_grow@?$QList@VQVariant@@@@AAEPAUNode@1@HH@Z 1002dd00     KrakenClassifyWorkerFactory.obj
 0002:00009d24       __tryblocktable$?detach_helper_grow@?$QList@VQVariant@@@@AAEPAUNode@1@HH@Z 1002dd24     KrakenClassifyWorkerFactory.obj
 0002:00009d4c       __unwindtable$?node_construct@?$QList@VQVariant@@@@AAEXPAUNode@1@ABVQVariant@@@Z 1002dd4c     KrakenClassifyWorkerFactory.obj
 0002:00009d5c       __ehfuncinfo$?node_construct@?$QList@VQVariant@@@@AAEXPAUNode@1@ABVQVariant@@@Z 1002dd5c     KrakenClassifyWorkerFactory.obj
 0002:00009d80       __catchsym$?node_copy@?$QList@VQVariant@@@@AAEXPAUNode@1@00@Z$6 1002dd80     KrakenClassifyWorkerFactory.obj
 0002:00009d90       __tryblocktable$?node_copy@?$QList@VQVariant@@@@AAEXPAUNode@1@00@Z 1002dd90     KrakenClassifyWorkerFactory.obj
 0002:00009da4       __ehfuncinfo$?node_copy@?$QList@VQVariant@@@@AAEXPAUNode@1@00@Z 1002dda4     KrakenClassifyWorkerFactory.obj
 0002:00009dc8       __unwindtable$?node_copy@?$QList@VQVariant@@@@AAEXPAUNode@1@00@Z 1002ddc8     KrakenClassifyWorkerFactory.obj
 0002:00009df8       __unwindtable$??__EalgoLog@U2@@YAXXZ 1002ddf8     KrakenClassifyWorkerFactory.obj
 0002:00009e00       __ehfuncinfo$??__EalgoLog@U2@@YAXXZ 1002de00     KrakenClassifyWorkerFactory.obj
 0002:00009e24       __unwindtable$??__EcmdLog@U2@@YAXXZ 1002de24     KrakenClassifyWorkerFactory.obj
 0002:00009e2c       __ehfuncinfo$??__EcmdLog@U2@@YAXXZ 1002de2c     KrakenClassifyWorkerFactory.obj
 0002:00009e50       __unwindtable$??__EcoreLog@U2@@YAXXZ 1002de50     KrakenClassifyWorkerFactory.obj
 0002:00009e58       __ehfuncinfo$??__EcoreLog@U2@@YAXXZ 1002de58     KrakenClassifyWorkerFactory.obj
 0002:00009e7c       __unwindtable$??__EioLog@U2@@YAXXZ 1002de7c     KrakenClassifyWorkerFactory.obj
 0002:00009e84       __ehfuncinfo$??__EioLog@U2@@YAXXZ 1002de84     KrakenClassifyWorkerFactory.obj
 0002:00009ea8       __unwindtable$??__EperfLog@U2@@YAXXZ 1002dea8     KrakenClassifyWorkerFactory.obj
 0002:00009eb0       __ehfuncinfo$??__EperfLog@U2@@YAXXZ 1002deb0     KrakenClassifyWorkerFactory.obj
 0002:00009ed4       __unwindtable$??__EscriptLog@U2@@YAXXZ 1002ded4     KrakenClassifyWorkerFactory.obj
 0002:00009edc       __ehfuncinfo$??__EscriptLog@U2@@YAXXZ 1002dedc     KrakenClassifyWorkerFactory.obj
 0002:00009f00       __unwindtable$??__EtaskLog@U2@@YAXXZ 1002df00     KrakenClassifyWorkerFactory.obj
 0002:00009f08       __ehfuncinfo$??__EtaskLog@U2@@YAXXZ 1002df08     KrakenClassifyWorkerFactory.obj
 0002:00009f2c       __unwindtable$??__EuiLog@U2@@YAXXZ 1002df2c     KrakenClassifyWorkerFactory.obj
 0002:00009f34       __ehfuncinfo$??__EuiLog@U2@@YAXXZ 1002df34     KrakenClassifyWorkerFactory.obj
 0002:00009f58       __unwindtable$??__EuserActLog@U2@@YAXXZ 1002df58     KrakenClassifyWorkerFactory.obj
 0002:00009f60       __ehfuncinfo$??__EuserActLog@U2@@YAXXZ 1002df60     KrakenClassifyWorkerFactory.obj
 0002:00009f84       __unwindtable$?createWorker@KrakenClassifyWorkerFactory@LocalWorkflow@U2@@UAEPAVWorker@Workflow@3@PAVActor@53@@Z 1002df84     KrakenClassifyWorkerFactory.obj
 0002:00009f8c       __ehfuncinfo$?createWorker@KrakenClassifyWorkerFactory@LocalWorkflow@U2@@UAEPAVWorker@Workflow@3@PAVActor@53@@Z 1002df8c     KrakenClassifyWorkerFactory.obj
 0002:00009fb0       __ehfuncinfo$?init@KrakenClassifyWorkerFactory@LocalWorkflow@U2@@SAXXZ 1002dfb0     KrakenClassifyWorkerFactory.obj
 0002:00009fd4       __unwindtable$?init@KrakenClassifyWorkerFactory@LocalWorkflow@U2@@SAXXZ 1002dfd4     KrakenClassifyWorkerFactory.obj
 0002:0000a4a4       __ehfuncinfo$??0KrakenSupport@U2@@QAE@ABVQString@@0@Z 1002e4a4     KrakenSupport.obj
 0002:0000a4c8       __unwindtable$??0KrakenSupport@U2@@QAE@ABVQString@@0@Z 1002e4c8     KrakenSupport.obj
 0002:0000a510       __ehfuncinfo$?getAdditionalPaths@KrakenSupport@U2@@UBE?AVQStringList@@XZ 1002e510     KrakenSupport.obj
 0002:0000a534       __unwindtable$?getAdditionalPaths@KrakenSupport@U2@@UBE?AVQStringList@@XZ 1002e534     KrakenSupport.obj
 0002:0000a57c       __unwindtable$?initBuild@KrakenSupport@U2@@AAEXXZ 1002e57c     KrakenSupport.obj
 0002:0000a584       __ehfuncinfo$?initBuild@KrakenSupport@U2@@AAEXXZ 1002e584     KrakenSupport.obj
 0002:0000a5a8       __unwindtable$?initClassify@KrakenSupport@U2@@AAEXXZ 1002e5a8     KrakenSupport.obj
 0002:0000a5b0       __ehfuncinfo$?initClassify@KrakenSupport@U2@@AAEXXZ 1002e5b0     KrakenSupport.obj
 0002:0000a5d4       __unwindtable$??__EalgoLog@U2@@YAXXZ 1002e5d4     KrakenSupportPlugin.obj
 0002:0000a5dc       __ehfuncinfo$??__EalgoLog@U2@@YAXXZ 1002e5dc     KrakenSupportPlugin.obj
 0002:0000a600       __unwindtable$??__EcmdLog@U2@@YAXXZ 1002e600     KrakenSupportPlugin.obj
 0002:0000a608       __ehfuncinfo$??__EcmdLog@U2@@YAXXZ 1002e608     KrakenSupportPlugin.obj
 0002:0000a62c       __unwindtable$??__EcoreLog@U2@@YAXXZ 1002e62c     KrakenSupportPlugin.obj
 0002:0000a634       __ehfuncinfo$??__EcoreLog@U2@@YAXXZ 1002e634     KrakenSupportPlugin.obj
 0002:0000a658       __unwindtable$??__EioLog@U2@@YAXXZ 1002e658     KrakenSupportPlugin.obj
 0002:0000a660       __ehfuncinfo$??__EioLog@U2@@YAXXZ 1002e660     KrakenSupportPlugin.obj
 0002:0000a684       __unwindtable$??__EperfLog@U2@@YAXXZ 1002e684     KrakenSupportPlugin.obj
 0002:0000a68c       __ehfuncinfo$??__EperfLog@U2@@YAXXZ 1002e68c     KrakenSupportPlugin.obj
 0002:0000a6b0       __unwindtable$??__EscriptLog@U2@@YAXXZ 1002e6b0     KrakenSupportPlugin.obj
 0002:0000a6b8       __ehfuncinfo$??__EscriptLog@U2@@YAXXZ 1002e6b8     KrakenSupportPlugin.obj
 0002:0000a6dc       __unwindtable$??__EtaskLog@U2@@YAXXZ 1002e6dc     KrakenSupportPlugin.obj
 0002:0000a6e4       __ehfuncinfo$??__EtaskLog@U2@@YAXXZ 1002e6e4     KrakenSupportPlugin.obj
 0002:0000a708       __unwindtable$??__EuiLog@U2@@YAXXZ 1002e708     KrakenSupportPlugin.obj
 0002:0000a710       __ehfuncinfo$??__EuiLog@U2@@YAXXZ 1002e710     KrakenSupportPlugin.obj
 0002:0000a734       __unwindtable$??__EuserActLog@U2@@YAXXZ 1002e734     KrakenSupportPlugin.obj
 0002:0000a73c       __ehfuncinfo$??__EuserActLog@U2@@YAXXZ 1002e73c     KrakenSupportPlugin.obj
 0002:0000a760       __unwindtable$??0KrakenSupportPlugin@U2@@QAE@XZ 1002e760     KrakenSupportPlugin.obj
 0002:0000a780       __ehfuncinfo$??0KrakenSupportPlugin@U2@@QAE@XZ 1002e780     KrakenSupportPlugin.obj
 0002:0000a7a4       __unwindtable$??1KrakenSupportPlugin@U2@@UAE@XZ 1002e7a4     KrakenSupportPlugin.obj
 0002:0000a7ac       __ehfuncinfo$??1KrakenSupportPlugin@U2@@UAE@XZ 1002e7ac     KrakenSupportPlugin.obj
 0002:0000a7d0       __unwindtable$??_GKrakenSupportPlugin@U2@@UAEPAXI@Z 1002e7d0     KrakenSupportPlugin.obj
 0002:0000a7d8       __ehfuncinfo$??_GKrakenSupportPlugin@U2@@UAEPAXI@Z 1002e7d8     KrakenSupportPlugin.obj
 0002:0000a7fc       __unwindtable$??__EalgoLog@U2@@YAXXZ 1002e7fc     KrakenTranslateLogParser.obj
 0002:0000a804       __ehfuncinfo$??__EalgoLog@U2@@YAXXZ 1002e804     KrakenTranslateLogParser.obj
 0002:0000a828       __unwindtable$??__EcmdLog@U2@@YAXXZ 1002e828     KrakenTranslateLogParser.obj
 0002:0000a830       __ehfuncinfo$??__EcmdLog@U2@@YAXXZ 1002e830     KrakenTranslateLogParser.obj
 0002:0000a854       __unwindtable$??__EcoreLog@U2@@YAXXZ 1002e854     KrakenTranslateLogParser.obj
 0002:0000a85c       __ehfuncinfo$??__EcoreLog@U2@@YAXXZ 1002e85c     KrakenTranslateLogParser.obj
 0002:0000a880       __unwindtable$??__EioLog@U2@@YAXXZ 1002e880     KrakenTranslateLogParser.obj
 0002:0000a888       __ehfuncinfo$??__EioLog@U2@@YAXXZ 1002e888     KrakenTranslateLogParser.obj
 0002:0000a8ac       __unwindtable$??__EperfLog@U2@@YAXXZ 1002e8ac     KrakenTranslateLogParser.obj
 0002:0000a8b4       __ehfuncinfo$??__EperfLog@U2@@YAXXZ 1002e8b4     KrakenTranslateLogParser.obj
 0002:0000a8d8       __unwindtable$??__EscriptLog@U2@@YAXXZ 1002e8d8     KrakenTranslateLogParser.obj
 0002:0000a8e0       __ehfuncinfo$??__EscriptLog@U2@@YAXXZ 1002e8e0     KrakenTranslateLogParser.obj
 0002:0000a904       __unwindtable$??__EtaskLog@U2@@YAXXZ 1002e904     KrakenTranslateLogParser.obj
 0002:0000a90c       __ehfuncinfo$??__EtaskLog@U2@@YAXXZ 1002e90c     KrakenTranslateLogParser.obj
 0002:0000a930       __unwindtable$??__EuiLog@U2@@YAXXZ 1002e930     KrakenTranslateLogParser.obj
 0002:0000a938       __ehfuncinfo$??__EuiLog@U2@@YAXXZ 1002e938     KrakenTranslateLogParser.obj
 0002:0000a95c       __unwindtable$??__EuserActLog@U2@@YAXXZ 1002e95c     KrakenTranslateLogParser.obj
 0002:0000a964       __ehfuncinfo$??__EuserActLog@U2@@YAXXZ 1002e964     KrakenTranslateLogParser.obj
 0002:0000a988       __unwindtable$?isError@KrakenTranslateLogParser@U2@@EBE_NABVQString@@@Z 1002e988     KrakenTranslateLogParser.obj
 0002:0000a990       __ehfuncinfo$?isError@KrakenTranslateLogParser@U2@@EBE_NABVQString@@@Z 1002e990     KrakenTranslateLogParser.obj
 0002:0000a9b4       __ehfuncinfo$?initWellKnownErrors@KrakenTranslateLogParser@U2@@CA?AVQStringList@@XZ 1002e9b4     KrakenTranslateLogParser.obj
 0002:0000a9d8       __unwindtable$?initWellKnownErrors@KrakenTranslateLogParser@U2@@CA?AVQStringList@@XZ 1002e9d8     KrakenTranslateLogParser.obj
 0002:0000aa08       __unwindtable$??__EalgoLog@U2@@YAXXZ 1002ea08     moc_KrakenBuildPrompter.obj
 0002:0000aa10       __ehfuncinfo$??__EalgoLog@U2@@YAXXZ 1002ea10     moc_KrakenBuildPrompter.obj
 0002:0000aa34       __unwindtable$??__EcmdLog@U2@@YAXXZ 1002ea34     moc_KrakenBuildPrompter.obj
 0002:0000aa3c       __ehfuncinfo$??__EcmdLog@U2@@YAXXZ 1002ea3c     moc_KrakenBuildPrompter.obj
 0002:0000aa60       __unwindtable$??__EcoreLog@U2@@YAXXZ 1002ea60     moc_KrakenBuildPrompter.obj
 0002:0000aa68       __ehfuncinfo$??__EcoreLog@U2@@YAXXZ 1002ea68     moc_KrakenBuildPrompter.obj
 0002:0000aa8c       __unwindtable$??__EioLog@U2@@YAXXZ 1002ea8c     moc_KrakenBuildPrompter.obj
 0002:0000aa94       __ehfuncinfo$??__EioLog@U2@@YAXXZ 1002ea94     moc_KrakenBuildPrompter.obj
 0002:0000aab8       __unwindtable$??__EperfLog@U2@@YAXXZ 1002eab8     moc_KrakenBuildPrompter.obj
 0002:0000aac0       __ehfuncinfo$??__EperfLog@U2@@YAXXZ 1002eac0     moc_KrakenBuildPrompter.obj
 0002:0000aae4       __unwindtable$??__EscriptLog@U2@@YAXXZ 1002eae4     moc_KrakenBuildPrompter.obj
 0002:0000aaec       __ehfuncinfo$??__EscriptLog@U2@@YAXXZ 1002eaec     moc_KrakenBuildPrompter.obj
 0002:0000ab10       __unwindtable$??__EtaskLog@U2@@YAXXZ 1002eb10     moc_KrakenBuildPrompter.obj
 0002:0000ab18       __ehfuncinfo$??__EtaskLog@U2@@YAXXZ 1002eb18     moc_KrakenBuildPrompter.obj
 0002:0000ab3c       __unwindtable$??__EuiLog@U2@@YAXXZ 1002eb3c     moc_KrakenBuildPrompter.obj
 0002:0000ab44       __ehfuncinfo$??__EuiLog@U2@@YAXXZ 1002eb44     moc_KrakenBuildPrompter.obj
 0002:0000ab68       __unwindtable$??__EuserActLog@U2@@YAXXZ 1002eb68     moc_KrakenBuildPrompter.obj
 0002:0000ab70       __ehfuncinfo$??__EuserActLog@U2@@YAXXZ 1002eb70     moc_KrakenBuildPrompter.obj
 0002:0000ab94       __unwindtable$??__EalgoLog@U2@@YAXXZ 1002eb94     moc_KrakenBuildTask.obj
 0002:0000ab9c       __ehfuncinfo$??__EalgoLog@U2@@YAXXZ 1002eb9c     moc_KrakenBuildTask.obj
 0002:0000abc0       __unwindtable$??__EcmdLog@U2@@YAXXZ 1002ebc0     moc_KrakenBuildTask.obj
 0002:0000abc8       __ehfuncinfo$??__EcmdLog@U2@@YAXXZ 1002ebc8     moc_KrakenBuildTask.obj
 0002:0000abec       __unwindtable$??__EcoreLog@U2@@YAXXZ 1002ebec     moc_KrakenBuildTask.obj
 0002:0000abf4       __ehfuncinfo$??__EcoreLog@U2@@YAXXZ 1002ebf4     moc_KrakenBuildTask.obj
 0002:0000ac18       __unwindtable$??__EioLog@U2@@YAXXZ 1002ec18     moc_KrakenBuildTask.obj
 0002:0000ac20       __ehfuncinfo$??__EioLog@U2@@YAXXZ 1002ec20     moc_KrakenBuildTask.obj
 0002:0000ac44       __unwindtable$??__EperfLog@U2@@YAXXZ 1002ec44     moc_KrakenBuildTask.obj
 0002:0000ac4c       __ehfuncinfo$??__EperfLog@U2@@YAXXZ 1002ec4c     moc_KrakenBuildTask.obj
 0002:0000ac70       __unwindtable$??__EscriptLog@U2@@YAXXZ 1002ec70     moc_KrakenBuildTask.obj
 0002:0000ac78       __ehfuncinfo$??__EscriptLog@U2@@YAXXZ 1002ec78     moc_KrakenBuildTask.obj
 0002:0000ac9c       __unwindtable$??__EtaskLog@U2@@YAXXZ 1002ec9c     moc_KrakenBuildTask.obj
 0002:0000aca4       __ehfuncinfo$??__EtaskLog@U2@@YAXXZ 1002eca4     moc_KrakenBuildTask.obj
 0002:0000acc8       __unwindtable$??__EuiLog@U2@@YAXXZ 1002ecc8     moc_KrakenBuildTask.obj
 0002:0000acd0       __ehfuncinfo$??__EuiLog@U2@@YAXXZ 1002ecd0     moc_KrakenBuildTask.obj
 0002:0000acf4       __unwindtable$??__EuserActLog@U2@@YAXXZ 1002ecf4     moc_KrakenBuildTask.obj
 0002:0000acfc       __ehfuncinfo$??__EuserActLog@U2@@YAXXZ 1002ecfc     moc_KrakenBuildTask.obj
 0002:0000ad20       __unwindtable$??__EalgoLog@U2@@YAXXZ 1002ed20     moc_KrakenBuildWorker.obj
 0002:0000ad28       __ehfuncinfo$??__EalgoLog@U2@@YAXXZ 1002ed28     moc_KrakenBuildWorker.obj
 0002:0000ad4c       __unwindtable$??__EcmdLog@U2@@YAXXZ 1002ed4c     moc_KrakenBuildWorker.obj
 0002:0000ad54       __ehfuncinfo$??__EcmdLog@U2@@YAXXZ 1002ed54     moc_KrakenBuildWorker.obj
 0002:0000ad78       __unwindtable$??__EcoreLog@U2@@YAXXZ 1002ed78     moc_KrakenBuildWorker.obj
 0002:0000ad80       __ehfuncinfo$??__EcoreLog@U2@@YAXXZ 1002ed80     moc_KrakenBuildWorker.obj
 0002:0000ada4       __unwindtable$??__EioLog@U2@@YAXXZ 1002eda4     moc_KrakenBuildWorker.obj
 0002:0000adac       __ehfuncinfo$??__EioLog@U2@@YAXXZ 1002edac     moc_KrakenBuildWorker.obj
 0002:0000add0       __unwindtable$??__EperfLog@U2@@YAXXZ 1002edd0     moc_KrakenBuildWorker.obj
 0002:0000add8       __ehfuncinfo$??__EperfLog@U2@@YAXXZ 1002edd8     moc_KrakenBuildWorker.obj
 0002:0000adfc       __unwindtable$??__EscriptLog@U2@@YAXXZ 1002edfc     moc_KrakenBuildWorker.obj
 0002:0000ae04       __ehfuncinfo$??__EscriptLog@U2@@YAXXZ 1002ee04     moc_KrakenBuildWorker.obj
 0002:0000ae28       __unwindtable$??__EtaskLog@U2@@YAXXZ 1002ee28     moc_KrakenBuildWorker.obj
 0002:0000ae30       __ehfuncinfo$??__EtaskLog@U2@@YAXXZ 1002ee30     moc_KrakenBuildWorker.obj
 0002:0000ae54       __unwindtable$??__EuiLog@U2@@YAXXZ 1002ee54     moc_KrakenBuildWorker.obj
 0002:0000ae5c       __ehfuncinfo$??__EuiLog@U2@@YAXXZ 1002ee5c     moc_KrakenBuildWorker.obj
 0002:0000ae80       __unwindtable$??__EuserActLog@U2@@YAXXZ 1002ee80     moc_KrakenBuildWorker.obj
 0002:0000ae88       __ehfuncinfo$??__EuserActLog@U2@@YAXXZ 1002ee88     moc_KrakenBuildWorker.obj
 0002:0000aeac       __unwindtable$?qt_metatype_id@?$QMetaTypeIdQObject@PAVTask@U2@@$00@@SAHXZ 1002eeac     moc_KrakenBuildWorker.obj
 0002:0000aeb4       __ehfuncinfo$?qt_metatype_id@?$QMetaTypeIdQObject@PAVTask@U2@@$00@@SAHXZ 1002eeb4     moc_KrakenBuildWorker.obj
 0002:0000aed8       __unwindtable$??__EalgoLog@U2@@YAXXZ 1002eed8     moc_KrakenClassifyPrompter.obj
 0002:0000aee0       __ehfuncinfo$??__EalgoLog@U2@@YAXXZ 1002eee0     moc_KrakenClassifyPrompter.obj
 0002:0000af04       __unwindtable$??__EcmdLog@U2@@YAXXZ 1002ef04     moc_KrakenClassifyPrompter.obj
 0002:0000af0c       __ehfuncinfo$??__EcmdLog@U2@@YAXXZ 1002ef0c     moc_KrakenClassifyPrompter.obj
 0002:0000af30       __unwindtable$??__EcoreLog@U2@@YAXXZ 1002ef30     moc_KrakenClassifyPrompter.obj
 0002:0000af38       __ehfuncinfo$??__EcoreLog@U2@@YAXXZ 1002ef38     moc_KrakenClassifyPrompter.obj
 0002:0000af5c       __unwindtable$??__EioLog@U2@@YAXXZ 1002ef5c     moc_KrakenClassifyPrompter.obj
 0002:0000af64       __ehfuncinfo$??__EioLog@U2@@YAXXZ 1002ef64     moc_KrakenClassifyPrompter.obj
 0002:0000af88       __unwindtable$??__EperfLog@U2@@YAXXZ 1002ef88     moc_KrakenClassifyPrompter.obj
 0002:0000af90       __ehfuncinfo$??__EperfLog@U2@@YAXXZ 1002ef90     moc_KrakenClassifyPrompter.obj
 0002:0000afb4       __unwindtable$??__EscriptLog@U2@@YAXXZ 1002efb4     moc_KrakenClassifyPrompter.obj
 0002:0000afbc       __ehfuncinfo$??__EscriptLog@U2@@YAXXZ 1002efbc     moc_KrakenClassifyPrompter.obj
 0002:0000afe0       __unwindtable$??__EtaskLog@U2@@YAXXZ 1002efe0     moc_KrakenClassifyPrompter.obj
 0002:0000afe8       __ehfuncinfo$??__EtaskLog@U2@@YAXXZ 1002efe8     moc_KrakenClassifyPrompter.obj
 0002:0000b00c       __unwindtable$??__EuiLog@U2@@YAXXZ 1002f00c     moc_KrakenClassifyPrompter.obj
 0002:0000b014       __ehfuncinfo$??__EuiLog@U2@@YAXXZ 1002f014     moc_KrakenClassifyPrompter.obj
 0002:0000b038       __unwindtable$??__EuserActLog@U2@@YAXXZ 1002f038     moc_KrakenClassifyPrompter.obj
 0002:0000b040       __ehfuncinfo$??__EuserActLog@U2@@YAXXZ 1002f040     moc_KrakenClassifyPrompter.obj
 0002:0000b064       __unwindtable$??__EalgoLog@U2@@YAXXZ 1002f064     moc_KrakenClassifyTask.obj
 0002:0000b06c       __ehfuncinfo$??__EalgoLog@U2@@YAXXZ 1002f06c     moc_KrakenClassifyTask.obj
 0002:0000b090       __unwindtable$??__EcmdLog@U2@@YAXXZ 1002f090     moc_KrakenClassifyTask.obj
 0002:0000b098       __ehfuncinfo$??__EcmdLog@U2@@YAXXZ 1002f098     moc_KrakenClassifyTask.obj
 0002:0000b0bc       __unwindtable$??__EcoreLog@U2@@YAXXZ 1002f0bc     moc_KrakenClassifyTask.obj
 0002:0000b0c4       __ehfuncinfo$??__EcoreLog@U2@@YAXXZ 1002f0c4     moc_KrakenClassifyTask.obj
 0002:0000b0e8       __unwindtable$??__EioLog@U2@@YAXXZ 1002f0e8     moc_KrakenClassifyTask.obj
 0002:0000b0f0       __ehfuncinfo$??__EioLog@U2@@YAXXZ 1002f0f0     moc_KrakenClassifyTask.obj
 0002:0000b114       __unwindtable$??__EperfLog@U2@@YAXXZ 1002f114     moc_KrakenClassifyTask.obj
 0002:0000b11c       __ehfuncinfo$??__EperfLog@U2@@YAXXZ 1002f11c     moc_KrakenClassifyTask.obj
 0002:0000b140       __unwindtable$??__EscriptLog@U2@@YAXXZ 1002f140     moc_KrakenClassifyTask.obj
 0002:0000b148       __ehfuncinfo$??__EscriptLog@U2@@YAXXZ 1002f148     moc_KrakenClassifyTask.obj
 0002:0000b16c       __unwindtable$??__EtaskLog@U2@@YAXXZ 1002f16c     moc_KrakenClassifyTask.obj
 0002:0000b174       __ehfuncinfo$??__EtaskLog@U2@@YAXXZ 1002f174     moc_KrakenClassifyTask.obj
 0002:0000b198       __unwindtable$??__EuiLog@U2@@YAXXZ 1002f198     moc_KrakenClassifyTask.obj
 0002:0000b1a0       __ehfuncinfo$??__EuiLog@U2@@YAXXZ 1002f1a0     moc_KrakenClassifyTask.obj
 0002:0000b1c4       __unwindtable$??__EuserActLog@U2@@YAXXZ 1002f1c4     moc_KrakenClassifyTask.obj
 0002:0000b1cc       __ehfuncinfo$??__EuserActLog@U2@@YAXXZ 1002f1cc     moc_KrakenClassifyTask.obj
 0002:0000b1f0       __unwindtable$??__EalgoLog@U2@@YAXXZ 1002f1f0     moc_KrakenClassifyWorker.obj
 0002:0000b1f8       __ehfuncinfo$??__EalgoLog@U2@@YAXXZ 1002f1f8     moc_KrakenClassifyWorker.obj
 0002:0000b21c       __unwindtable$??__EcmdLog@U2@@YAXXZ 1002f21c     moc_KrakenClassifyWorker.obj
 0002:0000b224       __ehfuncinfo$??__EcmdLog@U2@@YAXXZ 1002f224     moc_KrakenClassifyWorker.obj
 0002:0000b248       __unwindtable$??__EcoreLog@U2@@YAXXZ 1002f248     moc_KrakenClassifyWorker.obj
 0002:0000b250       __ehfuncinfo$??__EcoreLog@U2@@YAXXZ 1002f250     moc_KrakenClassifyWorker.obj
 0002:0000b274       __unwindtable$??__EioLog@U2@@YAXXZ 1002f274     moc_KrakenClassifyWorker.obj
 0002:0000b27c       __ehfuncinfo$??__EioLog@U2@@YAXXZ 1002f27c     moc_KrakenClassifyWorker.obj
 0002:0000b2a0       __unwindtable$??__EperfLog@U2@@YAXXZ 1002f2a0     moc_KrakenClassifyWorker.obj
 0002:0000b2a8       __ehfuncinfo$??__EperfLog@U2@@YAXXZ 1002f2a8     moc_KrakenClassifyWorker.obj
 0002:0000b2cc       __unwindtable$??__EscriptLog@U2@@YAXXZ 1002f2cc     moc_KrakenClassifyWorker.obj
 0002:0000b2d4       __ehfuncinfo$??__EscriptLog@U2@@YAXXZ 1002f2d4     moc_KrakenClassifyWorker.obj
 0002:0000b2f8       __unwindtable$??__EtaskLog@U2@@YAXXZ 1002f2f8     moc_KrakenClassifyWorker.obj
 0002:0000b300       __ehfuncinfo$??__EtaskLog@U2@@YAXXZ 1002f300     moc_KrakenClassifyWorker.obj
 0002:0000b324       __unwindtable$??__EuiLog@U2@@YAXXZ 1002f324     moc_KrakenClassifyWorker.obj
 0002:0000b32c       __ehfuncinfo$??__EuiLog@U2@@YAXXZ 1002f32c     moc_KrakenClassifyWorker.obj
 0002:0000b350       __unwindtable$??__EuserActLog@U2@@YAXXZ 1002f350     moc_KrakenClassifyWorker.obj
 0002:0000b358       __ehfuncinfo$??__EuserActLog@U2@@YAXXZ 1002f358     moc_KrakenClassifyWorker.obj
 0002:0000b380       __sehtable$__onexit        1002f380     MSVCRT:atonexit.obj
 0002:0000b3a0       __sehtable$___DllMainCRTStartup 1002f3a0     MSVCRT:crtdll.obj
 0002:0000b3c8       __sehtable$??_M@YGXPAXIHP6EX0@Z@Z 1002f3c8     MSVCRT:ehvecdtr.obj
 0002:0000b3e8       __sehtable$?__ArrayUnwind@@YGXPAXIHP6EX0@Z@Z 1002f3e8     MSVCRT:ehvecdtr.obj
 0002:0000b408       __sehtable$__IsNonwritableInCurrentImage 1002f408     MSVCRT:pesect.obj
 0002:0000b430       .edata                     1002f430     kraken_support.exp
 0002:0000b458       rgpv                       1002f458     kraken_support.exp
 0002:0000b45c       rgszName                   1002f45c     kraken_support.exp
 0002:0000b460       rgwOrd                     1002f460     kraken_support.exp
 0002:0000b462       szName                     1002f462     kraken_support.exp
 0002:0000b475       $N00001                    1002f475     kraken_support.exp
 0002:0000d730       .idata$6                   10031730     U2Core:U2Core.dll
 0002:0000d792       .idata$6                   10031792     U2Gui:U2Gui.dll
 0002:00010182       .idata$6                   10034182     U2Lang:U2Lang.dll
 0002:00011002       .idata$6                   10035002     U2Designer:U2Designer.dll
 0002:000119cc       .idata$6                   100359cc     ngs_reads_classification:ngs_reads_classification.dll
 0002:00011e2a       .idata$6                   10035e2a     Qt5Widgets:Qt5Widgets.dll
 0002:00011edc       .idata$6                   10035edc     Qt5Gui:Qt5Gui.dll
 0002:0001204e       .idata$6                   1003604e     Qt5Script:Qt5Script.dll
 0002:00013106       .idata$6                   10037106     Qt5Core:Qt5Core.dll
 0002:000131ac       .idata$6                   100371ac     msvcprt:MSVCP120.dll
 0002:00013230       .idata$6                   10037230     MSVCRT:MSVCR120.dll
 0002:00013444       .idata$6                   10037444     kernel32:KERNEL32.dll
 0003:00000c10       __Tuple_alloc              10038c10     DatabaseSizeRelation.obj
 0003:00000c11       _ignore                    10038c11     DatabaseSizeRelation.obj
 0003:00000c12       _allocator_arg             10038c12     DatabaseSizeRelation.obj
 0003:00000c13       _piecewise_construct       10038c13     DatabaseSizeRelation.obj
 0003:00000c14       _taskLog                   10038c14     DatabaseSizeRelation.obj
 0003:00000c1c       _algoLog                   10038c1c     DatabaseSizeRelation.obj
 0003:00000c24       _userActLog                10038c24     DatabaseSizeRelation.obj
 0003:00000c2c       _ioLog                     10038c2c     DatabaseSizeRelation.obj
 0003:00000c34       _coreLog                   10038c34     DatabaseSizeRelation.obj
 0003:00000c3c       _uiLog                     10038c3c     DatabaseSizeRelation.obj
 0003:00000c44       _scriptLog                 10038c44     DatabaseSizeRelation.obj
 0003:00000c4c       _perfLog                   10038c4c     DatabaseSizeRelation.obj
 0003:00000c54       _cmdLog                    10038c54     DatabaseSizeRelation.obj
 0003:00000c64       __Tuple_alloc              10038c64     KrakenBuildPrompter.obj
 0003:00000c65       _ignore                    10038c65     KrakenBuildPrompter.obj
 0003:00000c66       _allocator_arg             10038c66     KrakenBuildPrompter.obj
 0003:00000c67       _piecewise_construct       10038c67     KrakenBuildPrompter.obj
 0003:00000c68       _taskLog                   10038c68     KrakenBuildPrompter.obj
 0003:00000c70       _algoLog                   10038c70     KrakenBuildPrompter.obj
 0003:00000c78       _userActLog                10038c78     KrakenBuildPrompter.obj
 0003:00000c80       _ioLog                     10038c80     KrakenBuildPrompter.obj
 0003:00000c88       _coreLog                   10038c88     KrakenBuildPrompter.obj
 0003:00000c90       _uiLog                     10038c90     KrakenBuildPrompter.obj
 0003:00000c98       _scriptLog                 10038c98     KrakenBuildPrompter.obj
 0003:00000ca0       _perfLog                   10038ca0     KrakenBuildPrompter.obj
 0003:00000ca8       _cmdLog                    10038ca8     KrakenBuildPrompter.obj
 0003:00000cb0       __Tuple_alloc              10038cb0     KrakenBuildTask.obj
 0003:00000cb1       _ignore                    10038cb1     KrakenBuildTask.obj
 0003:00000cb2       _allocator_arg             10038cb2     KrakenBuildTask.obj
 0003:00000cb3       _piecewise_construct       10038cb3     KrakenBuildTask.obj
 0003:00000cb8       _taskLog                   10038cb8     KrakenBuildTask.obj
 0003:00000cc0       _algoLog                   10038cc0     KrakenBuildTask.obj
 0003:00000cc8       _userActLog                10038cc8     KrakenBuildTask.obj
 0003:00000cd0       _ioLog                     10038cd0     KrakenBuildTask.obj
 0003:00000cd8       _coreLog                   10038cd8     KrakenBuildTask.obj
 0003:00000ce0       _uiLog                     10038ce0     KrakenBuildTask.obj
 0003:00000ce8       _scriptLog                 10038ce8     KrakenBuildTask.obj
 0003:00000cf4       _perfLog                   10038cf4     KrakenBuildTask.obj
 0003:00000cfc       _cmdLog                    10038cfc     KrakenBuildTask.obj
 0003:00000d08       ?cvar@?1???0KrakenBuildTask@U2@@QAE@ABUKrakenBuildTaskSettings@2@@Z@4VGReportableCounter@2@A 10038d08     KrakenBuildTask.obj
 0003:00000d30       ?$S1@?1???0KrakenBuildTask@U2@@QAE@ABUKrakenBuildTaskSettings@2@@Z@4IA 10038d30     KrakenBuildTask.obj
 0003:00000d34       ?TAXONOMY_FILES_TO_COPY@?1??prepareTaxonomyData@KrakenBuildTask@U2@@AAE?AV?$QList@PAVTask@U2@@@@XZ@4VQStringList@@B 10038d34     KrakenBuildTask.obj
 0003:00000d38       ?$S2@?1??prepareTaxonomyData@KrakenBuildTask@U2@@AAE?AV?$QList@PAVTask@U2@@@@XZ@4IA 10038d38     KrakenBuildTask.obj
 0003:00000d3c       __Tuple_alloc              10038d3c     KrakenBuildValidator.obj
 0003:00000d3d       _ignore                    10038d3d     KrakenBuildValidator.obj
 0003:00000d3e       _allocator_arg             10038d3e     KrakenBuildValidator.obj
 0003:00000d3f       _piecewise_construct       10038d3f     KrakenBuildValidator.obj
 0003:00000d40       _taskLog                   10038d40     KrakenBuildValidator.obj
 0003:00000d48       _algoLog                   10038d48     KrakenBuildValidator.obj
 0003:00000d50       _userActLog                10038d50     KrakenBuildValidator.obj
 0003:00000d58       _ioLog                     10038d58     KrakenBuildValidator.obj
 0003:00000d60       _coreLog                   10038d60     KrakenBuildValidator.obj
 0003:00000d68       _uiLog                     10038d68     KrakenBuildValidator.obj
 0003:00000d70       _scriptLog                 10038d70     KrakenBuildValidator.obj
 0003:00000d78       _perfLog                   10038d78     KrakenBuildValidator.obj
 0003:00000d80       _cmdLog                    10038d80     KrakenBuildValidator.obj
 0003:00000d88       __Tuple_alloc              10038d88     KrakenBuildWorker.obj
 0003:00000d89       _ignore                    10038d89     KrakenBuildWorker.obj
 0003:00000d8a       _allocator_arg             10038d8a     KrakenBuildWorker.obj
 0003:00000d8b       _piecewise_construct       10038d8b     KrakenBuildWorker.obj
 0003:00000d8c       _taskLog                   10038d8c     KrakenBuildWorker.obj
 0003:00000d94       _algoLog                   10038d94     KrakenBuildWorker.obj
 0003:00000d9c       _userActLog                10038d9c     KrakenBuildWorker.obj
 0003:00000da4       _ioLog                     10038da4     KrakenBuildWorker.obj
 0003:00000dac       _coreLog                   10038dac     KrakenBuildWorker.obj
 0003:00000db4       _uiLog                     10038db4     KrakenBuildWorker.obj
 0003:00000dbc       _scriptLog                 10038dbc     KrakenBuildWorker.obj
 0003:00000dc4       _perfLog                   10038dc4     KrakenBuildWorker.obj
 0003:00000dcc       _cmdLog                    10038dcc     KrakenBuildWorker.obj
 0003:00000dd8       __Tuple_alloc              10038dd8     KrakenBuildWorkerFactory.obj
 0003:00000dd9       _ignore                    10038dd9     KrakenBuildWorkerFactory.obj
 0003:00000dda       _allocator_arg             10038dda     KrakenBuildWorkerFactory.obj
 0003:00000ddb       _piecewise_construct       10038ddb     KrakenBuildWorkerFactory.obj
 0003:00000de4       _taskLog                   10038de4     KrakenBuildWorkerFactory.obj
 0003:00000dec       _algoLog                   10038dec     KrakenBuildWorkerFactory.obj
 0003:00000df4       _userActLog                10038df4     KrakenBuildWorkerFactory.obj
 0003:00000dfc       _ioLog                     10038dfc     KrakenBuildWorkerFactory.obj
 0003:00000e04       _coreLog                   10038e04     KrakenBuildWorkerFactory.obj
 0003:00000e18       _uiLog                     10038e18     KrakenBuildWorkerFactory.obj
 0003:00000e24       _scriptLog                 10038e24     KrakenBuildWorkerFactory.obj
 0003:00000e2c       _perfLog                   10038e2c     KrakenBuildWorkerFactory.obj
 0003:00000e40       _cmdLog                    10038e40     KrakenBuildWorkerFactory.obj
 0003:00000e60       __Tuple_alloc              10038e60     KrakenClassifyLogParser.obj
 0003:00000e61       _ignore                    10038e61     KrakenClassifyLogParser.obj
 0003:00000e62       _allocator_arg             10038e62     KrakenClassifyLogParser.obj
 0003:00000e63       _piecewise_construct       10038e63     KrakenClassifyLogParser.obj
 0003:00000e64       _taskLog                   10038e64     KrakenClassifyLogParser.obj
 0003:00000e6c       _algoLog                   10038e6c     KrakenClassifyLogParser.obj
 0003:00000e74       _userActLog                10038e74     KrakenClassifyLogParser.obj
 0003:00000e7c       _ioLog                     10038e7c     KrakenClassifyLogParser.obj
 0003:00000e84       _coreLog                   10038e84     KrakenClassifyLogParser.obj
 0003:00000e8c       _uiLog                     10038e8c     KrakenClassifyLogParser.obj
 0003:00000e94       _scriptLog                 10038e94     KrakenClassifyLogParser.obj
 0003:00000e9c       _perfLog                   10038e9c     KrakenClassifyLogParser.obj
 0003:00000ea4       _cmdLog                    10038ea4     KrakenClassifyLogParser.obj
 0003:00000eb0       __Tuple_alloc              10038eb0     KrakenClassifyPrompter.obj
 0003:00000eb1       _ignore                    10038eb1     KrakenClassifyPrompter.obj
 0003:00000eb2       _allocator_arg             10038eb2     KrakenClassifyPrompter.obj
 0003:00000eb3       _piecewise_construct       10038eb3     KrakenClassifyPrompter.obj
 0003:00000eb4       _taskLog                   10038eb4     KrakenClassifyPrompter.obj
 0003:00000ebc       _algoLog                   10038ebc     KrakenClassifyPrompter.obj
 0003:00000ec4       _userActLog                10038ec4     KrakenClassifyPrompter.obj
 0003:00000ecc       _ioLog                     10038ecc     KrakenClassifyPrompter.obj
 0003:00000ed4       _coreLog                   10038ed4     KrakenClassifyPrompter.obj
 0003:00000edc       _uiLog                     10038edc     KrakenClassifyPrompter.obj
 0003:00000ee4       _scriptLog                 10038ee4     KrakenClassifyPrompter.obj
 0003:00000eec       _perfLog                   10038eec     KrakenClassifyPrompter.obj
 0003:00000ef4       _cmdLog                    10038ef4     KrakenClassifyPrompter.obj
 0003:00000efc       __Tuple_alloc              10038efc     KrakenClassifyTask.obj
 0003:00000efd       _ignore                    10038efd     KrakenClassifyTask.obj
 0003:00000efe       _allocator_arg             10038efe     KrakenClassifyTask.obj
 0003:00000eff       _piecewise_construct       10038eff     KrakenClassifyTask.obj
 0003:00000f00       _taskLog                   10038f00     KrakenClassifyTask.obj
 0003:00000f08       _algoLog                   10038f08     KrakenClassifyTask.obj
 0003:00000f14       _userActLog                10038f14     KrakenClassifyTask.obj
 0003:00000f1c       _ioLog                     10038f1c     KrakenClassifyTask.obj
 0003:00000f24       _coreLog                   10038f24     KrakenClassifyTask.obj
 0003:00000f2c       _uiLog                     10038f2c     KrakenClassifyTask.obj
 0003:00000f34       _scriptLog                 10038f34     KrakenClassifyTask.obj
 0003:00000f40       _perfLog                   10038f40     KrakenClassifyTask.obj
 0003:00000f48       _cmdLog                    10038f48     KrakenClassifyTask.obj
 0003:00000f50       ?cvar@?1???0KrakenClassifyTask@U2@@QAE@ABUKrakenClassifyTaskSettings@2@@Z@4VGReportableCounter@2@A 10038f50     KrakenClassifyTask.obj
 0003:00000f78       ?$S1@?1???0KrakenClassifyTask@U2@@QAE@ABUKrakenClassifyTaskSettings@2@@Z@4IA 10038f78     KrakenClassifyTask.obj
 0003:00000f7c       __Tuple_alloc              10038f7c     KrakenClassifyValidator.obj
 0003:00000f7d       _ignore                    10038f7d     KrakenClassifyValidator.obj
 0003:00000f7e       _allocator_arg             10038f7e     KrakenClassifyValidator.obj
 0003:00000f7f       _piecewise_construct       10038f7f     KrakenClassifyValidator.obj
 0003:00000f80       _taskLog                   10038f80     KrakenClassifyValidator.obj
 0003:00000f88       _algoLog                   10038f88     KrakenClassifyValidator.obj
 0003:00000f90       _userActLog                10038f90     KrakenClassifyValidator.obj
 0003:00000f98       _ioLog                     10038f98     KrakenClassifyValidator.obj
 0003:00000fa0       _coreLog                   10038fa0     KrakenClassifyValidator.obj
 0003:00000fa8       _uiLog                     10038fa8     KrakenClassifyValidator.obj
 0003:00000fb0       _scriptLog                 10038fb0     KrakenClassifyValidator.obj
 0003:00000fb8       _perfLog                   10038fb8     KrakenClassifyValidator.obj
 0003:00000fc0       _cmdLog                    10038fc0     KrakenClassifyValidator.obj
 0003:00000fc8       __Tuple_alloc              10038fc8     KrakenClassifyWorker.obj
 0003:00000fc9       _ignore                    10038fc9     KrakenClassifyWorker.obj
 0003:00000fca       _allocator_arg             10038fca     KrakenClassifyWorker.obj
 0003:00000fcb       _piecewise_construct       10038fcb     KrakenClassifyWorker.obj
 0003:00000fd0       _taskLog                   10038fd0     KrakenClassifyWorker.obj
 0003:00000fd8       _algoLog                   10038fd8     KrakenClassifyWorker.obj
 0003:00000fe0       _userActLog                10038fe0     KrakenClassifyWorker.obj
 0003:00000fe8       _ioLog                     10038fe8     KrakenClassifyWorker.obj
 0003:00000ff0       _coreLog                   10038ff0     KrakenClassifyWorker.obj
 0003:00000ff8       _uiLog                     10038ff8     KrakenClassifyWorker.obj
 0003:00001000       _scriptLog                 10039000     KrakenClassifyWorker.obj
 0003:00001008       _perfLog                   10039008     KrakenClassifyWorker.obj
 0003:00001010       _cmdLog                    10039010     KrakenClassifyWorker.obj
 0003:0000102c       __Tuple_alloc              1003902c     KrakenClassifyWorkerFactory.obj
 0003:0000102d       _ignore                    1003902d     KrakenClassifyWorkerFactory.obj
 0003:0000102e       _allocator_arg             1003902e     KrakenClassifyWorkerFactory.obj
 0003:0000102f       _piecewise_construct       1003902f     KrakenClassifyWorkerFactory.obj
 0003:00001048       _taskLog                   10039048     KrakenClassifyWorkerFactory.obj
 0003:00001050       _algoLog                   10039050     KrakenClassifyWorkerFactory.obj
 0003:00001058       _userActLog                10039058     KrakenClassifyWorkerFactory.obj
 0003:00001060       _ioLog                     10039060     KrakenClassifyWorkerFactory.obj
 0003:00001068       _coreLog                   10039068     KrakenClassifyWorkerFactory.obj
 0003:0000107c       _uiLog                     1003907c     KrakenClassifyWorkerFactory.obj
 0003:00001084       _scriptLog                 10039084     KrakenClassifyWorkerFactory.obj
 0003:00001090       _perfLog                   10039090     KrakenClassifyWorkerFactory.obj
 0003:00001098       _cmdLog                    10039098     KrakenClassifyWorkerFactory.obj
 0003:000010b4       __Tuple_alloc              100390b4     KrakenSupport.obj
 0003:000010b5       _ignore                    100390b5     KrakenSupport.obj
 0003:000010b6       _allocator_arg             100390b6     KrakenSupport.obj
 0003:000010b7       _piecewise_construct       100390b7     KrakenSupport.obj
 0003:000010cc       __Tuple_alloc              100390cc     KrakenSupportPlugin.obj
 0003:000010cd       _ignore                    100390cd     KrakenSupportPlugin.obj
 0003:000010ce       _allocator_arg             100390ce     KrakenSupportPlugin.obj
 0003:000010cf       _piecewise_construct       100390cf     KrakenSupportPlugin.obj
 0003:000010d0       _taskLog                   100390d0     KrakenSupportPlugin.obj
 0003:000010d8       _algoLog                   100390d8     KrakenSupportPlugin.obj
 0003:000010e0       _userActLog                100390e0     KrakenSupportPlugin.obj
 0003:000010e8       _ioLog                     100390e8     KrakenSupportPlugin.obj
 0003:000010f4       _coreLog                   100390f4     KrakenSupportPlugin.obj
 0003:000010fc       _uiLog                     100390fc     KrakenSupportPlugin.obj
 0003:00001104       _scriptLog                 10039104     KrakenSupportPlugin.obj
 0003:0000110c       _perfLog                   1003910c     KrakenSupportPlugin.obj
 0003:00001118       _cmdLog                    10039118     KrakenSupportPlugin.obj
 0003:00001120       __Tuple_alloc              10039120     KrakenTranslateLogParser.obj
 0003:00001121       _ignore                    10039121     KrakenTranslateLogParser.obj
 0003:00001122       _allocator_arg             10039122     KrakenTranslateLogParser.obj
 0003:00001123       _piecewise_construct       10039123     KrakenTranslateLogParser.obj
 0003:00001124       _taskLog                   10039124     KrakenTranslateLogParser.obj
 0003:0000112c       _algoLog                   1003912c     KrakenTranslateLogParser.obj
 0003:00001134       _userActLog                10039134     KrakenTranslateLogParser.obj
 0003:0000113c       _ioLog                     1003913c     KrakenTranslateLogParser.obj
 0003:00001148       _coreLog                   10039148     KrakenTranslateLogParser.obj
 0003:00001150       _uiLog                     10039150     KrakenTranslateLogParser.obj
 0003:00001158       _scriptLog                 10039158     KrakenTranslateLogParser.obj
 0003:00001160       _perfLog                   10039160     KrakenTranslateLogParser.obj
 0003:00001168       _cmdLog                    10039168     KrakenTranslateLogParser.obj
 0003:00001170       __Tuple_alloc              10039170     moc_KrakenBuildPrompter.obj
 0003:00001171       _ignore                    10039171     moc_KrakenBuildPrompter.obj
 0003:00001172       _allocator_arg             10039172     moc_KrakenBuildPrompter.obj
 0003:00001173       _piecewise_construct       10039173     moc_KrakenBuildPrompter.obj
 0003:00001174       _taskLog                   10039174     moc_KrakenBuildPrompter.obj
 0003:0000117c       _algoLog                   1003917c     moc_KrakenBuildPrompter.obj
 0003:00001184       _userActLog                10039184     moc_KrakenBuildPrompter.obj
 0003:0000118c       _ioLog                     1003918c     moc_KrakenBuildPrompter.obj
 0003:00001194       _coreLog                   10039194     moc_KrakenBuildPrompter.obj
 0003:0000119c       _uiLog                     1003919c     moc_KrakenBuildPrompter.obj
 0003:000011a4       _scriptLog                 100391a4     moc_KrakenBuildPrompter.obj
 0003:000011ac       _perfLog                   100391ac     moc_KrakenBuildPrompter.obj
 0003:000011b4       _cmdLog                    100391b4     moc_KrakenBuildPrompter.obj
 0003:000011bc       __Tuple_alloc              100391bc     moc_KrakenBuildTask.obj
 0003:000011bd       _ignore                    100391bd     moc_KrakenBuildTask.obj
 0003:000011be       _allocator_arg             100391be     moc_KrakenBuildTask.obj
 0003:000011bf       _piecewise_construct       100391bf     moc_KrakenBuildTask.obj
 0003:000011c0       _taskLog                   100391c0     moc_KrakenBuildTask.obj
 0003:000011c8       _algoLog                   100391c8     moc_KrakenBuildTask.obj
 0003:000011d0       _userActLog                100391d0     moc_KrakenBuildTask.obj
 0003:000011d8       _ioLog                     100391d8     moc_KrakenBuildTask.obj
 0003:000011e0       _coreLog                   100391e0     moc_KrakenBuildTask.obj
 0003:000011e8       _uiLog                     100391e8     moc_KrakenBuildTask.obj
 0003:000011f0       _scriptLog                 100391f0     moc_KrakenBuildTask.obj
 0003:000011f8       _perfLog                   100391f8     moc_KrakenBuildTask.obj
 0003:00001200       _cmdLog                    10039200     moc_KrakenBuildTask.obj
 0003:00001208       __Tuple_alloc              10039208     moc_KrakenBuildWorker.obj
 0003:00001209       _ignore                    10039209     moc_KrakenBuildWorker.obj
 0003:0000120a       _allocator_arg             1003920a     moc_KrakenBuildWorker.obj
 0003:0000120b       _piecewise_construct       1003920b     moc_KrakenBuildWorker.obj
 0003:0000120c       _taskLog                   1003920c     moc_KrakenBuildWorker.obj
 0003:00001214       _algoLog                   10039214     moc_KrakenBuildWorker.obj
 0003:0000121c       _userActLog                1003921c     moc_KrakenBuildWorker.obj
 0003:00001224       _ioLog                     10039224     moc_KrakenBuildWorker.obj
 0003:0000122c       _coreLog                   1003922c     moc_KrakenBuildWorker.obj
 0003:00001234       _uiLog                     10039234     moc_KrakenBuildWorker.obj
 0003:0000123c       _scriptLog                 1003923c     moc_KrakenBuildWorker.obj
 0003:00001244       _perfLog                   10039244     moc_KrakenBuildWorker.obj
 0003:0000124c       _cmdLog                    1003924c     moc_KrakenBuildWorker.obj
 0003:00001258       __Tuple_alloc              10039258     moc_KrakenClassifyPrompter.obj
 0003:00001259       _ignore                    10039259     moc_KrakenClassifyPrompter.obj
 0003:0000125a       _allocator_arg             1003925a     moc_KrakenClassifyPrompter.obj
 0003:0000125b       _piecewise_construct       1003925b     moc_KrakenClassifyPrompter.obj
 0003:0000125c       _taskLog                   1003925c     moc_KrakenClassifyPrompter.obj
 0003:00001264       _algoLog                   10039264     moc_KrakenClassifyPrompter.obj
 0003:0000126c       _userActLog                1003926c     moc_KrakenClassifyPrompter.obj
 0003:00001274       _ioLog                     10039274     moc_KrakenClassifyPrompter.obj
 0003:0000127c       _coreLog                   1003927c     moc_KrakenClassifyPrompter.obj
 0003:00001284       _uiLog                     10039284     moc_KrakenClassifyPrompter.obj
 0003:0000128c       _scriptLog                 1003928c     moc_KrakenClassifyPrompter.obj
 0003:00001294       _perfLog                   10039294     moc_KrakenClassifyPrompter.obj
 0003:0000129c       _cmdLog                    1003929c     moc_KrakenClassifyPrompter.obj
 0003:000012a4       __Tuple_alloc              100392a4     moc_KrakenClassifyTask.obj
 0003:000012a5       _ignore                    100392a5     moc_KrakenClassifyTask.obj
 0003:000012a6       _allocator_arg             100392a6     moc_KrakenClassifyTask.obj
 0003:000012a7       _piecewise_construct       100392a7     moc_KrakenClassifyTask.obj
 0003:000012a8       _taskLog                   100392a8     moc_KrakenClassifyTask.obj
 0003:000012b0       _algoLog                   100392b0     moc_KrakenClassifyTask.obj
 0003:000012b8       _userActLog                100392b8     moc_KrakenClassifyTask.obj
 0003:000012c0       _ioLog                     100392c0     moc_KrakenClassifyTask.obj
 0003:000012c8       _coreLog                   100392c8     moc_KrakenClassifyTask.obj
 0003:000012d0       _uiLog                     100392d0     moc_KrakenClassifyTask.obj
 0003:000012d8       _scriptLog                 100392d8     moc_KrakenClassifyTask.obj
 0003:000012e0       _perfLog                   100392e0     moc_KrakenClassifyTask.obj
 0003:000012e8       _cmdLog                    100392e8     moc_KrakenClassifyTask.obj
 0003:000012f0       __Tuple_alloc              100392f0     moc_KrakenClassifyWorker.obj
 0003:000012f1       _ignore                    100392f1     moc_KrakenClassifyWorker.obj
 0003:000012f2       _allocator_arg             100392f2     moc_KrakenClassifyWorker.obj
 0003:000012f3       _piecewise_construct       100392f3     moc_KrakenClassifyWorker.obj
 0003:000012f4       _taskLog                   100392f4     moc_KrakenClassifyWorker.obj
 0003:000012fc       _algoLog                   100392fc     moc_KrakenClassifyWorker.obj
 0003:00001304       _userActLog                10039304     moc_KrakenClassifyWorker.obj
 0003:0000130c       _ioLog                     1003930c     moc_KrakenClassifyWorker.obj
 0003:00001314       _coreLog                   10039314     moc_KrakenClassifyWorker.obj
 0003:0000131c       _uiLog                     1003931c     moc_KrakenClassifyWorker.obj
 0003:00001324       _scriptLog                 10039324     moc_KrakenClassifyWorker.obj
 0003:0000132c       _perfLog                   1003932c     moc_KrakenClassifyWorker.obj
 0003:00001334       _cmdLog                    10039334     moc_KrakenClassifyWorker.obj
 0003:0000133c       __Tuple_alloc              1003933c     moc_KrakenSupport.obj
 0003:0000133d       _ignore                    1003933d     moc_KrakenSupport.obj
 0003:0000133e       _allocator_arg             1003933e     moc_KrakenSupport.obj
 0003:0000133f       _piecewise_construct       1003933f     moc_KrakenSupport.obj
 0003:00001340       __Tuple_alloc              10039340     moc_KrakenSupportPlugin.obj
 0003:00001341       _ignore                    10039341     moc_KrakenSupportPlugin.obj
 0003:00001342       _allocator_arg             10039342     moc_KrakenSupportPlugin.obj
 0003:00001343       _piecewise_construct       10039343     moc_KrakenSupportPlugin.obj
 0003:00001344       ___proc_attached           10039344     MSVCRT:crtdll.obj
 0003:00001348       _GS_ExceptionRecord        10039348     MSVCRT:gs_report.obj
 0003:00001398       _GS_ContextRecord          10039398     MSVCRT:gs_report.obj
 0003:00001664       _DebuggerWasPresent        10039664     MSVCRT:gs_report.obj
 0004:00000060       $R000000                   1003a060     * linker generated manifest res *

 Exports

  ordinal    name

        1    _ugene_plugin_init
               exported name: ugene_plugin_init
